 dna_stat

 Timestamp is 5c762218 (Wed Feb 27 12:37:28 2019)

 Preferred load address is 10000000

 Start         Length     Name                   Class
 0001:00000000 00002608H .text$di                CODE
 0001:00002610 00011f98H .text$mn                CODE
 0001:000145b0 00002ec4H .text$x                 CODE
 0001:00017480 000009bbH .text$yd                CODE
 0002:00000000 000009acH .idata$5                DATA
 0002:000009ac 00000004H .CRT$XCA                DATA
 0002:000009b0 0000023cH .CRT$XCU                DATA
 0002:00000bec 00000004H .CRT$XCZ                DATA
 0002:00000bf0 00000004H .CRT$XIA                DATA
 0002:00000bf4 00000004H .CRT$XIAA               DATA
 0002:00000bf8 00000004H .CRT$XIC                DATA
 0002:00000bfc 00000004H .CRT$XIZ                DATA
 0002:00000c00 00002f10H .rdata                  DATA
 0002:00003b10 00000070H .rdata$debug            DATA
 0002:00003b80 000012d8H .rdata$r                DATA
 0002:00004e60 0000021cH .rdata$sxdata           DATA
 0002:0000507c 00000004H .rtc$IAA                DATA
 0002:00005080 00000004H .rtc$IZZ                DATA
 0002:00005084 00000004H .rtc$TAA                DATA
 0002:00005088 00000004H .rtc$TZZ                DATA
 0002:00005090 00002fa4H .xdata$x                DATA
 0002:00008040 00000051H .edata                  DATA
 0002:00008094 000000c8H .idata$2                DATA
 0002:0000815c 00000014H .idata$3                DATA
 0002:00008170 000009acH .idata$4                DATA
 0002:00008b1c 00006d2cH .idata$6                DATA
 0003:00000000 000002e4H .data                   DATA
 0003:000002e8 00000824H .data$r                 DATA
 0003:00000b10 0000057cH .bss                    DATA
 0004:00000000 00000058H .rsrc$01                DATA
 0004:00000060 00000180H .rsrc$02                DATA

  Address         Publics by Value              Rva+Base       Lib:Object

 0000:00000000       __except_list              00000000     <absolute>
 0000:00000000       ___guard_flags             00000000     <absolute>
 0000:00000000       ___guard_fids_count        00000000     <absolute>
 0000:00000000       ___guard_fids_table        00000000     <absolute>
 0000:00000087       ___safe_se_handler_count   00000087     <absolute>
 0000:00009876       __fltused                  00009876     <absolute>
 0000:00009876       __ldused                   00009876     <absolute>
 0000:00000000       ___ImageBase               10000000     <linker-defined>
 0001:00002610       ??$_Allocate@D@std@@YAPADIPAD@Z 10003610 f i DNAStatMSAProfileDialog.obj
 0001:00002640       ??$_Move@AAPAU?$QTypedArrayData@D@@@std@@YA$$QAPAU?$QTypedArrayData@D@@AAPAU1@@Z 10003640 f i DNAStatMSAProfileDialog.obj
 0001:00002650       ??$_Move@AAPAU?$QTypedArrayData@UColumnStat@DNAStatMSAProfileTask@U2@@@@@std@@YA$$QAPAU?$QTypedArrayData@UColumnStat@DNAStatMSAProfileTask@U2@@@@AAPAU1@@Z 10003650 f i DNAStatMSAProfileDialog.obj
 0001:00002660       ??$_Move@AAPAUData@QListData@@@std@@YA$$QAPAUData@QListData@@AAPAU12@@Z 10003660 f i DNAStatMSAProfileDialog.obj
 0001:00002670       ??$_Move@AAPAUQHashData@@@std@@YA$$QAPAUQHashData@@AAPAU1@@Z 10003670 f i DNAStatMSAProfileDialog.obj
 0001:00002680       ??$addressof@D@std@@YAPADAAD@Z 10003680 f i DNAStatMSAProfileDialog.obj
 0001:00002690       ??$atomic@H@?$QAtomicOpsBySize@$03@@CAPAJPAH@Z 10003690 f i DNAStatMSAProfileDialog.obj
 0001:000026a0       ??$construct@PADAAPAD@?$_Wrap_alloc@V?$allocator@D@std@@@std@@QAEXPAPADAAPAD@Z 100036a0 f i DNAStatMSAProfileDialog.obj
 0001:000026c0       ??$construct@PADAAPAD@?$allocator@D@std@@QAEXPAPADAAPAD@Z 100036c0 f i DNAStatMSAProfileDialog.obj
 0001:000026e0       ??$construct@PADAAPAD@?$allocator_traits@V?$allocator@D@std@@@std@@SAXAAV?$allocator@D@1@PAPADAAPAD@Z 100036e0 f i DNAStatMSAProfileDialog.obj
 0001:00002700       ??$deref@H@?$QAtomicOpsBySize@$03@@SA_NAAH@Z 10003700 f i DNAStatMSAProfileDialog.obj
 0001:00002720       ??$destroy@PAD@?$_Wrap_alloc@V?$allocator@D@std@@@std@@QAEXPAPAD@Z 10003720 f i DNAStatMSAProfileDialog.obj
 0001:00002730       ??$destroy@PAD@?$allocator@D@std@@QAEXPAPAD@Z 10003730 f i DNAStatMSAProfileDialog.obj
 0001:00002740       ??$destroy@PAD@?$allocator_traits@V?$allocator@D@std@@@std@@SAXAAV?$allocator@D@1@PAPAD@Z 10003740 f i DNAStatMSAProfileDialog.obj
 0001:00002750       ??$forward@AAPAD@std@@YAAAPADAAPAD@Z 10003750 f i DNAStatMSAProfileDialog.obj
 0001:00002760       ??$load@H@?$QGenericAtomicOps@U?$QAtomicOpsBySize@$03@@@@SAHABH@Z 10003760 f i DNAStatMSAProfileDialog.obj
 0001:00002770       ??$qMax@H@@YAABHABH0@Z     10003770 f i DNAStatMSAProfileDialog.obj
 0001:00002790       ??$qSwap@PAU?$QTypedArrayData@D@@@@YAXAAPAU?$QTypedArrayData@D@@0@Z 10003790 f i DNAStatMSAProfileDialog.obj
 0001:000027b0       ??$qSwap@PAU?$QTypedArrayData@UColumnStat@DNAStatMSAProfileTask@U2@@@@@@YAXAAPAU?$QTypedArrayData@UColumnStat@DNAStatMSAProfileTask@U2@@@@0@Z 100037b0 f i DNAStatMSAProfileDialog.obj
 0001:000027d0       ??$qSwap@PAUData@QListData@@@@YAXAAPAUData@QListData@@0@Z 100037d0 f i DNAStatMSAProfileDialog.obj
 0001:000027f0       ??$qSwap@PAUQHashData@@@@YAXAAPAUQHashData@@0@Z 100037f0 f i DNAStatMSAProfileDialog.obj
 0001:00002810       ??$ref@H@?$QAtomicOpsBySize@$03@@SA_NAAH@Z 10003810 f i DNAStatMSAProfileDialog.obj
 0001:00002830       ??$swap@PAU?$QTypedArrayData@D@@@std@@YAXAAPAU?$QTypedArrayData@D@@0@Z 10003830 f i DNAStatMSAProfileDialog.obj
 0001:00002850       ??$swap@PAU?$QTypedArrayData@UColumnStat@DNAStatMSAProfileTask@U2@@@@@std@@YAXAAPAU?$QTypedArrayData@UColumnStat@DNAStatMSAProfileTask@U2@@@@0@Z 10003850 f i DNAStatMSAProfileDialog.obj
 0001:00002870       ??$swap@PAUData@QListData@@@std@@YAXAAPAUData@QListData@@0@Z 10003870 f i DNAStatMSAProfileDialog.obj
 0001:00002890       ??$swap@PAUQHashData@@@std@@YAXAAPAUQHashData@@0@Z 10003890 f i DNAStatMSAProfileDialog.obj
 0001:000028b0       ??0?$AbstractId@H@U2@@IAE@ABH@Z 100038b0 f i DNAStatMSAProfileDialog.obj
 0001:000028d0       ??0?$QFlags@W4AlignmentFlag@Qt@@@@QAE@PQPrivate@0@H@Z 100038d0 f i DNAStatMSAProfileDialog.obj
 0001:000028e0       ??0?$QFlags@W4AllocationOption@QArrayData@@@@QAE@PQPrivate@0@H@Z 100038e0 f i DNAStatMSAProfileDialog.obj
 0001:000028f0       ??0?$QFlags@W4AllocationOption@QArrayData@@@@QAE@W4AllocationOption@QArrayData@@@Z 100038f0 f i DNAStatMSAProfileDialog.obj
 0001:00002900       ??0?$QFlags@W4OpenModeFlag@QIODevice@@@@QAE@VQFlag@@@Z 10003900 f i DNAStatMSAProfileDialog.obj
 0001:00002910       ??0?$QFlags@W4OpenModeFlag@QIODevice@@@@QAE@W4OpenModeFlag@QIODevice@@@Z 10003910 f i DNAStatMSAProfileDialog.obj
 0001:00002920       ??0?$QFlags@W4StandardButton@QDialogButtonBox@@@@QAE@VQFlag@@@Z 10003920 f i DNAStatMSAProfileDialog.obj
 0001:00002930       ??0?$QFlags@W4StandardButton@QDialogButtonBox@@@@QAE@W4StandardButton@QDialogButtonBox@@@Z 10003930 f i DNAStatMSAProfileDialog.obj
 0001:00002940       ??0?$QFlags@W4StandardButton@QMessageBox@@@@QAE@W4StandardButton@QMessageBox@@@Z 10003940 f i DNAStatMSAProfileDialog.obj
 0001:00002950       ??0?$QFlags@W4TaskFlag@U2@@@@QAE@VQFlag@@@Z 10003950 f i DNAStatMSAProfileDialog.obj
 0001:00002960       ??0?$QFlags@W4TaskFlag@U2@@@@QAE@W4TaskFlag@U2@@@Z 10003960 f i DNAStatMSAProfileDialog.obj
 0001:00002970       ??0?$QFlags@W4WindowType@Qt@@@@QAE@PQPrivate@0@H@Z 10003970 f i DNAStatMSAProfileDialog.obj
 0001:00002980       ??0?$QHash@DH@@QAE@XZ      10003980 f i DNAStatMSAProfileDialog.obj
 0001:00002990       ??0?$QHash@DUQHashDummyValue@@@@QAE@XZ 10003990 f i DNAStatMSAProfileDialog.obj
 0001:000029a0       ??0?$QHashNode@DH@@QAE@ABDABHIPAU0@@Z 100039a0 f i DNAStatMSAProfileDialog.obj
 0001:000029d0       ??0?$QHashNode@DUQHashDummyValue@@@@QAE@ABDABUQHashDummyValue@@IPAU0@@Z 100039d0 f i DNAStatMSAProfileDialog.obj
 0001:000029f0       ??0?$QList@VMultipleSequenceAlignmentRow@U2@@@@QAE@XZ 100039f0 f i DNAStatMSAProfileDialog.obj
 0001:00002a00       ??0?$QList@VQString@@@@QAE@XZ 10003a00 f i DNAStatMSAProfileDialog.obj
 0001:00002a10       ??0?$QSet@D@@QAE@XZ        10003a10 f i DNAStatMSAProfileDialog.obj
 0001:00002a20       ??0?$QVector@D@@QAE@ABV0@@Z 10003a20 f i DNAStatMSAProfileDialog.obj
 0001:00002ae0       ??0?$QVector@D@@QAE@XZ     10003ae0 f i DNAStatMSAProfileDialog.obj
 0001:00002af0       ??0?$QVector@H@@QAE@ABV0@@Z 10003af0 f i DNAStatMSAProfileDialog.obj
 0001:00002bb0       ??0?$QVector@H@@QAE@XZ     10003bb0 f i DNAStatMSAProfileDialog.obj
 0001:00002bc0       ??0?$QVector@UColumnStat@DNAStatMSAProfileTask@U2@@@@QAE@ABV0@@Z 10003bc0 f i DNAStatMSAProfileDialog.obj
 0001:00002c80       ??0?$QVector@UColumnStat@DNAStatMSAProfileTask@U2@@@@QAE@XZ 10003c80 f i DNAStatMSAProfileDialog.obj
 0001:00002c90       ??0?$_String_alloc@$0A@U?$_String_base_types@DV?$allocator@D@std@@@std@@@std@@QAE@ABV?$allocator@D@1@@Z 10003c90 f i DNAStatMSAProfileDialog.obj
 0001:00002cb0       ??0?$_String_val@U?$_Simple_types@D@std@@@std@@QAE@XZ 10003cb0 f i DNAStatMSAProfileDialog.obj
 0001:00002cd0       ??0?$_Wrap_alloc@V?$allocator@D@std@@@std@@QAE@XZ 10003cd0 f i DNAStatMSAProfileDialog.obj
 0001:00002ce0       ??0?$allocator@D@std@@QAE@XZ 10003ce0 f i DNAStatMSAProfileDialog.obj
 0001:00002cf0       ??0?$basic_string@DU?$char_traits@D@std@@V?$allocator@D@2@@std@@QAE@PBD@Z 10003cf0 f i DNAStatMSAProfileDialog.obj
 0001:00002d50       ??0AbstractInt32Id@U2@@IAE@H@Z 10003d50 f i DNAStatMSAProfileDialog.obj
 0001:00002d70       ??0ColumnStat@DNAStatMSAProfileTask@U2@@QAE@ABU012@@Z 10003d70 f i DNAStatMSAProfileDialog.obj
 0001:00002d90       ??0ColumnStat@DNAStatMSAProfileTask@U2@@QAE@XZ 10003d90 f i DNAStatMSAProfileDialog.obj
 0001:00002da0       ??0DNAStatMSAProfileDialog@U2@@QAE@PAVQWidget@@PAVMSAEditor@1@@Z 10003da0 f   DNAStatMSAProfileDialog.obj
 0001:00002f10       ??0DNAStatMSAProfileTask@U2@@QAE@ABVDNAStatMSAProfileTaskSettings@1@@Z 10003f10 f   DNAStatMSAProfileDialog.obj
 0001:00002ff0       ??0DNAStatMSAProfileTaskSettings@U2@@QAE@ABV01@@Z 10003ff0 f i DNAStatMSAProfileDialog.obj
 0001:000030a0       ??0DNAStatMSAProfileTaskSettings@U2@@QAE@XZ 100040a0 f i DNAStatMSAProfileDialog.obj
 0001:00003180       ??0QFlag@@QAE@H@Z          10004180 f i DNAStatMSAProfileDialog.obj
 0001:00003190       ??0QLatin1Char@@QAE@D@Z    10004190 f i DNAStatMSAProfileDialog.obj
 0001:000031a0       ??0QStringList@@QAE@XZ     100041a0 f i DNAStatMSAProfileDialog.obj
 0001:000031b0       ??0ServiceType@U2@@QAE@H@Z 100041b0 f i DNAStatMSAProfileDialog.obj
 0001:000031d0       ??0_Generic_error_category@std@@QAE@XZ 100041d0 f i DNAStatMSAProfileDialog.obj
 0001:000031e0       ??0_Ignore@std@@QAE@XZ     100041e0 f i DNAStatMSAProfileDialog.obj
 0001:000031f0       ??0_Iostream_error_category@std@@QAE@XZ 100041f0 f i DNAStatMSAProfileDialog.obj
 0001:00003200       ??0_System_error_category@std@@QAE@XZ 10004200 f i DNAStatMSAProfileDialog.obj
 0001:00003210       ??0error_category@std@@QAE@XZ 10004210 f i DNAStatMSAProfileDialog.obj
 0001:00003220       ??0error_condition@std@@QAE@HABVerror_category@1@@Z 10004220 f i DNAStatMSAProfileDialog.obj
 0001:00003240       ??0iterator@?$QHash@DUQHashDummyValue@@@@QAE@PAX@Z 10004240 f i DNAStatMSAProfileDialog.obj
 0001:00003250       ??0iterator@?$QSet@D@@QAE@V0?$QHash@DUQHashDummyValue@@@@@Z 10004250 f i DNAStatMSAProfileDialog.obj
 0001:00003260       ??1?$AbstractId@H@U2@@MAE@XZ 10004260 f i DNAStatMSAProfileDialog.obj
 0001:00003270       ??1?$QHash@DH@@QAE@XZ      10004270 f i DNAStatMSAProfileDialog.obj
 0001:000032a0       ??1?$QHash@DUQHashDummyValue@@@@QAE@XZ 100042a0 f i DNAStatMSAProfileDialog.obj
 0001:000032d0       ??1?$QList@VMultipleSequenceAlignmentRow@U2@@@@QAE@XZ 100042d0 f i DNAStatMSAProfileDialog.obj
 0001:00003300       ??1?$QList@VQString@@@@QAE@XZ 10004300 f i DNAStatMSAProfileDialog.obj
 0001:00003360       ??1?$QSet@D@@QAE@XZ        10004360 f i DNAStatMSAProfileDialog.obj
 0001:00003390       ??1?$QVector@D@@QAE@XZ     10004390 f i DNAStatMSAProfileDialog.obj
 0001:000033d0       ??1?$QVector@H@@QAE@XZ     100043d0 f i DNAStatMSAProfileDialog.obj
 0001:00003410       ??1?$QVector@UColumnStat@DNAStatMSAProfileTask@U2@@@@QAE@XZ 10004410 f i DNAStatMSAProfileDialog.obj
 0001:00003470       ??1?$basic_string@DU?$char_traits@D@std@@V?$allocator@D@2@@std@@QAE@XZ 10004470 f i DNAStatMSAProfileDialog.obj
 0001:000034a0       ??1AbstractInt32Id@U2@@UAE@XZ 100044a0 f i DNAStatMSAProfileDialog.obj
 0001:000034b0       ??1ColumnStat@DNAStatMSAProfileTask@U2@@QAE@XZ 100044b0 f i DNAStatMSAProfileDialog.obj
 0001:000034f0       ??1DNAStatMSAProfileDialog@U2@@UAE@XZ 100044f0 f i DNAStatMSAProfileDialog.obj
 0001:00003500       ??1DNAStatMSAProfileTask@U2@@UAE@XZ 10004500 f i DNAStatMSAProfileDialog.obj
 0001:000036c0       ??1DNAStatMSAProfileTaskSettings@U2@@QAE@XZ 100046c0 f i DNAStatMSAProfileDialog.obj
 0001:00003740       ??1QStringList@@QAE@XZ     10004740 f i DNAStatMSAProfileDialog.obj
 0001:00003750       ??1ServiceType@U2@@UAE@XZ  10004750 f i DNAStatMSAProfileDialog.obj
 0001:00003760       ??1_Generic_error_category@std@@UAE@XZ 10004760 f i DNAStatMSAProfileDialog.obj
 0001:00003770       ??1_Iostream_error_category@std@@UAE@XZ 10004770 f i DNAStatMSAProfileDialog.obj
 0001:00003780       ??1_System_error_category@std@@UAE@XZ 10004780 f i DNAStatMSAProfileDialog.obj
 0001:00003790       ??1error_category@std@@UAE@XZ 10004790 f i DNAStatMSAProfileDialog.obj
 0001:000037a0       ??2@YAPAXIPAX@Z            100047a0 f i DNAStatMSAProfileDialog.obj
 0001:000037b0       ??3@YAXPAX0@Z              100047b0 f i DNAStatMSAProfileDialog.obj
 0001:000037c0       ??4?$QHash@DH@@QAEAAV0@$$QAV0@@Z 100047c0 f i DNAStatMSAProfileDialog.obj
 0001:000037e0       ??4?$QHash@DUQHashDummyValue@@@@QAEAAV0@$$QAV0@@Z 100047e0 f i DNAStatMSAProfileDialog.obj
 0001:00003800       ??4?$QList@VQString@@@@QAEAAV0@$$QAV0@@Z 10004800 f i DNAStatMSAProfileDialog.obj
 0001:00003820       ??4?$QVector@D@@QAE?AV0@$$QAV0@@Z 10004820 f i DNAStatMSAProfileDialog.obj
 0001:00003850       ??4?$QVector@UColumnStat@DNAStatMSAProfileTask@U2@@@@QAE?AV0@$$QAV0@@Z 10004850 f i DNAStatMSAProfileDialog.obj
 0001:00003880       ??6QStringList@@QAEAAV0@ABVQString@@@Z 10004880 f i DNAStatMSAProfileDialog.obj
 0001:000038a0       ??8error_category@std@@QBE_NABV01@@Z 100048a0 f i DNAStatMSAProfileDialog.obj
 0001:000038b0       ??8error_condition@std@@QBE_NABV01@@Z 100048b0 f i DNAStatMSAProfileDialog.obj
 0001:000038d0       ??A?$QHash@DH@@QAEAAHABD@Z 100048d0 f i DNAStatMSAProfileDialog.obj
 0001:000039c0       ??A?$QVector@H@@QAEAAHH@Z  100049c0 f i DNAStatMSAProfileDialog.obj
 0001:00003a40       ??A?$QVector@UColumnStat@DNAStatMSAProfileTask@U2@@@@QAEAAUColumnStat@DNAStatMSAProfileTask@U2@@H@Z 10004a40 f i DNAStatMSAProfileDialog.obj
 0001:00003ac0       ??BQFlag@@QBEHXZ           10004ac0 f i DNAStatMSAProfileDialog.obj
 0001:00003ad0       ??H@YA?BVQString@@ABV0@0@Z 10004ad0 f i DNAStatMSAProfileDialog.obj
 0001:00003b40       ??H@YA?BVQString@@ABV0@PBD@Z 10004b40 f i DNAStatMSAProfileDialog.obj
 0001:00003be0       ??H@YA?BVQString@@PBDABV0@@Z 10004be0 f i DNAStatMSAProfileDialog.obj
 0001:00003eb0       ??U?$QFlags@W4OpenModeFlag@QIODevice@@@@QBE?AV0@W4OpenModeFlag@QIODevice@@@Z 10004eb0 f i DNAStatMSAProfileDialog.obj
 0001:00003ed0       ??U?$QFlags@W4StandardButton@QDialogButtonBox@@@@QBE?AV0@W4StandardButton@QDialogButtonBox@@@Z 10004ed0 f i DNAStatMSAProfileDialog.obj
 0001:00003ef0       ??U?$QFlags@W4TaskFlag@U2@@@@QBE?AV0@W4TaskFlag@U2@@@Z 10004ef0 f i DNAStatMSAProfileDialog.obj
 0001:00003f10       ??U@YA?AV?$QFlags@W4OpenModeFlag@QIODevice@@@@W4OpenModeFlag@QIODevice@@0@Z 10004f10 f i DNAStatMSAProfileDialog.obj
 0001:00003f20       ??U@YA?AV?$QFlags@W4StandardButton@QDialogButtonBox@@@@W4StandardButton@QDialogButtonBox@@0@Z 10004f20 f i DNAStatMSAProfileDialog.obj
 0001:00003f30       ??_EDNAStatMSAProfileDialog@U2@@W7AEPAXI@Z 10004f30 f i DNAStatMSAProfileDialog.obj
 0001:00003f38       ??_EQCheckBox@@W7AEPAXI@Z  10004f38 f i DNAStatMSAProfileDialog.obj
 0001:00003f40       ??_EQDialogButtonBox@@W7AEPAXI@Z 10004f40 f i DNAStatMSAProfileDialog.obj
 0001:00003f48       ??_EQGridLayout@@W7AEPAXI@Z 10004f48 f i DNAStatMSAProfileDialog.obj
 0001:00003f50       ??_EQGroupBox@@W7AEPAXI@Z  10004f50 f i DNAStatMSAProfileDialog.obj
 0001:00003f58       ??_EQLabel@@W7AEPAXI@Z     10004f58 f i DNAStatMSAProfileDialog.obj
 0001:00003f60       ??_EQLineEdit@@W7AEPAXI@Z  10004f60 f i DNAStatMSAProfileDialog.obj
 0001:00003f68       ??_EQRadioButton@@W7AEPAXI@Z 10004f68 f i DNAStatMSAProfileDialog.obj
 0001:00003f70       ??_EQToolButton@@W7AEPAXI@Z 10004f70 f i DNAStatMSAProfileDialog.obj
 0001:00003f78       ??_EQVBoxLayout@@W7AEPAXI@Z 10004f78 f i DNAStatMSAProfileDialog.obj
 0001:00003f80       ??_EWebWindow@U2@@W7AEPAXI@Z 10004f80 f i DNAStatMSAProfileDialog.obj
 0001:00003f90       ??_G?$AbstractId@H@U2@@MAEPAXI@Z 10004f90 f i DNAStatMSAProfileDialog.obj
 0001:00003f90       ??_E?$AbstractId@H@U2@@MAEPAXI@Z 10004f90 f i DNAStatMSAProfileDialog.obj
 0001:00003fc0       ??_GAbstractInt32Id@U2@@UAEPAXI@Z 10004fc0 f i DNAStatMSAProfileDialog.obj
 0001:00003fc0       ??_EAbstractInt32Id@U2@@UAEPAXI@Z 10004fc0 f i DNAStatMSAProfileDialog.obj
 0001:00003ff0       ??_GColumnStat@DNAStatMSAProfileTask@U2@@QAEPAXI@Z 10004ff0 f i DNAStatMSAProfileDialog.obj
 0001:00004050       ??_GDNAStatMSAProfileDialog@U2@@UAEPAXI@Z 10005050 f i DNAStatMSAProfileDialog.obj
 0001:00004050       ??_EDNAStatMSAProfileDialog@U2@@UAEPAXI@Z 10005050 f i DNAStatMSAProfileDialog.obj
 0001:00004080       ??_GDNAStatMSAProfileTask@U2@@UAEPAXI@Z 10005080 f i DNAStatMSAProfileDialog.obj
 0001:00004080       ??_EDNAStatMSAProfileTask@U2@@UAEPAXI@Z 10005080 f i DNAStatMSAProfileDialog.obj
 0001:000040b0       ??_EHelpButton@U2@@UAEPAXI@Z 100050b0 f i DNAStatMSAProfileDialog.obj
 0001:000040b0       ??_GHelpButton@U2@@UAEPAXI@Z 100050b0 f i DNAStatMSAProfileDialog.obj
 0001:000040e0       ??_EQCheckBox@@UAEPAXI@Z   100050e0 f i DNAStatMSAProfileDialog.obj
 0001:000040e0       ??_GQCheckBox@@UAEPAXI@Z   100050e0 f i DNAStatMSAProfileDialog.obj
 0001:00004110       ??_GQDialogButtonBox@@UAEPAXI@Z 10005110 f i DNAStatMSAProfileDialog.obj
 0001:00004110       ??_EQDialogButtonBox@@UAEPAXI@Z 10005110 f i DNAStatMSAProfileDialog.obj
 0001:00004140       ??_GQFile@@UAEPAXI@Z       10005140 f i DNAStatMSAProfileDialog.obj
 0001:00004140       ??_EQFile@@UAEPAXI@Z       10005140 f i DNAStatMSAProfileDialog.obj
 0001:00004170       ??_GQGridLayout@@UAEPAXI@Z 10005170 f i DNAStatMSAProfileDialog.obj
 0001:00004170       ??_EQGridLayout@@UAEPAXI@Z 10005170 f i DNAStatMSAProfileDialog.obj
 0001:000041a0       ??_EQGroupBox@@UAEPAXI@Z   100051a0 f i DNAStatMSAProfileDialog.obj
 0001:000041a0       ??_GQGroupBox@@UAEPAXI@Z   100051a0 f i DNAStatMSAProfileDialog.obj
 0001:000041d0       ??_GQLabel@@UAEPAXI@Z      100051d0 f i DNAStatMSAProfileDialog.obj
 0001:000041d0       ??_EQLabel@@UAEPAXI@Z      100051d0 f i DNAStatMSAProfileDialog.obj
 0001:00004200       ??_EQLineEdit@@UAEPAXI@Z   10005200 f i DNAStatMSAProfileDialog.obj
 0001:00004200       ??_GQLineEdit@@UAEPAXI@Z   10005200 f i DNAStatMSAProfileDialog.obj
 0001:00004230       ??_EQRadioButton@@UAEPAXI@Z 10005230 f i DNAStatMSAProfileDialog.obj
 0001:00004230       ??_GQRadioButton@@UAEPAXI@Z 10005230 f i DNAStatMSAProfileDialog.obj
 0001:00004260       ??_GQString@@QAEPAXI@Z     10005260 f i DNAStatMSAProfileDialog.obj
 0001:00004290       ??_EQToolButton@@UAEPAXI@Z 10005290 f i DNAStatMSAProfileDialog.obj
 0001:00004290       ??_GQToolButton@@UAEPAXI@Z 10005290 f i DNAStatMSAProfileDialog.obj
 0001:000042c0       ??_EQVBoxLayout@@UAEPAXI@Z 100052c0 f i DNAStatMSAProfileDialog.obj
 0001:000042c0       ??_GQVBoxLayout@@UAEPAXI@Z 100052c0 f i DNAStatMSAProfileDialog.obj
 0001:000042f0       ??_GSaveDocumentController@U2@@UAEPAXI@Z 100052f0 f i DNAStatMSAProfileDialog.obj
 0001:000042f0       ??_ESaveDocumentController@U2@@UAEPAXI@Z 100052f0 f i DNAStatMSAProfileDialog.obj
 0001:00004320       ??_EServiceType@U2@@UAEPAXI@Z 10005320 f i DNAStatMSAProfileDialog.obj
 0001:00004320       ??_GServiceType@U2@@UAEPAXI@Z 10005320 f i DNAStatMSAProfileDialog.obj
 0001:00004350       ??_GWebWindow@U2@@UAEPAXI@Z 10005350 f i DNAStatMSAProfileDialog.obj
 0001:00004350       ??_EWebWindow@U2@@UAEPAXI@Z 10005350 f i DNAStatMSAProfileDialog.obj
 0001:00004380       ??_E_Generic_error_category@std@@UAEPAXI@Z 10005380 f i DNAStatMSAProfileDialog.obj
 0001:00004380       ??_G_Generic_error_category@std@@UAEPAXI@Z 10005380 f i DNAStatMSAProfileDialog.obj
 0001:000043b0       ??_E_Iostream_error_category@std@@UAEPAXI@Z 100053b0 f i DNAStatMSAProfileDialog.obj
 0001:000043b0       ??_G_Iostream_error_category@std@@UAEPAXI@Z 100053b0 f i DNAStatMSAProfileDialog.obj
 0001:000043e0       ??_E_System_error_category@std@@UAEPAXI@Z 100053e0 f i DNAStatMSAProfileDialog.obj
 0001:000043e0       ??_G_System_error_category@std@@UAEPAXI@Z 100053e0 f i DNAStatMSAProfileDialog.obj
 0001:00004410       ??_Gerror_category@std@@UAEPAXI@Z 10005410 f i DNAStatMSAProfileDialog.obj
 0001:00004410       ??_Eerror_category@std@@UAEPAXI@Z 10005410 f i DNAStatMSAProfileDialog.obj
 0001:00004440       ?_Copy@?$basic_string@DU?$char_traits@D@std@@V?$allocator@D@2@@std@@QAEXII@Z 10005440 f i DNAStatMSAProfileDialog.obj
 0001:00004590       ?_Eos@?$basic_string@DU?$char_traits@D@std@@V?$allocator@D@2@@std@@QAEXI@Z 10005590 f i DNAStatMSAProfileDialog.obj
 0001:000045c0       ?_Getal@?$_String_alloc@$0A@U?$_String_base_types@DV?$allocator@D@std@@@std@@@std@@QBE?AU?$_Wrap_alloc@V?$allocator@D@std@@@2@XZ 100055c0 f i DNAStatMSAProfileDialog.obj
 0001:000045d0       ?_Grow@?$basic_string@DU?$char_traits@D@std@@V?$allocator@D@2@@std@@QAE_NI_N@Z 100055d0 f i DNAStatMSAProfileDialog.obj
 0001:00004680       ?_Inside@?$basic_string@DU?$char_traits@D@std@@V?$allocator@D@2@@std@@QAE_NPBD@Z 10005680 f i DNAStatMSAProfileDialog.obj
 0001:000046c0       ?_Myptr@?$_String_val@U?$_Simple_types@D@std@@@std@@QAEPADXZ 100056c0 f i DNAStatMSAProfileDialog.obj
 0001:000046d0       ?_Myptr@?$_String_val@U?$_Simple_types@D@std@@@std@@QBEPBDXZ 100056d0 f i DNAStatMSAProfileDialog.obj
 0001:000046e0       ?_Tidy@?$basic_string@DU?$char_traits@D@std@@V?$allocator@D@2@@std@@QAEX_NI@Z 100056e0 f i DNAStatMSAProfileDialog.obj
 0001:00004730       ?_Xlen@?$basic_string@DU?$char_traits@D@std@@V?$allocator@D@2@@std@@QBEXXZ 10005730 f i DNAStatMSAProfileDialog.obj
 0001:00004740       ?_Xran@?$basic_string@DU?$char_traits@D@std@@V?$allocator@D@2@@std@@QBEXXZ 10005740 f i DNAStatMSAProfileDialog.obj
 0001:00004750       ?accept@DNAStatMSAProfileDialog@U2@@UAEXXZ 10005750 f   DNAStatMSAProfileDialog.obj
 0001:00004960       ?alignOfNode@?$QHash@DH@@CAHXZ 10005960 f i DNAStatMSAProfileDialog.obj
 0001:00004970       ?alignOfNode@?$QHash@DUQHashDummyValue@@@@CAHXZ 10005970 f i DNAStatMSAProfileDialog.obj
 0001:00004980       ?allocate@?$QTypedArrayData@D@@SAPAU1@IV?$QFlags@W4AllocationOption@QArrayData@@@@@Z 10005980 f i DNAStatMSAProfileDialog.obj
 0001:000049a0       ?allocate@?$QTypedArrayData@H@@SAPAU1@IV?$QFlags@W4AllocationOption@QArrayData@@@@@Z 100059a0 f i DNAStatMSAProfileDialog.obj
 0001:000049c0       ?allocate@?$QTypedArrayData@UColumnStat@DNAStatMSAProfileTask@U2@@@@SAPAU1@IV?$QFlags@W4AllocationOption@QArrayData@@@@@Z 100059c0 f i DNAStatMSAProfileDialog.obj
 0001:000049e0       ?allocate@?$_Wrap_alloc@V?$allocator@D@std@@@std@@QAEPADI@Z 100059e0 f i DNAStatMSAProfileDialog.obj
 0001:00004a10       ?allocate@?$allocator@D@std@@QAEPADI@Z 10005a10 f i DNAStatMSAProfileDialog.obj
 0001:00004a40       ?append@?$QList@VQString@@@@QAEXABVQString@@@Z 10005a40 f i DNAStatMSAProfileDialog.obj
 0001:00004b30       ?assign@?$basic_string@DU?$char_traits@D@std@@V?$allocator@D@2@@std@@QAEAAV12@ABV12@II@Z 10005b30 f i DNAStatMSAProfileDialog.obj
 0001:00004c50       ?assign@?$basic_string@DU?$char_traits@D@std@@V?$allocator@D@2@@std@@QAEAAV12@PBD@Z 10005c50 f i DNAStatMSAProfileDialog.obj
 0001:00004c90       ?assign@?$basic_string@DU?$char_traits@D@std@@V?$allocator@D@2@@std@@QAEAAV12@PBDI@Z 10005c90 f i DNAStatMSAProfileDialog.obj
 0001:00004d90       ?assign@?$char_traits@D@std@@SAXAADABD@Z 10005d90 f i DNAStatMSAProfileDialog.obj
 0001:00004da0       ?begin@?$QTypedArrayData@D@@QAEPADPAD@Z 10005da0 f i DNAStatMSAProfileDialog.obj
 0001:00004db0       ?begin@?$QTypedArrayData@H@@QAEPAHPAH@Z 10005db0 f i DNAStatMSAProfileDialog.obj
 0001:00004dc0       ?begin@?$QTypedArrayData@UColumnStat@DNAStatMSAProfileTask@U2@@@@QAEPAUColumnStat@DNAStatMSAProfileTask@U2@@PAU234@@Z 10005dc0 f i DNAStatMSAProfileDialog.obj
 0001:00004dd0       ?category@error_code@std@@QBEABVerror_category@2@XZ 10005dd0 f i DNAStatMSAProfileDialog.obj
 0001:00004de0       ?category@error_condition@std@@QBEABVerror_category@2@XZ 10005de0 f i DNAStatMSAProfileDialog.obj
 0001:00004df0       ?clear@?$QHash@DH@@QAEXXZ  10005df0 f i DNAStatMSAProfileDialog.obj
 0001:00004e30       ?clear@?$QHash@DUQHashDummyValue@@@@QAEXXZ 10005e30 f i DNAStatMSAProfileDialog.obj
 0001:00004e70       ?clear@?$QList@VQString@@@@QAEXXZ 10005e70 f i DNAStatMSAProfileDialog.obj
 0001:00004e90       ?clear@?$QSet@D@@QAEXXZ    10005e90 f i DNAStatMSAProfileDialog.obj
 0001:00004ed0       ?clear@?$QVector@D@@QAEXXZ 10005ed0 f i DNAStatMSAProfileDialog.obj
 0001:00004fa0       ?clear@?$QVector@UColumnStat@DNAStatMSAProfileTask@U2@@@@QAEXXZ 10005fa0 f i DNAStatMSAProfileDialog.obj
 0001:00005090       ?computeStats@DNAStatMSAProfileTask@U2@@AAEXXZ 10006090 f   DNAStatMSAProfileDialog.obj
 0001:00005750       ?concrete@?$QHash@DH@@CAPAU?$QHashNode@DH@@PAUNode@QHashData@@@Z 10006750 f i DNAStatMSAProfileDialog.obj
 0001:00005760       ?concrete@?$QHash@DUQHashDummyValue@@@@CAPAU?$QHashNode@DUQHashDummyValue@@@@PAUNode@QHashData@@@Z 10006760 f i DNAStatMSAProfileDialog.obj
 0001:00005770       ?contains@?$QHash@DUQHashDummyValue@@@@QBE_NABD@Z 10006770 f i DNAStatMSAProfileDialog.obj
 0001:000057d0       ?contains@?$QSet@D@@QBE_NABD@Z 100067d0 f i DNAStatMSAProfileDialog.obj
 0001:000057e0       ?copy@?$char_traits@D@std@@SAPADPADPBDI@Z 100067e0 f i DNAStatMSAProfileDialog.obj
 0001:00005800       ?copyConstruct@?$QVector@D@@AAEXPBD0PAD@Z 10006800 f i DNAStatMSAProfileDialog.obj
 0001:00005820       ?copyConstruct@?$QVector@H@@AAEXPBH0PAH@Z 10006820 f i DNAStatMSAProfileDialog.obj
 0001:00005840       ?copyConstruct@?$QVector@UColumnStat@DNAStatMSAProfileTask@U2@@@@AAEXPBUColumnStat@DNAStatMSAProfileTask@U2@@0PAU234@@Z 10006840 f i DNAStatMSAProfileDialog.obj
 0001:000058c0       ?createNode@?$QHash@DH@@AAEPAU?$QHashNode@DH@@IABDABHPAPAU2@@Z 100068c0 f i DNAStatMSAProfileDialog.obj
 0001:00005920       ?createNode@?$QHash@DUQHashDummyValue@@@@AAEPAU?$QHashNode@DUQHashDummyValue@@@@IABDABUQHashDummyValue@@PAPAU2@@Z 10006920 f i DNAStatMSAProfileDialog.obj
 0001:00005970       ?data@?$QTypedArrayData@D@@QAEPADXZ 10006970 f i DNAStatMSAProfileDialog.obj
 0001:00005980       ?data@?$QTypedArrayData@H@@QAEPAHXZ 10006980 f i DNAStatMSAProfileDialog.obj
 0001:00005990       ?data@?$QTypedArrayData@UColumnStat@DNAStatMSAProfileTask@U2@@@@QAEPAUColumnStat@DNAStatMSAProfileTask@U2@@XZ 10006990 f i DNAStatMSAProfileDialog.obj
 0001:000059a0       ?data@?$QVector@H@@QAEPAHXZ 100069a0 f i DNAStatMSAProfileDialog.obj
 0001:00005a00       ?data@?$QVector@UColumnStat@DNAStatMSAProfileTask@U2@@@@QAEPAUColumnStat@DNAStatMSAProfileTask@U2@@XZ 10006a00 f i DNAStatMSAProfileDialog.obj
 0001:00005a60       ?data_ptr@?$QStaticStringData@$04@@QBEPAU?$QTypedArrayData@G@@XZ 10006a60 f i DNAStatMSAProfileDialog.obj
 0001:00005a70       ?data_ptr@?$QStaticStringData@$05@@QBEPAU?$QTypedArrayData@G@@XZ 10006a70 f i DNAStatMSAProfileDialog.obj
 0001:00005a80       ?data_ptr@?$QStaticStringData@$06@@QBEPAU?$QTypedArrayData@G@@XZ 10006a80 f i DNAStatMSAProfileDialog.obj
 0001:00005a90       ?data_ptr@?$QStaticStringData@$07@@QBEPAU?$QTypedArrayData@G@@XZ 10006a90 f i DNAStatMSAProfileDialog.obj
 0001:00005aa0       ?data_ptr@?$QStaticStringData@$08@@QBEPAU?$QTypedArrayData@G@@XZ 10006aa0 f i DNAStatMSAProfileDialog.obj
 0001:00005ab0       ?data_ptr@?$QStaticStringData@$09@@QBEPAU?$QTypedArrayData@G@@XZ 10006ab0 f i DNAStatMSAProfileDialog.obj
 0001:00005ac0       ?data_ptr@?$QStaticStringData@$0BA@@@QBEPAU?$QTypedArrayData@G@@XZ 10006ac0 f i DNAStatMSAProfileDialog.obj
 0001:00005ad0       ?data_ptr@?$QStaticStringData@$0BC@@@QBEPAU?$QTypedArrayData@G@@XZ 10006ad0 f i DNAStatMSAProfileDialog.obj
 0001:00005ae0       ?data_ptr@?$QStaticStringData@$0BH@@@QBEPAU?$QTypedArrayData@G@@XZ 10006ae0 f i DNAStatMSAProfileDialog.obj
 0001:00005af0       ?data_ptr@?$QStaticStringData@$0M@@@QBEPAU?$QTypedArrayData@G@@XZ 10006af0 f i DNAStatMSAProfileDialog.obj
 0001:00005b00       ?data_ptr@?$QStaticStringData@$0O@@@QBEPAU?$QTypedArrayData@G@@XZ 10006b00 f i DNAStatMSAProfileDialog.obj
 0001:00005b10       ?dealloc@?$QList@VMultipleSequenceAlignmentRow@U2@@@@AAEXPAUData@QListData@@@Z 10006b10 f i DNAStatMSAProfileDialog.obj
 0001:00005b60       ?dealloc@?$QList@VQString@@@@AAEXPAUData@QListData@@@Z 10006b60 f i DNAStatMSAProfileDialog.obj
 0001:00005ba0       ?deallocate@?$QTypedArrayData@D@@SAXPAUQArrayData@@@Z 10006ba0 f i DNAStatMSAProfileDialog.obj
 0001:00005bc0       ?deallocate@?$QTypedArrayData@H@@SAXPAUQArrayData@@@Z 10006bc0 f i DNAStatMSAProfileDialog.obj
 0001:00005be0       ?deallocate@?$QTypedArrayData@UColumnStat@DNAStatMSAProfileTask@U2@@@@SAXPAUQArrayData@@@Z 10006be0 f i DNAStatMSAProfileDialog.obj
 0001:00005c00       ?deallocate@?$_Wrap_alloc@V?$allocator@D@std@@@std@@QAEXPADI@Z 10006c00 f i DNAStatMSAProfileDialog.obj
 0001:00005c20       ?deallocate@?$allocator@D@std@@QAEXPADI@Z 10006c20 f i DNAStatMSAProfileDialog.obj
 0001:00005c40       ?defaultConstruct@?$QVector@D@@AAEXPAD0@Z 10006c40 f i DNAStatMSAProfileDialog.obj
 0001:00005c60       ?defaultConstruct@?$QVector@H@@AAEXPAH0@Z 10006c60 f i DNAStatMSAProfileDialog.obj
 0001:00005c80       ?defaultConstruct@?$QVector@UColumnStat@DNAStatMSAProfileTask@U2@@@@AAEXPAUColumnStat@DNAStatMSAProfileTask@U2@@0@Z 10006c80 f i DNAStatMSAProfileDialog.obj
 0001:00005cb0       ?default_error_condition@_System_error_category@std@@UBE?AVerror_condition@2@H@Z 10006cb0 f i DNAStatMSAProfileDialog.obj
 0001:00005cf0       ?default_error_condition@error_category@std@@UBE?AVerror_condition@2@H@Z 10006cf0 f i DNAStatMSAProfileDialog.obj
 0001:00005d10       ?deleteNode2@?$QHash@DH@@CAXPAUNode@QHashData@@@Z 10006d10 f i DNAStatMSAProfileDialog.obj
 0001:00005d20       ?deleteNode2@?$QHash@DUQHashDummyValue@@@@CAXPAUNode@QHashData@@@Z 10006d20 f i DNAStatMSAProfileDialog.obj
 0001:00005d30       ?deleteNode@?$QHash@DUQHashDummyValue@@@@AAEXPAU?$QHashNode@DUQHashDummyValue@@@@@Z 10006d30 f i DNAStatMSAProfileDialog.obj
 0001:00005d40       ?deref@?$QBasicAtomicInteger@H@@QAE_NXZ 10006d40 f i DNAStatMSAProfileDialog.obj
 0001:00005d50       ?deref@RefCount@QtPrivate@@QAE_NXZ 10006d50 f i DNAStatMSAProfileDialog.obj
 0001:00005d70       ?destruct@?$QVector@D@@AAEXPAD0@Z 10006d70 f i DNAStatMSAProfileDialog.obj
 0001:00005d80       ?destruct@?$QVector@H@@AAEXPAH0@Z 10006d80 f i DNAStatMSAProfileDialog.obj
 0001:00005d90       ?destruct@?$QVector@UColumnStat@DNAStatMSAProfileTask@U2@@@@AAEXPAUColumnStat@DNAStatMSAProfileTask@U2@@0@Z 10006d90 f i DNAStatMSAProfileDialog.obj
 0001:00005df0       ?detach@?$QHash@DH@@QAEXXZ 10006df0 f i DNAStatMSAProfileDialog.obj
 0001:00005e50       ?detach@?$QHash@DUQHashDummyValue@@@@QAEXXZ 10006e50 f i DNAStatMSAProfileDialog.obj
 0001:00005eb0       ?detach@?$QVector@H@@QAEXXZ 10006eb0 f i DNAStatMSAProfileDialog.obj
 0001:00005f00       ?detach@?$QVector@UColumnStat@DNAStatMSAProfileTask@U2@@@@QAEXXZ 10006f00 f i DNAStatMSAProfileDialog.obj
 0001:00005f50       ?detach_helper@?$QHash@DH@@AAEXXZ 10006f50 f i DNAStatMSAProfileDialog.obj
 0001:00005fa0       ?detach_helper@?$QHash@DUQHashDummyValue@@@@AAEXXZ 10006fa0 f i DNAStatMSAProfileDialog.obj
 0001:00005ff0       ?detach_helper_grow@?$QList@VQString@@@@AAEPAUNode@1@HH@Z 10006ff0 f i DNAStatMSAProfileDialog.obj
 0001:00006170       ?duplicateNode@?$QHash@DH@@CAXPAUNode@QHashData@@PAX@Z 10007170 f i DNAStatMSAProfileDialog.obj
 0001:000061a0       ?duplicateNode@?$QHash@DUQHashDummyValue@@@@CAXPAUNode@QHashData@@PAX@Z 100071a0 f i DNAStatMSAProfileDialog.obj
 0001:000061d0       ?end@?$QTypedArrayData@D@@QAEPADPAD@Z 100071d0 f i DNAStatMSAProfileDialog.obj
 0001:000061e0       ?end@?$QTypedArrayData@H@@QAEPAHPAH@Z 100071e0 f i DNAStatMSAProfileDialog.obj
 0001:00006200       ?end@?$QTypedArrayData@UColumnStat@DNAStatMSAProfileTask@U2@@@@QAEPAUColumnStat@DNAStatMSAProfileTask@U2@@PAU234@@Z 10007200 f i DNAStatMSAProfileDialog.obj
 0001:00006220       ?equivalent@error_category@std@@UBE_NABVerror_code@2@H@Z 10007220 f i DNAStatMSAProfileDialog.obj
 0001:00006240       ?equivalent@error_category@std@@UBE_NHABVerror_condition@2@@Z 10007240 f i DNAStatMSAProfileDialog.obj
 0001:00006280       ?erase@?$basic_string@DU?$char_traits@D@std@@V?$allocator@D@2@@std@@QAEAAV12@I@Z 10007280 f i DNAStatMSAProfileDialog.obj
 0001:000062c0       ?erase@?$basic_string@DU?$char_traits@D@std@@V?$allocator@D@2@@std@@QAEAAV12@II@Z 100072c0 f i DNAStatMSAProfileDialog.obj
 0001:00006360       ?findNode@?$QHash@DH@@ABEPAPAU?$QHashNode@DH@@ABDPAI@Z 10007360 f i DNAStatMSAProfileDialog.obj
 0001:000063d0       ?findNode@?$QHash@DUQHashDummyValue@@@@ABEPAPAU?$QHashNode@DUQHashDummyValue@@@@ABDPAI@Z 100073d0 f i DNAStatMSAProfileDialog.obj
 0001:00006440       ?freeData@?$QHash@DH@@AAEXPAUQHashData@@@Z 10007440 f i DNAStatMSAProfileDialog.obj
 0001:00006460       ?freeData@?$QHash@DUQHashDummyValue@@@@AAEXPAUQHashData@@@Z 10007460 f i DNAStatMSAProfileDialog.obj
 0001:00006480       ?freeData@?$QVector@D@@AAEXPAU?$QTypedArrayData@D@@@Z 10007480 f i DNAStatMSAProfileDialog.obj
 0001:000064b0       ?freeData@?$QVector@H@@AAEXPAU?$QTypedArrayData@H@@@Z 100074b0 f i DNAStatMSAProfileDialog.obj
 0001:000064e0       ?freeData@?$QVector@UColumnStat@DNAStatMSAProfileTask@U2@@@@AAEXPAU?$QTypedArrayData@UColumnStat@DNAStatMSAProfileTask@U2@@@@@Z 100074e0 f i DNAStatMSAProfileDialog.obj
 0001:00006520       ?generateReport@DNAStatMSAProfileTask@U2@@UBE?AVQString@@XZ 10007520 f   DNAStatMSAProfileDialog.obj
 0001:00006750       ?generic_category@std@@YAABVerror_category@1@XZ 10007750 f i DNAStatMSAProfileDialog.obj
 0001:00006760       ?initSaveController@DNAStatMSAProfileDialog@U2@@AAEXXZ 10007760 f   DNAStatMSAProfileDialog.obj
 0001:00006ac0       ?insert@?$QHash@DUQHashDummyValue@@@@QAE?AViterator@1@ABDABUQHashDummyValue@@@Z 10007ac0 f i DNAStatMSAProfileDialog.obj
 0001:00006b90       ?insert@?$QSet@D@@QAE?AViterator@1@ABD@Z 10007b90 f i DNAStatMSAProfileDialog.obj
 0001:00006bc0       ?isDetached@?$QVector@H@@QBE_NXZ 10007bc0 f i DNAStatMSAProfileDialog.obj
 0001:00006bf0       ?isDetached@?$QVector@UColumnStat@DNAStatMSAProfileTask@U2@@@@QBE_NXZ 10007bf0 f i DNAStatMSAProfileDialog.obj
 0001:00006c20       ?isEmpty@?$QHash@DUQHashDummyValue@@@@QBE_NXZ 10007c20 f i DNAStatMSAProfileDialog.obj
 0001:00006c30       ?isReportingEnabled@DNAStatMSAProfileTask@U2@@UBE_NXZ 10007c30 f   DNAStatMSAProfileDialog.obj
 0001:00006c60       ?isShared@RefCount@QtPrivate@@QBE_NXZ 10007c60 f i DNAStatMSAProfileDialog.obj
 0001:00006c80       ?isValid@AbstractInt32Id@U2@@UBE_NXZ 10007c80 f i DNAStatMSAProfileDialog.obj
 0001:00006c90       ?length@?$char_traits@D@std@@SAIPBD@Z 10007c90 f i DNAStatMSAProfileDialog.obj
 0001:00006cb0       ?load@?$QBasicAtomicInteger@H@@QBEHXZ 10007cb0 f i DNAStatMSAProfileDialog.obj
 0001:00006cc0       ?max_size@?$_Wrap_alloc@V?$allocator@D@std@@@std@@QBEIXZ 10007cc0 f i DNAStatMSAProfileDialog.obj
 0001:00006cd0       ?max_size@?$allocator@D@std@@QBEIXZ 10007cd0 f i DNAStatMSAProfileDialog.obj
 0001:00006ce0       ?max_size@?$allocator_traits@V?$allocator@D@std@@@std@@SAIABV?$allocator@D@2@@Z 10007ce0 f i DNAStatMSAProfileDialog.obj
 0001:00006cf0       ?max_size@?$basic_string@DU?$char_traits@D@std@@V?$allocator@D@2@@std@@QBEIXZ 10007cf0 f i DNAStatMSAProfileDialog.obj
 0001:00006d00       ?message@_Generic_error_category@std@@UBE?AV?$basic_string@DU?$char_traits@D@std@@V?$allocator@D@2@@2@H@Z 10007d00 f i DNAStatMSAProfileDialog.obj
 0001:00006d80       ?message@_Iostream_error_category@std@@UBE?AV?$basic_string@DU?$char_traits@D@std@@V?$allocator@D@2@@2@H@Z 10007d80 f i DNAStatMSAProfileDialog.obj
 0001:00006dd0       ?message@_System_error_category@std@@UBE?AV?$basic_string@DU?$char_traits@D@std@@V?$allocator@D@2@@2@H@Z 10007dd0 f i DNAStatMSAProfileDialog.obj
 0001:00006e50       ?move@?$char_traits@D@std@@SAPADPADPBDI@Z 10007e50 f i DNAStatMSAProfileDialog.obj
 0001:00006e70       ?name@_Generic_error_category@std@@UBEPBDXZ 10007e70 f i DNAStatMSAProfileDialog.obj
 0001:00006e80       ?name@_Iostream_error_category@std@@UBEPBDXZ 10007e80 f i DNAStatMSAProfileDialog.obj
 0001:00006e90       ?name@_System_error_category@std@@UBEPBDXZ 10007e90 f i DNAStatMSAProfileDialog.obj
 0001:00006ea0       ?node_construct@?$QList@VQString@@@@AAEXPAUNode@1@ABVQString@@@Z 10007ea0 f i DNAStatMSAProfileDialog.obj
 0001:00006ef0       ?node_copy@?$QList@VQString@@@@AAEXPAUNode@1@00@Z 10007ef0 f i DNAStatMSAProfileDialog.obj
 0001:00006f90       ?node_destruct@?$QList@VMultipleSequenceAlignmentRow@U2@@@@AAEXPAUNode@1@0@Z 10007f90 f i DNAStatMSAProfileDialog.obj
 0001:00006fc0       ?node_destruct@?$QList@VQString@@@@AAEXPAUNode@1@0@Z 10007fc0 f i DNAStatMSAProfileDialog.obj
 0001:00006ff0       ?node_destruct@?$QList@VQString@@@@AAEXPAUNode@1@@Z 10007ff0 f i DNAStatMSAProfileDialog.obj
 0001:00007000       ?qHash@@YAIDI@Z            10008000 f i DNAStatMSAProfileDialog.obj
 0001:00007010       ?qRound@@YAHN@Z            10008010 f i DNAStatMSAProfileDialog.obj
 0001:00007060       ?qt_noop@@YAXXZ            10008060 f i DNAStatMSAProfileDialog.obj
 0001:00007070       ?reallocData@?$QVector@D@@AAEXHHV?$QFlags@W4AllocationOption@QArrayData@@@@@Z 10008070 f i DNAStatMSAProfileDialog.obj
 0001:000072a0       ?reallocData@?$QVector@H@@AAEXHHV?$QFlags@W4AllocationOption@QArrayData@@@@@Z 100082a0 f i DNAStatMSAProfileDialog.obj
 0001:000074e0       ?reallocData@?$QVector@UColumnStat@DNAStatMSAProfileTask@U2@@@@AAEXHHV?$QFlags@W4AllocationOption@QArrayData@@@@@Z 100084e0 f i DNAStatMSAProfileDialog.obj
 0001:00007730       ?ref@?$QBasicAtomicInteger@H@@QAE_NXZ 10008730 f i DNAStatMSAProfileDialog.obj
 0001:00007750       ?ref@RefCount@QtPrivate@@QAE_NXZ 10008750 f i DNAStatMSAProfileDialog.obj
 0001:00007770       ?remove@?$QHash@DUQHashDummyValue@@@@QAEHABD@Z 10008770 f i DNAStatMSAProfileDialog.obj
 0001:00007840       ?remove@?$QSet@D@@QAE_NABD@Z 10008840 f i DNAStatMSAProfileDialog.obj
 0001:00007860       ?report@DNAStatMSAProfileTask@U2@@UAE?AW4ReportResult@Task@2@XZ 10008860 f   DNAStatMSAProfileDialog.obj
 0001:00007a50       ?resize@?$QVector@D@@QAEXH@Z 10008a50 f i DNAStatMSAProfileDialog.obj
 0001:00007aa0       ?resize@?$QVector@H@@QAEXH@Z 10008aa0 f i DNAStatMSAProfileDialog.obj
 0001:00007af0       ?resize@?$QVector@UColumnStat@DNAStatMSAProfileTask@U2@@@@QAEXH@Z 10008af0 f i DNAStatMSAProfileDialog.obj
 0001:00007b40       ?retranslateUi@Ui_DNAStatMSAProfileDialog@@QAEXPAVQDialog@@@Z 10008b40 f i DNAStatMSAProfileDialog.obj
 0001:00007e60       ?run@DNAStatMSAProfileTask@U2@@UAEXXZ 10008e60 f   DNAStatMSAProfileDialog.obj
 0001:000090d0       ?same_key@?$QHashNode@DH@@QBE_NIABD@Z 1000a0d0 f i DNAStatMSAProfileDialog.obj
 0001:00009100       ?same_key@?$QHashNode@DUQHashDummyValue@@@@QBE_NIABD@Z 1000a100 f i DNAStatMSAProfileDialog.obj
 0001:00009130       ?setupUi@Ui_DNAStatMSAProfileDialog@@QAEXPAVQDialog@@@Z 1000a130 f i DNAStatMSAProfileDialog.obj
 0001:00009ad0       ?sharedNull@?$QTypedArrayData@D@@SAPAU1@XZ 1000aad0 f i DNAStatMSAProfileDialog.obj
 0001:00009ae0       ?sharedNull@?$QTypedArrayData@H@@SAPAU1@XZ 1000aae0 f i DNAStatMSAProfileDialog.obj
 0001:00009af0       ?sharedNull@?$QTypedArrayData@UColumnStat@DNAStatMSAProfileTask@U2@@@@SAPAU1@XZ 1000aaf0 f i DNAStatMSAProfileDialog.obj
 0001:00009b00       ?size@?$QVector@UColumnStat@DNAStatMSAProfileTask@U2@@@@QBEHXZ 1000ab00 f i DNAStatMSAProfileDialog.obj
 0001:00009b10       ?size@?$basic_string@DU?$char_traits@D@std@@V?$allocator@D@2@@std@@QBEIXZ 1000ab10 f i DNAStatMSAProfileDialog.obj
 0001:00009b20       ?sl_formatChanged@DNAStatMSAProfileDialog@U2@@AAEXABVQString@@@Z 1000ab20 f   DNAStatMSAProfileDialog.obj
 0001:00009b60       ?sl_formatSelected@DNAStatMSAProfileDialog@U2@@AAEXXZ 1000ab60 f   DNAStatMSAProfileDialog.obj
 0001:00009b90       ?system_category@std@@YAABVerror_category@1@XZ 1000ab90 f i DNAStatMSAProfileDialog.obj
 0001:00009ba0       ?tr@DNAStatMSAProfileDialog@U2@@SA?AVQString@@PBD0H@Z 1000aba0 f i DNAStatMSAProfileDialog.obj
 0001:00009bd0       ?tr@DNAStatMSAProfileTask@U2@@SA?AVQString@@PBD0H@Z 1000abd0 f i DNAStatMSAProfileDialog.obj
 0001:00009c00       ?unsharableEmpty@?$QTypedArrayData@H@@SAPAU1@XZ 1000ac00 f i DNAStatMSAProfileDialog.obj
 0001:00009c20       ?unsharableEmpty@?$QTypedArrayData@UColumnStat@DNAStatMSAProfileTask@U2@@@@SAPAU1@XZ 1000ac20 f i DNAStatMSAProfileDialog.obj
 0001:00009c40       ?value@?$QHash@DH@@QBE?BHABD@Z 1000ac40 f i DNAStatMSAProfileDialog.obj
 0001:00009cb0       ?value@error_code@std@@QBEHXZ 1000acb0 f i DNAStatMSAProfileDialog.obj
 0001:00009cc0       ?value@error_condition@std@@QBEHXZ 1000acc0 f i DNAStatMSAProfileDialog.obj
 0001:00009cd0       _hypot                     1000acd0 f i DNAStatMSAProfileDialog.obj
 0001:00009d00       ??$?0VDNAStatMSAProfileDialog@U2@@@?$QWeakPointer@VQObject@@@@AAE@PAVDNAStatMSAProfileDialog@U2@@_N@Z 1000ad00 f i DNAStatPlugin.obj
 0001:00009d40       ??$?0VDistanceMatrixMSAProfileDialog@U2@@@?$QWeakPointer@VQObject@@@@AAE@PAVDistanceMatrixMSAProfileDialog@U2@@_N@Z 1000ad40 f i DNAStatPlugin.obj
 0001:00009d80       ??$qobject_cast@PAVGObjectViewAction@U2@@@@YAPAVGObjectViewAction@U2@@PAVQObject@@@Z 1000ad80 f i DNAStatPlugin.obj
 0001:00009da0       ??$qobject_cast@PAVMSAEditor@U2@@@@YAPAVMSAEditor@U2@@PAVQObject@@@Z 1000ada0 f i DNAStatPlugin.obj
 0001:00009dc0       ??0?$QForeachContainer@V?$QList@PAVGObjectViewAction@U2@@@@@@QAE@ABV?$QList@PAVGObjectViewAction@U2@@@@@Z 1000adc0 f i DNAStatPlugin.obj
 0001:00009e00       ??0?$QList@PAVGObjectViewAction@U2@@@@QAE@ABV0@@Z 1000ae00 f i DNAStatPlugin.obj
 0001:00009ec0       ??0?$QObjectScopedPointer@VDNAStatMSAProfileDialog@U2@@@U2@@QAE@PAVDNAStatMSAProfileDialog@1@@Z 1000aec0 f i DNAStatPlugin.obj
 0001:00009f00       ??0?$QObjectScopedPointer@VDistanceMatrixMSAProfileDialog@U2@@@U2@@QAE@PAVDistanceMatrixMSAProfileDialog@1@@Z 1000af00 f i DNAStatPlugin.obj
 0001:00009f40       ??0?$QPointer@VDNAStatMSAProfileDialog@U2@@@@QAE@PAVDNAStatMSAProfileDialog@U2@@@Z 1000af40 f i DNAStatPlugin.obj
 0001:00009f80       ??0?$QPointer@VDistanceMatrixMSAProfileDialog@U2@@@@QAE@PAVDistanceMatrixMSAProfileDialog@U2@@@Z 1000af80 f i DNAStatPlugin.obj
 0001:00009fc0       ??0DNAStatMSAEditorContext@U2@@QAE@PAVQObject@@@Z 1000afc0 f   DNAStatPlugin.obj
 0001:00009ff0       ??0DNAStatPlugin@U2@@QAE@XZ 1000aff0 f   DNAStatPlugin.obj
 0001:0000a120       ??0DistanceMatrixMSAEditorContext@U2@@QAE@PAVQObject@@@Z 1000b120 f   DNAStatPlugin.obj
 0001:0000a150       ??0const_iterator@?$QList@PAVGObjectViewAction@U2@@@@QAE@PAUNode@1@@Z 1000b150 f i DNAStatPlugin.obj
 0001:0000a160       ??1?$QForeachContainer@V?$QList@PAVGObjectViewAction@U2@@@@@@QAE@XZ 1000b160 f i DNAStatPlugin.obj
 0001:0000a190       ??1?$QList@PAVGObjectViewAction@U2@@@@QAE@XZ 1000b190 f i DNAStatPlugin.obj
 0001:0000a1c0       ??1?$QObjectScopedPointer@VDNAStatMSAProfileDialog@U2@@@U2@@QAE@XZ 1000b1c0 f i DNAStatPlugin.obj
 0001:0000a240       ??1?$QObjectScopedPointer@VDistanceMatrixMSAProfileDialog@U2@@@U2@@QAE@XZ 1000b240 f i DNAStatPlugin.obj
 0001:0000a2c0       ??1?$QPointer@VDNAStatMSAProfileDialog@U2@@@@QAE@XZ 1000b2c0 f i DNAStatPlugin.obj
 0001:0000a2e0       ??1?$QPointer@VDistanceMatrixMSAProfileDialog@U2@@@@QAE@XZ 1000b2e0 f i DNAStatPlugin.obj
 0001:0000a300       ??1?$QWeakPointer@VQObject@@@@QAE@XZ 1000b300 f i DNAStatPlugin.obj
 0001:0000a320       ??1DNAStatMSAEditorContext@U2@@UAE@XZ 1000b320 f i DNAStatPlugin.obj
 0001:0000a330       ??1DNAStatPlugin@U2@@UAE@XZ 1000b330 f i DNAStatPlugin.obj
 0001:0000a340       ??1DistanceMatrixMSAEditorContext@U2@@UAE@XZ 1000b340 f i DNAStatPlugin.obj
 0001:0000a350       ??1ExternalRefCountData@QtSharedPointer@@QAE@XZ 1000b350 f i DNAStatPlugin.obj
 0001:0000a360       ??3ExternalRefCountData@QtSharedPointer@@SAXPAX@Z 1000b360 f i DNAStatPlugin.obj
 0001:0000a370       ??9const_iterator@?$QList@PAVGObjectViewAction@U2@@@@QBE_NABV01@@Z 1000b370 f i DNAStatPlugin.obj
 0001:0000a390       ??C?$QObjectScopedPointer@VDNAStatMSAProfileDialog@U2@@@U2@@QBEPAVDNAStatMSAProfileDialog@1@XZ 1000b390 f i DNAStatPlugin.obj
 0001:0000a3b0       ??C?$QObjectScopedPointer@VDistanceMatrixMSAProfileDialog@U2@@@U2@@QBEPAVDistanceMatrixMSAProfileDialog@1@XZ 1000b3b0 f i DNAStatPlugin.obj
 0001:0000a3d0       ??C?$QPointer@VDNAStatMSAProfileDialog@U2@@@@QBEPAVDNAStatMSAProfileDialog@U2@@XZ 1000b3d0 f i DNAStatPlugin.obj
 0001:0000a3f0       ??C?$QPointer@VDistanceMatrixMSAProfileDialog@U2@@@@QBEPAVDistanceMatrixMSAProfileDialog@U2@@XZ 1000b3f0 f i DNAStatPlugin.obj
 0001:0000a410       ??Dconst_iterator@?$QList@PAVGObjectViewAction@U2@@@@QBEABQAVGObjectViewAction@U2@@XZ 1000b410 f i DNAStatPlugin.obj
 0001:0000a420       ??Econst_iterator@?$QList@PAVGObjectViewAction@U2@@@@QAEAAV01@XZ 1000b420 f i DNAStatPlugin.obj
 0001:0000a426       ??_EDNAStatMSAEditorContext@U2@@W7AEPAXI@Z 1000b426 f i DNAStatPlugin.obj
 0001:0000a42e       ??_EDistanceMatrixMSAEditorContext@U2@@W7AEPAXI@Z 1000b42e f i DNAStatPlugin.obj
 0001:0000a440       ??_GDNAStatMSAEditorContext@U2@@UAEPAXI@Z 1000b440 f i DNAStatPlugin.obj
 0001:0000a440       ??_EDNAStatMSAEditorContext@U2@@UAEPAXI@Z 1000b440 f i DNAStatPlugin.obj
 0001:0000a470       ??_EDNAStatPlugin@U2@@UAEPAXI@Z 1000b470 f i DNAStatPlugin.obj
 0001:0000a470       ??_GDNAStatPlugin@U2@@UAEPAXI@Z 1000b470 f i DNAStatPlugin.obj
 0001:0000a4a0       ??_GDistanceMatrixMSAEditorContext@U2@@UAEPAXI@Z 1000b4a0 f i DNAStatPlugin.obj
 0001:0000a4a0       ??_EDistanceMatrixMSAEditorContext@U2@@UAEPAXI@Z 1000b4a0 f i DNAStatPlugin.obj
 0001:0000a4d0       ??_GExternalRefCountData@QtSharedPointer@@QAEPAXI@Z 1000b4d0 f i DNAStatPlugin.obj
 0001:0000a4f0       ??_GGObjectViewAction@U2@@UAEPAXI@Z 1000b4f0 f i DNAStatPlugin.obj
 0001:0000a4f0       ??_EGObjectViewAction@U2@@UAEPAXI@Z 1000b4f0 f i DNAStatPlugin.obj
 0001:0000a520       ?begin@?$QList@PAVGObjectViewAction@U2@@@@QBE?AVconst_iterator@1@XZ 1000b520 f i DNAStatPlugin.obj
 0001:0000a540       ?buildMenu@DNAStatMSAEditorContext@U2@@MAEXPAVGObjectView@2@PAVQMenu@@@Z 1000b540 f   DNAStatPlugin.obj
 0001:0000a7d0       ?buildMenu@DistanceMatrixMSAEditorContext@U2@@MAEXPAVGObjectView@2@PAVQMenu@@@Z 1000b7d0 f   DNAStatPlugin.obj
 0001:0000aa60       ?data@?$QPointer@VDNAStatMSAProfileDialog@U2@@@@QBEPAVDNAStatMSAProfileDialog@U2@@XZ 1000ba60 f i DNAStatPlugin.obj
 0001:0000aa80       ?data@?$QPointer@VDistanceMatrixMSAProfileDialog@U2@@@@QBEPAVDistanceMatrixMSAProfileDialog@U2@@XZ 1000ba80 f i DNAStatPlugin.obj
 0001:0000aaa0       ?data@?$QWeakPointer@VQObject@@@@QBEPAVQObject@@XZ 1000baa0 f i DNAStatPlugin.obj
 0001:0000aac0       ?dealloc@?$QList@PAVGObjectViewAction@U2@@@@AAEXPAUData@QListData@@@Z 1000bac0 f i DNAStatPlugin.obj
 0001:0000aae0       ?end@?$QList@PAVGObjectViewAction@U2@@@@QBE?AVconst_iterator@1@XZ 1000bae0 f i DNAStatPlugin.obj
 0001:0000ab00       ?initViewContext@DNAStatMSAEditorContext@U2@@MAEXPAVGObjectView@2@@Z 1000bb00 f   DNAStatPlugin.obj
 0001:0000ac40       ?initViewContext@DistanceMatrixMSAEditorContext@U2@@MAEXPAVGObjectView@2@@Z 1000bc40 f   DNAStatPlugin.obj
 0001:0000ad80       ?node_copy@?$QList@PAVGObjectViewAction@U2@@@@AAEXPAUNode@1@00@Z 1000bd80 f i DNAStatPlugin.obj
 0001:0000adb0       ?node_destruct@?$QList@PAVGObjectViewAction@U2@@@@AAEXPAUNode@1@0@Z 1000bdb0 f i DNAStatPlugin.obj
 0001:0000adc0       ?sl_showDistanceMatrixDialog@DistanceMatrixMSAEditorContext@U2@@IAEXXZ 1000bdc0 f   DNAStatPlugin.obj
 0001:0000aed0       ?sl_showMSAProfileDialog@DNAStatMSAEditorContext@U2@@IAEXXZ 1000bed0 f   DNAStatPlugin.obj
 0001:0000afe0       ?t@Node@?$QList@PAVGObjectViewAction@U2@@@@QAEAAPAVGObjectViewAction@U2@@XZ 1000bfe0 f i DNAStatPlugin.obj
 0001:0000aff0       ?tr@DNAStatMSAEditorContext@U2@@SA?AVQString@@PBD0H@Z 1000bff0 f i DNAStatPlugin.obj
 0001:0000b020       ?tr@DNAStatPlugin@U2@@SA?AVQString@@PBD0H@Z 1000c020 f i DNAStatPlugin.obj
 0001:0000b050       ?tr@DistanceMatrixMSAEditorContext@U2@@SA?AVQString@@PBD0H@Z 1000c050 f i DNAStatPlugin.obj
 0001:0000b080       _ugene_plugin_init         1000c080 f   DNAStatPlugin.obj
 0001:0000b0b0       ??0?$QForeachContainer@V?$QList@UCharOccurResult@U2@@@@@@QAE@ABV?$QList@UCharOccurResult@U2@@@@@Z 1000c0b0 f i DNAStatProfileTask.obj
 0001:0000b0f0       ??0?$QList@PAVTask@U2@@@@QAE@$$QAV0@@Z 1000c0f0 f i DNAStatProfileTask.obj
 0001:0000b110       ??0?$QList@PAVTask@U2@@@@QAE@XZ 1000c110 f i DNAStatProfileTask.obj
 0001:0000b120       ??0?$QList@UCharOccurResult@U2@@@@QAE@ABV0@@Z 1000c120 f i DNAStatProfileTask.obj
 0001:0000b1e0       ??0DNAStatProfileTask@U2@@QAE@PAVADVSequenceObjectContext@1@@Z 1000c1e0 f   DNAStatProfileTask.obj
 0001:0000b4c0       ??0const_iterator@?$QList@UCharOccurResult@U2@@@@QAE@PAUNode@1@@Z 1000c4c0 f i DNAStatProfileTask.obj
 0001:0000b4d0       ??0const_iterator@?$QMap@VQByteArray@@_J@@QAE@ABViterator@1@@Z 1000c4d0 f i DNAStatProfileTask.obj
 0001:0000b4e0       ??0iterator@?$QMap@VQByteArray@@_J@@QAE@PAU?$QMapNode@VQByteArray@@_J@@@Z 1000c4e0 f i DNAStatProfileTask.obj
 0001:0000b4f0       ??1?$QForeachContainer@V?$QList@UCharOccurResult@U2@@@@@@QAE@XZ 1000c4f0 f i DNAStatProfileTask.obj
 0001:0000b500       ??1?$QList@PAVTask@U2@@@@QAE@XZ 1000c500 f i DNAStatProfileTask.obj
 0001:0000b530       ??1?$QList@UCharOccurResult@U2@@@@QAE@XZ 1000c530 f i DNAStatProfileTask.obj
 0001:0000b590       ??1?$QMap@VQByteArray@@_J@@QAE@XZ 1000c590 f i DNAStatProfileTask.obj
 0001:0000b600       ??1DNAStatProfileTask@U2@@UAE@XZ 1000c600 f i DNAStatProfileTask.obj
 0001:0000b680       ??9const_iterator@?$QList@UCharOccurResult@U2@@@@QBE_NABV01@@Z 1000c680 f i DNAStatProfileTask.obj
 0001:0000b6a0       ??9const_iterator@?$QMap@VQByteArray@@_J@@QBE_NABV01@@Z 1000c6a0 f i DNAStatProfileTask.obj
 0001:0000b6c0       ??Dconst_iterator@?$QList@UCharOccurResult@U2@@@@QBEABUCharOccurResult@U2@@XZ 1000c6c0 f i DNAStatProfileTask.obj
 0001:0000b6d0       ??Econst_iterator@?$QList@UCharOccurResult@U2@@@@QAEAAV01@XZ 1000c6d0 f i DNAStatProfileTask.obj
 0001:0000b6e0       ??Econst_iterator@?$QMap@VQByteArray@@_J@@QAE?AV01@H@Z 1000c6e0 f i DNAStatProfileTask.obj
 0001:0000b700       ??_GCharOccurTask@U2@@UAEPAXI@Z 1000c700 f i DNAStatProfileTask.obj
 0001:0000b700       ??_ECharOccurTask@U2@@UAEPAXI@Z 1000c700 f i DNAStatProfileTask.obj
 0001:0000b730       ??_EDNAStatProfileTask@U2@@UAEPAXI@Z 1000c730 f i DNAStatProfileTask.obj
 0001:0000b730       ??_GDNAStatProfileTask@U2@@UAEPAXI@Z 1000c730 f i DNAStatProfileTask.obj
 0001:0000b7c0       ??_EDNAStatisticsTask@U2@@UAEPAXI@Z 1000c7c0 f i DNAStatProfileTask.obj
 0001:0000b7c0       ??_GDNAStatisticsTask@U2@@UAEPAXI@Z 1000c7c0 f i DNAStatProfileTask.obj
 0001:0000b7f0       ??_EDinuclOccurTask@U2@@UAEPAXI@Z 1000c7f0 f i DNAStatProfileTask.obj
 0001:0000b7f0       ??_GDinuclOccurTask@U2@@UAEPAXI@Z 1000c7f0 f i DNAStatProfileTask.obj
 0001:0000b820       ??_GQByteArray@@QAEPAXI@Z  1000c820 f i DNAStatProfileTask.obj
 0001:0000b850       ?begin@?$QList@UCharOccurResult@U2@@@@QBE?AVconst_iterator@1@XZ 1000c850 f i DNAStatProfileTask.obj
 0001:0000b870       ?begin@?$QMap@VQByteArray@@_J@@QAE?AViterator@1@XZ 1000c870 f i DNAStatProfileTask.obj
 0001:0000b8b0       ?begin@?$QMapData@VQByteArray@@_J@@QAEPAU?$QMapNode@VQByteArray@@_J@@XZ 1000c8b0 f i DNAStatProfileTask.obj
 0001:0000b8c0       ?copy@?$QMapNode@VQByteArray@@_J@@QBEPAU1@PAU?$QMapData@VQByteArray@@_J@@@Z 1000c8c0 f i DNAStatProfileTask.obj
 0001:0000b950       ?create@?$QMapData@VQByteArray@@_J@@SAPAU1@XZ 1000c950 f i DNAStatProfileTask.obj
 0001:0000b960       ?createNode@?$QMapData@VQByteArray@@_J@@QAEPAU?$QMapNode@VQByteArray@@_J@@ABVQByteArray@@AB_JPAU2@_N@Z 1000c960 f i DNAStatProfileTask.obj
 0001:0000ba10       ?dealloc@?$QList@PAVTask@U2@@@@AAEXPAUData@QListData@@@Z 1000ca10 f i DNAStatProfileTask.obj
 0001:0000ba30       ?dealloc@?$QList@UCharOccurResult@U2@@@@AAEXPAUData@QListData@@@Z 1000ca30 f i DNAStatProfileTask.obj
 0001:0000ba80       ?destroy@?$QMapData@VQByteArray@@_J@@QAEXXZ 1000ca80 f i DNAStatProfileTask.obj
 0001:0000bad0       ?destroySubTree@?$QMapNode@VQByteArray@@_J@@QAEXXZ 1000cad0 f i DNAStatProfileTask.obj
 0001:0000bb00       ?detach@?$QMap@VQByteArray@@_J@@QAEXXZ 1000cb00 f i DNAStatProfileTask.obj
 0001:0000bb20       ?detach_helper@?$QMap@VQByteArray@@_J@@AAEXXZ 1000cb20 f i DNAStatProfileTask.obj
 0001:0000bbd0       ?end@?$QList@UCharOccurResult@U2@@@@QBE?AVconst_iterator@1@XZ 1000cbd0 f i DNAStatProfileTask.obj
 0001:0000bbf0       ?end@?$QMap@VQByteArray@@_J@@QAE?AViterator@1@XZ 1000cbf0 f i DNAStatProfileTask.obj
 0001:0000bc20       ?end@?$QMapData@VQByteArray@@_J@@QAEPAU?$QMapNode@VQByteArray@@_J@@XZ 1000cc20 f i DNAStatProfileTask.obj
 0001:0000bc30       ?formCharResultString@DNAStatProfileTask@U2@@ABE?AVQString@@XZ 1000cc30 f   DNAStatProfileTask.obj
 0001:0000bff0       ?formDinucResultString@DNAStatProfileTask@U2@@ABE?AVQString@@XZ 1000cff0 f   DNAStatProfileTask.obj
 0001:0000c400       ?formStatResultString@DNAStatProfileTask@U2@@ABE?AVQString@@XZ 1000d400 f   DNAStatProfileTask.obj
 0001:0000ce40       ?getChar@CharOccurResult@U2@@QBEDXZ 1000de40 f i DNAStatProfileTask.obj
 0001:0000ce50       ?getNumberOfOccur@CharOccurResult@U2@@QBE_JXZ 1000de50 f i DNAStatProfileTask.obj
 0001:0000ce60       ?getPercentage@CharOccurResult@U2@@QBENXZ 1000de60 f i DNAStatProfileTask.obj
 0001:0000ce70       ?getResult@DNAStatProfileTask@U2@@QBE?AVQString@@XZ 1000de70 f   DNAStatProfileTask.obj
 0001:0000cf40       ?isEmpty@?$QMap@VQByteArray@@_J@@QBE_NXZ 1000df40 f i DNAStatProfileTask.obj
 0001:0000cf50       ?key@const_iterator@?$QMap@VQByteArray@@_J@@QBEABVQByteArray@@XZ 1000df50 f i DNAStatProfileTask.obj
 0001:0000cf60       ?leftNode@?$QMapNode@VQByteArray@@_J@@QBEPAU1@XZ 1000df60 f i DNAStatProfileTask.obj
 0001:0000cf70       ?nextNode@?$QMapNode@VQByteArray@@_J@@QBEPBU1@XZ 1000df70 f i DNAStatProfileTask.obj
 0001:0000cf80       ?node_copy@?$QList@UCharOccurResult@U2@@@@AAEXPAUNode@1@00@Z 1000df80 f i DNAStatProfileTask.obj
 0001:0000d040       ?node_destruct@?$QList@PAVTask@U2@@@@AAEXPAUNode@1@0@Z 1000e040 f i DNAStatProfileTask.obj
 0001:0000d050       ?node_destruct@?$QList@UCharOccurResult@U2@@@@AAEXPAUNode@1@0@Z 1000e050 f i DNAStatProfileTask.obj
 0001:0000d080       ?onSubTaskFinished@DNAStatProfileTask@U2@@UAE?AV?$QList@PAVTask@U2@@@@PAVTask@2@@Z 1000e080 f   DNAStatProfileTask.obj
 0001:0000d180       ?rightNode@?$QMapNode@VQByteArray@@_J@@QBEPAU1@XZ 1000e180 f i DNAStatProfileTask.obj
 0001:0000d190       ?root@?$QMapData@VQByteArray@@_J@@QBEPAU?$QMapNode@VQByteArray@@_J@@XZ 1000e190 f i DNAStatProfileTask.obj
 0001:0000d1a0       ?t@Node@?$QList@UCharOccurResult@U2@@@@QAEAAUCharOccurResult@U2@@XZ 1000e1a0 f i DNAStatProfileTask.obj
 0001:0000d1b0       ?tr@DNAStatProfileTask@U2@@SA?AVQString@@PBD0H@Z 1000e1b0 f i DNAStatProfileTask.obj
 0001:0000d1e0       ?value@const_iterator@?$QMap@VQByteArray@@_J@@QBEAB_JXZ 1000e1e0 f i DNAStatProfileTask.obj
 0001:0000d1f0       ??$qobject_cast@PAVMSADistanceAlgorithm@U2@@@@YAPAVMSADistanceAlgorithm@U2@@PAVQObject@@@Z 1000e1f0 f i DistanceMatrixMSAProfileDialog.obj
 0001:0000d210       ??0?$QForeachContainer@V?$QList@PAVMSADistanceAlgorithmFactory@U2@@@@@@QAE@ABV?$QList@PAVMSADistanceAlgorithmFactory@U2@@@@@Z 1000e210 f i DistanceMatrixMSAProfileDialog.obj
 0001:0000d250       ??0?$QForeachContainer@V?$QVector@VU2Region@U2@@@@@@QAE@ABV?$QVector@VU2Region@U2@@@@@Z 1000e250 f i DistanceMatrixMSAProfileDialog.obj
 0001:0000d2d0       ??0?$QList@PAVMSADistanceAlgorithmFactory@U2@@@@QAE@ABV0@@Z 1000e2d0 f i DistanceMatrixMSAProfileDialog.obj
 0001:0000d390       ??0?$QVector@VU2Region@U2@@@@QAE@ABV0@@Z 1000e390 f i DistanceMatrixMSAProfileDialog.obj
 0001:0000d450       ??0?$QVector@VU2Region@U2@@@@QAE@XZ 1000e450 f i DistanceMatrixMSAProfileDialog.obj
 0001:0000d460       ??0DistanceMatrixMSAProfileDialog@U2@@QAE@PAVQWidget@@PAVMSAEditor@1@@Z 1000e460 f   DistanceMatrixMSAProfileDialog.obj
 0001:0000d7d0       ??0DistanceMatrixMSAProfileTask@U2@@QAE@ABVDistanceMatrixMSAProfileTaskSettings@1@@Z 1000e7d0 f   DistanceMatrixMSAProfileDialog.obj
 0001:0000d880       ??0DistanceMatrixMSAProfileTaskSettings@U2@@QAE@ABV01@@Z 1000e880 f i DistanceMatrixMSAProfileDialog.obj
 0001:0000d940       ??0DistanceMatrixMSAProfileTaskSettings@U2@@QAE@XZ 1000e940 f   DistanceMatrixMSAProfileDialog.obj
 0001:0000da30       ??0const_iterator@?$QList@PAVMSADistanceAlgorithmFactory@U2@@@@QAE@PAUNode@1@@Z 1000ea30 f i DistanceMatrixMSAProfileDialog.obj
 0001:0000da40       ??1?$QForeachContainer@V?$QList@PAVMSADistanceAlgorithmFactory@U2@@@@@@QAE@XZ 1000ea40 f i DistanceMatrixMSAProfileDialog.obj
 0001:0000da70       ??1?$QForeachContainer@V?$QVector@VU2Region@U2@@@@@@QAE@XZ 1000ea70 f i DistanceMatrixMSAProfileDialog.obj
 0001:0000dab0       ??1?$QList@PAVMSADistanceAlgorithmFactory@U2@@@@QAE@XZ 1000eab0 f i DistanceMatrixMSAProfileDialog.obj
 0001:0000dae0       ??1?$QVector@VU2Region@U2@@@@QAE@XZ 1000eae0 f i DistanceMatrixMSAProfileDialog.obj
 0001:0000db20       ??1DistanceMatrixMSAProfileDialog@U2@@UAE@XZ 1000eb20 f i DistanceMatrixMSAProfileDialog.obj
 0001:0000db30       ??1DistanceMatrixMSAProfileTask@U2@@UAE@XZ 1000eb30 f i DistanceMatrixMSAProfileDialog.obj
 0001:0000dbe0       ??1DistanceMatrixMSAProfileTaskSettings@U2@@QAE@XZ 1000ebe0 f i DistanceMatrixMSAProfileDialog.obj
 0001:0000dc60       ??9const_iterator@?$QList@PAVMSADistanceAlgorithmFactory@U2@@@@QBE_NABV01@@Z 1000ec60 f i DistanceMatrixMSAProfileDialog.obj
 0001:0000dc80       ??Dconst_iterator@?$QList@PAVMSADistanceAlgorithmFactory@U2@@@@QBEABQAVMSADistanceAlgorithmFactory@U2@@XZ 1000ec80 f i DistanceMatrixMSAProfileDialog.obj
 0001:0000dc90       ??Econst_iterator@?$QList@PAVMSADistanceAlgorithmFactory@U2@@@@QAEAAV01@XZ 1000ec90 f i DistanceMatrixMSAProfileDialog.obj
 0001:0000defa       ??_EDistanceMatrixMSAProfileDialog@U2@@W7AEPAXI@Z 1000eefa f i DistanceMatrixMSAProfileDialog.obj
 0001:0000df02       ??_EQComboBox@@W7AEPAXI@Z  1000ef02 f i DistanceMatrixMSAProfileDialog.obj
 0001:0000df0a       ??_EQHBoxLayout@@W7AEPAXI@Z 1000ef0a f i DistanceMatrixMSAProfileDialog.obj
 0001:0000df20       ??_EDistanceMatrixMSAProfileDialog@U2@@UAEPAXI@Z 1000ef20 f i DistanceMatrixMSAProfileDialog.obj
 0001:0000df20       ??_GDistanceMatrixMSAProfileDialog@U2@@UAEPAXI@Z 1000ef20 f i DistanceMatrixMSAProfileDialog.obj
 0001:0000df50       ??_GDistanceMatrixMSAProfileTask@U2@@UAEPAXI@Z 1000ef50 f i DistanceMatrixMSAProfileDialog.obj
 0001:0000df50       ??_EDistanceMatrixMSAProfileTask@U2@@UAEPAXI@Z 1000ef50 f i DistanceMatrixMSAProfileDialog.obj
 0001:0000df80       ??_EMultipleSequenceAlignmentRow@U2@@UAEPAXI@Z 1000ef80 f i DistanceMatrixMSAProfileDialog.obj
 0001:0000df80       ??_GMultipleSequenceAlignmentRow@U2@@UAEPAXI@Z 1000ef80 f i DistanceMatrixMSAProfileDialog.obj
 0001:0000dfb0       ??_EQComboBox@@UAEPAXI@Z   1000efb0 f i DistanceMatrixMSAProfileDialog.obj
 0001:0000dfb0       ??_GQComboBox@@UAEPAXI@Z   1000efb0 f i DistanceMatrixMSAProfileDialog.obj
 0001:0000dfe0       ??_GQHBoxLayout@@UAEPAXI@Z 1000efe0 f i DistanceMatrixMSAProfileDialog.obj
 0001:0000dfe0       ??_EQHBoxLayout@@UAEPAXI@Z 1000efe0 f i DistanceMatrixMSAProfileDialog.obj
 0001:0000e010       ??_EQSpacerItem@@UAEPAXI@Z 1000f010 f i DistanceMatrixMSAProfileDialog.obj
 0001:0000e010       ??_GQSpacerItem@@UAEPAXI@Z 1000f010 f i DistanceMatrixMSAProfileDialog.obj
 0001:0000e040       ?accept@DistanceMatrixMSAProfileDialog@U2@@UAEXXZ 1000f040 f   DistanceMatrixMSAProfileDialog.obj
 0001:0000e2a0       ?allocate@?$QTypedArrayData@VU2Region@U2@@@@SAPAU1@IV?$QFlags@W4AllocationOption@QArrayData@@@@@Z 1000f2a0 f i DistanceMatrixMSAProfileDialog.obj
 0001:0000e2c0       ?append@?$QList@VMultipleSequenceAlignmentRow@U2@@@@QAEXABVMultipleSequenceAlignmentRow@U2@@@Z 1000f2c0 f i DistanceMatrixMSAProfileDialog.obj
 0001:0000e3b0       ?at@?$QList@VMultipleSequenceAlignmentRow@U2@@@@QBEABVMultipleSequenceAlignmentRow@U2@@H@Z 1000f3b0 f i DistanceMatrixMSAProfileDialog.obj
 0001:0000e3d0       ?begin@?$QList@PAVMSADistanceAlgorithmFactory@U2@@@@QBE?AVconst_iterator@1@XZ 1000f3d0 f i DistanceMatrixMSAProfileDialog.obj
 0001:0000e3f0       ?begin@?$QTypedArrayData@VU2Region@U2@@@@QAEPAVU2Region@U2@@PAV23@@Z 1000f3f0 f i DistanceMatrixMSAProfileDialog.obj
 0001:0000e400       ?begin@?$QVector@VU2Region@U2@@@@QBEPBVU2Region@U2@@XZ 1000f400 f i DistanceMatrixMSAProfileDialog.obj
 0001:0000e410       ?constBegin@?$QTypedArrayData@VU2Region@U2@@@@QBEPBVU2Region@U2@@PBV23@@Z 1000f410 f i DistanceMatrixMSAProfileDialog.obj
 0001:0000e420       ?constEnd@?$QTypedArrayData@VU2Region@U2@@@@QBEPBVU2Region@U2@@PBV23@@Z 1000f420 f i DistanceMatrixMSAProfileDialog.obj
 0001:0000e440       ?copyConstruct@?$QVector@VU2Region@U2@@@@AAEXPBVU2Region@U2@@0PAV23@@Z 1000f440 f i DistanceMatrixMSAProfileDialog.obj
 0001:0000e460       ?createDistanceTable@DistanceMatrixMSAProfileTask@U2@@QAEXPAVMSADistanceAlgorithm@2@ABV?$QList@VMultipleSequenceAlignmentRow@U2@@@@PAVQFile@@@Z 1000f460 f   DistanceMatrixMSAProfileDialog.obj
 0001:0000eaa0       ?data@?$QTypedArrayData@VU2Region@U2@@@@QAEPAVU2Region@U2@@XZ 1000faa0 f i DistanceMatrixMSAProfileDialog.obj
 0001:0000eab0       ?data@?$QTypedArrayData@VU2Region@U2@@@@QBEPBVU2Region@U2@@XZ 1000fab0 f i DistanceMatrixMSAProfileDialog.obj
 0001:0000eac0       ?data_ptr@?$QStaticStringData@$0BE@@@QBEPAU?$QTypedArrayData@G@@XZ 1000fac0 f i DistanceMatrixMSAProfileDialog.obj
 0001:0000ead0       ?data_ptr@?$QStaticStringData@$0BO@@@QBEPAU?$QTypedArrayData@G@@XZ 1000fad0 f i DistanceMatrixMSAProfileDialog.obj
 0001:0000eae0       ?dealloc@?$QList@PAVMSADistanceAlgorithmFactory@U2@@@@AAEXPAUData@QListData@@@Z 1000fae0 f i DistanceMatrixMSAProfileDialog.obj
 0001:0000eb00       ?deallocate@?$QTypedArrayData@VU2Region@U2@@@@SAXPAUQArrayData@@@Z 1000fb00 f i DistanceMatrixMSAProfileDialog.obj
 0001:0000eb20       ?destruct@?$QVector@VU2Region@U2@@@@AAEXPAVU2Region@U2@@0@Z 1000fb20 f i DistanceMatrixMSAProfileDialog.obj
 0001:0000eb30       ?detach_helper_grow@?$QList@VMultipleSequenceAlignmentRow@U2@@@@AAEPAUNode@1@HH@Z 1000fb30 f i DistanceMatrixMSAProfileDialog.obj
 0001:0000ec80       ?end@?$QList@PAVMSADistanceAlgorithmFactory@U2@@@@QBE?AVconst_iterator@1@XZ 1000fc80 f i DistanceMatrixMSAProfileDialog.obj
 0001:0000eca0       ?end@?$QTypedArrayData@VU2Region@U2@@@@QAEPAVU2Region@U2@@PAV23@@Z 1000fca0 f i DistanceMatrixMSAProfileDialog.obj
 0001:0000ecc0       ?end@?$QVector@VU2Region@U2@@@@QBEPBVU2Region@U2@@XZ 1000fcc0 f i DistanceMatrixMSAProfileDialog.obj
 0001:0000ece0       ?freeData@?$QVector@VU2Region@U2@@@@AAEXPAU?$QTypedArrayData@VU2Region@U2@@@@@Z 1000fce0 f i DistanceMatrixMSAProfileDialog.obj
 0001:0000ed10       ?generateReport@DistanceMatrixMSAProfileTask@U2@@UBE?AVQString@@XZ 1000fd10 f   DistanceMatrixMSAProfileDialog.obj
 0001:0000ef20       ?initSaveController@DistanceMatrixMSAProfileDialog@U2@@AAEXXZ 1000ff20 f   DistanceMatrixMSAProfileDialog.obj
 0001:0000f280       ?isReportingEnabled@DistanceMatrixMSAProfileTask@U2@@UBE_NXZ 10010280 f   DistanceMatrixMSAProfileDialog.obj
 0001:0000f2b0       ?node_construct@?$QList@VMultipleSequenceAlignmentRow@U2@@@@AAEXPAUNode@1@ABVMultipleSequenceAlignmentRow@U2@@@Z 100102b0 f i DistanceMatrixMSAProfileDialog.obj
 0001:0000f340       ?node_copy@?$QList@PAVMSADistanceAlgorithmFactory@U2@@@@AAEXPAUNode@1@00@Z 10010340 f i DistanceMatrixMSAProfileDialog.obj
 0001:0000f370       ?node_copy@?$QList@VMultipleSequenceAlignmentRow@U2@@@@AAEXPAUNode@1@00@Z 10010370 f i DistanceMatrixMSAProfileDialog.obj
 0001:0000f440       ?node_destruct@?$QList@PAVMSADistanceAlgorithmFactory@U2@@@@AAEXPAUNode@1@0@Z 10010440 f i DistanceMatrixMSAProfileDialog.obj
 0001:0000f450       ?node_destruct@?$QList@VMultipleSequenceAlignmentRow@U2@@@@AAEXPAUNode@1@@Z 10010450 f i DistanceMatrixMSAProfileDialog.obj
 0001:0000f4a0       ?onSubTaskFinished@DistanceMatrixMSAProfileTask@U2@@UAE?AV?$QList@PAVTask@U2@@@@PAVTask@2@@Z 100104a0 f   DistanceMatrixMSAProfileDialog.obj
 0001:000108c0       ?prepare@DistanceMatrixMSAProfileTask@U2@@UAEXXZ 100118c0 f   DistanceMatrixMSAProfileDialog.obj
 0001:00010920       ?report@DistanceMatrixMSAProfileTask@U2@@UAE?AW4ReportResult@Task@2@XZ 10011920 f   DistanceMatrixMSAProfileDialog.obj
 0001:00010b10       ?retranslateUi@Ui_DistanceMatrixMSAProfileDialog@@QAEXPAVQDialog@@@Z 10011b10 f i DistanceMatrixMSAProfileDialog.obj
 0001:00010e10       ?setupUi@Ui_DistanceMatrixMSAProfileDialog@@QAEXPAVQDialog@@@Z 10011e10 f i DistanceMatrixMSAProfileDialog.obj
 0001:00011890       ?sharedNull@?$QTypedArrayData@VU2Region@U2@@@@SAPAU1@XZ 10012890 f i DistanceMatrixMSAProfileDialog.obj
 0001:000118a0       ?size@?$QList@VMultipleSequenceAlignmentRow@U2@@@@QBEHXZ 100128a0 f i DistanceMatrixMSAProfileDialog.obj
 0001:000118b0       ?size@?$QVector@VU2Region@U2@@@@QBEHXZ 100128b0 f i DistanceMatrixMSAProfileDialog.obj
 0001:000118c0       ?sl_formatChanged@DistanceMatrixMSAProfileDialog@U2@@AAEXABVQString@@@Z 100128c0 f   DistanceMatrixMSAProfileDialog.obj
 0001:00011900       ?sl_formatSelected@DistanceMatrixMSAProfileDialog@U2@@AAEXXZ 10012900 f   DistanceMatrixMSAProfileDialog.obj
 0001:00011930       ?t@Node@?$QList@PAVMSADistanceAlgorithmFactory@U2@@@@QAEAAPAVMSADistanceAlgorithmFactory@U2@@XZ 10012930 f i DistanceMatrixMSAProfileDialog.obj
 0001:00011940       ?t@Node@?$QList@VMultipleSequenceAlignmentRow@U2@@@@QAEAAVMultipleSequenceAlignmentRow@U2@@XZ 10012940 f i DistanceMatrixMSAProfileDialog.obj
 0001:00011950       ?tr@DistanceMatrixMSAProfileDialog@U2@@SA?AVQString@@PBD0H@Z 10012950 f i DistanceMatrixMSAProfileDialog.obj
 0001:00011980       ?tr@DistanceMatrixMSAProfileTask@U2@@SA?AVQString@@PBD0H@Z 10012980 f i DistanceMatrixMSAProfileDialog.obj
 0001:000119b0       ??C?$QScopedPointer@VQObjectData@@U?$QScopedPointerDeleter@VQObjectData@@@@@@QBEPAVQObjectData@@XZ 100129b0 f i moc_DNAStatMSAProfileDialog.obj
 0001:000119c0       ?metaObject@DNAStatMSAProfileDialog@U2@@UBEPBUQMetaObject@@XZ 100129c0 f   moc_DNAStatMSAProfileDialog.obj
 0001:000119e0       ?metaObject@DNAStatMSAProfileTask@U2@@UBEPBUQMetaObject@@XZ 100129e0 f   moc_DNAStatMSAProfileDialog.obj
 0001:00011a00       ?qt_metacall@DNAStatMSAProfileDialog@U2@@UAEHW4Call@QMetaObject@@HPAPAX@Z 10012a00 f   moc_DNAStatMSAProfileDialog.obj
 0001:00011a80       ?qt_metacall@DNAStatMSAProfileTask@U2@@UAEHW4Call@QMetaObject@@HPAPAX@Z 10012a80 f   moc_DNAStatMSAProfileDialog.obj
 0001:00011a90       ?qt_metacast@DNAStatMSAProfileDialog@U2@@UAEPAXPBD@Z 10012a90 f   moc_DNAStatMSAProfileDialog.obj
 0001:00011b30       ?qt_metacast@DNAStatMSAProfileTask@U2@@UAEPAXPBD@Z 10012b30 f   moc_DNAStatMSAProfileDialog.obj
 0001:00011b90       ?qt_static_metacall@DNAStatMSAProfileDialog@U2@@CAXPAVQObject@@W4Call@QMetaObject@@HPAPAX@Z 10012b90 f   moc_DNAStatMSAProfileDialog.obj
 0001:00011bc0       ?qt_static_metacall@DNAStatMSAProfileTask@U2@@CAXPAVQObject@@W4Call@QMetaObject@@HPAPAX@Z 10012bc0 f   moc_DNAStatMSAProfileDialog.obj
 0001:00011bd0       ??$acquireMemoryFence@H@?$QGenericAtomicOps@U?$QAtomicOpsBySize@$03@@@@SAXABH@Z 10012bd0 f i moc_DNAStatPlugin.obj
 0001:00011be0       ??$loadAcquire@H@?$QGenericAtomicOps@U?$QAtomicOpsBySize@$03@@@@SAHABH@Z 10012be0 f i moc_DNAStatPlugin.obj
 0001:00011bf0       ??$orderedMemoryFence@H@?$QGenericAtomicOps@U?$QAtomicOpsBySize@$03@@@@SAXABH@Z 10012bf0 f i moc_DNAStatPlugin.obj
 0001:00011c00       ??$qMetaTypeId@PAVGObjectView@U2@@@@YAHXZ 10012c00 f i moc_DNAStatPlugin.obj
 0001:00011c10       ??$qMetaTypeId@PAVQMenu@@@@YAHXZ 10012c10 f i moc_DNAStatPlugin.obj
 0001:00011c20       ??$qRegisterMetaType@PAVGObjectView@U2@@@@YAHXZ 10012c20 f i moc_DNAStatPlugin.obj
 0001:00011c30       ??$qRegisterMetaType@PAVQMenu@@@@YAHXZ 10012c30 f i moc_DNAStatPlugin.obj
 0001:00011c40       ??$qRegisterNormalizedMetaType@PAVGObjectView@U2@@@@YAHABVQByteArray@@PAPAVGObjectView@U2@@W4DefinedType@?$MetaTypeDefinedHelper@PAVGObjectView@U2@@$00@QtPrivate@@@Z 10012c40 f i moc_DNAStatPlugin.obj
 0001:00011ca0       ??$qRegisterNormalizedMetaType@PAVQMenu@@@@YAHABVQByteArray@@PAPAVQMenu@@W4DefinedType@?$MetaTypeDefinedHelper@PAVQMenu@@$00@QtPrivate@@@Z 10012ca0 f i moc_DNAStatPlugin.obj
 0001:00011d00       ??$releaseMemoryFence@H@?$QGenericAtomicOps@U?$QAtomicOpsBySize@$03@@@@SAXABH@Z 10012d00 f i moc_DNAStatPlugin.obj
 0001:00011d10       ??$storeRelease@HH@?$QGenericAtomicOps@U?$QAtomicOpsBySize@$03@@@@SAXAAHH@Z 10012d10 f i moc_DNAStatPlugin.obj
 0001:00011d20       ??0?$QFlags@W4TypeFlag@QMetaType@@@@QAE@VQFlag@@@Z 10012d20 f i moc_DNAStatPlugin.obj
 0001:00011d30       ??_5?$QFlags@W4TypeFlag@QMetaType@@@@QAEAAV0@W4TypeFlag@QMetaType@@@Z 10012d30 f i moc_DNAStatPlugin.obj
 0001:00011d40       ?Construct@?$QMetaTypeFunctionHelper@PAVGObjectView@U2@@$00@QtMetaTypePrivate@@SAPAXPAXPBX@Z 10012d40 f i moc_DNAStatPlugin.obj
 0001:00011d70       ?Construct@?$QMetaTypeFunctionHelper@PAVQMenu@@$00@QtMetaTypePrivate@@SAPAXPAXPBX@Z 10012d70 f i moc_DNAStatPlugin.obj
 0001:00011da0       ?Create@?$QMetaTypeFunctionHelper@PAVGObjectView@U2@@$00@QtMetaTypePrivate@@SAPAXPBX@Z 10012da0 f i moc_DNAStatPlugin.obj
 0001:00011de0       ?Create@?$QMetaTypeFunctionHelper@PAVQMenu@@$00@QtMetaTypePrivate@@SAPAXPBX@Z 10012de0 f i moc_DNAStatPlugin.obj
 0001:00011e20       ?Delete@?$QMetaTypeFunctionHelper@PAVGObjectView@U2@@$00@QtMetaTypePrivate@@SAXPAX@Z 10012e20 f i moc_DNAStatPlugin.obj
 0001:00011e30       ?Delete@?$QMetaTypeFunctionHelper@PAVQMenu@@$00@QtMetaTypePrivate@@SAXPAX@Z 10012e30 f i moc_DNAStatPlugin.obj
 0001:00011e40       ?Destruct@?$QMetaTypeFunctionHelper@PAVGObjectView@U2@@$00@QtMetaTypePrivate@@SAXPAX@Z 10012e40 f i moc_DNAStatPlugin.obj
 0001:00011e50       ?Destruct@?$QMetaTypeFunctionHelper@PAVQMenu@@$00@QtMetaTypePrivate@@SAXPAX@Z 10012e50 f i moc_DNAStatPlugin.obj
 0001:00011e60       ?loadAcquire@?$QBasicAtomicInteger@H@@QBEHXZ 10012e60 f i moc_DNAStatPlugin.obj
 0001:00011e70       ?metaObject@DNAStatMSAEditorContext@U2@@UBEPBUQMetaObject@@XZ 10012e70 f   moc_DNAStatPlugin.obj
 0001:00011e90       ?metaObject@DNAStatPlugin@U2@@UBEPBUQMetaObject@@XZ 10012e90 f   moc_DNAStatPlugin.obj
 0001:00011eb0       ?metaObject@DistanceMatrixMSAEditorContext@U2@@UBEPBUQMetaObject@@XZ 10012eb0 f   moc_DNAStatPlugin.obj
 0001:00011ed0       ?qt_metacall@DNAStatMSAEditorContext@U2@@UAEHW4Call@QMetaObject@@HPAPAX@Z 10012ed0 f   moc_DNAStatPlugin.obj
 0001:00011f30       ?qt_metacall@DNAStatPlugin@U2@@UAEHW4Call@QMetaObject@@HPAPAX@Z 10012f30 f   moc_DNAStatPlugin.obj
 0001:00011f40       ?qt_metacall@DistanceMatrixMSAEditorContext@U2@@UAEHW4Call@QMetaObject@@HPAPAX@Z 10012f40 f   moc_DNAStatPlugin.obj
 0001:00011fa0       ?qt_metacast@DNAStatMSAEditorContext@U2@@UAEPAXPBD@Z 10012fa0 f   moc_DNAStatPlugin.obj
 0001:00012000       ?qt_metacast@DNAStatPlugin@U2@@UAEPAXPBD@Z 10013000 f   moc_DNAStatPlugin.obj
 0001:00012060       ?qt_metacast@DistanceMatrixMSAEditorContext@U2@@UAEPAXPBD@Z 10013060 f   moc_DNAStatPlugin.obj
 0001:000120c0       ?qt_metatype_id@?$QMetaTypeId2@PAVGObjectView@U2@@@@SAHXZ 100130c0 f i moc_DNAStatPlugin.obj
 0001:000120d0       ?qt_metatype_id@?$QMetaTypeId2@PAVQMenu@@@@SAHXZ 100130d0 f i moc_DNAStatPlugin.obj
 0001:000120e0       ?qt_metatype_id@?$QMetaTypeIdHelper@PAVGObjectView@U2@@$00@QtPrivate@@SAHXZ 100130e0 f i moc_DNAStatPlugin.obj
 0001:000120f0       ?qt_metatype_id@?$QMetaTypeIdHelper@PAVQMenu@@$00@QtPrivate@@SAHXZ 100130f0 f i moc_DNAStatPlugin.obj
 0001:00012100       ?qt_metatype_id@?$QMetaTypeIdQObject@PAVGObjectView@U2@@$00@@SAHXZ 10013100 f i moc_DNAStatPlugin.obj
 0001:000121e0       ?qt_metatype_id@?$QMetaTypeIdQObject@PAVQMenu@@$00@@SAHXZ 100131e0 f i moc_DNAStatPlugin.obj
 0001:000122c0       ?qt_static_metacall@DNAStatMSAEditorContext@U2@@CAXPAVQObject@@W4Call@QMetaObject@@HPAPAX@Z 100132c0 f   moc_DNAStatPlugin.obj
 0001:00012350       ?qt_static_metacall@DNAStatPlugin@U2@@CAXPAVQObject@@W4Call@QMetaObject@@HPAPAX@Z 10013350 f   moc_DNAStatPlugin.obj
 0001:00012360       ?qt_static_metacall@DistanceMatrixMSAEditorContext@U2@@CAXPAVQObject@@W4Call@QMetaObject@@HPAPAX@Z 10013360 f   moc_DNAStatPlugin.obj
 0001:000123f0       ?registerConverter@?$AssociativeContainerConverterHelper@PAVGObjectView@U2@@$0A@@QtPrivate@@SA_NH@Z 100133f0 f i moc_DNAStatPlugin.obj
 0001:00012400       ?registerConverter@?$AssociativeContainerConverterHelper@PAVQMenu@@$0A@@QtPrivate@@SA_NH@Z 10013400 f i moc_DNAStatPlugin.obj
 0001:00012410       ?registerConverter@?$IsPair@PAVGObjectView@U2@@@QtPrivate@@SA_NH@Z 10013410 f i moc_DNAStatPlugin.obj
 0001:00012420       ?registerConverter@?$IsPair@PAVQMenu@@@QtPrivate@@SA_NH@Z 10013420 f i moc_DNAStatPlugin.obj
 0001:00012430       ?registerConverter@?$MetaTypeSmartPointerHelper@PAVGObjectView@U2@@X@QtPrivate@@SA_NH@Z 10013430 f i moc_DNAStatPlugin.obj
 0001:00012440       ?registerConverter@?$MetaTypeSmartPointerHelper@PAVQMenu@@X@QtPrivate@@SA_NH@Z 10013440 f i moc_DNAStatPlugin.obj
 0001:00012450       ?registerConverter@?$SequentialContainerConverterHelper@PAVGObjectView@U2@@$0A@@QtPrivate@@SA_NH@Z 10013450 f i moc_DNAStatPlugin.obj
 0001:00012460       ?registerConverter@?$SequentialContainerConverterHelper@PAVQMenu@@$0A@@QtPrivate@@SA_NH@Z 10013460 f i moc_DNAStatPlugin.obj
 0001:00012470       ?storeRelease@?$QBasicAtomicInteger@H@@QAEXH@Z 10013470 f i moc_DNAStatPlugin.obj
 0001:00012480       ?value@?$MetaObjectForType@PAVGObjectView@U2@@$00@QtPrivate@@SAPBUQMetaObject@@XZ 10013480 f i moc_DNAStatPlugin.obj
 0001:00012490       ?value@?$MetaObjectForType@PAVQMenu@@$00@QtPrivate@@SAPBUQMetaObject@@XZ 10013490 f i moc_DNAStatPlugin.obj
 0001:000124a0       ?metaObject@DNAStatProfileTask@U2@@UBEPBUQMetaObject@@XZ 100134a0 f   moc_DNAStatProfileTask.obj
 0001:000124c0       ?qt_metacall@DNAStatProfileTask@U2@@UAEHW4Call@QMetaObject@@HPAPAX@Z 100134c0 f   moc_DNAStatProfileTask.obj
 0001:000124d0       ?qt_metacast@DNAStatProfileTask@U2@@UAEPAXPBD@Z 100134d0 f   moc_DNAStatProfileTask.obj
 0001:00012530       ?qt_static_metacall@DNAStatProfileTask@U2@@CAXPAVQObject@@W4Call@QMetaObject@@HPAPAX@Z 10013530 f   moc_DNAStatProfileTask.obj
 0001:00012540       ?metaObject@DistanceMatrixMSAProfileDialog@U2@@UBEPBUQMetaObject@@XZ 10013540 f   moc_DistanceMatrixMSAProfileDialog.obj
 0001:00012560       ?metaObject@DistanceMatrixMSAProfileTask@U2@@UBEPBUQMetaObject@@XZ 10013560 f   moc_DistanceMatrixMSAProfileDialog.obj
 0001:00012580       ?qt_metacall@DistanceMatrixMSAProfileDialog@U2@@UAEHW4Call@QMetaObject@@HPAPAX@Z 10013580 f   moc_DistanceMatrixMSAProfileDialog.obj
 0001:00012600       ?qt_metacall@DistanceMatrixMSAProfileTask@U2@@UAEHW4Call@QMetaObject@@HPAPAX@Z 10013600 f   moc_DistanceMatrixMSAProfileDialog.obj
 0001:00012610       ?qt_metacast@DistanceMatrixMSAProfileDialog@U2@@UAEPAXPBD@Z 10013610 f   moc_DistanceMatrixMSAProfileDialog.obj
 0001:000126b0       ?qt_metacast@DistanceMatrixMSAProfileTask@U2@@UAEPAXPBD@Z 100136b0 f   moc_DistanceMatrixMSAProfileDialog.obj
 0001:00012710       ?qt_static_metacall@DistanceMatrixMSAProfileDialog@U2@@CAXPAVQObject@@W4Call@QMetaObject@@HPAPAX@Z 10013710 f   moc_DistanceMatrixMSAProfileDialog.obj
 0001:00012740       ?qt_static_metacall@DistanceMatrixMSAProfileTask@U2@@CAXPAVQObject@@W4Call@QMetaObject@@HPAPAX@Z 10013740 f   moc_DistanceMatrixMSAProfileDialog.obj
 0001:00012742       ?getMainWindow@AppContext@U2@@SAPAVMainWindow@2@XZ 10013742 f   U2Core:U2Core.dll
 0001:00012748       ?getTaskScheduler@AppContext@U2@@SAPAVTaskScheduler@2@XZ 10013748 f   U2Core:U2Core.dll
 0001:0001274e       ?getAlphabetChars@DNAAlphabet@U2@@QBE?AVQByteArray@@_N@Z 1001374e f   U2Core:U2Core.dll
 0001:00012754       ?dumpStringToFile@FileAndDirectoryUtils@U2@@SAXPAVQFile@@AAVQString@@@Z 10013754 f   U2Core:U2Core.dll
 0001:0001275a       ?getDefaultDataPath@GUrlUtils@U2@@SA?AVQString@@XZ 1001375a f   U2Core:U2Core.dll
 0001:00012760       ?fixFileName@GUrlUtils@U2@@SA?AVQString@@ABV3@@Z 10013760 f   U2Core:U2Core.dll
 0001:00012766       ??1MultipleAlignmentRow@U2@@UAE@XZ 10013766 f   U2Core:U2Core.dll
 0001:0001276c       ??1MultipleAlignment@U2@@UAE@XZ 1001376c f   U2Core:U2Core.dll
 0001:00012772       ?getAlphabet@MultipleAlignmentData@U2@@QBEPBVDNAAlphabet@2@XZ 10013772 f   U2Core:U2Core.dll
 0001:00012778       ?getLength@MultipleAlignmentData@U2@@QBEHXZ 10013778 f   U2Core:U2Core.dll
 0001:0001277e       ??0Logger@U2@@QAE@ABVQString@@@Z 1001377e f   U2Core:U2Core.dll
 0001:00012784       ??1Logger@U2@@UAE@XZ       10013784 f   U2Core:U2Core.dll
 0001:0001278a       ??CMultipleSequenceAlignmentRow@U2@@QAEPAVMultipleSequenceAlignmentRowData@1@XZ 1001378a f   U2Core:U2Core.dll
 0001:00012790       ??1MultipleSequenceAlignmentRow@U2@@UAE@XZ 10013790 f   U2Core:U2Core.dll
 0001:00012796       ??0MultipleSequenceAlignment@U2@@QAE@ABVQString@@PBVDNAAlphabet@1@ABV?$QList@VMultipleSequenceAlignmentRow@U2@@@@@Z 10013796 f   U2Core:U2Core.dll
 0001:0001279c       ??CMultipleSequenceAlignment@U2@@QAEPAVMultipleSequenceAlignmentData@1@XZ 1001379c f   U2Core:U2Core.dll
 0001:000127a2       ??1MultipleSequenceAlignment@U2@@UAE@XZ 100137a2 f   U2Core:U2Core.dll
 0001:000127a8       ??0MultipleSequenceAlignment@U2@@QAE@ABV01@@Z 100137a8 f   U2Core:U2Core.dll
 0001:000127ae       ??4MultipleSequenceAlignment@U2@@QAEAAV01@ABV01@@Z 100137ae f   U2Core:U2Core.dll
 0001:000127b4       ?getNumRows@MultipleSequenceAlignmentData@U2@@QBEHXZ 100137b4 f   U2Core:U2Core.dll
 0001:000127ba       ?getMsaRow@MultipleSequenceAlignmentData@U2@@QAE?AVMultipleSequenceAlignmentRow@2@H@Z 100137ba f   U2Core:U2Core.dll
 0001:000127c0       ?getMsaCopy@MultipleSequenceAlignmentObject@U2@@QBE?BVMultipleSequenceAlignment@2@XZ 100137c0 f   U2Core:U2Core.dll
 0001:000127c6       ??0Task@U2@@QAE@ABVQString@@V?$QFlags@W4TaskFlag@U2@@@@@Z 100137c6 f   U2Core:U2Core.dll
 0001:000127cc       ?hasError@Task@U2@@QBE_NXZ 100137cc f   U2Core:U2Core.dll
 0001:000127d2       ?getError@Task@U2@@QBE?AVQString@@XZ 100137d2 f   U2Core:U2Core.dll
 0001:000127d8       ?setVerboseLogMode@Task@U2@@QAEX_N@Z 100137d8 f   U2Core:U2Core.dll
 0001:000127de       ?setError@Task@U2@@QAEXABVQString@@@Z 100137de f   U2Core:U2Core.dll
 0001:000127e4       ??1Task@U2@@UAE@XZ         100137e4 f   U2Core:U2Core.dll
 0001:000127ea       ?cleanup@Task@U2@@UAEXXZ   100137ea f   U2Core:U2Core.dll
 0001:000127f0       ?getNumParallelSubtasks@Task@U2@@UBEHXZ 100137f0 f   U2Core:U2Core.dll
 0001:000127f6       ?getParentTask@Task@U2@@UBEPAV12@XZ 100137f6 f   U2Core:U2Core.dll
 0001:000127fc       ?getSubtaskWithErrors@Task@U2@@UBEPAV12@XZ 100137fc f   U2Core:U2Core.dll
 0001:00012802       ?getTaskId@Task@U2@@UBE_JXZ 10013802 f   U2Core:U2Core.dll
 0001:00012808       ?getTopLevelParentTask@Task@U2@@UAEPAV12@XZ 10013808 f   U2Core:U2Core.dll
 0001:0001280e       ?getWarnings@Task@U2@@UBE?AVQStringList@@XZ 1001380e f   U2Core:U2Core.dll
 0001:00012814       ?hasSubtasksWithErrors@Task@U2@@UBE_NXZ 10013814 f   U2Core:U2Core.dll
 0001:0001281a       ?hasWarning@Task@U2@@UBE_NXZ 1001381a f   U2Core:U2Core.dll
 0001:00012820       ?isNotificationReport@Task@U2@@UBE_NXZ 10013820 f   U2Core:U2Core.dll
 0001:00012826       ?isReportingSupported@Task@U2@@UBE_NXZ 10013826 f   U2Core:U2Core.dll
 0001:0001282c       ?isTopLevelTask@Task@U2@@UBE_NXZ 1001382c f   U2Core:U2Core.dll
 0001:00012832       ?onSubTaskFinished@Task@U2@@MAE?AV?$QList@PAVTask@U2@@@@PAV12@@Z 10013832 f   U2Core:U2Core.dll
 0001:00012838       ?prepare@Task@U2@@UAEXXZ   10013838 f   U2Core:U2Core.dll
 0001:0001283e       ?propagateSubtaskError@Task@U2@@UAE_NXZ 1001383e f   U2Core:U2Core.dll
 0001:00012844       ?setCollectChildrensWarningsFlag@Task@U2@@UAEX_N@Z 10013844 f   U2Core:U2Core.dll
 0001:0001284a       ?setNoAutoDelete@Task@U2@@UAEX_N@Z 1001384a f   U2Core:U2Core.dll
 0001:00012850       ?setNotificationReport@Task@U2@@UAEX_N@Z 10013850 f   U2Core:U2Core.dll
 0001:00012856       ?setReportingEnabled@Task@U2@@UAEX_N@Z 10013856 f   U2Core:U2Core.dll
 0001:0001285c       ?setReportingSupported@Task@U2@@UAEX_N@Z 1001385c f   U2Core:U2Core.dll
 0001:00012862       ?error@Logger@U2@@QAEXABVQString@@@Z 10013862 f   U2Core:U2Core.dll
 0001:00012868       ??0Plugin@U2@@QAE@ABVQString@@0_NW4PluginState@1@@Z 10013868 f   U2Core:U2Core.dll
 0001:0001286e       ??1Plugin@U2@@UAE@XZ       1001386e f   U2Core:U2Core.dll
 0001:00012874       ??1U2EntityRef@U2@@QAE@XZ  10013874 f   U2Core:U2Core.dll
 0001:0001287a       ?getAlphabet@U2SequenceObject@U2@@QBEPBVDNAAlphabet@2@XZ 1001387a f   U2Core:U2Core.dll
 0001:00012880       ?addSubTask@Task@U2@@QAEXPAV12@@Z 10013880 f   U2Core:U2Core.dll
 0001:00012886       ?generateReport@Task@U2@@UBE?AVQString@@XZ 10013886 f   U2Core:U2Core.dll
 0001:0001288c       ?isReportingEnabled@Task@U2@@UBE_NXZ 1001388c f   U2Core:U2Core.dll
 0001:00012892       ?metaObject@Task@U2@@UBEPBUQMetaObject@@XZ 10013892 f   U2Core:U2Core.dll
 0001:00012898       ?qt_metacall@Task@U2@@UAEHW4Call@QMetaObject@@HPAPAX@Z 10013898 f   U2Core:U2Core.dll
 0001:0001289e       ?qt_metacast@Task@U2@@UAEPAXPBD@Z 1001389e f   U2Core:U2Core.dll
 0001:000128a4       ?report@Task@U2@@UAE?AW4ReportResult@12@XZ 100138a4 f   U2Core:U2Core.dll
 0001:000128aa       ?run@Task@U2@@UAEXXZ       100138aa f   U2Core:U2Core.dll
 0001:000128b0       ??CMultipleSequenceAlignmentRow@U2@@QBEPBVMultipleSequenceAlignmentRowData@1@XZ 100138b0 f   U2Core:U2Core.dll
 0001:000128b6       ??0MultipleSequenceAlignmentRow@U2@@QAE@ABV01@@Z 100138b6 f   U2Core:U2Core.dll
 0001:000128bc       ?getExplicitCopy@MultipleSequenceAlignmentRowData@U2@@QBE?AVMultipleSequenceAlignmentRow@2@XZ 100138bc f   U2Core:U2Core.dll
 0001:000128c2       ?sortRowsBySimilarity@MultipleSequenceAlignmentData@U2@@QAE_NAAV?$QVector@VU2Region@U2@@@@@Z 100138c2 f   U2Core:U2Core.dll
 0001:000128c8       ?getMsaRows@MultipleSequenceAlignmentData@U2@@QBE?BV?$QList@VMultipleSequenceAlignmentRow@U2@@@@XZ 100138c8 f   U2Core:U2Core.dll
 0001:000128ce       ?getMSADistanceAlgorithmRegistry@AppContext@U2@@SAPAVMSADistanceAlgorithmRegistry@2@XZ 100138ce f   U2Core:U2Core.dll
 0001:000128d4       ?wrapForCSV@TextUtils@U2@@SAXAAVQString@@@Z 100138d4 f   U2Core:U2Core.dll
 0001:000128da       ?qt_metacast@Plugin@U2@@UAEPAXPBD@Z 100138da f   U2Core:U2Core.dll
 0001:000128e0       ?qt_metacall@Plugin@U2@@UAEHW4Call@QMetaObject@@HPAPAX@Z 100138e0 f   U2Core:U2Core.dll
 0001:000128e6       ?getId@MSADistanceAlgorithmFactory@U2@@QBE?AVQString@@XZ 100138e6 f   U2Algorithm:U2Algorithm.dll
 0001:000128ec       ?setFlag@MSADistanceAlgorithmFactory@U2@@QAEXW4DistanceAlgorithmFlag@2@@Z 100138ec f   U2Algorithm:U2Algorithm.dll
 0001:000128f2       ?resetFlag@MSADistanceAlgorithmFactory@U2@@QAEXW4DistanceAlgorithmFlag@2@@Z 100138f2 f   U2Algorithm:U2Algorithm.dll
 0001:000128f8       ?getSimilarity@MSADistanceAlgorithm@U2@@QAEHHH_N@Z 100138f8 f   U2Algorithm:U2Algorithm.dll
 0001:000128fe       ?getAlgorithmFactory@MSADistanceAlgorithmRegistry@U2@@QAEPAVMSADistanceAlgorithmFactory@2@ABVQString@@@Z 100138fe f   U2Algorithm:U2Algorithm.dll
 0001:00012904       ?getAlgorithmFactories@MSADistanceAlgorithmRegistry@U2@@QBE?AV?$QList@PAVMSADistanceAlgorithmFactory@U2@@@@XZ 10013904 f   U2Algorithm:U2Algorithm.dll
 0001:0001290a       ??0HelpButton@U2@@QAE@PAVQObject@@PAVQDialogButtonBox@@ABVQString@@@Z 1001390a f   U2Gui:U2Gui.dll
 0001:00012910       ??1HelpButton@U2@@UAE@XZ   10013910 f   U2Gui:U2Gui.dll
 0001:00012916       ??0LastUsedDirHelper@U2@@QAE@ABVQString@@0@Z 10013916 f   U2Gui:U2Gui.dll
 0001:0001291c       ??1LastUsedDirHelper@U2@@UAE@XZ 1001391c f   U2Gui:U2Gui.dll
 0001:00012922       ??0SaveDocumentControllerConfig@U2@@QAE@XZ 10013922 f   U2Gui:U2Gui.dll
 0001:00012928       ??1SaveDocumentControllerConfig@U2@@QAE@XZ 10013928 f   U2Gui:U2Gui.dll
 0001:0001292e       ?addFormat@SimpleFormatsInfo@SaveDocumentController@U2@@QAEXABVQString@@0ABVQStringList@@@Z 1001392e f   U2Gui:U2Gui.dll
 0001:00012934       ??0SimpleFormatsInfo@SaveDocumentController@U2@@QAE@XZ 10013934 f   U2Gui:U2Gui.dll
 0001:0001293a       ??1SimpleFormatsInfo@SaveDocumentController@U2@@QAE@XZ 1001393a f   U2Gui:U2Gui.dll
 0001:00012940       ??0SaveDocumentController@U2@@QAE@ABVSaveDocumentControllerConfig@1@ABVSimpleFormatsInfo@01@PAVQObject@@@Z 10013940 f   U2Gui:U2Gui.dll
 0001:00012946       ?setFormat@SaveDocumentController@U2@@QAEXABVQString@@@Z 10013946 f   U2Gui:U2Gui.dll
 0001:0001294c       ?getSaveFileName@SaveDocumentController@U2@@QBE?AVQString@@XZ 1001394c f   U2Gui:U2Gui.dll
 0001:00012952       ??1SaveDocumentController@U2@@UAE@XZ 10013952 f   U2Gui:U2Gui.dll
 0001:00012958       ??1MWMDIWindow@U2@@UAE@XZ  10013958 f   U2Gui:U2Gui.dll
 0001:0001295e       ?metaObject@HelpButton@U2@@UBEPBUQMetaObject@@XZ 1001395e f   U2Gui:U2Gui.dll
 0001:00012964       ?metaObject@SaveDocumentController@U2@@UBEPBUQMetaObject@@XZ 10013964 f   U2Gui:U2Gui.dll
 0001:0001296a       ?onCloseEvent@MWMDIWindow@U2@@MAE_NXZ 1001396a f   U2Gui:U2Gui.dll
 0001:00012970       ?qt_metacall@HelpButton@U2@@UAEHW4Call@QMetaObject@@HPAPAX@Z 10013970 f   U2Gui:U2Gui.dll
 0001:00012976       ?qt_metacall@SaveDocumentController@U2@@UAEHW4Call@QMetaObject@@HPAPAX@Z 10013976 f   U2Gui:U2Gui.dll
 0001:0001297c       ?qt_metacast@HelpButton@U2@@UAEPAXPBD@Z 1001397c f   U2Gui:U2Gui.dll
 0001:00012982       ?qt_metacast@SaveDocumentController@U2@@UAEPAXPBD@Z 10013982 f   U2Gui:U2Gui.dll
 0001:00012988       ?setupMDIToolbar@MWMDIWindow@U2@@UAEXPAVQToolBar@@@Z 10013988 f   U2Gui:U2Gui.dll
 0001:0001298e       ?setupViewMenu@MWMDIWindow@U2@@UAEXPAVQMenu@@@Z 1001398e f   U2Gui:U2Gui.dll
 0001:00012994       ?sl_buttonClicked@HelpButton@U2@@MAEXXZ 10013994 f   U2Gui:U2Gui.dll
 0001:0001299a       ?findSubMenu@GUIUtils@U2@@SAPAVQMenu@@PAV3@ABVQString@@@Z 1001399a f   U2Gui:U2Gui.dll
 0001:000129a0       ?getWidget@GObjectView@U2@@QAEPAVQWidget@@XZ 100139a0 f   U2Gui:U2Gui.dll
 0001:000129a6       ??0GObjectViewAction@U2@@QAE@PAVQObject@@PAVGObjectView@1@ABVQString@@H@Z 100139a6 f   U2Gui:U2Gui.dll
 0001:000129ac       ?getObjectView@GObjectViewAction@U2@@QBEPAVGObjectView@2@XZ 100139ac f   U2Gui:U2Gui.dll
 0001:000129b2       ??0GObjectViewWindowContext@U2@@QAE@PAVQObject@@ABVGObjectViewFactoryId@1@@Z 100139b2 f   U2Gui:U2Gui.dll
 0001:000129b8       ??1GObjectViewWindowContext@U2@@UAE@XZ 100139b8 f   U2Gui:U2Gui.dll
 0001:000129be       ?getViewActions@GObjectViewWindowContext@U2@@QBE?AV?$QList@PAVGObjectViewAction@U2@@@@PAVGObjectView@2@@Z 100139be f   U2Gui:U2Gui.dll
 0001:000129c4       ?addViewAction@GObjectViewWindowContext@U2@@IAEXPAVGObjectViewAction@2@@Z 100139c4 f   U2Gui:U2Gui.dll
 0001:000129ca       ?canHandle@GObjectViewObjectHandler@U2@@UAE_NPAVGObjectView@2@PAVGObject@2@@Z 100139ca f   U2Gui:U2Gui.dll
 0001:000129d0       ?disconnectView@GObjectViewWindowContext@U2@@MAEXPAVGObjectView@2@@Z 100139d0 f   U2Gui:U2Gui.dll
 0001:000129d6       ?init@GObjectViewWindowContext@U2@@UAEXXZ 100139d6 f   U2Gui:U2Gui.dll
 0001:000129dc       ?metaObject@GObjectViewAction@U2@@UBEPBUQMetaObject@@XZ 100139dc f   U2Gui:U2Gui.dll
 0001:000129e2       ?onObjectAdded@GObjectViewObjectHandler@U2@@UAEXPAVGObjectView@2@PAVGObject@2@@Z 100139e2 f   U2Gui:U2Gui.dll
 0001:000129e8       ?onObjectRemoved@GObjectViewWindowContext@U2@@UAEXPAVGObjectView@2@PAVGObject@2@@Z 100139e8 f   U2Gui:U2Gui.dll
 0001:000129ee       ?qt_metacall@GObjectViewAction@U2@@UAEHW4Call@QMetaObject@@HPAPAX@Z 100139ee f   U2Gui:U2Gui.dll
 0001:000129f4       ?qt_metacast@GObjectViewAction@U2@@UAEPAXPBD@Z 100139f4 f   U2Gui:U2Gui.dll
 0001:000129fa       ?sl_buildContextMenu@GObjectViewWindowContext@U2@@MAEXPAVGObjectView@2@PAVQMenu@@@Z 100139fa f   U2Gui:U2Gui.dll
 0001:00012a00       ?sl_buildStaticMenu@GObjectViewWindowContext@U2@@MAEXPAVGObjectView@2@PAVQMenu@@@Z 10013a00 f   U2Gui:U2Gui.dll
 0001:00012a06       ?sl_windowAdded@GObjectViewWindowContext@U2@@MAEXPAVMWMDIWindow@2@@Z 10013a06 f   U2Gui:U2Gui.dll
 0001:00012a0c       ?sl_windowClosing@GObjectViewWindowContext@U2@@MAEXPAVMWMDIWindow@2@@Z 10013a0c f   U2Gui:U2Gui.dll
 0001:00012a12       ?qt_metacast@GObjectViewWindowContext@U2@@UAEPAXPBD@Z 10013a12 f   U2Gui:U2Gui.dll
 0001:00012a18       ?qt_metacall@GObjectViewWindowContext@U2@@UAEHW4Call@QMetaObject@@HPAPAX@Z 10013a18 f   U2Gui:U2Gui.dll
 0001:00012a1e       ??0WebWindow@U2@@QAE@ABVQString@@0@Z 10013a1e f   U2View:U2View.dll
 0001:00012a24       ?metaObject@WebWindow@U2@@UBEPBUQMetaObject@@XZ 10013a24 f   U2View:U2View.dll
 0001:00012a2a       ?qt_metacall@WebWindow@U2@@UAEHW4Call@QMetaObject@@HPAPAX@Z 10013a2a f   U2View:U2View.dll
 0001:00012a30       ?qt_metacast@WebWindow@U2@@UAEPAXPBD@Z 10013a30 f   U2View:U2View.dll
 0001:00012a36       ?getResult@?$BackgroundTask@V?$QList@UCharOccurResult@U2@@@@@U2@@QBE?AV?$QList@UCharOccurResult@U2@@@@XZ 10013a36 f   U2View:U2View.dll
 0001:00012a3c       ??0CharOccurTask@U2@@QAE@PBVDNAAlphabet@1@VU2EntityRef@1@VU2Region@1@@Z 10013a3c f   U2View:U2View.dll
 0001:00012a42       ??1CharOccurTask@U2@@UAE@XZ 10013a42 f   U2View:U2View.dll
 0001:00012a48       ?getResult@?$BackgroundTask@V?$QMap@VQByteArray@@_J@@@U2@@QBE?AV?$QMap@VQByteArray@@_J@@XZ 10013a48 f   U2View:U2View.dll
 0001:00012a4e       ??0DinuclOccurTask@U2@@QAE@PBVDNAAlphabet@1@VU2EntityRef@1@VU2Region@1@@Z 10013a4e f   U2View:U2View.dll
 0001:00012a54       ??1DinuclOccurTask@U2@@UAE@XZ 10013a54 f   U2View:U2View.dll
 0001:00012a5a       ??0DNAStatisticsTask@U2@@QAE@PBVDNAAlphabet@1@VU2EntityRef@1@ABVU2Region@1@@Z 10013a5a f   U2View:U2View.dll
 0001:00012a60       ??1DNAStatisticsTask@U2@@UAE@XZ 10013a60 f   U2View:U2View.dll
 0001:00012a66       ?getSequenceGObject@SequenceObjectContext@U2@@QBEPAVGObject@2@XZ 10013a66 f   U2View:U2View.dll
 0001:00012a6c       ?getSequenceLength@SequenceObjectContext@U2@@QBE_JXZ 10013a6c f   U2View:U2View.dll
 0001:00012a72       ?getAlphabet@SequenceObjectContext@U2@@QBEPBVDNAAlphabet@2@XZ 10013a72 f   U2View:U2View.dll
 0001:00012a78       ?getSequenceRef@SequenceObjectContext@U2@@QBE?AVU2EntityRef@2@XZ 10013a78 f   U2View:U2View.dll
 0001:00012a7e       ?metaObject@DNAStatisticsTask@U2@@UBEPBUQMetaObject@@XZ 10013a7e f   U2View:U2View.dll
 0001:00012a84       ?qt_metacall@DNAStatisticsTask@U2@@UAEHW4Call@QMetaObject@@HPAPAX@Z 10013a84 f   U2View:U2View.dll
 0001:00012a8a       ?qt_metacast@DNAStatisticsTask@U2@@UAEPAXPBD@Z 10013a8a f   U2View:U2View.dll
 0001:00012a90       ?run@CharOccurTask@U2@@UAEXXZ 10013a90 f   U2View:U2View.dll
 0001:00012a96       ?run@DNAStatisticsTask@U2@@UAEXXZ 10013a96 f   U2View:U2View.dll
 0001:00012a9c       ?run@DinuclOccurTask@U2@@UAEXXZ 10013a9c f   U2View:U2View.dll
 0001:00012aa2       ?setWindowTitle@QWidget@@QAEXABVQString@@@Z 10013aa2 f   Qt5Widgets:Qt5Widgets.dll
 0001:00012aa8       ?setWindowIcon@QWidget@@QAEXABVQIcon@@@Z 10013aa8 f   Qt5Widgets:Qt5Widgets.dll
 0001:00012aae       ?resize@QWidget@@QAEXABVQSize@@@Z 10013aae f   Qt5Widgets:Qt5Widgets.dll
 0001:00012ab4       ??0QDialog@@QAE@PAVQWidget@@V?$QFlags@W4WindowType@Qt@@@@@Z 10013ab4 f   Qt5Widgets:Qt5Widgets.dll
 0001:00012aba       ??1QDialog@@UAE@XZ         10013aba f   Qt5Widgets:Qt5Widgets.dll
 0001:00012ac0       ?accept@QDialog@@UAEXXZ    10013ac0 f   Qt5Widgets:Qt5Widgets.dll
 0001:00012ac6       ?critical@QMessageBox@@SA?AW4StandardButton@1@PAVQWidget@@ABVQString@@1V?$QFlags@W4StandardButton@QMessageBox@@@@W421@@Z 10013ac6 f   Qt5Widgets:Qt5Widgets.dll
 0001:00012acc       ?setText@QAbstractButton@@QAEXABVQString@@@Z 10013acc f   Qt5Widgets:Qt5Widgets.dll
 0001:00012ad2       ?isChecked@QAbstractButton@@QBE_NXZ 10013ad2 f   Qt5Widgets:Qt5Widgets.dll
 0001:00012ad8       ?setChecked@QAbstractButton@@QAEX_N@Z 10013ad8 f   Qt5Widgets:Qt5Widgets.dll
 0001:00012ade       ??0QDialogButtonBox@@QAE@PAVQWidget@@@Z 10013ade f   Qt5Widgets:Qt5Widgets.dll
 0001:00012ae4       ??1QDialogButtonBox@@UAE@XZ 10013ae4 f   Qt5Widgets:Qt5Widgets.dll
 0001:00012aea       ?setStandardButtons@QDialogButtonBox@@QAEXV?$QFlags@W4StandardButton@QDialogButtonBox@@@@@Z 10013aea f   Qt5Widgets:Qt5Widgets.dll
 0001:00012af0       ?button@QDialogButtonBox@@QBEPAVQPushButton@@W4StandardButton@1@@Z 10013af0 f   Qt5Widgets:Qt5Widgets.dll
 0001:00012af6       ??0QLabel@@QAE@PAVQWidget@@V?$QFlags@W4WindowType@Qt@@@@@Z 10013af6 f   Qt5Widgets:Qt5Widgets.dll
 0001:00012afc       ??1QLabel@@UAE@XZ          10013afc f   Qt5Widgets:Qt5Widgets.dll
 0001:00012b02       ?setText@QLabel@@QAEXABVQString@@@Z 10013b02 f   Qt5Widgets:Qt5Widgets.dll
 0001:00012b08       ??0QCheckBox@@QAE@PAVQWidget@@@Z 10013b08 f   Qt5Widgets:Qt5Widgets.dll
 0001:00012b0e       ??1QCheckBox@@UAE@XZ       10013b0e f   Qt5Widgets:Qt5Widgets.dll
 0001:00012b14       ?addWidget@QBoxLayout@@QAEXPAVQWidget@@HV?$QFlags@W4AlignmentFlag@Qt@@@@@Z 10013b14 f   Qt5Widgets:Qt5Widgets.dll
 0001:00012b1a       ??0QVBoxLayout@@QAE@PAVQWidget@@@Z 10013b1a f   Qt5Widgets:Qt5Widgets.dll
 0001:00012b20       ??1QVBoxLayout@@UAE@XZ     10013b20 f   Qt5Widgets:Qt5Widgets.dll
 0001:00012b26       ??0QGridLayout@@QAE@PAVQWidget@@@Z 10013b26 f   Qt5Widgets:Qt5Widgets.dll
 0001:00012b2c       ??1QGridLayout@@UAE@XZ     10013b2c f   Qt5Widgets:Qt5Widgets.dll
 0001:00012b32       ?addWidget@QGridLayout@@QAEXPAVQWidget@@HHHHV?$QFlags@W4AlignmentFlag@Qt@@@@@Z 10013b32 f   Qt5Widgets:Qt5Widgets.dll
 0001:00012b38       ??0QGroupBox@@QAE@PAVQWidget@@@Z 10013b38 f   Qt5Widgets:Qt5Widgets.dll
 0001:00012b3e       ??1QGroupBox@@UAE@XZ       10013b3e f   Qt5Widgets:Qt5Widgets.dll
 0001:00012b44       ?setTitle@QGroupBox@@QAEXABVQString@@@Z 10013b44 f   Qt5Widgets:Qt5Widgets.dll
 0001:00012b4a       ?setCheckable@QGroupBox@@QAEX_N@Z 10013b4a f   Qt5Widgets:Qt5Widgets.dll
 0001:00012b50       ?isChecked@QGroupBox@@QBE_NXZ 10013b50 f   Qt5Widgets:Qt5Widgets.dll
 0001:00012b56       ?setChecked@QGroupBox@@QAEX_N@Z 10013b56 f   Qt5Widgets:Qt5Widgets.dll
 0001:00012b5c       ??0QLineEdit@@QAE@PAVQWidget@@@Z 10013b5c f   Qt5Widgets:Qt5Widgets.dll
 0001:00012b62       ??1QLineEdit@@UAE@XZ       10013b62 f   Qt5Widgets:Qt5Widgets.dll
 0001:00012b68       ??0QRadioButton@@QAE@PAVQWidget@@@Z 10013b68 f   Qt5Widgets:Qt5Widgets.dll
 0001:00012b6e       ??1QRadioButton@@UAE@XZ    10013b6e f   Qt5Widgets:Qt5Widgets.dll
 0001:00012b74       ??0QToolButton@@QAE@PAVQWidget@@@Z 10013b74 f   Qt5Widgets:Qt5Widgets.dll
 0001:00012b7a       ??1QToolButton@@UAE@XZ     10013b7a f   Qt5Widgets:Qt5Widgets.dll
 0001:00012b80       ?actionEvent@QToolButton@@MAEXPAVQActionEvent@@@Z 10013b80 f   Qt5Widgets:Qt5Widgets.dll
 0001:00012b86       ?actionEvent@QWidget@@MAEXPAVQActionEvent@@@Z 10013b86 f   Qt5Widgets:Qt5Widgets.dll
 0001:00012b8c       ?addItem@QBoxLayout@@UAEXPAVQLayoutItem@@@Z 10013b8c f   Qt5Widgets:Qt5Widgets.dll
 0001:00012b92       ?addItem@QGridLayout@@MAEXPAVQLayoutItem@@@Z 10013b92 f   Qt5Widgets:Qt5Widgets.dll
 0001:00012b98       ?changeEvent@QAbstractButton@@MAEXPAVQEvent@@@Z 10013b98 f   Qt5Widgets:Qt5Widgets.dll
 0001:00012b9e       ?changeEvent@QDialogButtonBox@@MAEXPAVQEvent@@@Z 10013b9e f   Qt5Widgets:Qt5Widgets.dll
 0001:00012ba4       ?changeEvent@QGroupBox@@MAEXPAVQEvent@@@Z 10013ba4 f   Qt5Widgets:Qt5Widgets.dll
 0001:00012baa       ?changeEvent@QLabel@@MAEXPAVQEvent@@@Z 10013baa f   Qt5Widgets:Qt5Widgets.dll
 0001:00012bb0       ?changeEvent@QLineEdit@@MAEXPAVQEvent@@@Z 10013bb0 f   Qt5Widgets:Qt5Widgets.dll
 0001:00012bb6       ?changeEvent@QToolButton@@MAEXPAVQEvent@@@Z 10013bb6 f   Qt5Widgets:Qt5Widgets.dll
 0001:00012bbc       ?changeEvent@QWidget@@MAEXPAVQEvent@@@Z 10013bbc f   Qt5Widgets:Qt5Widgets.dll
 0001:00012bc2       ?checkStateSet@QAbstractButton@@MAEXXZ 10013bc2 f   Qt5Widgets:Qt5Widgets.dll
 0001:00012bc8       ?checkStateSet@QCheckBox@@MAEXXZ 10013bc8 f   Qt5Widgets:Qt5Widgets.dll
 0001:00012bce       ?childEvent@QGroupBox@@MAEXPAVQChildEvent@@@Z 10013bce f   Qt5Widgets:Qt5Widgets.dll
 0001:00012bd4       ?childEvent@QLayout@@MAEXPAVQChildEvent@@@Z 10013bd4 f   Qt5Widgets:Qt5Widgets.dll
 0001:00012bda       ?closeEvent@QDialog@@MAEXPAVQCloseEvent@@@Z 10013bda f   Qt5Widgets:Qt5Widgets.dll
 0001:00012be0       ?closeEvent@QWidget@@MAEXPAVQCloseEvent@@@Z 10013be0 f   Qt5Widgets:Qt5Widgets.dll
 0001:00012be6       ?contextMenuEvent@QDialog@@MAEXPAVQContextMenuEvent@@@Z 10013be6 f   Qt5Widgets:Qt5Widgets.dll
 0001:00012bec       ?contextMenuEvent@QLabel@@MAEXPAVQContextMenuEvent@@@Z 10013bec f   Qt5Widgets:Qt5Widgets.dll
 0001:00012bf2       ?contextMenuEvent@QLineEdit@@MAEXPAVQContextMenuEvent@@@Z 10013bf2 f   Qt5Widgets:Qt5Widgets.dll
 0001:00012bf8       ?contextMenuEvent@QWidget@@MAEXPAVQContextMenuEvent@@@Z 10013bf8 f   Qt5Widgets:Qt5Widgets.dll
 0001:00012bfe       ?controlTypes@QLayout@@UBE?AV?$QFlags@W4ControlType@QSizePolicy@@@@XZ 10013bfe f   Qt5Widgets:Qt5Widgets.dll
 0001:00012c04       ?count@QBoxLayout@@UBEHXZ  10013c04 f   Qt5Widgets:Qt5Widgets.dll
 0001:00012c0a       ?count@QGridLayout@@UBEHXZ 10013c0a f   Qt5Widgets:Qt5Widgets.dll
 0001:00012c10       ?devType@QWidget@@UBEHXZ   10013c10 f   Qt5Widgets:Qt5Widgets.dll
 0001:00012c16       ?done@QDialog@@UAEXH@Z     10013c16 f   Qt5Widgets:Qt5Widgets.dll
 0001:00012c1c       ?dragEnterEvent@QLineEdit@@MAEXPAVQDragEnterEvent@@@Z 10013c1c f   Qt5Widgets:Qt5Widgets.dll
 0001:00012c22       ?dragEnterEvent@QWidget@@MAEXPAVQDragEnterEvent@@@Z 10013c22 f   Qt5Widgets:Qt5Widgets.dll
 0001:00012c28       ?dragLeaveEvent@QLineEdit@@MAEXPAVQDragLeaveEvent@@@Z 10013c28 f   Qt5Widgets:Qt5Widgets.dll
 0001:00012c2e       ?dragLeaveEvent@QWidget@@MAEXPAVQDragLeaveEvent@@@Z 10013c2e f   Qt5Widgets:Qt5Widgets.dll
 0001:00012c34       ?dragMoveEvent@QLineEdit@@MAEXPAVQDragMoveEvent@@@Z 10013c34 f   Qt5Widgets:Qt5Widgets.dll
 0001:00012c3a       ?dragMoveEvent@QWidget@@MAEXPAVQDragMoveEvent@@@Z 10013c3a f   Qt5Widgets:Qt5Widgets.dll
 0001:00012c40       ?dropEvent@QLineEdit@@MAEXPAVQDropEvent@@@Z 10013c40 f   Qt5Widgets:Qt5Widgets.dll
 0001:00012c46       ?dropEvent@QWidget@@MAEXPAVQDropEvent@@@Z 10013c46 f   Qt5Widgets:Qt5Widgets.dll
 0001:00012c4c       ?enterEvent@QToolButton@@MAEXPAVQEvent@@@Z 10013c4c f   Qt5Widgets:Qt5Widgets.dll
 0001:00012c52       ?enterEvent@QWidget@@MAEXPAVQEvent@@@Z 10013c52 f   Qt5Widgets:Qt5Widgets.dll
 0001:00012c58       ?event@QCheckBox@@MAE_NPAVQEvent@@@Z 10013c58 f   Qt5Widgets:Qt5Widgets.dll
 0001:00012c5e       ?event@QDialogButtonBox@@MAE_NPAVQEvent@@@Z 10013c5e f   Qt5Widgets:Qt5Widgets.dll
 0001:00012c64       ?event@QGroupBox@@MAE_NPAVQEvent@@@Z 10013c64 f   Qt5Widgets:Qt5Widgets.dll
 0001:00012c6a       ?event@QLabel@@MAE_NPAVQEvent@@@Z 10013c6a f   Qt5Widgets:Qt5Widgets.dll
 0001:00012c70       ?event@QLineEdit@@UAE_NPAVQEvent@@@Z 10013c70 f   Qt5Widgets:Qt5Widgets.dll
 0001:00012c76       ?event@QRadioButton@@MAE_NPAVQEvent@@@Z 10013c76 f   Qt5Widgets:Qt5Widgets.dll
 0001:00012c7c       ?event@QToolButton@@MAE_NPAVQEvent@@@Z 10013c7c f   Qt5Widgets:Qt5Widgets.dll
 0001:00012c82       ?event@QWidget@@MAE_NPAVQEvent@@@Z 10013c82 f   Qt5Widgets:Qt5Widgets.dll
 0001:00012c88       ?eventFilter@QDialog@@MAE_NPAVQObject@@PAVQEvent@@@Z 10013c88 f   Qt5Widgets:Qt5Widgets.dll
 0001:00012c8e       ?exec@QDialog@@UAEHXZ      10013c8e f   Qt5Widgets:Qt5Widgets.dll
 0001:00012c94       ?expandingDirections@QBoxLayout@@UBE?AV?$QFlags@W4Orientation@Qt@@@@XZ 10013c94 f   Qt5Widgets:Qt5Widgets.dll
 0001:00012c9a       ?expandingDirections@QGridLayout@@UBE?AV?$QFlags@W4Orientation@Qt@@@@XZ 10013c9a f   Qt5Widgets:Qt5Widgets.dll
 0001:00012ca0       ?focusInEvent@QAbstractButton@@MAEXPAVQFocusEvent@@@Z 10013ca0 f   Qt5Widgets:Qt5Widgets.dll
 0001:00012ca6       ?focusInEvent@QGroupBox@@MAEXPAVQFocusEvent@@@Z 10013ca6 f   Qt5Widgets:Qt5Widgets.dll
 0001:00012cac       ?focusInEvent@QLabel@@MAEXPAVQFocusEvent@@@Z 10013cac f   Qt5Widgets:Qt5Widgets.dll
 0001:00012cb2       ?focusInEvent@QLineEdit@@MAEXPAVQFocusEvent@@@Z 10013cb2 f   Qt5Widgets:Qt5Widgets.dll
 0001:00012cb8       ?focusInEvent@QWidget@@MAEXPAVQFocusEvent@@@Z 10013cb8 f   Qt5Widgets:Qt5Widgets.dll
 0001:00012cbe       ?focusNextPrevChild@QLabel@@MAE_N_N@Z 10013cbe f   Qt5Widgets:Qt5Widgets.dll
 0001:00012cc4       ?focusNextPrevChild@QWidget@@MAE_N_N@Z 10013cc4 f   Qt5Widgets:Qt5Widgets.dll
 0001:00012cca       ?focusOutEvent@QAbstractButton@@MAEXPAVQFocusEvent@@@Z 10013cca f   Qt5Widgets:Qt5Widgets.dll
 0001:00012cd0       ?focusOutEvent@QLabel@@MAEXPAVQFocusEvent@@@Z 10013cd0 f   Qt5Widgets:Qt5Widgets.dll
 0001:00012cd6       ?focusOutEvent@QLineEdit@@MAEXPAVQFocusEvent@@@Z 10013cd6 f   Qt5Widgets:Qt5Widgets.dll
 0001:00012cdc       ?focusOutEvent@QWidget@@MAEXPAVQFocusEvent@@@Z 10013cdc f   Qt5Widgets:Qt5Widgets.dll
 0001:00012ce2       ?geometry@QLayout@@UBE?AVQRect@@XZ 10013ce2 f   Qt5Widgets:Qt5Widgets.dll
 0001:00012ce8       ?hasHeightForWidth@QBoxLayout@@UBE_NXZ 10013ce8 f   Qt5Widgets:Qt5Widgets.dll
 0001:00012cee       ?hasHeightForWidth@QGridLayout@@UBE_NXZ 10013cee f   Qt5Widgets:Qt5Widgets.dll
 0001:00012cf4       ?hasHeightForWidth@QWidget@@UBE_NXZ 10013cf4 f   Qt5Widgets:Qt5Widgets.dll
 0001:00012cfa       ?heightForWidth@QBoxLayout@@UBEHH@Z 10013cfa f   Qt5Widgets:Qt5Widgets.dll
 0001:00012d00       ?heightForWidth@QGridLayout@@UBEHH@Z 10013d00 f   Qt5Widgets:Qt5Widgets.dll
 0001:00012d06       ?heightForWidth@QLabel@@UBEHH@Z 10013d06 f   Qt5Widgets:Qt5Widgets.dll
 0001:00012d0c       ?heightForWidth@QWidget@@UBEHH@Z 10013d0c f   Qt5Widgets:Qt5Widgets.dll
 0001:00012d12       ?hideEvent@QWidget@@MAEXPAVQHideEvent@@@Z 10013d12 f   Qt5Widgets:Qt5Widgets.dll
 0001:00012d18       ?hitButton@QCheckBox@@MBE_NABVQPoint@@@Z 10013d18 f   Qt5Widgets:Qt5Widgets.dll
 0001:00012d1e       ?hitButton@QRadioButton@@MBE_NABVQPoint@@@Z 10013d1e f   Qt5Widgets:Qt5Widgets.dll
 0001:00012d24       ?hitButton@QToolButton@@MBE_NABVQPoint@@@Z 10013d24 f   Qt5Widgets:Qt5Widgets.dll
 0001:00012d2a       ?indexOf@QLayout@@UBEHPAVQWidget@@@Z 10013d2a f   Qt5Widgets:Qt5Widgets.dll
 0001:00012d30       ?initPainter@QWidget@@MBEXPAVQPainter@@@Z 10013d30 f   Qt5Widgets:Qt5Widgets.dll
 0001:00012d36       ?inputMethodEvent@QLineEdit@@MAEXPAVQInputMethodEvent@@@Z 10013d36 f   Qt5Widgets:Qt5Widgets.dll
 0001:00012d3c       ?inputMethodEvent@QWidget@@MAEXPAVQInputMethodEvent@@@Z 10013d3c f   Qt5Widgets:Qt5Widgets.dll
 0001:00012d42       ?inputMethodQuery@QLineEdit@@UBE?AVQVariant@@W4InputMethodQuery@Qt@@@Z 10013d42 f   Qt5Widgets:Qt5Widgets.dll
 0001:00012d48       ?inputMethodQuery@QWidget@@UBE?AVQVariant@@W4InputMethodQuery@Qt@@@Z 10013d48 f   Qt5Widgets:Qt5Widgets.dll
 0001:00012d4e       ?invalidate@QBoxLayout@@UAEXXZ 10013d4e f   Qt5Widgets:Qt5Widgets.dll
 0001:00012d54       ?invalidate@QGridLayout@@UAEXXZ 10013d54 f   Qt5Widgets:Qt5Widgets.dll
 0001:00012d5a       ?isEmpty@QLayout@@UBE_NXZ  10013d5a f   Qt5Widgets:Qt5Widgets.dll
 0001:00012d60       ?itemAt@QBoxLayout@@UBEPAVQLayoutItem@@H@Z 10013d60 f   Qt5Widgets:Qt5Widgets.dll
 0001:00012d66       ?itemAt@QGridLayout@@UBEPAVQLayoutItem@@H@Z 10013d66 f   Qt5Widgets:Qt5Widgets.dll
 0001:00012d6c       ?keyPressEvent@QAbstractButton@@MAEXPAVQKeyEvent@@@Z 10013d6c f   Qt5Widgets:Qt5Widgets.dll
 0001:00012d72       ?keyPressEvent@QDialog@@MAEXPAVQKeyEvent@@@Z 10013d72 f   Qt5Widgets:Qt5Widgets.dll
 0001:00012d78       ?keyPressEvent@QLabel@@MAEXPAVQKeyEvent@@@Z 10013d78 f   Qt5Widgets:Qt5Widgets.dll
 0001:00012d7e       ?keyPressEvent@QLineEdit@@MAEXPAVQKeyEvent@@@Z 10013d7e f   Qt5Widgets:Qt5Widgets.dll
 0001:00012d84       ?keyPressEvent@QWidget@@MAEXPAVQKeyEvent@@@Z 10013d84 f   Qt5Widgets:Qt5Widgets.dll
 0001:00012d8a       ?keyReleaseEvent@QAbstractButton@@MAEXPAVQKeyEvent@@@Z 10013d8a f   Qt5Widgets:Qt5Widgets.dll
 0001:00012d90       ?keyReleaseEvent@QWidget@@MAEXPAVQKeyEvent@@@Z 10013d90 f   Qt5Widgets:Qt5Widgets.dll
 0001:00012d96       ?layout@QLayout@@UAEPAV1@XZ 10013d96 f   Qt5Widgets:Qt5Widgets.dll
 0001:00012d9c       ?leaveEvent@QToolButton@@MAEXPAVQEvent@@@Z 10013d9c f   Qt5Widgets:Qt5Widgets.dll
 0001:00012da2       ?leaveEvent@QWidget@@MAEXPAVQEvent@@@Z 10013da2 f   Qt5Widgets:Qt5Widgets.dll
 0001:00012da8       ?maximumSize@QBoxLayout@@UBE?AVQSize@@XZ 10013da8 f   Qt5Widgets:Qt5Widgets.dll
 0001:00012dae       ?maximumSize@QGridLayout@@UBE?AVQSize@@XZ 10013dae f   Qt5Widgets:Qt5Widgets.dll
 0001:00012db4       ?metaObject@QCheckBox@@UBEPBUQMetaObject@@XZ 10013db4 f   Qt5Widgets:Qt5Widgets.dll
 0001:00012dba       ?metaObject@QDialogButtonBox@@UBEPBUQMetaObject@@XZ 10013dba f   Qt5Widgets:Qt5Widgets.dll
 0001:00012dc0       ?metaObject@QGridLayout@@UBEPBUQMetaObject@@XZ 10013dc0 f   Qt5Widgets:Qt5Widgets.dll
 0001:00012dc6       ?metaObject@QGroupBox@@UBEPBUQMetaObject@@XZ 10013dc6 f   Qt5Widgets:Qt5Widgets.dll
 0001:00012dcc       ?metaObject@QLabel@@UBEPBUQMetaObject@@XZ 10013dcc f   Qt5Widgets:Qt5Widgets.dll
 0001:00012dd2       ?metaObject@QLineEdit@@UBEPBUQMetaObject@@XZ 10013dd2 f   Qt5Widgets:Qt5Widgets.dll
 0001:00012dd8       ?metaObject@QRadioButton@@UBEPBUQMetaObject@@XZ 10013dd8 f   Qt5Widgets:Qt5Widgets.dll
 0001:00012dde       ?metaObject@QToolButton@@UBEPBUQMetaObject@@XZ 10013dde f   Qt5Widgets:Qt5Widgets.dll
 0001:00012de4       ?metaObject@QVBoxLayout@@UBEPBUQMetaObject@@XZ 10013de4 f   Qt5Widgets:Qt5Widgets.dll
 0001:00012dea       ?metric@QWidget@@MBEHW4PaintDeviceMetric@QPaintDevice@@@Z 10013dea f   Qt5Widgets:Qt5Widgets.dll
 0001:00012df0       ?minimumHeightForWidth@QBoxLayout@@UBEHH@Z 10013df0 f   Qt5Widgets:Qt5Widgets.dll
 0001:00012df6       ?minimumHeightForWidth@QGridLayout@@UBEHH@Z 10013df6 f   Qt5Widgets:Qt5Widgets.dll
 0001:00012dfc       ?minimumSize@QBoxLayout@@UBE?AVQSize@@XZ 10013dfc f   Qt5Widgets:Qt5Widgets.dll
 0001:00012e02       ?minimumSize@QGridLayout@@UBE?AVQSize@@XZ 10013e02 f   Qt5Widgets:Qt5Widgets.dll
 0001:00012e08       ?minimumSizeHint@QCheckBox@@UBE?AVQSize@@XZ 10013e08 f   Qt5Widgets:Qt5Widgets.dll
 0001:00012e0e       ?minimumSizeHint@QDialog@@UBE?AVQSize@@XZ 10013e0e f   Qt5Widgets:Qt5Widgets.dll
 0001:00012e14       ?minimumSizeHint@QGroupBox@@UBE?AVQSize@@XZ 10013e14 f   Qt5Widgets:Qt5Widgets.dll
 0001:00012e1a       ?minimumSizeHint@QLabel@@UBE?AVQSize@@XZ 10013e1a f   Qt5Widgets:Qt5Widgets.dll
 0001:00012e20       ?minimumSizeHint@QLineEdit@@UBE?AVQSize@@XZ 10013e20 f   Qt5Widgets:Qt5Widgets.dll
 0001:00012e26       ?minimumSizeHint@QRadioButton@@UBE?AVQSize@@XZ 10013e26 f   Qt5Widgets:Qt5Widgets.dll
 0001:00012e2c       ?minimumSizeHint@QToolButton@@UBE?AVQSize@@XZ 10013e2c f   Qt5Widgets:Qt5Widgets.dll
 0001:00012e32       ?minimumSizeHint@QWidget@@UBE?AVQSize@@XZ 10013e32 f   Qt5Widgets:Qt5Widgets.dll
 0001:00012e38       ?mouseDoubleClickEvent@QLineEdit@@MAEXPAVQMouseEvent@@@Z 10013e38 f   Qt5Widgets:Qt5Widgets.dll
 0001:00012e3e       ?mouseDoubleClickEvent@QWidget@@MAEXPAVQMouseEvent@@@Z 10013e3e f   Qt5Widgets:Qt5Widgets.dll
 0001:00012e44       ?mouseMoveEvent@QAbstractButton@@MAEXPAVQMouseEvent@@@Z 10013e44 f   Qt5Widgets:Qt5Widgets.dll
 0001:00012e4a       ?mouseMoveEvent@QCheckBox@@MAEXPAVQMouseEvent@@@Z 10013e4a f   Qt5Widgets:Qt5Widgets.dll
 0001:00012e50       ?mouseMoveEvent@QGroupBox@@MAEXPAVQMouseEvent@@@Z 10013e50 f   Qt5Widgets:Qt5Widgets.dll
 0001:00012e56       ?mouseMoveEvent@QLabel@@MAEXPAVQMouseEvent@@@Z 10013e56 f   Qt5Widgets:Qt5Widgets.dll
 0001:00012e5c       ?mouseMoveEvent@QLineEdit@@MAEXPAVQMouseEvent@@@Z 10013e5c f   Qt5Widgets:Qt5Widgets.dll
 0001:00012e62       ?mouseMoveEvent@QRadioButton@@MAEXPAVQMouseEvent@@@Z 10013e62 f   Qt5Widgets:Qt5Widgets.dll
 0001:00012e68       ?mouseMoveEvent@QWidget@@MAEXPAVQMouseEvent@@@Z 10013e68 f   Qt5Widgets:Qt5Widgets.dll
 0001:00012e6e       ?mousePressEvent@QAbstractButton@@MAEXPAVQMouseEvent@@@Z 10013e6e f   Qt5Widgets:Qt5Widgets.dll
 0001:00012e74       ?mousePressEvent@QGroupBox@@MAEXPAVQMouseEvent@@@Z 10013e74 f   Qt5Widgets:Qt5Widgets.dll
 0001:00012e7a       ?mousePressEvent@QLabel@@MAEXPAVQMouseEvent@@@Z 10013e7a f   Qt5Widgets:Qt5Widgets.dll
 0001:00012e80       ?mousePressEvent@QLineEdit@@MAEXPAVQMouseEvent@@@Z 10013e80 f   Qt5Widgets:Qt5Widgets.dll
 0001:00012e86       ?mousePressEvent@QToolButton@@MAEXPAVQMouseEvent@@@Z 10013e86 f   Qt5Widgets:Qt5Widgets.dll
 0001:00012e8c       ?mousePressEvent@QWidget@@MAEXPAVQMouseEvent@@@Z 10013e8c f   Qt5Widgets:Qt5Widgets.dll
 0001:00012e92       ?mouseReleaseEvent@QAbstractButton@@MAEXPAVQMouseEvent@@@Z 10013e92 f   Qt5Widgets:Qt5Widgets.dll
 0001:00012e98       ?mouseReleaseEvent@QGroupBox@@MAEXPAVQMouseEvent@@@Z 10013e98 f   Qt5Widgets:Qt5Widgets.dll
 0001:00012e9e       ?mouseReleaseEvent@QLabel@@MAEXPAVQMouseEvent@@@Z 10013e9e f   Qt5Widgets:Qt5Widgets.dll
 0001:00012ea4       ?mouseReleaseEvent@QLineEdit@@MAEXPAVQMouseEvent@@@Z 10013ea4 f   Qt5Widgets:Qt5Widgets.dll
 0001:00012eaa       ?mouseReleaseEvent@QToolButton@@MAEXPAVQMouseEvent@@@Z 10013eaa f   Qt5Widgets:Qt5Widgets.dll
 0001:00012eb0       ?mouseReleaseEvent@QWidget@@MAEXPAVQMouseEvent@@@Z 10013eb0 f   Qt5Widgets:Qt5Widgets.dll
 0001:00012eb6       ?moveEvent@QWidget@@MAEXPAVQMoveEvent@@@Z 10013eb6 f   Qt5Widgets:Qt5Widgets.dll
 0001:00012ebc       ?nativeEvent@QWidget@@MAE_NABVQByteArray@@PAXPAJ@Z 10013ebc f   Qt5Widgets:Qt5Widgets.dll
 0001:00012ec2       ?nextCheckState@QAbstractButton@@MAEXXZ 10013ec2 f   Qt5Widgets:Qt5Widgets.dll
 0001:00012ec8       ?nextCheckState@QCheckBox@@MAEXXZ 10013ec8 f   Qt5Widgets:Qt5Widgets.dll
 0001:00012ece       ?nextCheckState@QToolButton@@MAEXXZ 10013ece f   Qt5Widgets:Qt5Widgets.dll
 0001:00012ed4       ?open@QDialog@@UAEXXZ      10013ed4 f   Qt5Widgets:Qt5Widgets.dll
 0001:00012eda       ?paintEngine@QWidget@@UBEPAVQPaintEngine@@XZ 10013eda f   Qt5Widgets:Qt5Widgets.dll
 0001:00012ee0       ?paintEvent@QCheckBox@@MAEXPAVQPaintEvent@@@Z 10013ee0 f   Qt5Widgets:Qt5Widgets.dll
 0001:00012ee6       ?paintEvent@QGroupBox@@MAEXPAVQPaintEvent@@@Z 10013ee6 f   Qt5Widgets:Qt5Widgets.dll
 0001:00012eec       ?paintEvent@QLabel@@MAEXPAVQPaintEvent@@@Z 10013eec f   Qt5Widgets:Qt5Widgets.dll
 0001:00012ef2       ?paintEvent@QLineEdit@@MAEXPAVQPaintEvent@@@Z 10013ef2 f   Qt5Widgets:Qt5Widgets.dll
 0001:00012ef8       ?paintEvent@QRadioButton@@MAEXPAVQPaintEvent@@@Z 10013ef8 f   Qt5Widgets:Qt5Widgets.dll
 0001:00012efe       ?paintEvent@QToolButton@@MAEXPAVQPaintEvent@@@Z 10013efe f   Qt5Widgets:Qt5Widgets.dll
 0001:00012f04       ?paintEvent@QWidget@@MAEXPAVQPaintEvent@@@Z 10013f04 f   Qt5Widgets:Qt5Widgets.dll
 0001:00012f0a       ?qt_metacall@QCheckBox@@UAEHW4Call@QMetaObject@@HPAPAX@Z 10013f0a f   Qt5Widgets:Qt5Widgets.dll
 0001:00012f10       ?qt_metacall@QDialogButtonBox@@UAEHW4Call@QMetaObject@@HPAPAX@Z 10013f10 f   Qt5Widgets:Qt5Widgets.dll
 0001:00012f16       ?qt_metacall@QGridLayout@@UAEHW4Call@QMetaObject@@HPAPAX@Z 10013f16 f   Qt5Widgets:Qt5Widgets.dll
 0001:00012f1c       ?qt_metacall@QGroupBox@@UAEHW4Call@QMetaObject@@HPAPAX@Z 10013f1c f   Qt5Widgets:Qt5Widgets.dll
 0001:00012f22       ?qt_metacall@QLabel@@UAEHW4Call@QMetaObject@@HPAPAX@Z 10013f22 f   Qt5Widgets:Qt5Widgets.dll
 0001:00012f28       ?qt_metacall@QLineEdit@@UAEHW4Call@QMetaObject@@HPAPAX@Z 10013f28 f   Qt5Widgets:Qt5Widgets.dll
 0001:00012f2e       ?qt_metacall@QRadioButton@@UAEHW4Call@QMetaObject@@HPAPAX@Z 10013f2e f   Qt5Widgets:Qt5Widgets.dll
 0001:00012f34       ?qt_metacall@QToolButton@@UAEHW4Call@QMetaObject@@HPAPAX@Z 10013f34 f   Qt5Widgets:Qt5Widgets.dll
 0001:00012f3a       ?qt_metacall@QVBoxLayout@@UAEHW4Call@QMetaObject@@HPAPAX@Z 10013f3a f   Qt5Widgets:Qt5Widgets.dll
 0001:00012f40       ?qt_metacast@QCheckBox@@UAEPAXPBD@Z 10013f40 f   Qt5Widgets:Qt5Widgets.dll
 0001:00012f46       ?qt_metacast@QDialogButtonBox@@UAEPAXPBD@Z 10013f46 f   Qt5Widgets:Qt5Widgets.dll
 0001:00012f4c       ?qt_metacast@QGridLayout@@UAEPAXPBD@Z 10013f4c f   Qt5Widgets:Qt5Widgets.dll
 0001:00012f52       ?qt_metacast@QGroupBox@@UAEPAXPBD@Z 10013f52 f   Qt5Widgets:Qt5Widgets.dll
 0001:00012f58       ?qt_metacast@QLabel@@UAEPAXPBD@Z 10013f58 f   Qt5Widgets:Qt5Widgets.dll
 0001:00012f5e       ?qt_metacast@QLineEdit@@UAEPAXPBD@Z 10013f5e f   Qt5Widgets:Qt5Widgets.dll
 0001:00012f64       ?qt_metacast@QRadioButton@@UAEPAXPBD@Z 10013f64 f   Qt5Widgets:Qt5Widgets.dll
 0001:00012f6a       ?qt_metacast@QToolButton@@UAEPAXPBD@Z 10013f6a f   Qt5Widgets:Qt5Widgets.dll
 0001:00012f70       ?qt_metacast@QVBoxLayout@@UAEPAXPBD@Z 10013f70 f   Qt5Widgets:Qt5Widgets.dll
 0001:00012f76       ?redirected@QWidget@@MBEPAVQPaintDevice@@PAVQPoint@@@Z 10013f76 f   Qt5Widgets:Qt5Widgets.dll
 0001:00012f7c       ?reject@QDialog@@UAEXXZ    10013f7c f   Qt5Widgets:Qt5Widgets.dll
 0001:00012f82       ?resizeEvent@QDialog@@MAEXPAVQResizeEvent@@@Z 10013f82 f   Qt5Widgets:Qt5Widgets.dll
 0001:00012f88       ?resizeEvent@QGroupBox@@MAEXPAVQResizeEvent@@@Z 10013f88 f   Qt5Widgets:Qt5Widgets.dll
 0001:00012f8e       ?resizeEvent@QWidget@@MAEXPAVQResizeEvent@@@Z 10013f8e f   Qt5Widgets:Qt5Widgets.dll
 0001:00012f94       ?setGeometry@QBoxLayout@@UAEXABVQRect@@@Z 10013f94 f   Qt5Widgets:Qt5Widgets.dll
 0001:00012f9a       ?setGeometry@QGridLayout@@UAEXABVQRect@@@Z 10013f9a f   Qt5Widgets:Qt5Widgets.dll
 0001:00012fa0       ?setVisible@QDialog@@UAEX_N@Z 10013fa0 f   Qt5Widgets:Qt5Widgets.dll
 0001:00012fa6       ?setVisible@QWidget@@UAEX_N@Z 10013fa6 f   Qt5Widgets:Qt5Widgets.dll
 0001:00012fac       ?sharedPainter@QWidget@@MBEPAVQPainter@@XZ 10013fac f   Qt5Widgets:Qt5Widgets.dll
 0001:00012fb2       ?showEvent@QDialog@@MAEXPAVQShowEvent@@@Z 10013fb2 f   Qt5Widgets:Qt5Widgets.dll
 0001:00012fb8       ?showEvent@QWidget@@MAEXPAVQShowEvent@@@Z 10013fb8 f   Qt5Widgets:Qt5Widgets.dll
 0001:00012fbe       ?sizeHint@QBoxLayout@@UBE?AVQSize@@XZ 10013fbe f   Qt5Widgets:Qt5Widgets.dll
 0001:00012fc4       ?sizeHint@QCheckBox@@UBE?AVQSize@@XZ 10013fc4 f   Qt5Widgets:Qt5Widgets.dll
 0001:00012fca       ?sizeHint@QDialog@@UBE?AVQSize@@XZ 10013fca f   Qt5Widgets:Qt5Widgets.dll
 0001:00012fd0       ?sizeHint@QGridLayout@@UBE?AVQSize@@XZ 10013fd0 f   Qt5Widgets:Qt5Widgets.dll
 0001:00012fd6       ?sizeHint@QLabel@@UBE?AVQSize@@XZ 10013fd6 f   Qt5Widgets:Qt5Widgets.dll
 0001:00012fdc       ?sizeHint@QLineEdit@@UBE?AVQSize@@XZ 10013fdc f   Qt5Widgets:Qt5Widgets.dll
 0001:00012fe2       ?sizeHint@QRadioButton@@UBE?AVQSize@@XZ 10013fe2 f   Qt5Widgets:Qt5Widgets.dll
 0001:00012fe8       ?sizeHint@QToolButton@@UBE?AVQSize@@XZ 10013fe8 f   Qt5Widgets:Qt5Widgets.dll
 0001:00012fee       ?sizeHint@QWidget@@UBE?AVQSize@@XZ 10013fee f   Qt5Widgets:Qt5Widgets.dll
 0001:00012ff4       ?spacerItem@QLayoutItem@@UAEPAVQSpacerItem@@XZ 10013ff4 f   Qt5Widgets:Qt5Widgets.dll
 0001:00012ffa       ?tabletEvent@QWidget@@MAEXPAVQTabletEvent@@@Z 10013ffa f   Qt5Widgets:Qt5Widgets.dll
 0001:00013000       ?takeAt@QBoxLayout@@UAEPAVQLayoutItem@@H@Z 10014000 f   Qt5Widgets:Qt5Widgets.dll
 0001:00013006       ?takeAt@QGridLayout@@UAEPAVQLayoutItem@@H@Z 10014006 f   Qt5Widgets:Qt5Widgets.dll
 0001:0001300c       ?timerEvent@QAbstractButton@@MAEXPAVQTimerEvent@@@Z 1001400c f   Qt5Widgets:Qt5Widgets.dll
 0001:00013012       ?timerEvent@QToolButton@@MAEXPAVQTimerEvent@@@Z 10014012 f   Qt5Widgets:Qt5Widgets.dll
 0001:00013018       ?wheelEvent@QWidget@@MAEXPAVQWheelEvent@@@Z 10014018 f   Qt5Widgets:Qt5Widgets.dll
 0001:0001301e       ?widget@QLayoutItem@@UAEPAVQWidget@@XZ 1001401e f   Qt5Widgets:Qt5Widgets.dll
 0001:00013024       ?addAction@QWidget@@QAEXPAVQAction@@@Z 10014024 f   Qt5Widgets:Qt5Widgets.dll
 0001:0001302a       ??1QAction@@UAE@XZ         1001402a f   Qt5Widgets:Qt5Widgets.dll
 0001:00013030       ?event@QAction@@MAE_NPAVQEvent@@@Z 10014030 f   Qt5Widgets:Qt5Widgets.dll
 0001:00013036       ?setEnabled@QWidget@@QAEX_N@Z 10014036 f   Qt5Widgets:Qt5Widgets.dll
 0001:0001303c       ?setTabOrder@QWidget@@SAXPAV1@0@Z 1001403c f   Qt5Widgets:Qt5Widgets.dll
 0001:00013042       ??0QSpacerItem@@QAE@HHW4Policy@QSizePolicy@@0@Z 10014042 f   Qt5Widgets:Qt5Widgets.dll
 0001:00013048       ??1QSpacerItem@@UAE@XZ     10014048 f   Qt5Widgets:Qt5Widgets.dll
 0001:0001304e       ?addLayout@QBoxLayout@@QAEXPAVQLayout@@H@Z 1001404e f   Qt5Widgets:Qt5Widgets.dll
 0001:00013054       ?setStretch@QBoxLayout@@QAEXHH@Z 10014054 f   Qt5Widgets:Qt5Widgets.dll
 0001:0001305a       ??0QHBoxLayout@@QAE@XZ     1001405a f   Qt5Widgets:Qt5Widgets.dll
 0001:00013060       ??1QHBoxLayout@@UAE@XZ     10014060 f   Qt5Widgets:Qt5Widgets.dll
 0001:00013066       ??0QComboBox@@QAE@PAVQWidget@@@Z 10014066 f   Qt5Widgets:Qt5Widgets.dll
 0001:0001306c       ??1QComboBox@@UAE@XZ       1001406c f   Qt5Widgets:Qt5Widgets.dll
 0001:00013072       ?count@QComboBox@@QBEHXZ   10014072 f   Qt5Widgets:Qt5Widgets.dll
 0001:00013078       ?currentData@QComboBox@@QBE?AVQVariant@@H@Z 10014078 f   Qt5Widgets:Qt5Widgets.dll
 0001:0001307e       ?insertItem@QComboBox@@QAEXHABVQIcon@@ABVQString@@ABVQVariant@@@Z 1001407e f   Qt5Widgets:Qt5Widgets.dll
 0001:00013084       ?changeEvent@QComboBox@@MAEXPAVQEvent@@@Z 10014084 f   Qt5Widgets:Qt5Widgets.dll
 0001:0001308a       ?contextMenuEvent@QComboBox@@MAEXPAVQContextMenuEvent@@@Z 1001408a f   Qt5Widgets:Qt5Widgets.dll
 0001:00013090       ?controlTypes@QLayoutItem@@UBE?AV?$QFlags@W4ControlType@QSizePolicy@@@@XZ 10014090 f   Qt5Widgets:Qt5Widgets.dll
 0001:00013096       ?event@QComboBox@@UAE_NPAVQEvent@@@Z 10014096 f   Qt5Widgets:Qt5Widgets.dll
 0001:0001309c       ?expandingDirections@QSpacerItem@@UBE?AV?$QFlags@W4Orientation@Qt@@@@XZ 1001409c f   Qt5Widgets:Qt5Widgets.dll
 0001:000130a2       ?focusInEvent@QComboBox@@MAEXPAVQFocusEvent@@@Z 100140a2 f   Qt5Widgets:Qt5Widgets.dll
 0001:000130a8       ?focusOutEvent@QComboBox@@MAEXPAVQFocusEvent@@@Z 100140a8 f   Qt5Widgets:Qt5Widgets.dll
 0001:000130ae       ?geometry@QSpacerItem@@UBE?AVQRect@@XZ 100140ae f   Qt5Widgets:Qt5Widgets.dll
 0001:000130b4       ?hasHeightForWidth@QLayoutItem@@UBE_NXZ 100140b4 f   Qt5Widgets:Qt5Widgets.dll
 0001:000130ba       ?heightForWidth@QLayoutItem@@UBEHH@Z 100140ba f   Qt5Widgets:Qt5Widgets.dll
 0001:000130c0       ?hideEvent@QComboBox@@MAEXPAVQHideEvent@@@Z 100140c0 f   Qt5Widgets:Qt5Widgets.dll
 0001:000130c6       ?hidePopup@QComboBox@@UAEXXZ 100140c6 f   Qt5Widgets:Qt5Widgets.dll
 0001:000130cc       ?inputMethodEvent@QComboBox@@MAEXPAVQInputMethodEvent@@@Z 100140cc f   Qt5Widgets:Qt5Widgets.dll
 0001:000130d2       ?inputMethodQuery@QComboBox@@UBE?AVQVariant@@W4InputMethodQuery@Qt@@@Z 100140d2 f   Qt5Widgets:Qt5Widgets.dll
 0001:000130d8       ?invalidate@QLayoutItem@@UAEXXZ 100140d8 f   Qt5Widgets:Qt5Widgets.dll
 0001:000130de       ?isEmpty@QSpacerItem@@UBE_NXZ 100140de f   Qt5Widgets:Qt5Widgets.dll
 0001:000130e4       ?keyPressEvent@QComboBox@@MAEXPAVQKeyEvent@@@Z 100140e4 f   Qt5Widgets:Qt5Widgets.dll
 0001:000130ea       ?keyReleaseEvent@QComboBox@@MAEXPAVQKeyEvent@@@Z 100140ea f   Qt5Widgets:Qt5Widgets.dll
 0001:000130f0       ?layout@QLayoutItem@@UAEPAVQLayout@@XZ 100140f0 f   Qt5Widgets:Qt5Widgets.dll
 0001:000130f6       ?maximumSize@QSpacerItem@@UBE?AVQSize@@XZ 100140f6 f   Qt5Widgets:Qt5Widgets.dll
 0001:000130fc       ?metaObject@QComboBox@@UBEPBUQMetaObject@@XZ 100140fc f   Qt5Widgets:Qt5Widgets.dll
 0001:00013102       ?metaObject@QHBoxLayout@@UBEPBUQMetaObject@@XZ 10014102 f   Qt5Widgets:Qt5Widgets.dll
 0001:00013108       ?minimumHeightForWidth@QLayoutItem@@UBEHH@Z 10014108 f   Qt5Widgets:Qt5Widgets.dll
 0001:0001310e       ?minimumSize@QSpacerItem@@UBE?AVQSize@@XZ 1001410e f   Qt5Widgets:Qt5Widgets.dll
 0001:00013114       ?minimumSizeHint@QComboBox@@UBE?AVQSize@@XZ 10014114 f   Qt5Widgets:Qt5Widgets.dll
 0001:0001311a       ?mousePressEvent@QComboBox@@MAEXPAVQMouseEvent@@@Z 1001411a f   Qt5Widgets:Qt5Widgets.dll
 0001:00013120       ?mouseReleaseEvent@QComboBox@@MAEXPAVQMouseEvent@@@Z 10014120 f   Qt5Widgets:Qt5Widgets.dll
 0001:00013126       ?paintEvent@QComboBox@@MAEXPAVQPaintEvent@@@Z 10014126 f   Qt5Widgets:Qt5Widgets.dll
 0001:0001312c       ?qt_metacall@QComboBox@@UAEHW4Call@QMetaObject@@HPAPAX@Z 1001412c f   Qt5Widgets:Qt5Widgets.dll
 0001:00013132       ?qt_metacall@QHBoxLayout@@UAEHW4Call@QMetaObject@@HPAPAX@Z 10014132 f   Qt5Widgets:Qt5Widgets.dll
 0001:00013138       ?qt_metacast@QComboBox@@UAEPAXPBD@Z 10014138 f   Qt5Widgets:Qt5Widgets.dll
 0001:0001313e       ?qt_metacast@QHBoxLayout@@UAEPAXPBD@Z 1001413e f   Qt5Widgets:Qt5Widgets.dll
 0001:00013144       ?resizeEvent@QComboBox@@MAEXPAVQResizeEvent@@@Z 10014144 f   Qt5Widgets:Qt5Widgets.dll
 0001:0001314a       ?setGeometry@QSpacerItem@@UAEXABVQRect@@@Z 1001414a f   Qt5Widgets:Qt5Widgets.dll
 0001:00013150       ?showEvent@QComboBox@@MAEXPAVQShowEvent@@@Z 10014150 f   Qt5Widgets:Qt5Widgets.dll
 0001:00013156       ?showPopup@QComboBox@@UAEXXZ 10014156 f   Qt5Widgets:Qt5Widgets.dll
 0001:0001315c       ?sizeHint@QComboBox@@UBE?AVQSize@@XZ 1001415c f   Qt5Widgets:Qt5Widgets.dll
 0001:00013162       ?sizeHint@QSpacerItem@@UBE?AVQSize@@XZ 10014162 f   Qt5Widgets:Qt5Widgets.dll
 0001:00013168       ?spacerItem@QSpacerItem@@UAEPAV1@XZ 10014168 f   Qt5Widgets:Qt5Widgets.dll
 0001:0001316e       ?wheelEvent@QComboBox@@MAEXPAVQWheelEvent@@@Z 1001416e f   Qt5Widgets:Qt5Widgets.dll
 0001:00013174       ?qt_metacast@QDialog@@UAEPAXPBD@Z 10014174 f   Qt5Widgets:Qt5Widgets.dll
 0001:0001317a       ?qt_metacall@QDialog@@UAEHW4Call@QMetaObject@@HPAPAX@Z 1001417a f   Qt5Widgets:Qt5Widgets.dll
 0001:00013180       ??0QIcon@@QAE@ABVQString@@@Z 10014180 f   Qt5Gui:Qt5Gui.dll
 0001:00013186       ??1QIcon@@QAE@XZ           10014186 f   Qt5Gui:Qt5Gui.dll
 0001:0001318c       ??0QIcon@@QAE@XZ           1001418c f   Qt5Gui:Qt5Gui.dll
 0001:00013192       ?qBadAlloc@@YAXXZ          10014192 f   Qt5Core:Qt5Core.dll
 0001:00013198       ??0QChar@@QAE@UQLatin1Char@@@Z 10014198 f   Qt5Core:Qt5Core.dll
 0001:0001319e       ?data@QArrayData@@QAEPAXXZ 1001419e f   Qt5Core:Qt5Core.dll
 0001:000131a4       ?allocate@QArrayData@@SAPAU1@IIIV?$QFlags@W4AllocationOption@QArrayData@@@@@Z 100141a4 f   Qt5Core:Qt5Core.dll
 0001:000131aa       ?deallocate@QArrayData@@SAXPAU1@II@Z 100141aa f   Qt5Core:Qt5Core.dll
 0001:000131b0       ??1QByteArray@@QAE@XZ      100141b0 f   Qt5Core:Qt5Core.dll
 0001:000131b6       ??AQByteArray@@QAE?AVQByteRef@@H@Z 100141b6 f   Qt5Core:Qt5Core.dll
 0001:000131bc       ??BQByteRef@@QBEDXZ        100141bc f   Qt5Core:Qt5Core.dll
 0001:000131c2       ??0QString@@QAE@XZ         100141c2 f   Qt5Core:Qt5Core.dll
 0001:000131c8       ??0QString@@QAE@VQChar@@@Z 100141c8 f   Qt5Core:Qt5Core.dll
 0001:000131ce       ??0QString@@QAE@ABV0@@Z    100141ce f   Qt5Core:Qt5Core.dll
 0001:000131d4       ??1QString@@QAE@XZ         100141d4 f   Qt5Core:Qt5Core.dll
 0001:000131da       ??4QString@@QAEAAV0@ABV0@@Z 100141da f   Qt5Core:Qt5Core.dll
 0001:000131e0       ??0QString@@QAE@$$QAV0@@Z  100141e0 f   Qt5Core:Qt5Core.dll
 0001:000131e6       ??4QString@@QAEAAV0@$$QAV0@@Z 100141e6 f   Qt5Core:Qt5Core.dll
 0001:000131ec       ?clear@QString@@QAEXXZ     100141ec f   Qt5Core:Qt5Core.dll
 0001:000131f2       ?arg@QString@@QBE?AV1@ABV1@HVQChar@@@Z 100141f2 f   Qt5Core:Qt5Core.dll
 0001:000131f8       ?toUpper@QString@@QBE?AV1@XZ 100141f8 f   Qt5Core:Qt5Core.dll
 0001:000131fe       ?append@QString@@QAEAAV1@ABV1@@Z 100141fe f   Qt5Core:Qt5Core.dll
 0001:00013204       ?toLocal8Bit@QString@@QBE?AVQByteArray@@XZ 10014204 f   Qt5Core:Qt5Core.dll
 0001:0001320a       ?fromUtf8@QString@@SA?AV1@PBDH@Z 1001420a f   Qt5Core:Qt5Core.dll
 0001:00013210       ?number@QString@@SA?AV1@HH@Z 10014210 f   Qt5Core:Qt5Core.dll
 0001:00013216       ??8@YA_NABVQString@@0@Z    10014216 f   Qt5Core:Qt5Core.dll
 0001:0001321c       ??4QString@@QAEAAV0@PBD@Z  1001421c f   Qt5Core:Qt5Core.dll
 0001:00013222       ??YQString@@QAEAAV0@PBD@Z  10014222 f   Qt5Core:Qt5Core.dll
 0001:00013228       ?fromAscii_helper@QString@@CAPAU?$QTypedArrayData@G@@PBDH@Z 10014228 f   Qt5Core:Qt5Core.dll
 0001:0001322e       ?tr@QMetaObject@@QBE?AVQString@@PBD0H@Z 1001422e f   Qt5Core:Qt5Core.dll
 0001:00013234       ?connectSlotsByName@QMetaObject@@SAXPAVQObject@@@Z 10014234 f   Qt5Core:Qt5Core.dll
 0001:0001323a       ??1Connection@QMetaObject@@QAE@XZ 1001423a f   Qt5Core:Qt5Core.dll
 0001:00013240       ?detach_grow@QListData@@QAEPAUData@1@PAHH@Z 10014240 f   Qt5Core:Qt5Core.dll
 0001:00013246       ?dispose@QListData@@SAXPAUData@1@@Z 10014246 f   Qt5Core:Qt5Core.dll
 0001:0001324c       ?append@QListData@@QAEPAPAXXZ 1001424c f   Qt5Core:Qt5Core.dll
 0001:00013252       ?objectName@QObject@@QBE?AVQString@@XZ 10014252 f   Qt5Core:Qt5Core.dll
 0001:00013258       ?setObjectName@QObject@@QAEXABVQString@@@Z 10014258 f   Qt5Core:Qt5Core.dll
 0001:0001325e       ?connect@QObject@@SA?AVConnection@QMetaObject@@PBV1@PBD01W4ConnectionType@Qt@@@Z 1001425e f   Qt5Core:Qt5Core.dll
 0001:00013264       ?connect@QObject@@QBE?AVConnection@QMetaObject@@PBV1@PBD1W4ConnectionType@Qt@@@Z 10014264 f   Qt5Core:Qt5Core.dll
 0001:0001326a       ?write@QIODevice@@QAE_JABVQByteArray@@@Z 1001426a f   Qt5Core:Qt5Core.dll
 0001:00013270       ??0QFile@@QAE@ABVQString@@@Z 10014270 f   Qt5Core:Qt5Core.dll
 0001:00013276       ??1QFile@@UAE@XZ           10014276 f   Qt5Core:Qt5Core.dll
 0001:0001327c       ?allocateNode@QHashData@@QAEPAXH@Z 1001427c f   Qt5Core:Qt5Core.dll
 0001:00013282       ?freeNode@QHashData@@QAEXPAX@Z 10014282 f   Qt5Core:Qt5Core.dll
 0001:00013288       ?detach_helper@QHashData@@QAEPAU1@P6AXPAUNode@1@PAX@ZP6AX0@ZHH@Z 10014288 f   Qt5Core:Qt5Core.dll
 0001:0001328e       ?hasShrunk@QHashData@@QAEXXZ 1001428e f   Qt5Core:Qt5Core.dll
 0001:00013294       ?rehash@QHashData@@QAEXH@Z 10014294 f   Qt5Core:Qt5Core.dll
 0001:0001329a       ?free_helper@QHashData@@QAEXP6AXPAUNode@1@@Z@Z 1001429a f   Qt5Core:Qt5Core.dll
 0001:000132a0       ?toNativeSeparators@QDir@@SA?AVQString@@ABV2@@Z 100142a0 f   Qt5Core:Qt5Core.dll
 0001:000132a6       ?translate@QCoreApplication@@SA?AVQString@@PBD00H@Z 100142a6 f   Qt5Core:Qt5Core.dll
 0001:000132ac       ?atEnd@QFileDevice@@UBE_NXZ 100142ac f   Qt5Core:Qt5Core.dll
 0001:000132b2       ?bytesAvailable@QIODevice@@UBE_JXZ 100142b2 f   Qt5Core:Qt5Core.dll
 0001:000132b8       ?bytesToWrite@QIODevice@@UBE_JXZ 100142b8 f   Qt5Core:Qt5Core.dll
 0001:000132be       ?canReadLine@QIODevice@@UBE_NXZ 100142be f   Qt5Core:Qt5Core.dll
 0001:000132c4       ?childEvent@QObject@@MAEXPAVQChildEvent@@@Z 100142c4 f   Qt5Core:Qt5Core.dll
 0001:000132ca       ?close@QFileDevice@@UAEXXZ 100142ca f   Qt5Core:Qt5Core.dll
 0001:000132d0       ?connectNotify@QObject@@MAEXABVQMetaMethod@@@Z 100142d0 f   Qt5Core:Qt5Core.dll
 0001:000132d6       ?customEvent@QObject@@MAEXPAVQEvent@@@Z 100142d6 f   Qt5Core:Qt5Core.dll
 0001:000132dc       ?disconnectNotify@QObject@@MAEXABVQMetaMethod@@@Z 100142dc f   Qt5Core:Qt5Core.dll
 0001:000132e2       ?event@QObject@@UAE_NPAVQEvent@@@Z 100142e2 f   Qt5Core:Qt5Core.dll
 0001:000132e8       ?eventFilter@QObject@@UAE_NPAV1@PAVQEvent@@@Z 100142e8 f   Qt5Core:Qt5Core.dll
 0001:000132ee       ?fileName@QFile@@UBE?AVQString@@XZ 100142ee f   Qt5Core:Qt5Core.dll
 0001:000132f4       ?isSequential@QFileDevice@@UBE_NXZ 100142f4 f   Qt5Core:Qt5Core.dll
 0001:000132fa       ?metaObject@QFile@@UBEPBUQMetaObject@@XZ 100142fa f   Qt5Core:Qt5Core.dll
 0001:00013300       ?open@QFile@@UAE_NV?$QFlags@W4OpenModeFlag@QIODevice@@@@@Z 10014300 f   Qt5Core:Qt5Core.dll
 0001:00013306       ?permissions@QFile@@UBE?AV?$QFlags@W4Permission@QFileDevice@@@@XZ 10014306 f   Qt5Core:Qt5Core.dll
 0001:0001330c       ?pos@QFileDevice@@UBE_JXZ  1001430c f   Qt5Core:Qt5Core.dll
 0001:00013312       ?qt_metacall@QFile@@UAEHW4Call@QMetaObject@@HPAPAX@Z 10014312 f   Qt5Core:Qt5Core.dll
 0001:00013318       ?qt_metacast@QFile@@UAEPAXPBD@Z 10014318 f   Qt5Core:Qt5Core.dll
 0001:0001331e       ?readData@QFileDevice@@MAE_JPAD_J@Z 1001431e f   Qt5Core:Qt5Core.dll
 0001:00013324       ?readLineData@QFileDevice@@MAE_JPAD_J@Z 10014324 f   Qt5Core:Qt5Core.dll
 0001:0001332a       ?reset@QIODevice@@UAE_NXZ  1001432a f   Qt5Core:Qt5Core.dll
 0001:00013330       ?resize@QFile@@UAE_N_J@Z   10014330 f   Qt5Core:Qt5Core.dll
 0001:00013336       ?seek@QFileDevice@@UAE_N_J@Z 10014336 f   Qt5Core:Qt5Core.dll
 0001:0001333c       ?setPermissions@QFile@@UAE_NV?$QFlags@W4Permission@QFileDevice@@@@@Z 1001433c f   Qt5Core:Qt5Core.dll
 0001:00013342       ?size@QFile@@UBE_JXZ       10014342 f   Qt5Core:Qt5Core.dll
 0001:00013348       ?timerEvent@QObject@@MAEXPAVQTimerEvent@@@Z 10014348 f   Qt5Core:Qt5Core.dll
 0001:0001334e       ?waitForBytesWritten@QIODevice@@UAE_NH@Z 1001434e f   Qt5Core:Qt5Core.dll
 0001:00013354       ?waitForReadyRead@QIODevice@@UAE_NH@Z 10014354 f   Qt5Core:Qt5Core.dll
 0001:0001335a       ?writeData@QFileDevice@@MAE_JPBD_J@Z 1001435a f   Qt5Core:Qt5Core.dll
 0001:00013360       ?arg@QString@@QBE?AV1@HHHVQChar@@@Z 10014360 f   Qt5Core:Qt5Core.dll
 0001:00013366       ?cast@QMetaObject@@QBEPAVQObject@@PAV2@@Z 10014366 f   Qt5Core:Qt5Core.dll
 0001:0001336c       ?detach@QListData@@QAEPAUData@1@H@Z 1001436c f   Qt5Core:Qt5Core.dll
 0001:00013372       ?sender@QObject@@IBEPAV1@XZ 10014372 f   Qt5Core:Qt5Core.dll
 0001:00013378       ?getAndRef@ExternalRefCountData@QtSharedPointer@@SAPAU12@PBVQObject@@@Z 10014378 f   Qt5Core:Qt5Core.dll
 0001:0001337e       ??0QByteArray@@QAE@ABV0@@Z 1001437e f   Qt5Core:Qt5Core.dll
 0001:00013384       ?arg@QString@@QBE?AV1@_JHHVQChar@@@Z 10014384 f   Qt5Core:Qt5Core.dll
 0001:0001338a       ?arg@QString@@QBE?AV1@NHDHVQChar@@@Z 1001438a f   Qt5Core:Qt5Core.dll
 0001:00013390       ?arg@QString@@QBE?AV1@DHVQChar@@@Z 10014390 f   Qt5Core:Qt5Core.dll
 0001:00013396       ?number@QString@@SA?AV1@_JH@Z 10014396 f   Qt5Core:Qt5Core.dll
 0001:0001339c       ?number@QString@@SA?AV1@NDH@Z 1001439c f   Qt5Core:Qt5Core.dll
 0001:000133a2       ??0QString@@QAE@ABVQByteArray@@@Z 100143a2 f   Qt5Core:Qt5Core.dll
 0001:000133a8       ?nextNode@QMapNodeBase@@QBEPBU1@XZ 100143a8 f   Qt5Core:Qt5Core.dll
 0001:000133ae       ?freeNodeAndRebalance@QMapDataBase@@QAEXPAUQMapNodeBase@@@Z 100143ae f   Qt5Core:Qt5Core.dll
 0001:000133b4       ?recalcMostLeftNode@QMapDataBase@@QAEXXZ 100143b4 f   Qt5Core:Qt5Core.dll
 0001:000133ba       ?createNode@QMapDataBase@@QAEPAUQMapNodeBase@@HHPAU2@_N@Z 100143ba f   Qt5Core:Qt5Core.dll
 0001:000133c0       ?freeTree@QMapDataBase@@QAEXPAUQMapNodeBase@@H@Z 100143c0 f   Qt5Core:Qt5Core.dll
 0001:000133c6       ?createData@QMapDataBase@@SAPAU1@XZ 100143c6 f   Qt5Core:Qt5Core.dll
 0001:000133cc       ?freeData@QMapDataBase@@SAXPAU1@@Z 100143cc f   Qt5Core:Qt5Core.dll
 0001:000133d2       ?qrand@@YAHXZ              100143d2 f   Qt5Core:Qt5Core.dll
 0001:000133d8       ?data@QArrayData@@QBEPBXXZ 100143d8 f   Qt5Core:Qt5Core.dll
 0001:000133de       ??1QDateTime@@QAE@XZ       100143de f   Qt5Core:Qt5Core.dll
 0001:000133e4       ?toTime_t@QDateTime@@QBEIXZ 100143e4 f   Qt5Core:Qt5Core.dll
 0001:000133ea       ?currentDateTime@QDateTime@@SA?AV1@XZ 100143ea f   Qt5Core:Qt5Core.dll
 0001:000133f0       ??1QVariant@@QAE@XZ        100143f0 f   Qt5Core:Qt5Core.dll
 0001:000133f6       ??0QVariant@@QAE@ABVQString@@@Z 100143f6 f   Qt5Core:Qt5Core.dll
 0001:000133fc       ?toString@QVariant@@QBE?AVQString@@XZ 100143fc f   Qt5Core:Qt5Core.dll
 0001:00013402       ?dynamicMetaObject@QObjectData@@QBEPAUQMetaObject@@XZ 10014402 f   Qt5Core:Qt5Core.dll
 0001:00013408       ??0QByteArray@@QAE@XZ      10014408 f   Qt5Core:Qt5Core.dll
 0001:0001340e       ?reserve@QByteArray@@QAEXH@Z 1001440e f   Qt5Core:Qt5Core.dll
 0001:00013414       ?append@QByteArray@@QAEAAV1@D@Z 10014414 f   Qt5Core:Qt5Core.dll
 0001:0001341a       ?append@QByteArray@@QAEAAV1@PBD@Z 1001441a f   Qt5Core:Qt5Core.dll
 0001:00013420       ?className@QMetaObject@@QBEPBDXZ 10014420 f   Qt5Core:Qt5Core.dll
 0001:00013426       ?registerNormalizedType@QMetaType@@SAHABVQByteArray@@P6AXPAX@ZP6APAXPBX@Z2P6APAX13@ZHV?$QFlags@W4TypeFlag@QMetaType@@@@PBUQMetaObject@@@Z 10014426 f   Qt5Core:Qt5Core.dll
 0001:0001342c       ?registerNormalizedTypedef@QMetaType@@SAHABVQByteArray@@H@Z 1001442c f   Qt5Core:Qt5Core.dll
 0001:00013432       ?_Xbad_alloc@std@@YAXXZ    10014432 f   msvcprt:MSVCP120.dll
 0001:00013438       ?_Xlength_error@std@@YAXPBD@Z 10014438 f   msvcprt:MSVCP120.dll
 0001:0001343e       ?_Xout_of_range@std@@YAXPBD@Z 1001443e f   msvcprt:MSVCP120.dll
 0001:00013444       ?_Syserror_map@std@@YAPBDH@Z 10014444 f   msvcprt:MSVCP120.dll
 0001:0001344a       ?_Winerror_map@std@@YAPBDH@Z 1001444a f   msvcprt:MSVCP120.dll
 0001:00013450       ??_M@YGXPAXIHP6EX0@Z@Z     10014450 f   MSVCRT:ehvecdtr.obj
 0001:000134d8       ?__ArrayUnwind@@YGXPAXIHP6EX0@Z@Z 100144d8 f   MSVCRT:ehvecdtr.obj
 0001:00013536       __purecall                 10014536 f   MSVCRT:MSVCR120.dll
 0001:0001353c       ??2@YAPAXI@Z               1001453c f   MSVCRT:MSVCR120.dll
 0001:00013542       ??3@YAXPAX@Z               10014542 f   MSVCRT:MSVCR120.dll
 0001:00013548       ___atonexitinit            10014548 f   MSVCRT:atonexit.obj
 0001:00013584       __onexit                   10014584 f   MSVCRT:atonexit.obj
 0001:0001362d       _atexit                    1001462d f   MSVCRT:atonexit.obj
 0001:00013642       _memmove                   10014642 f   MSVCRT:MSVCR120.dll
 0001:00013648       __hypot                    10014648 f   MSVCRT:MSVCR120.dll
 0001:0001364e       @__security_check_cookie@4 1001464e f   MSVCRT:secchk.obj
 0001:0001365e       __CxxThrowException@8      1001465e f   MSVCRT:MSVCR120.dll
 0001:00013664       ___CxxFrameHandler3        10014664 f   MSVCRT:MSVCR120.dll
 0001:0001366a       _memcpy                    1001466a f   MSVCRT:MSVCR120.dll
 0001:00013670       _memset                    10014670 f   MSVCRT:MSVCR120.dll
 0001:00013676       ??0type_info@@AAE@ABV0@@Z  10014676 f   MSVCRT:ti_inst.obj
 0001:00013681       ??4type_info@@AAEAAV0@ABV0@@Z 10014681 f   MSVCRT:ti_inst.obj
 0001:00013686       ??_Etype_info@@UAEPAXI@Z   10014686 f i MSVCRT:ti_inst.obj
 0001:000136d0       __ftoui3                   100146d0 f   MSVCRT:ftol3.obj
 0001:000136df       __ftoul3                   100146df f   MSVCRT:ftol3.obj
 0001:000136ee       __ftol3                    100146ee f   MSVCRT:ftol3.obj
 0001:000136fb       __ftol3_NaN                100146fb f   MSVCRT:ftol3.obj
 0001:00013713       __ftol3_work               10014713 f   MSVCRT:ftol3.obj
 0001:00013799       __ftol3_common             10014799 f   MSVCRT:ftol3.obj
 0001:0001385b       __ftol3_arg_error          1001485b f   MSVCRT:ftol3.obj
 0001:0001386d       __ftol3_except             1001486d f   MSVCRT:ftol3.obj
 0001:000138b1       __dtoui3                   100148b1 f   MSVCRT:ftol3.obj
 0001:000138c0       __dtoul3                   100148c0 f   MSVCRT:ftol3.obj
 0001:000138cf       __dtol3                    100148cf f   MSVCRT:ftol3.obj
 0001:000138dc       __dtol3_NaN                100148dc f   MSVCRT:ftol3.obj
 0001:000138f9       __dtol3_work               100148f9 f   MSVCRT:ftol3.obj
 0001:000139de       __ultod3                   100149de f   MSVCRT:ftol3.obj
 0001:00013a6f       __ltod3                    10014a6f f   MSVCRT:ftol3.obj
 0001:00013a9e       _srand                     10014a9e f   MSVCRT:MSVCR120.dll
 0001:00013ab0       __allrem                   10014ab0 f   MSVCRT:llrem.obj
 0001:00013bae       _NtCurrentTeb              10014bae f i MSVCRT:crtdll.obj
 0001:00013bb5       __CRT_INIT@12              10014bb5 f   MSVCRT:crtdll.obj
 0001:00013dac       __DllMainCRTStartup@12     10014dac f   MSVCRT:crtdll.obj
 0001:00013f02       ?terminate@@YAXXZ          10014f02 f   MSVCRT:MSVCR120.dll
 0001:00013f10       __SEH_prolog4              10014f10 f   MSVCRT:sehprolg4.obj
 0001:00013f55       __SEH_epilog4              10014f55 f   MSVCRT:sehprolg4.obj
 0001:00013f69       __except_handler4          10014f69 f   MSVCRT:chandler4gs.obj
 0001:00013f8c       __lock                     10014f8c f   MSVCRT:MSVCR120.dll
 0001:00013f92       __unlock                   10014f92 f   MSVCRT:MSVCR120.dll
 0001:00013f98       __calloc_crt               10014f98 f   MSVCRT:MSVCR120.dll
 0001:00013f9e       ___dllonexit               10014f9e f   MSVCRT:MSVCR120.dll
 0001:00013fa4       ___raise_securityfailure   10014fa4 f   MSVCRT:gs_report.obj
 0001:00013fe1       ___report_gsfailure        10014fe1 f   MSVCRT:gs_report.obj
 0001:000140dc       ___report_rangecheckfailure 100150dc f   MSVCRT:gs_report.obj
 0001:000140e8       ___report_securityfailure  100150e8 f   MSVCRT:gs_report.obj
 0001:000141b8       ___report_securityfailureEx 100151b8 f   MSVCRT:gs_report.obj
 0001:000142ce       ??1type_info@@UAE@XZ       100152ce f   MSVCRT:MSVCR120.dll
 0001:000142d4       __except1                  100152d4 f   MSVCRT:MSVCR120.dll
 0001:000142da       ___CppXcptFilter           100152da f   MSVCRT:MSVCR120.dll
 0001:000142e0       __amsg_exit                100152e0 f   MSVCRT:MSVCR120.dll
 0001:000142f0       __FindPESection            100152f0 f   MSVCRT:pesect.obj
 0001:00014340       __IsNonwritableInCurrentImage 10015340 f   MSVCRT:pesect.obj
 0001:00014400       __ValidateImageBase        10015400 f   MSVCRT:pesect.obj
 0001:00014432       _free                      10015432 f   MSVCRT:MSVCR120.dll
 0001:00014438       ___security_init_cookie    10015438 f   MSVCRT:gs_support.obj
 0001:000144d4       _DllMain@12                100154d4 f   MSVCRT:dllmain.obj
 0001:000144f6       __malloc_crt               100154f6 f   MSVCRT:MSVCR120.dll
 0001:000144fc       __RTC_Initialize           100154fc f   MSVCRT:initsect.obj
 0001:0001451c       __RTC_Terminate            1001551c f   MSVCRT:initsect.obj
 0001:0001453c       __initterm                 1001553c f   MSVCRT:MSVCR120.dll
 0001:00014542       __initterm_e               10015542 f   MSVCRT:MSVCR120.dll
 0001:00014548       ___clean_type_info_names   10015548 f   MSVCRT:tncleanup.obj
 0001:00014554       __except_handler4_common   10015554 f   MSVCRT:MSVCR120.dll
 0001:0001455a       __crt_debugger_hook        1001555a f   MSVCRT:MSVCR120.dll
 0001:00014560       ___crtUnhandledException   10015560 f   MSVCRT:MSVCR120.dll
 0001:00014566       ___crtTerminateProcess     10015566 f   MSVCRT:MSVCR120.dll
 0001:0001456c       ___clean_type_info_names_internal 1001556c f   MSVCRT:MSVCR120.dll
 0001:00014572       _EncodePointer@4           10015572 f   kernel32:KERNEL32.dll
 0001:00014578       _DecodePointer@4           10015578 f   kernel32:KERNEL32.dll
 0001:0001457e       _IsDebuggerPresent@0       1001557e f   kernel32:KERNEL32.dll
 0001:00014584       _IsProcessorFeaturePresent@4 10015584 f   kernel32:KERNEL32.dll
 0001:0001458a       _QueryPerformanceCounter@4 1001558a f   kernel32:KERNEL32.dll
 0001:00014590       _GetCurrentProcessId@0     10015590 f   kernel32:KERNEL32.dll
 0001:00014596       _GetCurrentThreadId@0      10015596 f   kernel32:KERNEL32.dll
 0001:0001459c       _GetSystemTimeAsFileTime@4 1001559c f   kernel32:KERNEL32.dll
 0001:000145a2       _DisableThreadLibraryCalls@4 100155a2 f   kernel32:KERNEL32.dll
 0002:00000000       __imp__DisableThreadLibraryCalls@4 10019000     kernel32:KERNEL32.dll
 0002:00000004       __imp__GetSystemTimeAsFileTime@4 10019004     kernel32:KERNEL32.dll
 0002:00000008       __imp__GetCurrentThreadId@0 10019008     kernel32:KERNEL32.dll
 0002:0000000c       __imp__GetCurrentProcessId@0 1001900c     kernel32:KERNEL32.dll
 0002:00000010       __imp__QueryPerformanceCounter@4 10019010     kernel32:KERNEL32.dll
 0002:00000014       __imp__IsProcessorFeaturePresent@4 10019014     kernel32:KERNEL32.dll
 0002:00000018       __imp__IsDebuggerPresent@0 10019018     kernel32:KERNEL32.dll
 0002:0000001c       __imp__DecodePointer@4     1001901c     kernel32:KERNEL32.dll
 0002:00000020       __imp__EncodePointer@4     10019020     kernel32:KERNEL32.dll
 0002:00000024       \177KERNEL32_NULL_THUNK_DATA 10019024     kernel32:KERNEL32.dll
 0002:00000028       __imp_?_Xlength_error@std@@YAXPBD@Z 10019028     msvcprt:MSVCP120.dll
 0002:0000002c       __imp_?_Xout_of_range@std@@YAXPBD@Z 1001902c     msvcprt:MSVCP120.dll
 0002:00000030       __imp_?_Syserror_map@std@@YAPBDH@Z 10019030     msvcprt:MSVCP120.dll
 0002:00000034       __imp_?_Winerror_map@std@@YAPBDH@Z 10019034     msvcprt:MSVCP120.dll
 0002:00000038       __imp_?_Xbad_alloc@std@@YAXXZ 10019038     msvcprt:MSVCP120.dll
 0002:0000003c       \177MSVCP120_NULL_THUNK_DATA 1001903c     msvcprt:MSVCP120.dll
 0002:00000040       __imp___initterm_e         10019040     MSVCRT:MSVCR120.dll
 0002:00000044       __imp___initterm           10019044     MSVCRT:MSVCR120.dll
 0002:00000048       __imp___malloc_crt         10019048     MSVCRT:MSVCR120.dll
 0002:0000004c       __imp__free                1001904c     MSVCRT:MSVCR120.dll
 0002:00000050       __imp___amsg_exit          10019050     MSVCRT:MSVCR120.dll
 0002:00000054       __imp____CppXcptFilter     10019054     MSVCRT:MSVCR120.dll
 0002:00000058       __imp___except1            10019058     MSVCRT:MSVCR120.dll
 0002:0000005c       __imp___except_handler4_common 1001905c     MSVCRT:MSVCR120.dll
 0002:00000060       __imp___onexit             10019060     MSVCRT:MSVCR120.dll
 0002:00000064       __imp____dllonexit         10019064     MSVCRT:MSVCR120.dll
 0002:00000068       __imp___calloc_crt         10019068     MSVCRT:MSVCR120.dll
 0002:0000006c       __imp___unlock             1001906c     MSVCRT:MSVCR120.dll
 0002:00000070       __imp___lock               10019070     MSVCRT:MSVCR120.dll
 0002:00000074       __imp_?terminate@@YAXXZ    10019074     MSVCRT:MSVCR120.dll
 0002:00000078       __imp__srand               10019078     MSVCRT:MSVCR120.dll
 0002:0000007c       __imp__memset              1001907c     MSVCRT:MSVCR120.dll
 0002:00000080       __imp__memcpy              10019080     MSVCRT:MSVCR120.dll
 0002:00000084       __imp____CxxFrameHandler3  10019084     MSVCRT:MSVCR120.dll
 0002:00000088       __imp___CxxThrowException@8 10019088     MSVCRT:MSVCR120.dll
 0002:0000008c       __imp___hypot              1001908c     MSVCRT:MSVCR120.dll
 0002:00000090       __imp__memmove             10019090     MSVCRT:MSVCR120.dll
 0002:00000094       __imp_??3@YAXPAX@Z         10019094     MSVCRT:MSVCR120.dll
 0002:00000098       __imp_??2@YAPAXI@Z         10019098     MSVCRT:MSVCR120.dll
 0002:0000009c       __imp___purecall           1001909c     MSVCRT:MSVCR120.dll
 0002:000000a0       __imp___crt_debugger_hook  100190a0     MSVCRT:MSVCR120.dll
 0002:000000a4       __imp____crtUnhandledException 100190a4     MSVCRT:MSVCR120.dll
 0002:000000a8       __imp____crtTerminateProcess 100190a8     MSVCRT:MSVCR120.dll
 0002:000000ac       __imp____clean_type_info_names_internal 100190ac     MSVCRT:MSVCR120.dll
 0002:000000b0       __imp_??1type_info@@UAE@XZ 100190b0     MSVCRT:MSVCR120.dll
 0002:000000b4       \177MSVCR120_NULL_THUNK_DATA 100190b4     MSVCRT:MSVCR120.dll
 0002:000000b8       __imp_?registerNormalizedTypedef@QMetaType@@SAHABVQByteArray@@H@Z 100190b8     Qt5Core:Qt5Core.dll
 0002:000000bc       __imp_?registerNormalizedType@QMetaType@@SAHABVQByteArray@@P6AXPAX@ZP6APAXPBX@Z2P6APAX13@ZHV?$QFlags@W4TypeFlag@QMetaType@@@@PBUQMetaObject@@@Z 100190bc     Qt5Core:Qt5Core.dll
 0002:000000c0       __imp_?className@QMetaObject@@QBEPBDXZ 100190c0     Qt5Core:Qt5Core.dll
 0002:000000c4       __imp_?append@QByteArray@@QAEAAV1@PBD@Z 100190c4     Qt5Core:Qt5Core.dll
 0002:000000c8       __imp_?append@QByteArray@@QAEAAV1@D@Z 100190c8     Qt5Core:Qt5Core.dll
 0002:000000cc       __imp_?reserve@QByteArray@@QAEXH@Z 100190cc     Qt5Core:Qt5Core.dll
 0002:000000d0       __imp_??0QByteArray@@QAE@XZ 100190d0     Qt5Core:Qt5Core.dll
 0002:000000d4       __imp_?dynamicMetaObject@QObjectData@@QBEPAUQMetaObject@@XZ 100190d4     Qt5Core:Qt5Core.dll
 0002:000000d8       __imp_?toString@QVariant@@QBE?AVQString@@XZ 100190d8     Qt5Core:Qt5Core.dll
 0002:000000dc       __imp_??0QVariant@@QAE@ABVQString@@@Z 100190dc     Qt5Core:Qt5Core.dll
 0002:000000e0       __imp_??1QVariant@@QAE@XZ  100190e0     Qt5Core:Qt5Core.dll
 0002:000000e4       __imp_?currentDateTime@QDateTime@@SA?AV1@XZ 100190e4     Qt5Core:Qt5Core.dll
 0002:000000e8       __imp_?toTime_t@QDateTime@@QBEIXZ 100190e8     Qt5Core:Qt5Core.dll
 0002:000000ec       __imp_??1QDateTime@@QAE@XZ 100190ec     Qt5Core:Qt5Core.dll
 0002:000000f0       __imp_?data@QArrayData@@QBEPBXXZ 100190f0     Qt5Core:Qt5Core.dll
 0002:000000f4       __imp_?qrand@@YAHXZ        100190f4     Qt5Core:Qt5Core.dll
 0002:000000f8       __imp_?freeData@QMapDataBase@@SAXPAU1@@Z 100190f8     Qt5Core:Qt5Core.dll
 0002:000000fc       __imp_?createData@QMapDataBase@@SAPAU1@XZ 100190fc     Qt5Core:Qt5Core.dll
 0002:00000100       __imp_?freeTree@QMapDataBase@@QAEXPAUQMapNodeBase@@H@Z 10019100     Qt5Core:Qt5Core.dll
 0002:00000104       __imp_?createNode@QMapDataBase@@QAEPAUQMapNodeBase@@HHPAU2@_N@Z 10019104     Qt5Core:Qt5Core.dll
 0002:00000108       __imp_?recalcMostLeftNode@QMapDataBase@@QAEXXZ 10019108     Qt5Core:Qt5Core.dll
 0002:0000010c       __imp_?freeNodeAndRebalance@QMapDataBase@@QAEXPAUQMapNodeBase@@@Z 1001910c     Qt5Core:Qt5Core.dll
 0002:00000110       __imp_?nextNode@QMapNodeBase@@QBEPBU1@XZ 10019110     Qt5Core:Qt5Core.dll
 0002:00000114       __imp_??0QString@@QAE@ABVQByteArray@@@Z 10019114     Qt5Core:Qt5Core.dll
 0002:00000118       __imp_?number@QString@@SA?AV1@NDH@Z 10019118     Qt5Core:Qt5Core.dll
 0002:0000011c       __imp_?number@QString@@SA?AV1@_JH@Z 1001911c     Qt5Core:Qt5Core.dll
 0002:00000120       __imp_?arg@QString@@QBE?AV1@DHVQChar@@@Z 10019120     Qt5Core:Qt5Core.dll
 0002:00000124       __imp_?arg@QString@@QBE?AV1@NHDHVQChar@@@Z 10019124     Qt5Core:Qt5Core.dll
 0002:00000128       __imp_?arg@QString@@QBE?AV1@_JHHVQChar@@@Z 10019128     Qt5Core:Qt5Core.dll
 0002:0000012c       __imp_??0QByteArray@@QAE@ABV0@@Z 1001912c     Qt5Core:Qt5Core.dll
 0002:00000130       __imp_?getAndRef@ExternalRefCountData@QtSharedPointer@@SAPAU12@PBVQObject@@@Z 10019130     Qt5Core:Qt5Core.dll
 0002:00000134       __imp_?sender@QObject@@IBEPAV1@XZ 10019134     Qt5Core:Qt5Core.dll
 0002:00000138       __imp_?detach@QListData@@QAEPAUData@1@H@Z 10019138     Qt5Core:Qt5Core.dll
 0002:0000013c       __imp_?cast@QMetaObject@@QBEPAVQObject@@PAV2@@Z 1001913c     Qt5Core:Qt5Core.dll
 0002:00000140       __imp_?arg@QString@@QBE?AV1@HHHVQChar@@@Z 10019140     Qt5Core:Qt5Core.dll
 0002:00000144       __imp_?shared_null@QHashData@@2U1@B 10019144     Qt5Core:Qt5Core.dll
 0002:00000148       __imp_?shared_null@QListData@@2UData@1@B 10019148     Qt5Core:Qt5Core.dll
 0002:0000014c       __imp_?shared_null@QArrayData@@2QBU1@B 1001914c     Qt5Core:Qt5Core.dll
 0002:00000150       __imp_?writeData@QFileDevice@@MAE_JPBD_J@Z 10019150     Qt5Core:Qt5Core.dll
 0002:00000154       __imp_?waitForReadyRead@QIODevice@@UAE_NH@Z 10019154     Qt5Core:Qt5Core.dll
 0002:00000158       __imp_?waitForBytesWritten@QIODevice@@UAE_NH@Z 10019158     Qt5Core:Qt5Core.dll
 0002:0000015c       __imp_?timerEvent@QObject@@MAEXPAVQTimerEvent@@@Z 1001915c     Qt5Core:Qt5Core.dll
 0002:00000160       __imp_?size@QFile@@UBE_JXZ 10019160     Qt5Core:Qt5Core.dll
 0002:00000164       __imp_?setPermissions@QFile@@UAE_NV?$QFlags@W4Permission@QFileDevice@@@@@Z 10019164     Qt5Core:Qt5Core.dll
 0002:00000168       __imp_?seek@QFileDevice@@UAE_N_J@Z 10019168     Qt5Core:Qt5Core.dll
 0002:0000016c       __imp_?resize@QFile@@UAE_N_J@Z 1001916c     Qt5Core:Qt5Core.dll
 0002:00000170       __imp_?reset@QIODevice@@UAE_NXZ 10019170     Qt5Core:Qt5Core.dll
 0002:00000174       __imp_?readLineData@QFileDevice@@MAE_JPAD_J@Z 10019174     Qt5Core:Qt5Core.dll
 0002:00000178       __imp_?readData@QFileDevice@@MAE_JPAD_J@Z 10019178     Qt5Core:Qt5Core.dll
 0002:0000017c       __imp_?qt_metacast@QFile@@UAEPAXPBD@Z 1001917c     Qt5Core:Qt5Core.dll
 0002:00000180       __imp_?qt_metacall@QFile@@UAEHW4Call@QMetaObject@@HPAPAX@Z 10019180     Qt5Core:Qt5Core.dll
 0002:00000184       __imp_?pos@QFileDevice@@UBE_JXZ 10019184     Qt5Core:Qt5Core.dll
 0002:00000188       __imp_?permissions@QFile@@UBE?AV?$QFlags@W4Permission@QFileDevice@@@@XZ 10019188     Qt5Core:Qt5Core.dll
 0002:0000018c       __imp_?open@QFile@@UAE_NV?$QFlags@W4OpenModeFlag@QIODevice@@@@@Z 1001918c     Qt5Core:Qt5Core.dll
 0002:00000190       __imp_?metaObject@QFile@@UBEPBUQMetaObject@@XZ 10019190     Qt5Core:Qt5Core.dll
 0002:00000194       __imp_?isSequential@QFileDevice@@UBE_NXZ 10019194     Qt5Core:Qt5Core.dll
 0002:00000198       __imp_?fileName@QFile@@UBE?AVQString@@XZ 10019198     Qt5Core:Qt5Core.dll
 0002:0000019c       __imp_?eventFilter@QObject@@UAE_NPAV1@PAVQEvent@@@Z 1001919c     Qt5Core:Qt5Core.dll
 0002:000001a0       __imp_?event@QObject@@UAE_NPAVQEvent@@@Z 100191a0     Qt5Core:Qt5Core.dll
 0002:000001a4       __imp_?disconnectNotify@QObject@@MAEXABVQMetaMethod@@@Z 100191a4     Qt5Core:Qt5Core.dll
 0002:000001a8       __imp_?customEvent@QObject@@MAEXPAVQEvent@@@Z 100191a8     Qt5Core:Qt5Core.dll
 0002:000001ac       __imp_?connectNotify@QObject@@MAEXABVQMetaMethod@@@Z 100191ac     Qt5Core:Qt5Core.dll
 0002:000001b0       __imp_?close@QFileDevice@@UAEXXZ 100191b0     Qt5Core:Qt5Core.dll
 0002:000001b4       __imp_?childEvent@QObject@@MAEXPAVQChildEvent@@@Z 100191b4     Qt5Core:Qt5Core.dll
 0002:000001b8       __imp_?canReadLine@QIODevice@@UBE_NXZ 100191b8     Qt5Core:Qt5Core.dll
 0002:000001bc       __imp_?bytesToWrite@QIODevice@@UBE_JXZ 100191bc     Qt5Core:Qt5Core.dll
 0002:000001c0       __imp_?bytesAvailable@QIODevice@@UBE_JXZ 100191c0     Qt5Core:Qt5Core.dll
 0002:000001c4       __imp_?atEnd@QFileDevice@@UBE_NXZ 100191c4     Qt5Core:Qt5Core.dll
 0002:000001c8       __imp_?translate@QCoreApplication@@SA?AVQString@@PBD00H@Z 100191c8     Qt5Core:Qt5Core.dll
 0002:000001cc       __imp_?toNativeSeparators@QDir@@SA?AVQString@@ABV2@@Z 100191cc     Qt5Core:Qt5Core.dll
 0002:000001d0       __imp_?free_helper@QHashData@@QAEXP6AXPAUNode@1@@Z@Z 100191d0     Qt5Core:Qt5Core.dll
 0002:000001d4       __imp_?rehash@QHashData@@QAEXH@Z 100191d4     Qt5Core:Qt5Core.dll
 0002:000001d8       __imp_?hasShrunk@QHashData@@QAEXXZ 100191d8     Qt5Core:Qt5Core.dll
 0002:000001dc       __imp_?detach_helper@QHashData@@QAEPAU1@P6AXPAUNode@1@PAX@ZP6AX0@ZHH@Z 100191dc     Qt5Core:Qt5Core.dll
 0002:000001e0       __imp_?freeNode@QHashData@@QAEXPAX@Z 100191e0     Qt5Core:Qt5Core.dll
 0002:000001e4       __imp_?allocateNode@QHashData@@QAEPAXH@Z 100191e4     Qt5Core:Qt5Core.dll
 0002:000001e8       __imp_??1QFile@@UAE@XZ     100191e8     Qt5Core:Qt5Core.dll
 0002:000001ec       __imp_??0QFile@@QAE@ABVQString@@@Z 100191ec     Qt5Core:Qt5Core.dll
 0002:000001f0       __imp_?write@QIODevice@@QAE_JABVQByteArray@@@Z 100191f0     Qt5Core:Qt5Core.dll
 0002:000001f4       __imp_?connect@QObject@@QBE?AVConnection@QMetaObject@@PBV1@PBD1W4ConnectionType@Qt@@@Z 100191f4     Qt5Core:Qt5Core.dll
 0002:000001f8       __imp_?connect@QObject@@SA?AVConnection@QMetaObject@@PBV1@PBD01W4ConnectionType@Qt@@@Z 100191f8     Qt5Core:Qt5Core.dll
 0002:000001fc       __imp_?setObjectName@QObject@@QAEXABVQString@@@Z 100191fc     Qt5Core:Qt5Core.dll
 0002:00000200       __imp_?objectName@QObject@@QBE?AVQString@@XZ 10019200     Qt5Core:Qt5Core.dll
 0002:00000204       __imp_?append@QListData@@QAEPAPAXXZ 10019204     Qt5Core:Qt5Core.dll
 0002:00000208       __imp_?dispose@QListData@@SAXPAUData@1@@Z 10019208     Qt5Core:Qt5Core.dll
 0002:0000020c       __imp_?detach_grow@QListData@@QAEPAUData@1@PAHH@Z 1001920c     Qt5Core:Qt5Core.dll
 0002:00000210       __imp_??1Connection@QMetaObject@@QAE@XZ 10019210     Qt5Core:Qt5Core.dll
 0002:00000214       __imp_?connectSlotsByName@QMetaObject@@SAXPAVQObject@@@Z 10019214     Qt5Core:Qt5Core.dll
 0002:00000218       __imp_?tr@QMetaObject@@QBE?AVQString@@PBD0H@Z 10019218     Qt5Core:Qt5Core.dll
 0002:0000021c       __imp_?fromAscii_helper@QString@@CAPAU?$QTypedArrayData@G@@PBDH@Z 1001921c     Qt5Core:Qt5Core.dll
 0002:00000220       __imp_??YQString@@QAEAAV0@PBD@Z 10019220     Qt5Core:Qt5Core.dll
 0002:00000224       __imp_??4QString@@QAEAAV0@PBD@Z 10019224     Qt5Core:Qt5Core.dll
 0002:00000228       __imp_??8@YA_NABVQString@@0@Z 10019228     Qt5Core:Qt5Core.dll
 0002:0000022c       __imp_?number@QString@@SA?AV1@HH@Z 1001922c     Qt5Core:Qt5Core.dll
 0002:00000230       __imp_?fromUtf8@QString@@SA?AV1@PBDH@Z 10019230     Qt5Core:Qt5Core.dll
 0002:00000234       __imp_?toLocal8Bit@QString@@QBE?AVQByteArray@@XZ 10019234     Qt5Core:Qt5Core.dll
 0002:00000238       __imp_?append@QString@@QAEAAV1@ABV1@@Z 10019238     Qt5Core:Qt5Core.dll
 0002:0000023c       __imp_?toUpper@QString@@QBE?AV1@XZ 1001923c     Qt5Core:Qt5Core.dll
 0002:00000240       __imp_?arg@QString@@QBE?AV1@ABV1@HVQChar@@@Z 10019240     Qt5Core:Qt5Core.dll
 0002:00000244       __imp_?clear@QString@@QAEXXZ 10019244     Qt5Core:Qt5Core.dll
 0002:00000248       __imp_??4QString@@QAEAAV0@$$QAV0@@Z 10019248     Qt5Core:Qt5Core.dll
 0002:0000024c       __imp_??0QString@@QAE@$$QAV0@@Z 1001924c     Qt5Core:Qt5Core.dll
 0002:00000250       __imp_??4QString@@QAEAAV0@ABV0@@Z 10019250     Qt5Core:Qt5Core.dll
 0002:00000254       __imp_??1QString@@QAE@XZ   10019254     Qt5Core:Qt5Core.dll
 0002:00000258       __imp_??0QString@@QAE@ABV0@@Z 10019258     Qt5Core:Qt5Core.dll
 0002:0000025c       __imp_??0QString@@QAE@VQChar@@@Z 1001925c     Qt5Core:Qt5Core.dll
 0002:00000260       __imp_??0QString@@QAE@XZ   10019260     Qt5Core:Qt5Core.dll
 0002:00000264       __imp_??BQByteRef@@QBEDXZ  10019264     Qt5Core:Qt5Core.dll
 0002:00000268       __imp_??AQByteArray@@QAE?AVQByteRef@@H@Z 10019268     Qt5Core:Qt5Core.dll
 0002:0000026c       __imp_??1QByteArray@@QAE@XZ 1001926c     Qt5Core:Qt5Core.dll
 0002:00000270       __imp_?allocate@QArrayData@@SAPAU1@IIIV?$QFlags@W4AllocationOption@QArrayData@@@@@Z 10019270     Qt5Core:Qt5Core.dll
 0002:00000274       __imp_?data@QArrayData@@QAEPAXXZ 10019274     Qt5Core:Qt5Core.dll
 0002:00000278       __imp_??0QChar@@QAE@UQLatin1Char@@@Z 10019278     Qt5Core:Qt5Core.dll
 0002:0000027c       __imp_?qBadAlloc@@YAXXZ    1001927c     Qt5Core:Qt5Core.dll
 0002:00000280       __imp_?deallocate@QArrayData@@SAXPAU1@II@Z 10019280     Qt5Core:Qt5Core.dll
 0002:00000284       \177Qt5Core_NULL_THUNK_DATA 10019284     Qt5Core:Qt5Core.dll
 0002:00000288       __imp_??1QIcon@@QAE@XZ     10019288     Qt5Gui:Qt5Gui.dll
 0002:0000028c       __imp_??0QIcon@@QAE@ABVQString@@@Z 1001928c     Qt5Gui:Qt5Gui.dll
 0002:00000290       __imp_??0QIcon@@QAE@XZ     10019290     Qt5Gui:Qt5Gui.dll
 0002:00000294       \177Qt5Gui_NULL_THUNK_DATA 10019294     Qt5Gui:Qt5Gui.dll
 0002:00000298       __imp_?setChecked@QAbstractButton@@QAEX_N@Z 10019298     Qt5Widgets:Qt5Widgets.dll
 0002:0000029c       __imp_??0QDialogButtonBox@@QAE@PAVQWidget@@@Z 1001929c     Qt5Widgets:Qt5Widgets.dll
 0002:000002a0       __imp_??1QDialogButtonBox@@UAE@XZ 100192a0     Qt5Widgets:Qt5Widgets.dll
 0002:000002a4       __imp_?setStandardButtons@QDialogButtonBox@@QAEXV?$QFlags@W4StandardButton@QDialogButtonBox@@@@@Z 100192a4     Qt5Widgets:Qt5Widgets.dll
 0002:000002a8       __imp_?button@QDialogButtonBox@@QBEPAVQPushButton@@W4StandardButton@1@@Z 100192a8     Qt5Widgets:Qt5Widgets.dll
 0002:000002ac       __imp_??0QLabel@@QAE@PAVQWidget@@V?$QFlags@W4WindowType@Qt@@@@@Z 100192ac     Qt5Widgets:Qt5Widgets.dll
 0002:000002b0       __imp_??1QLabel@@UAE@XZ    100192b0     Qt5Widgets:Qt5Widgets.dll
 0002:000002b4       __imp_?setText@QLabel@@QAEXABVQString@@@Z 100192b4     Qt5Widgets:Qt5Widgets.dll
 0002:000002b8       __imp_??0QCheckBox@@QAE@PAVQWidget@@@Z 100192b8     Qt5Widgets:Qt5Widgets.dll
 0002:000002bc       __imp_??1QCheckBox@@UAE@XZ 100192bc     Qt5Widgets:Qt5Widgets.dll
 0002:000002c0       __imp_?addWidget@QBoxLayout@@QAEXPAVQWidget@@HV?$QFlags@W4AlignmentFlag@Qt@@@@@Z 100192c0     Qt5Widgets:Qt5Widgets.dll
 0002:000002c4       __imp_??0QVBoxLayout@@QAE@PAVQWidget@@@Z 100192c4     Qt5Widgets:Qt5Widgets.dll
 0002:000002c8       __imp_??1QVBoxLayout@@UAE@XZ 100192c8     Qt5Widgets:Qt5Widgets.dll
 0002:000002cc       __imp_??0QGridLayout@@QAE@PAVQWidget@@@Z 100192cc     Qt5Widgets:Qt5Widgets.dll
 0002:000002d0       __imp_??1QGridLayout@@UAE@XZ 100192d0     Qt5Widgets:Qt5Widgets.dll
 0002:000002d4       __imp_?addWidget@QGridLayout@@QAEXPAVQWidget@@HHHHV?$QFlags@W4AlignmentFlag@Qt@@@@@Z 100192d4     Qt5Widgets:Qt5Widgets.dll
 0002:000002d8       __imp_??0QGroupBox@@QAE@PAVQWidget@@@Z 100192d8     Qt5Widgets:Qt5Widgets.dll
 0002:000002dc       __imp_??1QGroupBox@@UAE@XZ 100192dc     Qt5Widgets:Qt5Widgets.dll
 0002:000002e0       __imp_?setTitle@QGroupBox@@QAEXABVQString@@@Z 100192e0     Qt5Widgets:Qt5Widgets.dll
 0002:000002e4       __imp_?setCheckable@QGroupBox@@QAEX_N@Z 100192e4     Qt5Widgets:Qt5Widgets.dll
 0002:000002e8       __imp_?isChecked@QGroupBox@@QBE_NXZ 100192e8     Qt5Widgets:Qt5Widgets.dll
 0002:000002ec       __imp_?setChecked@QGroupBox@@QAEX_N@Z 100192ec     Qt5Widgets:Qt5Widgets.dll
 0002:000002f0       __imp_??0QLineEdit@@QAE@PAVQWidget@@@Z 100192f0     Qt5Widgets:Qt5Widgets.dll
 0002:000002f4       __imp_??1QLineEdit@@UAE@XZ 100192f4     Qt5Widgets:Qt5Widgets.dll
 0002:000002f8       __imp_??0QRadioButton@@QAE@PAVQWidget@@@Z 100192f8     Qt5Widgets:Qt5Widgets.dll
 0002:000002fc       __imp_??1QRadioButton@@UAE@XZ 100192fc     Qt5Widgets:Qt5Widgets.dll
 0002:00000300       __imp_??0QToolButton@@QAE@PAVQWidget@@@Z 10019300     Qt5Widgets:Qt5Widgets.dll
 0002:00000304       __imp_??1QToolButton@@UAE@XZ 10019304     Qt5Widgets:Qt5Widgets.dll
 0002:00000308       __imp_?actionEvent@QToolButton@@MAEXPAVQActionEvent@@@Z 10019308     Qt5Widgets:Qt5Widgets.dll
 0002:0000030c       __imp_?actionEvent@QWidget@@MAEXPAVQActionEvent@@@Z 1001930c     Qt5Widgets:Qt5Widgets.dll
 0002:00000310       __imp_?addItem@QBoxLayout@@UAEXPAVQLayoutItem@@@Z 10019310     Qt5Widgets:Qt5Widgets.dll
 0002:00000314       __imp_?addItem@QGridLayout@@MAEXPAVQLayoutItem@@@Z 10019314     Qt5Widgets:Qt5Widgets.dll
 0002:00000318       __imp_?changeEvent@QAbstractButton@@MAEXPAVQEvent@@@Z 10019318     Qt5Widgets:Qt5Widgets.dll
 0002:0000031c       __imp_?changeEvent@QDialogButtonBox@@MAEXPAVQEvent@@@Z 1001931c     Qt5Widgets:Qt5Widgets.dll
 0002:00000320       __imp_?changeEvent@QGroupBox@@MAEXPAVQEvent@@@Z 10019320     Qt5Widgets:Qt5Widgets.dll
 0002:00000324       __imp_?changeEvent@QLabel@@MAEXPAVQEvent@@@Z 10019324     Qt5Widgets:Qt5Widgets.dll
 0002:00000328       __imp_?changeEvent@QLineEdit@@MAEXPAVQEvent@@@Z 10019328     Qt5Widgets:Qt5Widgets.dll
 0002:0000032c       __imp_?changeEvent@QToolButton@@MAEXPAVQEvent@@@Z 1001932c     Qt5Widgets:Qt5Widgets.dll
 0002:00000330       __imp_?changeEvent@QWidget@@MAEXPAVQEvent@@@Z 10019330     Qt5Widgets:Qt5Widgets.dll
 0002:00000334       __imp_?checkStateSet@QAbstractButton@@MAEXXZ 10019334     Qt5Widgets:Qt5Widgets.dll
 0002:00000338       __imp_?checkStateSet@QCheckBox@@MAEXXZ 10019338     Qt5Widgets:Qt5Widgets.dll
 0002:0000033c       __imp_?childEvent@QGroupBox@@MAEXPAVQChildEvent@@@Z 1001933c     Qt5Widgets:Qt5Widgets.dll
 0002:00000340       __imp_?childEvent@QLayout@@MAEXPAVQChildEvent@@@Z 10019340     Qt5Widgets:Qt5Widgets.dll
 0002:00000344       __imp_?closeEvent@QDialog@@MAEXPAVQCloseEvent@@@Z 10019344     Qt5Widgets:Qt5Widgets.dll
 0002:00000348       __imp_?closeEvent@QWidget@@MAEXPAVQCloseEvent@@@Z 10019348     Qt5Widgets:Qt5Widgets.dll
 0002:0000034c       __imp_?contextMenuEvent@QDialog@@MAEXPAVQContextMenuEvent@@@Z 1001934c     Qt5Widgets:Qt5Widgets.dll
 0002:00000350       __imp_?contextMenuEvent@QLabel@@MAEXPAVQContextMenuEvent@@@Z 10019350     Qt5Widgets:Qt5Widgets.dll
 0002:00000354       __imp_?contextMenuEvent@QLineEdit@@MAEXPAVQContextMenuEvent@@@Z 10019354     Qt5Widgets:Qt5Widgets.dll
 0002:00000358       __imp_?contextMenuEvent@QWidget@@MAEXPAVQContextMenuEvent@@@Z 10019358     Qt5Widgets:Qt5Widgets.dll
 0002:0000035c       __imp_?controlTypes@QLayout@@UBE?AV?$QFlags@W4ControlType@QSizePolicy@@@@XZ 1001935c     Qt5Widgets:Qt5Widgets.dll
 0002:00000360       __imp_?count@QBoxLayout@@UBEHXZ 10019360     Qt5Widgets:Qt5Widgets.dll
 0002:00000364       __imp_?count@QGridLayout@@UBEHXZ 10019364     Qt5Widgets:Qt5Widgets.dll
 0002:00000368       __imp_?devType@QWidget@@UBEHXZ 10019368     Qt5Widgets:Qt5Widgets.dll
 0002:0000036c       __imp_?done@QDialog@@UAEXH@Z 1001936c     Qt5Widgets:Qt5Widgets.dll
 0002:00000370       __imp_?dragEnterEvent@QLineEdit@@MAEXPAVQDragEnterEvent@@@Z 10019370     Qt5Widgets:Qt5Widgets.dll
 0002:00000374       __imp_?dragEnterEvent@QWidget@@MAEXPAVQDragEnterEvent@@@Z 10019374     Qt5Widgets:Qt5Widgets.dll
 0002:00000378       __imp_?dragLeaveEvent@QLineEdit@@MAEXPAVQDragLeaveEvent@@@Z 10019378     Qt5Widgets:Qt5Widgets.dll
 0002:0000037c       __imp_?dragLeaveEvent@QWidget@@MAEXPAVQDragLeaveEvent@@@Z 1001937c     Qt5Widgets:Qt5Widgets.dll
 0002:00000380       __imp_?dragMoveEvent@QLineEdit@@MAEXPAVQDragMoveEvent@@@Z 10019380     Qt5Widgets:Qt5Widgets.dll
 0002:00000384       __imp_?dragMoveEvent@QWidget@@MAEXPAVQDragMoveEvent@@@Z 10019384     Qt5Widgets:Qt5Widgets.dll
 0002:00000388       __imp_?dropEvent@QLineEdit@@MAEXPAVQDropEvent@@@Z 10019388     Qt5Widgets:Qt5Widgets.dll
 0002:0000038c       __imp_?dropEvent@QWidget@@MAEXPAVQDropEvent@@@Z 1001938c     Qt5Widgets:Qt5Widgets.dll
 0002:00000390       __imp_?enterEvent@QToolButton@@MAEXPAVQEvent@@@Z 10019390     Qt5Widgets:Qt5Widgets.dll
 0002:00000394       __imp_?enterEvent@QWidget@@MAEXPAVQEvent@@@Z 10019394     Qt5Widgets:Qt5Widgets.dll
 0002:00000398       __imp_?event@QCheckBox@@MAE_NPAVQEvent@@@Z 10019398     Qt5Widgets:Qt5Widgets.dll
 0002:0000039c       __imp_??1QDialog@@UAE@XZ   1001939c     Qt5Widgets:Qt5Widgets.dll
 0002:000003a0       __imp_?event@QGroupBox@@MAE_NPAVQEvent@@@Z 100193a0     Qt5Widgets:Qt5Widgets.dll
 0002:000003a4       __imp_?event@QLabel@@MAE_NPAVQEvent@@@Z 100193a4     Qt5Widgets:Qt5Widgets.dll
 0002:000003a8       __imp_?event@QLineEdit@@UAE_NPAVQEvent@@@Z 100193a8     Qt5Widgets:Qt5Widgets.dll
 0002:000003ac       __imp_?event@QRadioButton@@MAE_NPAVQEvent@@@Z 100193ac     Qt5Widgets:Qt5Widgets.dll
 0002:000003b0       __imp_?event@QToolButton@@MAE_NPAVQEvent@@@Z 100193b0     Qt5Widgets:Qt5Widgets.dll
 0002:000003b4       __imp_?event@QWidget@@MAE_NPAVQEvent@@@Z 100193b4     Qt5Widgets:Qt5Widgets.dll
 0002:000003b8       __imp_?eventFilter@QDialog@@MAE_NPAVQObject@@PAVQEvent@@@Z 100193b8     Qt5Widgets:Qt5Widgets.dll
 0002:000003bc       __imp_?exec@QDialog@@UAEHXZ 100193bc     Qt5Widgets:Qt5Widgets.dll
 0002:000003c0       __imp_?expandingDirections@QBoxLayout@@UBE?AV?$QFlags@W4Orientation@Qt@@@@XZ 100193c0     Qt5Widgets:Qt5Widgets.dll
 0002:000003c4       __imp_?expandingDirections@QGridLayout@@UBE?AV?$QFlags@W4Orientation@Qt@@@@XZ 100193c4     Qt5Widgets:Qt5Widgets.dll
 0002:000003c8       __imp_?focusInEvent@QAbstractButton@@MAEXPAVQFocusEvent@@@Z 100193c8     Qt5Widgets:Qt5Widgets.dll
 0002:000003cc       __imp_?focusInEvent@QGroupBox@@MAEXPAVQFocusEvent@@@Z 100193cc     Qt5Widgets:Qt5Widgets.dll
 0002:000003d0       __imp_?focusInEvent@QLabel@@MAEXPAVQFocusEvent@@@Z 100193d0     Qt5Widgets:Qt5Widgets.dll
 0002:000003d4       __imp_?focusInEvent@QLineEdit@@MAEXPAVQFocusEvent@@@Z 100193d4     Qt5Widgets:Qt5Widgets.dll
 0002:000003d8       __imp_?focusInEvent@QWidget@@MAEXPAVQFocusEvent@@@Z 100193d8     Qt5Widgets:Qt5Widgets.dll
 0002:000003dc       __imp_?focusNextPrevChild@QLabel@@MAE_N_N@Z 100193dc     Qt5Widgets:Qt5Widgets.dll
 0002:000003e0       __imp_?focusNextPrevChild@QWidget@@MAE_N_N@Z 100193e0     Qt5Widgets:Qt5Widgets.dll
 0002:000003e4       __imp_?focusOutEvent@QAbstractButton@@MAEXPAVQFocusEvent@@@Z 100193e4     Qt5Widgets:Qt5Widgets.dll
 0002:000003e8       __imp_?focusOutEvent@QLabel@@MAEXPAVQFocusEvent@@@Z 100193e8     Qt5Widgets:Qt5Widgets.dll
 0002:000003ec       __imp_?focusOutEvent@QLineEdit@@MAEXPAVQFocusEvent@@@Z 100193ec     Qt5Widgets:Qt5Widgets.dll
 0002:000003f0       __imp_?focusOutEvent@QWidget@@MAEXPAVQFocusEvent@@@Z 100193f0     Qt5Widgets:Qt5Widgets.dll
 0002:000003f4       __imp_?geometry@QLayout@@UBE?AVQRect@@XZ 100193f4     Qt5Widgets:Qt5Widgets.dll
 0002:000003f8       __imp_?hasHeightForWidth@QBoxLayout@@UBE_NXZ 100193f8     Qt5Widgets:Qt5Widgets.dll
 0002:000003fc       __imp_?hasHeightForWidth@QGridLayout@@UBE_NXZ 100193fc     Qt5Widgets:Qt5Widgets.dll
 0002:00000400       __imp_?hasHeightForWidth@QWidget@@UBE_NXZ 10019400     Qt5Widgets:Qt5Widgets.dll
 0002:00000404       __imp_?heightForWidth@QBoxLayout@@UBEHH@Z 10019404     Qt5Widgets:Qt5Widgets.dll
 0002:00000408       __imp_?heightForWidth@QGridLayout@@UBEHH@Z 10019408     Qt5Widgets:Qt5Widgets.dll
 0002:0000040c       __imp_?heightForWidth@QLabel@@UBEHH@Z 1001940c     Qt5Widgets:Qt5Widgets.dll
 0002:00000410       __imp_?heightForWidth@QWidget@@UBEHH@Z 10019410     Qt5Widgets:Qt5Widgets.dll
 0002:00000414       __imp_?hideEvent@QWidget@@MAEXPAVQHideEvent@@@Z 10019414     Qt5Widgets:Qt5Widgets.dll
 0002:00000418       __imp_?hitButton@QCheckBox@@MBE_NABVQPoint@@@Z 10019418     Qt5Widgets:Qt5Widgets.dll
 0002:0000041c       __imp_?hitButton@QRadioButton@@MBE_NABVQPoint@@@Z 1001941c     Qt5Widgets:Qt5Widgets.dll
 0002:00000420       __imp_?hitButton@QToolButton@@MBE_NABVQPoint@@@Z 10019420     Qt5Widgets:Qt5Widgets.dll
 0002:00000424       __imp_?indexOf@QLayout@@UBEHPAVQWidget@@@Z 10019424     Qt5Widgets:Qt5Widgets.dll
 0002:00000428       __imp_?initPainter@QWidget@@MBEXPAVQPainter@@@Z 10019428     Qt5Widgets:Qt5Widgets.dll
 0002:0000042c       __imp_?inputMethodEvent@QLineEdit@@MAEXPAVQInputMethodEvent@@@Z 1001942c     Qt5Widgets:Qt5Widgets.dll
 0002:00000430       __imp_?inputMethodEvent@QWidget@@MAEXPAVQInputMethodEvent@@@Z 10019430     Qt5Widgets:Qt5Widgets.dll
 0002:00000434       __imp_?inputMethodQuery@QLineEdit@@UBE?AVQVariant@@W4InputMethodQuery@Qt@@@Z 10019434     Qt5Widgets:Qt5Widgets.dll
 0002:00000438       __imp_?inputMethodQuery@QWidget@@UBE?AVQVariant@@W4InputMethodQuery@Qt@@@Z 10019438     Qt5Widgets:Qt5Widgets.dll
 0002:0000043c       __imp_?invalidate@QBoxLayout@@UAEXXZ 1001943c     Qt5Widgets:Qt5Widgets.dll
 0002:00000440       __imp_?invalidate@QGridLayout@@UAEXXZ 10019440     Qt5Widgets:Qt5Widgets.dll
 0002:00000444       __imp_?isEmpty@QLayout@@UBE_NXZ 10019444     Qt5Widgets:Qt5Widgets.dll
 0002:00000448       __imp_?itemAt@QBoxLayout@@UBEPAVQLayoutItem@@H@Z 10019448     Qt5Widgets:Qt5Widgets.dll
 0002:0000044c       __imp_?itemAt@QGridLayout@@UBEPAVQLayoutItem@@H@Z 1001944c     Qt5Widgets:Qt5Widgets.dll
 0002:00000450       __imp_?keyPressEvent@QAbstractButton@@MAEXPAVQKeyEvent@@@Z 10019450     Qt5Widgets:Qt5Widgets.dll
 0002:00000454       __imp_?keyPressEvent@QDialog@@MAEXPAVQKeyEvent@@@Z 10019454     Qt5Widgets:Qt5Widgets.dll
 0002:00000458       __imp_?keyPressEvent@QLabel@@MAEXPAVQKeyEvent@@@Z 10019458     Qt5Widgets:Qt5Widgets.dll
 0002:0000045c       __imp_?keyPressEvent@QLineEdit@@MAEXPAVQKeyEvent@@@Z 1001945c     Qt5Widgets:Qt5Widgets.dll
 0002:00000460       __imp_?keyPressEvent@QWidget@@MAEXPAVQKeyEvent@@@Z 10019460     Qt5Widgets:Qt5Widgets.dll
 0002:00000464       __imp_?keyReleaseEvent@QAbstractButton@@MAEXPAVQKeyEvent@@@Z 10019464     Qt5Widgets:Qt5Widgets.dll
 0002:00000468       __imp_?keyReleaseEvent@QWidget@@MAEXPAVQKeyEvent@@@Z 10019468     Qt5Widgets:Qt5Widgets.dll
 0002:0000046c       __imp_?layout@QLayout@@UAEPAV1@XZ 1001946c     Qt5Widgets:Qt5Widgets.dll
 0002:00000470       __imp_?leaveEvent@QToolButton@@MAEXPAVQEvent@@@Z 10019470     Qt5Widgets:Qt5Widgets.dll
 0002:00000474       __imp_?leaveEvent@QWidget@@MAEXPAVQEvent@@@Z 10019474     Qt5Widgets:Qt5Widgets.dll
 0002:00000478       __imp_?maximumSize@QBoxLayout@@UBE?AVQSize@@XZ 10019478     Qt5Widgets:Qt5Widgets.dll
 0002:0000047c       __imp_?maximumSize@QGridLayout@@UBE?AVQSize@@XZ 1001947c     Qt5Widgets:Qt5Widgets.dll
 0002:00000480       __imp_?metaObject@QCheckBox@@UBEPBUQMetaObject@@XZ 10019480     Qt5Widgets:Qt5Widgets.dll
 0002:00000484       __imp_?metaObject@QDialogButtonBox@@UBEPBUQMetaObject@@XZ 10019484     Qt5Widgets:Qt5Widgets.dll
 0002:00000488       __imp_?metaObject@QGridLayout@@UBEPBUQMetaObject@@XZ 10019488     Qt5Widgets:Qt5Widgets.dll
 0002:0000048c       __imp_?metaObject@QGroupBox@@UBEPBUQMetaObject@@XZ 1001948c     Qt5Widgets:Qt5Widgets.dll
 0002:00000490       __imp_?metaObject@QLabel@@UBEPBUQMetaObject@@XZ 10019490     Qt5Widgets:Qt5Widgets.dll
 0002:00000494       __imp_?metaObject@QLineEdit@@UBEPBUQMetaObject@@XZ 10019494     Qt5Widgets:Qt5Widgets.dll
 0002:00000498       __imp_?metaObject@QRadioButton@@UBEPBUQMetaObject@@XZ 10019498     Qt5Widgets:Qt5Widgets.dll
 0002:0000049c       __imp_?metaObject@QToolButton@@UBEPBUQMetaObject@@XZ 1001949c     Qt5Widgets:Qt5Widgets.dll
 0002:000004a0       __imp_?metaObject@QVBoxLayout@@UBEPBUQMetaObject@@XZ 100194a0     Qt5Widgets:Qt5Widgets.dll
 0002:000004a4       __imp_?metric@QWidget@@MBEHW4PaintDeviceMetric@QPaintDevice@@@Z 100194a4     Qt5Widgets:Qt5Widgets.dll
 0002:000004a8       __imp_?minimumHeightForWidth@QBoxLayout@@UBEHH@Z 100194a8     Qt5Widgets:Qt5Widgets.dll
 0002:000004ac       __imp_?minimumHeightForWidth@QGridLayout@@UBEHH@Z 100194ac     Qt5Widgets:Qt5Widgets.dll
 0002:000004b0       __imp_?minimumSize@QBoxLayout@@UBE?AVQSize@@XZ 100194b0     Qt5Widgets:Qt5Widgets.dll
 0002:000004b4       __imp_?minimumSize@QGridLayout@@UBE?AVQSize@@XZ 100194b4     Qt5Widgets:Qt5Widgets.dll
 0002:000004b8       __imp_?minimumSizeHint@QCheckBox@@UBE?AVQSize@@XZ 100194b8     Qt5Widgets:Qt5Widgets.dll
 0002:000004bc       __imp_?minimumSizeHint@QDialog@@UBE?AVQSize@@XZ 100194bc     Qt5Widgets:Qt5Widgets.dll
 0002:000004c0       __imp_?minimumSizeHint@QGroupBox@@UBE?AVQSize@@XZ 100194c0     Qt5Widgets:Qt5Widgets.dll
 0002:000004c4       __imp_?minimumSizeHint@QLabel@@UBE?AVQSize@@XZ 100194c4     Qt5Widgets:Qt5Widgets.dll
 0002:000004c8       __imp_?minimumSizeHint@QLineEdit@@UBE?AVQSize@@XZ 100194c8     Qt5Widgets:Qt5Widgets.dll
 0002:000004cc       __imp_?minimumSizeHint@QRadioButton@@UBE?AVQSize@@XZ 100194cc     Qt5Widgets:Qt5Widgets.dll
 0002:000004d0       __imp_?minimumSizeHint@QToolButton@@UBE?AVQSize@@XZ 100194d0     Qt5Widgets:Qt5Widgets.dll
 0002:000004d4       __imp_?isChecked@QAbstractButton@@QBE_NXZ 100194d4     Qt5Widgets:Qt5Widgets.dll
 0002:000004d8       __imp_?mouseDoubleClickEvent@QLineEdit@@MAEXPAVQMouseEvent@@@Z 100194d8     Qt5Widgets:Qt5Widgets.dll
 0002:000004dc       __imp_?mouseDoubleClickEvent@QWidget@@MAEXPAVQMouseEvent@@@Z 100194dc     Qt5Widgets:Qt5Widgets.dll
 0002:000004e0       __imp_?mouseMoveEvent@QAbstractButton@@MAEXPAVQMouseEvent@@@Z 100194e0     Qt5Widgets:Qt5Widgets.dll
 0002:000004e4       __imp_?mouseMoveEvent@QCheckBox@@MAEXPAVQMouseEvent@@@Z 100194e4     Qt5Widgets:Qt5Widgets.dll
 0002:000004e8       __imp_?mouseMoveEvent@QGroupBox@@MAEXPAVQMouseEvent@@@Z 100194e8     Qt5Widgets:Qt5Widgets.dll
 0002:000004ec       __imp_?mouseMoveEvent@QLabel@@MAEXPAVQMouseEvent@@@Z 100194ec     Qt5Widgets:Qt5Widgets.dll
 0002:000004f0       __imp_?mouseMoveEvent@QLineEdit@@MAEXPAVQMouseEvent@@@Z 100194f0     Qt5Widgets:Qt5Widgets.dll
 0002:000004f4       __imp_?mouseMoveEvent@QRadioButton@@MAEXPAVQMouseEvent@@@Z 100194f4     Qt5Widgets:Qt5Widgets.dll
 0002:000004f8       __imp_?mouseMoveEvent@QWidget@@MAEXPAVQMouseEvent@@@Z 100194f8     Qt5Widgets:Qt5Widgets.dll
 0002:000004fc       __imp_?mousePressEvent@QAbstractButton@@MAEXPAVQMouseEvent@@@Z 100194fc     Qt5Widgets:Qt5Widgets.dll
 0002:00000500       __imp_?mousePressEvent@QGroupBox@@MAEXPAVQMouseEvent@@@Z 10019500     Qt5Widgets:Qt5Widgets.dll
 0002:00000504       __imp_?mousePressEvent@QLabel@@MAEXPAVQMouseEvent@@@Z 10019504     Qt5Widgets:Qt5Widgets.dll
 0002:00000508       __imp_?mousePressEvent@QLineEdit@@MAEXPAVQMouseEvent@@@Z 10019508     Qt5Widgets:Qt5Widgets.dll
 0002:0000050c       __imp_?mousePressEvent@QToolButton@@MAEXPAVQMouseEvent@@@Z 1001950c     Qt5Widgets:Qt5Widgets.dll
 0002:00000510       __imp_?mousePressEvent@QWidget@@MAEXPAVQMouseEvent@@@Z 10019510     Qt5Widgets:Qt5Widgets.dll
 0002:00000514       __imp_?mouseReleaseEvent@QAbstractButton@@MAEXPAVQMouseEvent@@@Z 10019514     Qt5Widgets:Qt5Widgets.dll
 0002:00000518       __imp_?mouseReleaseEvent@QGroupBox@@MAEXPAVQMouseEvent@@@Z 10019518     Qt5Widgets:Qt5Widgets.dll
 0002:0000051c       __imp_?mouseReleaseEvent@QLabel@@MAEXPAVQMouseEvent@@@Z 1001951c     Qt5Widgets:Qt5Widgets.dll
 0002:00000520       __imp_?mouseReleaseEvent@QLineEdit@@MAEXPAVQMouseEvent@@@Z 10019520     Qt5Widgets:Qt5Widgets.dll
 0002:00000524       __imp_?mouseReleaseEvent@QToolButton@@MAEXPAVQMouseEvent@@@Z 10019524     Qt5Widgets:Qt5Widgets.dll
 0002:00000528       __imp_?mouseReleaseEvent@QWidget@@MAEXPAVQMouseEvent@@@Z 10019528     Qt5Widgets:Qt5Widgets.dll
 0002:0000052c       __imp_?moveEvent@QWidget@@MAEXPAVQMoveEvent@@@Z 1001952c     Qt5Widgets:Qt5Widgets.dll
 0002:00000530       __imp_?nativeEvent@QWidget@@MAE_NABVQByteArray@@PAXPAJ@Z 10019530     Qt5Widgets:Qt5Widgets.dll
 0002:00000534       __imp_?nextCheckState@QAbstractButton@@MAEXXZ 10019534     Qt5Widgets:Qt5Widgets.dll
 0002:00000538       __imp_?nextCheckState@QCheckBox@@MAEXXZ 10019538     Qt5Widgets:Qt5Widgets.dll
 0002:0000053c       __imp_?nextCheckState@QToolButton@@MAEXXZ 1001953c     Qt5Widgets:Qt5Widgets.dll
 0002:00000540       __imp_?open@QDialog@@UAEXXZ 10019540     Qt5Widgets:Qt5Widgets.dll
 0002:00000544       __imp_?paintEngine@QWidget@@UBEPAVQPaintEngine@@XZ 10019544     Qt5Widgets:Qt5Widgets.dll
 0002:00000548       __imp_?paintEvent@QCheckBox@@MAEXPAVQPaintEvent@@@Z 10019548     Qt5Widgets:Qt5Widgets.dll
 0002:0000054c       __imp_?paintEvent@QGroupBox@@MAEXPAVQPaintEvent@@@Z 1001954c     Qt5Widgets:Qt5Widgets.dll
 0002:00000550       __imp_?paintEvent@QLabel@@MAEXPAVQPaintEvent@@@Z 10019550     Qt5Widgets:Qt5Widgets.dll
 0002:00000554       __imp_?paintEvent@QLineEdit@@MAEXPAVQPaintEvent@@@Z 10019554     Qt5Widgets:Qt5Widgets.dll
 0002:00000558       __imp_?paintEvent@QRadioButton@@MAEXPAVQPaintEvent@@@Z 10019558     Qt5Widgets:Qt5Widgets.dll
 0002:0000055c       __imp_?paintEvent@QToolButton@@MAEXPAVQPaintEvent@@@Z 1001955c     Qt5Widgets:Qt5Widgets.dll
 0002:00000560       __imp_?paintEvent@QWidget@@MAEXPAVQPaintEvent@@@Z 10019560     Qt5Widgets:Qt5Widgets.dll
 0002:00000564       __imp_?qt_metacall@QCheckBox@@UAEHW4Call@QMetaObject@@HPAPAX@Z 10019564     Qt5Widgets:Qt5Widgets.dll
 0002:00000568       __imp_?qt_metacall@QDialogButtonBox@@UAEHW4Call@QMetaObject@@HPAPAX@Z 10019568     Qt5Widgets:Qt5Widgets.dll
 0002:0000056c       __imp_?qt_metacall@QGridLayout@@UAEHW4Call@QMetaObject@@HPAPAX@Z 1001956c     Qt5Widgets:Qt5Widgets.dll
 0002:00000570       __imp_?qt_metacall@QGroupBox@@UAEHW4Call@QMetaObject@@HPAPAX@Z 10019570     Qt5Widgets:Qt5Widgets.dll
 0002:00000574       __imp_?qt_metacall@QLabel@@UAEHW4Call@QMetaObject@@HPAPAX@Z 10019574     Qt5Widgets:Qt5Widgets.dll
 0002:00000578       __imp_?qt_metacall@QLineEdit@@UAEHW4Call@QMetaObject@@HPAPAX@Z 10019578     Qt5Widgets:Qt5Widgets.dll
 0002:0000057c       __imp_?qt_metacall@QRadioButton@@UAEHW4Call@QMetaObject@@HPAPAX@Z 1001957c     Qt5Widgets:Qt5Widgets.dll
 0002:00000580       __imp_?qt_metacall@QToolButton@@UAEHW4Call@QMetaObject@@HPAPAX@Z 10019580     Qt5Widgets:Qt5Widgets.dll
 0002:00000584       __imp_?qt_metacall@QVBoxLayout@@UAEHW4Call@QMetaObject@@HPAPAX@Z 10019584     Qt5Widgets:Qt5Widgets.dll
 0002:00000588       __imp_?qt_metacast@QCheckBox@@UAEPAXPBD@Z 10019588     Qt5Widgets:Qt5Widgets.dll
 0002:0000058c       __imp_?qt_metacast@QDialogButtonBox@@UAEPAXPBD@Z 1001958c     Qt5Widgets:Qt5Widgets.dll
 0002:00000590       __imp_?qt_metacast@QGridLayout@@UAEPAXPBD@Z 10019590     Qt5Widgets:Qt5Widgets.dll
 0002:00000594       __imp_?qt_metacast@QGroupBox@@UAEPAXPBD@Z 10019594     Qt5Widgets:Qt5Widgets.dll
 0002:00000598       __imp_?qt_metacast@QLabel@@UAEPAXPBD@Z 10019598     Qt5Widgets:Qt5Widgets.dll
 0002:0000059c       __imp_?qt_metacast@QLineEdit@@UAEPAXPBD@Z 1001959c     Qt5Widgets:Qt5Widgets.dll
 0002:000005a0       __imp_?qt_metacast@QRadioButton@@UAEPAXPBD@Z 100195a0     Qt5Widgets:Qt5Widgets.dll
 0002:000005a4       __imp_?qt_metacast@QToolButton@@UAEPAXPBD@Z 100195a4     Qt5Widgets:Qt5Widgets.dll
 0002:000005a8       __imp_?qt_metacast@QVBoxLayout@@UAEPAXPBD@Z 100195a8     Qt5Widgets:Qt5Widgets.dll
 0002:000005ac       __imp_?redirected@QWidget@@MBEPAVQPaintDevice@@PAVQPoint@@@Z 100195ac     Qt5Widgets:Qt5Widgets.dll
 0002:000005b0       __imp_?reject@QDialog@@UAEXXZ 100195b0     Qt5Widgets:Qt5Widgets.dll
 0002:000005b4       __imp_?resizeEvent@QDialog@@MAEXPAVQResizeEvent@@@Z 100195b4     Qt5Widgets:Qt5Widgets.dll
 0002:000005b8       __imp_?resizeEvent@QGroupBox@@MAEXPAVQResizeEvent@@@Z 100195b8     Qt5Widgets:Qt5Widgets.dll
 0002:000005bc       __imp_?resizeEvent@QWidget@@MAEXPAVQResizeEvent@@@Z 100195bc     Qt5Widgets:Qt5Widgets.dll
 0002:000005c0       __imp_?setGeometry@QBoxLayout@@UAEXABVQRect@@@Z 100195c0     Qt5Widgets:Qt5Widgets.dll
 0002:000005c4       __imp_?setGeometry@QGridLayout@@UAEXABVQRect@@@Z 100195c4     Qt5Widgets:Qt5Widgets.dll
 0002:000005c8       __imp_?setVisible@QDialog@@UAEX_N@Z 100195c8     Qt5Widgets:Qt5Widgets.dll
 0002:000005cc       __imp_?setVisible@QWidget@@UAEX_N@Z 100195cc     Qt5Widgets:Qt5Widgets.dll
 0002:000005d0       __imp_?sharedPainter@QWidget@@MBEPAVQPainter@@XZ 100195d0     Qt5Widgets:Qt5Widgets.dll
 0002:000005d4       __imp_?showEvent@QDialog@@MAEXPAVQShowEvent@@@Z 100195d4     Qt5Widgets:Qt5Widgets.dll
 0002:000005d8       __imp_?showEvent@QWidget@@MAEXPAVQShowEvent@@@Z 100195d8     Qt5Widgets:Qt5Widgets.dll
 0002:000005dc       __imp_?sizeHint@QBoxLayout@@UBE?AVQSize@@XZ 100195dc     Qt5Widgets:Qt5Widgets.dll
 0002:000005e0       __imp_?sizeHint@QCheckBox@@UBE?AVQSize@@XZ 100195e0     Qt5Widgets:Qt5Widgets.dll
 0002:000005e4       __imp_?sizeHint@QDialog@@UBE?AVQSize@@XZ 100195e4     Qt5Widgets:Qt5Widgets.dll
 0002:000005e8       __imp_?sizeHint@QGridLayout@@UBE?AVQSize@@XZ 100195e8     Qt5Widgets:Qt5Widgets.dll
 0002:000005ec       __imp_?sizeHint@QLabel@@UBE?AVQSize@@XZ 100195ec     Qt5Widgets:Qt5Widgets.dll
 0002:000005f0       __imp_?sizeHint@QLineEdit@@UBE?AVQSize@@XZ 100195f0     Qt5Widgets:Qt5Widgets.dll
 0002:000005f4       __imp_?sizeHint@QRadioButton@@UBE?AVQSize@@XZ 100195f4     Qt5Widgets:Qt5Widgets.dll
 0002:000005f8       __imp_?sizeHint@QToolButton@@UBE?AVQSize@@XZ 100195f8     Qt5Widgets:Qt5Widgets.dll
 0002:000005fc       __imp_?sizeHint@QWidget@@UBE?AVQSize@@XZ 100195fc     Qt5Widgets:Qt5Widgets.dll
 0002:00000600       __imp_?spacerItem@QLayoutItem@@UAEPAVQSpacerItem@@XZ 10019600     Qt5Widgets:Qt5Widgets.dll
 0002:00000604       __imp_?tabletEvent@QWidget@@MAEXPAVQTabletEvent@@@Z 10019604     Qt5Widgets:Qt5Widgets.dll
 0002:00000608       __imp_?takeAt@QBoxLayout@@UAEPAVQLayoutItem@@H@Z 10019608     Qt5Widgets:Qt5Widgets.dll
 0002:0000060c       __imp_?takeAt@QGridLayout@@UAEPAVQLayoutItem@@H@Z 1001960c     Qt5Widgets:Qt5Widgets.dll
 0002:00000610       __imp_?timerEvent@QAbstractButton@@MAEXPAVQTimerEvent@@@Z 10019610     Qt5Widgets:Qt5Widgets.dll
 0002:00000614       __imp_?timerEvent@QToolButton@@MAEXPAVQTimerEvent@@@Z 10019614     Qt5Widgets:Qt5Widgets.dll
 0002:00000618       __imp_?wheelEvent@QWidget@@MAEXPAVQWheelEvent@@@Z 10019618     Qt5Widgets:Qt5Widgets.dll
 0002:0000061c       __imp_?widget@QLayoutItem@@UAEPAVQWidget@@XZ 1001961c     Qt5Widgets:Qt5Widgets.dll
 0002:00000620       __imp_?addAction@QWidget@@QAEXPAVQAction@@@Z 10019620     Qt5Widgets:Qt5Widgets.dll
 0002:00000624       __imp_??1QAction@@UAE@XZ   10019624     Qt5Widgets:Qt5Widgets.dll
 0002:00000628       __imp_?event@QAction@@MAE_NPAVQEvent@@@Z 10019628     Qt5Widgets:Qt5Widgets.dll
 0002:0000062c       __imp_?setEnabled@QWidget@@QAEX_N@Z 1001962c     Qt5Widgets:Qt5Widgets.dll
 0002:00000630       __imp_?setTabOrder@QWidget@@SAXPAV1@0@Z 10019630     Qt5Widgets:Qt5Widgets.dll
 0002:00000634       __imp_??0QSpacerItem@@QAE@HHW4Policy@QSizePolicy@@0@Z 10019634     Qt5Widgets:Qt5Widgets.dll
 0002:00000638       __imp_??1QSpacerItem@@UAE@XZ 10019638     Qt5Widgets:Qt5Widgets.dll
 0002:0000063c       __imp_?addLayout@QBoxLayout@@QAEXPAVQLayout@@H@Z 1001963c     Qt5Widgets:Qt5Widgets.dll
 0002:00000640       __imp_?setStretch@QBoxLayout@@QAEXHH@Z 10019640     Qt5Widgets:Qt5Widgets.dll
 0002:00000644       __imp_??0QHBoxLayout@@QAE@XZ 10019644     Qt5Widgets:Qt5Widgets.dll
 0002:00000648       __imp_??1QHBoxLayout@@UAE@XZ 10019648     Qt5Widgets:Qt5Widgets.dll
 0002:0000064c       __imp_??0QComboBox@@QAE@PAVQWidget@@@Z 1001964c     Qt5Widgets:Qt5Widgets.dll
 0002:00000650       __imp_??1QComboBox@@UAE@XZ 10019650     Qt5Widgets:Qt5Widgets.dll
 0002:00000654       __imp_?count@QComboBox@@QBEHXZ 10019654     Qt5Widgets:Qt5Widgets.dll
 0002:00000658       __imp_?currentData@QComboBox@@QBE?AVQVariant@@H@Z 10019658     Qt5Widgets:Qt5Widgets.dll
 0002:0000065c       __imp_?insertItem@QComboBox@@QAEXHABVQIcon@@ABVQString@@ABVQVariant@@@Z 1001965c     Qt5Widgets:Qt5Widgets.dll
 0002:00000660       __imp_?changeEvent@QComboBox@@MAEXPAVQEvent@@@Z 10019660     Qt5Widgets:Qt5Widgets.dll
 0002:00000664       __imp_?contextMenuEvent@QComboBox@@MAEXPAVQContextMenuEvent@@@Z 10019664     Qt5Widgets:Qt5Widgets.dll
 0002:00000668       __imp_?controlTypes@QLayoutItem@@UBE?AV?$QFlags@W4ControlType@QSizePolicy@@@@XZ 10019668     Qt5Widgets:Qt5Widgets.dll
 0002:0000066c       __imp_?event@QComboBox@@UAE_NPAVQEvent@@@Z 1001966c     Qt5Widgets:Qt5Widgets.dll
 0002:00000670       __imp_?expandingDirections@QSpacerItem@@UBE?AV?$QFlags@W4Orientation@Qt@@@@XZ 10019670     Qt5Widgets:Qt5Widgets.dll
 0002:00000674       __imp_?focusInEvent@QComboBox@@MAEXPAVQFocusEvent@@@Z 10019674     Qt5Widgets:Qt5Widgets.dll
 0002:00000678       __imp_?focusOutEvent@QComboBox@@MAEXPAVQFocusEvent@@@Z 10019678     Qt5Widgets:Qt5Widgets.dll
 0002:0000067c       __imp_?geometry@QSpacerItem@@UBE?AVQRect@@XZ 1001967c     Qt5Widgets:Qt5Widgets.dll
 0002:00000680       __imp_?hasHeightForWidth@QLayoutItem@@UBE_NXZ 10019680     Qt5Widgets:Qt5Widgets.dll
 0002:00000684       __imp_?heightForWidth@QLayoutItem@@UBEHH@Z 10019684     Qt5Widgets:Qt5Widgets.dll
 0002:00000688       __imp_?hideEvent@QComboBox@@MAEXPAVQHideEvent@@@Z 10019688     Qt5Widgets:Qt5Widgets.dll
 0002:0000068c       __imp_?hidePopup@QComboBox@@UAEXXZ 1001968c     Qt5Widgets:Qt5Widgets.dll
 0002:00000690       __imp_?inputMethodEvent@QComboBox@@MAEXPAVQInputMethodEvent@@@Z 10019690     Qt5Widgets:Qt5Widgets.dll
 0002:00000694       __imp_?inputMethodQuery@QComboBox@@UBE?AVQVariant@@W4InputMethodQuery@Qt@@@Z 10019694     Qt5Widgets:Qt5Widgets.dll
 0002:00000698       __imp_?invalidate@QLayoutItem@@UAEXXZ 10019698     Qt5Widgets:Qt5Widgets.dll
 0002:0000069c       __imp_?isEmpty@QSpacerItem@@UBE_NXZ 1001969c     Qt5Widgets:Qt5Widgets.dll
 0002:000006a0       __imp_?keyPressEvent@QComboBox@@MAEXPAVQKeyEvent@@@Z 100196a0     Qt5Widgets:Qt5Widgets.dll
 0002:000006a4       __imp_?keyReleaseEvent@QComboBox@@MAEXPAVQKeyEvent@@@Z 100196a4     Qt5Widgets:Qt5Widgets.dll
 0002:000006a8       __imp_?layout@QLayoutItem@@UAEPAVQLayout@@XZ 100196a8     Qt5Widgets:Qt5Widgets.dll
 0002:000006ac       __imp_?maximumSize@QSpacerItem@@UBE?AVQSize@@XZ 100196ac     Qt5Widgets:Qt5Widgets.dll
 0002:000006b0       __imp_?metaObject@QComboBox@@UBEPBUQMetaObject@@XZ 100196b0     Qt5Widgets:Qt5Widgets.dll
 0002:000006b4       __imp_?metaObject@QHBoxLayout@@UBEPBUQMetaObject@@XZ 100196b4     Qt5Widgets:Qt5Widgets.dll
 0002:000006b8       __imp_?minimumHeightForWidth@QLayoutItem@@UBEHH@Z 100196b8     Qt5Widgets:Qt5Widgets.dll
 0002:000006bc       __imp_?minimumSize@QSpacerItem@@UBE?AVQSize@@XZ 100196bc     Qt5Widgets:Qt5Widgets.dll
 0002:000006c0       __imp_?minimumSizeHint@QComboBox@@UBE?AVQSize@@XZ 100196c0     Qt5Widgets:Qt5Widgets.dll
 0002:000006c4       __imp_?mousePressEvent@QComboBox@@MAEXPAVQMouseEvent@@@Z 100196c4     Qt5Widgets:Qt5Widgets.dll
 0002:000006c8       __imp_?mouseReleaseEvent@QComboBox@@MAEXPAVQMouseEvent@@@Z 100196c8     Qt5Widgets:Qt5Widgets.dll
 0002:000006cc       __imp_?paintEvent@QComboBox@@MAEXPAVQPaintEvent@@@Z 100196cc     Qt5Widgets:Qt5Widgets.dll
 0002:000006d0       __imp_?qt_metacall@QComboBox@@UAEHW4Call@QMetaObject@@HPAPAX@Z 100196d0     Qt5Widgets:Qt5Widgets.dll
 0002:000006d4       __imp_?qt_metacall@QHBoxLayout@@UAEHW4Call@QMetaObject@@HPAPAX@Z 100196d4     Qt5Widgets:Qt5Widgets.dll
 0002:000006d8       __imp_?qt_metacast@QComboBox@@UAEPAXPBD@Z 100196d8     Qt5Widgets:Qt5Widgets.dll
 0002:000006dc       __imp_?qt_metacast@QHBoxLayout@@UAEPAXPBD@Z 100196dc     Qt5Widgets:Qt5Widgets.dll
 0002:000006e0       __imp_?resizeEvent@QComboBox@@MAEXPAVQResizeEvent@@@Z 100196e0     Qt5Widgets:Qt5Widgets.dll
 0002:000006e4       __imp_?setGeometry@QSpacerItem@@UAEXABVQRect@@@Z 100196e4     Qt5Widgets:Qt5Widgets.dll
 0002:000006e8       __imp_?showEvent@QComboBox@@MAEXPAVQShowEvent@@@Z 100196e8     Qt5Widgets:Qt5Widgets.dll
 0002:000006ec       __imp_?showPopup@QComboBox@@UAEXXZ 100196ec     Qt5Widgets:Qt5Widgets.dll
 0002:000006f0       __imp_?sizeHint@QComboBox@@UBE?AVQSize@@XZ 100196f0     Qt5Widgets:Qt5Widgets.dll
 0002:000006f4       __imp_?sizeHint@QSpacerItem@@UBE?AVQSize@@XZ 100196f4     Qt5Widgets:Qt5Widgets.dll
 0002:000006f8       __imp_?spacerItem@QSpacerItem@@UAEPAV1@XZ 100196f8     Qt5Widgets:Qt5Widgets.dll
 0002:000006fc       __imp_?wheelEvent@QComboBox@@MAEXPAVQWheelEvent@@@Z 100196fc     Qt5Widgets:Qt5Widgets.dll
 0002:00000700       __imp_?qt_metacast@QDialog@@UAEPAXPBD@Z 10019700     Qt5Widgets:Qt5Widgets.dll
 0002:00000704       __imp_?qt_metacall@QDialog@@UAEHW4Call@QMetaObject@@HPAPAX@Z 10019704     Qt5Widgets:Qt5Widgets.dll
 0002:00000708       __imp_?staticMetaObject@QDialog@@2UQMetaObject@@B 10019708     Qt5Widgets:Qt5Widgets.dll
 0002:0000070c       __imp_?staticMetaObject@QMenu@@2UQMetaObject@@B 1001970c     Qt5Widgets:Qt5Widgets.dll
 0002:00000710       __imp_?setText@QAbstractButton@@QAEXABVQString@@@Z 10019710     Qt5Widgets:Qt5Widgets.dll
 0002:00000714       __imp_?critical@QMessageBox@@SA?AW4StandardButton@1@PAVQWidget@@ABVQString@@1V?$QFlags@W4StandardButton@QMessageBox@@@@W421@@Z 10019714     Qt5Widgets:Qt5Widgets.dll
 0002:00000718       __imp_?minimumSizeHint@QWidget@@UBE?AVQSize@@XZ 10019718     Qt5Widgets:Qt5Widgets.dll
 0002:0000071c       __imp_?accept@QDialog@@UAEXXZ 1001971c     Qt5Widgets:Qt5Widgets.dll
 0002:00000720       __imp_??0QDialog@@QAE@PAVQWidget@@V?$QFlags@W4WindowType@Qt@@@@@Z 10019720     Qt5Widgets:Qt5Widgets.dll
 0002:00000724       __imp_?resize@QWidget@@QAEXABVQSize@@@Z 10019724     Qt5Widgets:Qt5Widgets.dll
 0002:00000728       __imp_?setWindowIcon@QWidget@@QAEXABVQIcon@@@Z 10019728     Qt5Widgets:Qt5Widgets.dll
 0002:0000072c       __imp_?setWindowTitle@QWidget@@QAEXABVQString@@@Z 1001972c     Qt5Widgets:Qt5Widgets.dll
 0002:00000730       __imp_?event@QDialogButtonBox@@MAE_NPAVQEvent@@@Z 10019730     Qt5Widgets:Qt5Widgets.dll
 0002:00000734       \177Qt5Widgets_NULL_THUNK_DATA 10019734     Qt5Widgets:Qt5Widgets.dll
 0002:00000738       __imp_?getAlgorithmFactory@MSADistanceAlgorithmRegistry@U2@@QAEPAVMSADistanceAlgorithmFactory@2@ABVQString@@@Z 10019738     U2Algorithm:U2Algorithm.dll
 0002:0000073c       __imp_?resetFlag@MSADistanceAlgorithmFactory@U2@@QAEXW4DistanceAlgorithmFlag@2@@Z 1001973c     U2Algorithm:U2Algorithm.dll
 0002:00000740       __imp_?getSimilarity@MSADistanceAlgorithm@U2@@QAEHHH_N@Z 10019740     U2Algorithm:U2Algorithm.dll
 0002:00000744       __imp_?getAlgorithmFactories@MSADistanceAlgorithmRegistry@U2@@QBE?AV?$QList@PAVMSADistanceAlgorithmFactory@U2@@@@XZ 10019744     U2Algorithm:U2Algorithm.dll
 0002:00000748       __imp_?staticMetaObject@MSADistanceAlgorithm@U2@@2UQMetaObject@@B 10019748     U2Algorithm:U2Algorithm.dll
 0002:0000074c       __imp_?getId@MSADistanceAlgorithmFactory@U2@@QBE?AVQString@@XZ 1001974c     U2Algorithm:U2Algorithm.dll
 0002:00000750       __imp_?setFlag@MSADistanceAlgorithmFactory@U2@@QAEXW4DistanceAlgorithmFlag@2@@Z 10019750     U2Algorithm:U2Algorithm.dll
 0002:00000754       \177U2Algorithm_NULL_THUNK_DATA 10019754     U2Algorithm:U2Algorithm.dll
 0002:00000758       __imp_?getAlphabet@MultipleAlignmentData@U2@@QBEPBVDNAAlphabet@2@XZ 10019758     U2Core:U2Core.dll
 0002:0000075c       __imp_?getLength@MultipleAlignmentData@U2@@QBEHXZ 1001975c     U2Core:U2Core.dll
 0002:00000760       __imp_??0Logger@U2@@QAE@ABVQString@@@Z 10019760     U2Core:U2Core.dll
 0002:00000764       __imp_??1Logger@U2@@UAE@XZ 10019764     U2Core:U2Core.dll
 0002:00000768       __imp_??CMultipleSequenceAlignmentRow@U2@@QAEPAVMultipleSequenceAlignmentRowData@1@XZ 10019768     U2Core:U2Core.dll
 0002:0000076c       __imp_??1MultipleSequenceAlignmentRow@U2@@UAE@XZ 1001976c     U2Core:U2Core.dll
 0002:00000770       __imp_??0MultipleSequenceAlignment@U2@@QAE@ABVQString@@PBVDNAAlphabet@1@ABV?$QList@VMultipleSequenceAlignmentRow@U2@@@@@Z 10019770     U2Core:U2Core.dll
 0002:00000774       __imp_??CMultipleSequenceAlignment@U2@@QAEPAVMultipleSequenceAlignmentData@1@XZ 10019774     U2Core:U2Core.dll
 0002:00000778       __imp_??1MultipleSequenceAlignment@U2@@UAE@XZ 10019778     U2Core:U2Core.dll
 0002:0000077c       __imp_??0MultipleSequenceAlignment@U2@@QAE@ABV01@@Z 1001977c     U2Core:U2Core.dll
 0002:00000780       __imp_??4MultipleSequenceAlignment@U2@@QAEAAV01@ABV01@@Z 10019780     U2Core:U2Core.dll
 0002:00000784       __imp_?getNumRows@MultipleSequenceAlignmentData@U2@@QBEHXZ 10019784     U2Core:U2Core.dll
 0002:00000788       __imp_?getMsaRow@MultipleSequenceAlignmentData@U2@@QAE?AVMultipleSequenceAlignmentRow@2@H@Z 10019788     U2Core:U2Core.dll
 0002:0000078c       __imp_?getMsaCopy@MultipleSequenceAlignmentObject@U2@@QBE?BVMultipleSequenceAlignment@2@XZ 1001978c     U2Core:U2Core.dll
 0002:00000790       __imp_??0Task@U2@@QAE@ABVQString@@V?$QFlags@W4TaskFlag@U2@@@@@Z 10019790     U2Core:U2Core.dll
 0002:00000794       __imp_?hasError@Task@U2@@QBE_NXZ 10019794     U2Core:U2Core.dll
 0002:00000798       __imp_?getError@Task@U2@@QBE?AVQString@@XZ 10019798     U2Core:U2Core.dll
 0002:0000079c       __imp_?setVerboseLogMode@Task@U2@@QAEX_N@Z 1001979c     U2Core:U2Core.dll
 0002:000007a0       __imp_?setError@Task@U2@@QAEXABVQString@@@Z 100197a0     U2Core:U2Core.dll
 0002:000007a4       __imp_??1Task@U2@@UAE@XZ   100197a4     U2Core:U2Core.dll
 0002:000007a8       __imp_?cleanup@Task@U2@@UAEXXZ 100197a8     U2Core:U2Core.dll
 0002:000007ac       __imp_?getNumParallelSubtasks@Task@U2@@UBEHXZ 100197ac     U2Core:U2Core.dll
 0002:000007b0       __imp_?getParentTask@Task@U2@@UBEPAV12@XZ 100197b0     U2Core:U2Core.dll
 0002:000007b4       __imp_?getSubtaskWithErrors@Task@U2@@UBEPAV12@XZ 100197b4     U2Core:U2Core.dll
 0002:000007b8       __imp_?getTaskId@Task@U2@@UBE_JXZ 100197b8     U2Core:U2Core.dll
 0002:000007bc       __imp_?getTopLevelParentTask@Task@U2@@UAEPAV12@XZ 100197bc     U2Core:U2Core.dll
 0002:000007c0       __imp_?getWarnings@Task@U2@@UBE?AVQStringList@@XZ 100197c0     U2Core:U2Core.dll
 0002:000007c4       __imp_?hasSubtasksWithErrors@Task@U2@@UBE_NXZ 100197c4     U2Core:U2Core.dll
 0002:000007c8       __imp_?hasWarning@Task@U2@@UBE_NXZ 100197c8     U2Core:U2Core.dll
 0002:000007cc       __imp_?isNotificationReport@Task@U2@@UBE_NXZ 100197cc     U2Core:U2Core.dll
 0002:000007d0       __imp_?isReportingSupported@Task@U2@@UBE_NXZ 100197d0     U2Core:U2Core.dll
 0002:000007d4       __imp_?isTopLevelTask@Task@U2@@UBE_NXZ 100197d4     U2Core:U2Core.dll
 0002:000007d8       __imp_?onSubTaskFinished@Task@U2@@MAE?AV?$QList@PAVTask@U2@@@@PAV12@@Z 100197d8     U2Core:U2Core.dll
 0002:000007dc       __imp_??1MultipleAlignment@U2@@UAE@XZ 100197dc     U2Core:U2Core.dll
 0002:000007e0       __imp_?propagateSubtaskError@Task@U2@@UAE_NXZ 100197e0     U2Core:U2Core.dll
 0002:000007e4       __imp_?setCollectChildrensWarningsFlag@Task@U2@@UAEX_N@Z 100197e4     U2Core:U2Core.dll
 0002:000007e8       __imp_?setNoAutoDelete@Task@U2@@UAEX_N@Z 100197e8     U2Core:U2Core.dll
 0002:000007ec       __imp_?setNotificationReport@Task@U2@@UAEX_N@Z 100197ec     U2Core:U2Core.dll
 0002:000007f0       __imp_?setReportingEnabled@Task@U2@@UAEX_N@Z 100197f0     U2Core:U2Core.dll
 0002:000007f4       __imp_?setReportingSupported@Task@U2@@UAEX_N@Z 100197f4     U2Core:U2Core.dll
 0002:000007f8       __imp_?GAP_CHAR@U2Msa@U2@@2DB 100197f8     U2Core:U2Core.dll
 0002:000007fc       __imp_?error@Logger@U2@@QAEXABVQString@@@Z 100197fc     U2Core:U2Core.dll
 0002:00000800       __imp_??0Plugin@U2@@QAE@ABVQString@@0_NW4PluginState@1@@Z 10019800     U2Core:U2Core.dll
 0002:00000804       __imp_??1Plugin@U2@@UAE@XZ 10019804     U2Core:U2Core.dll
 0002:00000808       __imp_??1U2EntityRef@U2@@QAE@XZ 10019808     U2Core:U2Core.dll
 0002:0000080c       __imp_?getAlphabet@U2SequenceObject@U2@@QBEPBVDNAAlphabet@2@XZ 1001980c     U2Core:U2Core.dll
 0002:00000810       __imp_?addSubTask@Task@U2@@QAEXPAV12@@Z 10019810     U2Core:U2Core.dll
 0002:00000814       __imp_?generateReport@Task@U2@@UBE?AVQString@@XZ 10019814     U2Core:U2Core.dll
 0002:00000818       __imp_?isReportingEnabled@Task@U2@@UBE_NXZ 10019818     U2Core:U2Core.dll
 0002:0000081c       __imp_?metaObject@Task@U2@@UBEPBUQMetaObject@@XZ 1001981c     U2Core:U2Core.dll
 0002:00000820       __imp_?qt_metacall@Task@U2@@UAEHW4Call@QMetaObject@@HPAPAX@Z 10019820     U2Core:U2Core.dll
 0002:00000824       __imp_?qt_metacast@Task@U2@@UAEPAXPBD@Z 10019824     U2Core:U2Core.dll
 0002:00000828       __imp_?report@Task@U2@@UAE?AW4ReportResult@12@XZ 10019828     U2Core:U2Core.dll
 0002:0000082c       __imp_?run@Task@U2@@UAEXXZ 1001982c     U2Core:U2Core.dll
 0002:00000830       __imp_??CMultipleSequenceAlignmentRow@U2@@QBEPBVMultipleSequenceAlignmentRowData@1@XZ 10019830     U2Core:U2Core.dll
 0002:00000834       __imp_??0MultipleSequenceAlignmentRow@U2@@QAE@ABV01@@Z 10019834     U2Core:U2Core.dll
 0002:00000838       __imp_?getExplicitCopy@MultipleSequenceAlignmentRowData@U2@@QBE?AVMultipleSequenceAlignmentRow@2@XZ 10019838     U2Core:U2Core.dll
 0002:0000083c       __imp_?sortRowsBySimilarity@MultipleSequenceAlignmentData@U2@@QAE_NAAV?$QVector@VU2Region@U2@@@@@Z 1001983c     U2Core:U2Core.dll
 0002:00000840       __imp_?getMsaRows@MultipleSequenceAlignmentData@U2@@QBE?BV?$QList@VMultipleSequenceAlignmentRow@U2@@@@XZ 10019840     U2Core:U2Core.dll
 0002:00000844       __imp_?getMSADistanceAlgorithmRegistry@AppContext@U2@@SAPAVMSADistanceAlgorithmRegistry@2@XZ 10019844     U2Core:U2Core.dll
 0002:00000848       __imp_?wrapForCSV@TextUtils@U2@@SAXAAVQString@@@Z 10019848     U2Core:U2Core.dll
 0002:0000084c       __imp_?staticMetaObject@Task@U2@@2UQMetaObject@@B 1001984c     U2Core:U2Core.dll
 0002:00000850       __imp_?qt_metacast@Plugin@U2@@UAEPAXPBD@Z 10019850     U2Core:U2Core.dll
 0002:00000854       __imp_?qt_metacall@Plugin@U2@@UAEHW4Call@QMetaObject@@HPAPAX@Z 10019854     U2Core:U2Core.dll
 0002:00000858       __imp_?staticMetaObject@Plugin@U2@@2UQMetaObject@@B 10019858     U2Core:U2Core.dll
 0002:0000085c       __imp_??1MultipleAlignmentRow@U2@@UAE@XZ 1001985c     U2Core:U2Core.dll
 0002:00000860       __imp_?fixFileName@GUrlUtils@U2@@SA?AVQString@@ABV3@@Z 10019860     U2Core:U2Core.dll
 0002:00000864       __imp_?getDefaultDataPath@GUrlUtils@U2@@SA?AVQString@@XZ 10019864     U2Core:U2Core.dll
 0002:00000868       __imp_?dumpStringToFile@FileAndDirectoryUtils@U2@@SAXPAVQFile@@AAVQString@@@Z 10019868     U2Core:U2Core.dll
 0002:0000086c       __imp_?getMainWindow@AppContext@U2@@SAPAVMainWindow@2@XZ 1001986c     U2Core:U2Core.dll
 0002:00000870       __imp_?getAlphabetChars@DNAAlphabet@U2@@QBE?AVQByteArray@@_N@Z 10019870     U2Core:U2Core.dll
 0002:00000874       __imp_?getTaskScheduler@AppContext@U2@@SAPAVTaskScheduler@2@XZ 10019874     U2Core:U2Core.dll
 0002:00000878       __imp_?prepare@Task@U2@@UAEXXZ 10019878     U2Core:U2Core.dll
 0002:0000087c       \177U2Core_NULL_THUNK_DATA 1001987c     U2Core:U2Core.dll
 0002:00000880       __imp_??0HelpButton@U2@@QAE@PAVQObject@@PAVQDialogButtonBox@@ABVQString@@@Z 10019880     U2Gui:U2Gui.dll
 0002:00000884       __imp_??1HelpButton@U2@@UAE@XZ 10019884     U2Gui:U2Gui.dll
 0002:00000888       __imp_??0LastUsedDirHelper@U2@@QAE@ABVQString@@0@Z 10019888     U2Gui:U2Gui.dll
 0002:0000088c       __imp_??1LastUsedDirHelper@U2@@UAE@XZ 1001988c     U2Gui:U2Gui.dll
 0002:00000890       __imp_??0SaveDocumentControllerConfig@U2@@QAE@XZ 10019890     U2Gui:U2Gui.dll
 0002:00000894       __imp_??1SaveDocumentControllerConfig@U2@@QAE@XZ 10019894     U2Gui:U2Gui.dll
 0002:00000898       __imp_?addFormat@SimpleFormatsInfo@SaveDocumentController@U2@@QAEXABVQString@@0ABVQStringList@@@Z 10019898     U2Gui:U2Gui.dll
 0002:0000089c       __imp_??0SimpleFormatsInfo@SaveDocumentController@U2@@QAE@XZ 1001989c     U2Gui:U2Gui.dll
 0002:000008a0       __imp_??1SimpleFormatsInfo@SaveDocumentController@U2@@QAE@XZ 100198a0     U2Gui:U2Gui.dll
 0002:000008a4       __imp_??0SaveDocumentController@U2@@QAE@ABVSaveDocumentControllerConfig@1@ABVSimpleFormatsInfo@01@PAVQObject@@@Z 100198a4     U2Gui:U2Gui.dll
 0002:000008a8       __imp_?setFormat@SaveDocumentController@U2@@QAEXABVQString@@@Z 100198a8     U2Gui:U2Gui.dll
 0002:000008ac       __imp_?getSaveFileName@SaveDocumentController@U2@@QBE?AVQString@@XZ 100198ac     U2Gui:U2Gui.dll
 0002:000008b0       __imp_??1SaveDocumentController@U2@@UAE@XZ 100198b0     U2Gui:U2Gui.dll
 0002:000008b4       __imp_??1MWMDIWindow@U2@@UAE@XZ 100198b4     U2Gui:U2Gui.dll
 0002:000008b8       __imp_?metaObject@HelpButton@U2@@UBEPBUQMetaObject@@XZ 100198b8     U2Gui:U2Gui.dll
 0002:000008bc       __imp_?metaObject@SaveDocumentController@U2@@UBEPBUQMetaObject@@XZ 100198bc     U2Gui:U2Gui.dll
 0002:000008c0       __imp_?onCloseEvent@MWMDIWindow@U2@@MAE_NXZ 100198c0     U2Gui:U2Gui.dll
 0002:000008c4       __imp_?qt_metacall@HelpButton@U2@@UAEHW4Call@QMetaObject@@HPAPAX@Z 100198c4     U2Gui:U2Gui.dll
 0002:000008c8       __imp_?qt_metacall@SaveDocumentController@U2@@UAEHW4Call@QMetaObject@@HPAPAX@Z 100198c8     U2Gui:U2Gui.dll
 0002:000008cc       __imp_?qt_metacast@HelpButton@U2@@UAEPAXPBD@Z 100198cc     U2Gui:U2Gui.dll
 0002:000008d0       __imp_?qt_metacast@SaveDocumentController@U2@@UAEPAXPBD@Z 100198d0     U2Gui:U2Gui.dll
 0002:000008d4       __imp_?setupMDIToolbar@MWMDIWindow@U2@@UAEXPAVQToolBar@@@Z 100198d4     U2Gui:U2Gui.dll
 0002:000008d8       __imp_?setupViewMenu@MWMDIWindow@U2@@UAEXPAVQMenu@@@Z 100198d8     U2Gui:U2Gui.dll
 0002:000008dc       __imp_?sl_buttonClicked@HelpButton@U2@@MAEXXZ 100198dc     U2Gui:U2Gui.dll
 0002:000008e0       __imp_?findSubMenu@GUIUtils@U2@@SAPAVQMenu@@PAV3@ABVQString@@@Z 100198e0     U2Gui:U2Gui.dll
 0002:000008e4       __imp_?getWidget@GObjectView@U2@@QAEPAVQWidget@@XZ 100198e4     U2Gui:U2Gui.dll
 0002:000008e8       __imp_??0GObjectViewAction@U2@@QAE@PAVQObject@@PAVGObjectView@1@ABVQString@@H@Z 100198e8     U2Gui:U2Gui.dll
 0002:000008ec       __imp_?getObjectView@GObjectViewAction@U2@@QBEPAVGObjectView@2@XZ 100198ec     U2Gui:U2Gui.dll
 0002:000008f0       __imp_??0GObjectViewWindowContext@U2@@QAE@PAVQObject@@ABVGObjectViewFactoryId@1@@Z 100198f0     U2Gui:U2Gui.dll
 0002:000008f4       __imp_??1GObjectViewWindowContext@U2@@UAE@XZ 100198f4     U2Gui:U2Gui.dll
 0002:000008f8       __imp_?getViewActions@GObjectViewWindowContext@U2@@QBE?AV?$QList@PAVGObjectViewAction@U2@@@@PAVGObjectView@2@@Z 100198f8     U2Gui:U2Gui.dll
 0002:000008fc       __imp_?addViewAction@GObjectViewWindowContext@U2@@IAEXPAVGObjectViewAction@2@@Z 100198fc     U2Gui:U2Gui.dll
 0002:00000900       __imp_?canHandle@GObjectViewObjectHandler@U2@@UAE_NPAVGObjectView@2@PAVGObject@2@@Z 10019900     U2Gui:U2Gui.dll
 0002:00000904       __imp_?disconnectView@GObjectViewWindowContext@U2@@MAEXPAVGObjectView@2@@Z 10019904     U2Gui:U2Gui.dll
 0002:00000908       __imp_?init@GObjectViewWindowContext@U2@@UAEXXZ 10019908     U2Gui:U2Gui.dll
 0002:0000090c       __imp_?metaObject@GObjectViewAction@U2@@UBEPBUQMetaObject@@XZ 1001990c     U2Gui:U2Gui.dll
 0002:00000910       __imp_?onObjectAdded@GObjectViewObjectHandler@U2@@UAEXPAVGObjectView@2@PAVGObject@2@@Z 10019910     U2Gui:U2Gui.dll
 0002:00000914       __imp_?onObjectRemoved@GObjectViewWindowContext@U2@@UAEXPAVGObjectView@2@PAVGObject@2@@Z 10019914     U2Gui:U2Gui.dll
 0002:00000918       __imp_?qt_metacall@GObjectViewAction@U2@@UAEHW4Call@QMetaObject@@HPAPAX@Z 10019918     U2Gui:U2Gui.dll
 0002:0000091c       __imp_?qt_metacast@GObjectViewAction@U2@@UAEPAXPBD@Z 1001991c     U2Gui:U2Gui.dll
 0002:00000920       __imp_?sl_buildContextMenu@GObjectViewWindowContext@U2@@MAEXPAVGObjectView@2@PAVQMenu@@@Z 10019920     U2Gui:U2Gui.dll
 0002:00000924       __imp_?sl_buildStaticMenu@GObjectViewWindowContext@U2@@MAEXPAVGObjectView@2@PAVQMenu@@@Z 10019924     U2Gui:U2Gui.dll
 0002:00000928       __imp_?sl_windowAdded@GObjectViewWindowContext@U2@@MAEXPAVMWMDIWindow@2@@Z 10019928     U2Gui:U2Gui.dll
 0002:0000092c       __imp_?sl_windowClosing@GObjectViewWindowContext@U2@@MAEXPAVMWMDIWindow@2@@Z 1001992c     U2Gui:U2Gui.dll
 0002:00000930       __imp_?staticMetaObject@GObjectViewAction@U2@@2UQMetaObject@@B 10019930     U2Gui:U2Gui.dll
 0002:00000934       __imp_?qt_metacast@GObjectViewWindowContext@U2@@UAEPAXPBD@Z 10019934     U2Gui:U2Gui.dll
 0002:00000938       __imp_?qt_metacall@GObjectViewWindowContext@U2@@UAEHW4Call@QMetaObject@@HPAPAX@Z 10019938     U2Gui:U2Gui.dll
 0002:0000093c       __imp_?staticMetaObject@GObjectView@U2@@2UQMetaObject@@B 1001993c     U2Gui:U2Gui.dll
 0002:00000940       __imp_?staticMetaObject@GObjectViewWindowContext@U2@@2UQMetaObject@@B 10019940     U2Gui:U2Gui.dll
 0002:00000944       \177U2Gui_NULL_THUNK_DATA  10019944     U2Gui:U2Gui.dll
 0002:00000948       __imp_??0WebWindow@U2@@QAE@ABVQString@@0@Z 10019948     U2View:U2View.dll
 0002:0000094c       __imp_?metaObject@WebWindow@U2@@UBEPBUQMetaObject@@XZ 1001994c     U2View:U2View.dll
 0002:00000950       __imp_?qt_metacall@WebWindow@U2@@UAEHW4Call@QMetaObject@@HPAPAX@Z 10019950     U2View:U2View.dll
 0002:00000954       __imp_?qt_metacast@WebWindow@U2@@UAEPAXPBD@Z 10019954     U2View:U2View.dll
 0002:00000958       __imp_?staticMetaObject@MSAEditor@U2@@2UQMetaObject@@B 10019958     U2View:U2View.dll
 0002:0000095c       __imp_?ID@MsaEditorFactory@U2@@2VGObjectViewFactoryId@2@B 1001995c     U2View:U2View.dll
 0002:00000960       __imp_?getResult@?$BackgroundTask@V?$QList@UCharOccurResult@U2@@@@@U2@@QBE?AV?$QList@UCharOccurResult@U2@@@@XZ 10019960     U2View:U2View.dll
 0002:00000964       __imp_??0CharOccurTask@U2@@QAE@PBVDNAAlphabet@1@VU2EntityRef@1@VU2Region@1@@Z 10019964     U2View:U2View.dll
 0002:00000968       __imp_??1CharOccurTask@U2@@UAE@XZ 10019968     U2View:U2View.dll
 0002:0000096c       __imp_?getResult@?$BackgroundTask@V?$QMap@VQByteArray@@_J@@@U2@@QBE?AV?$QMap@VQByteArray@@_J@@XZ 1001996c     U2View:U2View.dll
 0002:00000970       __imp_??0DinuclOccurTask@U2@@QAE@PBVDNAAlphabet@1@VU2EntityRef@1@VU2Region@1@@Z 10019970     U2View:U2View.dll
 0002:00000974       __imp_??1DinuclOccurTask@U2@@UAE@XZ 10019974     U2View:U2View.dll
 0002:00000978       __imp_??0DNAStatisticsTask@U2@@QAE@PBVDNAAlphabet@1@VU2EntityRef@1@ABVU2Region@1@@Z 10019978     U2View:U2View.dll
 0002:0000097c       __imp_??1DNAStatisticsTask@U2@@UAE@XZ 1001997c     U2View:U2View.dll
 0002:00000980       __imp_?getSequenceGObject@SequenceObjectContext@U2@@QBEPAVGObject@2@XZ 10019980     U2View:U2View.dll
 0002:00000984       __imp_?getSequenceLength@SequenceObjectContext@U2@@QBE_JXZ 10019984     U2View:U2View.dll
 0002:00000988       __imp_?getAlphabet@SequenceObjectContext@U2@@QBEPBVDNAAlphabet@2@XZ 10019988     U2View:U2View.dll
 0002:0000098c       __imp_?getSequenceRef@SequenceObjectContext@U2@@QBE?AVU2EntityRef@2@XZ 1001998c     U2View:U2View.dll
 0002:00000990       __imp_?metaObject@DNAStatisticsTask@U2@@UBEPBUQMetaObject@@XZ 10019990     U2View:U2View.dll
 0002:00000994       __imp_?qt_metacall@DNAStatisticsTask@U2@@UAEHW4Call@QMetaObject@@HPAPAX@Z 10019994     U2View:U2View.dll
 0002:00000998       __imp_?qt_metacast@DNAStatisticsTask@U2@@UAEPAXPBD@Z 10019998     U2View:U2View.dll
 0002:0000099c       __imp_?run@CharOccurTask@U2@@UAEXXZ 1001999c     U2View:U2View.dll
 0002:000009a0       __imp_?run@DNAStatisticsTask@U2@@UAEXXZ 100199a0     U2View:U2View.dll
 0002:000009a4       __imp_?run@DinuclOccurTask@U2@@UAEXXZ 100199a4     U2View:U2View.dll
 0002:000009a8       \177U2View_NULL_THUNK_DATA 100199a8     U2View:U2View.dll
 0002:000009ac       ___xc_a                    100199ac     MSVCRT:cinitexe.obj
 0002:00000bec       ___xc_z                    10019bec     MSVCRT:cinitexe.obj
 0002:00000bf0       ___xi_a                    10019bf0     MSVCRT:cinitexe.obj
 0002:00000bfc       ___xi_z                    10019bfc     MSVCRT:cinitexe.obj
 0002:00000c3c       ??_7error_category@std@@6B@ 10019c3c     DNAStatMSAProfileDialog.obj
 0002:00000c58       ??_7_Generic_error_category@std@@6B@ 10019c58     DNAStatMSAProfileDialog.obj
 0002:00000c70       ??_C@_07DCLBNMLN@generic?$AA@ 10019c70     DNAStatMSAProfileDialog.obj
 0002:00000c78       ??_C@_0O@BFJCFAAK@unknown?5error?$AA@ 10019c78     DNAStatMSAProfileDialog.obj
 0002:00000c8c       ??_7_Iostream_error_category@std@@6B@ 10019c8c     DNAStatMSAProfileDialog.obj
 0002:00000ca4       ??_C@_08LLGCOLLL@iostream?$AA@ 10019ca4     DNAStatMSAProfileDialog.obj
 0002:00000cb0       ??_C@_0BG@PADBLCHM@iostream?5stream?5error?$AA@ 10019cb0     DNAStatMSAProfileDialog.obj
 0002:00000ccc       ??_7_System_error_category@std@@6B@ 10019ccc     DNAStatMSAProfileDialog.obj
 0002:00000ce4       ??_C@_06FHFOAHML@system?$AA@ 10019ce4     DNAStatMSAProfileDialog.obj
 0002:00000cf4       ??_SQFile@@6B@             10019cf4     DNAStatMSAProfileDialog.obj
 0002:00000d74       ??_7?$AbstractId@H@U2@@6B@ 10019d74     DNAStatMSAProfileDialog.obj
 0002:00000d80       ??_7AbstractInt32Id@U2@@6B@ 10019d80     DNAStatMSAProfileDialog.obj
 0002:00000d8c       ??_7ServiceType@U2@@6B@    10019d8c     DNAStatMSAProfileDialog.obj
 0002:00000d94       ??_C@_0L@JLHNEGIN@Algorithms?$AA@ 10019d94     DNAStatMSAProfileDialog.obj
 0002:00000da0       ??_C@_07PGLPGHFC@Console?$AA@ 10019da0     DNAStatMSAProfileDialog.obj
 0002:00000da8       ??_C@_0O@BOFHOPCF@Core?5Services?$AA@ 10019da8     DNAStatMSAProfileDialog.obj
 0002:00000db8       ??_C@_0N@PPADAKBM@Input?1Output?$AA@ 10019db8     DNAStatMSAProfileDialog.obj
 0002:00000dc8       ??_C@_0M@KPPBKPKK@Performance?$AA@ 10019dc8     DNAStatMSAProfileDialog.obj
 0002:00000dd4       ??_C@_07BFDHHBBI@Scripts?$AA@ 10019dd4     DNAStatMSAProfileDialog.obj
 0002:00000ddc       ??_C@_05EEGKELMG@Tasks?$AA@ 10019ddc     DNAStatMSAProfileDialog.obj
 0002:00000de4       ??_C@_0P@NIIOBHGA@User?5Interface?$AA@ 10019de4     DNAStatMSAProfileDialog.obj
 0002:00000df4       ??_C@_0N@JINCGGMN@User?5Actions?$AA@ 10019df4     DNAStatMSAProfileDialog.obj
 0002:00000e0c       ??_SQDialogButtonBox@@6BQObject@@@ 10019e0c     DNAStatMSAProfileDialog.obj
 0002:00000ec4       ??_SQDialogButtonBox@@6BQPaintDevice@@@ 10019ec4     DNAStatMSAProfileDialog.obj
 0002:00000ee4       ??_SHelpButton@U2@@6B@     10019ee4     DNAStatMSAProfileDialog.obj
 0002:00000f18       ??_SSaveDocumentController@U2@@6B@ 10019f18     DNAStatMSAProfileDialog.obj
 0002:00000f4c       ??_SQLabel@@6BQObject@@@   10019f4c     DNAStatMSAProfileDialog.obj
 0002:00001004       ??_SQLabel@@6BQPaintDevice@@@ 1001a004     DNAStatMSAProfileDialog.obj
 0002:00001024       ??_SWebWindow@U2@@6BQObject@@@ 1001a024     DNAStatMSAProfileDialog.obj
 0002:000010e8       ??_SWebWindow@U2@@6BQPaintDevice@@@ 1001a0e8     DNAStatMSAProfileDialog.obj
 0002:0000110c       ??_SQCheckBox@@6BQObject@@@ 1001a10c     DNAStatMSAProfileDialog.obj
 0002:000011d0       ??_SQCheckBox@@6BQPaintDevice@@@ 1001a1d0     DNAStatMSAProfileDialog.obj
 0002:000011f4       ??_SQVBoxLayout@@6BQObject@@@ 1001a1f4     DNAStatMSAProfileDialog.obj
 0002:0000123c       ??_SQVBoxLayout@@6BQLayoutItem@@@ 1001a23c     DNAStatMSAProfileDialog.obj
 0002:00001284       ??_SQGridLayout@@6BQObject@@@ 1001a284     DNAStatMSAProfileDialog.obj
 0002:000012cc       ??_SQGridLayout@@6BQLayoutItem@@@ 1001a2cc     DNAStatMSAProfileDialog.obj
 0002:00001314       ??_SQGroupBox@@6BQObject@@@ 1001a314     DNAStatMSAProfileDialog.obj
 0002:000013cc       ??_SQGroupBox@@6BQPaintDevice@@@ 1001a3cc     DNAStatMSAProfileDialog.obj
 0002:000013ec       ??_SQLineEdit@@6BQObject@@@ 1001a3ec     DNAStatMSAProfileDialog.obj
 0002:000014a4       ??_SQLineEdit@@6BQPaintDevice@@@ 1001a4a4     DNAStatMSAProfileDialog.obj
 0002:000014c4       ??_SQRadioButton@@6BQObject@@@ 1001a4c4     DNAStatMSAProfileDialog.obj
 0002:00001588       ??_SQRadioButton@@6BQPaintDevice@@@ 1001a588     DNAStatMSAProfileDialog.obj
 0002:000015ac       ??_SQToolButton@@6BQObject@@@ 1001a5ac     DNAStatMSAProfileDialog.obj
 0002:00001670       ??_SQToolButton@@6BQPaintDevice@@@ 1001a670     DNAStatMSAProfileDialog.obj
 0002:0000168c       ??_C@_09DMINLBG@1accept?$CI?$CJ?$AA@ 1001a68c     DNAStatMSAProfileDialog.obj
 0002:00001698       ??_C@_0M@MBACPLBI@2accepted?$CI?$CJ?$AA@ 1001a698     DNAStatMSAProfileDialog.obj
 0002:000016a4       ??_C@_09OCDCAEKE@1reject?$CI?$CJ?$AA@ 1001a6a4     DNAStatMSAProfileDialog.obj
 0002:000016b0       ??_C@_0M@BJNBJJN@2rejected?$CI?$CJ?$AA@ 1001a6b0     DNAStatMSAProfileDialog.obj
 0002:000016bc       ??_C@_0BL@FIFFIGDP@Generate?5Alignment?5Profile?$AA@ 1001a6bc     DNAStatMSAProfileDialog.obj
 0002:000016d8       ??_C@_0BI@PDEICGEI@DNAStatMSAProfileDialog?$AA@ 1001a6d8     DNAStatMSAProfileDialog.obj
 0002:000016f0       ??_C@_0N@NCLAMLGG@Profile?5mode?$AA@ 1001a6f0     DNAStatMSAProfileDialog.obj
 0002:00001700       ??_C@_05IJGIMMHE@Count?$AA@ 1001a700     DNAStatMSAProfileDialog.obj
 0002:00001708       ??_C@_0L@GKJDIJEO@Percentage?$AA@ 1001a708     DNAStatMSAProfileDialog.obj
 0002:00001714       ??_C@_0P@BMPMOGPF@Custom?5options?$AA@ 1001a714     DNAStatMSAProfileDialog.obj
 0002:00001724       ??_C@_0BF@HJCLGAAJ@Show?5scores?5for?5gaps?$AA@ 1001a724     DNAStatMSAProfileDialog.obj
 0002:0000173c       ??_C@_0CO@MPDDNDLJ@Show?5scores?5for?5symbols?5not?5used@ 1001a73c     DNAStatMSAProfileDialog.obj
 0002:0000176c       ??_C@_0CL@MGGCOGOM@Skip?5gaps?5in?5consensus?5position?5@ 1001a76c     DNAStatMSAProfileDialog.obj
 0002:00001798       ??_C@_0BF@PMLJNFKC@Save?5profile?5to?5file?$AA@ 1001a798     DNAStatMSAProfileDialog.obj
 0002:000017b0       ??_C@_04PBAHLACE@File?$AA@ 1001a7b0     DNAStatMSAProfileDialog.obj
 0002:000017b8       ??_C@_03KHICJKCI@?4?4?4?$AA@ 1001a7b8     DNAStatMSAProfileDialog.obj
 0002:000017bc       ??_C@_0BD@FHHMANNL@Hypertext?5?5?$CI?4HTML?$CJ?$AA@ 1001a7bc     DNAStatMSAProfileDialog.obj
 0002:000017d0       ??_C@_0BI@HCJDPFEH@Comma?5separated?5?$CI?5?4CSV?$CJ?$AA@ 1001a7d0     DNAStatMSAProfileDialog.obj
 0002:00001adc       ??_7DNAStatMSAProfileDialog@U2@@6BQObject@@@ 1001aadc     DNAStatMSAProfileDialog.obj
 0002:00001ba8       ??_7DNAStatMSAProfileDialog@U2@@6BQPaintDevice@@@ 1001aba8     DNAStatMSAProfileDialog.obj
 0002:00001bc8       ??_7DNAStatMSAProfileTask@U2@@6B@ 1001abc8     DNAStatMSAProfileDialog.obj
 0002:00001c54       ??_C@_04PNIFHPHN@html?$AA@ 1001ac54     DNAStatMSAProfileDialog.obj
 0002:00001c5c       ??_C@_03NIPKHAHH@csv?$AA@  1001ac5c     DNAStatMSAProfileDialog.obj
 0002:00001c60       ??_C@_08ECIBIFMC@23331104?$AA@ 1001ac60     DNAStatMSAProfileDialog.obj
 0002:00001c6c       ??_C@_02GIPFHKNO@OK?$AA@   1001ac6c     DNAStatMSAProfileDialog.obj
 0002:00001c70       ??_C@_06FMBNCPDL@Cancel?$AA@ 1001ac70     DNAStatMSAProfileDialog.obj
 0002:00001c78       ??_C@_0BA@GFHNPDJL@plugin_dna_stat?$AA@ 1001ac78     DNAStatMSAProfileDialog.obj
 0002:00001c88       ??_C@_01LFCBOECM@?4?$AA@   1001ac88     DNAStatMSAProfileDialog.obj
 0002:00001c8c       ??_C@_0O@JNEKMCPB@_grid_profile?$AA@ 1001ac8c     DNAStatMSAProfileDialog.obj
 0002:00001c9c       ??_C@_01KMDKNFGN@?1?$AA@   1001ac9c     DNAStatMSAProfileDialog.obj
 0002:00001ca0       ??_C@_09LIEIFGIE@Save?5file?$AA@ 1001aca0     DNAStatMSAProfileDialog.obj
 0002:00001cac       ??_C@_0CD@PNEKAAGJ@1sl_formatChanged?$CIconst?5QString?5@ 1001acac     DNAStatMSAProfileDialog.obj
 0002:00001cd0       ??_C@_0CD@JLKBONEP@2si_formatChanged?$CIconst?5QString?5@ 1001acd0     DNAStatMSAProfileDialog.obj
 0002:00001cf4       ??_C@_0BF@DPHBBMMI@1sl_formatSelected?$CI?$CJ?$AA@ 1001acf4     DNAStatMSAProfileDialog.obj
 0002:00001d0c       ??_C@_0P@POCECEMJ@2toggled?$CIbool?$CJ?$AA@ 1001ad0c     DNAStatMSAProfileDialog.obj
 0002:00001d1c       ??_C@_0BC@KJBBCNNI@File?5URL?5is?5empty?$AA@ 1001ad1c     DNAStatMSAProfileDialog.obj
 0002:00001d30       ??_C@_05NAOIJFC@Error?$AA@ 1001ad30     DNAStatMSAProfileDialog.obj
 0002:00001d38       ??_C@_0BL@PMGFFMFJ@Generate?5alignment?5profile?$AA@ 1001ad38     DNAStatMSAProfileDialog.obj
 0002:00001d54       ??_C@_0BO@EHEHGJKA@No?5output?5file?5name?5specified?$AA@ 1001ad54     DNAStatMSAProfileDialog.obj
 0002:00001d74       ??_C@_0BO@JJAOCCEM@Can?8t?5open?5file?5for?5write?3?5?$CF1?$AA@ 1001ad74     DNAStatMSAProfileDialog.obj
 0002:00001d94       ??_C@_07PFEKAKBD@?$CDff5555?$AA@ 1001ad94     DNAStatMSAProfileDialog.obj
 0002:00001d9c       ??_C@_07KFGAIBMC@?$CDff9c00?$AA@ 1001ad9c     DNAStatMSAProfileDialog.obj
 0002:00001da4       ??_C@_07NBPPCLLH@?$CD60ff00?$AA@ 1001ada4     DNAStatMSAProfileDialog.obj
 0002:00001dac       ??_C@_07MHMLFDEO@?$CDa1d1e5?$AA@ 1001adac     DNAStatMSAProfileDialog.obj
 0002:00001db4       ??_C@_07JHABBMBP@?$CDdddddd?$AA@ 1001adb4     DNAStatMSAProfileDialog.obj
 0002:00001dbc       ??_C@_0BO@KJOHEOEO@?$DMSTYLE?5TYPE?$DN?$CCtext?1css?$CC?$DO?$DM?$CB?9?9?5?6?$AA@ 1001adbc     DNAStatMSAProfileDialog.obj
 0002:00001de0       ??_C@_0GL@KLMLHOGI@table?4tbl?5?5?5?$HL?6?5border?9width?3?51px@ 1001ade0     DNAStatMSAProfileDialog.obj
 0002:00001e50       ??_C@_0FO@IAPKICCH@table?4tbl?5td?$HL?6?5max?9width?3?5200px?$DL@ 1001ae50     DNAStatMSAProfileDialog.obj
 0002:00001eb0       ??_C@_0CK@IMOOKFDN@border?9style?3?5solid?$DL?6?5padding?3?50@ 1001aeb0     DNAStatMSAProfileDialog.obj
 0002:00001edc       ??_C@_0N@BFLNFKNH@?9?9?$DO?$DM?1STYLE?$DO?6?$AA@ 1001aedc     DNAStatMSAProfileDialog.obj
 0002:00001eec       ??_C@_0L@FFDHMNNK@?$DM?1h2?$DO?$DMbr?$DO?6?$AA@ 1001aeec     DNAStatMSAProfileDialog.obj
 0002:00001ef8       ??_C@_0CJ@ICHLHFM@Multiple?5Sequence?5Alignment?5Grid@ 1001aef8     DNAStatMSAProfileDialog.obj
 0002:00001f24       ??_C@_04MFLEKIAK@?$DMh2?$DO?$AA@ 1001af24     DNAStatMSAProfileDialog.obj
 0002:00001f2c       ??_C@_08BFDEBDJA@?$DMtable?$DO?6?$AA@ 1001af2c     DNAStatMSAProfileDialog.obj
 0002:00001f38       ??_C@_0M@GOEAPLMM@?$DM?1td?$DO?$DM?1tr?$DO?6?$AA@ 1001af38     DNAStatMSAProfileDialog.obj
 0002:00001f44       ??_C@_01EOFPKCAF@?$EA?$AA@ 1001af44     DNAStatMSAProfileDialog.obj
 0002:00001f48       ??_C@_0O@ENJPPLKE@?$DM?1b?$DO?$DM?1td?$DO?$DMtd?$DO?$AA@ 1001af48     DNAStatMSAProfileDialog.obj
 0002:00001f58       ??_C@_0BA@ILLDKCAG@Alignment?5file?3?$AA@ 1001af58     DNAStatMSAProfileDialog.obj
 0002:00001f68       ??_C@_0M@DIOHJHAK@?$DMtr?$DO?$DMtd?$DO?$DMb?$DO?$AA@ 1001af68     DNAStatMSAProfileDialog.obj
 0002:00001f74       ??_C@_0BA@MPOHFJPL@symbol?5percents?$AA@ 1001af74     DNAStatMSAProfileDialog.obj
 0002:00001f84       ??_C@_0O@KGHOIFAP@symbol?5counts?$AA@ 1001af84     DNAStatMSAProfileDialog.obj
 0002:00001f94       ??_C@_0P@MLFHHFMB@Table?5content?3?$AA@ 1001af94     DNAStatMSAProfileDialog.obj
 0002:00001fa4       ??_C@_09PHDFHDEK@?$DM?1table?$DO?6?$AA@ 1001afa4     DNAStatMSAProfileDialog.obj
 0002:00001fb0       ??_C@_09IPGALPAD@?$DMbr?$DO?$DMbr?$DO?6?$AA@ 1001afb0     DNAStatMSAProfileDialog.obj
 0002:00001fbc       ??_C@_0BC@KDCLJJNB@?$DMtable?5class?$DNtbl?$DO?$AA@ 1001afbc     DNAStatMSAProfileDialog.obj
 0002:00001fd0       ??_C@_0O@MOFFIKKK@?$DMtr?$DO?$DMtd?$DO?$DM?1td?$DO?$AA@ 1001afd0     DNAStatMSAProfileDialog.obj
 0002:00001fe0       ??_C@_06ODLOODK@?$CGnbsp?$DL?$AA@ 1001afe0     DNAStatMSAProfileDialog.obj
 0002:00001fe8       ??_C@_05JEFCGOBF@?$DM?1td?$DO?$AA@ 1001afe8     DNAStatMSAProfileDialog.obj
 0002:00001ff0       ??_C@_0O@FCKLFBLD@?$DMtd?5width?$DN20?$DO?$AA@ 1001aff0     DNAStatMSAProfileDialog.obj
 0002:00002000       ??_C@_06OCNEFGEM@?$DM?1tr?$DO?6?$AA@ 1001b000     DNAStatMSAProfileDialog.obj
 0002:00002008       ??_C@_0BJ@DJCCBGCF@?$DMtr?$DO?$DMtd?$DO?5Consensus?5?$DM?1td?$DO?$AA@ 1001b008     DNAStatMSAProfileDialog.obj
 0002:00002024       ??_C@_09IDAPPBMN@?$DM?1b?$DO?$DM?1td?$DO?$AA@ 1001b024     DNAStatMSAProfileDialog.obj
 0002:00002030       ??_C@_07GNIHJKBN@?$DMtd?$DO?$DMb?$DO?$AA@ 1001b030     DNAStatMSAProfileDialog.obj
 0002:00002038       ??_C@_04KPOBMNON@?$DMtr?$DO?$AA@ 1001b038     DNAStatMSAProfileDialog.obj
 0002:00002040       ??_C@_05DOOCFDOJ@?$DMtd?$DO?5?$AA@ 1001b040     DNAStatMSAProfileDialog.obj
 0002:00002048       ??_C@_09LKHFPGLH@?5bgcolor?$DN?$AA@ 1001b048     DNAStatMSAProfileDialog.obj
 0002:00002054       ??_C@_01PPODPGHN@?$DO?$AA@ 1001b054     DNAStatMSAProfileDialog.obj
 0002:00002058       ??_C@_03DGCPAJNF@?$DMtd?$AA@ 1001b058     DNAStatMSAProfileDialog.obj
 0002:0000205c       ??_C@_0BC@MALKIKLP@?$CGnbsp?$DL?$CGnbsp?$DL?$DM?1b?$DO?6?$AA@ 1001b05c     DNAStatMSAProfileDialog.obj
 0002:00002070       ??_C@_07MIMMGOBM@Legend?3?$AA@ 1001b070     DNAStatMSAProfileDialog.obj
 0002:00002078       ??_C@_0BD@DGHNFOEI@?$DMtable?$DO?$DMtr?$DO?$DMtd?$DO?$DMb?$DO?$AA@ 1001b078     DNAStatMSAProfileDialog.obj
 0002:0000208c       ??_C@_0L@DMHBFGB@?$DO10?$CF?$DM?1td?$DO?6?$AA@ 1001b08c     DNAStatMSAProfileDialog.obj
 0002:00002098       ??_C@_0N@MAJNDKG@?$DMtd?5bgcolor?$DN?$AA@ 1001b098     DNAStatMSAProfileDialog.obj
 0002:000020a8       ??_C@_0L@KCGHOLCN@?$DO25?$CF?$DM?1td?$DO?6?$AA@ 1001b0a8     DNAStatMSAProfileDialog.obj
 0002:000020b4       ??_C@_0L@KCMLFBL@?$DO50?$CF?$DM?1td?$DO?6?$AA@ 1001b0b4     DNAStatMSAProfileDialog.obj
 0002:000020c0       ??_C@_0L@ONJGFCG@?$DO70?$CF?$DM?1td?$DO?6?$AA@ 1001b0c0     DNAStatMSAProfileDialog.obj
 0002:000020cc       ??_C@_0L@BABAFFJF@?$DO90?$CF?$DM?1td?$DO?6?$AA@ 1001b0cc     DNAStatMSAProfileDialog.obj
 0002:000020d8       ??_C@_0BD@BMCAHECI@?$DM?1tr?$DO?$DM?1table?$DO?$DMbr?$DO?6?$AA@ 1001b0d8     DNAStatMSAProfileDialog.obj
 0002:000020f0       ??_C@_0HP@NLFMIHF@There?5is?5not?5enough?5memory?5to?5sh@ 1001b0f0     DNAStatMSAProfileDialog.obj
 0002:00002170       ??_C@_0ED@LFIMCHHN@There?5is?5not?5enough?5memory?5to?5ge@ 1001b170     DNAStatMSAProfileDialog.obj
 0002:000021b4       ??_C@_01IHBHIGKO@?0?$AA@   1001b1b4     DNAStatMSAProfileDialog.obj
 0002:000021b8       ??_C@_01EEMJAFIK@?6?$AA@   1001b1b8     DNAStatMSAProfileDialog.obj
 0002:000021bc       ??_C@_0CE@IALHPIPP@Task?5was?5finished?5with?5an?5error?3@ 1001b1bc     DNAStatMSAProfileDialog.obj
 0002:000021e0       ??_C@_0BD@INJPPOBO@Task?5was?5canceled?4?$AA@ 1001b1e0     DNAStatMSAProfileDialog.obj
 0002:000021f4       ??_C@_04NKJDMFKO@?$DMbr?$DO?$AA@ 1001b1f4     DNAStatMSAProfileDialog.obj
 0002:000021fc       ??_C@_0CJ@DAKAACDF@Grid?5profile?5for?5?$CF1?3?5?$DMa?5href?$DN?8?$CF2@ 1001b1fc     DNAStatMSAProfileDialog.obj
 0002:00002228       ??_C@_0BC@PAEEBLPN@Alignment?5profile?$AA@ 1001b228     DNAStatMSAProfileDialog.obj
 0002:0000223c       ??_C@_0BJ@HEOEHIEB@Alignment?5profile?5for?5?$CF1?$AA@ 1001b23c     DNAStatMSAProfileDialog.obj
 0002:00002258       ??_C@_0BL@MOMIHLAO@?3core?1images?1chart_bar?4png?$AA@ 1001b258     DNAStatMSAProfileDialog.obj
 0002:00002274       ??_C@_0BA@JFNIOLAK@string?5too?5long?$AA@ 1001b274     DNAStatMSAProfileDialog.obj
 0002:00002284       ??_C@_0BI@CFPLBAOH@invalid?5string?5position?$AA@ 1001b284     DNAStatMSAProfileDialog.obj
 0002:000022a0       __real@0000000000000000    1001b2a0     DNAStatMSAProfileDialog.obj
 0002:000022a8       __real@3fe0000000000000    1001b2a8     DNAStatMSAProfileDialog.obj
 0002:000022b0       __real@3ff0000000000000    1001b2b0     DNAStatMSAProfileDialog.obj
 0002:000022b8       __real@4059000000000000    1001b2b8     DNAStatMSAProfileDialog.obj
 0002:000022c4       ??_SGObjectViewAction@U2@@6B@ 1001b2c4     DNAStatPlugin.obj
 0002:000022f4       ??_7DNAStatPlugin@U2@@6B@  1001b2f4     DNAStatPlugin.obj
 0002:00002324       ??_7DNAStatMSAEditorContext@U2@@6BQObject@@@ 1001b324     DNAStatPlugin.obj
 0002:00002374       ??_7DNAStatMSAEditorContext@U2@@6BGObjectViewObjectHandler@1@@ 1001b374     DNAStatPlugin.obj
 0002:00002388       ??_7DistanceMatrixMSAEditorContext@U2@@6BQObject@@@ 1001b388     DNAStatPlugin.obj
 0002:000023d8       ??_7DistanceMatrixMSAEditorContext@U2@@6BGObjectViewObjectHandler@1@@ 1001b3d8     DNAStatPlugin.obj
 0002:000023e8       ??_C@_0DK@KLPDFNMH@Provides?5statistical?5reports?5for@ 1001b3e8     DNAStatPlugin.obj
 0002:00002424       ??_C@_0P@HADIJAHI@DNA?5Statistics?$AA@ 1001b424     DNAStatPlugin.obj
 0002:00002434       ??_C@_0BJ@MEJPONLE@Generate?5grid?5profile?4?4?4?$AA@ 1001b434     DNAStatPlugin.obj
 0002:00002450       ??_C@_0BG@BHEPDIGG@Generate?5grid?5profile?$AA@ 1001b450     DNAStatPlugin.obj
 0002:00002468       ??_C@_0BL@FDPDGKCK@1sl_showMSAProfileDialog?$CI?$CJ?$AA@ 1001b468     DNAStatPlugin.obj
 0002:00002484       ??_C@_0N@NBJIAFIH@2triggered?$CI?$CJ?$AA@ 1001b484     DNAStatPlugin.obj
 0002:00002494       ??_C@_0BF@EBOOBJB@MSAE_MENU_STATISTICS?$AA@ 1001b494     DNAStatPlugin.obj
 0002:000024ac       ??_C@_0CK@IGBIANDN@Trying?5to?5recover?5from?5error?3?5?$CF1@ 1001b4ac     DNAStatPlugin.obj
 0002:000024d8       ??_C@_08PJCKHDPN@statMenu?$AA@ 1001b4d8     DNAStatPlugin.obj
 0002:000024e4       ??_C@_0BG@BBPDOGMK@src?2DNAStatPlugin?4cpp?$AA@ 1001b4e4     DNAStatPlugin.obj
 0002:000024fc       ??_C@_0BM@OJMKEGNN@Generate?5distance?5matrix?4?4?4?$AA@ 1001b4fc     DNAStatPlugin.obj
 0002:00002518       ??_C@_0BJ@JPALMHNI@Generate?5distance?5matrix?$AA@ 1001b518     DNAStatPlugin.obj
 0002:00002534       ??_C@_0BP@JIPKJILK@1sl_showDistanceMatrixDialog?$CI?$CJ?$AA@ 1001b534     DNAStatPlugin.obj
 0002:0000255c       ??_SCharOccurTask@U2@@6B@  1001b55c     DNAStatProfileTask.obj
 0002:000025ec       ??_SDinuclOccurTask@U2@@6B@ 1001b5ec     DNAStatProfileTask.obj
 0002:0000267c       ??_SDNAStatisticsTask@U2@@6B@ 1001b67c     DNAStatProfileTask.obj
 0002:0000270c       ??_7DNAStatProfileTask@U2@@6B@ 1001b70c     DNAStatProfileTask.obj
 0002:00002798       ??_C@_0CF@FGJNJHEF@Generate?5sequence?5statistics?5pro@ 1001b798     DNAStatProfileTask.obj
 0002:000027c0       ??_C@_0BJ@GJFCMHEC@Sequence?5context?5is?5NULL?$AA@ 1001b7c0     DNAStatProfileTask.obj
 0002:000027dc       ??_C@_0DE@HBJGLAGL@border?9style?3?5solid?$DL?6?5margin?30px@ 1001b7dc     DNAStatProfileTask.obj
 0002:00002810       ??_C@_0L@MLCIMCIJ@?$DM?1td?$DO?$DM?1tr?$DO?$AA@ 1001b810     DNAStatProfileTask.obj
 0002:0000281c       ??_C@_0BC@GIAHDAPG@Symbol?5percents?5?$CF?$AA@ 1001b81c     DNAStatProfileTask.obj
 0002:00002830       ??_C@_09NEPGDDMB@?$DM?1td?$DO?$DMtd?$DO?$AA@ 1001b830     DNAStatProfileTask.obj
 0002:0000283c       ??_C@_0O@GLBKPNNH@Symbol?5counts?$AA@ 1001b83c     DNAStatProfileTask.obj
 0002:0000284c       ??_C@_0BC@PLPDDLFM@?$DMtr?$DO?$DMtd?$DO?$DM?1td?$DO?$DMtd?$DO?$AA@ 1001b84c     DNAStatProfileTask.obj
 0002:00002860       ??_C@_0DC@JOAMBFPA@?$DMtr?$DO?$DMtd?$DO?$DMb?$DO?$CF1?$DM?1b?$DO?$DM?1td?$DO?$DMtd?$DO?$CF2?$DM?1td@ 1001b860     DNAStatProfileTask.obj
 0002:00002894       ??_C@_0BI@LIHODLKA@Dinucleotide?5percents?5?$CF?$AA@ 1001b894     DNAStatProfileTask.obj
 0002:000028ac       ??_C@_0BE@KDDFBFOH@Dinucleotide?5counts?$AA@ 1001b8ac     DNAStatProfileTask.obj
 0002:000028c0       ??_C@_0BE@JEAEGDMC@Sequence?5Statistics?$AA@ 1001b8c0     DNAStatProfileTask.obj
 0002:000028d4       ??_C@_0BB@NDEOCOKM@Sequence?5length?3?$AA@ 1001b8d4     DNAStatProfileTask.obj
 0002:000028e8       ??_C@_0BG@NCMOAAMG@?$DM?1td?$DO?$DM?1tr?$DO?$DMtr?$DO?$DMtd?$DO?$DMb?$DO?$AA@ 1001b8e8     DNAStatProfileTask.obj
 0002:00002900       ??_C@_0P@OIACICBL@Sequence?5file?3?$AA@ 1001b900     DNAStatProfileTask.obj
 0002:00002910       ??_C@_0CH@CLBKKCFP@?$DMtr?$DO?$DMtd?$DO?$DMb?$DOMolecule?5Type?3?$DM?1b?$DO?$DM?1t@ 1001b910     DNAStatProfileTask.obj
 0002:00002938       ??_C@_04KINFKBFF@?$CF1?5?$CF?$AA@ 1001b938     DNAStatProfileTask.obj
 0002:00002940       ??_C@_0M@BLEDAKDA@GC?5content?3?$AA@ 1001b940     DNAStatProfileTask.obj
 0002:0000294c       ??_C@_05COFKILCL@?$CF1?5Da?$AA@ 1001b94c     DNAStatProfileTask.obj
 0002:00002954       ??_C@_0O@DHIMBMMF@Molar?5Weight?3?$AA@ 1001b954     DNAStatProfileTask.obj
 0002:00002964       ??_C@_0BF@GAOJLDNA@?$CF1?5I?1mol?5?$CIat?5260?5nm?$CJ?$AA@ 1001b964     DNAStatProfileTask.obj
 0002:0000297c       ??_C@_0BC@BKJCKPBG@Molar?5ext?4?5coef?4?3?$AA@ 1001b97c     DNAStatProfileTask.obj
 0002:00002990       ??_C@_0DB@JGJMOLI@?$CF1?5C?5?$CIat?5salt?5CC?550?5mM?0?5primer?5C@ 1001b990     DNAStatProfileTask.obj
 0002:000029c4       ??_C@_0M@IMCFEBOC@Melting?5Tm?3?$AA@ 1001b9c4     DNAStatProfileTask.obj
 0002:000029d0       ??_C@_02PIGFKFFE@?$CF1?$AA@ 1001b9d0     DNAStatProfileTask.obj
 0002:000029d4       ??_C@_0BC@BKBADJJM@Molecular?5Weight?3?$AA@ 1001b9d4     DNAStatProfileTask.obj
 0002:000029e8       ??_C@_0BI@PCBJEBNA@Isoelectric?5Point?5?$CIpI?$CJ?3?$AA@ 1001b9e8     DNAStatProfileTask.obj
 0002:00002a00       ??_C@_00CNPNBAHC@?$AA@     1001ba00     DistanceMatrixMSAProfileDialog.obj
 0002:00002a08       ??_SMultipleSequenceAlignmentRow@U2@@6B@ 1001ba08     DistanceMatrixMSAProfileDialog.obj
 0002:00002a14       ??_SQSpacerItem@@6B@       1001ba14     DistanceMatrixMSAProfileDialog.obj
 0002:00002a5c       ??_SQHBoxLayout@@6BQObject@@@ 1001ba5c     DistanceMatrixMSAProfileDialog.obj
 0002:00002aa4       ??_SQHBoxLayout@@6BQLayoutItem@@@ 1001baa4     DistanceMatrixMSAProfileDialog.obj
 0002:00002aec       ??_SQComboBox@@6BQObject@@@ 1001baec     DistanceMatrixMSAProfileDialog.obj
 0002:00002bac       ??_SQComboBox@@6BQPaintDevice@@@ 1001bbac     DistanceMatrixMSAProfileDialog.obj
 0002:00002bc8       ??_C@_0BJ@EHIJIFDJ@Generate?5Distance?5Matrix?$AA@ 1001bbc8     DistanceMatrixMSAProfileDialog.obj
 0002:00002be4       ??_C@_0BP@LENMGFMF@DistanceMatrixMSAProfileDialog?$AA@ 1001bbe4     DistanceMatrixMSAProfileDialog.obj
 0002:00002c04       ??_C@_0BD@BIFBICGM@Distance?5algorithm?$AA@ 1001bc04     DistanceMatrixMSAProfileDialog.obj
 0002:00002c18       ??_C@_0N@LIFOEPPJ@Exclude?5gaps?$AA@ 1001bc18     DistanceMatrixMSAProfileDialog.obj
 0002:00002c28       ??_C@_0CM@BGPJHPG@Show?5group?5statistics?5of?5multipl@ 1001bc28     DistanceMatrixMSAProfileDialog.obj
 0002:00002f70       ??_7DistanceMatrixMSAProfileDialog@U2@@6BQObject@@@ 1001bf70     DistanceMatrixMSAProfileDialog.obj
 0002:0000303c       ??_7DistanceMatrixMSAProfileDialog@U2@@6BQPaintDevice@@@ 1001c03c     DistanceMatrixMSAProfileDialog.obj
 0002:0000305c       ??_7DistanceMatrixMSAProfileTask@U2@@6B@ 1001c05c     DistanceMatrixMSAProfileDialog.obj
 0002:000030e8       ??_C@_08FLJKLEID@23331105?$AA@ 1001c0e8     DistanceMatrixMSAProfileDialog.obj
 0002:000030f4       ??_C@_08PDEEPOLG@Generate?$AA@ 1001c0f4     DistanceMatrixMSAProfileDialog.obj
 0002:00003100       ??_C@_0BB@NKMAAJCG@_distance_matrix?$AA@ 1001c100     DistanceMatrixMSAProfileDialog.obj
 0002:00003118       ??_C@_0FO@FAGNEKK@table?4tbl?5td?$HL?6?5max?9width?3?5400px?$DL@ 1001c118     DistanceMatrixMSAProfileDialog.obj
 0002:00003178       ??_C@_0CM@BEBCHLBJ@border?9style?3?5solid?$DL?6?5?6?5padding?3@ 1001c178     DistanceMatrixMSAProfileDialog.obj
 0002:000031a4       ??_C@_0CM@KEHMCE@Multiple?5Sequence?5Alignment?5Dist@ 1001c1a4     DistanceMatrixMSAProfileDialog.obj
 0002:000031d0       ??_C@_0M@BCBJPCNJ@?5in?5percent?$AA@ 1001c1d0     DistanceMatrixMSAProfileDialog.obj
 0002:000031e0       ??_C@_0IC@CNBHFKAK@There?5is?5not?5enough?5memory?5to?5sh@ 1001c1e0     DistanceMatrixMSAProfileDialog.obj
 0002:00003264       ??_C@_0CH@GLCJIKEL@Group?5statistics?5of?5multiple?5ali@ 1001c264     DistanceMatrixMSAProfileDialog.obj
 0002:0000328c       ??_C@_01PKGAHCOL@?$CJ?$AA@ 1001c28c     DistanceMatrixMSAProfileDialog.obj
 0002:00003290       ??_C@_01ODHLEDKK@?$CI?$AA@ 1001c290     DistanceMatrixMSAProfileDialog.obj
 0002:00003294       ??_C@_0L@OINHGIBC@Group?5?$CF1?3?5?$AA@ 1001c294     DistanceMatrixMSAProfileDialog.obj
 0002:000032a0       ??_C@_02KEGNLNML@?0?5?$AA@ 1001c2a0     DistanceMatrixMSAProfileDialog.obj
 0002:000032a4       ??_C@_01CLKCMJKC@?5?$AA@   1001c2a4     DistanceMatrixMSAProfileDialog.obj
 0002:000032a8       ??_C@_01FGNFDNOH@?$CF?$AA@ 1001c2a8     DistanceMatrixMSAProfileDialog.obj
 0002:000032ac       ??_C@_0DG@BNEMNJDC@There?5is?5not?5enough?5groups?5to?5cr@ 1001c2ac     DistanceMatrixMSAProfileDialog.obj
 0002:000032e4       ??_C@_0BD@LJICBFB@?$DMtable?5class?$DNtbl?$DO?6?$AA@ 1001c2e4     DistanceMatrixMSAProfileDialog.obj
 0002:000032f8       ??_C@_0CM@FLFOMHOK@Distanse?5matrix?5for?5?$CF1?3?5?$DMa?5href?$DN@ 1001c2f8     DistanceMatrixMSAProfileDialog.obj
 0002:00003324       ??_C@_0BA@BBEOIEND@Distance?5matrix?$AA@ 1001c324     DistanceMatrixMSAProfileDialog.obj
 0002:00003334       ??_C@_0BH@CDCFKAOK@Distance?5matrix?5for?5?$CF1?$AA@ 1001c334     DistanceMatrixMSAProfileDialog.obj
 0002:000034c8       ??_C@_0BL@EBLDEBKO@Ui_DNAStatMSAProfileDialog?$AA@ 1001c4c8     moc_DNAStatMSAProfileDialog.obj
 0002:000039f0       ??_C@_0CC@EJMCCOFH@Ui_DistanceMatrixMSAProfileDialo@ 1001c9f0     moc_DistanceMatrixMSAProfileDialog.obj
 0002:00003a12       ?value@?$integral_constant@_N$0A@@std@@2_NB 1001ca12     MSVCRT:ti_inst.obj
 0002:00003a13       ?value@?$integral_constant@_N$00@std@@2_NB 1001ca13     MSVCRT:ti_inst.obj
 0002:00003a18       ??_7type_info@@6B@         1001ca18     MSVCRT:ti_inst.obj
 0002:00003aa4       __pDefaultRawDllMain       1001caa4     MSVCRT:crtdll.obj
 0002:00003aa4       __pRawDllMain              1001caa4     MSVCRT:crtdll.obj
 0002:00003ab0       ?ProcessDetach@NativeDll@<CrtImplementationDetails>@@0IB 1001cab0     MSVCRT:initsect.obj
 0002:00003ab4       ?ProcessAttach@NativeDll@<CrtImplementationDetails>@@0IB 1001cab4     MSVCRT:initsect.obj
 0002:00003ab8       ?ThreadAttach@NativeDll@<CrtImplementationDetails>@@0IB 1001cab8     MSVCRT:initsect.obj
 0002:00003abc       ?ThreadDetach@NativeDll@<CrtImplementationDetails>@@0IB 1001cabc     MSVCRT:initsect.obj
 0002:00003ac0       ?ProcessVerifier@NativeDll@<CrtImplementationDetails>@@0IB 1001cac0     MSVCRT:initsect.obj
 0002:00003ac8       __load_config_used         1001cac8     MSVCRT:loadcfg.obj
 0002:00003b80       ??_R4error_category@std@@6B@ 1001cb80     DNAStatMSAProfileDialog.obj
 0002:00003b94       ??_R3error_category@std@@8 1001cb94     DNAStatMSAProfileDialog.obj
 0002:00003ba4       ??_R2error_category@std@@8 1001cba4     DNAStatMSAProfileDialog.obj
 0002:00003bac       ??_R1A@?0A@EA@error_category@std@@8 1001cbac     DNAStatMSAProfileDialog.obj
 0002:00003bc8       ??_R4_Generic_error_category@std@@6B@ 1001cbc8     DNAStatMSAProfileDialog.obj
 0002:00003bdc       ??_R3_Generic_error_category@std@@8 1001cbdc     DNAStatMSAProfileDialog.obj
 0002:00003bec       ??_R2_Generic_error_category@std@@8 1001cbec     DNAStatMSAProfileDialog.obj
 0002:00003bf8       ??_R1A@?0A@EA@_Generic_error_category@std@@8 1001cbf8     DNAStatMSAProfileDialog.obj
 0002:00003c14       ??_R4_Iostream_error_category@std@@6B@ 1001cc14     DNAStatMSAProfileDialog.obj
 0002:00003c28       ??_R3_Iostream_error_category@std@@8 1001cc28     DNAStatMSAProfileDialog.obj
 0002:00003c38       ??_R2_Iostream_error_category@std@@8 1001cc38     DNAStatMSAProfileDialog.obj
 0002:00003c48       ??_R1A@?0A@EA@_Iostream_error_category@std@@8 1001cc48     DNAStatMSAProfileDialog.obj
 0002:00003c64       ??_R4_System_error_category@std@@6B@ 1001cc64     DNAStatMSAProfileDialog.obj
 0002:00003c78       ??_R3_System_error_category@std@@8 1001cc78     DNAStatMSAProfileDialog.obj
 0002:00003c88       ??_R2_System_error_category@std@@8 1001cc88     DNAStatMSAProfileDialog.obj
 0002:00003c98       ??_R1A@?0A@EA@_System_error_category@std@@8 1001cc98     DNAStatMSAProfileDialog.obj
 0002:00003cb4       ??_R4QFile@@6B@            1001ccb4     DNAStatMSAProfileDialog.obj
 0002:00003cc8       ??_R3QFile@@8              1001ccc8     DNAStatMSAProfileDialog.obj
 0002:00003cd8       ??_R2QFile@@8              1001ccd8     DNAStatMSAProfileDialog.obj
 0002:00003cec       ??_R1A@?0A@EA@QFile@@8     1001ccec     DNAStatMSAProfileDialog.obj
 0002:00003d08       ??_R1A@?0A@EA@QFileDevice@@8 1001cd08     DNAStatMSAProfileDialog.obj
 0002:00003d24       ??_R3QFileDevice@@8        1001cd24     DNAStatMSAProfileDialog.obj
 0002:00003d34       ??_R2QFileDevice@@8        1001cd34     DNAStatMSAProfileDialog.obj
 0002:00003d44       ??_R1A@?0A@EA@QIODevice@@8 1001cd44     DNAStatMSAProfileDialog.obj
 0002:00003d60       ??_R3QIODevice@@8          1001cd60     DNAStatMSAProfileDialog.obj
 0002:00003d70       ??_R2QIODevice@@8          1001cd70     DNAStatMSAProfileDialog.obj
 0002:00003d7c       ??_R1A@?0A@EA@QObject@@8   1001cd7c     DNAStatMSAProfileDialog.obj
 0002:00003d98       ??_R3QObject@@8            1001cd98     DNAStatMSAProfileDialog.obj
 0002:00003da8       ??_R2QObject@@8            1001cda8     DNAStatMSAProfileDialog.obj
 0002:00003db0       ??_R4QLabel@@6BQObject@@@  1001cdb0     DNAStatMSAProfileDialog.obj
 0002:00003dc4       ??_R3QLabel@@8             1001cdc4     DNAStatMSAProfileDialog.obj
 0002:00003dd4       ??_R2QLabel@@8             1001cdd4     DNAStatMSAProfileDialog.obj
 0002:00003dec       ??_R1A@?0A@EA@QLabel@@8    1001cdec     DNAStatMSAProfileDialog.obj
 0002:00003e08       ??_R1A@?0A@EA@QFrame@@8    1001ce08     DNAStatMSAProfileDialog.obj
 0002:00003e24       ??_R3QFrame@@8             1001ce24     DNAStatMSAProfileDialog.obj
 0002:00003e34       ??_R2QFrame@@8             1001ce34     DNAStatMSAProfileDialog.obj
 0002:00003e48       ??_R1A@?0A@EA@QWidget@@8   1001ce48     DNAStatMSAProfileDialog.obj
 0002:00003e64       ??_R3QWidget@@8            1001ce64     DNAStatMSAProfileDialog.obj
 0002:00003e74       ??_R2QWidget@@8            1001ce74     DNAStatMSAProfileDialog.obj
 0002:00003e84       ??_R17?0A@EA@QPaintDevice@@8 1001ce84     DNAStatMSAProfileDialog.obj
 0002:00003ea0       ??_R3QPaintDevice@@8       1001cea0     DNAStatMSAProfileDialog.obj
 0002:00003eb0       ??_R2QPaintDevice@@8       1001ceb0     DNAStatMSAProfileDialog.obj
 0002:00003eb8       ??_R1A@?0A@EA@QPaintDevice@@8 1001ceb8     DNAStatMSAProfileDialog.obj
 0002:00003ed4       ??_R4QLabel@@6BQPaintDevice@@@ 1001ced4     DNAStatMSAProfileDialog.obj
 0002:00003ee8       ??_R4QCheckBox@@6BQObject@@@ 1001cee8     DNAStatMSAProfileDialog.obj
 0002:00003efc       ??_R3QCheckBox@@8          1001cefc     DNAStatMSAProfileDialog.obj
 0002:00003f0c       ??_R2QCheckBox@@8          1001cf0c     DNAStatMSAProfileDialog.obj
 0002:00003f24       ??_R1A@?0A@EA@QCheckBox@@8 1001cf24     DNAStatMSAProfileDialog.obj
 0002:00003f40       ??_R1A@?0A@EA@QAbstractButton@@8 1001cf40     DNAStatMSAProfileDialog.obj
 0002:00003f5c       ??_R3QAbstractButton@@8    1001cf5c     DNAStatMSAProfileDialog.obj
 0002:00003f6c       ??_R2QAbstractButton@@8    1001cf6c     DNAStatMSAProfileDialog.obj
 0002:00003f80       ??_R4QCheckBox@@6BQPaintDevice@@@ 1001cf80     DNAStatMSAProfileDialog.obj
 0002:00003f94       ??_R4AbstractInt32Id@U2@@6B@ 1001cf94     DNAStatMSAProfileDialog.obj
 0002:00003fa8       ??_R3AbstractInt32Id@U2@@8 1001cfa8     DNAStatMSAProfileDialog.obj
 0002:00003fb8       ??_R2AbstractInt32Id@U2@@8 1001cfb8     DNAStatMSAProfileDialog.obj
 0002:00003fc4       ??_R1A@?0A@EA@AbstractInt32Id@U2@@8 1001cfc4     DNAStatMSAProfileDialog.obj
 0002:00003fe0       ??_R1A@?0A@EA@?$AbstractId@H@U2@@8 1001cfe0     DNAStatMSAProfileDialog.obj
 0002:00003ffc       ??_R3?$AbstractId@H@U2@@8  1001cffc     DNAStatMSAProfileDialog.obj
 0002:0000400c       ??_R2?$AbstractId@H@U2@@8  1001d00c     DNAStatMSAProfileDialog.obj
 0002:00004014       ??_R4?$AbstractId@H@U2@@6B@ 1001d014     DNAStatMSAProfileDialog.obj
 0002:00004028       ??_R4ServiceType@U2@@6B@   1001d028     DNAStatMSAProfileDialog.obj
 0002:0000403c       ??_R3ServiceType@U2@@8     1001d03c     DNAStatMSAProfileDialog.obj
 0002:0000404c       ??_R2ServiceType@U2@@8     1001d04c     DNAStatMSAProfileDialog.obj
 0002:0000405c       ??_R1A@?0A@EA@ServiceType@U2@@8 1001d05c     DNAStatMSAProfileDialog.obj
 0002:00004078       ??_R4QDialogButtonBox@@6BQObject@@@ 1001d078     DNAStatMSAProfileDialog.obj
 0002:0000408c       ??_R3QDialogButtonBox@@8   1001d08c     DNAStatMSAProfileDialog.obj
 0002:0000409c       ??_R2QDialogButtonBox@@8   1001d09c     DNAStatMSAProfileDialog.obj
 0002:000040b0       ??_R1A@?0A@EA@QDialogButtonBox@@8 1001d0b0     DNAStatMSAProfileDialog.obj
 0002:000040cc       ??_R4QDialogButtonBox@@6BQPaintDevice@@@ 1001d0cc     DNAStatMSAProfileDialog.obj
 0002:000040e0       ??_R4HelpButton@U2@@6B@    1001d0e0     DNAStatMSAProfileDialog.obj
 0002:000040f4       ??_R3HelpButton@U2@@8      1001d0f4     DNAStatMSAProfileDialog.obj
 0002:00004104       ??_R2HelpButton@U2@@8      1001d104     DNAStatMSAProfileDialog.obj
 0002:00004110       ??_R1A@?0A@EA@HelpButton@U2@@8 1001d110     DNAStatMSAProfileDialog.obj
 0002:0000412c       ??_R4QLineEdit@@6BQObject@@@ 1001d12c     DNAStatMSAProfileDialog.obj
 0002:00004140       ??_R3QLineEdit@@8          1001d140     DNAStatMSAProfileDialog.obj
 0002:00004150       ??_R2QLineEdit@@8          1001d150     DNAStatMSAProfileDialog.obj
 0002:00004164       ??_R1A@?0A@EA@QLineEdit@@8 1001d164     DNAStatMSAProfileDialog.obj
 0002:00004180       ??_R4QLineEdit@@6BQPaintDevice@@@ 1001d180     DNAStatMSAProfileDialog.obj
 0002:00004194       ??_R4SaveDocumentController@U2@@6B@ 1001d194     DNAStatMSAProfileDialog.obj
 0002:000041a8       ??_R3SaveDocumentController@U2@@8 1001d1a8     DNAStatMSAProfileDialog.obj
 0002:000041b8       ??_R2SaveDocumentController@U2@@8 1001d1b8     DNAStatMSAProfileDialog.obj
 0002:000041c4       ??_R1A@?0A@EA@SaveDocumentController@U2@@8 1001d1c4     DNAStatMSAProfileDialog.obj
 0002:000041e0       ??_R4QToolButton@@6BQObject@@@ 1001d1e0     DNAStatMSAProfileDialog.obj
 0002:000041f4       ??_R3QToolButton@@8        1001d1f4     DNAStatMSAProfileDialog.obj
 0002:00004204       ??_R2QToolButton@@8        1001d204     DNAStatMSAProfileDialog.obj
 0002:0000421c       ??_R1A@?0A@EA@QToolButton@@8 1001d21c     DNAStatMSAProfileDialog.obj
 0002:00004238       ??_R4QToolButton@@6BQPaintDevice@@@ 1001d238     DNAStatMSAProfileDialog.obj
 0002:0000424c       ??_R4QGridLayout@@6BQObject@@@ 1001d24c     DNAStatMSAProfileDialog.obj
 0002:00004260       ??_R3QGridLayout@@8        1001d260     DNAStatMSAProfileDialog.obj
 0002:00004270       ??_R2QGridLayout@@8        1001d270     DNAStatMSAProfileDialog.obj
 0002:00004284       ??_R1A@?0A@EA@QGridLayout@@8 1001d284     DNAStatMSAProfileDialog.obj
 0002:000042a0       ??_R1A@?0A@EA@QLayout@@8   1001d2a0     DNAStatMSAProfileDialog.obj
 0002:000042bc       ??_R3QLayout@@8            1001d2bc     DNAStatMSAProfileDialog.obj
 0002:000042cc       ??_R2QLayout@@8            1001d2cc     DNAStatMSAProfileDialog.obj
 0002:000042dc       ??_R17?0A@EA@QLayoutItem@@8 1001d2dc     DNAStatMSAProfileDialog.obj
 0002:000042f8       ??_R3QLayoutItem@@8        1001d2f8     DNAStatMSAProfileDialog.obj
 0002:00004308       ??_R2QLayoutItem@@8        1001d308     DNAStatMSAProfileDialog.obj
 0002:00004310       ??_R1A@?0A@EA@QLayoutItem@@8 1001d310     DNAStatMSAProfileDialog.obj
 0002:0000432c       ??_R4QGridLayout@@6BQLayoutItem@@@ 1001d32c     DNAStatMSAProfileDialog.obj
 0002:00004340       ??_R4QVBoxLayout@@6BQObject@@@ 1001d340     DNAStatMSAProfileDialog.obj
 0002:00004354       ??_R3QVBoxLayout@@8        1001d354     DNAStatMSAProfileDialog.obj
 0002:00004364       ??_R2QVBoxLayout@@8        1001d364     DNAStatMSAProfileDialog.obj
 0002:0000437c       ??_R1A@?0A@EA@QVBoxLayout@@8 1001d37c     DNAStatMSAProfileDialog.obj
 0002:00004398       ??_R1A@?0A@EA@QBoxLayout@@8 1001d398     DNAStatMSAProfileDialog.obj
 0002:000043b4       ??_R3QBoxLayout@@8         1001d3b4     DNAStatMSAProfileDialog.obj
 0002:000043c4       ??_R2QBoxLayout@@8         1001d3c4     DNAStatMSAProfileDialog.obj
 0002:000043d8       ??_R4QVBoxLayout@@6BQLayoutItem@@@ 1001d3d8     DNAStatMSAProfileDialog.obj
 0002:000043ec       ??_R4WebWindow@U2@@6BQObject@@@ 1001d3ec     DNAStatMSAProfileDialog.obj
 0002:00004400       ??_R3WebWindow@U2@@8       1001d400     DNAStatMSAProfileDialog.obj
 0002:00004410       ??_R2WebWindow@U2@@8       1001d410     DNAStatMSAProfileDialog.obj
 0002:00004428       ??_R1A@?0A@EA@WebWindow@U2@@8 1001d428     DNAStatMSAProfileDialog.obj
 0002:00004444       ??_R1A@?0A@EA@MWMDIWindow@U2@@8 1001d444     DNAStatMSAProfileDialog.obj
 0002:00004460       ??_R3MWMDIWindow@U2@@8     1001d460     DNAStatMSAProfileDialog.obj
 0002:00004470       ??_R2MWMDIWindow@U2@@8     1001d470     DNAStatMSAProfileDialog.obj
 0002:00004484       ??_R4WebWindow@U2@@6BQPaintDevice@@@ 1001d484     DNAStatMSAProfileDialog.obj
 0002:00004498       ??_R4QGroupBox@@6BQObject@@@ 1001d498     DNAStatMSAProfileDialog.obj
 0002:000044ac       ??_R3QGroupBox@@8          1001d4ac     DNAStatMSAProfileDialog.obj
 0002:000044bc       ??_R2QGroupBox@@8          1001d4bc     DNAStatMSAProfileDialog.obj
 0002:000044d0       ??_R1A@?0A@EA@QGroupBox@@8 1001d4d0     DNAStatMSAProfileDialog.obj
 0002:000044ec       ??_R4QGroupBox@@6BQPaintDevice@@@ 1001d4ec     DNAStatMSAProfileDialog.obj
 0002:00004500       ??_R4QRadioButton@@6BQObject@@@ 1001d500     DNAStatMSAProfileDialog.obj
 0002:00004514       ??_R3QRadioButton@@8       1001d514     DNAStatMSAProfileDialog.obj
 0002:00004524       ??_R2QRadioButton@@8       1001d524     DNAStatMSAProfileDialog.obj
 0002:0000453c       ??_R1A@?0A@EA@QRadioButton@@8 1001d53c     DNAStatMSAProfileDialog.obj
 0002:00004558       ??_R4QRadioButton@@6BQPaintDevice@@@ 1001d558     DNAStatMSAProfileDialog.obj
 0002:0000456c       ??_R4DNAStatMSAProfileDialog@U2@@6BQObject@@@ 1001d56c     DNAStatMSAProfileDialog.obj
 0002:00004580       ??_R3DNAStatMSAProfileDialog@U2@@8 1001d580     DNAStatMSAProfileDialog.obj
 0002:00004590       ??_R2DNAStatMSAProfileDialog@U2@@8 1001d590     DNAStatMSAProfileDialog.obj
 0002:000045ac       ??_R1A@?0A@EA@DNAStatMSAProfileDialog@U2@@8 1001d5ac     DNAStatMSAProfileDialog.obj
 0002:000045c8       ??_R1A@?0A@EA@QDialog@@8   1001d5c8     DNAStatMSAProfileDialog.obj
 0002:000045e4       ??_R3QDialog@@8            1001d5e4     DNAStatMSAProfileDialog.obj
 0002:000045f4       ??_R2QDialog@@8            1001d5f4     DNAStatMSAProfileDialog.obj
 0002:00004608       ??_R1BI@?0A@EA@Ui_DNAStatMSAProfileDialog@@8 1001d608     DNAStatMSAProfileDialog.obj
 0002:00004624       ??_R3Ui_DNAStatMSAProfileDialog@@8 1001d624     DNAStatMSAProfileDialog.obj
 0002:00004634       ??_R2Ui_DNAStatMSAProfileDialog@@8 1001d634     DNAStatMSAProfileDialog.obj
 0002:0000463c       ??_R1A@?0A@EA@Ui_DNAStatMSAProfileDialog@@8 1001d63c     DNAStatMSAProfileDialog.obj
 0002:00004658       ??_R4DNAStatMSAProfileDialog@U2@@6BQPaintDevice@@@ 1001d658     DNAStatMSAProfileDialog.obj
 0002:0000466c       ??_R4DNAStatMSAProfileTask@U2@@6B@ 1001d66c     DNAStatMSAProfileDialog.obj
 0002:00004680       ??_R3DNAStatMSAProfileTask@U2@@8 1001d680     DNAStatMSAProfileDialog.obj
 0002:00004690       ??_R2DNAStatMSAProfileTask@U2@@8 1001d690     DNAStatMSAProfileDialog.obj
 0002:000046a0       ??_R1A@?0A@EA@DNAStatMSAProfileTask@U2@@8 1001d6a0     DNAStatMSAProfileDialog.obj
 0002:000046bc       ??_R1A@?0A@EA@Task@U2@@8   1001d6bc     DNAStatMSAProfileDialog.obj
 0002:000046d8       ??_R3Task@U2@@8            1001d6d8     DNAStatMSAProfileDialog.obj
 0002:000046e8       ??_R2Task@U2@@8            1001d6e8     DNAStatMSAProfileDialog.obj
 0002:000046f4       ??_R4GObjectViewAction@U2@@6B@ 1001d6f4     DNAStatPlugin.obj
 0002:00004708       ??_R3GObjectViewAction@U2@@8 1001d708     DNAStatPlugin.obj
 0002:00004718       ??_R2GObjectViewAction@U2@@8 1001d718     DNAStatPlugin.obj
 0002:00004728       ??_R1A@?0A@EA@GObjectViewAction@U2@@8 1001d728     DNAStatPlugin.obj
 0002:00004744       ??_R1A@?0A@EA@QAction@@8   1001d744     DNAStatPlugin.obj
 0002:00004760       ??_R3QAction@@8            1001d760     DNAStatPlugin.obj
 0002:00004770       ??_R2QAction@@8            1001d770     DNAStatPlugin.obj
 0002:0000477c       ??_R4DNAStatPlugin@U2@@6B@ 1001d77c     DNAStatPlugin.obj
 0002:00004790       ??_R3DNAStatPlugin@U2@@8   1001d790     DNAStatPlugin.obj
 0002:000047a0       ??_R2DNAStatPlugin@U2@@8   1001d7a0     DNAStatPlugin.obj
 0002:000047b0       ??_R1A@?0A@EA@DNAStatPlugin@U2@@8 1001d7b0     DNAStatPlugin.obj
 0002:000047cc       ??_R1A@?0A@EA@Plugin@U2@@8 1001d7cc     DNAStatPlugin.obj
 0002:000047e8       ??_R3Plugin@U2@@8          1001d7e8     DNAStatPlugin.obj
 0002:000047f8       ??_R2Plugin@U2@@8          1001d7f8     DNAStatPlugin.obj
 0002:00004804       ??_R4DNAStatMSAEditorContext@U2@@6BQObject@@@ 1001d804     DNAStatPlugin.obj
 0002:00004818       ??_R3DNAStatMSAEditorContext@U2@@8 1001d818     DNAStatPlugin.obj
 0002:00004828       ??_R2DNAStatMSAEditorContext@U2@@8 1001d828     DNAStatPlugin.obj
 0002:0000483c       ??_R1A@?0A@EA@DNAStatMSAEditorContext@U2@@8 1001d83c     DNAStatPlugin.obj
 0002:00004858       ??_R1A@?0A@EA@GObjectViewWindowContext@U2@@8 1001d858     DNAStatPlugin.obj
 0002:00004874       ??_R3GObjectViewWindowContext@U2@@8 1001d874     DNAStatPlugin.obj
 0002:00004884       ??_R2GObjectViewWindowContext@U2@@8 1001d884     DNAStatPlugin.obj
 0002:00004894       ??_R17?0A@EA@GObjectViewObjectHandler@U2@@8 1001d894     DNAStatPlugin.obj
 0002:000048b0       ??_R3GObjectViewObjectHandler@U2@@8 1001d8b0     DNAStatPlugin.obj
 0002:000048c0       ??_R2GObjectViewObjectHandler@U2@@8 1001d8c0     DNAStatPlugin.obj
 0002:000048c8       ??_R1A@?0A@EA@GObjectViewObjectHandler@U2@@8 1001d8c8     DNAStatPlugin.obj
 0002:000048e4       ??_R4DNAStatMSAEditorContext@U2@@6BGObjectViewObjectHandler@1@@ 1001d8e4     DNAStatPlugin.obj
 0002:000048f8       ??_R4DistanceMatrixMSAEditorContext@U2@@6BQObject@@@ 1001d8f8     DNAStatPlugin.obj
 0002:0000490c       ??_R3DistanceMatrixMSAEditorContext@U2@@8 1001d90c     DNAStatPlugin.obj
 0002:0000491c       ??_R2DistanceMatrixMSAEditorContext@U2@@8 1001d91c     DNAStatPlugin.obj
 0002:00004930       ??_R1A@?0A@EA@DistanceMatrixMSAEditorContext@U2@@8 1001d930     DNAStatPlugin.obj
 0002:0000494c       ??_R4DistanceMatrixMSAEditorContext@U2@@6BGObjectViewObjectHandler@1@@ 1001d94c     DNAStatPlugin.obj
 0002:00004960       ??_R4CharOccurTask@U2@@6B@ 1001d960     DNAStatProfileTask.obj
 0002:00004974       ??_R3CharOccurTask@U2@@8   1001d974     DNAStatProfileTask.obj
 0002:00004984       ??_R2CharOccurTask@U2@@8   1001d984     DNAStatProfileTask.obj
 0002:00004998       ??_R1A@?0A@EA@CharOccurTask@U2@@8 1001d998     DNAStatProfileTask.obj
 0002:000049b4       ??_R1A@?0A@EA@?$BackgroundTask@V?$QList@UCharOccurResult@U2@@@@@U2@@8 1001d9b4     DNAStatProfileTask.obj
 0002:000049d0       ??_R3?$BackgroundTask@V?$QList@UCharOccurResult@U2@@@@@U2@@8 1001d9d0     DNAStatProfileTask.obj
 0002:000049e0       ??_R2?$BackgroundTask@V?$QList@UCharOccurResult@U2@@@@@U2@@8 1001d9e0     DNAStatProfileTask.obj
 0002:000049f0       ??_R4DinuclOccurTask@U2@@6B@ 1001d9f0     DNAStatProfileTask.obj
 0002:00004a04       ??_R3DinuclOccurTask@U2@@8 1001da04     DNAStatProfileTask.obj
 0002:00004a14       ??_R2DinuclOccurTask@U2@@8 1001da14     DNAStatProfileTask.obj
 0002:00004a28       ??_R1A@?0A@EA@DinuclOccurTask@U2@@8 1001da28     DNAStatProfileTask.obj
 0002:00004a44       ??_R1A@?0A@EA@?$BackgroundTask@V?$QMap@VQByteArray@@_J@@@U2@@8 1001da44     DNAStatProfileTask.obj
 0002:00004a60       ??_R3?$BackgroundTask@V?$QMap@VQByteArray@@_J@@@U2@@8 1001da60     DNAStatProfileTask.obj
 0002:00004a70       ??_R2?$BackgroundTask@V?$QMap@VQByteArray@@_J@@@U2@@8 1001da70     DNAStatProfileTask.obj
 0002:00004a80       ??_R4DNAStatisticsTask@U2@@6B@ 1001da80     DNAStatProfileTask.obj
 0002:00004a94       ??_R3DNAStatisticsTask@U2@@8 1001da94     DNAStatProfileTask.obj
 0002:00004aa4       ??_R2DNAStatisticsTask@U2@@8 1001daa4     DNAStatProfileTask.obj
 0002:00004ab8       ??_R1A@?0A@EA@DNAStatisticsTask@U2@@8 1001dab8     DNAStatProfileTask.obj
 0002:00004ad4       ??_R1A@?0A@EA@?$BackgroundTask@UDNAStatistics@U2@@@U2@@8 1001dad4     DNAStatProfileTask.obj
 0002:00004af0       ??_R3?$BackgroundTask@UDNAStatistics@U2@@@U2@@8 1001daf0     DNAStatProfileTask.obj
 0002:00004b00       ??_R2?$BackgroundTask@UDNAStatistics@U2@@@U2@@8 1001db00     DNAStatProfileTask.obj
 0002:00004b10       ??_R4DNAStatProfileTask@U2@@6B@ 1001db10     DNAStatProfileTask.obj
 0002:00004b24       ??_R3DNAStatProfileTask@U2@@8 1001db24     DNAStatProfileTask.obj
 0002:00004b34       ??_R2DNAStatProfileTask@U2@@8 1001db34     DNAStatProfileTask.obj
 0002:00004b44       ??_R1A@?0A@EA@DNAStatProfileTask@U2@@8 1001db44     DNAStatProfileTask.obj
 0002:00004b60       ??_R4MultipleSequenceAlignmentRow@U2@@6B@ 1001db60     DistanceMatrixMSAProfileDialog.obj
 0002:00004b74       ??_R3MultipleSequenceAlignmentRow@U2@@8 1001db74     DistanceMatrixMSAProfileDialog.obj
 0002:00004b84       ??_R2MultipleSequenceAlignmentRow@U2@@8 1001db84     DistanceMatrixMSAProfileDialog.obj
 0002:00004b90       ??_R1A@?0A@EA@MultipleSequenceAlignmentRow@U2@@8 1001db90     DistanceMatrixMSAProfileDialog.obj
 0002:00004bac       ??_R1A@?0A@EA@MultipleAlignmentRow@U2@@8 1001dbac     DistanceMatrixMSAProfileDialog.obj
 0002:00004bc8       ??_R3MultipleAlignmentRow@U2@@8 1001dbc8     DistanceMatrixMSAProfileDialog.obj
 0002:00004bd8       ??_R2MultipleAlignmentRow@U2@@8 1001dbd8     DistanceMatrixMSAProfileDialog.obj
 0002:00004be0       ??_R4QComboBox@@6BQObject@@@ 1001dbe0     DistanceMatrixMSAProfileDialog.obj
 0002:00004bf4       ??_R3QComboBox@@8          1001dbf4     DistanceMatrixMSAProfileDialog.obj
 0002:00004c04       ??_R2QComboBox@@8          1001dc04     DistanceMatrixMSAProfileDialog.obj
 0002:00004c18       ??_R1A@?0A@EA@QComboBox@@8 1001dc18     DistanceMatrixMSAProfileDialog.obj
 0002:00004c34       ??_R4QComboBox@@6BQPaintDevice@@@ 1001dc34     DistanceMatrixMSAProfileDialog.obj
 0002:00004c48       ??_R4QSpacerItem@@6B@      1001dc48     DistanceMatrixMSAProfileDialog.obj
 0002:00004c5c       ??_R3QSpacerItem@@8        1001dc5c     DistanceMatrixMSAProfileDialog.obj
 0002:00004c6c       ??_R2QSpacerItem@@8        1001dc6c     DistanceMatrixMSAProfileDialog.obj
 0002:00004c78       ??_R1A@?0A@EA@QSpacerItem@@8 1001dc78     DistanceMatrixMSAProfileDialog.obj
 0002:00004c94       ??_R4QHBoxLayout@@6BQObject@@@ 1001dc94     DistanceMatrixMSAProfileDialog.obj
 0002:00004ca8       ??_R3QHBoxLayout@@8        1001dca8     DistanceMatrixMSAProfileDialog.obj
 0002:00004cb8       ??_R2QHBoxLayout@@8        1001dcb8     DistanceMatrixMSAProfileDialog.obj
 0002:00004cd0       ??_R1A@?0A@EA@QHBoxLayout@@8 1001dcd0     DistanceMatrixMSAProfileDialog.obj
 0002:00004cec       ??_R4QHBoxLayout@@6BQLayoutItem@@@ 1001dcec     DistanceMatrixMSAProfileDialog.obj
 0002:00004d00       ??_R4DistanceMatrixMSAProfileDialog@U2@@6BQObject@@@ 1001dd00     DistanceMatrixMSAProfileDialog.obj
 0002:00004d14       ??_R3DistanceMatrixMSAProfileDialog@U2@@8 1001dd14     DistanceMatrixMSAProfileDialog.obj
 0002:00004d24       ??_R2DistanceMatrixMSAProfileDialog@U2@@8 1001dd24     DistanceMatrixMSAProfileDialog.obj
 0002:00004d40       ??_R1A@?0A@EA@DistanceMatrixMSAProfileDialog@U2@@8 1001dd40     DistanceMatrixMSAProfileDialog.obj
 0002:00004d5c       ??_R1BI@?0A@EA@Ui_DistanceMatrixMSAProfileDialog@@8 1001dd5c     DistanceMatrixMSAProfileDialog.obj
 0002:00004d78       ??_R3Ui_DistanceMatrixMSAProfileDialog@@8 1001dd78     DistanceMatrixMSAProfileDialog.obj
 0002:00004d88       ??_R2Ui_DistanceMatrixMSAProfileDialog@@8 1001dd88     DistanceMatrixMSAProfileDialog.obj
 0002:00004d90       ??_R1A@?0A@EA@Ui_DistanceMatrixMSAProfileDialog@@8 1001dd90     DistanceMatrixMSAProfileDialog.obj
 0002:00004dac       ??_R4DistanceMatrixMSAProfileDialog@U2@@6BQPaintDevice@@@ 1001ddac     DistanceMatrixMSAProfileDialog.obj
 0002:00004dc0       ??_R4DistanceMatrixMSAProfileTask@U2@@6B@ 1001ddc0     DistanceMatrixMSAProfileDialog.obj
 0002:00004dd4       ??_R3DistanceMatrixMSAProfileTask@U2@@8 1001ddd4     DistanceMatrixMSAProfileDialog.obj
 0002:00004de4       ??_R2DistanceMatrixMSAProfileTask@U2@@8 1001dde4     DistanceMatrixMSAProfileDialog.obj
 0002:00004df4       ??_R1A@?0A@EA@DistanceMatrixMSAProfileTask@U2@@8 1001ddf4     DistanceMatrixMSAProfileDialog.obj
 0002:00004e10       ??_R4type_info@@6B@        1001de10     MSVCRT:ti_inst.obj
 0002:00004e24       ??_R3type_info@@8          1001de24     MSVCRT:ti_inst.obj
 0002:00004e34       ??_R2type_info@@8          1001de34     MSVCRT:ti_inst.obj
 0002:00004e3c       ??_R1A@?0A@EA@type_info@@8 1001de3c     MSVCRT:ti_inst.obj
 0002:00004e60       ___safe_se_handler_table   1001de60     <linker-defined>
 0002:0000507c       ___rtc_iaa                 1001e07c     MSVCRT:initsect.obj
 0002:00005080       ___rtc_izz                 1001e080     MSVCRT:initsect.obj
 0002:00005084       ___rtc_taa                 1001e084     MSVCRT:initsect.obj
 0002:00005088       ___rtc_tzz                 1001e088     MSVCRT:initsect.obj
 0002:00008094       __IMPORT_DESCRIPTOR_U2Core 10021094     U2Core:U2Core.dll
 0002:000080a8       __IMPORT_DESCRIPTOR_U2Algorithm 100210a8     U2Algorithm:U2Algorithm.dll
 0002:000080bc       __IMPORT_DESCRIPTOR_U2Gui  100210bc     U2Gui:U2Gui.dll
 0002:000080d0       __IMPORT_DESCRIPTOR_U2View 100210d0     U2View:U2View.dll
 0002:000080e4       __IMPORT_DESCRIPTOR_Qt5Widgets 100210e4     Qt5Widgets:Qt5Widgets.dll
 0002:000080f8       __IMPORT_DESCRIPTOR_Qt5Gui 100210f8     Qt5Gui:Qt5Gui.dll
 0002:0000810c       __IMPORT_DESCRIPTOR_Qt5Core 1002110c     Qt5Core:Qt5Core.dll
 0002:00008120       __IMPORT_DESCRIPTOR_MSVCP120 10021120     msvcprt:MSVCP120.dll
 0002:00008134       __IMPORT_DESCRIPTOR_MSVCR120 10021134     MSVCRT:MSVCR120.dll
 0002:00008148       __IMPORT_DESCRIPTOR_KERNEL32 10021148     kernel32:KERNEL32.dll
 0002:0000815c       __NULL_IMPORT_DESCRIPTOR   1002115c     U2Core:U2Core.dll
 0003:00000000       ?_Generic_object@?$_Error_objects@H@std@@2V_Generic_error_category@2@A 10029000     DNAStatMSAProfileDialog.obj
 0003:00000004       ?_Iostream_object@?$_Error_objects@H@std@@2V_Iostream_error_category@2@A 10029004     DNAStatMSAProfileDialog.obj
 0003:00000008       ?_System_object@?$_Error_objects@H@std@@2V_System_error_category@2@A 10029008     DNAStatMSAProfileDialog.obj
 0003:000001ac       ?staticMetaObject@DNAStatMSAProfileDialog@U2@@2UQMetaObject@@B 100291ac     moc_DNAStatMSAProfileDialog.obj
 0003:000001c4       ?staticMetaObject@DNAStatMSAProfileTask@U2@@2UQMetaObject@@B 100291c4     moc_DNAStatMSAProfileDialog.obj
 0003:00000244       ?staticMetaObject@DNAStatPlugin@U2@@2UQMetaObject@@B 10029244     moc_DNAStatPlugin.obj
 0003:0000025c       ?staticMetaObject@DNAStatMSAEditorContext@U2@@2UQMetaObject@@B 1002925c     moc_DNAStatPlugin.obj
 0003:00000274       ?staticMetaObject@DistanceMatrixMSAEditorContext@U2@@2UQMetaObject@@B 10029274     moc_DNAStatPlugin.obj
 0003:0000028c       ?staticMetaObject@DNAStatProfileTask@U2@@2UQMetaObject@@B 1002928c     moc_DNAStatProfileTask.obj
 0003:000002a4       ?staticMetaObject@DistanceMatrixMSAProfileDialog@U2@@2UQMetaObject@@B 100292a4     moc_DistanceMatrixMSAProfileDialog.obj
 0003:000002bc       ?staticMetaObject@DistanceMatrixMSAProfileTask@U2@@2UQMetaObject@@B 100292bc     moc_DistanceMatrixMSAProfileDialog.obj
 0003:000002d4       ___security_cookie         100292d4     MSVCRT:gs_cookie.obj
 0003:000002d8       ___security_cookie_complement 100292d8     MSVCRT:gs_cookie.obj
 0003:000002e0       ___native_dllmain_reason   100292e0     MSVCRT:natstart.obj
 0003:000002e8       ??_R0?AVbad_alloc@std@@@8  100292e8     DNAStatMSAProfileDialog.obj
 0003:00000304       ??_R0?AVerror_category@std@@@8 10029304     DNAStatMSAProfileDialog.obj
 0003:00000328       ??_R0?AV_Generic_error_category@std@@@8 10029328     DNAStatMSAProfileDialog.obj
 0003:00000354       ??_R0?AV_Iostream_error_category@std@@@8 10029354     DNAStatMSAProfileDialog.obj
 0003:00000380       ??_R0?AV_System_error_category@std@@@8 10029380     DNAStatMSAProfileDialog.obj
 0003:000003ac       ??_R0?AVQFile@@@8          100293ac     DNAStatMSAProfileDialog.obj
 0003:000003c0       ??_R0?AVQFileDevice@@@8    100293c0     DNAStatMSAProfileDialog.obj
 0003:000003dc       ??_R0?AVQIODevice@@@8      100293dc     DNAStatMSAProfileDialog.obj
 0003:000003f4       ??_R0?AVQObject@@@8        100293f4     DNAStatMSAProfileDialog.obj
 0003:0000040c       ??_R0?AVQLabel@@@8         1002940c     DNAStatMSAProfileDialog.obj
 0003:00000424       ??_R0?AVQFrame@@@8         10029424     DNAStatMSAProfileDialog.obj
 0003:0000043c       ??_R0?AVQWidget@@@8        1002943c     DNAStatMSAProfileDialog.obj
 0003:00000454       ??_R0?AVQPaintDevice@@@8   10029454     DNAStatMSAProfileDialog.obj
 0003:00000470       ??_R0?AVQCheckBox@@@8      10029470     DNAStatMSAProfileDialog.obj
 0003:00000488       ??_R0?AVQAbstractButton@@@8 10029488     DNAStatMSAProfileDialog.obj
 0003:000004a8       ??_R0?AVAbstractInt32Id@U2@@@8 100294a8     DNAStatMSAProfileDialog.obj
 0003:000004cc       ??_R0?AV?$AbstractId@H@U2@@@8 100294cc     DNAStatMSAProfileDialog.obj
 0003:000004ec       ??_R0?AVServiceType@U2@@@8 100294ec     DNAStatMSAProfileDialog.obj
 0003:0000050c       ??_R0?AVQDialogButtonBox@@@8 1002950c     DNAStatMSAProfileDialog.obj
 0003:0000052c       ??_R0?AVHelpButton@U2@@@8  1002952c     DNAStatMSAProfileDialog.obj
 0003:00000548       ??_R0?AVQLineEdit@@@8      10029548     DNAStatMSAProfileDialog.obj
 0003:00000560       ??_R0?AVSaveDocumentController@U2@@@8 10029560     DNAStatMSAProfileDialog.obj
 0003:00000588       ??_R0?AVQToolButton@@@8    10029588     DNAStatMSAProfileDialog.obj
 0003:000005a4       ??_R0?AVQGridLayout@@@8    100295a4     DNAStatMSAProfileDialog.obj
 0003:000005c0       ??_R0?AVQLayout@@@8        100295c0     DNAStatMSAProfileDialog.obj
 0003:000005d8       ??_R0?AVQLayoutItem@@@8    100295d8     DNAStatMSAProfileDialog.obj
 0003:000005f4       ??_R0?AVQVBoxLayout@@@8    100295f4     DNAStatMSAProfileDialog.obj
 0003:00000610       ??_R0?AVQBoxLayout@@@8     10029610     DNAStatMSAProfileDialog.obj
 0003:0000062c       ??_R0?AVWebWindow@U2@@@8   1002962c     DNAStatMSAProfileDialog.obj
 0003:00000648       ??_R0?AVMWMDIWindow@U2@@@8 10029648     DNAStatMSAProfileDialog.obj
 0003:00000668       ??_R0?AVQGroupBox@@@8      10029668     DNAStatMSAProfileDialog.obj
 0003:00000680       ??_R0?AVQRadioButton@@@8   10029680     DNAStatMSAProfileDialog.obj
 0003:0000069c       ??_R0?AVDNAStatMSAProfileDialog@U2@@@8 1002969c     DNAStatMSAProfileDialog.obj
 0003:000006c8       ??_R0?AVQDialog@@@8        100296c8     DNAStatMSAProfileDialog.obj
 0003:000006e0       ??_R0?AVUi_DNAStatMSAProfileDialog@@@8 100296e0     DNAStatMSAProfileDialog.obj
 0003:0000070c       ??_R0?AVDNAStatMSAProfileTask@U2@@@8 1002970c     DNAStatMSAProfileDialog.obj
 0003:00000734       ??_R0?AVTask@U2@@@8        10029734     DNAStatMSAProfileDialog.obj
 0003:0000074c       ??_R0?AVGObjectViewAction@U2@@@8 1002974c     DNAStatPlugin.obj
 0003:00000770       ??_R0?AVQAction@@@8        10029770     DNAStatPlugin.obj
 0003:00000788       ??_R0?AVDNAStatPlugin@U2@@@8 10029788     DNAStatPlugin.obj
 0003:000007a8       ??_R0?AVPlugin@U2@@@8      100297a8     DNAStatPlugin.obj
 0003:000007c0       ??_R0?AVDNAStatMSAEditorContext@U2@@@8 100297c0     DNAStatPlugin.obj
 0003:000007ec       ??_R0?AVGObjectViewWindowContext@U2@@@8 100297ec     DNAStatPlugin.obj
 0003:00000818       ??_R0?AVGObjectViewObjectHandler@U2@@@8 10029818     DNAStatPlugin.obj
 0003:00000844       ??_R0?AVDistanceMatrixMSAEditorContext@U2@@@8 10029844     DNAStatPlugin.obj
 0003:00000874       ??_R0?AVCharOccurTask@U2@@@8 10029874     DNAStatProfileTask.obj
 0003:00000898       ??_R0?AV?$BackgroundTask@V?$QList@UCharOccurResult@U2@@@@@U2@@@8 10029898     DNAStatProfileTask.obj
 0003:000008dc       ??_R0?AVDinuclOccurTask@U2@@@8 100298dc     DNAStatProfileTask.obj
 0003:00000900       ??_R0?AV?$BackgroundTask@V?$QMap@VQByteArray@@_J@@@U2@@@8 10029900     DNAStatProfileTask.obj
 0003:0000093c       ??_R0?AVDNAStatisticsTask@U2@@@8 1002993c     DNAStatProfileTask.obj
 0003:00000960       ??_R0?AV?$BackgroundTask@UDNAStatistics@U2@@@U2@@@8 10029960     DNAStatProfileTask.obj
 0003:00000998       ??_R0?AVDNAStatProfileTask@U2@@@8 10029998     DNAStatProfileTask.obj
 0003:000009bc       ??_R0?AVMultipleSequenceAlignmentRow@U2@@@8 100299bc     DistanceMatrixMSAProfileDialog.obj
 0003:000009ec       ??_R0?AVMultipleAlignmentRow@U2@@@8 100299ec     DistanceMatrixMSAProfileDialog.obj
 0003:00000a14       ??_R0?AVQComboBox@@@8      10029a14     DistanceMatrixMSAProfileDialog.obj
 0003:00000a2c       ??_R0?AVQSpacerItem@@@8    10029a2c     DistanceMatrixMSAProfileDialog.obj
 0003:00000a48       ??_R0?AVQHBoxLayout@@@8    10029a48     DistanceMatrixMSAProfileDialog.obj
 0003:00000a64       ??_R0?AVDistanceMatrixMSAProfileDialog@U2@@@8 10029a64     DistanceMatrixMSAProfileDialog.obj
 0003:00000a94       ??_R0?AVUi_DistanceMatrixMSAProfileDialog@@@8 10029a94     DistanceMatrixMSAProfileDialog.obj
 0003:00000ac4       ??_R0?AVDistanceMatrixMSAProfileTask@U2@@@8 10029ac4     DistanceMatrixMSAProfileDialog.obj
 0003:00000af4       ??_R0?AVtype_info@@@8      10029af4     MSVCRT:ti_inst.obj
 0003:00000b34       ?CSV@DNAStatMSAProfileDialog@U2@@0VQString@@B 10029b34     DNAStatMSAProfileDialog.obj
 0003:00000b60       ?HTML@DNAStatMSAProfileDialog@U2@@0VQString@@B 10029b60     DNAStatMSAProfileDialog.obj
 0003:00000b64       ?id@?$num_put@DV?$back_insert_iterator@V?$basic_string@DU?$char_traits@D@std@@V?$allocator@D@2@@std@@@std@@@std@@2V0locale@2@A 10029b64     DNAStatMSAProfileDialog.obj
 0003:00000b68       ?id@?$num_put@_WV?$back_insert_iterator@V?$basic_string@_WU?$char_traits@_W@std@@V?$allocator@_W@2@@std@@@std@@@std@@2V0locale@2@A 10029b68     DNAStatMSAProfileDialog.obj
 0003:00000c30       ?HTML@DistanceMatrixMSAProfileDialog@U2@@0VQString@@B 10029c30     DistanceMatrixMSAProfileDialog.obj
 0003:00000c44       ?CSV@DistanceMatrixMSAProfileDialog@U2@@0VQString@@B 10029c44     DistanceMatrixMSAProfileDialog.obj
 0003:00000ca8       ?metatype_id@?1??qt_metatype_id@?$QMetaTypeIdQObject@PAVGObjectView@U2@@$00@@SAHXZ@4V?$QBasicAtomicInteger@H@@A 10029ca8     moc_DNAStatPlugin.obj
 0003:00000cac       ?metatype_id@?1??qt_metatype_id@?$QMetaTypeIdQObject@PAVQMenu@@$00@@SAHXZ@4V?$QBasicAtomicInteger@H@@A 10029cac     moc_DNAStatPlugin.obj
 0003:00001070       ?__type_info_root_node@@3U__type_info_node@@A 1002a070     MSVCRT:tncleanup.obj
 0003:00001078       ___native_startup_lock     1002a078     <common>
 0003:0000107c       ___native_startup_state    1002a07c     <common>
 0003:00001080       ___dyn_tls_init_callback   1002a080     <common>
 0003:00001084       ___onexitend               1002a084     <common>
 0003:00001088       ___onexitbegin             1002a088     <common>

 entry point at        0001:00013dac

 Static symbols

 0001:fffff000       __ehhandler$?_Copy@?$basic_string@DU?$char_traits@D@std@@V?$allocator@D@2@@std@@QAEXII@Z 10000000 f   DNAStatPlugin.obj
 0000:fffd0000       .debug$S                   10000000     MSVCRT:MSVCR120.dll
 0000:fffd0000       .debug$S                   10000000     MSVCRT:MSVCR120.dll
 0000:fffd0000       .debug$S                   10000000     MSVCRT:MSVCR120.dll
 0000:fffd0000       .debug$S                   10000000     MSVCRT:MSVCR120.dll
 0000:fffd0000       .debug$S                   10000000     MSVCRT:MSVCR120.dll
 0000:fffd0000       .debug$S                   10000000     MSVCRT:MSVCR120.dll
 0000:fffd0000       .debug$S                   10000000     MSVCRT:MSVCR120.dll
 0000:fffd0000       .debug$S                   10000000     MSVCRT:MSVCR120.dll
 0000:fffd0000       .debug$S                   10000000     MSVCRT:MSVCR120.dll
 0000:fffd0000       .debug$S                   10000000     MSVCRT:MSVCR120.dll
 0000:fffd0000       .debug$S                   10000000     MSVCRT:MSVCR120.dll
 0000:fffd0000       .debug$S                   10000000     MSVCRT:MSVCR120.dll
 0000:fffd0000       .debug$S                   10000000     MSVCRT:MSVCR120.dll
 0000:fffd0000       .debug$S                   10000000     MSVCRT:MSVCR120.dll
 0000:fffd0000       .debug$S                   10000000     MSVCRT:MSVCR120.dll
 0000:fffd0000       .debug$S                   10000000     MSVCRT:MSVCR120.dll
 0000:fffd0000       .debug$S                   10000000     MSVCRT:MSVCR120.dll
 0000:fffd0000       .debug$S                   10000000     MSVCRT:MSVCR120.dll
 0000:fffd0000       .debug$S                   10000000     MSVCRT:MSVCR120.dll
 0000:fffd0000       .debug$S                   10000000     MSVCRT:MSVCR120.dll
 0000:fffd0000       .debug$S                   10000000     MSVCRT:MSVCR120.dll
 0000:fffd0000       .debug$S                   10000000     MSVCRT:MSVCR120.dll
 0000:fffd0000       .debug$S                   10000000     MSVCRT:MSVCR120.dll
 0000:fffd0000       .debug$S                   10000000     MSVCRT:MSVCR120.dll
 0000:fffd0000       .debug$S                   10000000     MSVCRT:MSVCR120.dll
 0000:fffd0000       .debug$S                   10000000     MSVCRT:MSVCR120.dll
 0000:fffd0000       .debug$S                   10000000     MSVCRT:MSVCR120.dll
 0000:fffd0000       .debug$S                   10000000     MSVCRT:MSVCR120.dll
 0000:fffd0000       .debug$S                   10000000     msvcprt:MSVCP120.dll
 0000:fffd0000       .debug$S                   10000000     msvcprt:MSVCP120.dll
 0000:fffd0000       .debug$S                   10000000     msvcprt:MSVCP120.dll
 0000:fffd0000       .debug$S                   10000000     msvcprt:MSVCP120.dll
 0000:fffd0000       .debug$S                   10000000     msvcprt:MSVCP120.dll
 0000:fffd0000       .debug$S                   10000000     kernel32:KERNEL32.dll
 0000:fffd0000       .debug$S                   10000000     kernel32:KERNEL32.dll
 0000:fffd0000       .debug$S                   10000000     kernel32:KERNEL32.dll
 0001:fffff000       __ehhandler$?_Copy@?$basic_string@DU?$char_traits@D@std@@V?$allocator@D@2@@std@@QAEXII@Z 10000000 f   moc_DistanceMatrixMSAProfileDialog.obj
 0000:fffd0000       .debug$S                   10000000     kernel32:KERNEL32.dll
 0000:fffd0000       .debug$S                   10000000     kernel32:KERNEL32.dll
 0000:fffd0000       .debug$S                   10000000     kernel32:KERNEL32.dll
 0000:fffd0000       .debug$S                   10000000     kernel32:KERNEL32.dll
 0000:fffd0000       .debug$S                   10000000     kernel32:KERNEL32.dll
 0000:fffd0000       .debug$S                   10000000     kernel32:KERNEL32.dll
 0000:fffd0000       .debug$S                   10000000     Qt5Core:Qt5Core.dll
 0000:fffd0000       .debug$S                   10000000     Qt5Core:Qt5Core.dll
 0000:fffd0000       .debug$S                   10000000     Qt5Core:Qt5Core.dll
 0000:fffd0000       .debug$S                   10000000     Qt5Core:Qt5Core.dll
 0000:fffd0000       .debug$S                   10000000     Qt5Core:Qt5Core.dll
 0000:fffd0000       .debug$S                   10000000     Qt5Core:Qt5Core.dll
 0000:fffd0000       .debug$S                   10000000     Qt5Core:Qt5Core.dll
 0000:fffd0000       .debug$S                   10000000     Qt5Core:Qt5Core.dll
 0000:fffd0000       .debug$S                   10000000     Qt5Core:Qt5Core.dll
 0000:fffd0000       .debug$S                   10000000     Qt5Core:Qt5Core.dll
 0000:fffd0000       .debug$S                   10000000     Qt5Core:Qt5Core.dll
 0000:fffd0000       .debug$S                   10000000     Qt5Core:Qt5Core.dll
 0000:fffd0000       .debug$S                   10000000     Qt5Core:Qt5Core.dll
 0000:fffd0000       .debug$S                   10000000     Qt5Core:Qt5Core.dll
 0000:fffd0000       .debug$S                   10000000     Qt5Core:Qt5Core.dll
 0000:fffd0000       .debug$S                   10000000     Qt5Core:Qt5Core.dll
 0000:fffd0000       .debug$S                   10000000     Qt5Core:Qt5Core.dll
 0000:fffd0000       .debug$S                   10000000     Qt5Core:Qt5Core.dll
 0002:fffe7000       __catchsym$?_Copy@?$basic_string@DU?$char_traits@D@std@@V?$allocator@D@2@@std@@QAEXII@Z$5 10000000     moc_DistanceMatrixMSAProfileDialog.obj
 0000:fffd0000       .debug$S                   10000000     Qt5Core:Qt5Core.dll
 0000:fffd0000       .debug$S                   10000000     Qt5Core:Qt5Core.dll
 0000:fffd0000       .debug$S                   10000000     Qt5Core:Qt5Core.dll
 0000:fffd0000       .debug$S                   10000000     Qt5Core:Qt5Core.dll
 0000:fffd0000       .debug$S                   10000000     Qt5Core:Qt5Core.dll
 0000:fffd0000       .debug$S                   10000000     Qt5Core:Qt5Core.dll
 0000:fffd0000       .debug$S                   10000000     Qt5Core:Qt5Core.dll
 0000:fffd0000       .debug$S                   10000000     Qt5Core:Qt5Core.dll
 0000:fffd0000       .debug$S                   10000000     Qt5Core:Qt5Core.dll
 0000:fffd0000       .debug$S                   10000000     Qt5Core:Qt5Core.dll
 0000:fffd0000       .debug$S                   10000000     Qt5Core:Qt5Core.dll
 0000:fffd0000       .debug$S                   10000000     Qt5Core:Qt5Core.dll
 0000:fffd0000       .debug$S                   10000000     Qt5Core:Qt5Core.dll
 0000:fffd0000       .debug$S                   10000000     Qt5Core:Qt5Core.dll
 0000:fffd0000       .debug$S                   10000000     Qt5Core:Qt5Core.dll
 0000:fffd0000       .debug$S                   10000000     Qt5Core:Qt5Core.dll
 0000:fffd0000       .debug$S                   10000000     Qt5Core:Qt5Core.dll
 0000:fffd0000       .debug$S                   10000000     Qt5Core:Qt5Core.dll
 0000:fffd0000       .debug$S                   10000000     Qt5Core:Qt5Core.dll
 0000:fffd0000       .debug$S                   10000000     Qt5Core:Qt5Core.dll
 0000:fffd0000       .debug$S                   10000000     Qt5Core:Qt5Core.dll
 0000:fffd0000       .debug$S                   10000000     Qt5Core:Qt5Core.dll
 0000:fffd0000       .debug$S                   10000000     Qt5Core:Qt5Core.dll
 0000:fffd0000       .debug$S                   10000000     Qt5Core:Qt5Core.dll
 0000:fffd0000       .debug$S                   10000000     Qt5Core:Qt5Core.dll
 0000:fffd0000       .debug$S                   10000000     Qt5Core:Qt5Core.dll
 0000:fffd0000       .debug$S                   10000000     Qt5Core:Qt5Core.dll
 0000:fffd0000       .debug$S                   10000000     Qt5Core:Qt5Core.dll
 0000:fffd0000       .debug$S                   10000000     Qt5Core:Qt5Core.dll
 0000:fffd0000       .debug$S                   10000000     Qt5Core:Qt5Core.dll
 0000:fffd0000       .debug$S                   10000000     Qt5Core:Qt5Core.dll
 0000:fffd0000       .debug$S                   10000000     Qt5Core:Qt5Core.dll
 0000:fffd0000       .debug$S                   10000000     Qt5Core:Qt5Core.dll
 0000:fffd0000       .debug$S                   10000000     Qt5Core:Qt5Core.dll
 0000:fffd0000       .debug$S                   10000000     Qt5Core:Qt5Core.dll
 0000:fffd0000       .debug$S                   10000000     Qt5Core:Qt5Core.dll
 0000:fffd0000       .debug$S                   10000000     Qt5Core:Qt5Core.dll
 0000:fffd0000       .debug$S                   10000000     Qt5Core:Qt5Core.dll
 0000:fffd0000       .debug$S                   10000000     Qt5Core:Qt5Core.dll
 0000:fffd0000       .debug$S                   10000000     Qt5Core:Qt5Core.dll
 0000:fffd0000       .debug$S                   10000000     Qt5Core:Qt5Core.dll
 0000:fffd0000       .debug$S                   10000000     Qt5Core:Qt5Core.dll
 0002:fffe7000       ?_Generic_object$initializer$@?$_Error_objects@H@std@@2P6AXXZA 10000000     moc_DistanceMatrixMSAProfileDialog.obj
 0002:fffe7000       ?_Iostream_object$initializer$@?$_Error_objects@H@std@@2P6AXXZA 10000000     moc_DistanceMatrixMSAProfileDialog.obj
 0002:fffe7000       ?_System_object$initializer$@?$_Error_objects@H@std@@2P6AXXZA 10000000     moc_DistanceMatrixMSAProfileDialog.obj
 0000:fffd0000       .debug$S                   10000000     Qt5Core:Qt5Core.dll
 0000:fffd0000       .debug$S                   10000000     Qt5Core:Qt5Core.dll
 0000:fffd0000       .debug$S                   10000000     Qt5Core:Qt5Core.dll
 0000:fffd0000       .debug$S                   10000000     Qt5Core:Qt5Core.dll
 0000:fffd0000       .debug$S                   10000000     Qt5Core:Qt5Core.dll
 0000:fffd0000       .debug$S                   10000000     Qt5Core:Qt5Core.dll
 0000:fffd0000       .debug$S                   10000000     Qt5Core:Qt5Core.dll
 0000:fffd0000       .debug$S                   10000000     Qt5Core:Qt5Core.dll
 0000:fffd0000       .debug$S                   10000000     Qt5Core:Qt5Core.dll
 0000:fffd0000       .debug$S                   10000000     Qt5Core:Qt5Core.dll
 0000:fffd0000       .debug$S                   10000000     Qt5Core:Qt5Core.dll
 0000:fffd0000       .debug$S                   10000000     Qt5Core:Qt5Core.dll
 0000:fffd0000       .debug$S                   10000000     Qt5Core:Qt5Core.dll
 0000:fffd0000       .debug$S                   10000000     Qt5Core:Qt5Core.dll
 0000:fffd0000       .debug$S                   10000000     Qt5Core:Qt5Core.dll
 0000:fffd0000       .debug$S                   10000000     Qt5Core:Qt5Core.dll
 0000:fffd0000       .debug$S                   10000000     Qt5Core:Qt5Core.dll
 0000:fffd0000       .debug$S                   10000000     Qt5Core:Qt5Core.dll
 0000:fffd0000       .debug$S                   10000000     Qt5Core:Qt5Core.dll
 0000:fffd0000       .debug$S                   10000000     Qt5Core:Qt5Core.dll
 0000:fffd0000       .debug$S                   10000000     Qt5Core:Qt5Core.dll
 0000:fffd0000       .debug$S                   10000000     Qt5Core:Qt5Core.dll
 0000:fffd0000       .debug$S                   10000000     Qt5Core:Qt5Core.dll
 0000:fffd0000       .debug$S                   10000000     Qt5Core:Qt5Core.dll
 0000:fffd0000       .debug$S                   10000000     Qt5Core:Qt5Core.dll
 0000:fffd0000       .debug$S                   10000000     Qt5Core:Qt5Core.dll
 0000:fffd0000       .debug$S                   10000000     Qt5Core:Qt5Core.dll
 0001:fffff000       __ehhandler$?_Copy@?$basic_string@DU?$char_traits@D@std@@V?$allocator@D@2@@std@@QAEXII@Z 10000000 f   moc_DNAStatProfileTask.obj
 0000:fffd0000       .debug$S                   10000000     Qt5Core:Qt5Core.dll
 0000:fffd0000       .debug$S                   10000000     Qt5Core:Qt5Core.dll
 0000:fffd0000       .debug$S                   10000000     Qt5Core:Qt5Core.dll
 0000:fffd0000       .debug$S                   10000000     Qt5Core:Qt5Core.dll
 0000:fffd0000       .debug$S                   10000000     Qt5Core:Qt5Core.dll
 0000:fffd0000       .debug$S                   10000000     Qt5Core:Qt5Core.dll
 0000:fffd0000       .debug$S                   10000000     Qt5Core:Qt5Core.dll
 0000:fffd0000       .debug$S                   10000000     Qt5Core:Qt5Core.dll
 0000:fffd0000       .debug$S                   10000000     Qt5Core:Qt5Core.dll
 0000:fffd0000       .debug$S                   10000000     Qt5Core:Qt5Core.dll
 0000:fffd0000       .debug$S                   10000000     Qt5Core:Qt5Core.dll
 0000:fffd0000       .debug$S                   10000000     Qt5Core:Qt5Core.dll
 0000:fffd0000       .debug$S                   10000000     Qt5Core:Qt5Core.dll
 0000:fffd0000       .debug$S                   10000000     Qt5Core:Qt5Core.dll
 0000:fffd0000       .debug$S                   10000000     Qt5Core:Qt5Core.dll
 0000:fffd0000       .debug$S                   10000000     Qt5Core:Qt5Core.dll
 0000:fffd0000       .debug$S                   10000000     Qt5Core:Qt5Core.dll
 0000:fffd0000       .debug$S                   10000000     Qt5Core:Qt5Core.dll
 0000:fffd0000       .debug$S                   10000000     Qt5Core:Qt5Core.dll
 0000:fffd0000       .debug$S                   10000000     Qt5Core:Qt5Core.dll
 0000:fffd0000       .debug$S                   10000000     Qt5Core:Qt5Core.dll
 0000:fffd0000       .debug$S                   10000000     Qt5Core:Qt5Core.dll
 0000:fffd0000       .debug$S                   10000000     Qt5Core:Qt5Core.dll
 0000:fffd0000       .debug$S                   10000000     Qt5Core:Qt5Core.dll
 0002:fffe7000       __catchsym$?_Copy@?$basic_string@DU?$char_traits@D@std@@V?$allocator@D@2@@std@@QAEXII@Z$5 10000000     moc_DNAStatProfileTask.obj
 0000:fffd0000       .debug$S                   10000000     Qt5Core:Qt5Core.dll
 0000:fffd0000       .debug$S                   10000000     Qt5Core:Qt5Core.dll
 0000:fffd0000       .debug$S                   10000000     Qt5Core:Qt5Core.dll
 0000:fffd0000       .debug$S                   10000000     Qt5Core:Qt5Core.dll
 0000:fffd0000       .debug$S                   10000000     Qt5Gui:Qt5Gui.dll
 0000:fffd0000       .debug$S                   10000000     Qt5Gui:Qt5Gui.dll
 0000:fffd0000       .debug$S                   10000000     Qt5Gui:Qt5Gui.dll
 0000:fffd0000       .debug$S                   10000000     Qt5Widgets:Qt5Widgets.dll
 0000:fffd0000       .debug$S                   10000000     Qt5Widgets:Qt5Widgets.dll
 0000:fffd0000       .debug$S                   10000000     Qt5Widgets:Qt5Widgets.dll
 0000:fffd0000       .debug$S                   10000000     Qt5Widgets:Qt5Widgets.dll
 0000:fffd0000       .debug$S                   10000000     Qt5Widgets:Qt5Widgets.dll
 0000:fffd0000       .debug$S                   10000000     Qt5Widgets:Qt5Widgets.dll
 0000:fffd0000       .debug$S                   10000000     Qt5Widgets:Qt5Widgets.dll
 0000:fffd0000       .debug$S                   10000000     Qt5Widgets:Qt5Widgets.dll
 0000:fffd0000       .debug$S                   10000000     Qt5Widgets:Qt5Widgets.dll
 0000:fffd0000       .debug$S                   10000000     Qt5Widgets:Qt5Widgets.dll
 0000:fffd0000       .debug$S                   10000000     Qt5Widgets:Qt5Widgets.dll
 0000:fffd0000       .debug$S                   10000000     Qt5Widgets:Qt5Widgets.dll
 0000:fffd0000       .debug$S                   10000000     Qt5Widgets:Qt5Widgets.dll
 0000:fffd0000       .debug$S                   10000000     Qt5Widgets:Qt5Widgets.dll
 0000:fffd0000       .debug$S                   10000000     Qt5Widgets:Qt5Widgets.dll
 0000:fffd0000       .debug$S                   10000000     Qt5Widgets:Qt5Widgets.dll
 0000:fffd0000       .debug$S                   10000000     Qt5Widgets:Qt5Widgets.dll
 0000:fffd0000       .debug$S                   10000000     Qt5Widgets:Qt5Widgets.dll
 0000:fffd0000       .debug$S                   10000000     Qt5Widgets:Qt5Widgets.dll
 0000:fffd0000       .debug$S                   10000000     Qt5Widgets:Qt5Widgets.dll
 0000:fffd0000       .debug$S                   10000000     Qt5Widgets:Qt5Widgets.dll
 0000:fffd0000       .debug$S                   10000000     Qt5Widgets:Qt5Widgets.dll
 0000:fffd0000       .debug$S                   10000000     Qt5Widgets:Qt5Widgets.dll
 0000:fffd0000       .debug$S                   10000000     Qt5Widgets:Qt5Widgets.dll
 0000:fffd0000       .debug$S                   10000000     Qt5Widgets:Qt5Widgets.dll
 0000:fffd0000       .debug$S                   10000000     Qt5Widgets:Qt5Widgets.dll
 0000:fffd0000       .debug$S                   10000000     Qt5Widgets:Qt5Widgets.dll
 0000:fffd0000       .debug$S                   10000000     Qt5Widgets:Qt5Widgets.dll
 0000:fffd0000       .debug$S                   10000000     Qt5Widgets:Qt5Widgets.dll
 0000:fffd0000       .debug$S                   10000000     Qt5Widgets:Qt5Widgets.dll
 0000:fffd0000       .debug$S                   10000000     Qt5Widgets:Qt5Widgets.dll
 0000:fffd0000       .debug$S                   10000000     Qt5Widgets:Qt5Widgets.dll
 0000:fffd0000       .debug$S                   10000000     Qt5Widgets:Qt5Widgets.dll
 0000:fffd0000       .debug$S                   10000000     Qt5Widgets:Qt5Widgets.dll
 0002:fffe7000       ?_Generic_object$initializer$@?$_Error_objects@H@std@@2P6AXXZA 10000000     moc_DNAStatProfileTask.obj
 0002:fffe7000       ?_Iostream_object$initializer$@?$_Error_objects@H@std@@2P6AXXZA 10000000     moc_DNAStatProfileTask.obj
 0002:fffe7000       ?_System_object$initializer$@?$_Error_objects@H@std@@2P6AXXZA 10000000     moc_DNAStatProfileTask.obj
 0000:fffd0000       .debug$S                   10000000     Qt5Widgets:Qt5Widgets.dll
 0000:fffd0000       .debug$S                   10000000     Qt5Widgets:Qt5Widgets.dll
 0000:fffd0000       .debug$S                   10000000     Qt5Widgets:Qt5Widgets.dll
 0000:fffd0000       .debug$S                   10000000     Qt5Widgets:Qt5Widgets.dll
 0000:fffd0000       .debug$S                   10000000     Qt5Widgets:Qt5Widgets.dll
 0000:fffd0000       .debug$S                   10000000     Qt5Widgets:Qt5Widgets.dll
 0000:fffd0000       .debug$S                   10000000     Qt5Widgets:Qt5Widgets.dll
 0000:fffd0000       .debug$S                   10000000     Qt5Widgets:Qt5Widgets.dll
 0000:fffd0000       .debug$S                   10000000     Qt5Widgets:Qt5Widgets.dll
 0000:fffd0000       .debug$S                   10000000     Qt5Widgets:Qt5Widgets.dll
 0000:fffd0000       .debug$S                   10000000     Qt5Widgets:Qt5Widgets.dll
 0000:fffd0000       .debug$S                   10000000     Qt5Widgets:Qt5Widgets.dll
 0000:fffd0000       .debug$S                   10000000     Qt5Widgets:Qt5Widgets.dll
 0000:fffd0000       .debug$S                   10000000     Qt5Widgets:Qt5Widgets.dll
 0000:fffd0000       .debug$S                   10000000     Qt5Widgets:Qt5Widgets.dll
 0000:fffd0000       .debug$S                   10000000     Qt5Widgets:Qt5Widgets.dll
 0000:fffd0000       .debug$S                   10000000     Qt5Widgets:Qt5Widgets.dll
 0000:fffd0000       .debug$S                   10000000     Qt5Widgets:Qt5Widgets.dll
 0000:fffd0000       .debug$S                   10000000     Qt5Widgets:Qt5Widgets.dll
 0000:fffd0000       .debug$S                   10000000     Qt5Widgets:Qt5Widgets.dll
 0000:fffd0000       .debug$S                   10000000     Qt5Widgets:Qt5Widgets.dll
 0000:fffd0000       .debug$S                   10000000     Qt5Widgets:Qt5Widgets.dll
 0000:fffd0000       .debug$S                   10000000     Qt5Widgets:Qt5Widgets.dll
 0000:fffd0000       .debug$S                   10000000     Qt5Widgets:Qt5Widgets.dll
 0000:fffd0000       .debug$S                   10000000     Qt5Widgets:Qt5Widgets.dll
 0000:fffd0000       .debug$S                   10000000     Qt5Widgets:Qt5Widgets.dll
 0000:fffd0000       .debug$S                   10000000     Qt5Widgets:Qt5Widgets.dll
 0000:fffd0000       .debug$S                   10000000     Qt5Widgets:Qt5Widgets.dll
 0000:fffd0000       .debug$S                   10000000     Qt5Widgets:Qt5Widgets.dll
 0000:fffd0000       .debug$S                   10000000     Qt5Widgets:Qt5Widgets.dll
 0000:fffd0000       .debug$S                   10000000     Qt5Widgets:Qt5Widgets.dll
 0000:fffd0000       .debug$S                   10000000     Qt5Widgets:Qt5Widgets.dll
 0000:fffd0000       .debug$S                   10000000     Qt5Widgets:Qt5Widgets.dll
 0000:fffd0000       .debug$S                   10000000     Qt5Widgets:Qt5Widgets.dll
 0000:fffd0000       .debug$S                   10000000     Qt5Widgets:Qt5Widgets.dll
 0000:fffd0000       .debug$S                   10000000     Qt5Widgets:Qt5Widgets.dll
 0000:fffd0000       .debug$S                   10000000     Qt5Widgets:Qt5Widgets.dll
 0000:fffd0000       .debug$S                   10000000     Qt5Widgets:Qt5Widgets.dll
 0000:fffd0000       .debug$S                   10000000     Qt5Widgets:Qt5Widgets.dll
 0000:fffd0000       .debug$S                   10000000     Qt5Widgets:Qt5Widgets.dll
 0000:fffd0000       .debug$S                   10000000     Qt5Widgets:Qt5Widgets.dll
 0001:fffff000       __ehhandler$?_Copy@?$basic_string@DU?$char_traits@D@std@@V?$allocator@D@2@@std@@QAEXII@Z 10000000 f   moc_DNAStatPlugin.obj
 0000:fffd0000       .debug$S                   10000000     Qt5Widgets:Qt5Widgets.dll
 0000:fffd0000       .debug$S                   10000000     Qt5Widgets:Qt5Widgets.dll
 0000:fffd0000       .debug$S                   10000000     Qt5Widgets:Qt5Widgets.dll
 0000:fffd0000       .debug$S                   10000000     Qt5Widgets:Qt5Widgets.dll
 0000:fffd0000       .debug$S                   10000000     Qt5Widgets:Qt5Widgets.dll
 0000:fffd0000       .debug$S                   10000000     Qt5Widgets:Qt5Widgets.dll
 0000:fffd0000       .debug$S                   10000000     Qt5Widgets:Qt5Widgets.dll
 0000:fffd0000       .debug$S                   10000000     Qt5Widgets:Qt5Widgets.dll
 0000:fffd0000       .debug$S                   10000000     Qt5Widgets:Qt5Widgets.dll
 0000:fffd0000       .debug$S                   10000000     Qt5Widgets:Qt5Widgets.dll
 0002:fffe7000       __catchsym$?_Copy@?$basic_string@DU?$char_traits@D@std@@V?$allocator@D@2@@std@@QAEXII@Z$5 10000000     moc_DNAStatPlugin.obj
 0000:fffd0000       .debug$S                   10000000     Qt5Widgets:Qt5Widgets.dll
 0000:fffd0000       .debug$S                   10000000     Qt5Widgets:Qt5Widgets.dll
 0000:fffd0000       .debug$S                   10000000     Qt5Widgets:Qt5Widgets.dll
 0000:fffd0000       .debug$S                   10000000     Qt5Widgets:Qt5Widgets.dll
 0000:fffd0000       .debug$S                   10000000     Qt5Widgets:Qt5Widgets.dll
 0000:fffd0000       .debug$S                   10000000     Qt5Widgets:Qt5Widgets.dll
 0000:fffd0000       .debug$S                   10000000     Qt5Widgets:Qt5Widgets.dll
 0000:fffd0000       .debug$S                   10000000     Qt5Widgets:Qt5Widgets.dll
 0000:fffd0000       .debug$S                   10000000     Qt5Widgets:Qt5Widgets.dll
 0000:fffd0000       .debug$S                   10000000     Qt5Widgets:Qt5Widgets.dll
 0000:fffd0000       .debug$S                   10000000     Qt5Widgets:Qt5Widgets.dll
 0000:fffd0000       .debug$S                   10000000     Qt5Widgets:Qt5Widgets.dll
 0000:fffd0000       .debug$S                   10000000     Qt5Widgets:Qt5Widgets.dll
 0000:fffd0000       .debug$S                   10000000     Qt5Widgets:Qt5Widgets.dll
 0000:fffd0000       .debug$S                   10000000     Qt5Widgets:Qt5Widgets.dll
 0000:fffd0000       .debug$S                   10000000     Qt5Widgets:Qt5Widgets.dll
 0000:fffd0000       .debug$S                   10000000     Qt5Widgets:Qt5Widgets.dll
 0000:fffd0000       .debug$S                   10000000     Qt5Widgets:Qt5Widgets.dll
 0000:fffd0000       .debug$S                   10000000     Qt5Widgets:Qt5Widgets.dll
 0000:fffd0000       .debug$S                   10000000     Qt5Widgets:Qt5Widgets.dll
 0000:fffd0000       .debug$S                   10000000     Qt5Widgets:Qt5Widgets.dll
 0000:fffd0000       .debug$S                   10000000     Qt5Widgets:Qt5Widgets.dll
 0000:fffd0000       .debug$S                   10000000     Qt5Widgets:Qt5Widgets.dll
 0000:fffd0000       .debug$S                   10000000     Qt5Widgets:Qt5Widgets.dll
 0000:fffd0000       .debug$S                   10000000     Qt5Widgets:Qt5Widgets.dll
 0000:fffd0000       .debug$S                   10000000     Qt5Widgets:Qt5Widgets.dll
 0000:fffd0000       .debug$S                   10000000     Qt5Widgets:Qt5Widgets.dll
 0000:fffd0000       .debug$S                   10000000     Qt5Widgets:Qt5Widgets.dll
 0000:fffd0000       .debug$S                   10000000     Qt5Widgets:Qt5Widgets.dll
 0000:fffd0000       .debug$S                   10000000     Qt5Widgets:Qt5Widgets.dll
 0000:fffd0000       .debug$S                   10000000     Qt5Widgets:Qt5Widgets.dll
 0000:fffd0000       .debug$S                   10000000     Qt5Widgets:Qt5Widgets.dll
 0000:fffd0000       .debug$S                   10000000     Qt5Widgets:Qt5Widgets.dll
 0000:fffd0000       .debug$S                   10000000     Qt5Widgets:Qt5Widgets.dll
 0000:fffd0000       .debug$S                   10000000     Qt5Widgets:Qt5Widgets.dll
 0000:fffd0000       .debug$S                   10000000     Qt5Widgets:Qt5Widgets.dll
 0000:fffd0000       .debug$S                   10000000     Qt5Widgets:Qt5Widgets.dll
 0002:fffe7000       ?_Generic_object$initializer$@?$_Error_objects@H@std@@2P6AXXZA 10000000     moc_DNAStatPlugin.obj
 0002:fffe7000       ?_Iostream_object$initializer$@?$_Error_objects@H@std@@2P6AXXZA 10000000     moc_DNAStatPlugin.obj
 0002:fffe7000       ?_System_object$initializer$@?$_Error_objects@H@std@@2P6AXXZA 10000000     moc_DNAStatPlugin.obj
 0000:fffd0000       .debug$S                   10000000     Qt5Widgets:Qt5Widgets.dll
 0000:fffd0000       .debug$S                   10000000     Qt5Widgets:Qt5Widgets.dll
 0000:fffd0000       .debug$S                   10000000     Qt5Widgets:Qt5Widgets.dll
 0000:fffd0000       .debug$S                   10000000     Qt5Widgets:Qt5Widgets.dll
 0000:fffd0000       .debug$S                   10000000     Qt5Widgets:Qt5Widgets.dll
 0000:fffd0000       .debug$S                   10000000     Qt5Widgets:Qt5Widgets.dll
 0000:fffd0000       .debug$S                   10000000     Qt5Widgets:Qt5Widgets.dll
 0000:fffd0000       .debug$S                   10000000     Qt5Widgets:Qt5Widgets.dll
 0000:fffd0000       .debug$S                   10000000     Qt5Widgets:Qt5Widgets.dll
 0000:fffd0000       .debug$S                   10000000     Qt5Widgets:Qt5Widgets.dll
 0000:fffd0000       .debug$S                   10000000     Qt5Widgets:Qt5Widgets.dll
 0000:fffd0000       .debug$S                   10000000     Qt5Widgets:Qt5Widgets.dll
 0000:fffd0000       .debug$S                   10000000     Qt5Widgets:Qt5Widgets.dll
 0000:fffd0000       .debug$S                   10000000     Qt5Widgets:Qt5Widgets.dll
 0000:fffd0000       .debug$S                   10000000     Qt5Widgets:Qt5Widgets.dll
 0000:fffd0000       .debug$S                   10000000     Qt5Widgets:Qt5Widgets.dll
 0000:fffd0000       .debug$S                   10000000     Qt5Widgets:Qt5Widgets.dll
 0000:fffd0000       .debug$S                   10000000     Qt5Widgets:Qt5Widgets.dll
 0000:fffd0000       .debug$S                   10000000     Qt5Widgets:Qt5Widgets.dll
 0000:fffd0000       .debug$S                   10000000     Qt5Widgets:Qt5Widgets.dll
 0000:fffd0000       .debug$S                   10000000     Qt5Widgets:Qt5Widgets.dll
 0000:fffd0000       .debug$S                   10000000     Qt5Widgets:Qt5Widgets.dll
 0000:fffd0000       .debug$S                   10000000     Qt5Widgets:Qt5Widgets.dll
 0000:fffd0000       .debug$S                   10000000     Qt5Widgets:Qt5Widgets.dll
 0000:fffd0000       .debug$S                   10000000     Qt5Widgets:Qt5Widgets.dll
 0000:fffd0000       .debug$S                   10000000     Qt5Widgets:Qt5Widgets.dll
 0000:fffd0000       .debug$S                   10000000     Qt5Widgets:Qt5Widgets.dll
 0000:fffd0000       .debug$S                   10000000     Qt5Widgets:Qt5Widgets.dll
 0000:fffd0000       .debug$S                   10000000     Qt5Widgets:Qt5Widgets.dll
 0000:fffd0000       .debug$S                   10000000     Qt5Widgets:Qt5Widgets.dll
 0001:fffff000       __ehhandler$?_Copy@?$basic_string@DU?$char_traits@D@std@@V?$allocator@D@2@@std@@QAEXII@Z 10000000 f   moc_DNAStatMSAProfileDialog.obj
 0000:fffd0000       .debug$S                   10000000     Qt5Widgets:Qt5Widgets.dll
 0000:fffd0000       .debug$S                   10000000     Qt5Widgets:Qt5Widgets.dll
 0000:fffd0000       .debug$S                   10000000     Qt5Widgets:Qt5Widgets.dll
 0000:fffd0000       .debug$S                   10000000     Qt5Widgets:Qt5Widgets.dll
 0000:fffd0000       .debug$S                   10000000     Qt5Widgets:Qt5Widgets.dll
 0000:fffd0000       .debug$S                   10000000     Qt5Widgets:Qt5Widgets.dll
 0000:fffd0000       .debug$S                   10000000     Qt5Widgets:Qt5Widgets.dll
 0000:fffd0000       .debug$S                   10000000     Qt5Widgets:Qt5Widgets.dll
 0000:fffd0000       .debug$S                   10000000     Qt5Widgets:Qt5Widgets.dll
 0000:fffd0000       .debug$S                   10000000     Qt5Widgets:Qt5Widgets.dll
 0000:fffd0000       .debug$S                   10000000     Qt5Widgets:Qt5Widgets.dll
 0000:fffd0000       .debug$S                   10000000     Qt5Widgets:Qt5Widgets.dll
 0000:fffd0000       .debug$S                   10000000     Qt5Widgets:Qt5Widgets.dll
 0000:fffd0000       .debug$S                   10000000     Qt5Widgets:Qt5Widgets.dll
 0000:fffd0000       .debug$S                   10000000     Qt5Widgets:Qt5Widgets.dll
 0000:fffd0000       .debug$S                   10000000     Qt5Widgets:Qt5Widgets.dll
 0000:fffd0000       .debug$S                   10000000     Qt5Widgets:Qt5Widgets.dll
 0000:fffd0000       .debug$S                   10000000     Qt5Widgets:Qt5Widgets.dll
 0000:fffd0000       .debug$S                   10000000     Qt5Widgets:Qt5Widgets.dll
 0000:fffd0000       .debug$S                   10000000     Qt5Widgets:Qt5Widgets.dll
 0000:fffd0000       .debug$S                   10000000     Qt5Widgets:Qt5Widgets.dll
 0000:fffd0000       .debug$S                   10000000     Qt5Widgets:Qt5Widgets.dll
 0000:fffd0000       .debug$S                   10000000     Qt5Widgets:Qt5Widgets.dll
 0000:fffd0000       .debug$S                   10000000     Qt5Widgets:Qt5Widgets.dll
 0002:fffe7000       __catchsym$?_Copy@?$basic_string@DU?$char_traits@D@std@@V?$allocator@D@2@@std@@QAEXII@Z$5 10000000     moc_DNAStatMSAProfileDialog.obj
 0000:fffd0000       .debug$S                   10000000     Qt5Widgets:Qt5Widgets.dll
 0000:fffd0000       .debug$S                   10000000     Qt5Widgets:Qt5Widgets.dll
 0000:fffd0000       .debug$S                   10000000     Qt5Widgets:Qt5Widgets.dll
 0000:fffd0000       .debug$S                   10000000     Qt5Widgets:Qt5Widgets.dll
 0000:fffd0000       .debug$S                   10000000     Qt5Widgets:Qt5Widgets.dll
 0000:fffd0000       .debug$S                   10000000     Qt5Widgets:Qt5Widgets.dll
 0000:fffd0000       .debug$S                   10000000     Qt5Widgets:Qt5Widgets.dll
 0000:fffd0000       .debug$S                   10000000     Qt5Widgets:Qt5Widgets.dll
 0000:fffd0000       .debug$S                   10000000     Qt5Widgets:Qt5Widgets.dll
 0000:fffd0000       .debug$S                   10000000     Qt5Widgets:Qt5Widgets.dll
 0000:fffd0000       .debug$S                   10000000     Qt5Widgets:Qt5Widgets.dll
 0000:fffd0000       .debug$S                   10000000     Qt5Widgets:Qt5Widgets.dll
 0000:fffd0000       .debug$S                   10000000     Qt5Widgets:Qt5Widgets.dll
 0000:fffd0000       .debug$S                   10000000     Qt5Widgets:Qt5Widgets.dll
 0000:fffd0000       .debug$S                   10000000     Qt5Widgets:Qt5Widgets.dll
 0000:fffd0000       .debug$S                   10000000     Qt5Widgets:Qt5Widgets.dll
 0000:fffd0000       .debug$S                   10000000     Qt5Widgets:Qt5Widgets.dll
 0000:fffd0000       .debug$S                   10000000     Qt5Widgets:Qt5Widgets.dll
 0000:fffd0000       .debug$S                   10000000     Qt5Widgets:Qt5Widgets.dll
 0000:fffd0000       .debug$S                   10000000     Qt5Widgets:Qt5Widgets.dll
 0000:fffd0000       .debug$S                   10000000     Qt5Widgets:Qt5Widgets.dll
 0000:fffd0000       .debug$S                   10000000     Qt5Widgets:Qt5Widgets.dll
 0000:fffd0000       .debug$S                   10000000     Qt5Widgets:Qt5Widgets.dll
 0000:fffd0000       .debug$S                   10000000     Qt5Widgets:Qt5Widgets.dll
 0000:fffd0000       .debug$S                   10000000     Qt5Widgets:Qt5Widgets.dll
 0000:fffd0000       .debug$S                   10000000     Qt5Widgets:Qt5Widgets.dll
 0000:fffd0000       .debug$S                   10000000     Qt5Widgets:Qt5Widgets.dll
 0000:fffd0000       .debug$S                   10000000     Qt5Widgets:Qt5Widgets.dll
 0000:fffd0000       .debug$S                   10000000     Qt5Widgets:Qt5Widgets.dll
 0000:fffd0000       .debug$S                   10000000     Qt5Widgets:Qt5Widgets.dll
 0000:fffd0000       .debug$S                   10000000     Qt5Widgets:Qt5Widgets.dll
 0000:fffd0000       .debug$S                   10000000     Qt5Widgets:Qt5Widgets.dll
 0000:fffd0000       .debug$S                   10000000     Qt5Widgets:Qt5Widgets.dll
 0000:fffd0000       .debug$S                   10000000     Qt5Widgets:Qt5Widgets.dll
 0000:fffd0000       .debug$S                   10000000     Qt5Widgets:Qt5Widgets.dll
 0000:fffd0000       .debug$S                   10000000     Qt5Widgets:Qt5Widgets.dll
 0000:fffd0000       .debug$S                   10000000     Qt5Widgets:Qt5Widgets.dll
 0000:fffd0000       .debug$S                   10000000     Qt5Widgets:Qt5Widgets.dll
 0000:fffd0000       .debug$S                   10000000     Qt5Widgets:Qt5Widgets.dll
 0000:fffd0000       .debug$S                   10000000     Qt5Widgets:Qt5Widgets.dll
 0000:fffd0000       .debug$S                   10000000     Qt5Widgets:Qt5Widgets.dll
 0000:fffd0000       .debug$S                   10000000     Qt5Widgets:Qt5Widgets.dll
 0002:fffe7000       ?_Generic_object$initializer$@?$_Error_objects@H@std@@2P6AXXZA 10000000     moc_DNAStatMSAProfileDialog.obj
 0002:fffe7000       ?_Iostream_object$initializer$@?$_Error_objects@H@std@@2P6AXXZA 10000000     moc_DNAStatMSAProfileDialog.obj
 0002:fffe7000       ?_System_object$initializer$@?$_Error_objects@H@std@@2P6AXXZA 10000000     moc_DNAStatMSAProfileDialog.obj
 0000:fffd0000       .debug$S                   10000000     Qt5Widgets:Qt5Widgets.dll
 0000:fffd0000       .debug$S                   10000000     Qt5Widgets:Qt5Widgets.dll
 0000:fffd0000       .debug$S                   10000000     Qt5Widgets:Qt5Widgets.dll
 0000:fffd0000       .debug$S                   10000000     Qt5Widgets:Qt5Widgets.dll
 0000:fffd0000       .debug$S                   10000000     Qt5Widgets:Qt5Widgets.dll
 0000:fffd0000       .debug$S                   10000000     Qt5Widgets:Qt5Widgets.dll
 0000:fffd0000       .debug$S                   10000000     Qt5Widgets:Qt5Widgets.dll
 0000:fffd0000       .debug$S                   10000000     Qt5Widgets:Qt5Widgets.dll
 0000:fffd0000       .debug$S                   10000000     Qt5Widgets:Qt5Widgets.dll
 0000:fffd0000       .debug$S                   10000000     Qt5Widgets:Qt5Widgets.dll
 0000:fffd0000       .debug$S                   10000000     Qt5Widgets:Qt5Widgets.dll
 0000:fffd0000       .debug$S                   10000000     Qt5Widgets:Qt5Widgets.dll
 0000:fffd0000       .debug$S                   10000000     Qt5Widgets:Qt5Widgets.dll
 0000:fffd0000       .debug$S                   10000000     Qt5Widgets:Qt5Widgets.dll
 0000:fffd0000       .debug$S                   10000000     Qt5Widgets:Qt5Widgets.dll
 0000:fffd0000       .debug$S                   10000000     Qt5Widgets:Qt5Widgets.dll
 0000:fffd0000       .debug$S                   10000000     Qt5Widgets:Qt5Widgets.dll
 0000:fffd0000       .debug$S                   10000000     Qt5Widgets:Qt5Widgets.dll
 0000:fffd0000       .debug$S                   10000000     Qt5Widgets:Qt5Widgets.dll
 0000:fffd0000       .debug$S                   10000000     Qt5Widgets:Qt5Widgets.dll
 0000:fffd0000       .debug$S                   10000000     Qt5Widgets:Qt5Widgets.dll
 0000:fffd0000       .debug$S                   10000000     Qt5Widgets:Qt5Widgets.dll
 0000:fffd0000       .debug$S                   10000000     Qt5Widgets:Qt5Widgets.dll
 0000:fffd0000       .debug$S                   10000000     Qt5Widgets:Qt5Widgets.dll
 0000:fffd0000       .debug$S                   10000000     Qt5Widgets:Qt5Widgets.dll
 0000:fffd0000       .debug$S                   10000000     Qt5Widgets:Qt5Widgets.dll
 0000:fffd0000       .debug$S                   10000000     Qt5Widgets:Qt5Widgets.dll
 0000:fffd0000       .debug$S                   10000000     Qt5Widgets:Qt5Widgets.dll
 0000:fffd0000       .debug$S                   10000000     Qt5Widgets:Qt5Widgets.dll
 0000:fffd0000       .debug$S                   10000000     Qt5Widgets:Qt5Widgets.dll
 0000:fffd0000       .debug$S                   10000000     Qt5Widgets:Qt5Widgets.dll
 0000:fffd0000       .debug$S                   10000000     Qt5Widgets:Qt5Widgets.dll
 0000:fffd0000       .debug$S                   10000000     Qt5Widgets:Qt5Widgets.dll
 0000:fffd0000       .debug$S                   10000000     Qt5Widgets:Qt5Widgets.dll
 0000:fffd0000       .debug$S                   10000000     Qt5Widgets:Qt5Widgets.dll
 0000:fffd0000       .debug$S                   10000000     Qt5Widgets:Qt5Widgets.dll
 0000:fffd0000       .debug$S                   10000000     Qt5Widgets:Qt5Widgets.dll
 0000:fffd0000       .debug$S                   10000000     Qt5Widgets:Qt5Widgets.dll
 0000:fffd0000       .debug$S                   10000000     Qt5Widgets:Qt5Widgets.dll
 0000:fffd0000       .debug$S                   10000000     Qt5Widgets:Qt5Widgets.dll
 0000:fffd0000       .debug$S                   10000000     Qt5Widgets:Qt5Widgets.dll
 0000:fffd0000       .debug$S                   10000000     Qt5Widgets:Qt5Widgets.dll
 0000:fffd0000       .debug$S                   10000000     Qt5Widgets:Qt5Widgets.dll
 0000:fffd0000       .debug$S                   10000000     Qt5Widgets:Qt5Widgets.dll
 0000:fffd0000       .debug$S                   10000000     Qt5Widgets:Qt5Widgets.dll
 0000:fffd0000       .debug$S                   10000000     Qt5Widgets:Qt5Widgets.dll
 0000:fffd0000       .debug$S                   10000000     Qt5Widgets:Qt5Widgets.dll
 0000:fffd0000       .debug$S                   10000000     Qt5Widgets:Qt5Widgets.dll
 0000:fffd0000       .debug$S                   10000000     Qt5Widgets:Qt5Widgets.dll
 0000:fffd0000       .debug$S                   10000000     Qt5Widgets:Qt5Widgets.dll
 0000:fffd0000       .debug$S                   10000000     Qt5Widgets:Qt5Widgets.dll
 0000:fffd0000       .debug$S                   10000000     Qt5Widgets:Qt5Widgets.dll
 0000:fffd0000       .debug$S                   10000000     Qt5Widgets:Qt5Widgets.dll
 0000:fffd0000       .debug$S                   10000000     Qt5Widgets:Qt5Widgets.dll
 0000:fffd0000       .debug$S                   10000000     Qt5Widgets:Qt5Widgets.dll
 0000:fffd0000       .debug$S                   10000000     Qt5Widgets:Qt5Widgets.dll
 0000:fffd0000       .debug$S                   10000000     Qt5Widgets:Qt5Widgets.dll
 0000:fffd0000       .debug$S                   10000000     Qt5Widgets:Qt5Widgets.dll
 0000:fffd0000       .debug$S                   10000000     Qt5Widgets:Qt5Widgets.dll
 0000:fffd0000       .debug$S                   10000000     Qt5Widgets:Qt5Widgets.dll
 0000:fffd0000       .debug$S                   10000000     Qt5Widgets:Qt5Widgets.dll
 0000:fffd0000       .debug$S                   10000000     Qt5Widgets:Qt5Widgets.dll
 0000:fffd0000       .debug$S                   10000000     Qt5Widgets:Qt5Widgets.dll
 0000:fffd0000       .debug$S                   10000000     Qt5Widgets:Qt5Widgets.dll
 0000:fffd0000       .debug$S                   10000000     Qt5Widgets:Qt5Widgets.dll
 0000:fffd0000       .debug$S                   10000000     Qt5Widgets:Qt5Widgets.dll
 0000:fffd0000       .debug$S                   10000000     Qt5Widgets:Qt5Widgets.dll
 0000:fffd0000       .debug$S                   10000000     Qt5Widgets:Qt5Widgets.dll
 0000:fffd0000       .debug$S                   10000000     Qt5Widgets:Qt5Widgets.dll
 0000:fffd0000       .debug$S                   10000000     Qt5Widgets:Qt5Widgets.dll
 0000:fffd0000       .debug$S                   10000000     Qt5Widgets:Qt5Widgets.dll
 0000:fffd0000       .debug$S                   10000000     Qt5Widgets:Qt5Widgets.dll
 0000:fffd0000       .debug$S                   10000000     Qt5Widgets:Qt5Widgets.dll
 0001:fffff000       __ehhandler$?_Copy@?$basic_string@DU?$char_traits@D@std@@V?$allocator@D@2@@std@@QAEXII@Z 10000000 f   DistanceMatrixMSAProfileDialog.obj
 0000:fffd0000       .debug$S                   10000000     Qt5Widgets:Qt5Widgets.dll
 0000:fffd0000       .debug$S                   10000000     Qt5Widgets:Qt5Widgets.dll
 0000:fffd0000       .debug$S                   10000000     Qt5Widgets:Qt5Widgets.dll
 0001:fffff000       __unwindfunclet$??H@YA?BVQString@@ABV0@0@Z$0 10000000 f   DistanceMatrixMSAProfileDialog.obj
 0000:fffd0000       .debug$S                   10000000     Qt5Widgets:Qt5Widgets.dll
 0001:fffff000       __unwindfunclet$??H@YA?BVQString@@ABV0@PBD@Z$0 10000000 f   DistanceMatrixMSAProfileDialog.obj
 0000:fffd0000       .debug$S                   10000000     U2View:U2View.dll
 0000:fffd0000       .debug$S                   10000000     U2View:U2View.dll
 0001:fffff000       __unwindfunclet$??H@YA?BVQString@@PBDABV0@@Z$0 10000000 f   DistanceMatrixMSAProfileDialog.obj
 0000:fffd0000       .debug$S                   10000000     U2View:U2View.dll
 0000:fffd0000       .debug$S                   10000000     U2View:U2View.dll
 0000:fffd0000       .debug$S                   10000000     U2View:U2View.dll
 0001:fffff000       __unwindfunclet$?append@?$QList@VQString@@@@QAEXABVQString@@@Z$7 10000000 f   DistanceMatrixMSAProfileDialog.obj
 0000:fffd0000       .debug$S                   10000000     U2View:U2View.dll
 0001:fffff000       __ehhandler$?detach_helper_grow@?$QList@VQString@@@@AAEPAUNode@1@HH@Z 10000000 f   DistanceMatrixMSAProfileDialog.obj
 0000:fffd0000       .debug$S                   10000000     U2View:U2View.dll
 0000:fffd0000       .debug$S                   10000000     U2View:U2View.dll
 0000:fffd0000       .debug$S                   10000000     U2View:U2View.dll
 0001:fffff000       __unwindfunclet$?node_construct@?$QList@VQString@@@@AAEXPAUNode@1@ABVQString@@@Z$1 10000000 f   DistanceMatrixMSAProfileDialog.obj
 0000:fffd0000       .debug$S                   10000000     U2View:U2View.dll
 0000:fffd0000       .debug$S                   10000000     U2View:U2View.dll
 0001:fffff000       __unwindfunclet$?node_copy@?$QList@VQString@@@@AAEXPAUNode@1@00@Z$5 10000000 f   DistanceMatrixMSAProfileDialog.obj
 0000:fffd0000       .debug$S                   10000000     U2View:U2View.dll
 0000:fffd0000       .debug$S                   10000000     U2View:U2View.dll
 0000:fffd0000       .debug$S                   10000000     U2View:U2View.dll
 0000:fffd0000       .debug$S                   10000000     U2View:U2View.dll
 0000:fffd0000       .debug$S                   10000000     U2View:U2View.dll
 0000:fffd0000       .debug$S                   10000000     U2View:U2View.dll
 0000:fffd0000       .debug$S                   10000000     U2View:U2View.dll
 0000:fffd0000       .debug$S                   10000000     U2View:U2View.dll
 0000:fffd0000       .debug$S                   10000000     U2View:U2View.dll
 0000:fffd0000       .debug$S                   10000000     U2View:U2View.dll
 0000:fffd0000       .debug$S                   10000000     U2View:U2View.dll
 0000:fffd0000       .debug$S                   10000000     U2View:U2View.dll
 0000:fffd0000       .debug$S                   10000000     U2View:U2View.dll
 0000:fffd0000       .debug$S                   10000000     U2Gui:U2Gui.dll
 0000:fffd0000       .debug$S                   10000000     U2Gui:U2Gui.dll
 0000:fffd0000       .debug$S                   10000000     U2Gui:U2Gui.dll
 0000:fffd0000       .debug$S                   10000000     U2Gui:U2Gui.dll
 0000:fffd0000       .debug$S                   10000000     U2Gui:U2Gui.dll
 0000:fffd0000       .debug$S                   10000000     U2Gui:U2Gui.dll
 0000:fffd0000       .debug$S                   10000000     U2Gui:U2Gui.dll
 0000:fffd0000       .debug$S                   10000000     U2Gui:U2Gui.dll
 0000:fffd0000       .debug$S                   10000000     U2Gui:U2Gui.dll
 0000:fffd0000       .debug$S                   10000000     U2Gui:U2Gui.dll
 0000:fffd0000       .debug$S                   10000000     U2Gui:U2Gui.dll
 0000:fffd0000       .debug$S                   10000000     U2Gui:U2Gui.dll
 0000:fffd0000       .debug$S                   10000000     U2Gui:U2Gui.dll
 0000:fffd0000       .debug$S                   10000000     U2Gui:U2Gui.dll
 0000:fffd0000       .debug$S                   10000000     U2Gui:U2Gui.dll
 0000:fffd0000       .debug$S                   10000000     U2Gui:U2Gui.dll
 0000:fffd0000       .debug$S                   10000000     U2Gui:U2Gui.dll
 0000:fffd0000       .debug$S                   10000000     U2Gui:U2Gui.dll
 0000:fffd0000       .debug$S                   10000000     U2Gui:U2Gui.dll
 0000:fffd0000       .debug$S                   10000000     U2Gui:U2Gui.dll
 0000:fffd0000       .debug$S                   10000000     U2Gui:U2Gui.dll
 0000:fffd0000       .debug$S                   10000000     U2Gui:U2Gui.dll
 0000:fffd0000       .debug$S                   10000000     U2Gui:U2Gui.dll
 0000:fffd0000       .debug$S                   10000000     U2Gui:U2Gui.dll
 0000:fffd0000       .debug$S                   10000000     U2Gui:U2Gui.dll
 0000:fffd0000       .debug$S                   10000000     U2Gui:U2Gui.dll
 0000:fffd0000       .debug$S                   10000000     U2Gui:U2Gui.dll
 0000:fffd0000       .debug$S                   10000000     U2Gui:U2Gui.dll
 0000:fffd0000       .debug$S                   10000000     U2Gui:U2Gui.dll
 0000:fffd0000       .debug$S                   10000000     U2Gui:U2Gui.dll
 0000:fffd0000       .debug$S                   10000000     U2Gui:U2Gui.dll
 0000:fffd0000       .debug$S                   10000000     U2Gui:U2Gui.dll
 0000:fffd0000       .debug$S                   10000000     U2Gui:U2Gui.dll
 0000:fffd0000       .debug$S                   10000000     U2Gui:U2Gui.dll
 0000:fffd0000       .debug$S                   10000000     U2Gui:U2Gui.dll
 0000:fffd0000       .debug$S                   10000000     U2Gui:U2Gui.dll
 0000:fffd0000       .debug$S                   10000000     U2Gui:U2Gui.dll
 0000:fffd0000       .debug$S                   10000000     U2Gui:U2Gui.dll
 0000:fffd0000       .debug$S                   10000000     U2Gui:U2Gui.dll
 0000:fffd0000       .debug$S                   10000000     U2Gui:U2Gui.dll
 0000:fffd0000       .debug$S                   10000000     U2Gui:U2Gui.dll
 0000:fffd0000       .debug$S                   10000000     U2Gui:U2Gui.dll
 0000:fffd0000       .debug$S                   10000000     U2Gui:U2Gui.dll
 0000:fffd0000       .debug$S                   10000000     U2Gui:U2Gui.dll
 0000:fffd0000       .debug$S                   10000000     U2Gui:U2Gui.dll
 0000:fffd0000       .debug$S                   10000000     U2Gui:U2Gui.dll
 0000:fffd0000       .debug$S                   10000000     U2Gui:U2Gui.dll
 0000:fffd0000       .debug$S                   10000000     U2Gui:U2Gui.dll
 0000:fffd0000       .debug$S                   10000000     U2Gui:U2Gui.dll
 0000:fffd0000       .debug$S                   10000000     U2Algorithm:U2Algorithm.dll
 0000:fffd0000       .debug$S                   10000000     U2Algorithm:U2Algorithm.dll
 0000:fffd0000       .debug$S                   10000000     U2Algorithm:U2Algorithm.dll
 0000:fffd0000       .debug$S                   10000000     U2Algorithm:U2Algorithm.dll
 0000:fffd0000       .debug$S                   10000000     U2Algorithm:U2Algorithm.dll
 0000:fffd0000       .debug$S                   10000000     U2Algorithm:U2Algorithm.dll
 0000:fffd0000       .debug$S                   10000000     U2Algorithm:U2Algorithm.dll
 0000:fffd0000       .debug$S                   10000000     U2Core:U2Core.dll
 0000:fffd0000       .debug$S                   10000000     U2Core:U2Core.dll
 0000:fffd0000       .debug$S                   10000000     U2Core:U2Core.dll
 0000:fffd0000       .debug$S                   10000000     U2Core:U2Core.dll
 0000:fffd0000       .debug$S                   10000000     U2Core:U2Core.dll
 0000:fffd0000       .debug$S                   10000000     U2Core:U2Core.dll
 0000:fffd0000       .debug$S                   10000000     U2Core:U2Core.dll
 0000:fffd0000       .debug$S                   10000000     U2Core:U2Core.dll
 0000:fffd0000       .debug$S                   10000000     U2Core:U2Core.dll
 0000:fffd0000       .debug$S                   10000000     U2Core:U2Core.dll
 0000:fffd0000       .debug$S                   10000000     U2Core:U2Core.dll
 0000:fffd0000       .debug$S                   10000000     U2Core:U2Core.dll
 0000:fffd0000       .debug$S                   10000000     U2Core:U2Core.dll
 0000:fffd0000       .debug$S                   10000000     U2Core:U2Core.dll
 0000:fffd0000       .debug$S                   10000000     U2Core:U2Core.dll
 0000:fffd0000       .debug$S                   10000000     U2Core:U2Core.dll
 0000:fffd0000       .debug$S                   10000000     U2Core:U2Core.dll
 0000:fffd0000       .debug$S                   10000000     U2Core:U2Core.dll
 0000:fffd0000       .debug$S                   10000000     U2Core:U2Core.dll
 0000:fffd0000       .debug$S                   10000000     U2Core:U2Core.dll
 0000:fffd0000       .debug$S                   10000000     U2Core:U2Core.dll
 0000:fffd0000       .debug$S                   10000000     U2Core:U2Core.dll
 0000:fffd0000       .debug$S                   10000000     U2Core:U2Core.dll
 0000:fffd0000       .debug$S                   10000000     U2Core:U2Core.dll
 0000:fffd0000       .debug$S                   10000000     U2Core:U2Core.dll
 0000:fffd0000       .debug$S                   10000000     U2Core:U2Core.dll
 0000:fffd0000       .debug$S                   10000000     U2Core:U2Core.dll
 0000:fffd0000       .debug$S                   10000000     U2Core:U2Core.dll
 0000:fffd0000       .debug$S                   10000000     U2Core:U2Core.dll
 0000:fffd0000       .debug$S                   10000000     U2Core:U2Core.dll
 0000:fffd0000       .debug$S                   10000000     U2Core:U2Core.dll
 0000:fffd0000       .debug$S                   10000000     U2Core:U2Core.dll
 0000:fffd0000       .debug$S                   10000000     U2Core:U2Core.dll
 0000:fffd0000       .debug$S                   10000000     U2Core:U2Core.dll
 0000:fffd0000       .debug$S                   10000000     U2Core:U2Core.dll
 0000:fffd0000       .debug$S                   10000000     U2Core:U2Core.dll
 0000:fffd0000       .debug$S                   10000000     U2Core:U2Core.dll
 0000:fffd0000       .debug$S                   10000000     U2Core:U2Core.dll
 0000:fffd0000       .debug$S                   10000000     U2Core:U2Core.dll
 0000:fffd0000       .debug$S                   10000000     U2Core:U2Core.dll
 0000:fffd0000       .debug$S                   10000000     U2Core:U2Core.dll
 0000:fffd0000       .debug$S                   10000000     U2Core:U2Core.dll
 0000:fffd0000       .debug$S                   10000000     U2Core:U2Core.dll
 0000:fffd0000       .debug$S                   10000000     U2Core:U2Core.dll
 0000:fffd0000       .debug$S                   10000000     U2Core:U2Core.dll
 0000:fffd0000       .debug$S                   10000000     U2Core:U2Core.dll
 0000:fffd0000       .debug$S                   10000000     U2Core:U2Core.dll
 0000:fffd0000       .debug$S                   10000000     U2Core:U2Core.dll
 0000:fffd0000       .debug$S                   10000000     U2Core:U2Core.dll
 0000:fffd0000       .debug$S                   10000000     U2Core:U2Core.dll
 0000:fffd0000       .debug$S                   10000000     U2Core:U2Core.dll
 0000:fffd0000       .debug$S                   10000000     U2Core:U2Core.dll
 0000:fffd0000       .debug$S                   10000000     U2Core:U2Core.dll
 0000:fffd0000       .debug$S                   10000000     U2Core:U2Core.dll
 0000:fffd0000       .debug$S                   10000000     U2Core:U2Core.dll
 0000:fffd0000       .debug$S                   10000000     U2Core:U2Core.dll
 0000:fffd0000       .debug$S                   10000000     U2Core:U2Core.dll
 0000:fffd0000       .debug$S                   10000000     U2Core:U2Core.dll
 0000:fffd0000       .debug$S                   10000000     U2Core:U2Core.dll
 0000:fffd0000       .debug$S                   10000000     U2Core:U2Core.dll
 0000:fffd0000       .debug$S                   10000000     U2Core:U2Core.dll
 0000:fffd0000       .debug$S                   10000000     U2Core:U2Core.dll
 0000:fffd0000       .debug$S                   10000000     U2Core:U2Core.dll
 0000:fffd0000       .debug$S                   10000000     U2Core:U2Core.dll
 0000:fffd0000       .debug$S                   10000000     U2Core:U2Core.dll
 0000:fffd0000       .debug$S                   10000000     U2Core:U2Core.dll
 0000:fffd0000       .debug$S                   10000000     U2Core:U2Core.dll
 0000:fffd0000       .debug$S                   10000000     U2Core:U2Core.dll
 0000:fffd0000       .debug$S                   10000000     U2Core:U2Core.dll
 0000:fffd0000       .debug$S                   10000000     U2Core:U2Core.dll
 0000:fffd0000       .debug$S                   10000000     U2Core:U2Core.dll
 0000:fffd0000       .debug$S                   10000000     U2Core:U2Core.dll
 0000:fffd0000       .debug$S                   10000000     U2Core:U2Core.dll
 0002:fffe7000       ?_System_object$initializer$@?$_Error_objects@H@std@@2P6AXXZA 10000000     DNAStatPlugin.obj
 0002:fffe7000       ?_Iostream_object$initializer$@?$_Error_objects@H@std@@2P6AXXZA 10000000     DNAStatPlugin.obj
 0002:fffe7000       ?_Generic_object$initializer$@?$_Error_objects@H@std@@2P6AXXZA 10000000     DNAStatPlugin.obj
 0002:fffe7000       __catchsym$?_Copy@?$basic_string@DU?$char_traits@D@std@@V?$allocator@D@2@@std@@QAEXII@Z$5 10000000     DNAStatPlugin.obj
 0000:fffd0000       .debug$S                   10000000     MSVCRT:MSVCR120.dll
 0002:fffe7000       ?_System_object$initializer$@?$_Error_objects@H@std@@2P6AXXZA 10000000     DNAStatProfileTask.obj
 0002:fffe7000       ?_Iostream_object$initializer$@?$_Error_objects@H@std@@2P6AXXZA 10000000     DNAStatProfileTask.obj
 0002:fffe7000       ?_Generic_object$initializer$@?$_Error_objects@H@std@@2P6AXXZA 10000000     DNAStatProfileTask.obj
 0002:fffe7000       __unwindtable$??H@YA?BVQString@@PBDABV0@@Z 10000000     DNAStatProfileTask.obj
 0002:fffe7000       __unwindtable$??H@YA?BVQString@@ABV0@PBD@Z 10000000     DNAStatProfileTask.obj
 0002:fffe7000       __unwindtable$??H@YA?BVQString@@ABV0@0@Z 10000000     DNAStatProfileTask.obj
 0002:fffe7000       __catchsym$?_Copy@?$basic_string@DU?$char_traits@D@std@@V?$allocator@D@2@@std@@QAEXII@Z$5 10000000     DNAStatProfileTask.obj
 0001:fffff000       __unwindfunclet$??H@YA?BVQString@@PBDABV0@@Z$0 10000000 f   DNAStatProfileTask.obj
 0001:fffff000       __unwindfunclet$??H@YA?BVQString@@ABV0@PBD@Z$0 10000000 f   DNAStatProfileTask.obj
 0001:fffff000       __unwindfunclet$??H@YA?BVQString@@ABV0@0@Z$0 10000000 f   DNAStatProfileTask.obj
 0001:fffff000       __ehhandler$?_Copy@?$basic_string@DU?$char_traits@D@std@@V?$allocator@D@2@@std@@QAEXII@Z 10000000 f   DNAStatProfileTask.obj
 0002:fffe7000       ?_System_object$initializer$@?$_Error_objects@H@std@@2P6AXXZA 10000000     DistanceMatrixMSAProfileDialog.obj
 0002:fffe7000       ?_Iostream_object$initializer$@?$_Error_objects@H@std@@2P6AXXZA 10000000     DistanceMatrixMSAProfileDialog.obj
 0002:fffe7000       ?_Generic_object$initializer$@?$_Error_objects@H@std@@2P6AXXZA 10000000     DistanceMatrixMSAProfileDialog.obj
 0002:fffe7000       __catchsym$?node_copy@?$QList@VQString@@@@AAEXPAUNode@1@00@Z$6 10000000     DistanceMatrixMSAProfileDialog.obj
 0002:fffe7000       __unwindtable$?node_construct@?$QList@VQString@@@@AAEXPAUNode@1@ABVQString@@@Z 10000000     DistanceMatrixMSAProfileDialog.obj
 0002:fffe7000       __catchsym$?detach_helper_grow@?$QList@VQString@@@@AAEPAUNode@1@HH@Z$5 10000000     DistanceMatrixMSAProfileDialog.obj
 0002:fffe7000       __catchsym$?append@?$QList@VQString@@@@QAEXABVQString@@@Z$13 10000000     DistanceMatrixMSAProfileDialog.obj
 0002:fffe7000       __unwindtable$??H@YA?BVQString@@PBDABV0@@Z 10000000     DistanceMatrixMSAProfileDialog.obj
 0002:fffe7000       __unwindtable$??H@YA?BVQString@@ABV0@PBD@Z 10000000     DistanceMatrixMSAProfileDialog.obj
 0002:fffe7000       __unwindtable$??H@YA?BVQString@@ABV0@0@Z 10000000     DistanceMatrixMSAProfileDialog.obj
 0002:fffe7000       __catchsym$?_Copy@?$basic_string@DU?$char_traits@D@std@@V?$allocator@D@2@@std@@QAEXII@Z$5 10000000     DistanceMatrixMSAProfileDialog.obj
 0002:fffe7008       __ehfuncinfo$??H@YA?BVQString@@ABV0@0@Z 10000008     DNAStatProfileTask.obj
 0002:fffe7008       __ehfuncinfo$??H@YA?BVQString@@PBDABV0@@Z 10000008     DNAStatProfileTask.obj
 0002:fffe7008       __ehfuncinfo$??H@YA?BVQString@@ABV0@0@Z 10000008     DistanceMatrixMSAProfileDialog.obj
 0002:fffe7008       __ehfuncinfo$??H@YA?BVQString@@PBDABV0@@Z 10000008     DistanceMatrixMSAProfileDialog.obj
 0002:fffe7010       __ehfuncinfo$?node_construct@?$QList@VQString@@@@AAEXPAUNode@1@ABVQString@@@Z 10000010     DistanceMatrixMSAProfileDialog.obj
 0002:fffe7010       __tryblocktable$?node_copy@?$QList@VQString@@@@AAEXPAUNode@1@00@Z 10000010     DistanceMatrixMSAProfileDialog.obj
 0002:fffe7010       __catchsym$?append@?$QList@VQString@@@@QAEXABVQString@@@Z$12 10000010     DistanceMatrixMSAProfileDialog.obj
 0002:fffe7010       __catchsym$?_Copy@?$basic_string@DU?$char_traits@D@std@@V?$allocator@D@2@@std@@QAEXII@Z$4 10000010     moc_DNAStatPlugin.obj
 0002:fffe7010       __catchsym$?_Copy@?$basic_string@DU?$char_traits@D@std@@V?$allocator@D@2@@std@@QAEXII@Z$4 10000010     DistanceMatrixMSAProfileDialog.obj
 0002:fffe7010       __catchsym$?_Copy@?$basic_string@DU?$char_traits@D@std@@V?$allocator@D@2@@std@@QAEXII@Z$4 10000010     DNAStatPlugin.obj
 0002:fffe7010       __catchsym$?_Copy@?$basic_string@DU?$char_traits@D@std@@V?$allocator@D@2@@std@@QAEXII@Z$4 10000010     moc_DNAStatMSAProfileDialog.obj
 0002:fffe7010       __catchsym$?_Copy@?$basic_string@DU?$char_traits@D@std@@V?$allocator@D@2@@std@@QAEXII@Z$4 10000010     moc_DistanceMatrixMSAProfileDialog.obj
 0002:fffe7010       __catchsym$?detach_helper_grow@?$QList@VQString@@@@AAEPAUNode@1@HH@Z$4 10000010     DistanceMatrixMSAProfileDialog.obj
 0002:fffe7010       __catchsym$?_Copy@?$basic_string@DU?$char_traits@D@std@@V?$allocator@D@2@@std@@QAEXII@Z$4 10000010     DNAStatProfileTask.obj
 0002:fffe7010       __catchsym$?_Copy@?$basic_string@DU?$char_traits@D@std@@V?$allocator@D@2@@std@@QAEXII@Z$4 10000010     moc_DNAStatProfileTask.obj
 0002:fffe7010       __ehfuncinfo$??H@YA?BVQString@@ABV0@PBD@Z 10000010     DNAStatProfileTask.obj
 0002:fffe7010       __ehfuncinfo$??H@YA?BVQString@@ABV0@PBD@Z 10000010     DistanceMatrixMSAProfileDialog.obj
 0001:fffff011       __unwindfunclet$?append@?$QList@VQString@@@@QAEXABVQString@@@Z$11 10000011 f   DistanceMatrixMSAProfileDialog.obj
 0001:fffff011       __ehhandler$?node_construct@?$QList@VQString@@@@AAEXPAUNode@1@ABVQString@@@Z 10000011 f   DistanceMatrixMSAProfileDialog.obj
 0001:fffff011       __ehhandler$?node_copy@?$QList@VQString@@@@AAEXPAUNode@1@00@Z 10000011 f   DistanceMatrixMSAProfileDialog.obj
 0001:fffff01a       __ehhandler$??H@YA?BVQString@@ABV0@0@Z 1000001a f   DNAStatProfileTask.obj
 0001:fffff01a       __unwindfunclet$??H@YA?BVQString@@ABV0@PBD@Z$1 1000001a f   DistanceMatrixMSAProfileDialog.obj
 0001:fffff01a       __ehhandler$??H@YA?BVQString@@PBDABV0@@Z 1000001a f   DNAStatProfileTask.obj
 0001:fffff01a       __ehhandler$??H@YA?BVQString@@PBDABV0@@Z 1000001a f   DistanceMatrixMSAProfileDialog.obj
 0001:fffff01a       __unwindfunclet$??H@YA?BVQString@@ABV0@PBD@Z$1 1000001a f   DNAStatProfileTask.obj
 0001:fffff01a       __ehhandler$??H@YA?BVQString@@ABV0@0@Z 1000001a f   DistanceMatrixMSAProfileDialog.obj
 0002:fffe7020       __unwindtable$?_Copy@?$basic_string@DU?$char_traits@D@std@@V?$allocator@D@2@@std@@QAEXII@Z 10000020     DNAStatPlugin.obj
 0002:fffe7020       __unwindtable$?_Copy@?$basic_string@DU?$char_traits@D@std@@V?$allocator@D@2@@std@@QAEXII@Z 10000020     DNAStatProfileTask.obj
 0002:fffe7020       __unwindtable$?_Copy@?$basic_string@DU?$char_traits@D@std@@V?$allocator@D@2@@std@@QAEXII@Z 10000020     moc_DNAStatPlugin.obj
 0002:fffe7020       __unwindtable$?detach_helper_grow@?$QList@VQString@@@@AAEPAUNode@1@HH@Z 10000020     DistanceMatrixMSAProfileDialog.obj
 0002:fffe7020       __unwindtable$?_Copy@?$basic_string@DU?$char_traits@D@std@@V?$allocator@D@2@@std@@QAEXII@Z 10000020     moc_DistanceMatrixMSAProfileDialog.obj
 0002:fffe7020       __unwindtable$?_Copy@?$basic_string@DU?$char_traits@D@std@@V?$allocator@D@2@@std@@QAEXII@Z 10000020     moc_DNAStatMSAProfileDialog.obj
 0002:fffe7020       __ehfuncinfo$?append@?$QList@VQString@@@@QAEXABVQString@@@Z 10000020     DistanceMatrixMSAProfileDialog.obj
 0002:fffe7020       __unwindtable$?_Copy@?$basic_string@DU?$char_traits@D@std@@V?$allocator@D@2@@std@@QAEXII@Z 10000020     moc_DNAStatProfileTask.obj
 0002:fffe7020       __unwindtable$?_Copy@?$basic_string@DU?$char_traits@D@std@@V?$allocator@D@2@@std@@QAEXII@Z 10000020     DistanceMatrixMSAProfileDialog.obj
 0001:fffff022       __ehhandler$?append@?$QList@VQString@@@@QAEXABVQString@@@Z 10000022 f   DistanceMatrixMSAProfileDialog.obj
 0001:fffff023       __ehhandler$??H@YA?BVQString@@ABV0@PBD@Z 10000023 f   DNAStatProfileTask.obj
 0001:fffff023       __ehhandler$??H@YA?BVQString@@ABV0@PBD@Z 10000023 f   DistanceMatrixMSAProfileDialog.obj
 0002:fffe7024       __ehfuncinfo$?node_copy@?$QList@VQString@@@@AAEXPAUNode@1@00@Z 10000024     DistanceMatrixMSAProfileDialog.obj
 0002:fffe7040       __ehfuncinfo$?_Copy@?$basic_string@DU?$char_traits@D@std@@V?$allocator@D@2@@std@@QAEXII@Z 10000040     DNAStatProfileTask.obj
 0002:fffe7040       __ehfuncinfo$?detach_helper_grow@?$QList@VQString@@@@AAEPAUNode@1@HH@Z 10000040     DistanceMatrixMSAProfileDialog.obj
 0002:fffe7040       __ehfuncinfo$?_Copy@?$basic_string@DU?$char_traits@D@std@@V?$allocator@D@2@@std@@QAEXII@Z 10000040     DistanceMatrixMSAProfileDialog.obj
 0002:fffe7040       __ehfuncinfo$?_Copy@?$basic_string@DU?$char_traits@D@std@@V?$allocator@D@2@@std@@QAEXII@Z 10000040     moc_DistanceMatrixMSAProfileDialog.obj
 0002:fffe7040       __ehfuncinfo$?_Copy@?$basic_string@DU?$char_traits@D@std@@V?$allocator@D@2@@std@@QAEXII@Z 10000040     moc_DNAStatMSAProfileDialog.obj
 0002:fffe7040       __ehfuncinfo$?_Copy@?$basic_string@DU?$char_traits@D@std@@V?$allocator@D@2@@std@@QAEXII@Z 10000040     moc_DNAStatProfileTask.obj
 0002:fffe7040       __ehfuncinfo$?_Copy@?$basic_string@DU?$char_traits@D@std@@V?$allocator@D@2@@std@@QAEXII@Z 10000040     moc_DNAStatPlugin.obj
 0002:fffe7040       __ehfuncinfo$?_Copy@?$basic_string@DU?$char_traits@D@std@@V?$allocator@D@2@@std@@QAEXII@Z 10000040     DNAStatPlugin.obj
 0002:fffe7044       __tryblocktable$?append@?$QList@VQString@@@@QAEXABVQString@@@Z 10000044     DistanceMatrixMSAProfileDialog.obj
 0002:fffe7048       __unwindtable$?node_copy@?$QList@VQString@@@@AAEXPAUNode@1@00@Z 10000048     DistanceMatrixMSAProfileDialog.obj
 0001:fffff062       __catch$?node_copy@?$QList@VQString@@@@AAEXPAUNode@1@00@Z$2 10000062 f   DistanceMatrixMSAProfileDialog.obj
 0002:fffe7064       __tryblocktable$?detach_helper_grow@?$QList@VQString@@@@AAEPAUNode@1@HH@Z 10000064     DistanceMatrixMSAProfileDialog.obj
 0002:fffe7064       __tryblocktable$?_Copy@?$basic_string@DU?$char_traits@D@std@@V?$allocator@D@2@@std@@QAEXII@Z 10000064     moc_DistanceMatrixMSAProfileDialog.obj
 0002:fffe7064       __tryblocktable$?_Copy@?$basic_string@DU?$char_traits@D@std@@V?$allocator@D@2@@std@@QAEXII@Z 10000064     DNAStatProfileTask.obj
 0002:fffe7064       __tryblocktable$?_Copy@?$basic_string@DU?$char_traits@D@std@@V?$allocator@D@2@@std@@QAEXII@Z 10000064     DNAStatPlugin.obj
 0002:fffe7064       __tryblocktable$?_Copy@?$basic_string@DU?$char_traits@D@std@@V?$allocator@D@2@@std@@QAEXII@Z 10000064     moc_DNAStatPlugin.obj
 0002:fffe7064       __tryblocktable$?_Copy@?$basic_string@DU?$char_traits@D@std@@V?$allocator@D@2@@std@@QAEXII@Z 10000064     DistanceMatrixMSAProfileDialog.obj
 0002:fffe7064       __tryblocktable$?_Copy@?$basic_string@DU?$char_traits@D@std@@V?$allocator@D@2@@std@@QAEXII@Z 10000064     moc_DNAStatMSAProfileDialog.obj
 0002:fffe7064       __tryblocktable$?_Copy@?$basic_string@DU?$char_traits@D@std@@V?$allocator@D@2@@std@@QAEXII@Z 10000064     moc_DNAStatProfileTask.obj
 0002:fffe706c       __unwindtable$?append@?$QList@VQString@@@@QAEXABVQString@@@Z 1000006c     DistanceMatrixMSAProfileDialog.obj
 0001:fffff07d       __catch$?append@?$QList@VQString@@@@QAEXABVQString@@@Z$0 1000007d f   DistanceMatrixMSAProfileDialog.obj
 0001:fffff096       __catch$?_Copy@?$basic_string@DU?$char_traits@D@std@@V?$allocator@D@2@@std@@QAEXII@Z$0 10000096 f   moc_DNAStatProfileTask.obj
 0001:fffff096       __catch$?_Copy@?$basic_string@DU?$char_traits@D@std@@V?$allocator@D@2@@std@@QAEXII@Z$0 10000096 f   DNAStatPlugin.obj
 0001:fffff096       __catch$?_Copy@?$basic_string@DU?$char_traits@D@std@@V?$allocator@D@2@@std@@QAEXII@Z$0 10000096 f   DNAStatProfileTask.obj
 0001:fffff096       __catch$?_Copy@?$basic_string@DU?$char_traits@D@std@@V?$allocator@D@2@@std@@QAEXII@Z$0 10000096 f   moc_DistanceMatrixMSAProfileDialog.obj
 0001:fffff096       __catch$?_Copy@?$basic_string@DU?$char_traits@D@std@@V?$allocator@D@2@@std@@QAEXII@Z$0 10000096 f   moc_DNAStatPlugin.obj
 0001:fffff096       __catch$?_Copy@?$basic_string@DU?$char_traits@D@std@@V?$allocator@D@2@@std@@QAEXII@Z$0 10000096 f   DistanceMatrixMSAProfileDialog.obj
 0001:fffff096       __catch$?_Copy@?$basic_string@DU?$char_traits@D@std@@V?$allocator@D@2@@std@@QAEXII@Z$0 10000096 f   moc_DNAStatMSAProfileDialog.obj
 0001:fffff0ce       __catch$?append@?$QList@VQString@@@@QAEXABVQString@@@Z$4 100000ce f   DistanceMatrixMSAProfileDialog.obj
 0001:fffff0d3       __catch$?_Copy@?$basic_string@DU?$char_traits@D@std@@V?$allocator@D@2@@std@@QAEXII@Z$1 100000d3 f   moc_DNAStatProfileTask.obj
 0001:fffff0d3       __catch$?_Copy@?$basic_string@DU?$char_traits@D@std@@V?$allocator@D@2@@std@@QAEXII@Z$1 100000d3 f   moc_DNAStatPlugin.obj
 0001:fffff0d3       __catch$?_Copy@?$basic_string@DU?$char_traits@D@std@@V?$allocator@D@2@@std@@QAEXII@Z$1 100000d3 f   moc_DNAStatMSAProfileDialog.obj
 0001:fffff0d3       __catch$?_Copy@?$basic_string@DU?$char_traits@D@std@@V?$allocator@D@2@@std@@QAEXII@Z$1 100000d3 f   DNAStatPlugin.obj
 0001:fffff0d3       __catch$?_Copy@?$basic_string@DU?$char_traits@D@std@@V?$allocator@D@2@@std@@QAEXII@Z$1 100000d3 f   DNAStatProfileTask.obj
 0001:fffff0d3       __catch$?_Copy@?$basic_string@DU?$char_traits@D@std@@V?$allocator@D@2@@std@@QAEXII@Z$1 100000d3 f   moc_DistanceMatrixMSAProfileDialog.obj
 0001:fffff0d3       __catch$?_Copy@?$basic_string@DU?$char_traits@D@std@@V?$allocator@D@2@@std@@QAEXII@Z$1 100000d3 f   DistanceMatrixMSAProfileDialog.obj
 0001:fffff11e       __catch$?detach_helper_grow@?$QList@VQString@@@@AAEPAUNode@1@HH@Z$2 1000011e f   DistanceMatrixMSAProfileDialog.obj
 0001:fffff159       __catch$?detach_helper_grow@?$QList@VQString@@@@AAEPAUNode@1@HH@Z$0 10000159 f   DistanceMatrixMSAProfileDialog.obj
 0001:00000000       ??__E?CSV@DNAStatMSAProfileDialog@U2@@0VQString@@B@@YAXXZ 10001000 f   DNAStatMSAProfileDialog.obj
 0001:00000020       ??__E?HTML@DNAStatMSAProfileDialog@U2@@0VQString@@B@@YAXXZ 10001020 f   DNAStatMSAProfileDialog.obj
 0001:00000040       ??__E?_Generic_object@?$_Error_objects@H@std@@2V_Generic_error_category@2@A@@YAXXZ 10001040 f   DNAStatMSAProfileDialog.obj
 0001:00000050       ??__E?_Iostream_object@?$_Error_objects@H@std@@2V_Iostream_error_category@2@A@@YAXXZ 10001050 f   DNAStatMSAProfileDialog.obj
 0001:00000060       ??__E?_System_object@?$_Error_objects@H@std@@2V_System_error_category@2@A@@YAXXZ 10001060 f   DNAStatMSAProfileDialog.obj
 0001:00000070       ??__EService_DNAExport@U2@@YAXXZ 10001070 f   DNAStatMSAProfileDialog.obj
 0001:00000080       ??__EService_DNAGraphPack@U2@@YAXXZ 10001080 f   DNAStatMSAProfileDialog.obj
 0001:00000090       ??__EService_ExternalToolSupport@U2@@YAXXZ 10001090 f   DNAStatMSAProfileDialog.obj
 0001:000000a0       ??__EService_GUITesting@U2@@YAXXZ 100010a0 f   DNAStatMSAProfileDialog.obj
 0001:000000b0       ??__EService_MaxCoreServiceId@U2@@YAXXZ 100010b0 f   DNAStatMSAProfileDialog.obj
 0001:000000c0       ??__EService_MinCoreServiceId@U2@@YAXXZ 100010c0 f   DNAStatMSAProfileDialog.obj
 0001:000000d0       ??__EService_PluginViewer@U2@@YAXXZ 100010d0 f   DNAStatMSAProfileDialog.obj
 0001:000000e0       ??__EService_Project@U2@@YAXXZ 100010e0 f   DNAStatMSAProfileDialog.obj
 0001:000000f0       ??__EService_ProjectView@U2@@YAXXZ 100010f0 f   DNAStatMSAProfileDialog.obj
 0001:00000100       ??__EService_QueryDesigner@U2@@YAXXZ 10001100 f   DNAStatMSAProfileDialog.obj
 0001:00000110       ??__EService_ScriptRegistry@U2@@YAXXZ 10001110 f   DNAStatMSAProfileDialog.obj
 0001:00000120       ??__EService_TestRunner@U2@@YAXXZ 10001120 f   DNAStatMSAProfileDialog.obj
 0001:00000130       ??__EService_WorkflowDesigner@U2@@YAXXZ 10001130 f   DNAStatMSAProfileDialog.obj
 0001:00000140       ??__EalgoLog@U2@@YAXXZ     10001140 f   DNAStatMSAProfileDialog.obj
 0001:000001c0       ??__EcmdLog@U2@@YAXXZ      100011c0 f   DNAStatMSAProfileDialog.obj
 0001:00000240       ??__EcoreLog@U2@@YAXXZ     10001240 f   DNAStatMSAProfileDialog.obj
 0001:000002c0       ??__EioLog@U2@@YAXXZ       100012c0 f   DNAStatMSAProfileDialog.obj
 0001:00000340       ??__EperfLog@U2@@YAXXZ     10001340 f   DNAStatMSAProfileDialog.obj
 0001:000003c0       ??__EscriptLog@U2@@YAXXZ   100013c0 f   DNAStatMSAProfileDialog.obj
 0001:00000440       ??__EtaskLog@U2@@YAXXZ     10001440 f   DNAStatMSAProfileDialog.obj
 0001:000004c0       ??__EuiLog@U2@@YAXXZ       100014c0 f   DNAStatMSAProfileDialog.obj
 0001:00000540       ??__EuserActLog@U2@@YAXXZ  10001540 f   DNAStatMSAProfileDialog.obj
 0001:000005c0       ??__E?_Generic_object@?$_Error_objects@H@std@@2V_Generic_error_category@2@A@@YAXXZ 100015c0 f   DNAStatPlugin.obj
 0001:000005d0       ??__E?_Iostream_object@?$_Error_objects@H@std@@2V_Iostream_error_category@2@A@@YAXXZ 100015d0 f   DNAStatPlugin.obj
 0001:000005e0       ??__E?_System_object@?$_Error_objects@H@std@@2V_System_error_category@2@A@@YAXXZ 100015e0 f   DNAStatPlugin.obj
 0001:000005f0       ??__EService_DNAExport@U2@@YAXXZ 100015f0 f   DNAStatPlugin.obj
 0001:00000600       ??__EService_DNAGraphPack@U2@@YAXXZ 10001600 f   DNAStatPlugin.obj
 0001:00000610       ??__EService_ExternalToolSupport@U2@@YAXXZ 10001610 f   DNAStatPlugin.obj
 0001:00000620       ??__EService_GUITesting@U2@@YAXXZ 10001620 f   DNAStatPlugin.obj
 0001:00000630       ??__EService_MaxCoreServiceId@U2@@YAXXZ 10001630 f   DNAStatPlugin.obj
 0001:00000640       ??__EService_MinCoreServiceId@U2@@YAXXZ 10001640 f   DNAStatPlugin.obj
 0001:00000650       ??__EService_PluginViewer@U2@@YAXXZ 10001650 f   DNAStatPlugin.obj
 0001:00000660       ??__EService_Project@U2@@YAXXZ 10001660 f   DNAStatPlugin.obj
 0001:00000670       ??__EService_ProjectView@U2@@YAXXZ 10001670 f   DNAStatPlugin.obj
 0001:00000680       ??__EService_QueryDesigner@U2@@YAXXZ 10001680 f   DNAStatPlugin.obj
 0001:00000690       ??__EService_ScriptRegistry@U2@@YAXXZ 10001690 f   DNAStatPlugin.obj
 0001:000006a0       ??__EService_TestRunner@U2@@YAXXZ 100016a0 f   DNAStatPlugin.obj
 0001:000006b0       ??__EService_WorkflowDesigner@U2@@YAXXZ 100016b0 f   DNAStatPlugin.obj
 0001:000006c0       ??__EalgoLog@U2@@YAXXZ     100016c0 f   DNAStatPlugin.obj
 0001:00000740       ??__EcmdLog@U2@@YAXXZ      10001740 f   DNAStatPlugin.obj
 0001:000007c0       ??__EcoreLog@U2@@YAXXZ     100017c0 f   DNAStatPlugin.obj
 0001:00000840       ??__EioLog@U2@@YAXXZ       10001840 f   DNAStatPlugin.obj
 0001:000008c0       ??__EperfLog@U2@@YAXXZ     100018c0 f   DNAStatPlugin.obj
 0001:00000940       ??__EscriptLog@U2@@YAXXZ   10001940 f   DNAStatPlugin.obj
 0001:000009c0       ??__EtaskLog@U2@@YAXXZ     100019c0 f   DNAStatPlugin.obj
 0001:00000a40       ??__EuiLog@U2@@YAXXZ       10001a40 f   DNAStatPlugin.obj
 0001:00000ac0       ??__EuserActLog@U2@@YAXXZ  10001ac0 f   DNAStatPlugin.obj
 0001:00000b40       ??__E?_Generic_object@?$_Error_objects@H@std@@2V_Generic_error_category@2@A@@YAXXZ 10001b40 f   DNAStatProfileTask.obj
 0001:00000b50       ??__E?_Iostream_object@?$_Error_objects@H@std@@2V_Iostream_error_category@2@A@@YAXXZ 10001b50 f   DNAStatProfileTask.obj
 0001:00000b60       ??__E?_System_object@?$_Error_objects@H@std@@2V_System_error_category@2@A@@YAXXZ 10001b60 f   DNAStatProfileTask.obj
 0001:00000b70       ??__EService_DNAExport@U2@@YAXXZ 10001b70 f   DNAStatProfileTask.obj
 0001:00000b80       ??__EService_DNAGraphPack@U2@@YAXXZ 10001b80 f   DNAStatProfileTask.obj
 0001:00000b90       ??__EService_ExternalToolSupport@U2@@YAXXZ 10001b90 f   DNAStatProfileTask.obj
 0001:00000ba0       ??__EService_GUITesting@U2@@YAXXZ 10001ba0 f   DNAStatProfileTask.obj
 0001:00000bb0       ??__EService_MaxCoreServiceId@U2@@YAXXZ 10001bb0 f   DNAStatProfileTask.obj
 0001:00000bc0       ??__EService_MinCoreServiceId@U2@@YAXXZ 10001bc0 f   DNAStatProfileTask.obj
 0001:00000bd0       ??__EService_PluginViewer@U2@@YAXXZ 10001bd0 f   DNAStatProfileTask.obj
 0001:00000be0       ??__EService_Project@U2@@YAXXZ 10001be0 f   DNAStatProfileTask.obj
 0001:00000bf0       ??__EService_ProjectView@U2@@YAXXZ 10001bf0 f   DNAStatProfileTask.obj
 0001:00000c00       ??__EService_QueryDesigner@U2@@YAXXZ 10001c00 f   DNAStatProfileTask.obj
 0001:00000c10       ??__EService_ScriptRegistry@U2@@YAXXZ 10001c10 f   DNAStatProfileTask.obj
 0001:00000c20       ??__EService_TestRunner@U2@@YAXXZ 10001c20 f   DNAStatProfileTask.obj
 0001:00000c30       ??__EService_WorkflowDesigner@U2@@YAXXZ 10001c30 f   DNAStatProfileTask.obj
 0001:00000c40       ??__EalgoLog@U2@@YAXXZ     10001c40 f   DNAStatProfileTask.obj
 0001:00000cc0       ??__EcmdLog@U2@@YAXXZ      10001cc0 f   DNAStatProfileTask.obj
 0001:00000d40       ??__EcoreLog@U2@@YAXXZ     10001d40 f   DNAStatProfileTask.obj
 0001:00000dc0       ??__EioLog@U2@@YAXXZ       10001dc0 f   DNAStatProfileTask.obj
 0001:00000e40       ??__EperfLog@U2@@YAXXZ     10001e40 f   DNAStatProfileTask.obj
 0001:00000ec0       ??__EscriptLog@U2@@YAXXZ   10001ec0 f   DNAStatProfileTask.obj
 0001:00000f40       ??__EtaskLog@U2@@YAXXZ     10001f40 f   DNAStatProfileTask.obj
 0001:00000fc0       ??__EuiLog@U2@@YAXXZ       10001fc0 f   DNAStatProfileTask.obj
 0001:00001040       ??__EuserActLog@U2@@YAXXZ  10002040 f   DNAStatProfileTask.obj
 0001:000010c0       ??__E?CSV@DistanceMatrixMSAProfileDialog@U2@@0VQString@@B@@YAXXZ 100020c0 f   DistanceMatrixMSAProfileDialog.obj
 0001:000010e0       ??__E?HTML@DistanceMatrixMSAProfileDialog@U2@@0VQString@@B@@YAXXZ 100020e0 f   DistanceMatrixMSAProfileDialog.obj
 0001:00001100       ??__E?_Generic_object@?$_Error_objects@H@std@@2V_Generic_error_category@2@A@@YAXXZ 10002100 f   DistanceMatrixMSAProfileDialog.obj
 0001:00001110       ??__E?_Iostream_object@?$_Error_objects@H@std@@2V_Iostream_error_category@2@A@@YAXXZ 10002110 f   DistanceMatrixMSAProfileDialog.obj
 0001:00001120       ??__E?_System_object@?$_Error_objects@H@std@@2V_System_error_category@2@A@@YAXXZ 10002120 f   DistanceMatrixMSAProfileDialog.obj
 0001:00001130       ??__EService_DNAExport@U2@@YAXXZ 10002130 f   DistanceMatrixMSAProfileDialog.obj
 0001:00001140       ??__EService_DNAGraphPack@U2@@YAXXZ 10002140 f   DistanceMatrixMSAProfileDialog.obj
 0001:00001150       ??__EService_ExternalToolSupport@U2@@YAXXZ 10002150 f   DistanceMatrixMSAProfileDialog.obj
 0001:00001160       ??__EService_GUITesting@U2@@YAXXZ 10002160 f   DistanceMatrixMSAProfileDialog.obj
 0001:00001170       ??__EService_MaxCoreServiceId@U2@@YAXXZ 10002170 f   DistanceMatrixMSAProfileDialog.obj
 0001:00001180       ??__EService_MinCoreServiceId@U2@@YAXXZ 10002180 f   DistanceMatrixMSAProfileDialog.obj
 0001:00001190       ??__EService_PluginViewer@U2@@YAXXZ 10002190 f   DistanceMatrixMSAProfileDialog.obj
 0001:000011a0       ??__EService_Project@U2@@YAXXZ 100021a0 f   DistanceMatrixMSAProfileDialog.obj
 0001:000011b0       ??__EService_ProjectView@U2@@YAXXZ 100021b0 f   DistanceMatrixMSAProfileDialog.obj
 0001:000011c0       ??__EService_QueryDesigner@U2@@YAXXZ 100021c0 f   DistanceMatrixMSAProfileDialog.obj
 0001:000011d0       ??__EService_ScriptRegistry@U2@@YAXXZ 100021d0 f   DistanceMatrixMSAProfileDialog.obj
 0001:000011e0       ??__EService_TestRunner@U2@@YAXXZ 100021e0 f   DistanceMatrixMSAProfileDialog.obj
 0001:000011f0       ??__EService_WorkflowDesigner@U2@@YAXXZ 100021f0 f   DistanceMatrixMSAProfileDialog.obj
 0001:00001200       ??__EalgoLog@U2@@YAXXZ     10002200 f   DistanceMatrixMSAProfileDialog.obj
 0001:00001280       ??__EcmdLog@U2@@YAXXZ      10002280 f   DistanceMatrixMSAProfileDialog.obj
 0001:00001300       ??__EcoreLog@U2@@YAXXZ     10002300 f   DistanceMatrixMSAProfileDialog.obj
 0001:00001380       ??__EioLog@U2@@YAXXZ       10002380 f   DistanceMatrixMSAProfileDialog.obj
 0001:00001400       ??__EperfLog@U2@@YAXXZ     10002400 f   DistanceMatrixMSAProfileDialog.obj
 0001:00001480       ??__EscriptLog@U2@@YAXXZ   10002480 f   DistanceMatrixMSAProfileDialog.obj
 0001:00001500       ??__EtaskLog@U2@@YAXXZ     10002500 f   DistanceMatrixMSAProfileDialog.obj
 0001:00001580       ??__EuiLog@U2@@YAXXZ       10002580 f   DistanceMatrixMSAProfileDialog.obj
 0001:00001600       ??__EuserActLog@U2@@YAXXZ  10002600 f   DistanceMatrixMSAProfileDialog.obj
 0001:00001680       ??__E?_Generic_object@?$_Error_objects@H@std@@2V_Generic_error_category@2@A@@YAXXZ 10002680 f   moc_DNAStatMSAProfileDialog.obj
 0001:00001690       ??__E?_Iostream_object@?$_Error_objects@H@std@@2V_Iostream_error_category@2@A@@YAXXZ 10002690 f   moc_DNAStatMSAProfileDialog.obj
 0001:000016a0       ??__E?_System_object@?$_Error_objects@H@std@@2V_System_error_category@2@A@@YAXXZ 100026a0 f   moc_DNAStatMSAProfileDialog.obj
 0001:000016b0       ??__E?staticMetaObject@DNAStatMSAProfileDialog@U2@@2UQMetaObject@@B@@YAXXZ 100026b0 f   moc_DNAStatMSAProfileDialog.obj
 0001:000016c0       ??__E?staticMetaObject@DNAStatMSAProfileTask@U2@@2UQMetaObject@@B@@YAXXZ 100026c0 f   moc_DNAStatMSAProfileDialog.obj
 0001:000016d0       ??__EalgoLog@U2@@YAXXZ     100026d0 f   moc_DNAStatMSAProfileDialog.obj
 0001:00001750       ??__EcmdLog@U2@@YAXXZ      10002750 f   moc_DNAStatMSAProfileDialog.obj
 0001:000017d0       ??__EcoreLog@U2@@YAXXZ     100027d0 f   moc_DNAStatMSAProfileDialog.obj
 0001:00001850       ??__EioLog@U2@@YAXXZ       10002850 f   moc_DNAStatMSAProfileDialog.obj
 0001:000018d0       ??__EperfLog@U2@@YAXXZ     100028d0 f   moc_DNAStatMSAProfileDialog.obj
 0001:00001950       ??__EscriptLog@U2@@YAXXZ   10002950 f   moc_DNAStatMSAProfileDialog.obj
 0001:000019d0       ??__EtaskLog@U2@@YAXXZ     100029d0 f   moc_DNAStatMSAProfileDialog.obj
 0001:00001a50       ??__EuiLog@U2@@YAXXZ       10002a50 f   moc_DNAStatMSAProfileDialog.obj
 0001:00001ad0       ??__EuserActLog@U2@@YAXXZ  10002ad0 f   moc_DNAStatMSAProfileDialog.obj
 0001:00001b50       ??__E?_Generic_object@?$_Error_objects@H@std@@2V_Generic_error_category@2@A@@YAXXZ 10002b50 f   moc_DNAStatPlugin.obj
 0001:00001b60       ??__E?_Iostream_object@?$_Error_objects@H@std@@2V_Iostream_error_category@2@A@@YAXXZ 10002b60 f   moc_DNAStatPlugin.obj
 0001:00001b70       ??__E?_System_object@?$_Error_objects@H@std@@2V_System_error_category@2@A@@YAXXZ 10002b70 f   moc_DNAStatPlugin.obj
 0001:00001b80       ??__E?staticMetaObject@DNAStatMSAEditorContext@U2@@2UQMetaObject@@B@@YAXXZ 10002b80 f   moc_DNAStatPlugin.obj
 0001:00001b90       ??__E?staticMetaObject@DNAStatPlugin@U2@@2UQMetaObject@@B@@YAXXZ 10002b90 f   moc_DNAStatPlugin.obj
 0001:00001ba0       ??__E?staticMetaObject@DistanceMatrixMSAEditorContext@U2@@2UQMetaObject@@B@@YAXXZ 10002ba0 f   moc_DNAStatPlugin.obj
 0001:00001bb0       ??__EService_DNAExport@U2@@YAXXZ 10002bb0 f   moc_DNAStatPlugin.obj
 0001:00001bc0       ??__EService_DNAGraphPack@U2@@YAXXZ 10002bc0 f   moc_DNAStatPlugin.obj
 0001:00001bd0       ??__EService_ExternalToolSupport@U2@@YAXXZ 10002bd0 f   moc_DNAStatPlugin.obj
 0001:00001be0       ??__EService_GUITesting@U2@@YAXXZ 10002be0 f   moc_DNAStatPlugin.obj
 0001:00001bf0       ??__EService_MaxCoreServiceId@U2@@YAXXZ 10002bf0 f   moc_DNAStatPlugin.obj
 0001:00001c00       ??__EService_MinCoreServiceId@U2@@YAXXZ 10002c00 f   moc_DNAStatPlugin.obj
 0001:00001c10       ??__EService_PluginViewer@U2@@YAXXZ 10002c10 f   moc_DNAStatPlugin.obj
 0001:00001c20       ??__EService_Project@U2@@YAXXZ 10002c20 f   moc_DNAStatPlugin.obj
 0001:00001c30       ??__EService_ProjectView@U2@@YAXXZ 10002c30 f   moc_DNAStatPlugin.obj
 0001:00001c40       ??__EService_QueryDesigner@U2@@YAXXZ 10002c40 f   moc_DNAStatPlugin.obj
 0001:00001c50       ??__EService_ScriptRegistry@U2@@YAXXZ 10002c50 f   moc_DNAStatPlugin.obj
 0001:00001c60       ??__EService_TestRunner@U2@@YAXXZ 10002c60 f   moc_DNAStatPlugin.obj
 0001:00001c70       ??__EService_WorkflowDesigner@U2@@YAXXZ 10002c70 f   moc_DNAStatPlugin.obj
 0001:00001c80       ??__E?_Generic_object@?$_Error_objects@H@std@@2V_Generic_error_category@2@A@@YAXXZ 10002c80 f   moc_DNAStatProfileTask.obj
 0001:00001c90       ??__E?_Iostream_object@?$_Error_objects@H@std@@2V_Iostream_error_category@2@A@@YAXXZ 10002c90 f   moc_DNAStatProfileTask.obj
 0001:00001ca0       ??__E?_System_object@?$_Error_objects@H@std@@2V_System_error_category@2@A@@YAXXZ 10002ca0 f   moc_DNAStatProfileTask.obj
 0001:00001cb0       ??__E?staticMetaObject@DNAStatProfileTask@U2@@2UQMetaObject@@B@@YAXXZ 10002cb0 f   moc_DNAStatProfileTask.obj
 0001:00001cc0       ??__EalgoLog@U2@@YAXXZ     10002cc0 f   moc_DNAStatProfileTask.obj
 0001:00001d40       ??__EcmdLog@U2@@YAXXZ      10002d40 f   moc_DNAStatProfileTask.obj
 0001:00001dc0       ??__EcoreLog@U2@@YAXXZ     10002dc0 f   moc_DNAStatProfileTask.obj
 0001:00001e40       ??__EioLog@U2@@YAXXZ       10002e40 f   moc_DNAStatProfileTask.obj
 0001:00001ec0       ??__EperfLog@U2@@YAXXZ     10002ec0 f   moc_DNAStatProfileTask.obj
 0001:00001f40       ??__EscriptLog@U2@@YAXXZ   10002f40 f   moc_DNAStatProfileTask.obj
 0001:00001fc0       ??__EtaskLog@U2@@YAXXZ     10002fc0 f   moc_DNAStatProfileTask.obj
 0001:00002040       ??__EuiLog@U2@@YAXXZ       10003040 f   moc_DNAStatProfileTask.obj
 0001:000020c0       ??__EuserActLog@U2@@YAXXZ  100030c0 f   moc_DNAStatProfileTask.obj
 0001:00002140       ??__E?_Generic_object@?$_Error_objects@H@std@@2V_Generic_error_category@2@A@@YAXXZ 10003140 f   moc_DistanceMatrixMSAProfileDialog.obj
 0001:00002150       ??__E?_Iostream_object@?$_Error_objects@H@std@@2V_Iostream_error_category@2@A@@YAXXZ 10003150 f   moc_DistanceMatrixMSAProfileDialog.obj
 0001:00002160       ??__E?_System_object@?$_Error_objects@H@std@@2V_System_error_category@2@A@@YAXXZ 10003160 f   moc_DistanceMatrixMSAProfileDialog.obj
 0001:00002170       ??__E?staticMetaObject@DistanceMatrixMSAProfileDialog@U2@@2UQMetaObject@@B@@YAXXZ 10003170 f   moc_DistanceMatrixMSAProfileDialog.obj
 0001:00002180       ??__E?staticMetaObject@DistanceMatrixMSAProfileTask@U2@@2UQMetaObject@@B@@YAXXZ 10003180 f   moc_DistanceMatrixMSAProfileDialog.obj
 0001:00002190       ??__EalgoLog@U2@@YAXXZ     10003190 f   moc_DistanceMatrixMSAProfileDialog.obj
 0001:00002210       ??__EcmdLog@U2@@YAXXZ      10003210 f   moc_DistanceMatrixMSAProfileDialog.obj
 0001:00002290       ??__EcoreLog@U2@@YAXXZ     10003290 f   moc_DistanceMatrixMSAProfileDialog.obj
 0001:00002310       ??__EioLog@U2@@YAXXZ       10003310 f   moc_DistanceMatrixMSAProfileDialog.obj
 0001:00002390       ??__EperfLog@U2@@YAXXZ     10003390 f   moc_DistanceMatrixMSAProfileDialog.obj
 0001:00002410       ??__EscriptLog@U2@@YAXXZ   10003410 f   moc_DistanceMatrixMSAProfileDialog.obj
 0001:00002490       ??__EtaskLog@U2@@YAXXZ     10003490 f   moc_DistanceMatrixMSAProfileDialog.obj
 0001:00002510       ??__EuiLog@U2@@YAXXZ       10003510 f   moc_DistanceMatrixMSAProfileDialog.obj
 0001:00002590       ??__EuserActLog@U2@@YAXXZ  10003590 f   moc_DistanceMatrixMSAProfileDialog.obj
 0001:00003c50       ??R<lambda_0b89744300e523de31da4f8ed196539f>@@QBE?AVQString@@XZ 10004c50 f   DNAStatMSAProfileDialog.obj
 0001:00003c70       ??R<lambda_332f86a55e7649bbbc7d152cfc1d46e6>@@QBE?AVQString@@XZ 10004c70 f   DNAStatMSAProfileDialog.obj
 0001:00003c90       ??R<lambda_369cdf7999dc0faee62b5b90af0d786b>@@QBE?AVQString@@XZ 10004c90 f   DNAStatMSAProfileDialog.obj
 0001:00003cb0       ??R<lambda_376d37d6abfed47a5cb9bd756b76dca8>@@QBE?AVQString@@XZ 10004cb0 f   DNAStatMSAProfileDialog.obj
 0001:00003cd0       ??R<lambda_3921f84164ed29f15fc743b6ab68e204>@@QBE?AVQString@@XZ 10004cd0 f   DNAStatMSAProfileDialog.obj
 0001:00003cf0       ??R<lambda_3f118f97850a866f6d5ae3fbb0dc2aed>@@QBE?AVQString@@XZ 10004cf0 f   DNAStatMSAProfileDialog.obj
 0001:00003d10       ??R<lambda_459d3513592b8ff4f9b393a392f7e1dc>@@QBE?AVQString@@XZ 10004d10 f   DNAStatMSAProfileDialog.obj
 0001:00003d30       ??R<lambda_4a12a9b4f8aa2ea3a7fffd7d958ae388>@@QBE?AVQString@@XZ 10004d30 f   DNAStatMSAProfileDialog.obj
 0001:00003d50       ??R<lambda_545371d98571d04f1b39b4582be52899>@@QBE?AVQString@@XZ 10004d50 f   DNAStatMSAProfileDialog.obj
 0001:00003d70       ??R<lambda_580e10368bf5988093bdeab019318dc2>@@QBE?AVQString@@XZ 10004d70 f   DNAStatMSAProfileDialog.obj
 0001:00003d90       ??R<lambda_59946a197341b3528bd575f770f586ea>@@QBE?AVQString@@XZ 10004d90 f   DNAStatMSAProfileDialog.obj
 0001:00003db0       ??R<lambda_664313d2fa9b135bdb11bebee3978435>@@QBE?AVQString@@XZ 10004db0 f   DNAStatMSAProfileDialog.obj
 0001:00003dd0       ??R<lambda_9ef6d0056c3e3c198c7a1006e54d249c>@@QBE?AVQString@@XZ 10004dd0 f   DNAStatMSAProfileDialog.obj
 0001:00003df0       ??R<lambda_9f6a8b438001a51b240e5bf18f0afdd2>@@QBE?AVQString@@XZ 10004df0 f   DNAStatMSAProfileDialog.obj
 0001:00003e10       ??R<lambda_a3a39629b9536d4dab532972692be556>@@QBE?AVQString@@XZ 10004e10 f   DNAStatMSAProfileDialog.obj
 0001:00003e30       ??R<lambda_a89643c798c7c6488c2208d0e325f35b>@@QBE?AVQString@@XZ 10004e30 f   DNAStatMSAProfileDialog.obj
 0001:00003e50       ??R<lambda_bd9b46c5af1ae431bf97a2b6b358b9a7>@@QBE?AVQString@@XZ 10004e50 f   DNAStatMSAProfileDialog.obj
 0001:00003e70       ??R<lambda_bda637ed11183b6068483cf30a484448>@@QBE?AVQString@@XZ 10004e70 f   DNAStatMSAProfileDialog.obj
 0001:00003e90       ??R<lambda_fab6138414a91a0c3bced0a99c7ba19f>@@QBE?AVQString@@XZ 10004e90 f   DNAStatMSAProfileDialog.obj
 0001:000044d6       __catch$?_Copy@?$basic_string@DU?$char_traits@D@std@@V?$allocator@D@2@@std@@QAEXII@Z$0 100054d6 f i DNAStatMSAProfileDialog.obj
 0001:00004513       __catch$?_Copy@?$basic_string@DU?$char_traits@D@std@@V?$allocator@D@2@@std@@QAEXII@Z$1 10005513 f i DNAStatMSAProfileDialog.obj
 0001:00004abd       __catch$?append@?$QList@VQString@@@@QAEXABVQString@@@Z$0 10005abd f i DNAStatMSAProfileDialog.obj
 0001:00004b0e       __catch$?append@?$QList@VQString@@@@QAEXABVQString@@@Z$4 10005b0e f i DNAStatMSAProfileDialog.obj
 0001:0000610e       __catch$?detach_helper_grow@?$QList@VQString@@@@AAEPAUNode@1@HH@Z$2 1000710e f i DNAStatMSAProfileDialog.obj
 0001:00006149       __catch$?detach_helper_grow@?$QList@VQString@@@@AAEPAUNode@1@HH@Z$0 10007149 f i DNAStatMSAProfileDialog.obj
 0001:00006f52       __catch$?node_copy@?$QList@VQString@@@@AAEXPAUNode@1@00@Z$2 10007f52 f i DNAStatMSAProfileDialog.obj
 0001:00007203       __catch$?reallocData@?$QVector@D@@AAEXHHV?$QFlags@W4AllocationOption@QArrayData@@@@@Z$0 10008203 f i DNAStatMSAProfileDialog.obj
 0001:00007215       __catch$?reallocData@?$QVector@D@@AAEXHHV?$QFlags@W4AllocationOption@QArrayData@@@@@Z$2 10008215 f i DNAStatMSAProfileDialog.obj
 0001:00007444       __catch$?reallocData@?$QVector@H@@AAEXHHV?$QFlags@W4AllocationOption@QArrayData@@@@@Z$0 10008444 f i DNAStatMSAProfileDialog.obj
 0001:00007456       __catch$?reallocData@?$QVector@H@@AAEXHHV?$QFlags@W4AllocationOption@QArrayData@@@@@Z$2 10008456 f i DNAStatMSAProfileDialog.obj
 0001:000076a6       __catch$?reallocData@?$QVector@UColumnStat@DNAStatMSAProfileTask@U2@@@@AAEXHHV?$QFlags@W4AllocationOption@QArrayData@@@@@Z$0 100086a6 f i DNAStatMSAProfileDialog.obj
 0001:000076c4       __catch$?reallocData@?$QVector@UColumnStat@DNAStatMSAProfileTask@U2@@@@AAEXHHV?$QFlags@W4AllocationOption@QArrayData@@@@@Z$2 100086c4 f i DNAStatMSAProfileDialog.obj
 0001:00008ff9       __catch$?run@DNAStatMSAProfileTask@U2@@UAEXXZ$0 10009ff9 f   DNAStatMSAProfileDialog.obj
 0001:00009e9e       __catch$??0?$QList@PAVGObjectViewAction@U2@@@@QAE@ABV0@@Z$0 1000ae9e f i DNAStatPlugin.obj
 0001:0000b1be       __catch$??0?$QList@UCharOccurResult@U2@@@@QAE@ABV0@@Z$0 1000c1be f i DNAStatProfileTask.obj
 0001:0000b9eb       __catch$?createNode@?$QMapData@VQByteArray@@_J@@QAEPAU?$QMapNode@VQByteArray@@_J@@ABVQByteArray@@AB_JPAU2@_N@Z$2 1000c9eb f i DNAStatProfileTask.obj
 0001:0000cffa       __catch$?node_copy@?$QList@UCharOccurResult@U2@@@@AAEXPAUNode@1@00@Z$0 1000dffa f i DNAStatProfileTask.obj
 0001:0000d36e       __catch$??0?$QList@PAVMSADistanceAlgorithmFactory@U2@@@@QAE@ABV0@@Z$0 1000e36e f i DistanceMatrixMSAProfileDialog.obj
 0001:0000dca0       ??R<lambda_22328789e56fd3e3b770fcf81371bdbf>@@QBE?AVQString@@XZ 1000eca0 f   DistanceMatrixMSAProfileDialog.obj
 0001:0000dcc0       ??R<lambda_257a9ba125789c78778143779c7aa17e>@@QBE?AVQString@@XZ 1000ecc0 f   DistanceMatrixMSAProfileDialog.obj
 0001:0000dce0       ??R<lambda_346f61b4a197c7796b06dee8cb9eb1b6>@@QBE?AVQString@@XZ 1000ece0 f   DistanceMatrixMSAProfileDialog.obj
 0001:0000dd00       ??R<lambda_3af62e2b98c1502753882d3498ff5cca>@@QBE?AVQString@@XZ 1000ed00 f   DistanceMatrixMSAProfileDialog.obj
 0001:0000dd20       ??R<lambda_3b9e00bd2f9235c0e5410d79eb0eadce>@@QBE?AVQString@@XZ 1000ed20 f   DistanceMatrixMSAProfileDialog.obj
 0001:0000dd40       ??R<lambda_4149c1a5601b404cb9e3099d72fa0a0a>@@QBE?AVQString@@XZ 1000ed40 f   DistanceMatrixMSAProfileDialog.obj
 0001:0000dd60       ??R<lambda_477f2371469cb72a5ef263890104105f>@@QBE?AVQString@@XZ 1000ed60 f   DistanceMatrixMSAProfileDialog.obj
 0001:0000dd80       ??R<lambda_4c9d5f56d49016978bbb8760a7e3d910>@@QBE?AVQString@@XZ 1000ed80 f   DistanceMatrixMSAProfileDialog.obj
 0001:0000dda0       ??R<lambda_667cf19c3b93807e72a75e35313c6da5>@@QBE?AVQString@@XZ 1000eda0 f   DistanceMatrixMSAProfileDialog.obj
 0001:0000ddc0       ??R<lambda_7d1f8454ec166fb6929aab69d9b35ec8>@@QBE?AVQString@@XZ 1000edc0 f   DistanceMatrixMSAProfileDialog.obj
 0001:0000dde0       ??R<lambda_840dc314801588f3307f74f67d327cab>@@QBE?AVQString@@XZ 1000ede0 f   DistanceMatrixMSAProfileDialog.obj
 0001:0000de00       ??R<lambda_aaa0d8f07c2dd2193aa6aadb22c08d2b>@@QBE?AVQString@@XZ 1000ee00 f   DistanceMatrixMSAProfileDialog.obj
 0001:0000de20       ??R<lambda_b420bad46777224f9d1a7dddab21eac2>@@QBE?AVQString@@XZ 1000ee20 f   DistanceMatrixMSAProfileDialog.obj
 0001:0000de40       ??R<lambda_cd3023c81d757c47026fd3c6565acb82>@@QBE?AVQString@@XZ 1000ee40 f   DistanceMatrixMSAProfileDialog.obj
 0001:0000de60       ??R<lambda_d91a2c0f8c8907c0767dda3038aeabd8>@@QBE?AVQString@@XZ 1000ee60 f   DistanceMatrixMSAProfileDialog.obj
 0001:0000de80       ??R<lambda_d92ac2e6e619141498e0b5df5f617cb4>@@QBE?AVQString@@XZ 1000ee80 f   DistanceMatrixMSAProfileDialog.obj
 0001:0000dea0       ??R<lambda_df5a57b07f782d6c431b0eadd5e7983a>@@QBE?AVQString@@XZ 1000eea0 f   DistanceMatrixMSAProfileDialog.obj
 0001:0000dec0       ??R<lambda_f076482335b87e84dc878d3bc1c37823>@@QBE?AVQString@@XZ 1000eec0 f   DistanceMatrixMSAProfileDialog.obj
 0001:0000dee0       ??R<lambda_f3813fcbb1e170019aa0d3012117af7b>@@QBE?AVQString@@XZ 1000eee0 f   DistanceMatrixMSAProfileDialog.obj
 0001:0000e36c       __catch$?append@?$QList@VMultipleSequenceAlignmentRow@U2@@@@QAEXABVMultipleSequenceAlignmentRow@U2@@@Z$0 1000f36c f i DistanceMatrixMSAProfileDialog.obj
 0001:0000e36c       __catch$?append@?$QList@VMultipleSequenceAlignmentRow@U2@@@@QAEXABVMultipleSequenceAlignmentRow@U2@@@Z$2 1000f36c f i DistanceMatrixMSAProfileDialog.obj
 0001:0000ec1f       __catch$?detach_helper_grow@?$QList@VMultipleSequenceAlignmentRow@U2@@@@AAEPAUNode@1@HH@Z$2 1000fc1f f i DistanceMatrixMSAProfileDialog.obj
 0001:0000ec5a       __catch$?detach_helper_grow@?$QList@VMultipleSequenceAlignmentRow@U2@@@@AAEPAUNode@1@HH@Z$0 1000fc5a f i DistanceMatrixMSAProfileDialog.obj
 0001:0000f3f5       __catch$?node_copy@?$QList@VMultipleSequenceAlignmentRow@U2@@@@AAEXPAUNode@1@00@Z$0 100103f5 f i DistanceMatrixMSAProfileDialog.obj
 0001:00010773       __catch$?onSubTaskFinished@DistanceMatrixMSAProfileTask@U2@@UAE?AV?$QList@PAVTask@U2@@@@PAVTask@2@@Z$2 10011773 f   DistanceMatrixMSAProfileDialog.obj
 0001:000107e1       __catch$?onSubTaskFinished@DistanceMatrixMSAProfileTask@U2@@UAE?AV?$QList@PAVTask@U2@@@@PAVTask@2@@Z$0 100117e1 f   DistanceMatrixMSAProfileDialog.obj
 0001:000134bf       ?ArrayUnwindFilter@@YAHPAU_EXCEPTION_POINTERS@@@Z 100144bf f   MSVCRT:ehvecdtr.obj
 0001:000136d0       $$000000                   100146d0     MSVCRT:ftol3.obj
 0001:00013ab0       $$000000                   10014ab0     MSVCRT:llrem.obj
 0001:00013b62       _pre_c_init                10014b62 f   MSVCRT:crtdll.obj
 0001:00013dcf       ___DllMainCRTStartup       10014dcf f   MSVCRT:crtdll.obj
 0001:00013f10       $$000000                   10014f10     MSVCRT:sehprolg4.obj
 0001:000145b0       __unwindfunclet$??0DNAStatMSAProfileDialog@U2@@QAE@PAVQWidget@@PAVMSAEditor@1@@Z$0 100155b0 f   DNAStatMSAProfileDialog.obj
 0001:000145b9       __unwindfunclet$??0DNAStatMSAProfileDialog@U2@@QAE@PAVQWidget@@PAVMSAEditor@1@@Z$1 100155b9 f   DNAStatMSAProfileDialog.obj
 0001:000145c4       __unwindfunclet$??0DNAStatMSAProfileDialog@U2@@QAE@PAVQWidget@@PAVMSAEditor@1@@Z$2 100155c4 f   DNAStatMSAProfileDialog.obj
 0001:000145de       __unwindfunclet$??0DNAStatMSAProfileDialog@U2@@QAE@PAVQWidget@@PAVMSAEditor@1@@Z$3 100155de f   DNAStatMSAProfileDialog.obj
 0001:000145e7       __unwindfunclet$??0DNAStatMSAProfileDialog@U2@@QAE@PAVQWidget@@PAVMSAEditor@1@@Z$4 100155e7 f   DNAStatMSAProfileDialog.obj
 0001:000145f0       __ehhandler$??0DNAStatMSAProfileDialog@U2@@QAE@PAVQWidget@@PAVMSAEditor@1@@Z 100155f0 f   DNAStatMSAProfileDialog.obj
 0001:00014610       __unwindfunclet$??0DNAStatMSAProfileTask@U2@@QAE@ABVDNAStatMSAProfileTaskSettings@1@@Z$0 10015610 f   DNAStatMSAProfileDialog.obj
 0001:00014619       __unwindfunclet$??0DNAStatMSAProfileTask@U2@@QAE@ABVDNAStatMSAProfileTaskSettings@1@@Z$1 10015619 f   DNAStatMSAProfileDialog.obj
 0001:00014622       __unwindfunclet$??0DNAStatMSAProfileTask@U2@@QAE@ABVDNAStatMSAProfileTaskSettings@1@@Z$2 10015622 f   DNAStatMSAProfileDialog.obj
 0001:00014630       __unwindfunclet$??0DNAStatMSAProfileTask@U2@@QAE@ABVDNAStatMSAProfileTaskSettings@1@@Z$3 10015630 f   DNAStatMSAProfileDialog.obj
 0001:0001463e       __unwindfunclet$??0DNAStatMSAProfileTask@U2@@QAE@ABVDNAStatMSAProfileTaskSettings@1@@Z$4 1001563e f   DNAStatMSAProfileDialog.obj
 0001:0001464c       __unwindfunclet$??0DNAStatMSAProfileTask@U2@@QAE@ABVDNAStatMSAProfileTaskSettings@1@@Z$5 1001564c f   DNAStatMSAProfileDialog.obj
 0001:0001465a       __unwindfunclet$??0DNAStatMSAProfileTask@U2@@QAE@ABVDNAStatMSAProfileTaskSettings@1@@Z$6 1001565a f   DNAStatMSAProfileDialog.obj
 0001:00014668       __unwindfunclet$??0DNAStatMSAProfileTask@U2@@QAE@ABVDNAStatMSAProfileTaskSettings@1@@Z$7 10015668 f   DNAStatMSAProfileDialog.obj
 0001:00014676       __unwindfunclet$??0DNAStatMSAProfileTask@U2@@QAE@ABVDNAStatMSAProfileTaskSettings@1@@Z$8 10015676 f   DNAStatMSAProfileDialog.obj
 0001:00014685       __ehhandler$??0DNAStatMSAProfileTask@U2@@QAE@ABVDNAStatMSAProfileTaskSettings@1@@Z 10015685 f   DNAStatMSAProfileDialog.obj
 0001:000146a0       __unwindfunclet$??0DNAStatMSAProfileTaskSettings@U2@@QAE@ABV01@@Z$0 100156a0 f   DNAStatMSAProfileDialog.obj
 0001:000146a9       __unwindfunclet$??0DNAStatMSAProfileTaskSettings@U2@@QAE@ABV01@@Z$1 100156a9 f   DNAStatMSAProfileDialog.obj
 0001:000146b5       __unwindfunclet$??0DNAStatMSAProfileTaskSettings@U2@@QAE@ABV01@@Z$2 100156b5 f   DNAStatMSAProfileDialog.obj
 0001:000146c1       __ehhandler$??0DNAStatMSAProfileTaskSettings@U2@@QAE@ABV01@@Z 100156c1 f   DNAStatMSAProfileDialog.obj
 0001:000146e0       __unwindfunclet$??0DNAStatMSAProfileTaskSettings@U2@@QAE@XZ$0 100156e0 f   DNAStatMSAProfileDialog.obj
 0001:000146e9       __unwindfunclet$??0DNAStatMSAProfileTaskSettings@U2@@QAE@XZ$1 100156e9 f   DNAStatMSAProfileDialog.obj
 0001:000146f5       __unwindfunclet$??0DNAStatMSAProfileTaskSettings@U2@@QAE@XZ$2 100156f5 f   DNAStatMSAProfileDialog.obj
 0001:000146fd       __unwindfunclet$??0DNAStatMSAProfileTaskSettings@U2@@QAE@XZ$3 100156fd f   DNAStatMSAProfileDialog.obj
 0001:00014706       __unwindfunclet$??0DNAStatMSAProfileTaskSettings@U2@@QAE@XZ$4 10015706 f   DNAStatMSAProfileDialog.obj
 0001:00014712       __ehhandler$??0DNAStatMSAProfileTaskSettings@U2@@QAE@XZ 10015712 f   DNAStatMSAProfileDialog.obj
 0001:00014730       __unwindfunclet$??1DNAStatMSAProfileTask@U2@@UAE@XZ$0 10015730 f   DNAStatMSAProfileDialog.obj
 0001:00014739       __unwindfunclet$??1DNAStatMSAProfileTask@U2@@UAE@XZ$1 10015739 f   DNAStatMSAProfileDialog.obj
 0001:00014747       __unwindfunclet$??1DNAStatMSAProfileTask@U2@@UAE@XZ$2 10015747 f   DNAStatMSAProfileDialog.obj
 0001:00014755       __unwindfunclet$??1DNAStatMSAProfileTask@U2@@UAE@XZ$3 10015755 f   DNAStatMSAProfileDialog.obj
 0001:00014763       __unwindfunclet$??1DNAStatMSAProfileTask@U2@@UAE@XZ$4 10015763 f   DNAStatMSAProfileDialog.obj
 0001:00014771       __unwindfunclet$??1DNAStatMSAProfileTask@U2@@UAE@XZ$5 10015771 f   DNAStatMSAProfileDialog.obj
 0001:0001477f       __unwindfunclet$??1DNAStatMSAProfileTask@U2@@UAE@XZ$6 1001577f f   DNAStatMSAProfileDialog.obj
 0001:0001478d       __unwindfunclet$??1DNAStatMSAProfileTask@U2@@UAE@XZ$10 1001578d f   DNAStatMSAProfileDialog.obj
 0001:00014796       __unwindfunclet$??1DNAStatMSAProfileTask@U2@@UAE@XZ$11 10015796 f   DNAStatMSAProfileDialog.obj
 0001:000147a2       __unwindfunclet$??1DNAStatMSAProfileTask@U2@@UAE@XZ$12 100157a2 f   DNAStatMSAProfileDialog.obj
 0001:000147ae       __ehhandler$??1DNAStatMSAProfileTask@U2@@UAE@XZ 100157ae f   DNAStatMSAProfileDialog.obj
 0001:000147d0       __unwindfunclet$??1DNAStatMSAProfileTaskSettings@U2@@QAE@XZ$0 100157d0 f   DNAStatMSAProfileDialog.obj
 0001:000147d9       __unwindfunclet$??1DNAStatMSAProfileTaskSettings@U2@@QAE@XZ$1 100157d9 f   DNAStatMSAProfileDialog.obj
 0001:000147e5       __unwindfunclet$??1DNAStatMSAProfileTaskSettings@U2@@QAE@XZ$2 100157e5 f   DNAStatMSAProfileDialog.obj
 0001:000147f1       __ehhandler$??1DNAStatMSAProfileTaskSettings@U2@@QAE@XZ 100157f1 f   DNAStatMSAProfileDialog.obj
 0001:00014810       __unwindfunclet$??H@YA?BVQString@@ABV0@0@Z$0 10015810 f   DNAStatMSAProfileDialog.obj
 0001:0001482a       __ehhandler$??H@YA?BVQString@@ABV0@0@Z 1001582a f   DNAStatMSAProfileDialog.obj
 0001:00014850       __unwindfunclet$??H@YA?BVQString@@ABV0@PBD@Z$0 10015850 f   DNAStatMSAProfileDialog.obj
 0001:0001486a       __unwindfunclet$??H@YA?BVQString@@ABV0@PBD@Z$1 1001586a f   DNAStatMSAProfileDialog.obj
 0001:00014873       __ehhandler$??H@YA?BVQString@@ABV0@PBD@Z 10015873 f   DNAStatMSAProfileDialog.obj
 0001:00014890       __unwindfunclet$??H@YA?BVQString@@PBDABV0@@Z$0 10015890 f   DNAStatMSAProfileDialog.obj
 0001:000148aa       __ehhandler$??H@YA?BVQString@@PBDABV0@@Z 100158aa f   DNAStatMSAProfileDialog.obj
 0001:000148d0       __unwindfunclet$??__EalgoLog@U2@@YAXXZ$0 100158d0 f   DNAStatMSAProfileDialog.obj
 0001:000148d9       __ehhandler$??__EalgoLog@U2@@YAXXZ 100158d9 f   DNAStatMSAProfileDialog.obj
 0001:00014900       __unwindfunclet$??__EcmdLog@U2@@YAXXZ$0 10015900 f   DNAStatMSAProfileDialog.obj
 0001:00014909       __ehhandler$??__EcmdLog@U2@@YAXXZ 10015909 f   DNAStatMSAProfileDialog.obj
 0001:00014930       __unwindfunclet$??__EcoreLog@U2@@YAXXZ$0 10015930 f   DNAStatMSAProfileDialog.obj
 0001:00014939       __ehhandler$??__EcoreLog@U2@@YAXXZ 10015939 f   DNAStatMSAProfileDialog.obj
 0001:00014960       __unwindfunclet$??__EioLog@U2@@YAXXZ$0 10015960 f   DNAStatMSAProfileDialog.obj
 0001:00014969       __ehhandler$??__EioLog@U2@@YAXXZ 10015969 f   DNAStatMSAProfileDialog.obj
 0001:00014990       __unwindfunclet$??__EperfLog@U2@@YAXXZ$0 10015990 f   DNAStatMSAProfileDialog.obj
 0001:00014999       __ehhandler$??__EperfLog@U2@@YAXXZ 10015999 f   DNAStatMSAProfileDialog.obj
 0001:000149c0       __unwindfunclet$??__EscriptLog@U2@@YAXXZ$0 100159c0 f   DNAStatMSAProfileDialog.obj
 0001:000149c9       __ehhandler$??__EscriptLog@U2@@YAXXZ 100159c9 f   DNAStatMSAProfileDialog.obj
 0001:000149f0       __unwindfunclet$??__EtaskLog@U2@@YAXXZ$0 100159f0 f   DNAStatMSAProfileDialog.obj
 0001:000149f9       __ehhandler$??__EtaskLog@U2@@YAXXZ 100159f9 f   DNAStatMSAProfileDialog.obj
 0001:00014a20       __unwindfunclet$??__EuiLog@U2@@YAXXZ$0 10015a20 f   DNAStatMSAProfileDialog.obj
 0001:00014a29       __ehhandler$??__EuiLog@U2@@YAXXZ 10015a29 f   DNAStatMSAProfileDialog.obj
 0001:00014a50       __unwindfunclet$??__EuserActLog@U2@@YAXXZ$0 10015a50 f   DNAStatMSAProfileDialog.obj
 0001:00014a59       __ehhandler$??__EuserActLog@U2@@YAXXZ 10015a59 f   DNAStatMSAProfileDialog.obj
 0001:00014a80       __ehhandler$?_Copy@?$basic_string@DU?$char_traits@D@std@@V?$allocator@D@2@@std@@QAEXII@Z 10015a80 f   DNAStatMSAProfileDialog.obj
 0001:00014aa0       __unwindfunclet$?accept@DNAStatMSAProfileDialog@U2@@UAEXXZ$0 10015aa0 f   DNAStatMSAProfileDialog.obj
 0001:00014aa8       __unwindfunclet$?accept@DNAStatMSAProfileDialog@U2@@UAEXXZ$1 10015aa8 f   DNAStatMSAProfileDialog.obj
 0001:00014ab1       __unwindfunclet$?accept@DNAStatMSAProfileDialog@U2@@UAEXXZ$2 10015ab1 f   DNAStatMSAProfileDialog.obj
 0001:00014aba       __unwindfunclet$?accept@DNAStatMSAProfileDialog@U2@@UAEXXZ$3 10015aba f   DNAStatMSAProfileDialog.obj
 0001:00014ac3       __unwindfunclet$?accept@DNAStatMSAProfileDialog@U2@@UAEXXZ$4 10015ac3 f   DNAStatMSAProfileDialog.obj
 0001:00014acc       __unwindfunclet$?accept@DNAStatMSAProfileDialog@U2@@UAEXXZ$5 10015acc f   DNAStatMSAProfileDialog.obj
 0001:00014ad7       __unwindfunclet$?accept@DNAStatMSAProfileDialog@U2@@UAEXXZ$7 10015ad7 f   DNAStatMSAProfileDialog.obj
 0001:00014ae0       __unwindfunclet$?accept@DNAStatMSAProfileDialog@U2@@UAEXXZ$8 10015ae0 f   DNAStatMSAProfileDialog.obj
 0001:00014ae9       __unwindfunclet$?accept@DNAStatMSAProfileDialog@U2@@UAEXXZ$9 10015ae9 f   DNAStatMSAProfileDialog.obj
 0001:00014af2       __ehhandler$?accept@DNAStatMSAProfileDialog@U2@@UAEXXZ 10015af2 f   DNAStatMSAProfileDialog.obj
 0001:00014b10       __unwindfunclet$?append@?$QList@VQString@@@@QAEXABVQString@@@Z$7 10015b10 f   DNAStatMSAProfileDialog.obj
 0001:00014b21       __unwindfunclet$?append@?$QList@VQString@@@@QAEXABVQString@@@Z$11 10015b21 f   DNAStatMSAProfileDialog.obj
 0001:00014b32       __ehhandler$?append@?$QList@VQString@@@@QAEXABVQString@@@Z 10015b32 f   DNAStatMSAProfileDialog.obj
 0001:00014b50       __unwindfunclet$?clear@?$QVector@D@@QAEXXZ$0 10015b50 f   DNAStatMSAProfileDialog.obj
 0001:00014b58       __ehhandler$?clear@?$QVector@D@@QAEXXZ 10015b58 f   DNAStatMSAProfileDialog.obj
 0001:00014b80       __unwindfunclet$?clear@?$QVector@UColumnStat@DNAStatMSAProfileTask@U2@@@@QAEXXZ$0 10015b80 f   DNAStatMSAProfileDialog.obj
 0001:00014b88       __ehhandler$?clear@?$QVector@UColumnStat@DNAStatMSAProfileTask@U2@@@@QAEXXZ 10015b88 f   DNAStatMSAProfileDialog.obj
 0001:00014bb0       __unwindfunclet$?computeStats@DNAStatMSAProfileTask@U2@@AAEXXZ$0 10015bb0 f   DNAStatMSAProfileDialog.obj
 0001:00014bb9       __unwindfunclet$?computeStats@DNAStatMSAProfileTask@U2@@AAEXXZ$1 10015bb9 f   DNAStatMSAProfileDialog.obj
 0001:00014bc2       __unwindfunclet$?computeStats@DNAStatMSAProfileTask@U2@@AAEXXZ$2 10015bc2 f   DNAStatMSAProfileDialog.obj
 0001:00014bcb       __ehhandler$?computeStats@DNAStatMSAProfileTask@U2@@AAEXXZ 10015bcb f   DNAStatMSAProfileDialog.obj
 0001:00014bf0       __unwindfunclet$?copyConstruct@?$QVector@UColumnStat@DNAStatMSAProfileTask@U2@@@@AAEXPBUColumnStat@DNAStatMSAProfileTask@U2@@0PAU234@@Z$0 10015bf0 f   DNAStatMSAProfileDialog.obj
 0001:00014c01       __ehhandler$?copyConstruct@?$QVector@UColumnStat@DNAStatMSAProfileTask@U2@@@@AAEXPBUColumnStat@DNAStatMSAProfileTask@U2@@0PAU234@@Z 10015c01 f   DNAStatMSAProfileDialog.obj
 0001:00014c20       __ehhandler$?detach_helper_grow@?$QList@VQString@@@@AAEPAUNode@1@HH@Z 10015c20 f   DNAStatMSAProfileDialog.obj
 0001:00014c40       __unwindfunclet$?generateReport@DNAStatMSAProfileTask@U2@@UBE?AVQString@@XZ$0 10015c40 f   DNAStatMSAProfileDialog.obj
 0001:00014c49       __unwindfunclet$?generateReport@DNAStatMSAProfileTask@U2@@UBE?AVQString@@XZ$1 10015c49 f   DNAStatMSAProfileDialog.obj
 0001:00014c52       __unwindfunclet$?generateReport@DNAStatMSAProfileTask@U2@@UBE?AVQString@@XZ$2 10015c52 f   DNAStatMSAProfileDialog.obj
 0001:00014c6c       __unwindfunclet$?generateReport@DNAStatMSAProfileTask@U2@@UBE?AVQString@@XZ$3 10015c6c f   DNAStatMSAProfileDialog.obj
 0001:00014c75       __unwindfunclet$?generateReport@DNAStatMSAProfileTask@U2@@UBE?AVQString@@XZ$4 10015c75 f   DNAStatMSAProfileDialog.obj
 0001:00014c7e       __unwindfunclet$?generateReport@DNAStatMSAProfileTask@U2@@UBE?AVQString@@XZ$5 10015c7e f   DNAStatMSAProfileDialog.obj
 0001:00014c87       __unwindfunclet$?generateReport@DNAStatMSAProfileTask@U2@@UBE?AVQString@@XZ$6 10015c87 f   DNAStatMSAProfileDialog.obj
 0001:00014c90       __unwindfunclet$?generateReport@DNAStatMSAProfileTask@U2@@UBE?AVQString@@XZ$7 10015c90 f   DNAStatMSAProfileDialog.obj
 0001:00014c99       __unwindfunclet$?generateReport@DNAStatMSAProfileTask@U2@@UBE?AVQString@@XZ$8 10015c99 f   DNAStatMSAProfileDialog.obj
 0001:00014ca2       __ehhandler$?generateReport@DNAStatMSAProfileTask@U2@@UBE?AVQString@@XZ 10015ca2 f   DNAStatMSAProfileDialog.obj
 0001:00014cc0       __unwindfunclet$?initSaveController@DNAStatMSAProfileDialog@U2@@AAEXXZ$0 10015cc0 f   DNAStatMSAProfileDialog.obj
 0001:00014cc9       __unwindfunclet$?initSaveController@DNAStatMSAProfileDialog@U2@@AAEXXZ$1 10015cc9 f   DNAStatMSAProfileDialog.obj
 0001:00014cd2       __unwindfunclet$?initSaveController@DNAStatMSAProfileDialog@U2@@AAEXXZ$2 10015cd2 f   DNAStatMSAProfileDialog.obj
 0001:00014cdb       __unwindfunclet$?initSaveController@DNAStatMSAProfileDialog@U2@@AAEXXZ$3 10015cdb f   DNAStatMSAProfileDialog.obj
 0001:00014ce4       __unwindfunclet$?initSaveController@DNAStatMSAProfileDialog@U2@@AAEXXZ$4 10015ce4 f   DNAStatMSAProfileDialog.obj
 0001:00014ced       __unwindfunclet$?initSaveController@DNAStatMSAProfileDialog@U2@@AAEXXZ$5 10015ced f   DNAStatMSAProfileDialog.obj
 0001:00014cf6       __unwindfunclet$?initSaveController@DNAStatMSAProfileDialog@U2@@AAEXXZ$6 10015cf6 f   DNAStatMSAProfileDialog.obj
 0001:00014cff       __unwindfunclet$?initSaveController@DNAStatMSAProfileDialog@U2@@AAEXXZ$7 10015cff f   DNAStatMSAProfileDialog.obj
 0001:00014d08       __unwindfunclet$?initSaveController@DNAStatMSAProfileDialog@U2@@AAEXXZ$8 10015d08 f   DNAStatMSAProfileDialog.obj
 0001:00014d11       __unwindfunclet$?initSaveController@DNAStatMSAProfileDialog@U2@@AAEXXZ$9 10015d11 f   DNAStatMSAProfileDialog.obj
 0001:00014d1a       __unwindfunclet$?initSaveController@DNAStatMSAProfileDialog@U2@@AAEXXZ$10 10015d1a f   DNAStatMSAProfileDialog.obj
 0001:00014d23       __unwindfunclet$?initSaveController@DNAStatMSAProfileDialog@U2@@AAEXXZ$11 10015d23 f   DNAStatMSAProfileDialog.obj
 0001:00014d2c       __unwindfunclet$?initSaveController@DNAStatMSAProfileDialog@U2@@AAEXXZ$12 10015d2c f   DNAStatMSAProfileDialog.obj
 0001:00014d34       __unwindfunclet$?initSaveController@DNAStatMSAProfileDialog@U2@@AAEXXZ$13 10015d34 f   DNAStatMSAProfileDialog.obj
 0001:00014d3d       __unwindfunclet$?initSaveController@DNAStatMSAProfileDialog@U2@@AAEXXZ$14 10015d3d f   DNAStatMSAProfileDialog.obj
 0001:00014d45       __unwindfunclet$?initSaveController@DNAStatMSAProfileDialog@U2@@AAEXXZ$15 10015d45 f   DNAStatMSAProfileDialog.obj
 0001:00014d4e       __unwindfunclet$?initSaveController@DNAStatMSAProfileDialog@U2@@AAEXXZ$16 10015d4e f   DNAStatMSAProfileDialog.obj
 0001:00014d59       __ehhandler$?initSaveController@DNAStatMSAProfileDialog@U2@@AAEXXZ 10015d59 f   DNAStatMSAProfileDialog.obj
 0001:00014d80       __unwindfunclet$?node_construct@?$QList@VQString@@@@AAEXPAUNode@1@ABVQString@@@Z$1 10015d80 f   DNAStatMSAProfileDialog.obj
 0001:00014d91       __ehhandler$?node_construct@?$QList@VQString@@@@AAEXPAUNode@1@ABVQString@@@Z 10015d91 f   DNAStatMSAProfileDialog.obj
 0001:00014db0       __unwindfunclet$?node_copy@?$QList@VQString@@@@AAEXPAUNode@1@00@Z$5 10015db0 f   DNAStatMSAProfileDialog.obj
 0001:00014dc1       __ehhandler$?node_copy@?$QList@VQString@@@@AAEXPAUNode@1@00@Z 10015dc1 f   DNAStatMSAProfileDialog.obj
 0001:00014de0       __ehhandler$?reallocData@?$QVector@D@@AAEXHHV?$QFlags@W4AllocationOption@QArrayData@@@@@Z 10015de0 f   DNAStatMSAProfileDialog.obj
 0001:00014e00       __ehhandler$?reallocData@?$QVector@H@@AAEXHHV?$QFlags@W4AllocationOption@QArrayData@@@@@Z 10015e00 f   DNAStatMSAProfileDialog.obj
 0001:00014e20       __unwindfunclet$?reallocData@?$QVector@UColumnStat@DNAStatMSAProfileTask@U2@@@@AAEXHHV?$QFlags@W4AllocationOption@QArrayData@@@@@Z$4 10015e20 f   DNAStatMSAProfileDialog.obj
 0001:00014e31       __ehhandler$?reallocData@?$QVector@UColumnStat@DNAStatMSAProfileTask@U2@@@@AAEXHHV?$QFlags@W4AllocationOption@QArrayData@@@@@Z 10015e31 f   DNAStatMSAProfileDialog.obj
 0001:00014e50       __unwindfunclet$?report@DNAStatMSAProfileTask@U2@@UAE?AW4ReportResult@Task@2@XZ$0 10015e50 f   DNAStatMSAProfileDialog.obj
 0001:00014e6a       __unwindfunclet$?report@DNAStatMSAProfileTask@U2@@UAE?AW4ReportResult@Task@2@XZ$1 10015e6a f   DNAStatMSAProfileDialog.obj
 0001:00014e84       __unwindfunclet$?report@DNAStatMSAProfileTask@U2@@UAE?AW4ReportResult@Task@2@XZ$2 10015e84 f   DNAStatMSAProfileDialog.obj
 0001:00014e9e       __unwindfunclet$?report@DNAStatMSAProfileTask@U2@@UAE?AW4ReportResult@Task@2@XZ$3 10015e9e f   DNAStatMSAProfileDialog.obj
 0001:00014ea7       __unwindfunclet$?report@DNAStatMSAProfileTask@U2@@UAE?AW4ReportResult@Task@2@XZ$4 10015ea7 f   DNAStatMSAProfileDialog.obj
 0001:00014eb2       __unwindfunclet$?report@DNAStatMSAProfileTask@U2@@UAE?AW4ReportResult@Task@2@XZ$5 10015eb2 f   DNAStatMSAProfileDialog.obj
 0001:00014ebb       __unwindfunclet$?report@DNAStatMSAProfileTask@U2@@UAE?AW4ReportResult@Task@2@XZ$6 10015ebb f   DNAStatMSAProfileDialog.obj
 0001:00014ec4       __ehhandler$?report@DNAStatMSAProfileTask@U2@@UAE?AW4ReportResult@Task@2@XZ 10015ec4 f   DNAStatMSAProfileDialog.obj
 0001:00014ee0       __unwindfunclet$?retranslateUi@Ui_DNAStatMSAProfileDialog@@QAEXPAVQDialog@@@Z$0 10015ee0 f   DNAStatMSAProfileDialog.obj
 0001:00014ee9       __unwindfunclet$?retranslateUi@Ui_DNAStatMSAProfileDialog@@QAEXPAVQDialog@@@Z$1 10015ee9 f   DNAStatMSAProfileDialog.obj
 0001:00014ef2       __unwindfunclet$?retranslateUi@Ui_DNAStatMSAProfileDialog@@QAEXPAVQDialog@@@Z$2 10015ef2 f   DNAStatMSAProfileDialog.obj
 0001:00014efb       __unwindfunclet$?retranslateUi@Ui_DNAStatMSAProfileDialog@@QAEXPAVQDialog@@@Z$3 10015efb f   DNAStatMSAProfileDialog.obj
 0001:00014f04       __unwindfunclet$?retranslateUi@Ui_DNAStatMSAProfileDialog@@QAEXPAVQDialog@@@Z$4 10015f04 f   DNAStatMSAProfileDialog.obj
 0001:00014f0d       __unwindfunclet$?retranslateUi@Ui_DNAStatMSAProfileDialog@@QAEXPAVQDialog@@@Z$5 10015f0d f   DNAStatMSAProfileDialog.obj
 0001:00014f16       __unwindfunclet$?retranslateUi@Ui_DNAStatMSAProfileDialog@@QAEXPAVQDialog@@@Z$6 10015f16 f   DNAStatMSAProfileDialog.obj
 0001:00014f1f       __unwindfunclet$?retranslateUi@Ui_DNAStatMSAProfileDialog@@QAEXPAVQDialog@@@Z$7 10015f1f f   DNAStatMSAProfileDialog.obj
 0001:00014f28       __unwindfunclet$?retranslateUi@Ui_DNAStatMSAProfileDialog@@QAEXPAVQDialog@@@Z$8 10015f28 f   DNAStatMSAProfileDialog.obj
 0001:00014f31       __unwindfunclet$?retranslateUi@Ui_DNAStatMSAProfileDialog@@QAEXPAVQDialog@@@Z$9 10015f31 f   DNAStatMSAProfileDialog.obj
 0001:00014f3a       __unwindfunclet$?retranslateUi@Ui_DNAStatMSAProfileDialog@@QAEXPAVQDialog@@@Z$10 10015f3a f   DNAStatMSAProfileDialog.obj
 0001:00014f43       __unwindfunclet$?retranslateUi@Ui_DNAStatMSAProfileDialog@@QAEXPAVQDialog@@@Z$11 10015f43 f   DNAStatMSAProfileDialog.obj
 0001:00014f4c       __unwindfunclet$?retranslateUi@Ui_DNAStatMSAProfileDialog@@QAEXPAVQDialog@@@Z$12 10015f4c f   DNAStatMSAProfileDialog.obj
 0001:00014f55       __ehhandler$?retranslateUi@Ui_DNAStatMSAProfileDialog@@QAEXPAVQDialog@@@Z 10015f55 f   DNAStatMSAProfileDialog.obj
 0001:00014f70       __unwindfunclet$?run@DNAStatMSAProfileTask@U2@@UAEXXZ$2 10015f70 f   DNAStatMSAProfileDialog.obj
 0001:00014f79       __unwindfunclet$?run@DNAStatMSAProfileTask@U2@@UAEXXZ$67 10015f79 f   DNAStatMSAProfileDialog.obj
 0001:00014f84       __unwindfunclet$?run@DNAStatMSAProfileTask@U2@@UAEXXZ$68 10015f84 f   DNAStatMSAProfileDialog.obj
 0001:00014f8d       __unwindfunclet$?run@DNAStatMSAProfileTask@U2@@UAEXXZ$69 10015f8d f   DNAStatMSAProfileDialog.obj
 0001:00014f96       __unwindfunclet$?run@DNAStatMSAProfileTask@U2@@UAEXXZ$70 10015f96 f   DNAStatMSAProfileDialog.obj
 0001:00014f9f       __unwindfunclet$?run@DNAStatMSAProfileTask@U2@@UAEXXZ$71 10015f9f f   DNAStatMSAProfileDialog.obj
 0001:00014fa8       __unwindfunclet$?run@DNAStatMSAProfileTask@U2@@UAEXXZ$72 10015fa8 f   DNAStatMSAProfileDialog.obj
 0001:00014fb1       __unwindfunclet$?run@DNAStatMSAProfileTask@U2@@UAEXXZ$73 10015fb1 f   DNAStatMSAProfileDialog.obj
 0001:00014fba       __unwindfunclet$?run@DNAStatMSAProfileTask@U2@@UAEXXZ$3 10015fba f   DNAStatMSAProfileDialog.obj
 0001:00014fc5       __unwindfunclet$?run@DNAStatMSAProfileTask@U2@@UAEXXZ$4 10015fc5 f   DNAStatMSAProfileDialog.obj
 0001:00014fce       __unwindfunclet$?run@DNAStatMSAProfileTask@U2@@UAEXXZ$5 10015fce f   DNAStatMSAProfileDialog.obj
 0001:00014fd7       __unwindfunclet$?run@DNAStatMSAProfileTask@U2@@UAEXXZ$6 10015fd7 f   DNAStatMSAProfileDialog.obj
 0001:00014fe0       __unwindfunclet$?run@DNAStatMSAProfileTask@U2@@UAEXXZ$7 10015fe0 f   DNAStatMSAProfileDialog.obj
 0001:00014fe9       __unwindfunclet$?run@DNAStatMSAProfileTask@U2@@UAEXXZ$8 10015fe9 f   DNAStatMSAProfileDialog.obj
 0001:00014ff2       __unwindfunclet$?run@DNAStatMSAProfileTask@U2@@UAEXXZ$9 10015ff2 f   DNAStatMSAProfileDialog.obj
 0001:00014ffb       __unwindfunclet$?run@DNAStatMSAProfileTask@U2@@UAEXXZ$11 10015ffb f   DNAStatMSAProfileDialog.obj
 0001:0001500f       __unwindfunclet$?run@DNAStatMSAProfileTask@U2@@UAEXXZ$12 1001600f f   DNAStatMSAProfileDialog.obj
 0001:00015018       __unwindfunclet$?run@DNAStatMSAProfileTask@U2@@UAEXXZ$13 10016018 f   DNAStatMSAProfileDialog.obj
 0001:00015021       __unwindfunclet$?run@DNAStatMSAProfileTask@U2@@UAEXXZ$14 10016021 f   DNAStatMSAProfileDialog.obj
 0001:0001502a       __unwindfunclet$?run@DNAStatMSAProfileTask@U2@@UAEXXZ$15 1001602a f   DNAStatMSAProfileDialog.obj
 0001:00015033       __unwindfunclet$?run@DNAStatMSAProfileTask@U2@@UAEXXZ$16 10016033 f   DNAStatMSAProfileDialog.obj
 0001:0001503c       __unwindfunclet$?run@DNAStatMSAProfileTask@U2@@UAEXXZ$17 1001603c f   DNAStatMSAProfileDialog.obj
 0001:00015045       __unwindfunclet$?run@DNAStatMSAProfileTask@U2@@UAEXXZ$18 10016045 f   DNAStatMSAProfileDialog.obj
 0001:0001504e       __unwindfunclet$?run@DNAStatMSAProfileTask@U2@@UAEXXZ$19 1001604e f   DNAStatMSAProfileDialog.obj
 0001:00015057       __unwindfunclet$?run@DNAStatMSAProfileTask@U2@@UAEXXZ$20 10016057 f   DNAStatMSAProfileDialog.obj
 0001:00015060       __unwindfunclet$?run@DNAStatMSAProfileTask@U2@@UAEXXZ$21 10016060 f   DNAStatMSAProfileDialog.obj
 0001:00015069       __unwindfunclet$?run@DNAStatMSAProfileTask@U2@@UAEXXZ$22 10016069 f   DNAStatMSAProfileDialog.obj
 0001:00015083       __unwindfunclet$?run@DNAStatMSAProfileTask@U2@@UAEXXZ$23 10016083 f   DNAStatMSAProfileDialog.obj
 0001:0001509d       __unwindfunclet$?run@DNAStatMSAProfileTask@U2@@UAEXXZ$24 1001609d f   DNAStatMSAProfileDialog.obj
 0001:000150a6       __unwindfunclet$?run@DNAStatMSAProfileTask@U2@@UAEXXZ$25 100160a6 f   DNAStatMSAProfileDialog.obj
 0001:000150af       __unwindfunclet$?run@DNAStatMSAProfileTask@U2@@UAEXXZ$26 100160af f   DNAStatMSAProfileDialog.obj
 0001:000150b8       __unwindfunclet$?run@DNAStatMSAProfileTask@U2@@UAEXXZ$27 100160b8 f   DNAStatMSAProfileDialog.obj
 0001:000150c1       __unwindfunclet$?run@DNAStatMSAProfileTask@U2@@UAEXXZ$28 100160c1 f   DNAStatMSAProfileDialog.obj
 0001:000150ca       __unwindfunclet$?run@DNAStatMSAProfileTask@U2@@UAEXXZ$29 100160ca f   DNAStatMSAProfileDialog.obj
 0001:000150d3       __unwindfunclet$?run@DNAStatMSAProfileTask@U2@@UAEXXZ$31 100160d3 f   DNAStatMSAProfileDialog.obj
 0001:000150ed       __unwindfunclet$?run@DNAStatMSAProfileTask@U2@@UAEXXZ$30 100160ed f   DNAStatMSAProfileDialog.obj
 0001:00015107       __unwindfunclet$?run@DNAStatMSAProfileTask@U2@@UAEXXZ$32 10016107 f   DNAStatMSAProfileDialog.obj
 0001:00015110       __unwindfunclet$?run@DNAStatMSAProfileTask@U2@@UAEXXZ$33 10016110 f   DNAStatMSAProfileDialog.obj
 0001:00015119       __unwindfunclet$?run@DNAStatMSAProfileTask@U2@@UAEXXZ$34 10016119 f   DNAStatMSAProfileDialog.obj
 0001:00015122       __unwindfunclet$?run@DNAStatMSAProfileTask@U2@@UAEXXZ$35 10016122 f   DNAStatMSAProfileDialog.obj
 0001:0001512b       __unwindfunclet$?run@DNAStatMSAProfileTask@U2@@UAEXXZ$36 1001612b f   DNAStatMSAProfileDialog.obj
 0001:00015134       __unwindfunclet$?run@DNAStatMSAProfileTask@U2@@UAEXXZ$37 10016134 f   DNAStatMSAProfileDialog.obj
 0001:0001513d       __unwindfunclet$?run@DNAStatMSAProfileTask@U2@@UAEXXZ$38 1001613d f   DNAStatMSAProfileDialog.obj
 0001:00015146       __unwindfunclet$?run@DNAStatMSAProfileTask@U2@@UAEXXZ$39 10016146 f   DNAStatMSAProfileDialog.obj
 0001:0001514f       __unwindfunclet$?run@DNAStatMSAProfileTask@U2@@UAEXXZ$40 1001614f f   DNAStatMSAProfileDialog.obj
 0001:00015158       __unwindfunclet$?run@DNAStatMSAProfileTask@U2@@UAEXXZ$41 10016158 f   DNAStatMSAProfileDialog.obj
 0001:00015161       __unwindfunclet$?run@DNAStatMSAProfileTask@U2@@UAEXXZ$42 10016161 f   DNAStatMSAProfileDialog.obj
 0001:0001516a       __unwindfunclet$?run@DNAStatMSAProfileTask@U2@@UAEXXZ$43 1001616a f   DNAStatMSAProfileDialog.obj
 0001:00015173       __unwindfunclet$?run@DNAStatMSAProfileTask@U2@@UAEXXZ$44 10016173 f   DNAStatMSAProfileDialog.obj
 0001:0001517c       __unwindfunclet$?run@DNAStatMSAProfileTask@U2@@UAEXXZ$45 1001617c f   DNAStatMSAProfileDialog.obj
 0001:00015185       __unwindfunclet$?run@DNAStatMSAProfileTask@U2@@UAEXXZ$46 10016185 f   DNAStatMSAProfileDialog.obj
 0001:0001518e       __unwindfunclet$?run@DNAStatMSAProfileTask@U2@@UAEXXZ$47 1001618e f   DNAStatMSAProfileDialog.obj
 0001:00015197       __unwindfunclet$?run@DNAStatMSAProfileTask@U2@@UAEXXZ$48 10016197 f   DNAStatMSAProfileDialog.obj
 0001:000151a0       __unwindfunclet$?run@DNAStatMSAProfileTask@U2@@UAEXXZ$49 100161a0 f   DNAStatMSAProfileDialog.obj
 0001:000151a9       __unwindfunclet$?run@DNAStatMSAProfileTask@U2@@UAEXXZ$50 100161a9 f   DNAStatMSAProfileDialog.obj
 0001:000151b2       __unwindfunclet$?run@DNAStatMSAProfileTask@U2@@UAEXXZ$51 100161b2 f   DNAStatMSAProfileDialog.obj
 0001:000151bb       __unwindfunclet$?run@DNAStatMSAProfileTask@U2@@UAEXXZ$52 100161bb f   DNAStatMSAProfileDialog.obj
 0001:000151c4       __unwindfunclet$?run@DNAStatMSAProfileTask@U2@@UAEXXZ$53 100161c4 f   DNAStatMSAProfileDialog.obj
 0001:000151cd       __unwindfunclet$?run@DNAStatMSAProfileTask@U2@@UAEXXZ$54 100161cd f   DNAStatMSAProfileDialog.obj
 0001:000151d6       __unwindfunclet$?run@DNAStatMSAProfileTask@U2@@UAEXXZ$55 100161d6 f   DNAStatMSAProfileDialog.obj
 0001:000151df       __unwindfunclet$?run@DNAStatMSAProfileTask@U2@@UAEXXZ$56 100161df f   DNAStatMSAProfileDialog.obj
 0001:000151e8       __unwindfunclet$?run@DNAStatMSAProfileTask@U2@@UAEXXZ$57 100161e8 f   DNAStatMSAProfileDialog.obj
 0001:000151f1       __unwindfunclet$?run@DNAStatMSAProfileTask@U2@@UAEXXZ$58 100161f1 f   DNAStatMSAProfileDialog.obj
 0001:000151fa       __unwindfunclet$?run@DNAStatMSAProfileTask@U2@@UAEXXZ$59 100161fa f   DNAStatMSAProfileDialog.obj
 0001:00015203       __unwindfunclet$?run@DNAStatMSAProfileTask@U2@@UAEXXZ$60 10016203 f   DNAStatMSAProfileDialog.obj
 0001:0001520c       __unwindfunclet$?run@DNAStatMSAProfileTask@U2@@UAEXXZ$61 1001620c f   DNAStatMSAProfileDialog.obj
 0001:00015215       __unwindfunclet$?run@DNAStatMSAProfileTask@U2@@UAEXXZ$62 10016215 f   DNAStatMSAProfileDialog.obj
 0001:0001521e       __unwindfunclet$?run@DNAStatMSAProfileTask@U2@@UAEXXZ$63 1001621e f   DNAStatMSAProfileDialog.obj
 0001:00015227       __unwindfunclet$?run@DNAStatMSAProfileTask@U2@@UAEXXZ$64 10016227 f   DNAStatMSAProfileDialog.obj
 0001:00015230       __unwindfunclet$?run@DNAStatMSAProfileTask@U2@@UAEXXZ$74 10016230 f   DNAStatMSAProfileDialog.obj
 0001:00015239       __unwindfunclet$?run@DNAStatMSAProfileTask@U2@@UAEXXZ$65 10016239 f   DNAStatMSAProfileDialog.obj
 0001:00015242       __unwindfunclet$?run@DNAStatMSAProfileTask@U2@@UAEXXZ$66 10016242 f   DNAStatMSAProfileDialog.obj
 0001:0001524b       __ehhandler$?run@DNAStatMSAProfileTask@U2@@UAEXXZ 1001624b f   DNAStatMSAProfileDialog.obj
 0001:00015280       __unwindfunclet$?setupUi@Ui_DNAStatMSAProfileDialog@@QAEXPAVQDialog@@@Z$1 10016280 f   DNAStatMSAProfileDialog.obj
 0001:00015289       __unwindfunclet$?setupUi@Ui_DNAStatMSAProfileDialog@@QAEXPAVQDialog@@@Z$2 10016289 f   DNAStatMSAProfileDialog.obj
 0001:00015294       __unwindfunclet$?setupUi@Ui_DNAStatMSAProfileDialog@@QAEXPAVQDialog@@@Z$3 10016294 f   DNAStatMSAProfileDialog.obj
 0001:0001529d       __unwindfunclet$?setupUi@Ui_DNAStatMSAProfileDialog@@QAEXPAVQDialog@@@Z$4 1001629d f   DNAStatMSAProfileDialog.obj
 0001:000152a8       __unwindfunclet$?setupUi@Ui_DNAStatMSAProfileDialog@@QAEXPAVQDialog@@@Z$5 100162a8 f   DNAStatMSAProfileDialog.obj
 0001:000152b1       __unwindfunclet$?setupUi@Ui_DNAStatMSAProfileDialog@@QAEXPAVQDialog@@@Z$6 100162b1 f   DNAStatMSAProfileDialog.obj
 0001:000152bc       __unwindfunclet$?setupUi@Ui_DNAStatMSAProfileDialog@@QAEXPAVQDialog@@@Z$7 100162bc f   DNAStatMSAProfileDialog.obj
 0001:000152c5       __unwindfunclet$?setupUi@Ui_DNAStatMSAProfileDialog@@QAEXPAVQDialog@@@Z$8 100162c5 f   DNAStatMSAProfileDialog.obj
 0001:000152d0       __unwindfunclet$?setupUi@Ui_DNAStatMSAProfileDialog@@QAEXPAVQDialog@@@Z$9 100162d0 f   DNAStatMSAProfileDialog.obj
 0001:000152d9       __unwindfunclet$?setupUi@Ui_DNAStatMSAProfileDialog@@QAEXPAVQDialog@@@Z$10 100162d9 f   DNAStatMSAProfileDialog.obj
 0001:000152e4       __unwindfunclet$?setupUi@Ui_DNAStatMSAProfileDialog@@QAEXPAVQDialog@@@Z$11 100162e4 f   DNAStatMSAProfileDialog.obj
 0001:000152ed       __unwindfunclet$?setupUi@Ui_DNAStatMSAProfileDialog@@QAEXPAVQDialog@@@Z$12 100162ed f   DNAStatMSAProfileDialog.obj
 0001:000152f8       __unwindfunclet$?setupUi@Ui_DNAStatMSAProfileDialog@@QAEXPAVQDialog@@@Z$13 100162f8 f   DNAStatMSAProfileDialog.obj
 0001:00015301       __unwindfunclet$?setupUi@Ui_DNAStatMSAProfileDialog@@QAEXPAVQDialog@@@Z$14 10016301 f   DNAStatMSAProfileDialog.obj
 0001:0001530c       __unwindfunclet$?setupUi@Ui_DNAStatMSAProfileDialog@@QAEXPAVQDialog@@@Z$15 1001630c f   DNAStatMSAProfileDialog.obj
 0001:00015315       __unwindfunclet$?setupUi@Ui_DNAStatMSAProfileDialog@@QAEXPAVQDialog@@@Z$16 10016315 f   DNAStatMSAProfileDialog.obj
 0001:00015320       __unwindfunclet$?setupUi@Ui_DNAStatMSAProfileDialog@@QAEXPAVQDialog@@@Z$17 10016320 f   DNAStatMSAProfileDialog.obj
 0001:00015329       __unwindfunclet$?setupUi@Ui_DNAStatMSAProfileDialog@@QAEXPAVQDialog@@@Z$18 10016329 f   DNAStatMSAProfileDialog.obj
 0001:00015334       __unwindfunclet$?setupUi@Ui_DNAStatMSAProfileDialog@@QAEXPAVQDialog@@@Z$19 10016334 f   DNAStatMSAProfileDialog.obj
 0001:0001533d       __unwindfunclet$?setupUi@Ui_DNAStatMSAProfileDialog@@QAEXPAVQDialog@@@Z$20 1001633d f   DNAStatMSAProfileDialog.obj
 0001:00015348       __unwindfunclet$?setupUi@Ui_DNAStatMSAProfileDialog@@QAEXPAVQDialog@@@Z$21 10016348 f   DNAStatMSAProfileDialog.obj
 0001:00015351       __unwindfunclet$?setupUi@Ui_DNAStatMSAProfileDialog@@QAEXPAVQDialog@@@Z$22 10016351 f   DNAStatMSAProfileDialog.obj
 0001:0001535c       __unwindfunclet$?setupUi@Ui_DNAStatMSAProfileDialog@@QAEXPAVQDialog@@@Z$23 1001635c f   DNAStatMSAProfileDialog.obj
 0001:00015365       __unwindfunclet$?setupUi@Ui_DNAStatMSAProfileDialog@@QAEXPAVQDialog@@@Z$24 10016365 f   DNAStatMSAProfileDialog.obj
 0001:00015370       __unwindfunclet$?setupUi@Ui_DNAStatMSAProfileDialog@@QAEXPAVQDialog@@@Z$25 10016370 f   DNAStatMSAProfileDialog.obj
 0001:00015379       __unwindfunclet$?setupUi@Ui_DNAStatMSAProfileDialog@@QAEXPAVQDialog@@@Z$26 10016379 f   DNAStatMSAProfileDialog.obj
 0001:00015384       __unwindfunclet$?setupUi@Ui_DNAStatMSAProfileDialog@@QAEXPAVQDialog@@@Z$27 10016384 f   DNAStatMSAProfileDialog.obj
 0001:0001538d       __unwindfunclet$?setupUi@Ui_DNAStatMSAProfileDialog@@QAEXPAVQDialog@@@Z$28 1001638d f   DNAStatMSAProfileDialog.obj
 0001:00015398       __unwindfunclet$?setupUi@Ui_DNAStatMSAProfileDialog@@QAEXPAVQDialog@@@Z$29 10016398 f   DNAStatMSAProfileDialog.obj
 0001:000153a1       __unwindfunclet$?setupUi@Ui_DNAStatMSAProfileDialog@@QAEXPAVQDialog@@@Z$30 100163a1 f   DNAStatMSAProfileDialog.obj
 0001:000153ac       __unwindfunclet$?setupUi@Ui_DNAStatMSAProfileDialog@@QAEXPAVQDialog@@@Z$31 100163ac f   DNAStatMSAProfileDialog.obj
 0001:000153b5       __unwindfunclet$?setupUi@Ui_DNAStatMSAProfileDialog@@QAEXPAVQDialog@@@Z$32 100163b5 f   DNAStatMSAProfileDialog.obj
 0001:000153c0       __unwindfunclet$?setupUi@Ui_DNAStatMSAProfileDialog@@QAEXPAVQDialog@@@Z$33 100163c0 f   DNAStatMSAProfileDialog.obj
 0001:000153c9       __unwindfunclet$?setupUi@Ui_DNAStatMSAProfileDialog@@QAEXPAVQDialog@@@Z$34 100163c9 f   DNAStatMSAProfileDialog.obj
 0001:000153d4       __unwindfunclet$?setupUi@Ui_DNAStatMSAProfileDialog@@QAEXPAVQDialog@@@Z$35 100163d4 f   DNAStatMSAProfileDialog.obj
 0001:000153dd       __unwindfunclet$?setupUi@Ui_DNAStatMSAProfileDialog@@QAEXPAVQDialog@@@Z$36 100163dd f   DNAStatMSAProfileDialog.obj
 0001:000153e8       __unwindfunclet$?setupUi@Ui_DNAStatMSAProfileDialog@@QAEXPAVQDialog@@@Z$37 100163e8 f   DNAStatMSAProfileDialog.obj
 0001:000153f1       __ehhandler$?setupUi@Ui_DNAStatMSAProfileDialog@@QAEXPAVQDialog@@@Z 100163f1 f   DNAStatMSAProfileDialog.obj
 0001:00015410       __ehhandler$??0?$QList@PAVGObjectViewAction@U2@@@@QAE@ABV0@@Z 10016410 f   DNAStatPlugin.obj
 0001:00015430       __unwindfunclet$??0DNAStatPlugin@U2@@QAE@XZ$0 10016430 f   DNAStatPlugin.obj
 0001:00015439       __unwindfunclet$??0DNAStatPlugin@U2@@QAE@XZ$1 10016439 f   DNAStatPlugin.obj
 0001:00015442       __unwindfunclet$??0DNAStatPlugin@U2@@QAE@XZ$2 10016442 f   DNAStatPlugin.obj
 0001:0001544b       __unwindfunclet$??0DNAStatPlugin@U2@@QAE@XZ$3 1001644b f   DNAStatPlugin.obj
 0001:00015456       __unwindfunclet$??0DNAStatPlugin@U2@@QAE@XZ$4 10016456 f   DNAStatPlugin.obj
 0001:00015461       __ehhandler$??0DNAStatPlugin@U2@@QAE@XZ 10016461 f   DNAStatPlugin.obj
 0001:00015480       __unwindfunclet$??1?$QObjectScopedPointer@VDNAStatMSAProfileDialog@U2@@@U2@@QAE@XZ$0 10016480 f   DNAStatPlugin.obj
 0001:00015488       __ehhandler$??1?$QObjectScopedPointer@VDNAStatMSAProfileDialog@U2@@@U2@@QAE@XZ 10016488 f   DNAStatPlugin.obj
 0001:000154b0       __unwindfunclet$??1?$QObjectScopedPointer@VDistanceMatrixMSAProfileDialog@U2@@@U2@@QAE@XZ$0 100164b0 f   DNAStatPlugin.obj
 0001:000154b8       __ehhandler$??1?$QObjectScopedPointer@VDistanceMatrixMSAProfileDialog@U2@@@U2@@QAE@XZ 100164b8 f   DNAStatPlugin.obj
 0001:000154e0       __unwindfunclet$??__EalgoLog@U2@@YAXXZ$0 100164e0 f   DNAStatPlugin.obj
 0001:000154e9       __ehhandler$??__EalgoLog@U2@@YAXXZ 100164e9 f   DNAStatPlugin.obj
 0001:00015510       __unwindfunclet$??__EcmdLog@U2@@YAXXZ$0 10016510 f   DNAStatPlugin.obj
 0001:00015519       __ehhandler$??__EcmdLog@U2@@YAXXZ 10016519 f   DNAStatPlugin.obj
 0001:00015540       __unwindfunclet$??__EcoreLog@U2@@YAXXZ$0 10016540 f   DNAStatPlugin.obj
 0001:00015549       __ehhandler$??__EcoreLog@U2@@YAXXZ 10016549 f   DNAStatPlugin.obj
 0001:00015570       __unwindfunclet$??__EioLog@U2@@YAXXZ$0 10016570 f   DNAStatPlugin.obj
 0001:00015579       __ehhandler$??__EioLog@U2@@YAXXZ 10016579 f   DNAStatPlugin.obj
 0001:000155a0       __unwindfunclet$??__EperfLog@U2@@YAXXZ$0 100165a0 f   DNAStatPlugin.obj
 0001:000155a9       __ehhandler$??__EperfLog@U2@@YAXXZ 100165a9 f   DNAStatPlugin.obj
 0001:000155d0       __unwindfunclet$??__EscriptLog@U2@@YAXXZ$0 100165d0 f   DNAStatPlugin.obj
 0001:000155d9       __ehhandler$??__EscriptLog@U2@@YAXXZ 100165d9 f   DNAStatPlugin.obj
 0001:00015600       __unwindfunclet$??__EtaskLog@U2@@YAXXZ$0 10016600 f   DNAStatPlugin.obj
 0001:00015609       __ehhandler$??__EtaskLog@U2@@YAXXZ 10016609 f   DNAStatPlugin.obj
 0001:00015630       __unwindfunclet$??__EuiLog@U2@@YAXXZ$0 10016630 f   DNAStatPlugin.obj
 0001:00015639       __ehhandler$??__EuiLog@U2@@YAXXZ 10016639 f   DNAStatPlugin.obj
 0001:00015660       __unwindfunclet$??__EuserActLog@U2@@YAXXZ$0 10016660 f   DNAStatPlugin.obj
 0001:00015669       __ehhandler$??__EuserActLog@U2@@YAXXZ 10016669 f   DNAStatPlugin.obj
 0001:00015690       __unwindfunclet$?buildMenu@DNAStatMSAEditorContext@U2@@MAEXPAVGObjectView@2@PAVQMenu@@@Z$0 10016690 f   DNAStatPlugin.obj
 0001:00015698       __unwindfunclet$?buildMenu@DNAStatMSAEditorContext@U2@@MAEXPAVGObjectView@2@PAVQMenu@@@Z$1 10016698 f   DNAStatPlugin.obj
 0001:000156a1       __unwindfunclet$?buildMenu@DNAStatMSAEditorContext@U2@@MAEXPAVGObjectView@2@PAVQMenu@@@Z$2 100166a1 f   DNAStatPlugin.obj
 0001:000156aa       __unwindfunclet$?buildMenu@DNAStatMSAEditorContext@U2@@MAEXPAVGObjectView@2@PAVQMenu@@@Z$3 100166aa f   DNAStatPlugin.obj
 0001:000156b3       __unwindfunclet$?buildMenu@DNAStatMSAEditorContext@U2@@MAEXPAVGObjectView@2@PAVQMenu@@@Z$4 100166b3 f   DNAStatPlugin.obj
 0001:000156bc       __unwindfunclet$?buildMenu@DNAStatMSAEditorContext@U2@@MAEXPAVGObjectView@2@PAVQMenu@@@Z$5 100166bc f   DNAStatPlugin.obj
 0001:000156c5       __unwindfunclet$?buildMenu@DNAStatMSAEditorContext@U2@@MAEXPAVGObjectView@2@PAVQMenu@@@Z$6 100166c5 f   DNAStatPlugin.obj
 0001:000156ce       __unwindfunclet$?buildMenu@DNAStatMSAEditorContext@U2@@MAEXPAVGObjectView@2@PAVQMenu@@@Z$7 100166ce f   DNAStatPlugin.obj
 0001:000156d7       __unwindfunclet$?buildMenu@DNAStatMSAEditorContext@U2@@MAEXPAVGObjectView@2@PAVQMenu@@@Z$8 100166d7 f   DNAStatPlugin.obj
 0001:000156df       __ehhandler$?buildMenu@DNAStatMSAEditorContext@U2@@MAEXPAVGObjectView@2@PAVQMenu@@@Z 100166df f   DNAStatPlugin.obj
 0001:00015700       __unwindfunclet$?buildMenu@DistanceMatrixMSAEditorContext@U2@@MAEXPAVGObjectView@2@PAVQMenu@@@Z$0 10016700 f   DNAStatPlugin.obj
 0001:00015708       __unwindfunclet$?buildMenu@DistanceMatrixMSAEditorContext@U2@@MAEXPAVGObjectView@2@PAVQMenu@@@Z$1 10016708 f   DNAStatPlugin.obj
 0001:00015711       __unwindfunclet$?buildMenu@DistanceMatrixMSAEditorContext@U2@@MAEXPAVGObjectView@2@PAVQMenu@@@Z$2 10016711 f   DNAStatPlugin.obj
 0001:0001571a       __unwindfunclet$?buildMenu@DistanceMatrixMSAEditorContext@U2@@MAEXPAVGObjectView@2@PAVQMenu@@@Z$3 1001671a f   DNAStatPlugin.obj
 0001:00015723       __unwindfunclet$?buildMenu@DistanceMatrixMSAEditorContext@U2@@MAEXPAVGObjectView@2@PAVQMenu@@@Z$4 10016723 f   DNAStatPlugin.obj
 0001:0001572c       __unwindfunclet$?buildMenu@DistanceMatrixMSAEditorContext@U2@@MAEXPAVGObjectView@2@PAVQMenu@@@Z$5 1001672c f   DNAStatPlugin.obj
 0001:00015735       __unwindfunclet$?buildMenu@DistanceMatrixMSAEditorContext@U2@@MAEXPAVGObjectView@2@PAVQMenu@@@Z$6 10016735 f   DNAStatPlugin.obj
 0001:0001573e       __unwindfunclet$?buildMenu@DistanceMatrixMSAEditorContext@U2@@MAEXPAVGObjectView@2@PAVQMenu@@@Z$7 1001673e f   DNAStatPlugin.obj
 0001:00015747       __unwindfunclet$?buildMenu@DistanceMatrixMSAEditorContext@U2@@MAEXPAVGObjectView@2@PAVQMenu@@@Z$8 10016747 f   DNAStatPlugin.obj
 0001:0001574f       __ehhandler$?buildMenu@DistanceMatrixMSAEditorContext@U2@@MAEXPAVGObjectView@2@PAVQMenu@@@Z 1001674f f   DNAStatPlugin.obj
 0001:00015770       __unwindfunclet$?initViewContext@DNAStatMSAEditorContext@U2@@MAEXPAVGObjectView@2@@Z$0 10016770 f   DNAStatPlugin.obj
 0001:0001577b       __unwindfunclet$?initViewContext@DNAStatMSAEditorContext@U2@@MAEXPAVGObjectView@2@@Z$1 1001677b f   DNAStatPlugin.obj
 0001:00015795       __unwindfunclet$?initViewContext@DNAStatMSAEditorContext@U2@@MAEXPAVGObjectView@2@@Z$2 10016795 f   DNAStatPlugin.obj
 0001:0001579e       __ehhandler$?initViewContext@DNAStatMSAEditorContext@U2@@MAEXPAVGObjectView@2@@Z 1001679e f   DNAStatPlugin.obj
 0001:000157c0       __unwindfunclet$?initViewContext@DistanceMatrixMSAEditorContext@U2@@MAEXPAVGObjectView@2@@Z$0 100167c0 f   DNAStatPlugin.obj
 0001:000157cb       __unwindfunclet$?initViewContext@DistanceMatrixMSAEditorContext@U2@@MAEXPAVGObjectView@2@@Z$1 100167cb f   DNAStatPlugin.obj
 0001:000157e5       __unwindfunclet$?initViewContext@DistanceMatrixMSAEditorContext@U2@@MAEXPAVGObjectView@2@@Z$2 100167e5 f   DNAStatPlugin.obj
 0001:000157ee       __ehhandler$?initViewContext@DistanceMatrixMSAEditorContext@U2@@MAEXPAVGObjectView@2@@Z 100167ee f   DNAStatPlugin.obj
 0001:00015810       __unwindfunclet$?sl_showDistanceMatrixDialog@DistanceMatrixMSAEditorContext@U2@@IAEXXZ$0 10016810 f   DNAStatPlugin.obj
 0001:0001581b       __unwindfunclet$?sl_showDistanceMatrixDialog@DistanceMatrixMSAEditorContext@U2@@IAEXXZ$1 1001681b f   DNAStatPlugin.obj
 0001:00015823       __unwindfunclet$?sl_showDistanceMatrixDialog@DistanceMatrixMSAEditorContext@U2@@IAEXXZ$4 10016823 f   DNAStatPlugin.obj
 0001:0001582b       __ehhandler$?sl_showDistanceMatrixDialog@DistanceMatrixMSAEditorContext@U2@@IAEXXZ 1001682b f   DNAStatPlugin.obj
 0001:00015850       __unwindfunclet$?sl_showMSAProfileDialog@DNAStatMSAEditorContext@U2@@IAEXXZ$0 10016850 f   DNAStatPlugin.obj
 0001:0001585b       __unwindfunclet$?sl_showMSAProfileDialog@DNAStatMSAEditorContext@U2@@IAEXXZ$1 1001685b f   DNAStatPlugin.obj
 0001:00015863       __unwindfunclet$?sl_showMSAProfileDialog@DNAStatMSAEditorContext@U2@@IAEXXZ$4 10016863 f   DNAStatPlugin.obj
 0001:0001586b       __ehhandler$?sl_showMSAProfileDialog@DNAStatMSAEditorContext@U2@@IAEXXZ 1001686b f   DNAStatPlugin.obj
 0001:00015890       __ehhandler$??0?$QList@UCharOccurResult@U2@@@@QAE@ABV0@@Z 10016890 f   DNAStatProfileTask.obj
 0001:000158b0       __unwindfunclet$??0DNAStatProfileTask@U2@@QAE@PAVADVSequenceObjectContext@1@@Z$0 100168b0 f   DNAStatProfileTask.obj
 0001:000158b9       __unwindfunclet$??0DNAStatProfileTask@U2@@QAE@PAVADVSequenceObjectContext@1@@Z$1 100168b9 f   DNAStatProfileTask.obj
 0001:000158c2       __unwindfunclet$??0DNAStatProfileTask@U2@@QAE@PAVADVSequenceObjectContext@1@@Z$2 100168c2 f   DNAStatProfileTask.obj
 0001:000158d1       __unwindfunclet$??0DNAStatProfileTask@U2@@QAE@PAVADVSequenceObjectContext@1@@Z$3 100168d1 f   DNAStatProfileTask.obj
 0001:000158e0       __unwindfunclet$??0DNAStatProfileTask@U2@@QAE@PAVADVSequenceObjectContext@1@@Z$4 100168e0 f   DNAStatProfileTask.obj
 0001:000158ef       __unwindfunclet$??0DNAStatProfileTask@U2@@QAE@PAVADVSequenceObjectContext@1@@Z$5 100168ef f   DNAStatProfileTask.obj
 0001:000158f8       __unwindfunclet$??0DNAStatProfileTask@U2@@QAE@PAVADVSequenceObjectContext@1@@Z$6 100168f8 f   DNAStatProfileTask.obj
 0001:00015903       __unwindfunclet$??0DNAStatProfileTask@U2@@QAE@PAVADVSequenceObjectContext@1@@Z$7 10016903 f   DNAStatProfileTask.obj
 0001:0001590c       __unwindfunclet$??0DNAStatProfileTask@U2@@QAE@PAVADVSequenceObjectContext@1@@Z$8 1001690c f   DNAStatProfileTask.obj
 0001:00015917       __unwindfunclet$??0DNAStatProfileTask@U2@@QAE@PAVADVSequenceObjectContext@1@@Z$9 10016917 f   DNAStatProfileTask.obj
 0001:00015920       __unwindfunclet$??0DNAStatProfileTask@U2@@QAE@PAVADVSequenceObjectContext@1@@Z$10 10016920 f   DNAStatProfileTask.obj
 0001:0001592b       __unwindfunclet$??0DNAStatProfileTask@U2@@QAE@PAVADVSequenceObjectContext@1@@Z$11 1001692b f   DNAStatProfileTask.obj
 0001:00015934       __ehhandler$??0DNAStatProfileTask@U2@@QAE@PAVADVSequenceObjectContext@1@@Z 10016934 f   DNAStatProfileTask.obj
 0001:00015950       __unwindfunclet$??1DNAStatProfileTask@U2@@UAE@XZ$0 10016950 f   DNAStatProfileTask.obj
 0001:00015959       __unwindfunclet$??1DNAStatProfileTask@U2@@UAE@XZ$1 10016959 f   DNAStatProfileTask.obj
 0001:00015968       __unwindfunclet$??1DNAStatProfileTask@U2@@UAE@XZ$2 10016968 f   DNAStatProfileTask.obj
 0001:00015977       __ehhandler$??1DNAStatProfileTask@U2@@UAE@XZ 10016977 f   DNAStatProfileTask.obj
 0001:000159a0       __unwindfunclet$??_GDNAStatProfileTask@U2@@UAEPAXI@Z$0 100169a0 f   DNAStatProfileTask.obj
 0001:000159a9       __unwindfunclet$??_GDNAStatProfileTask@U2@@UAEPAXI@Z$1 100169a9 f   DNAStatProfileTask.obj
 0001:000159b8       __unwindfunclet$??_GDNAStatProfileTask@U2@@UAEPAXI@Z$2 100169b8 f   DNAStatProfileTask.obj
 0001:000159c7       __ehhandler$??_GDNAStatProfileTask@U2@@UAEPAXI@Z 100169c7 f   DNAStatProfileTask.obj
 0001:000159f0       __unwindfunclet$??__EalgoLog@U2@@YAXXZ$0 100169f0 f   DNAStatProfileTask.obj
 0001:000159f9       __ehhandler$??__EalgoLog@U2@@YAXXZ 100169f9 f   DNAStatProfileTask.obj
 0001:00015a20       __unwindfunclet$??__EcmdLog@U2@@YAXXZ$0 10016a20 f   DNAStatProfileTask.obj
 0001:00015a29       __ehhandler$??__EcmdLog@U2@@YAXXZ 10016a29 f   DNAStatProfileTask.obj
 0001:00015a50       __unwindfunclet$??__EcoreLog@U2@@YAXXZ$0 10016a50 f   DNAStatProfileTask.obj
 0001:00015a59       __ehhandler$??__EcoreLog@U2@@YAXXZ 10016a59 f   DNAStatProfileTask.obj
 0001:00015a80       __unwindfunclet$??__EioLog@U2@@YAXXZ$0 10016a80 f   DNAStatProfileTask.obj
 0001:00015a89       __ehhandler$??__EioLog@U2@@YAXXZ 10016a89 f   DNAStatProfileTask.obj
 0001:00015ab0       __unwindfunclet$??__EperfLog@U2@@YAXXZ$0 10016ab0 f   DNAStatProfileTask.obj
 0001:00015ab9       __ehhandler$??__EperfLog@U2@@YAXXZ 10016ab9 f   DNAStatProfileTask.obj
 0001:00015ae0       __unwindfunclet$??__EscriptLog@U2@@YAXXZ$0 10016ae0 f   DNAStatProfileTask.obj
 0001:00015ae9       __ehhandler$??__EscriptLog@U2@@YAXXZ 10016ae9 f   DNAStatProfileTask.obj
 0001:00015b10       __unwindfunclet$??__EtaskLog@U2@@YAXXZ$0 10016b10 f   DNAStatProfileTask.obj
 0001:00015b19       __ehhandler$??__EtaskLog@U2@@YAXXZ 10016b19 f   DNAStatProfileTask.obj
 0001:00015b40       __unwindfunclet$??__EuiLog@U2@@YAXXZ$0 10016b40 f   DNAStatProfileTask.obj
 0001:00015b49       __ehhandler$??__EuiLog@U2@@YAXXZ 10016b49 f   DNAStatProfileTask.obj
 0001:00015b70       __unwindfunclet$??__EuserActLog@U2@@YAXXZ$0 10016b70 f   DNAStatProfileTask.obj
 0001:00015b79       __ehhandler$??__EuserActLog@U2@@YAXXZ 10016b79 f   DNAStatProfileTask.obj
 0001:00015ba0       __unwindfunclet$?createNode@?$QMapData@VQByteArray@@_J@@QAEPAU?$QMapNode@VQByteArray@@_J@@ABVQByteArray@@AB_JPAU2@_N@Z$4 10016ba0 f   DNAStatProfileTask.obj
 0001:00015bb4       __ehhandler$?createNode@?$QMapData@VQByteArray@@_J@@QAEPAU?$QMapNode@VQByteArray@@_J@@ABVQByteArray@@AB_JPAU2@_N@Z 10016bb4 f   DNAStatProfileTask.obj
 0001:00015bd0       __unwindfunclet$?formCharResultString@DNAStatProfileTask@U2@@ABE?AVQString@@XZ$0 10016bd0 f   DNAStatProfileTask.obj
 0001:00015bd8       __unwindfunclet$?formCharResultString@DNAStatProfileTask@U2@@ABE?AVQString@@XZ$1 10016bd8 f   DNAStatProfileTask.obj
 0001:00015bf2       __unwindfunclet$?formCharResultString@DNAStatProfileTask@U2@@ABE?AVQString@@XZ$2 10016bf2 f   DNAStatProfileTask.obj
 0001:00015bfb       __unwindfunclet$?formCharResultString@DNAStatProfileTask@U2@@ABE?AVQString@@XZ$3 10016bfb f   DNAStatProfileTask.obj
 0001:00015c04       __unwindfunclet$?formCharResultString@DNAStatProfileTask@U2@@ABE?AVQString@@XZ$4 10016c04 f   DNAStatProfileTask.obj
 0001:00015c0d       __unwindfunclet$?formCharResultString@DNAStatProfileTask@U2@@ABE?AVQString@@XZ$5 10016c0d f   DNAStatProfileTask.obj
 0001:00015c16       __unwindfunclet$?formCharResultString@DNAStatProfileTask@U2@@ABE?AVQString@@XZ$6 10016c16 f   DNAStatProfileTask.obj
 0001:00015c1f       __unwindfunclet$?formCharResultString@DNAStatProfileTask@U2@@ABE?AVQString@@XZ$7 10016c1f f   DNAStatProfileTask.obj
 0001:00015c28       __unwindfunclet$?formCharResultString@DNAStatProfileTask@U2@@ABE?AVQString@@XZ$8 10016c28 f   DNAStatProfileTask.obj
 0001:00015c30       __unwindfunclet$?formCharResultString@DNAStatProfileTask@U2@@ABE?AVQString@@XZ$9 10016c30 f   DNAStatProfileTask.obj
 0001:00015c39       __unwindfunclet$?formCharResultString@DNAStatProfileTask@U2@@ABE?AVQString@@XZ$10 10016c39 f   DNAStatProfileTask.obj
 0001:00015c42       __unwindfunclet$?formCharResultString@DNAStatProfileTask@U2@@ABE?AVQString@@XZ$11 10016c42 f   DNAStatProfileTask.obj
 0001:00015c4b       __unwindfunclet$?formCharResultString@DNAStatProfileTask@U2@@ABE?AVQString@@XZ$12 10016c4b f   DNAStatProfileTask.obj
 0001:00015c54       __unwindfunclet$?formCharResultString@DNAStatProfileTask@U2@@ABE?AVQString@@XZ$13 10016c54 f   DNAStatProfileTask.obj
 0001:00015c5d       __unwindfunclet$?formCharResultString@DNAStatProfileTask@U2@@ABE?AVQString@@XZ$14 10016c5d f   DNAStatProfileTask.obj
 0001:00015c66       __ehhandler$?formCharResultString@DNAStatProfileTask@U2@@ABE?AVQString@@XZ 10016c66 f   DNAStatProfileTask.obj
 0001:00015c90       __unwindfunclet$?formDinucResultString@DNAStatProfileTask@U2@@ABE?AVQString@@XZ$0 10016c90 f   DNAStatProfileTask.obj
 0001:00015caa       __unwindfunclet$?formDinucResultString@DNAStatProfileTask@U2@@ABE?AVQString@@XZ$1 10016caa f   DNAStatProfileTask.obj
 0001:00015cb2       __unwindfunclet$?formDinucResultString@DNAStatProfileTask@U2@@ABE?AVQString@@XZ$2 10016cb2 f   DNAStatProfileTask.obj
 0001:00015cbb       __unwindfunclet$?formDinucResultString@DNAStatProfileTask@U2@@ABE?AVQString@@XZ$3 10016cbb f   DNAStatProfileTask.obj
 0001:00015cc4       __unwindfunclet$?formDinucResultString@DNAStatProfileTask@U2@@ABE?AVQString@@XZ$4 10016cc4 f   DNAStatProfileTask.obj
 0001:00015ccd       __unwindfunclet$?formDinucResultString@DNAStatProfileTask@U2@@ABE?AVQString@@XZ$5 10016ccd f   DNAStatProfileTask.obj
 0001:00015cd6       __unwindfunclet$?formDinucResultString@DNAStatProfileTask@U2@@ABE?AVQString@@XZ$6 10016cd6 f   DNAStatProfileTask.obj
 0001:00015cdf       __unwindfunclet$?formDinucResultString@DNAStatProfileTask@U2@@ABE?AVQString@@XZ$7 10016cdf f   DNAStatProfileTask.obj
 0001:00015ce8       __unwindfunclet$?formDinucResultString@DNAStatProfileTask@U2@@ABE?AVQString@@XZ$8 10016ce8 f   DNAStatProfileTask.obj
 0001:00015cf1       __unwindfunclet$?formDinucResultString@DNAStatProfileTask@U2@@ABE?AVQString@@XZ$9 10016cf1 f   DNAStatProfileTask.obj
 0001:00015cfa       __unwindfunclet$?formDinucResultString@DNAStatProfileTask@U2@@ABE?AVQString@@XZ$10 10016cfa f   DNAStatProfileTask.obj
 0001:00015d03       __unwindfunclet$?formDinucResultString@DNAStatProfileTask@U2@@ABE?AVQString@@XZ$11 10016d03 f   DNAStatProfileTask.obj
 0001:00015d0c       __unwindfunclet$?formDinucResultString@DNAStatProfileTask@U2@@ABE?AVQString@@XZ$12 10016d0c f   DNAStatProfileTask.obj
 0001:00015d15       __unwindfunclet$?formDinucResultString@DNAStatProfileTask@U2@@ABE?AVQString@@XZ$13 10016d15 f   DNAStatProfileTask.obj
 0001:00015d1e       __unwindfunclet$?formDinucResultString@DNAStatProfileTask@U2@@ABE?AVQString@@XZ$14 10016d1e f   DNAStatProfileTask.obj
 0001:00015d27       __unwindfunclet$?formDinucResultString@DNAStatProfileTask@U2@@ABE?AVQString@@XZ$15 10016d27 f   DNAStatProfileTask.obj
 0001:00015d30       __unwindfunclet$?formDinucResultString@DNAStatProfileTask@U2@@ABE?AVQString@@XZ$16 10016d30 f   DNAStatProfileTask.obj
 0001:00015d39       __ehhandler$?formDinucResultString@DNAStatProfileTask@U2@@ABE?AVQString@@XZ 10016d39 f   DNAStatProfileTask.obj
 0001:00015d60       __unwindfunclet$?formStatResultString@DNAStatProfileTask@U2@@ABE?AVQString@@XZ$0 10016d60 f   DNAStatProfileTask.obj
 0001:00015d69       __unwindfunclet$?formStatResultString@DNAStatProfileTask@U2@@ABE?AVQString@@XZ$1 10016d69 f   DNAStatProfileTask.obj
 0001:00015d72       __unwindfunclet$?formStatResultString@DNAStatProfileTask@U2@@ABE?AVQString@@XZ$2 10016d72 f   DNAStatProfileTask.obj
 0001:00015d8c       __unwindfunclet$?formStatResultString@DNAStatProfileTask@U2@@ABE?AVQString@@XZ$3 10016d8c f   DNAStatProfileTask.obj
 0001:00015d95       __unwindfunclet$?formStatResultString@DNAStatProfileTask@U2@@ABE?AVQString@@XZ$4 10016d95 f   DNAStatProfileTask.obj
 0001:00015d9e       __unwindfunclet$?formStatResultString@DNAStatProfileTask@U2@@ABE?AVQString@@XZ$5 10016d9e f   DNAStatProfileTask.obj
 0001:00015da7       __unwindfunclet$?formStatResultString@DNAStatProfileTask@U2@@ABE?AVQString@@XZ$6 10016da7 f   DNAStatProfileTask.obj
 0001:00015db0       __unwindfunclet$?formStatResultString@DNAStatProfileTask@U2@@ABE?AVQString@@XZ$7 10016db0 f   DNAStatProfileTask.obj
 0001:00015db9       __unwindfunclet$?formStatResultString@DNAStatProfileTask@U2@@ABE?AVQString@@XZ$8 10016db9 f   DNAStatProfileTask.obj
 0001:00015dc2       __unwindfunclet$?formStatResultString@DNAStatProfileTask@U2@@ABE?AVQString@@XZ$9 10016dc2 f   DNAStatProfileTask.obj
 0001:00015dcb       __unwindfunclet$?formStatResultString@DNAStatProfileTask@U2@@ABE?AVQString@@XZ$10 10016dcb f   DNAStatProfileTask.obj
 0001:00015dd4       __unwindfunclet$?formStatResultString@DNAStatProfileTask@U2@@ABE?AVQString@@XZ$11 10016dd4 f   DNAStatProfileTask.obj
 0001:00015ddd       __unwindfunclet$?formStatResultString@DNAStatProfileTask@U2@@ABE?AVQString@@XZ$12 10016ddd f   DNAStatProfileTask.obj
 0001:00015de6       __unwindfunclet$?formStatResultString@DNAStatProfileTask@U2@@ABE?AVQString@@XZ$13 10016de6 f   DNAStatProfileTask.obj
 0001:00015def       __unwindfunclet$?formStatResultString@DNAStatProfileTask@U2@@ABE?AVQString@@XZ$14 10016def f   DNAStatProfileTask.obj
 0001:00015df8       __unwindfunclet$?formStatResultString@DNAStatProfileTask@U2@@ABE?AVQString@@XZ$15 10016df8 f   DNAStatProfileTask.obj
 0001:00015e01       __unwindfunclet$?formStatResultString@DNAStatProfileTask@U2@@ABE?AVQString@@XZ$16 10016e01 f   DNAStatProfileTask.obj
 0001:00015e0a       __unwindfunclet$?formStatResultString@DNAStatProfileTask@U2@@ABE?AVQString@@XZ$17 10016e0a f   DNAStatProfileTask.obj
 0001:00015e13       __unwindfunclet$?formStatResultString@DNAStatProfileTask@U2@@ABE?AVQString@@XZ$18 10016e13 f   DNAStatProfileTask.obj
 0001:00015e1c       __unwindfunclet$?formStatResultString@DNAStatProfileTask@U2@@ABE?AVQString@@XZ$19 10016e1c f   DNAStatProfileTask.obj
 0001:00015e25       __unwindfunclet$?formStatResultString@DNAStatProfileTask@U2@@ABE?AVQString@@XZ$20 10016e25 f   DNAStatProfileTask.obj
 0001:00015e2e       __unwindfunclet$?formStatResultString@DNAStatProfileTask@U2@@ABE?AVQString@@XZ$21 10016e2e f   DNAStatProfileTask.obj
 0001:00015e37       __unwindfunclet$?formStatResultString@DNAStatProfileTask@U2@@ABE?AVQString@@XZ$22 10016e37 f   DNAStatProfileTask.obj
 0001:00015e40       __unwindfunclet$?formStatResultString@DNAStatProfileTask@U2@@ABE?AVQString@@XZ$23 10016e40 f   DNAStatProfileTask.obj
 0001:00015e49       __unwindfunclet$?formStatResultString@DNAStatProfileTask@U2@@ABE?AVQString@@XZ$24 10016e49 f   DNAStatProfileTask.obj
 0001:00015e52       __unwindfunclet$?formStatResultString@DNAStatProfileTask@U2@@ABE?AVQString@@XZ$25 10016e52 f   DNAStatProfileTask.obj
 0001:00015e5b       __unwindfunclet$?formStatResultString@DNAStatProfileTask@U2@@ABE?AVQString@@XZ$26 10016e5b f   DNAStatProfileTask.obj
 0001:00015e64       __unwindfunclet$?formStatResultString@DNAStatProfileTask@U2@@ABE?AVQString@@XZ$27 10016e64 f   DNAStatProfileTask.obj
 0001:00015e6d       __unwindfunclet$?formStatResultString@DNAStatProfileTask@U2@@ABE?AVQString@@XZ$28 10016e6d f   DNAStatProfileTask.obj
 0001:00015e76       __unwindfunclet$?formStatResultString@DNAStatProfileTask@U2@@ABE?AVQString@@XZ$29 10016e76 f   DNAStatProfileTask.obj
 0001:00015e7f       __unwindfunclet$?formStatResultString@DNAStatProfileTask@U2@@ABE?AVQString@@XZ$30 10016e7f f   DNAStatProfileTask.obj
 0001:00015e88       __unwindfunclet$?formStatResultString@DNAStatProfileTask@U2@@ABE?AVQString@@XZ$31 10016e88 f   DNAStatProfileTask.obj
 0001:00015e91       __unwindfunclet$?formStatResultString@DNAStatProfileTask@U2@@ABE?AVQString@@XZ$32 10016e91 f   DNAStatProfileTask.obj
 0001:00015e9a       __unwindfunclet$?formStatResultString@DNAStatProfileTask@U2@@ABE?AVQString@@XZ$33 10016e9a f   DNAStatProfileTask.obj
 0001:00015ea3       __unwindfunclet$?formStatResultString@DNAStatProfileTask@U2@@ABE?AVQString@@XZ$34 10016ea3 f   DNAStatProfileTask.obj
 0001:00015eac       __unwindfunclet$?formStatResultString@DNAStatProfileTask@U2@@ABE?AVQString@@XZ$35 10016eac f   DNAStatProfileTask.obj
 0001:00015eb5       __unwindfunclet$?formStatResultString@DNAStatProfileTask@U2@@ABE?AVQString@@XZ$36 10016eb5 f   DNAStatProfileTask.obj
 0001:00015ebe       __unwindfunclet$?formStatResultString@DNAStatProfileTask@U2@@ABE?AVQString@@XZ$37 10016ebe f   DNAStatProfileTask.obj
 0001:00015ec7       __unwindfunclet$?formStatResultString@DNAStatProfileTask@U2@@ABE?AVQString@@XZ$38 10016ec7 f   DNAStatProfileTask.obj
 0001:00015ed0       __unwindfunclet$?formStatResultString@DNAStatProfileTask@U2@@ABE?AVQString@@XZ$39 10016ed0 f   DNAStatProfileTask.obj
 0001:00015ed9       __unwindfunclet$?formStatResultString@DNAStatProfileTask@U2@@ABE?AVQString@@XZ$40 10016ed9 f   DNAStatProfileTask.obj
 0001:00015ee2       __unwindfunclet$?formStatResultString@DNAStatProfileTask@U2@@ABE?AVQString@@XZ$41 10016ee2 f   DNAStatProfileTask.obj
 0001:00015eeb       __unwindfunclet$?formStatResultString@DNAStatProfileTask@U2@@ABE?AVQString@@XZ$42 10016eeb f   DNAStatProfileTask.obj
 0001:00015ef4       __unwindfunclet$?formStatResultString@DNAStatProfileTask@U2@@ABE?AVQString@@XZ$43 10016ef4 f   DNAStatProfileTask.obj
 0001:00015efd       __unwindfunclet$?formStatResultString@DNAStatProfileTask@U2@@ABE?AVQString@@XZ$44 10016efd f   DNAStatProfileTask.obj
 0001:00015f06       __unwindfunclet$?formStatResultString@DNAStatProfileTask@U2@@ABE?AVQString@@XZ$45 10016f06 f   DNAStatProfileTask.obj
 0001:00015f0f       __unwindfunclet$?formStatResultString@DNAStatProfileTask@U2@@ABE?AVQString@@XZ$46 10016f0f f   DNAStatProfileTask.obj
 0001:00015f18       __unwindfunclet$?formStatResultString@DNAStatProfileTask@U2@@ABE?AVQString@@XZ$47 10016f18 f   DNAStatProfileTask.obj
 0001:00015f21       __unwindfunclet$?formStatResultString@DNAStatProfileTask@U2@@ABE?AVQString@@XZ$48 10016f21 f   DNAStatProfileTask.obj
 0001:00015f2a       __unwindfunclet$?formStatResultString@DNAStatProfileTask@U2@@ABE?AVQString@@XZ$49 10016f2a f   DNAStatProfileTask.obj
 0001:00015f33       __unwindfunclet$?formStatResultString@DNAStatProfileTask@U2@@ABE?AVQString@@XZ$50 10016f33 f   DNAStatProfileTask.obj
 0001:00015f3c       __unwindfunclet$?formStatResultString@DNAStatProfileTask@U2@@ABE?AVQString@@XZ$51 10016f3c f   DNAStatProfileTask.obj
 0001:00015f45       __unwindfunclet$?formStatResultString@DNAStatProfileTask@U2@@ABE?AVQString@@XZ$52 10016f45 f   DNAStatProfileTask.obj
 0001:00015f4e       __unwindfunclet$?formStatResultString@DNAStatProfileTask@U2@@ABE?AVQString@@XZ$53 10016f4e f   DNAStatProfileTask.obj
 0001:00015f57       __unwindfunclet$?formStatResultString@DNAStatProfileTask@U2@@ABE?AVQString@@XZ$54 10016f57 f   DNAStatProfileTask.obj
 0001:00015f60       __unwindfunclet$?formStatResultString@DNAStatProfileTask@U2@@ABE?AVQString@@XZ$55 10016f60 f   DNAStatProfileTask.obj
 0001:00015f69       __unwindfunclet$?formStatResultString@DNAStatProfileTask@U2@@ABE?AVQString@@XZ$56 10016f69 f   DNAStatProfileTask.obj
 0001:00015f72       __unwindfunclet$?formStatResultString@DNAStatProfileTask@U2@@ABE?AVQString@@XZ$57 10016f72 f   DNAStatProfileTask.obj
 0001:00015f7b       __unwindfunclet$?formStatResultString@DNAStatProfileTask@U2@@ABE?AVQString@@XZ$58 10016f7b f   DNAStatProfileTask.obj
 0001:00015f84       __unwindfunclet$?formStatResultString@DNAStatProfileTask@U2@@ABE?AVQString@@XZ$59 10016f84 f   DNAStatProfileTask.obj
 0001:00015f8d       __unwindfunclet$?formStatResultString@DNAStatProfileTask@U2@@ABE?AVQString@@XZ$60 10016f8d f   DNAStatProfileTask.obj
 0001:00015f96       __unwindfunclet$?formStatResultString@DNAStatProfileTask@U2@@ABE?AVQString@@XZ$61 10016f96 f   DNAStatProfileTask.obj
 0001:00015f9f       __unwindfunclet$?formStatResultString@DNAStatProfileTask@U2@@ABE?AVQString@@XZ$62 10016f9f f   DNAStatProfileTask.obj
 0001:00015fa8       __ehhandler$?formStatResultString@DNAStatProfileTask@U2@@ABE?AVQString@@XZ 10016fa8 f   DNAStatProfileTask.obj
 0001:00015fd0       __unwindfunclet$?getResult@DNAStatProfileTask@U2@@QBE?AVQString@@XZ$0 10016fd0 f   DNAStatProfileTask.obj
 0001:00015fea       __ehhandler$?getResult@DNAStatProfileTask@U2@@QBE?AVQString@@XZ 10016fea f   DNAStatProfileTask.obj
 0001:00016010       __ehhandler$?node_copy@?$QList@UCharOccurResult@U2@@@@AAEXPAUNode@1@00@Z 10017010 f   DNAStatProfileTask.obj
 0001:00016030       __unwindfunclet$?onSubTaskFinished@DNAStatProfileTask@U2@@UAE?AV?$QList@PAVTask@U2@@@@PAVTask@2@@Z$0 10017030 f   DNAStatProfileTask.obj
 0001:00016049       __unwindfunclet$?onSubTaskFinished@DNAStatProfileTask@U2@@UAE?AV?$QList@PAVTask@U2@@@@PAVTask@2@@Z$1 10017049 f   DNAStatProfileTask.obj
 0001:00016052       __unwindfunclet$?onSubTaskFinished@DNAStatProfileTask@U2@@UAE?AV?$QList@PAVTask@U2@@@@PAVTask@2@@Z$2 10017052 f   DNAStatProfileTask.obj
 0001:0001605b       __unwindfunclet$?onSubTaskFinished@DNAStatProfileTask@U2@@UAE?AV?$QList@PAVTask@U2@@@@PAVTask@2@@Z$3 1001705b f   DNAStatProfileTask.obj
 0001:00016064       __ehhandler$?onSubTaskFinished@DNAStatProfileTask@U2@@UAE?AV?$QList@PAVTask@U2@@@@PAVTask@2@@Z 10017064 f   DNAStatProfileTask.obj
 0001:00016080       __unwindfunclet$??0?$QForeachContainer@V?$QVector@VU2Region@U2@@@@@@QAE@ABV?$QVector@VU2Region@U2@@@@@Z$0 10017080 f   DistanceMatrixMSAProfileDialog.obj
 0001:00016088       __ehhandler$??0?$QForeachContainer@V?$QVector@VU2Region@U2@@@@@@QAE@ABV?$QVector@VU2Region@U2@@@@@Z 10017088 f   DistanceMatrixMSAProfileDialog.obj
 0001:000160b0       __ehhandler$??0?$QList@PAVMSADistanceAlgorithmFactory@U2@@@@QAE@ABV0@@Z 100170b0 f   DistanceMatrixMSAProfileDialog.obj
 0001:000160d0       __unwindfunclet$??0DistanceMatrixMSAProfileDialog@U2@@QAE@PAVQWidget@@PAVMSAEditor@1@@Z$0 100170d0 f   DistanceMatrixMSAProfileDialog.obj
 0001:000160d9       __unwindfunclet$??0DistanceMatrixMSAProfileDialog@U2@@QAE@PAVQWidget@@PAVMSAEditor@1@@Z$1 100170d9 f   DistanceMatrixMSAProfileDialog.obj
 0001:000160e4       __unwindfunclet$??0DistanceMatrixMSAProfileDialog@U2@@QAE@PAVQWidget@@PAVMSAEditor@1@@Z$2 100170e4 f   DistanceMatrixMSAProfileDialog.obj
 0001:000160fe       __unwindfunclet$??0DistanceMatrixMSAProfileDialog@U2@@QAE@PAVQWidget@@PAVMSAEditor@1@@Z$3 100170fe f   DistanceMatrixMSAProfileDialog.obj
 0001:00016107       __unwindfunclet$??0DistanceMatrixMSAProfileDialog@U2@@QAE@PAVQWidget@@PAVMSAEditor@1@@Z$4 10017107 f   DistanceMatrixMSAProfileDialog.obj
 0001:00016110       __unwindfunclet$??0DistanceMatrixMSAProfileDialog@U2@@QAE@PAVQWidget@@PAVMSAEditor@1@@Z$5 10017110 f   DistanceMatrixMSAProfileDialog.obj
 0001:00016118       __unwindfunclet$??0DistanceMatrixMSAProfileDialog@U2@@QAE@PAVQWidget@@PAVMSAEditor@1@@Z$6 10017118 f   DistanceMatrixMSAProfileDialog.obj
 0001:00016120       __unwindfunclet$??0DistanceMatrixMSAProfileDialog@U2@@QAE@PAVQWidget@@PAVMSAEditor@1@@Z$7 10017120 f   DistanceMatrixMSAProfileDialog.obj
 0001:00016129       __unwindfunclet$??0DistanceMatrixMSAProfileDialog@U2@@QAE@PAVQWidget@@PAVMSAEditor@1@@Z$8 10017129 f   DistanceMatrixMSAProfileDialog.obj
 0001:00016132       __unwindfunclet$??0DistanceMatrixMSAProfileDialog@U2@@QAE@PAVQWidget@@PAVMSAEditor@1@@Z$9 10017132 f   DistanceMatrixMSAProfileDialog.obj
 0001:0001613b       __unwindfunclet$??0DistanceMatrixMSAProfileDialog@U2@@QAE@PAVQWidget@@PAVMSAEditor@1@@Z$13 1001713b f   DistanceMatrixMSAProfileDialog.obj
 0001:00016144       __unwindfunclet$??0DistanceMatrixMSAProfileDialog@U2@@QAE@PAVQWidget@@PAVMSAEditor@1@@Z$10 10017144 f   DistanceMatrixMSAProfileDialog.obj
 0001:0001614c       __unwindfunclet$??0DistanceMatrixMSAProfileDialog@U2@@QAE@PAVQWidget@@PAVMSAEditor@1@@Z$11 1001714c f   DistanceMatrixMSAProfileDialog.obj
 0001:00016155       __ehhandler$??0DistanceMatrixMSAProfileDialog@U2@@QAE@PAVQWidget@@PAVMSAEditor@1@@Z 10017155 f   DistanceMatrixMSAProfileDialog.obj
 0001:00016170       __unwindfunclet$??0DistanceMatrixMSAProfileTask@U2@@QAE@ABVDistanceMatrixMSAProfileTaskSettings@1@@Z$0 10017170 f   DistanceMatrixMSAProfileDialog.obj
 0001:00016179       __unwindfunclet$??0DistanceMatrixMSAProfileTask@U2@@QAE@ABVDistanceMatrixMSAProfileTaskSettings@1@@Z$1 10017179 f   DistanceMatrixMSAProfileDialog.obj
 0001:00016182       __unwindfunclet$??0DistanceMatrixMSAProfileTask@U2@@QAE@ABVDistanceMatrixMSAProfileTaskSettings@1@@Z$2 10017182 f   DistanceMatrixMSAProfileDialog.obj
 0001:00016190       __unwindfunclet$??0DistanceMatrixMSAProfileTask@U2@@QAE@ABVDistanceMatrixMSAProfileTaskSettings@1@@Z$3 10017190 f   DistanceMatrixMSAProfileDialog.obj
 0001:0001619f       __ehhandler$??0DistanceMatrixMSAProfileTask@U2@@QAE@ABVDistanceMatrixMSAProfileTaskSettings@1@@Z 1001719f f   DistanceMatrixMSAProfileDialog.obj
 0001:000161c0       __unwindfunclet$??0DistanceMatrixMSAProfileTaskSettings@U2@@QAE@ABV01@@Z$0 100171c0 f   DistanceMatrixMSAProfileDialog.obj
 0001:000161c9       __unwindfunclet$??0DistanceMatrixMSAProfileTaskSettings@U2@@QAE@ABV01@@Z$1 100171c9 f   DistanceMatrixMSAProfileDialog.obj
 0001:000161d5       __unwindfunclet$??0DistanceMatrixMSAProfileTaskSettings@U2@@QAE@ABV01@@Z$2 100171d5 f   DistanceMatrixMSAProfileDialog.obj
 0001:000161e1       __unwindfunclet$??0DistanceMatrixMSAProfileTaskSettings@U2@@QAE@ABV01@@Z$3 100171e1 f   DistanceMatrixMSAProfileDialog.obj
 0001:000161ed       __ehhandler$??0DistanceMatrixMSAProfileTaskSettings@U2@@QAE@ABV01@@Z 100171ed f   DistanceMatrixMSAProfileDialog.obj
 0001:00016210       __unwindfunclet$??0DistanceMatrixMSAProfileTaskSettings@U2@@QAE@XZ$0 10017210 f   DistanceMatrixMSAProfileDialog.obj
 0001:00016219       __unwindfunclet$??0DistanceMatrixMSAProfileTaskSettings@U2@@QAE@XZ$1 10017219 f   DistanceMatrixMSAProfileDialog.obj
 0001:00016225       __unwindfunclet$??0DistanceMatrixMSAProfileTaskSettings@U2@@QAE@XZ$2 10017225 f   DistanceMatrixMSAProfileDialog.obj
 0001:00016231       __unwindfunclet$??0DistanceMatrixMSAProfileTaskSettings@U2@@QAE@XZ$3 10017231 f   DistanceMatrixMSAProfileDialog.obj
 0001:00016239       __unwindfunclet$??0DistanceMatrixMSAProfileTaskSettings@U2@@QAE@XZ$4 10017239 f   DistanceMatrixMSAProfileDialog.obj
 0001:00016242       __unwindfunclet$??0DistanceMatrixMSAProfileTaskSettings@U2@@QAE@XZ$5 10017242 f   DistanceMatrixMSAProfileDialog.obj
 0001:0001624e       __ehhandler$??0DistanceMatrixMSAProfileTaskSettings@U2@@QAE@XZ 1001724e f   DistanceMatrixMSAProfileDialog.obj
 0001:00016270       __unwindfunclet$??1DistanceMatrixMSAProfileTask@U2@@UAE@XZ$0 10017270 f   DistanceMatrixMSAProfileDialog.obj
 0001:00016279       __unwindfunclet$??1DistanceMatrixMSAProfileTask@U2@@UAE@XZ$1 10017279 f   DistanceMatrixMSAProfileDialog.obj
 0001:00016287       __unwindfunclet$??1DistanceMatrixMSAProfileTask@U2@@UAE@XZ$3 10017287 f   DistanceMatrixMSAProfileDialog.obj
 0001:00016290       __unwindfunclet$??1DistanceMatrixMSAProfileTask@U2@@UAE@XZ$4 10017290 f   DistanceMatrixMSAProfileDialog.obj
 0001:0001629c       __unwindfunclet$??1DistanceMatrixMSAProfileTask@U2@@UAE@XZ$5 1001729c f   DistanceMatrixMSAProfileDialog.obj
 0001:000162a8       __unwindfunclet$??1DistanceMatrixMSAProfileTask@U2@@UAE@XZ$6 100172a8 f   DistanceMatrixMSAProfileDialog.obj
 0001:000162b4       __ehhandler$??1DistanceMatrixMSAProfileTask@U2@@UAE@XZ 100172b4 f   DistanceMatrixMSAProfileDialog.obj
 0001:000162d0       __unwindfunclet$??1DistanceMatrixMSAProfileTaskSettings@U2@@QAE@XZ$0 100172d0 f   DistanceMatrixMSAProfileDialog.obj
 0001:000162d9       __unwindfunclet$??1DistanceMatrixMSAProfileTaskSettings@U2@@QAE@XZ$1 100172d9 f   DistanceMatrixMSAProfileDialog.obj
 0001:000162e5       __unwindfunclet$??1DistanceMatrixMSAProfileTaskSettings@U2@@QAE@XZ$2 100172e5 f   DistanceMatrixMSAProfileDialog.obj
 0001:000162f1       __unwindfunclet$??1DistanceMatrixMSAProfileTaskSettings@U2@@QAE@XZ$3 100172f1 f   DistanceMatrixMSAProfileDialog.obj
 0001:000162fd       __ehhandler$??1DistanceMatrixMSAProfileTaskSettings@U2@@QAE@XZ 100172fd f   DistanceMatrixMSAProfileDialog.obj
 0001:00016320       __unwindfunclet$??__EalgoLog@U2@@YAXXZ$0 10017320 f   DistanceMatrixMSAProfileDialog.obj
 0001:00016329       __ehhandler$??__EalgoLog@U2@@YAXXZ 10017329 f   DistanceMatrixMSAProfileDialog.obj
 0001:00016350       __unwindfunclet$??__EcmdLog@U2@@YAXXZ$0 10017350 f   DistanceMatrixMSAProfileDialog.obj
 0001:00016359       __ehhandler$??__EcmdLog@U2@@YAXXZ 10017359 f   DistanceMatrixMSAProfileDialog.obj
 0001:00016380       __unwindfunclet$??__EcoreLog@U2@@YAXXZ$0 10017380 f   DistanceMatrixMSAProfileDialog.obj
 0001:00016389       __ehhandler$??__EcoreLog@U2@@YAXXZ 10017389 f   DistanceMatrixMSAProfileDialog.obj
 0001:000163b0       __unwindfunclet$??__EioLog@U2@@YAXXZ$0 100173b0 f   DistanceMatrixMSAProfileDialog.obj
 0001:000163b9       __ehhandler$??__EioLog@U2@@YAXXZ 100173b9 f   DistanceMatrixMSAProfileDialog.obj
 0001:000163e0       __unwindfunclet$??__EperfLog@U2@@YAXXZ$0 100173e0 f   DistanceMatrixMSAProfileDialog.obj
 0001:000163e9       __ehhandler$??__EperfLog@U2@@YAXXZ 100173e9 f   DistanceMatrixMSAProfileDialog.obj
 0001:00016410       __unwindfunclet$??__EscriptLog@U2@@YAXXZ$0 10017410 f   DistanceMatrixMSAProfileDialog.obj
 0001:00016419       __ehhandler$??__EscriptLog@U2@@YAXXZ 10017419 f   DistanceMatrixMSAProfileDialog.obj
 0001:00016440       __unwindfunclet$??__EtaskLog@U2@@YAXXZ$0 10017440 f   DistanceMatrixMSAProfileDialog.obj
 0001:00016449       __ehhandler$??__EtaskLog@U2@@YAXXZ 10017449 f   DistanceMatrixMSAProfileDialog.obj
 0001:00016470       __unwindfunclet$??__EuiLog@U2@@YAXXZ$0 10017470 f   DistanceMatrixMSAProfileDialog.obj
 0001:00016479       __ehhandler$??__EuiLog@U2@@YAXXZ 10017479 f   DistanceMatrixMSAProfileDialog.obj
 0001:000164a0       __unwindfunclet$??__EuserActLog@U2@@YAXXZ$0 100174a0 f   DistanceMatrixMSAProfileDialog.obj
 0001:000164a9       __ehhandler$??__EuserActLog@U2@@YAXXZ 100174a9 f   DistanceMatrixMSAProfileDialog.obj
 0001:000164d0       __unwindfunclet$?accept@DistanceMatrixMSAProfileDialog@U2@@UAEXXZ$0 100174d0 f   DistanceMatrixMSAProfileDialog.obj
 0001:000164d8       __unwindfunclet$?accept@DistanceMatrixMSAProfileDialog@U2@@UAEXXZ$1 100174d8 f   DistanceMatrixMSAProfileDialog.obj
 0001:000164e1       __unwindfunclet$?accept@DistanceMatrixMSAProfileDialog@U2@@UAEXXZ$2 100174e1 f   DistanceMatrixMSAProfileDialog.obj
 0001:000164ea       __unwindfunclet$?accept@DistanceMatrixMSAProfileDialog@U2@@UAEXXZ$3 100174ea f   DistanceMatrixMSAProfileDialog.obj
 0001:000164f3       __unwindfunclet$?accept@DistanceMatrixMSAProfileDialog@U2@@UAEXXZ$4 100174f3 f   DistanceMatrixMSAProfileDialog.obj
 0001:000164fc       __unwindfunclet$?accept@DistanceMatrixMSAProfileDialog@U2@@UAEXXZ$5 100174fc f   DistanceMatrixMSAProfileDialog.obj
 0001:00016505       __unwindfunclet$?accept@DistanceMatrixMSAProfileDialog@U2@@UAEXXZ$6 10017505 f   DistanceMatrixMSAProfileDialog.obj
 0001:0001650e       __unwindfunclet$?accept@DistanceMatrixMSAProfileDialog@U2@@UAEXXZ$7 1001750e f   DistanceMatrixMSAProfileDialog.obj
 0001:00016519       __unwindfunclet$?accept@DistanceMatrixMSAProfileDialog@U2@@UAEXXZ$9 10017519 f   DistanceMatrixMSAProfileDialog.obj
 0001:00016522       __unwindfunclet$?accept@DistanceMatrixMSAProfileDialog@U2@@UAEXXZ$10 10017522 f   DistanceMatrixMSAProfileDialog.obj
 0001:0001652b       __unwindfunclet$?accept@DistanceMatrixMSAProfileDialog@U2@@UAEXXZ$11 1001752b f   DistanceMatrixMSAProfileDialog.obj
 0001:00016534       __unwindfunclet$?accept@DistanceMatrixMSAProfileDialog@U2@@UAEXXZ$12 10017534 f   DistanceMatrixMSAProfileDialog.obj
 0001:0001653d       __ehhandler$?accept@DistanceMatrixMSAProfileDialog@U2@@UAEXXZ 1001753d f   DistanceMatrixMSAProfileDialog.obj
 0001:00016560       __unwindfunclet$?append@?$QList@VMultipleSequenceAlignmentRow@U2@@@@QAEXABVMultipleSequenceAlignmentRow@U2@@@Z$6 10017560 f   DistanceMatrixMSAProfileDialog.obj
 0001:0001656b       __ehhandler$?append@?$QList@VMultipleSequenceAlignmentRow@U2@@@@QAEXABVMultipleSequenceAlignmentRow@U2@@@Z 1001756b f   DistanceMatrixMSAProfileDialog.obj
 0001:00016590       __unwindfunclet$?createDistanceTable@DistanceMatrixMSAProfileTask@U2@@QAEXPAVMSADistanceAlgorithm@2@ABV?$QList@VMultipleSequenceAlignmentRow@U2@@@@PAVQFile@@@Z$0 10017590 f   DistanceMatrixMSAProfileDialog.obj
 0001:00016599       __unwindfunclet$?createDistanceTable@DistanceMatrixMSAProfileTask@U2@@QAEXPAVMSADistanceAlgorithm@2@ABV?$QList@VMultipleSequenceAlignmentRow@U2@@@@PAVQFile@@@Z$1 10017599 f   DistanceMatrixMSAProfileDialog.obj
 0001:000165a2       __unwindfunclet$?createDistanceTable@DistanceMatrixMSAProfileTask@U2@@QAEXPAVMSADistanceAlgorithm@2@ABV?$QList@VMultipleSequenceAlignmentRow@U2@@@@PAVQFile@@@Z$2 100175a2 f   DistanceMatrixMSAProfileDialog.obj
 0001:000165ab       __unwindfunclet$?createDistanceTable@DistanceMatrixMSAProfileTask@U2@@QAEXPAVMSADistanceAlgorithm@2@ABV?$QList@VMultipleSequenceAlignmentRow@U2@@@@PAVQFile@@@Z$3 100175ab f   DistanceMatrixMSAProfileDialog.obj
 0001:000165b4       __unwindfunclet$?createDistanceTable@DistanceMatrixMSAProfileTask@U2@@QAEXPAVMSADistanceAlgorithm@2@ABV?$QList@VMultipleSequenceAlignmentRow@U2@@@@PAVQFile@@@Z$5 100175b4 f   DistanceMatrixMSAProfileDialog.obj
 0001:000165c8       __unwindfunclet$?createDistanceTable@DistanceMatrixMSAProfileTask@U2@@QAEXPAVMSADistanceAlgorithm@2@ABV?$QList@VMultipleSequenceAlignmentRow@U2@@@@PAVQFile@@@Z$6 100175c8 f   DistanceMatrixMSAProfileDialog.obj
 0001:000165d1       __unwindfunclet$?createDistanceTable@DistanceMatrixMSAProfileTask@U2@@QAEXPAVMSADistanceAlgorithm@2@ABV?$QList@VMultipleSequenceAlignmentRow@U2@@@@PAVQFile@@@Z$7 100175d1 f   DistanceMatrixMSAProfileDialog.obj
 0001:000165da       __unwindfunclet$?createDistanceTable@DistanceMatrixMSAProfileTask@U2@@QAEXPAVMSADistanceAlgorithm@2@ABV?$QList@VMultipleSequenceAlignmentRow@U2@@@@PAVQFile@@@Z$8 100175da f   DistanceMatrixMSAProfileDialog.obj
 0001:000165e3       __unwindfunclet$?createDistanceTable@DistanceMatrixMSAProfileTask@U2@@QAEXPAVMSADistanceAlgorithm@2@ABV?$QList@VMultipleSequenceAlignmentRow@U2@@@@PAVQFile@@@Z$9 100175e3 f   DistanceMatrixMSAProfileDialog.obj
 0001:000165ec       __unwindfunclet$?createDistanceTable@DistanceMatrixMSAProfileTask@U2@@QAEXPAVMSADistanceAlgorithm@2@ABV?$QList@VMultipleSequenceAlignmentRow@U2@@@@PAVQFile@@@Z$10 100175ec f   DistanceMatrixMSAProfileDialog.obj
 0001:000165f5       __unwindfunclet$?createDistanceTable@DistanceMatrixMSAProfileTask@U2@@QAEXPAVMSADistanceAlgorithm@2@ABV?$QList@VMultipleSequenceAlignmentRow@U2@@@@PAVQFile@@@Z$11 100175f5 f   DistanceMatrixMSAProfileDialog.obj
 0001:000165fe       __unwindfunclet$?createDistanceTable@DistanceMatrixMSAProfileTask@U2@@QAEXPAVMSADistanceAlgorithm@2@ABV?$QList@VMultipleSequenceAlignmentRow@U2@@@@PAVQFile@@@Z$12 100175fe f   DistanceMatrixMSAProfileDialog.obj
 0001:00016607       __unwindfunclet$?createDistanceTable@DistanceMatrixMSAProfileTask@U2@@QAEXPAVMSADistanceAlgorithm@2@ABV?$QList@VMultipleSequenceAlignmentRow@U2@@@@PAVQFile@@@Z$13 10017607 f   DistanceMatrixMSAProfileDialog.obj
 0001:00016613       __unwindfunclet$?createDistanceTable@DistanceMatrixMSAProfileTask@U2@@QAEXPAVMSADistanceAlgorithm@2@ABV?$QList@VMultipleSequenceAlignmentRow@U2@@@@PAVQFile@@@Z$14 10017613 f   DistanceMatrixMSAProfileDialog.obj
 0001:0001661c       __unwindfunclet$?createDistanceTable@DistanceMatrixMSAProfileTask@U2@@QAEXPAVMSADistanceAlgorithm@2@ABV?$QList@VMultipleSequenceAlignmentRow@U2@@@@PAVQFile@@@Z$15 1001761c f   DistanceMatrixMSAProfileDialog.obj
 0001:00016625       __unwindfunclet$?createDistanceTable@DistanceMatrixMSAProfileTask@U2@@QAEXPAVMSADistanceAlgorithm@2@ABV?$QList@VMultipleSequenceAlignmentRow@U2@@@@PAVQFile@@@Z$16 10017625 f   DistanceMatrixMSAProfileDialog.obj
 0001:0001662e       __unwindfunclet$?createDistanceTable@DistanceMatrixMSAProfileTask@U2@@QAEXPAVMSADistanceAlgorithm@2@ABV?$QList@VMultipleSequenceAlignmentRow@U2@@@@PAVQFile@@@Z$17 1001762e f   DistanceMatrixMSAProfileDialog.obj
 0001:00016637       __unwindfunclet$?createDistanceTable@DistanceMatrixMSAProfileTask@U2@@QAEXPAVMSADistanceAlgorithm@2@ABV?$QList@VMultipleSequenceAlignmentRow@U2@@@@PAVQFile@@@Z$19 10017637 f   DistanceMatrixMSAProfileDialog.obj
 0001:00016640       __unwindfunclet$?createDistanceTable@DistanceMatrixMSAProfileTask@U2@@QAEXPAVMSADistanceAlgorithm@2@ABV?$QList@VMultipleSequenceAlignmentRow@U2@@@@PAVQFile@@@Z$18 10017640 f   DistanceMatrixMSAProfileDialog.obj
 0001:00016649       __unwindfunclet$?createDistanceTable@DistanceMatrixMSAProfileTask@U2@@QAEXPAVMSADistanceAlgorithm@2@ABV?$QList@VMultipleSequenceAlignmentRow@U2@@@@PAVQFile@@@Z$20 10017649 f   DistanceMatrixMSAProfileDialog.obj
 0001:00016652       __unwindfunclet$?createDistanceTable@DistanceMatrixMSAProfileTask@U2@@QAEXPAVMSADistanceAlgorithm@2@ABV?$QList@VMultipleSequenceAlignmentRow@U2@@@@PAVQFile@@@Z$21 10017652 f   DistanceMatrixMSAProfileDialog.obj
 0001:0001665b       __unwindfunclet$?createDistanceTable@DistanceMatrixMSAProfileTask@U2@@QAEXPAVMSADistanceAlgorithm@2@ABV?$QList@VMultipleSequenceAlignmentRow@U2@@@@PAVQFile@@@Z$22 1001765b f   DistanceMatrixMSAProfileDialog.obj
 0001:00016664       __unwindfunclet$?createDistanceTable@DistanceMatrixMSAProfileTask@U2@@QAEXPAVMSADistanceAlgorithm@2@ABV?$QList@VMultipleSequenceAlignmentRow@U2@@@@PAVQFile@@@Z$23 10017664 f   DistanceMatrixMSAProfileDialog.obj
 0001:0001666d       __unwindfunclet$?createDistanceTable@DistanceMatrixMSAProfileTask@U2@@QAEXPAVMSADistanceAlgorithm@2@ABV?$QList@VMultipleSequenceAlignmentRow@U2@@@@PAVQFile@@@Z$24 1001766d f   DistanceMatrixMSAProfileDialog.obj
 0001:00016676       __unwindfunclet$?createDistanceTable@DistanceMatrixMSAProfileTask@U2@@QAEXPAVMSADistanceAlgorithm@2@ABV?$QList@VMultipleSequenceAlignmentRow@U2@@@@PAVQFile@@@Z$25 10017676 f   DistanceMatrixMSAProfileDialog.obj
 0001:0001667f       __unwindfunclet$?createDistanceTable@DistanceMatrixMSAProfileTask@U2@@QAEXPAVMSADistanceAlgorithm@2@ABV?$QList@VMultipleSequenceAlignmentRow@U2@@@@PAVQFile@@@Z$26 1001767f f   DistanceMatrixMSAProfileDialog.obj
 0001:00016688       __ehhandler$?createDistanceTable@DistanceMatrixMSAProfileTask@U2@@QAEXPAVMSADistanceAlgorithm@2@ABV?$QList@VMultipleSequenceAlignmentRow@U2@@@@PAVQFile@@@Z 10017688 f   DistanceMatrixMSAProfileDialog.obj
 0001:000166b0       __ehhandler$?detach_helper_grow@?$QList@VMultipleSequenceAlignmentRow@U2@@@@AAEPAUNode@1@HH@Z 100176b0 f   DistanceMatrixMSAProfileDialog.obj
 0001:000166d0       __unwindfunclet$?generateReport@DistanceMatrixMSAProfileTask@U2@@UBE?AVQString@@XZ$3 100176d0 f   DistanceMatrixMSAProfileDialog.obj
 0001:000166d9       __unwindfunclet$?generateReport@DistanceMatrixMSAProfileTask@U2@@UBE?AVQString@@XZ$4 100176d9 f   DistanceMatrixMSAProfileDialog.obj
 0001:000166e2       __unwindfunclet$?generateReport@DistanceMatrixMSAProfileTask@U2@@UBE?AVQString@@XZ$5 100176e2 f   DistanceMatrixMSAProfileDialog.obj
 0001:000166eb       __unwindfunclet$?generateReport@DistanceMatrixMSAProfileTask@U2@@UBE?AVQString@@XZ$6 100176eb f   DistanceMatrixMSAProfileDialog.obj
 0001:000166f4       __unwindfunclet$?generateReport@DistanceMatrixMSAProfileTask@U2@@UBE?AVQString@@XZ$7 100176f4 f   DistanceMatrixMSAProfileDialog.obj
 0001:000166fd       __unwindfunclet$?generateReport@DistanceMatrixMSAProfileTask@U2@@UBE?AVQString@@XZ$8 100176fd f   DistanceMatrixMSAProfileDialog.obj
 0001:00016706       __unwindfunclet$?generateReport@DistanceMatrixMSAProfileTask@U2@@UBE?AVQString@@XZ$0 10017706 f   DistanceMatrixMSAProfileDialog.obj
 0001:0001670f       __unwindfunclet$?generateReport@DistanceMatrixMSAProfileTask@U2@@UBE?AVQString@@XZ$1 1001770f f   DistanceMatrixMSAProfileDialog.obj
 0001:00016718       __unwindfunclet$?generateReport@DistanceMatrixMSAProfileTask@U2@@UBE?AVQString@@XZ$2 10017718 f   DistanceMatrixMSAProfileDialog.obj
 0001:00016732       __ehhandler$?generateReport@DistanceMatrixMSAProfileTask@U2@@UBE?AVQString@@XZ 10017732 f   DistanceMatrixMSAProfileDialog.obj
 0001:00016750       __unwindfunclet$?initSaveController@DistanceMatrixMSAProfileDialog@U2@@AAEXXZ$0 10017750 f   DistanceMatrixMSAProfileDialog.obj
 0001:00016759       __unwindfunclet$?initSaveController@DistanceMatrixMSAProfileDialog@U2@@AAEXXZ$1 10017759 f   DistanceMatrixMSAProfileDialog.obj
 0001:00016762       __unwindfunclet$?initSaveController@DistanceMatrixMSAProfileDialog@U2@@AAEXXZ$2 10017762 f   DistanceMatrixMSAProfileDialog.obj
 0001:0001676b       __unwindfunclet$?initSaveController@DistanceMatrixMSAProfileDialog@U2@@AAEXXZ$3 1001776b f   DistanceMatrixMSAProfileDialog.obj
 0001:00016774       __unwindfunclet$?initSaveController@DistanceMatrixMSAProfileDialog@U2@@AAEXXZ$4 10017774 f   DistanceMatrixMSAProfileDialog.obj
 0001:0001677d       __unwindfunclet$?initSaveController@DistanceMatrixMSAProfileDialog@U2@@AAEXXZ$5 1001777d f   DistanceMatrixMSAProfileDialog.obj
 0001:00016786       __unwindfunclet$?initSaveController@DistanceMatrixMSAProfileDialog@U2@@AAEXXZ$6 10017786 f   DistanceMatrixMSAProfileDialog.obj
 0001:0001678f       __unwindfunclet$?initSaveController@DistanceMatrixMSAProfileDialog@U2@@AAEXXZ$7 1001778f f   DistanceMatrixMSAProfileDialog.obj
 0001:00016798       __unwindfunclet$?initSaveController@DistanceMatrixMSAProfileDialog@U2@@AAEXXZ$8 10017798 f   DistanceMatrixMSAProfileDialog.obj
 0001:000167a1       __unwindfunclet$?initSaveController@DistanceMatrixMSAProfileDialog@U2@@AAEXXZ$9 100177a1 f   DistanceMatrixMSAProfileDialog.obj
 0001:000167aa       __unwindfunclet$?initSaveController@DistanceMatrixMSAProfileDialog@U2@@AAEXXZ$10 100177aa f   DistanceMatrixMSAProfileDialog.obj
 0001:000167b3       __unwindfunclet$?initSaveController@DistanceMatrixMSAProfileDialog@U2@@AAEXXZ$11 100177b3 f   DistanceMatrixMSAProfileDialog.obj
 0001:000167bc       __unwindfunclet$?initSaveController@DistanceMatrixMSAProfileDialog@U2@@AAEXXZ$12 100177bc f   DistanceMatrixMSAProfileDialog.obj
 0001:000167c4       __unwindfunclet$?initSaveController@DistanceMatrixMSAProfileDialog@U2@@AAEXXZ$13 100177c4 f   DistanceMatrixMSAProfileDialog.obj
 0001:000167cd       __unwindfunclet$?initSaveController@DistanceMatrixMSAProfileDialog@U2@@AAEXXZ$14 100177cd f   DistanceMatrixMSAProfileDialog.obj
 0001:000167d5       __unwindfunclet$?initSaveController@DistanceMatrixMSAProfileDialog@U2@@AAEXXZ$15 100177d5 f   DistanceMatrixMSAProfileDialog.obj
 0001:000167de       __unwindfunclet$?initSaveController@DistanceMatrixMSAProfileDialog@U2@@AAEXXZ$16 100177de f   DistanceMatrixMSAProfileDialog.obj
 0001:000167e9       __ehhandler$?initSaveController@DistanceMatrixMSAProfileDialog@U2@@AAEXXZ 100177e9 f   DistanceMatrixMSAProfileDialog.obj
 0001:00016810       __unwindfunclet$?node_construct@?$QList@VMultipleSequenceAlignmentRow@U2@@@@AAEXPAUNode@1@ABVMultipleSequenceAlignmentRow@U2@@@Z$0 10017810 f   DistanceMatrixMSAProfileDialog.obj
 0001:0001681b       __ehhandler$?node_construct@?$QList@VMultipleSequenceAlignmentRow@U2@@@@AAEXPAUNode@1@ABVMultipleSequenceAlignmentRow@U2@@@Z 1001781b f   DistanceMatrixMSAProfileDialog.obj
 0001:00016840       __unwindfunclet$?node_copy@?$QList@VMultipleSequenceAlignmentRow@U2@@@@AAEXPAUNode@1@00@Z$4 10017840 f   DistanceMatrixMSAProfileDialog.obj
 0001:0001684b       __ehhandler$?node_copy@?$QList@VMultipleSequenceAlignmentRow@U2@@@@AAEXPAUNode@1@00@Z 1001784b f   DistanceMatrixMSAProfileDialog.obj
 0001:00016870       __unwindfunclet$?onSubTaskFinished@DistanceMatrixMSAProfileTask@U2@@UAE?AV?$QList@PAVTask@U2@@@@PAVTask@2@@Z$4 10017870 f   DistanceMatrixMSAProfileDialog.obj
 0001:00016878       __unwindfunclet$?onSubTaskFinished@DistanceMatrixMSAProfileTask@U2@@UAE?AV?$QList@PAVTask@U2@@@@PAVTask@2@@Z$7 10017878 f   DistanceMatrixMSAProfileDialog.obj
 0001:00016881       __unwindfunclet$?onSubTaskFinished@DistanceMatrixMSAProfileTask@U2@@UAE?AV?$QList@PAVTask@U2@@@@PAVTask@2@@Z$84 10017881 f   DistanceMatrixMSAProfileDialog.obj
 0001:0001688c       __unwindfunclet$?onSubTaskFinished@DistanceMatrixMSAProfileTask@U2@@UAE?AV?$QList@PAVTask@U2@@@@PAVTask@2@@Z$85 1001788c f   DistanceMatrixMSAProfileDialog.obj
 0001:00016895       __unwindfunclet$?onSubTaskFinished@DistanceMatrixMSAProfileTask@U2@@UAE?AV?$QList@PAVTask@U2@@@@PAVTask@2@@Z$86 10017895 f   DistanceMatrixMSAProfileDialog.obj
 0001:0001689e       __unwindfunclet$?onSubTaskFinished@DistanceMatrixMSAProfileTask@U2@@UAE?AV?$QList@PAVTask@U2@@@@PAVTask@2@@Z$87 1001789e f   DistanceMatrixMSAProfileDialog.obj
 0001:000168aa       __unwindfunclet$?onSubTaskFinished@DistanceMatrixMSAProfileTask@U2@@UAE?AV?$QList@PAVTask@U2@@@@PAVTask@2@@Z$88 100178aa f   DistanceMatrixMSAProfileDialog.obj
 0001:000168b3       __unwindfunclet$?onSubTaskFinished@DistanceMatrixMSAProfileTask@U2@@UAE?AV?$QList@PAVTask@U2@@@@PAVTask@2@@Z$89 100178b3 f   DistanceMatrixMSAProfileDialog.obj
 0001:000168bc       __unwindfunclet$?onSubTaskFinished@DistanceMatrixMSAProfileTask@U2@@UAE?AV?$QList@PAVTask@U2@@@@PAVTask@2@@Z$90 100178bc f   DistanceMatrixMSAProfileDialog.obj
 0001:000168c8       __unwindfunclet$?onSubTaskFinished@DistanceMatrixMSAProfileTask@U2@@UAE?AV?$QList@PAVTask@U2@@@@PAVTask@2@@Z$91 100178c8 f   DistanceMatrixMSAProfileDialog.obj
 0001:000168d1       __unwindfunclet$?onSubTaskFinished@DistanceMatrixMSAProfileTask@U2@@UAE?AV?$QList@PAVTask@U2@@@@PAVTask@2@@Z$92 100178d1 f   DistanceMatrixMSAProfileDialog.obj
 0001:000168da       __unwindfunclet$?onSubTaskFinished@DistanceMatrixMSAProfileTask@U2@@UAE?AV?$QList@PAVTask@U2@@@@PAVTask@2@@Z$93 100178da f   DistanceMatrixMSAProfileDialog.obj
 0001:000168e3       __unwindfunclet$?onSubTaskFinished@DistanceMatrixMSAProfileTask@U2@@UAE?AV?$QList@PAVTask@U2@@@@PAVTask@2@@Z$94 100178e3 f   DistanceMatrixMSAProfileDialog.obj
 0001:000168ec       __unwindfunclet$?onSubTaskFinished@DistanceMatrixMSAProfileTask@U2@@UAE?AV?$QList@PAVTask@U2@@@@PAVTask@2@@Z$8 100178ec f   DistanceMatrixMSAProfileDialog.obj
 0001:000168f7       __unwindfunclet$?onSubTaskFinished@DistanceMatrixMSAProfileTask@U2@@UAE?AV?$QList@PAVTask@U2@@@@PAVTask@2@@Z$9 100178f7 f   DistanceMatrixMSAProfileDialog.obj
 0001:00016900       __unwindfunclet$?onSubTaskFinished@DistanceMatrixMSAProfileTask@U2@@UAE?AV?$QList@PAVTask@U2@@@@PAVTask@2@@Z$10 10017900 f   DistanceMatrixMSAProfileDialog.obj
 0001:00016909       __unwindfunclet$?onSubTaskFinished@DistanceMatrixMSAProfileTask@U2@@UAE?AV?$QList@PAVTask@U2@@@@PAVTask@2@@Z$11 10017909 f   DistanceMatrixMSAProfileDialog.obj
 0001:00016912       __unwindfunclet$?onSubTaskFinished@DistanceMatrixMSAProfileTask@U2@@UAE?AV?$QList@PAVTask@U2@@@@PAVTask@2@@Z$12 10017912 f   DistanceMatrixMSAProfileDialog.obj
 0001:0001691b       __unwindfunclet$?onSubTaskFinished@DistanceMatrixMSAProfileTask@U2@@UAE?AV?$QList@PAVTask@U2@@@@PAVTask@2@@Z$13 1001791b f   DistanceMatrixMSAProfileDialog.obj
 0001:00016924       __unwindfunclet$?onSubTaskFinished@DistanceMatrixMSAProfileTask@U2@@UAE?AV?$QList@PAVTask@U2@@@@PAVTask@2@@Z$14 10017924 f   DistanceMatrixMSAProfileDialog.obj
 0001:0001692d       __unwindfunclet$?onSubTaskFinished@DistanceMatrixMSAProfileTask@U2@@UAE?AV?$QList@PAVTask@U2@@@@PAVTask@2@@Z$16 1001792d f   DistanceMatrixMSAProfileDialog.obj
 0001:00016941       __unwindfunclet$?onSubTaskFinished@DistanceMatrixMSAProfileTask@U2@@UAE?AV?$QList@PAVTask@U2@@@@PAVTask@2@@Z$17 10017941 f   DistanceMatrixMSAProfileDialog.obj
 0001:0001694a       __unwindfunclet$?onSubTaskFinished@DistanceMatrixMSAProfileTask@U2@@UAE?AV?$QList@PAVTask@U2@@@@PAVTask@2@@Z$18 1001794a f   DistanceMatrixMSAProfileDialog.obj
 0001:00016953       __unwindfunclet$?onSubTaskFinished@DistanceMatrixMSAProfileTask@U2@@UAE?AV?$QList@PAVTask@U2@@@@PAVTask@2@@Z$19 10017953 f   DistanceMatrixMSAProfileDialog.obj
 0001:0001695c       __unwindfunclet$?onSubTaskFinished@DistanceMatrixMSAProfileTask@U2@@UAE?AV?$QList@PAVTask@U2@@@@PAVTask@2@@Z$20 1001795c f   DistanceMatrixMSAProfileDialog.obj
 0001:00016965       __unwindfunclet$?onSubTaskFinished@DistanceMatrixMSAProfileTask@U2@@UAE?AV?$QList@PAVTask@U2@@@@PAVTask@2@@Z$21 10017965 f   DistanceMatrixMSAProfileDialog.obj
 0001:0001696e       __unwindfunclet$?onSubTaskFinished@DistanceMatrixMSAProfileTask@U2@@UAE?AV?$QList@PAVTask@U2@@@@PAVTask@2@@Z$22 1001796e f   DistanceMatrixMSAProfileDialog.obj
 0001:00016977       __unwindfunclet$?onSubTaskFinished@DistanceMatrixMSAProfileTask@U2@@UAE?AV?$QList@PAVTask@U2@@@@PAVTask@2@@Z$23 10017977 f   DistanceMatrixMSAProfileDialog.obj
 0001:00016980       __unwindfunclet$?onSubTaskFinished@DistanceMatrixMSAProfileTask@U2@@UAE?AV?$QList@PAVTask@U2@@@@PAVTask@2@@Z$24 10017980 f   DistanceMatrixMSAProfileDialog.obj
 0001:00016989       __unwindfunclet$?onSubTaskFinished@DistanceMatrixMSAProfileTask@U2@@UAE?AV?$QList@PAVTask@U2@@@@PAVTask@2@@Z$25 10017989 f   DistanceMatrixMSAProfileDialog.obj
 0001:00016992       __unwindfunclet$?onSubTaskFinished@DistanceMatrixMSAProfileTask@U2@@UAE?AV?$QList@PAVTask@U2@@@@PAVTask@2@@Z$26 10017992 f   DistanceMatrixMSAProfileDialog.obj
 0001:0001699b       __unwindfunclet$?onSubTaskFinished@DistanceMatrixMSAProfileTask@U2@@UAE?AV?$QList@PAVTask@U2@@@@PAVTask@2@@Z$27 1001799b f   DistanceMatrixMSAProfileDialog.obj
 0001:000169b5       __unwindfunclet$?onSubTaskFinished@DistanceMatrixMSAProfileTask@U2@@UAE?AV?$QList@PAVTask@U2@@@@PAVTask@2@@Z$28 100179b5 f   DistanceMatrixMSAProfileDialog.obj
 0001:000169cf       __unwindfunclet$?onSubTaskFinished@DistanceMatrixMSAProfileTask@U2@@UAE?AV?$QList@PAVTask@U2@@@@PAVTask@2@@Z$29 100179cf f   DistanceMatrixMSAProfileDialog.obj
 0001:000169e9       __unwindfunclet$?onSubTaskFinished@DistanceMatrixMSAProfileTask@U2@@UAE?AV?$QList@PAVTask@U2@@@@PAVTask@2@@Z$30 100179e9 f   DistanceMatrixMSAProfileDialog.obj
 0001:000169f2       __unwindfunclet$?onSubTaskFinished@DistanceMatrixMSAProfileTask@U2@@UAE?AV?$QList@PAVTask@U2@@@@PAVTask@2@@Z$31 100179f2 f   DistanceMatrixMSAProfileDialog.obj
 0001:000169fb       __unwindfunclet$?onSubTaskFinished@DistanceMatrixMSAProfileTask@U2@@UAE?AV?$QList@PAVTask@U2@@@@PAVTask@2@@Z$32 100179fb f   DistanceMatrixMSAProfileDialog.obj
 0001:00016a04       __unwindfunclet$?onSubTaskFinished@DistanceMatrixMSAProfileTask@U2@@UAE?AV?$QList@PAVTask@U2@@@@PAVTask@2@@Z$33 10017a04 f   DistanceMatrixMSAProfileDialog.obj
 0001:00016a0d       __unwindfunclet$?onSubTaskFinished@DistanceMatrixMSAProfileTask@U2@@UAE?AV?$QList@PAVTask@U2@@@@PAVTask@2@@Z$34 10017a0d f   DistanceMatrixMSAProfileDialog.obj
 0001:00016a16       __unwindfunclet$?onSubTaskFinished@DistanceMatrixMSAProfileTask@U2@@UAE?AV?$QList@PAVTask@U2@@@@PAVTask@2@@Z$35 10017a16 f   DistanceMatrixMSAProfileDialog.obj
 0001:00016a1e       __unwindfunclet$?onSubTaskFinished@DistanceMatrixMSAProfileTask@U2@@UAE?AV?$QList@PAVTask@U2@@@@PAVTask@2@@Z$37 10017a1e f   DistanceMatrixMSAProfileDialog.obj
 0001:00016a27       __unwindfunclet$?onSubTaskFinished@DistanceMatrixMSAProfileTask@U2@@UAE?AV?$QList@PAVTask@U2@@@@PAVTask@2@@Z$38 10017a27 f   DistanceMatrixMSAProfileDialog.obj
 0001:00016a30       __unwindfunclet$?onSubTaskFinished@DistanceMatrixMSAProfileTask@U2@@UAE?AV?$QList@PAVTask@U2@@@@PAVTask@2@@Z$39 10017a30 f   DistanceMatrixMSAProfileDialog.obj
 0001:00016a39       __unwindfunclet$?onSubTaskFinished@DistanceMatrixMSAProfileTask@U2@@UAE?AV?$QList@PAVTask@U2@@@@PAVTask@2@@Z$40 10017a39 f   DistanceMatrixMSAProfileDialog.obj
 0001:00016a41       __unwindfunclet$?onSubTaskFinished@DistanceMatrixMSAProfileTask@U2@@UAE?AV?$QList@PAVTask@U2@@@@PAVTask@2@@Z$41 10017a41 f   DistanceMatrixMSAProfileDialog.obj
 0001:00016a49       __unwindfunclet$?onSubTaskFinished@DistanceMatrixMSAProfileTask@U2@@UAE?AV?$QList@PAVTask@U2@@@@PAVTask@2@@Z$42 10017a49 f   DistanceMatrixMSAProfileDialog.obj
 0001:00016a52       __unwindfunclet$?onSubTaskFinished@DistanceMatrixMSAProfileTask@U2@@UAE?AV?$QList@PAVTask@U2@@@@PAVTask@2@@Z$43 10017a52 f   DistanceMatrixMSAProfileDialog.obj
 0001:00016a5d       __unwindfunclet$?onSubTaskFinished@DistanceMatrixMSAProfileTask@U2@@UAE?AV?$QList@PAVTask@U2@@@@PAVTask@2@@Z$44 10017a5d f   DistanceMatrixMSAProfileDialog.obj
 0001:00016a69       __unwindfunclet$?onSubTaskFinished@DistanceMatrixMSAProfileTask@U2@@UAE?AV?$QList@PAVTask@U2@@@@PAVTask@2@@Z$45 10017a69 f   DistanceMatrixMSAProfileDialog.obj
 0001:00016a75       __unwindfunclet$?onSubTaskFinished@DistanceMatrixMSAProfileTask@U2@@UAE?AV?$QList@PAVTask@U2@@@@PAVTask@2@@Z$46 10017a75 f   DistanceMatrixMSAProfileDialog.obj
 0001:00016a7e       __unwindfunclet$?onSubTaskFinished@DistanceMatrixMSAProfileTask@U2@@UAE?AV?$QList@PAVTask@U2@@@@PAVTask@2@@Z$47 10017a7e f   DistanceMatrixMSAProfileDialog.obj
 0001:00016a8a       __unwindfunclet$?onSubTaskFinished@DistanceMatrixMSAProfileTask@U2@@UAE?AV?$QList@PAVTask@U2@@@@PAVTask@2@@Z$48 10017a8a f   DistanceMatrixMSAProfileDialog.obj
 0001:00016a96       __unwindfunclet$?onSubTaskFinished@DistanceMatrixMSAProfileTask@U2@@UAE?AV?$QList@PAVTask@U2@@@@PAVTask@2@@Z$49 10017a96 f   DistanceMatrixMSAProfileDialog.obj
 0001:00016aa2       __unwindfunclet$?onSubTaskFinished@DistanceMatrixMSAProfileTask@U2@@UAE?AV?$QList@PAVTask@U2@@@@PAVTask@2@@Z$50 10017aa2 f   DistanceMatrixMSAProfileDialog.obj
 0001:00016aae       __unwindfunclet$?onSubTaskFinished@DistanceMatrixMSAProfileTask@U2@@UAE?AV?$QList@PAVTask@U2@@@@PAVTask@2@@Z$51 10017aae f   DistanceMatrixMSAProfileDialog.obj
 0001:00016aba       __unwindfunclet$?onSubTaskFinished@DistanceMatrixMSAProfileTask@U2@@UAE?AV?$QList@PAVTask@U2@@@@PAVTask@2@@Z$52 10017aba f   DistanceMatrixMSAProfileDialog.obj
 0001:00016ac6       __unwindfunclet$?onSubTaskFinished@DistanceMatrixMSAProfileTask@U2@@UAE?AV?$QList@PAVTask@U2@@@@PAVTask@2@@Z$53 10017ac6 f   DistanceMatrixMSAProfileDialog.obj
 0001:00016acf       __unwindfunclet$?onSubTaskFinished@DistanceMatrixMSAProfileTask@U2@@UAE?AV?$QList@PAVTask@U2@@@@PAVTask@2@@Z$54 10017acf f   DistanceMatrixMSAProfileDialog.obj
 0001:00016ad8       __unwindfunclet$?onSubTaskFinished@DistanceMatrixMSAProfileTask@U2@@UAE?AV?$QList@PAVTask@U2@@@@PAVTask@2@@Z$55 10017ad8 f   DistanceMatrixMSAProfileDialog.obj
 0001:00016ae4       __unwindfunclet$?onSubTaskFinished@DistanceMatrixMSAProfileTask@U2@@UAE?AV?$QList@PAVTask@U2@@@@PAVTask@2@@Z$56 10017ae4 f   DistanceMatrixMSAProfileDialog.obj
 0001:00016aed       __unwindfunclet$?onSubTaskFinished@DistanceMatrixMSAProfileTask@U2@@UAE?AV?$QList@PAVTask@U2@@@@PAVTask@2@@Z$57 10017aed f   DistanceMatrixMSAProfileDialog.obj
 0001:00016af9       __unwindfunclet$?onSubTaskFinished@DistanceMatrixMSAProfileTask@U2@@UAE?AV?$QList@PAVTask@U2@@@@PAVTask@2@@Z$58 10017af9 f   DistanceMatrixMSAProfileDialog.obj
 0001:00016b02       __unwindfunclet$?onSubTaskFinished@DistanceMatrixMSAProfileTask@U2@@UAE?AV?$QList@PAVTask@U2@@@@PAVTask@2@@Z$59 10017b02 f   DistanceMatrixMSAProfileDialog.obj
 0001:00016b0b       __unwindfunclet$?onSubTaskFinished@DistanceMatrixMSAProfileTask@U2@@UAE?AV?$QList@PAVTask@U2@@@@PAVTask@2@@Z$61 10017b0b f   DistanceMatrixMSAProfileDialog.obj
 0001:00016b14       __unwindfunclet$?onSubTaskFinished@DistanceMatrixMSAProfileTask@U2@@UAE?AV?$QList@PAVTask@U2@@@@PAVTask@2@@Z$62 10017b14 f   DistanceMatrixMSAProfileDialog.obj
 0001:00016b1d       __unwindfunclet$?onSubTaskFinished@DistanceMatrixMSAProfileTask@U2@@UAE?AV?$QList@PAVTask@U2@@@@PAVTask@2@@Z$63 10017b1d f   DistanceMatrixMSAProfileDialog.obj
 0001:00016b26       __unwindfunclet$?onSubTaskFinished@DistanceMatrixMSAProfileTask@U2@@UAE?AV?$QList@PAVTask@U2@@@@PAVTask@2@@Z$64 10017b26 f   DistanceMatrixMSAProfileDialog.obj
 0001:00016b2f       __unwindfunclet$?onSubTaskFinished@DistanceMatrixMSAProfileTask@U2@@UAE?AV?$QList@PAVTask@U2@@@@PAVTask@2@@Z$65 10017b2f f   DistanceMatrixMSAProfileDialog.obj
 0001:00016b38       __unwindfunclet$?onSubTaskFinished@DistanceMatrixMSAProfileTask@U2@@UAE?AV?$QList@PAVTask@U2@@@@PAVTask@2@@Z$66 10017b38 f   DistanceMatrixMSAProfileDialog.obj
 0001:00016b41       __unwindfunclet$?onSubTaskFinished@DistanceMatrixMSAProfileTask@U2@@UAE?AV?$QList@PAVTask@U2@@@@PAVTask@2@@Z$67 10017b41 f   DistanceMatrixMSAProfileDialog.obj
 0001:00016b4a       __unwindfunclet$?onSubTaskFinished@DistanceMatrixMSAProfileTask@U2@@UAE?AV?$QList@PAVTask@U2@@@@PAVTask@2@@Z$68 10017b4a f   DistanceMatrixMSAProfileDialog.obj
 0001:00016b56       __unwindfunclet$?onSubTaskFinished@DistanceMatrixMSAProfileTask@U2@@UAE?AV?$QList@PAVTask@U2@@@@PAVTask@2@@Z$69 10017b56 f   DistanceMatrixMSAProfileDialog.obj
 0001:00016b5f       __unwindfunclet$?onSubTaskFinished@DistanceMatrixMSAProfileTask@U2@@UAE?AV?$QList@PAVTask@U2@@@@PAVTask@2@@Z$70 10017b5f f   DistanceMatrixMSAProfileDialog.obj
 0001:00016b68       __unwindfunclet$?onSubTaskFinished@DistanceMatrixMSAProfileTask@U2@@UAE?AV?$QList@PAVTask@U2@@@@PAVTask@2@@Z$71 10017b68 f   DistanceMatrixMSAProfileDialog.obj
 0001:00016b71       __unwindfunclet$?onSubTaskFinished@DistanceMatrixMSAProfileTask@U2@@UAE?AV?$QList@PAVTask@U2@@@@PAVTask@2@@Z$72 10017b71 f   DistanceMatrixMSAProfileDialog.obj
 0001:00016b7a       __unwindfunclet$?onSubTaskFinished@DistanceMatrixMSAProfileTask@U2@@UAE?AV?$QList@PAVTask@U2@@@@PAVTask@2@@Z$73 10017b7a f   DistanceMatrixMSAProfileDialog.obj
 0001:00016b83       __unwindfunclet$?onSubTaskFinished@DistanceMatrixMSAProfileTask@U2@@UAE?AV?$QList@PAVTask@U2@@@@PAVTask@2@@Z$74 10017b83 f   DistanceMatrixMSAProfileDialog.obj
 0001:00016b8c       __unwindfunclet$?onSubTaskFinished@DistanceMatrixMSAProfileTask@U2@@UAE?AV?$QList@PAVTask@U2@@@@PAVTask@2@@Z$75 10017b8c f   DistanceMatrixMSAProfileDialog.obj
 0001:00016b95       __unwindfunclet$?onSubTaskFinished@DistanceMatrixMSAProfileTask@U2@@UAE?AV?$QList@PAVTask@U2@@@@PAVTask@2@@Z$76 10017b95 f   DistanceMatrixMSAProfileDialog.obj
 0001:00016b9e       __unwindfunclet$?onSubTaskFinished@DistanceMatrixMSAProfileTask@U2@@UAE?AV?$QList@PAVTask@U2@@@@PAVTask@2@@Z$77 10017b9e f   DistanceMatrixMSAProfileDialog.obj
 0001:00016ba7       __unwindfunclet$?onSubTaskFinished@DistanceMatrixMSAProfileTask@U2@@UAE?AV?$QList@PAVTask@U2@@@@PAVTask@2@@Z$78 10017ba7 f   DistanceMatrixMSAProfileDialog.obj
 0001:00016bb3       __unwindfunclet$?onSubTaskFinished@DistanceMatrixMSAProfileTask@U2@@UAE?AV?$QList@PAVTask@U2@@@@PAVTask@2@@Z$79 10017bb3 f   DistanceMatrixMSAProfileDialog.obj
 0001:00016bbc       __unwindfunclet$?onSubTaskFinished@DistanceMatrixMSAProfileTask@U2@@UAE?AV?$QList@PAVTask@U2@@@@PAVTask@2@@Z$80 10017bbc f   DistanceMatrixMSAProfileDialog.obj
 0001:00016bc5       __unwindfunclet$?onSubTaskFinished@DistanceMatrixMSAProfileTask@U2@@UAE?AV?$QList@PAVTask@U2@@@@PAVTask@2@@Z$81 10017bc5 f   DistanceMatrixMSAProfileDialog.obj
 0001:00016bce       __unwindfunclet$?onSubTaskFinished@DistanceMatrixMSAProfileTask@U2@@UAE?AV?$QList@PAVTask@U2@@@@PAVTask@2@@Z$82 10017bce f   DistanceMatrixMSAProfileDialog.obj
 0001:00016bd7       __unwindfunclet$?onSubTaskFinished@DistanceMatrixMSAProfileTask@U2@@UAE?AV?$QList@PAVTask@U2@@@@PAVTask@2@@Z$83 10017bd7 f   DistanceMatrixMSAProfileDialog.obj
 0001:00016be0       __unwindfunclet$?onSubTaskFinished@DistanceMatrixMSAProfileTask@U2@@UAE?AV?$QList@PAVTask@U2@@@@PAVTask@2@@Z$95 10017be0 f   DistanceMatrixMSAProfileDialog.obj
 0001:00016be9       __unwindfunclet$?onSubTaskFinished@DistanceMatrixMSAProfileTask@U2@@UAE?AV?$QList@PAVTask@U2@@@@PAVTask@2@@Z$60 10017be9 f   DistanceMatrixMSAProfileDialog.obj
 0001:00016bf2       __unwindfunclet$?onSubTaskFinished@DistanceMatrixMSAProfileTask@U2@@UAE?AV?$QList@PAVTask@U2@@@@PAVTask@2@@Z$36 10017bf2 f   DistanceMatrixMSAProfileDialog.obj
 0001:00016bfb       __unwindfunclet$?onSubTaskFinished@DistanceMatrixMSAProfileTask@U2@@UAE?AV?$QList@PAVTask@U2@@@@PAVTask@2@@Z$5 10017bfb f   DistanceMatrixMSAProfileDialog.obj
 0001:00016c04       __unwindfunclet$?onSubTaskFinished@DistanceMatrixMSAProfileTask@U2@@UAE?AV?$QList@PAVTask@U2@@@@PAVTask@2@@Z$6 10017c04 f   DistanceMatrixMSAProfileDialog.obj
 0001:00016c20       __ehhandler$?onSubTaskFinished@DistanceMatrixMSAProfileTask@U2@@UAE?AV?$QList@PAVTask@U2@@@@PAVTask@2@@Z 10017c20 f   DistanceMatrixMSAProfileDialog.obj
 0001:00016c50       __unwindfunclet$?report@DistanceMatrixMSAProfileTask@U2@@UAE?AW4ReportResult@Task@2@XZ$0 10017c50 f   DistanceMatrixMSAProfileDialog.obj
 0001:00016c6a       __unwindfunclet$?report@DistanceMatrixMSAProfileTask@U2@@UAE?AW4ReportResult@Task@2@XZ$1 10017c6a f   DistanceMatrixMSAProfileDialog.obj
 0001:00016c84       __unwindfunclet$?report@DistanceMatrixMSAProfileTask@U2@@UAE?AW4ReportResult@Task@2@XZ$2 10017c84 f   DistanceMatrixMSAProfileDialog.obj
 0001:00016c9e       __unwindfunclet$?report@DistanceMatrixMSAProfileTask@U2@@UAE?AW4ReportResult@Task@2@XZ$3 10017c9e f   DistanceMatrixMSAProfileDialog.obj
 0001:00016ca7       __unwindfunclet$?report@DistanceMatrixMSAProfileTask@U2@@UAE?AW4ReportResult@Task@2@XZ$4 10017ca7 f   DistanceMatrixMSAProfileDialog.obj
 0001:00016cb2       __unwindfunclet$?report@DistanceMatrixMSAProfileTask@U2@@UAE?AW4ReportResult@Task@2@XZ$5 10017cb2 f   DistanceMatrixMSAProfileDialog.obj
 0001:00016cbb       __unwindfunclet$?report@DistanceMatrixMSAProfileTask@U2@@UAE?AW4ReportResult@Task@2@XZ$6 10017cbb f   DistanceMatrixMSAProfileDialog.obj
 0001:00016cc4       __ehhandler$?report@DistanceMatrixMSAProfileTask@U2@@UAE?AW4ReportResult@Task@2@XZ 10017cc4 f   DistanceMatrixMSAProfileDialog.obj
 0001:00016ce0       __unwindfunclet$?retranslateUi@Ui_DistanceMatrixMSAProfileDialog@@QAEXPAVQDialog@@@Z$0 10017ce0 f   DistanceMatrixMSAProfileDialog.obj
 0001:00016ce9       __unwindfunclet$?retranslateUi@Ui_DistanceMatrixMSAProfileDialog@@QAEXPAVQDialog@@@Z$1 10017ce9 f   DistanceMatrixMSAProfileDialog.obj
 0001:00016cf2       __unwindfunclet$?retranslateUi@Ui_DistanceMatrixMSAProfileDialog@@QAEXPAVQDialog@@@Z$2 10017cf2 f   DistanceMatrixMSAProfileDialog.obj
 0001:00016cfb       __unwindfunclet$?retranslateUi@Ui_DistanceMatrixMSAProfileDialog@@QAEXPAVQDialog@@@Z$3 10017cfb f   DistanceMatrixMSAProfileDialog.obj
 0001:00016d04       __unwindfunclet$?retranslateUi@Ui_DistanceMatrixMSAProfileDialog@@QAEXPAVQDialog@@@Z$4 10017d04 f   DistanceMatrixMSAProfileDialog.obj
 0001:00016d0d       __unwindfunclet$?retranslateUi@Ui_DistanceMatrixMSAProfileDialog@@QAEXPAVQDialog@@@Z$5 10017d0d f   DistanceMatrixMSAProfileDialog.obj
 0001:00016d16       __unwindfunclet$?retranslateUi@Ui_DistanceMatrixMSAProfileDialog@@QAEXPAVQDialog@@@Z$6 10017d16 f   DistanceMatrixMSAProfileDialog.obj
 0001:00016d1f       __unwindfunclet$?retranslateUi@Ui_DistanceMatrixMSAProfileDialog@@QAEXPAVQDialog@@@Z$7 10017d1f f   DistanceMatrixMSAProfileDialog.obj
 0001:00016d28       __unwindfunclet$?retranslateUi@Ui_DistanceMatrixMSAProfileDialog@@QAEXPAVQDialog@@@Z$8 10017d28 f   DistanceMatrixMSAProfileDialog.obj
 0001:00016d31       __unwindfunclet$?retranslateUi@Ui_DistanceMatrixMSAProfileDialog@@QAEXPAVQDialog@@@Z$9 10017d31 f   DistanceMatrixMSAProfileDialog.obj
 0001:00016d3a       __unwindfunclet$?retranslateUi@Ui_DistanceMatrixMSAProfileDialog@@QAEXPAVQDialog@@@Z$10 10017d3a f   DistanceMatrixMSAProfileDialog.obj
 0001:00016d43       __unwindfunclet$?retranslateUi@Ui_DistanceMatrixMSAProfileDialog@@QAEXPAVQDialog@@@Z$11 10017d43 f   DistanceMatrixMSAProfileDialog.obj
 0001:00016d4c       __ehhandler$?retranslateUi@Ui_DistanceMatrixMSAProfileDialog@@QAEXPAVQDialog@@@Z 10017d4c f   DistanceMatrixMSAProfileDialog.obj
 0001:00016d70       __unwindfunclet$?setupUi@Ui_DistanceMatrixMSAProfileDialog@@QAEXPAVQDialog@@@Z$1 10017d70 f   DistanceMatrixMSAProfileDialog.obj
 0001:00016d79       __unwindfunclet$?setupUi@Ui_DistanceMatrixMSAProfileDialog@@QAEXPAVQDialog@@@Z$2 10017d79 f   DistanceMatrixMSAProfileDialog.obj
 0001:00016d84       __unwindfunclet$?setupUi@Ui_DistanceMatrixMSAProfileDialog@@QAEXPAVQDialog@@@Z$3 10017d84 f   DistanceMatrixMSAProfileDialog.obj
 0001:00016d8d       __unwindfunclet$?setupUi@Ui_DistanceMatrixMSAProfileDialog@@QAEXPAVQDialog@@@Z$4 10017d8d f   DistanceMatrixMSAProfileDialog.obj
 0001:00016d98       __unwindfunclet$?setupUi@Ui_DistanceMatrixMSAProfileDialog@@QAEXPAVQDialog@@@Z$5 10017d98 f   DistanceMatrixMSAProfileDialog.obj
 0001:00016da1       __unwindfunclet$?setupUi@Ui_DistanceMatrixMSAProfileDialog@@QAEXPAVQDialog@@@Z$6 10017da1 f   DistanceMatrixMSAProfileDialog.obj
 0001:00016dac       __unwindfunclet$?setupUi@Ui_DistanceMatrixMSAProfileDialog@@QAEXPAVQDialog@@@Z$7 10017dac f   DistanceMatrixMSAProfileDialog.obj
 0001:00016db5       __unwindfunclet$?setupUi@Ui_DistanceMatrixMSAProfileDialog@@QAEXPAVQDialog@@@Z$8 10017db5 f   DistanceMatrixMSAProfileDialog.obj
 0001:00016dc0       __unwindfunclet$?setupUi@Ui_DistanceMatrixMSAProfileDialog@@QAEXPAVQDialog@@@Z$9 10017dc0 f   DistanceMatrixMSAProfileDialog.obj
 0001:00016dc9       __unwindfunclet$?setupUi@Ui_DistanceMatrixMSAProfileDialog@@QAEXPAVQDialog@@@Z$10 10017dc9 f   DistanceMatrixMSAProfileDialog.obj
 0001:00016dd4       __unwindfunclet$?setupUi@Ui_DistanceMatrixMSAProfileDialog@@QAEXPAVQDialog@@@Z$11 10017dd4 f   DistanceMatrixMSAProfileDialog.obj
 0001:00016ddd       __unwindfunclet$?setupUi@Ui_DistanceMatrixMSAProfileDialog@@QAEXPAVQDialog@@@Z$12 10017ddd f   DistanceMatrixMSAProfileDialog.obj
 0001:00016de8       __unwindfunclet$?setupUi@Ui_DistanceMatrixMSAProfileDialog@@QAEXPAVQDialog@@@Z$13 10017de8 f   DistanceMatrixMSAProfileDialog.obj
 0001:00016df1       __unwindfunclet$?setupUi@Ui_DistanceMatrixMSAProfileDialog@@QAEXPAVQDialog@@@Z$14 10017df1 f   DistanceMatrixMSAProfileDialog.obj
 0001:00016dfc       __unwindfunclet$?setupUi@Ui_DistanceMatrixMSAProfileDialog@@QAEXPAVQDialog@@@Z$15 10017dfc f   DistanceMatrixMSAProfileDialog.obj
 0001:00016e05       __unwindfunclet$?setupUi@Ui_DistanceMatrixMSAProfileDialog@@QAEXPAVQDialog@@@Z$16 10017e05 f   DistanceMatrixMSAProfileDialog.obj
 0001:00016e10       __unwindfunclet$?setupUi@Ui_DistanceMatrixMSAProfileDialog@@QAEXPAVQDialog@@@Z$17 10017e10 f   DistanceMatrixMSAProfileDialog.obj
 0001:00016e19       __unwindfunclet$?setupUi@Ui_DistanceMatrixMSAProfileDialog@@QAEXPAVQDialog@@@Z$18 10017e19 f   DistanceMatrixMSAProfileDialog.obj
 0001:00016e24       __unwindfunclet$?setupUi@Ui_DistanceMatrixMSAProfileDialog@@QAEXPAVQDialog@@@Z$19 10017e24 f   DistanceMatrixMSAProfileDialog.obj
 0001:00016e2d       __unwindfunclet$?setupUi@Ui_DistanceMatrixMSAProfileDialog@@QAEXPAVQDialog@@@Z$20 10017e2d f   DistanceMatrixMSAProfileDialog.obj
 0001:00016e38       __unwindfunclet$?setupUi@Ui_DistanceMatrixMSAProfileDialog@@QAEXPAVQDialog@@@Z$21 10017e38 f   DistanceMatrixMSAProfileDialog.obj
 0001:00016e41       __unwindfunclet$?setupUi@Ui_DistanceMatrixMSAProfileDialog@@QAEXPAVQDialog@@@Z$22 10017e41 f   DistanceMatrixMSAProfileDialog.obj
 0001:00016e4c       __unwindfunclet$?setupUi@Ui_DistanceMatrixMSAProfileDialog@@QAEXPAVQDialog@@@Z$23 10017e4c f   DistanceMatrixMSAProfileDialog.obj
 0001:00016e55       __unwindfunclet$?setupUi@Ui_DistanceMatrixMSAProfileDialog@@QAEXPAVQDialog@@@Z$24 10017e55 f   DistanceMatrixMSAProfileDialog.obj
 0001:00016e60       __unwindfunclet$?setupUi@Ui_DistanceMatrixMSAProfileDialog@@QAEXPAVQDialog@@@Z$25 10017e60 f   DistanceMatrixMSAProfileDialog.obj
 0001:00016e69       __unwindfunclet$?setupUi@Ui_DistanceMatrixMSAProfileDialog@@QAEXPAVQDialog@@@Z$26 10017e69 f   DistanceMatrixMSAProfileDialog.obj
 0001:00016e74       __unwindfunclet$?setupUi@Ui_DistanceMatrixMSAProfileDialog@@QAEXPAVQDialog@@@Z$27 10017e74 f   DistanceMatrixMSAProfileDialog.obj
 0001:00016e7d       __unwindfunclet$?setupUi@Ui_DistanceMatrixMSAProfileDialog@@QAEXPAVQDialog@@@Z$28 10017e7d f   DistanceMatrixMSAProfileDialog.obj
 0001:00016e88       __unwindfunclet$?setupUi@Ui_DistanceMatrixMSAProfileDialog@@QAEXPAVQDialog@@@Z$29 10017e88 f   DistanceMatrixMSAProfileDialog.obj
 0001:00016e91       __unwindfunclet$?setupUi@Ui_DistanceMatrixMSAProfileDialog@@QAEXPAVQDialog@@@Z$30 10017e91 f   DistanceMatrixMSAProfileDialog.obj
 0001:00016e9c       __unwindfunclet$?setupUi@Ui_DistanceMatrixMSAProfileDialog@@QAEXPAVQDialog@@@Z$31 10017e9c f   DistanceMatrixMSAProfileDialog.obj
 0001:00016ea5       __unwindfunclet$?setupUi@Ui_DistanceMatrixMSAProfileDialog@@QAEXPAVQDialog@@@Z$32 10017ea5 f   DistanceMatrixMSAProfileDialog.obj
 0001:00016eb0       __unwindfunclet$?setupUi@Ui_DistanceMatrixMSAProfileDialog@@QAEXPAVQDialog@@@Z$33 10017eb0 f   DistanceMatrixMSAProfileDialog.obj
 0001:00016eb9       __unwindfunclet$?setupUi@Ui_DistanceMatrixMSAProfileDialog@@QAEXPAVQDialog@@@Z$34 10017eb9 f   DistanceMatrixMSAProfileDialog.obj
 0001:00016ec4       __unwindfunclet$?setupUi@Ui_DistanceMatrixMSAProfileDialog@@QAEXPAVQDialog@@@Z$35 10017ec4 f   DistanceMatrixMSAProfileDialog.obj
 0001:00016ecd       __unwindfunclet$?setupUi@Ui_DistanceMatrixMSAProfileDialog@@QAEXPAVQDialog@@@Z$36 10017ecd f   DistanceMatrixMSAProfileDialog.obj
 0001:00016ed8       __unwindfunclet$?setupUi@Ui_DistanceMatrixMSAProfileDialog@@QAEXPAVQDialog@@@Z$37 10017ed8 f   DistanceMatrixMSAProfileDialog.obj
 0001:00016ee3       __unwindfunclet$?setupUi@Ui_DistanceMatrixMSAProfileDialog@@QAEXPAVQDialog@@@Z$38 10017ee3 f   DistanceMatrixMSAProfileDialog.obj
 0001:00016eec       __ehhandler$?setupUi@Ui_DistanceMatrixMSAProfileDialog@@QAEXPAVQDialog@@@Z 10017eec f   DistanceMatrixMSAProfileDialog.obj
 0001:00016f10       __unwindfunclet$??__EalgoLog@U2@@YAXXZ$0 10017f10 f   moc_DNAStatMSAProfileDialog.obj
 0001:00016f19       __ehhandler$??__EalgoLog@U2@@YAXXZ 10017f19 f   moc_DNAStatMSAProfileDialog.obj
 0001:00016f40       __unwindfunclet$??__EcmdLog@U2@@YAXXZ$0 10017f40 f   moc_DNAStatMSAProfileDialog.obj
 0001:00016f49       __ehhandler$??__EcmdLog@U2@@YAXXZ 10017f49 f   moc_DNAStatMSAProfileDialog.obj
 0001:00016f70       __unwindfunclet$??__EcoreLog@U2@@YAXXZ$0 10017f70 f   moc_DNAStatMSAProfileDialog.obj
 0001:00016f79       __ehhandler$??__EcoreLog@U2@@YAXXZ 10017f79 f   moc_DNAStatMSAProfileDialog.obj
 0001:00016fa0       __unwindfunclet$??__EioLog@U2@@YAXXZ$0 10017fa0 f   moc_DNAStatMSAProfileDialog.obj
 0001:00016fa9       __ehhandler$??__EioLog@U2@@YAXXZ 10017fa9 f   moc_DNAStatMSAProfileDialog.obj
 0001:00016fd0       __unwindfunclet$??__EperfLog@U2@@YAXXZ$0 10017fd0 f   moc_DNAStatMSAProfileDialog.obj
 0001:00016fd9       __ehhandler$??__EperfLog@U2@@YAXXZ 10017fd9 f   moc_DNAStatMSAProfileDialog.obj
 0001:00017000       __unwindfunclet$??__EscriptLog@U2@@YAXXZ$0 10018000 f   moc_DNAStatMSAProfileDialog.obj
 0001:00017009       __ehhandler$??__EscriptLog@U2@@YAXXZ 10018009 f   moc_DNAStatMSAProfileDialog.obj
 0001:00017030       __unwindfunclet$??__EtaskLog@U2@@YAXXZ$0 10018030 f   moc_DNAStatMSAProfileDialog.obj
 0001:00017039       __ehhandler$??__EtaskLog@U2@@YAXXZ 10018039 f   moc_DNAStatMSAProfileDialog.obj
 0001:00017060       __unwindfunclet$??__EuiLog@U2@@YAXXZ$0 10018060 f   moc_DNAStatMSAProfileDialog.obj
 0001:00017069       __ehhandler$??__EuiLog@U2@@YAXXZ 10018069 f   moc_DNAStatMSAProfileDialog.obj
 0001:00017090       __unwindfunclet$??__EuserActLog@U2@@YAXXZ$0 10018090 f   moc_DNAStatMSAProfileDialog.obj
 0001:00017099       __ehhandler$??__EuserActLog@U2@@YAXXZ 10018099 f   moc_DNAStatMSAProfileDialog.obj
 0001:000170c0       __unwindfunclet$?qt_metatype_id@?$QMetaTypeIdQObject@PAVGObjectView@U2@@$00@@SAHXZ$0 100180c0 f   moc_DNAStatPlugin.obj
 0001:000170c9       __ehhandler$?qt_metatype_id@?$QMetaTypeIdQObject@PAVGObjectView@U2@@$00@@SAHXZ 100180c9 f   moc_DNAStatPlugin.obj
 0001:000170f0       __unwindfunclet$?qt_metatype_id@?$QMetaTypeIdQObject@PAVQMenu@@$00@@SAHXZ$0 100180f0 f   moc_DNAStatPlugin.obj
 0001:000170f9       __ehhandler$?qt_metatype_id@?$QMetaTypeIdQObject@PAVQMenu@@$00@@SAHXZ 100180f9 f   moc_DNAStatPlugin.obj
 0001:00017120       __unwindfunclet$??__EalgoLog@U2@@YAXXZ$0 10018120 f   moc_DNAStatProfileTask.obj
 0001:00017129       __ehhandler$??__EalgoLog@U2@@YAXXZ 10018129 f   moc_DNAStatProfileTask.obj
 0001:00017150       __unwindfunclet$??__EcmdLog@U2@@YAXXZ$0 10018150 f   moc_DNAStatProfileTask.obj
 0001:00017159       __ehhandler$??__EcmdLog@U2@@YAXXZ 10018159 f   moc_DNAStatProfileTask.obj
 0001:00017180       __unwindfunclet$??__EcoreLog@U2@@YAXXZ$0 10018180 f   moc_DNAStatProfileTask.obj
 0001:00017189       __ehhandler$??__EcoreLog@U2@@YAXXZ 10018189 f   moc_DNAStatProfileTask.obj
 0001:000171b0       __unwindfunclet$??__EioLog@U2@@YAXXZ$0 100181b0 f   moc_DNAStatProfileTask.obj
 0001:000171b9       __ehhandler$??__EioLog@U2@@YAXXZ 100181b9 f   moc_DNAStatProfileTask.obj
 0001:000171e0       __unwindfunclet$??__EperfLog@U2@@YAXXZ$0 100181e0 f   moc_DNAStatProfileTask.obj
 0001:000171e9       __ehhandler$??__EperfLog@U2@@YAXXZ 100181e9 f   moc_DNAStatProfileTask.obj
 0001:00017210       __unwindfunclet$??__EscriptLog@U2@@YAXXZ$0 10018210 f   moc_DNAStatProfileTask.obj
 0001:00017219       __ehhandler$??__EscriptLog@U2@@YAXXZ 10018219 f   moc_DNAStatProfileTask.obj
 0001:00017240       __unwindfunclet$??__EtaskLog@U2@@YAXXZ$0 10018240 f   moc_DNAStatProfileTask.obj
 0001:00017249       __ehhandler$??__EtaskLog@U2@@YAXXZ 10018249 f   moc_DNAStatProfileTask.obj
 0001:00017270       __unwindfunclet$??__EuiLog@U2@@YAXXZ$0 10018270 f   moc_DNAStatProfileTask.obj
 0001:00017279       __ehhandler$??__EuiLog@U2@@YAXXZ 10018279 f   moc_DNAStatProfileTask.obj
 0001:000172a0       __unwindfunclet$??__EuserActLog@U2@@YAXXZ$0 100182a0 f   moc_DNAStatProfileTask.obj
 0001:000172a9       __ehhandler$??__EuserActLog@U2@@YAXXZ 100182a9 f   moc_DNAStatProfileTask.obj
 0001:000172d0       __unwindfunclet$??__EalgoLog@U2@@YAXXZ$0 100182d0 f   moc_DistanceMatrixMSAProfileDialog.obj
 0001:000172d9       __ehhandler$??__EalgoLog@U2@@YAXXZ 100182d9 f   moc_DistanceMatrixMSAProfileDialog.obj
 0001:00017300       __unwindfunclet$??__EcmdLog@U2@@YAXXZ$0 10018300 f   moc_DistanceMatrixMSAProfileDialog.obj
 0001:00017309       __ehhandler$??__EcmdLog@U2@@YAXXZ 10018309 f   moc_DistanceMatrixMSAProfileDialog.obj
 0001:00017330       __unwindfunclet$??__EcoreLog@U2@@YAXXZ$0 10018330 f   moc_DistanceMatrixMSAProfileDialog.obj
 0001:00017339       __ehhandler$??__EcoreLog@U2@@YAXXZ 10018339 f   moc_DistanceMatrixMSAProfileDialog.obj
 0001:00017360       __unwindfunclet$??__EioLog@U2@@YAXXZ$0 10018360 f   moc_DistanceMatrixMSAProfileDialog.obj
 0001:00017369       __ehhandler$??__EioLog@U2@@YAXXZ 10018369 f   moc_DistanceMatrixMSAProfileDialog.obj
 0001:00017390       __unwindfunclet$??__EperfLog@U2@@YAXXZ$0 10018390 f   moc_DistanceMatrixMSAProfileDialog.obj
 0001:00017399       __ehhandler$??__EperfLog@U2@@YAXXZ 10018399 f   moc_DistanceMatrixMSAProfileDialog.obj
 0001:000173c0       __unwindfunclet$??__EscriptLog@U2@@YAXXZ$0 100183c0 f   moc_DistanceMatrixMSAProfileDialog.obj
 0001:000173c9       __ehhandler$??__EscriptLog@U2@@YAXXZ 100183c9 f   moc_DistanceMatrixMSAProfileDialog.obj
 0001:000173f0       __unwindfunclet$??__EtaskLog@U2@@YAXXZ$0 100183f0 f   moc_DistanceMatrixMSAProfileDialog.obj
 0001:000173f9       __ehhandler$??__EtaskLog@U2@@YAXXZ 100183f9 f   moc_DistanceMatrixMSAProfileDialog.obj
 0001:00017420       __unwindfunclet$??__EuiLog@U2@@YAXXZ$0 10018420 f   moc_DistanceMatrixMSAProfileDialog.obj
 0001:00017429       __ehhandler$??__EuiLog@U2@@YAXXZ 10018429 f   moc_DistanceMatrixMSAProfileDialog.obj
 0001:00017450       __unwindfunclet$??__EuserActLog@U2@@YAXXZ$0 10018450 f   moc_DistanceMatrixMSAProfileDialog.obj
 0001:00017459       __ehhandler$??__EuserActLog@U2@@YAXXZ 10018459 f   moc_DistanceMatrixMSAProfileDialog.obj
 0001:00017480       ??__F?CSV@DNAStatMSAProfileDialog@U2@@0VQString@@B@@YAXXZ 10018480 f   DNAStatMSAProfileDialog.obj
 0001:00017490       ??__F?HTML@DNAStatMSAProfileDialog@U2@@0VQString@@B@@YAXXZ 10018490 f   DNAStatMSAProfileDialog.obj
 0001:000174a0       ??__F?_Generic_object@?$_Error_objects@H@std@@2V_Generic_error_category@2@A@@YAXXZ 100184a0 f   DNAStatMSAProfileDialog.obj
 0001:000174b0       ??__F?_Iostream_object@?$_Error_objects@H@std@@2V_Iostream_error_category@2@A@@YAXXZ 100184b0 f   DNAStatMSAProfileDialog.obj
 0001:000174c0       ??__F?_System_object@?$_Error_objects@H@std@@2V_System_error_category@2@A@@YAXXZ 100184c0 f   DNAStatMSAProfileDialog.obj
 0001:000174d0       ??__FService_DNAExport@U2@@YAXXZ 100184d0 f   DNAStatMSAProfileDialog.obj
 0001:000174e0       ??__FService_DNAGraphPack@U2@@YAXXZ 100184e0 f   DNAStatMSAProfileDialog.obj
 0001:000174f0       ??__FService_ExternalToolSupport@U2@@YAXXZ 100184f0 f   DNAStatMSAProfileDialog.obj
 0001:00017500       ??__FService_GUITesting@U2@@YAXXZ 10018500 f   DNAStatMSAProfileDialog.obj
 0001:00017510       ??__FService_MaxCoreServiceId@U2@@YAXXZ 10018510 f   DNAStatMSAProfileDialog.obj
 0001:00017520       ??__FService_MinCoreServiceId@U2@@YAXXZ 10018520 f   DNAStatMSAProfileDialog.obj
 0001:00017530       ??__FService_PluginViewer@U2@@YAXXZ 10018530 f   DNAStatMSAProfileDialog.obj
 0001:00017540       ??__FService_Project@U2@@YAXXZ 10018540 f   DNAStatMSAProfileDialog.obj
 0001:00017550       ??__FService_ProjectView@U2@@YAXXZ 10018550 f   DNAStatMSAProfileDialog.obj
 0001:00017560       ??__FService_QueryDesigner@U2@@YAXXZ 10018560 f   DNAStatMSAProfileDialog.obj
 0001:00017570       ??__FService_ScriptRegistry@U2@@YAXXZ 10018570 f   DNAStatMSAProfileDialog.obj
 0001:00017580       ??__FService_TestRunner@U2@@YAXXZ 10018580 f   DNAStatMSAProfileDialog.obj
 0001:00017590       ??__FService_WorkflowDesigner@U2@@YAXXZ 10018590 f   DNAStatMSAProfileDialog.obj
 0001:000175a0       ??__FalgoLog@U2@@YAXXZ     100185a0 f   DNAStatMSAProfileDialog.obj
 0001:000175b0       ??__FcmdLog@U2@@YAXXZ      100185b0 f   DNAStatMSAProfileDialog.obj
 0001:000175c0       ??__FcoreLog@U2@@YAXXZ     100185c0 f   DNAStatMSAProfileDialog.obj
 0001:000175d0       ??__FioLog@U2@@YAXXZ       100185d0 f   DNAStatMSAProfileDialog.obj
 0001:000175e0       ??__FperfLog@U2@@YAXXZ     100185e0 f   DNAStatMSAProfileDialog.obj
 0001:000175f0       ??__FscriptLog@U2@@YAXXZ   100185f0 f   DNAStatMSAProfileDialog.obj
 0001:00017600       ??__FtaskLog@U2@@YAXXZ     10018600 f   DNAStatMSAProfileDialog.obj
 0001:00017610       ??__FuiLog@U2@@YAXXZ       10018610 f   DNAStatMSAProfileDialog.obj
 0001:00017620       ??__FuserActLog@U2@@YAXXZ  10018620 f   DNAStatMSAProfileDialog.obj
 0001:00017630       ??__F?_Generic_object@?$_Error_objects@H@std@@2V_Generic_error_category@2@A@@YAXXZ 10018630 f   DNAStatPlugin.obj
 0001:00017640       ??__F?_Iostream_object@?$_Error_objects@H@std@@2V_Iostream_error_category@2@A@@YAXXZ 10018640 f   DNAStatPlugin.obj
 0001:00017650       ??__F?_System_object@?$_Error_objects@H@std@@2V_System_error_category@2@A@@YAXXZ 10018650 f   DNAStatPlugin.obj
 0001:00017660       ??__FService_DNAExport@U2@@YAXXZ 10018660 f   DNAStatPlugin.obj
 0001:00017670       ??__FService_DNAGraphPack@U2@@YAXXZ 10018670 f   DNAStatPlugin.obj
 0001:00017680       ??__FService_ExternalToolSupport@U2@@YAXXZ 10018680 f   DNAStatPlugin.obj
 0001:00017690       ??__FService_GUITesting@U2@@YAXXZ 10018690 f   DNAStatPlugin.obj
 0001:000176a0       ??__FService_MaxCoreServiceId@U2@@YAXXZ 100186a0 f   DNAStatPlugin.obj
 0001:000176b0       ??__FService_MinCoreServiceId@U2@@YAXXZ 100186b0 f   DNAStatPlugin.obj
 0001:000176c0       ??__FService_PluginViewer@U2@@YAXXZ 100186c0 f   DNAStatPlugin.obj
 0001:000176d0       ??__FService_Project@U2@@YAXXZ 100186d0 f   DNAStatPlugin.obj
 0001:000176e0       ??__FService_ProjectView@U2@@YAXXZ 100186e0 f   DNAStatPlugin.obj
 0001:000176f0       ??__FService_QueryDesigner@U2@@YAXXZ 100186f0 f   DNAStatPlugin.obj
 0001:00017700       ??__FService_ScriptRegistry@U2@@YAXXZ 10018700 f   DNAStatPlugin.obj
 0001:00017710       ??__FService_TestRunner@U2@@YAXXZ 10018710 f   DNAStatPlugin.obj
 0001:00017720       ??__FService_WorkflowDesigner@U2@@YAXXZ 10018720 f   DNAStatPlugin.obj
 0001:00017730       ??__FalgoLog@U2@@YAXXZ     10018730 f   DNAStatPlugin.obj
 0001:00017740       ??__FcmdLog@U2@@YAXXZ      10018740 f   DNAStatPlugin.obj
 0001:00017750       ??__FcoreLog@U2@@YAXXZ     10018750 f   DNAStatPlugin.obj
 0001:00017760       ??__FioLog@U2@@YAXXZ       10018760 f   DNAStatPlugin.obj
 0001:00017770       ??__FperfLog@U2@@YAXXZ     10018770 f   DNAStatPlugin.obj
 0001:00017780       ??__FscriptLog@U2@@YAXXZ   10018780 f   DNAStatPlugin.obj
 0001:00017790       ??__FtaskLog@U2@@YAXXZ     10018790 f   DNAStatPlugin.obj
 0001:000177a0       ??__FuiLog@U2@@YAXXZ       100187a0 f   DNAStatPlugin.obj
 0001:000177b0       ??__FuserActLog@U2@@YAXXZ  100187b0 f   DNAStatPlugin.obj
 0001:000177c0       ??__F?_Generic_object@?$_Error_objects@H@std@@2V_Generic_error_category@2@A@@YAXXZ 100187c0 f   DNAStatProfileTask.obj
 0001:000177d0       ??__F?_Iostream_object@?$_Error_objects@H@std@@2V_Iostream_error_category@2@A@@YAXXZ 100187d0 f   DNAStatProfileTask.obj
 0001:000177e0       ??__F?_System_object@?$_Error_objects@H@std@@2V_System_error_category@2@A@@YAXXZ 100187e0 f   DNAStatProfileTask.obj
 0001:000177f0       ??__FService_DNAExport@U2@@YAXXZ 100187f0 f   DNAStatProfileTask.obj
 0001:00017800       ??__FService_DNAGraphPack@U2@@YAXXZ 10018800 f   DNAStatProfileTask.obj
 0001:00017810       ??__FService_ExternalToolSupport@U2@@YAXXZ 10018810 f   DNAStatProfileTask.obj
 0001:00017820       ??__FService_GUITesting@U2@@YAXXZ 10018820 f   DNAStatProfileTask.obj
 0001:00017830       ??__FService_MaxCoreServiceId@U2@@YAXXZ 10018830 f   DNAStatProfileTask.obj
 0001:00017840       ??__FService_MinCoreServiceId@U2@@YAXXZ 10018840 f   DNAStatProfileTask.obj
 0001:00017850       ??__FService_PluginViewer@U2@@YAXXZ 10018850 f   DNAStatProfileTask.obj
 0001:00017860       ??__FService_Project@U2@@YAXXZ 10018860 f   DNAStatProfileTask.obj
 0001:00017870       ??__FService_ProjectView@U2@@YAXXZ 10018870 f   DNAStatProfileTask.obj
 0001:00017880       ??__FService_QueryDesigner@U2@@YAXXZ 10018880 f   DNAStatProfileTask.obj
 0001:00017890       ??__FService_ScriptRegistry@U2@@YAXXZ 10018890 f   DNAStatProfileTask.obj
 0001:000178a0       ??__FService_TestRunner@U2@@YAXXZ 100188a0 f   DNAStatProfileTask.obj
 0001:000178b0       ??__FService_WorkflowDesigner@U2@@YAXXZ 100188b0 f   DNAStatProfileTask.obj
 0001:000178c0       ??__FalgoLog@U2@@YAXXZ     100188c0 f   DNAStatProfileTask.obj
 0001:000178d0       ??__FcmdLog@U2@@YAXXZ      100188d0 f   DNAStatProfileTask.obj
 0001:000178e0       ??__FcoreLog@U2@@YAXXZ     100188e0 f   DNAStatProfileTask.obj
 0001:000178f0       ??__FioLog@U2@@YAXXZ       100188f0 f   DNAStatProfileTask.obj
 0001:00017900       ??__FperfLog@U2@@YAXXZ     10018900 f   DNAStatProfileTask.obj
 0001:00017910       ??__FscriptLog@U2@@YAXXZ   10018910 f   DNAStatProfileTask.obj
 0001:00017920       ??__FtaskLog@U2@@YAXXZ     10018920 f   DNAStatProfileTask.obj
 0001:00017930       ??__FuiLog@U2@@YAXXZ       10018930 f   DNAStatProfileTask.obj
 0001:00017940       ??__FuserActLog@U2@@YAXXZ  10018940 f   DNAStatProfileTask.obj
 0001:00017950       ??__F?CSV@DistanceMatrixMSAProfileDialog@U2@@0VQString@@B@@YAXXZ 10018950 f   DistanceMatrixMSAProfileDialog.obj
 0001:00017960       ??__F?HTML@DistanceMatrixMSAProfileDialog@U2@@0VQString@@B@@YAXXZ 10018960 f   DistanceMatrixMSAProfileDialog.obj
 0001:00017970       ??__F?_Generic_object@?$_Error_objects@H@std@@2V_Generic_error_category@2@A@@YAXXZ 10018970 f   DistanceMatrixMSAProfileDialog.obj
 0001:00017980       ??__F?_Iostream_object@?$_Error_objects@H@std@@2V_Iostream_error_category@2@A@@YAXXZ 10018980 f   DistanceMatrixMSAProfileDialog.obj
 0001:00017990       ??__F?_System_object@?$_Error_objects@H@std@@2V_System_error_category@2@A@@YAXXZ 10018990 f   DistanceMatrixMSAProfileDialog.obj
 0001:000179a0       ??__FService_DNAExport@U2@@YAXXZ 100189a0 f   DistanceMatrixMSAProfileDialog.obj
 0001:000179b0       ??__FService_DNAGraphPack@U2@@YAXXZ 100189b0 f   DistanceMatrixMSAProfileDialog.obj
 0001:000179c0       ??__FService_ExternalToolSupport@U2@@YAXXZ 100189c0 f   DistanceMatrixMSAProfileDialog.obj
 0001:000179d0       ??__FService_GUITesting@U2@@YAXXZ 100189d0 f   DistanceMatrixMSAProfileDialog.obj
 0001:000179e0       ??__FService_MaxCoreServiceId@U2@@YAXXZ 100189e0 f   DistanceMatrixMSAProfileDialog.obj
 0001:000179f0       ??__FService_MinCoreServiceId@U2@@YAXXZ 100189f0 f   DistanceMatrixMSAProfileDialog.obj
 0001:00017a00       ??__FService_PluginViewer@U2@@YAXXZ 10018a00 f   DistanceMatrixMSAProfileDialog.obj
 0001:00017a10       ??__FService_Project@U2@@YAXXZ 10018a10 f   DistanceMatrixMSAProfileDialog.obj
 0001:00017a20       ??__FService_ProjectView@U2@@YAXXZ 10018a20 f   DistanceMatrixMSAProfileDialog.obj
 0001:00017a30       ??__FService_QueryDesigner@U2@@YAXXZ 10018a30 f   DistanceMatrixMSAProfileDialog.obj
 0001:00017a40       ??__FService_ScriptRegistry@U2@@YAXXZ 10018a40 f   DistanceMatrixMSAProfileDialog.obj
 0001:00017a50       ??__FService_TestRunner@U2@@YAXXZ 10018a50 f   DistanceMatrixMSAProfileDialog.obj
 0001:00017a60       ??__FService_WorkflowDesigner@U2@@YAXXZ 10018a60 f   DistanceMatrixMSAProfileDialog.obj
 0001:00017a70       ??__FalgoLog@U2@@YAXXZ     10018a70 f   DistanceMatrixMSAProfileDialog.obj
 0001:00017a80       ??__FcmdLog@U2@@YAXXZ      10018a80 f   DistanceMatrixMSAProfileDialog.obj
 0001:00017a90       ??__FcoreLog@U2@@YAXXZ     10018a90 f   DistanceMatrixMSAProfileDialog.obj
 0001:00017aa0       ??__FioLog@U2@@YAXXZ       10018aa0 f   DistanceMatrixMSAProfileDialog.obj
 0001:00017ab0       ??__FperfLog@U2@@YAXXZ     10018ab0 f   DistanceMatrixMSAProfileDialog.obj
 0001:00017ac0       ??__FscriptLog@U2@@YAXXZ   10018ac0 f   DistanceMatrixMSAProfileDialog.obj
 0001:00017ad0       ??__FtaskLog@U2@@YAXXZ     10018ad0 f   DistanceMatrixMSAProfileDialog.obj
 0001:00017ae0       ??__FuiLog@U2@@YAXXZ       10018ae0 f   DistanceMatrixMSAProfileDialog.obj
 0001:00017af0       ??__FuserActLog@U2@@YAXXZ  10018af0 f   DistanceMatrixMSAProfileDialog.obj
 0001:00017b00       ??__F?_Generic_object@?$_Error_objects@H@std@@2V_Generic_error_category@2@A@@YAXXZ 10018b00 f   moc_DNAStatMSAProfileDialog.obj
 0001:00017b10       ??__F?_Iostream_object@?$_Error_objects@H@std@@2V_Iostream_error_category@2@A@@YAXXZ 10018b10 f   moc_DNAStatMSAProfileDialog.obj
 0001:00017b20       ??__F?_System_object@?$_Error_objects@H@std@@2V_System_error_category@2@A@@YAXXZ 10018b20 f   moc_DNAStatMSAProfileDialog.obj
 0001:00017b30       ??__FalgoLog@U2@@YAXXZ     10018b30 f   moc_DNAStatMSAProfileDialog.obj
 0001:00017b40       ??__FcmdLog@U2@@YAXXZ      10018b40 f   moc_DNAStatMSAProfileDialog.obj
 0001:00017b50       ??__FcoreLog@U2@@YAXXZ     10018b50 f   moc_DNAStatMSAProfileDialog.obj
 0001:00017b60       ??__FioLog@U2@@YAXXZ       10018b60 f   moc_DNAStatMSAProfileDialog.obj
 0001:00017b70       ??__FperfLog@U2@@YAXXZ     10018b70 f   moc_DNAStatMSAProfileDialog.obj
 0001:00017b80       ??__FscriptLog@U2@@YAXXZ   10018b80 f   moc_DNAStatMSAProfileDialog.obj
 0001:00017b90       ??__FtaskLog@U2@@YAXXZ     10018b90 f   moc_DNAStatMSAProfileDialog.obj
 0001:00017ba0       ??__FuiLog@U2@@YAXXZ       10018ba0 f   moc_DNAStatMSAProfileDialog.obj
 0001:00017bb0       ??__FuserActLog@U2@@YAXXZ  10018bb0 f   moc_DNAStatMSAProfileDialog.obj
 0001:00017bc0       ??__F?_Generic_object@?$_Error_objects@H@std@@2V_Generic_error_category@2@A@@YAXXZ 10018bc0 f   moc_DNAStatPlugin.obj
 0001:00017bd0       ??__F?_Iostream_object@?$_Error_objects@H@std@@2V_Iostream_error_category@2@A@@YAXXZ 10018bd0 f   moc_DNAStatPlugin.obj
 0001:00017be0       ??__F?_System_object@?$_Error_objects@H@std@@2V_System_error_category@2@A@@YAXXZ 10018be0 f   moc_DNAStatPlugin.obj
 0001:00017bf0       ??__FService_DNAExport@U2@@YAXXZ 10018bf0 f   moc_DNAStatPlugin.obj
 0001:00017c00       ??__FService_DNAGraphPack@U2@@YAXXZ 10018c00 f   moc_DNAStatPlugin.obj
 0001:00017c10       ??__FService_ExternalToolSupport@U2@@YAXXZ 10018c10 f   moc_DNAStatPlugin.obj
 0001:00017c20       ??__FService_GUITesting@U2@@YAXXZ 10018c20 f   moc_DNAStatPlugin.obj
 0001:00017c30       ??__FService_MaxCoreServiceId@U2@@YAXXZ 10018c30 f   moc_DNAStatPlugin.obj
 0001:00017c40       ??__FService_MinCoreServiceId@U2@@YAXXZ 10018c40 f   moc_DNAStatPlugin.obj
 0001:00017c50       ??__FService_PluginViewer@U2@@YAXXZ 10018c50 f   moc_DNAStatPlugin.obj
 0001:00017c60       ??__FService_Project@U2@@YAXXZ 10018c60 f   moc_DNAStatPlugin.obj
 0001:00017c70       ??__FService_ProjectView@U2@@YAXXZ 10018c70 f   moc_DNAStatPlugin.obj
 0001:00017c80       ??__FService_QueryDesigner@U2@@YAXXZ 10018c80 f   moc_DNAStatPlugin.obj
 0001:00017c90       ??__FService_ScriptRegistry@U2@@YAXXZ 10018c90 f   moc_DNAStatPlugin.obj
 0001:00017ca0       ??__FService_TestRunner@U2@@YAXXZ 10018ca0 f   moc_DNAStatPlugin.obj
 0001:00017cb0       ??__FService_WorkflowDesigner@U2@@YAXXZ 10018cb0 f   moc_DNAStatPlugin.obj
 0001:00017cc0       ??__F?_Generic_object@?$_Error_objects@H@std@@2V_Generic_error_category@2@A@@YAXXZ 10018cc0 f   moc_DNAStatProfileTask.obj
 0001:00017cd0       ??__F?_Iostream_object@?$_Error_objects@H@std@@2V_Iostream_error_category@2@A@@YAXXZ 10018cd0 f   moc_DNAStatProfileTask.obj
 0001:00017ce0       ??__F?_System_object@?$_Error_objects@H@std@@2V_System_error_category@2@A@@YAXXZ 10018ce0 f   moc_DNAStatProfileTask.obj
 0001:00017cf0       ??__FalgoLog@U2@@YAXXZ     10018cf0 f   moc_DNAStatProfileTask.obj
 0001:00017d00       ??__FcmdLog@U2@@YAXXZ      10018d00 f   moc_DNAStatProfileTask.obj
 0001:00017d10       ??__FcoreLog@U2@@YAXXZ     10018d10 f   moc_DNAStatProfileTask.obj
 0001:00017d20       ??__FioLog@U2@@YAXXZ       10018d20 f   moc_DNAStatProfileTask.obj
 0001:00017d30       ??__FperfLog@U2@@YAXXZ     10018d30 f   moc_DNAStatProfileTask.obj
 0001:00017d40       ??__FscriptLog@U2@@YAXXZ   10018d40 f   moc_DNAStatProfileTask.obj
 0001:00017d50       ??__FtaskLog@U2@@YAXXZ     10018d50 f   moc_DNAStatProfileTask.obj
 0001:00017d60       ??__FuiLog@U2@@YAXXZ       10018d60 f   moc_DNAStatProfileTask.obj
 0001:00017d70       ??__FuserActLog@U2@@YAXXZ  10018d70 f   moc_DNAStatProfileTask.obj
 0001:00017d80       ??__F?_Generic_object@?$_Error_objects@H@std@@2V_Generic_error_category@2@A@@YAXXZ 10018d80 f   moc_DistanceMatrixMSAProfileDialog.obj
 0001:00017d90       ??__F?_Iostream_object@?$_Error_objects@H@std@@2V_Iostream_error_category@2@A@@YAXXZ 10018d90 f   moc_DistanceMatrixMSAProfileDialog.obj
 0001:00017da0       ??__F?_System_object@?$_Error_objects@H@std@@2V_System_error_category@2@A@@YAXXZ 10018da0 f   moc_DistanceMatrixMSAProfileDialog.obj
 0001:00017db0       ??__FalgoLog@U2@@YAXXZ     10018db0 f   moc_DistanceMatrixMSAProfileDialog.obj
 0001:00017dc0       ??__FcmdLog@U2@@YAXXZ      10018dc0 f   moc_DistanceMatrixMSAProfileDialog.obj
 0001:00017dd0       ??__FcoreLog@U2@@YAXXZ     10018dd0 f   moc_DistanceMatrixMSAProfileDialog.obj
 0001:00017de0       ??__FioLog@U2@@YAXXZ       10018de0 f   moc_DistanceMatrixMSAProfileDialog.obj
 0001:00017df0       ??__FperfLog@U2@@YAXXZ     10018df0 f   moc_DistanceMatrixMSAProfileDialog.obj
 0001:00017e00       ??__FscriptLog@U2@@YAXXZ   10018e00 f   moc_DistanceMatrixMSAProfileDialog.obj
 0001:00017e10       ??__FtaskLog@U2@@YAXXZ     10018e10 f   moc_DistanceMatrixMSAProfileDialog.obj
 0001:00017e20       ??__FuiLog@U2@@YAXXZ       10018e20 f   moc_DistanceMatrixMSAProfileDialog.obj
 0001:00017e30       ??__FuserActLog@U2@@YAXXZ  10018e30 f   moc_DistanceMatrixMSAProfileDialog.obj
 0002:000009b0       _algoLog$initializer$      100199b0     DNAStatMSAProfileDialog.obj
 0002:000009b4       _cmdLog$initializer$       100199b4     DNAStatMSAProfileDialog.obj
 0002:000009b8       _coreLog$initializer$      100199b8     DNAStatMSAProfileDialog.obj
 0002:000009bc       _ioLog$initializer$        100199bc     DNAStatMSAProfileDialog.obj
 0002:000009c0       _perfLog$initializer$      100199c0     DNAStatMSAProfileDialog.obj
 0002:000009c4       _scriptLog$initializer$    100199c4     DNAStatMSAProfileDialog.obj
 0002:000009c8       _taskLog$initializer$      100199c8     DNAStatMSAProfileDialog.obj
 0002:000009cc       _uiLog$initializer$        100199cc     DNAStatMSAProfileDialog.obj
 0002:000009d0       _userActLog$initializer$   100199d0     DNAStatMSAProfileDialog.obj
 0002:000009d4       _Service_PluginViewer$initializer$ 100199d4     DNAStatMSAProfileDialog.obj
 0002:000009d8       _Service_Project$initializer$ 100199d8     DNAStatMSAProfileDialog.obj
 0002:000009dc       _Service_ProjectView$initializer$ 100199dc     DNAStatMSAProfileDialog.obj
 0002:000009e0       _Service_DNAGraphPack$initializer$ 100199e0     DNAStatMSAProfileDialog.obj
 0002:000009e4       _Service_DNAExport$initializer$ 100199e4     DNAStatMSAProfileDialog.obj
 0002:000009e8       _Service_TestRunner$initializer$ 100199e8     DNAStatMSAProfileDialog.obj
 0002:000009ec       _Service_ScriptRegistry$initializer$ 100199ec     DNAStatMSAProfileDialog.obj
 0002:000009f0       _Service_ExternalToolSupport$initializer$ 100199f0     DNAStatMSAProfileDialog.obj
 0002:000009f4       _Service_GUITesting$initializer$ 100199f4     DNAStatMSAProfileDialog.obj
 0002:000009f8       _Service_WorkflowDesigner$initializer$ 100199f8     DNAStatMSAProfileDialog.obj
 0002:000009fc       _Service_QueryDesigner$initializer$ 100199fc     DNAStatMSAProfileDialog.obj
 0002:00000a00       _Service_MinCoreServiceId$initializer$ 10019a00     DNAStatMSAProfileDialog.obj
 0002:00000a04       _Service_MaxCoreServiceId$initializer$ 10019a04     DNAStatMSAProfileDialog.obj
 0002:00000a08       ?HTML$initializer$@DNAStatMSAProfileDialog@U2@@0P6AXXZA 10019a08     DNAStatMSAProfileDialog.obj
 0002:00000a0c       ?CSV$initializer$@DNAStatMSAProfileDialog@U2@@0P6AXXZA 10019a0c     DNAStatMSAProfileDialog.obj
 0002:00000a10       ?_Generic_object$initializer$@?$_Error_objects@H@std@@2P6AXXZA 10019a10     DNAStatMSAProfileDialog.obj
 0002:00000a14       ?_Iostream_object$initializer$@?$_Error_objects@H@std@@2P6AXXZA 10019a14     DNAStatMSAProfileDialog.obj
 0002:00000a18       ?_System_object$initializer$@?$_Error_objects@H@std@@2P6AXXZA 10019a18     DNAStatMSAProfileDialog.obj
 0002:00000a1c       _algoLog$initializer$      10019a1c     DNAStatPlugin.obj
 0002:00000a20       _cmdLog$initializer$       10019a20     DNAStatPlugin.obj
 0002:00000a24       _coreLog$initializer$      10019a24     DNAStatPlugin.obj
 0002:00000a28       _ioLog$initializer$        10019a28     DNAStatPlugin.obj
 0002:00000a2c       _perfLog$initializer$      10019a2c     DNAStatPlugin.obj
 0002:00000a30       _scriptLog$initializer$    10019a30     DNAStatPlugin.obj
 0002:00000a34       _taskLog$initializer$      10019a34     DNAStatPlugin.obj
 0002:00000a38       _uiLog$initializer$        10019a38     DNAStatPlugin.obj
 0002:00000a3c       _userActLog$initializer$   10019a3c     DNAStatPlugin.obj
 0002:00000a40       _Service_PluginViewer$initializer$ 10019a40     DNAStatPlugin.obj
 0002:00000a44       _Service_Project$initializer$ 10019a44     DNAStatPlugin.obj
 0002:00000a48       _Service_ProjectView$initializer$ 10019a48     DNAStatPlugin.obj
 0002:00000a4c       _Service_DNAGraphPack$initializer$ 10019a4c     DNAStatPlugin.obj
 0002:00000a50       _Service_DNAExport$initializer$ 10019a50     DNAStatPlugin.obj
 0002:00000a54       _Service_TestRunner$initializer$ 10019a54     DNAStatPlugin.obj
 0002:00000a58       _Service_ScriptRegistry$initializer$ 10019a58     DNAStatPlugin.obj
 0002:00000a5c       _Service_ExternalToolSupport$initializer$ 10019a5c     DNAStatPlugin.obj
 0002:00000a60       _Service_GUITesting$initializer$ 10019a60     DNAStatPlugin.obj
 0002:00000a64       _Service_WorkflowDesigner$initializer$ 10019a64     DNAStatPlugin.obj
 0002:00000a68       _Service_QueryDesigner$initializer$ 10019a68     DNAStatPlugin.obj
 0002:00000a6c       _Service_MinCoreServiceId$initializer$ 10019a6c     DNAStatPlugin.obj
 0002:00000a70       _Service_MaxCoreServiceId$initializer$ 10019a70     DNAStatPlugin.obj
 0002:00000a74       _algoLog$initializer$      10019a74     DNAStatProfileTask.obj
 0002:00000a78       _cmdLog$initializer$       10019a78     DNAStatProfileTask.obj
 0002:00000a7c       _coreLog$initializer$      10019a7c     DNAStatProfileTask.obj
 0002:00000a80       _ioLog$initializer$        10019a80     DNAStatProfileTask.obj
 0002:00000a84       _perfLog$initializer$      10019a84     DNAStatProfileTask.obj
 0002:00000a88       _scriptLog$initializer$    10019a88     DNAStatProfileTask.obj
 0002:00000a8c       _taskLog$initializer$      10019a8c     DNAStatProfileTask.obj
 0002:00000a90       _uiLog$initializer$        10019a90     DNAStatProfileTask.obj
 0002:00000a94       _userActLog$initializer$   10019a94     DNAStatProfileTask.obj
 0002:00000a98       _Service_PluginViewer$initializer$ 10019a98     DNAStatProfileTask.obj
 0002:00000a9c       _Service_Project$initializer$ 10019a9c     DNAStatProfileTask.obj
 0002:00000aa0       _Service_ProjectView$initializer$ 10019aa0     DNAStatProfileTask.obj
 0002:00000aa4       _Service_DNAGraphPack$initializer$ 10019aa4     DNAStatProfileTask.obj
 0002:00000aa8       _Service_DNAExport$initializer$ 10019aa8     DNAStatProfileTask.obj
 0002:00000aac       _Service_TestRunner$initializer$ 10019aac     DNAStatProfileTask.obj
 0002:00000ab0       _Service_ScriptRegistry$initializer$ 10019ab0     DNAStatProfileTask.obj
 0002:00000ab4       _Service_ExternalToolSupport$initializer$ 10019ab4     DNAStatProfileTask.obj
 0002:00000ab8       _Service_GUITesting$initializer$ 10019ab8     DNAStatProfileTask.obj
 0002:00000abc       _Service_WorkflowDesigner$initializer$ 10019abc     DNAStatProfileTask.obj
 0002:00000ac0       _Service_QueryDesigner$initializer$ 10019ac0     DNAStatProfileTask.obj
 0002:00000ac4       _Service_MinCoreServiceId$initializer$ 10019ac4     DNAStatProfileTask.obj
 0002:00000ac8       _Service_MaxCoreServiceId$initializer$ 10019ac8     DNAStatProfileTask.obj
 0002:00000acc       _algoLog$initializer$      10019acc     DistanceMatrixMSAProfileDialog.obj
 0002:00000ad0       _cmdLog$initializer$       10019ad0     DistanceMatrixMSAProfileDialog.obj
 0002:00000ad4       _coreLog$initializer$      10019ad4     DistanceMatrixMSAProfileDialog.obj
 0002:00000ad8       _ioLog$initializer$        10019ad8     DistanceMatrixMSAProfileDialog.obj
 0002:00000adc       _perfLog$initializer$      10019adc     DistanceMatrixMSAProfileDialog.obj
 0002:00000ae0       _scriptLog$initializer$    10019ae0     DistanceMatrixMSAProfileDialog.obj
 0002:00000ae4       _taskLog$initializer$      10019ae4     DistanceMatrixMSAProfileDialog.obj
 0002:00000ae8       _uiLog$initializer$        10019ae8     DistanceMatrixMSAProfileDialog.obj
 0002:00000aec       _userActLog$initializer$   10019aec     DistanceMatrixMSAProfileDialog.obj
 0002:00000af0       _Service_PluginViewer$initializer$ 10019af0     DistanceMatrixMSAProfileDialog.obj
 0002:00000af4       _Service_Project$initializer$ 10019af4     DistanceMatrixMSAProfileDialog.obj
 0002:00000af8       _Service_ProjectView$initializer$ 10019af8     DistanceMatrixMSAProfileDialog.obj
 0002:00000afc       _Service_DNAGraphPack$initializer$ 10019afc     DistanceMatrixMSAProfileDialog.obj
 0002:00000b00       _Service_DNAExport$initializer$ 10019b00     DistanceMatrixMSAProfileDialog.obj
 0002:00000b04       _Service_TestRunner$initializer$ 10019b04     DistanceMatrixMSAProfileDialog.obj
 0002:00000b08       _Service_ScriptRegistry$initializer$ 10019b08     DistanceMatrixMSAProfileDialog.obj
 0002:00000b0c       _Service_ExternalToolSupport$initializer$ 10019b0c     DistanceMatrixMSAProfileDialog.obj
 0002:00000b10       _Service_GUITesting$initializer$ 10019b10     DistanceMatrixMSAProfileDialog.obj
 0002:00000b14       _Service_WorkflowDesigner$initializer$ 10019b14     DistanceMatrixMSAProfileDialog.obj
 0002:00000b18       _Service_QueryDesigner$initializer$ 10019b18     DistanceMatrixMSAProfileDialog.obj
 0002:00000b1c       _Service_MinCoreServiceId$initializer$ 10019b1c     DistanceMatrixMSAProfileDialog.obj
 0002:00000b20       _Service_MaxCoreServiceId$initializer$ 10019b20     DistanceMatrixMSAProfileDialog.obj
 0002:00000b24       ?HTML$initializer$@DistanceMatrixMSAProfileDialog@U2@@0P6AXXZA 10019b24     DistanceMatrixMSAProfileDialog.obj
 0002:00000b28       ?CSV$initializer$@DistanceMatrixMSAProfileDialog@U2@@0P6AXXZA 10019b28     DistanceMatrixMSAProfileDialog.obj
 0002:00000b2c       _algoLog$initializer$      10019b2c     moc_DNAStatMSAProfileDialog.obj
 0002:00000b30       _cmdLog$initializer$       10019b30     moc_DNAStatMSAProfileDialog.obj
 0002:00000b34       _coreLog$initializer$      10019b34     moc_DNAStatMSAProfileDialog.obj
 0002:00000b38       _ioLog$initializer$        10019b38     moc_DNAStatMSAProfileDialog.obj
 0002:00000b3c       _perfLog$initializer$      10019b3c     moc_DNAStatMSAProfileDialog.obj
 0002:00000b40       _scriptLog$initializer$    10019b40     moc_DNAStatMSAProfileDialog.obj
 0002:00000b44       _taskLog$initializer$      10019b44     moc_DNAStatMSAProfileDialog.obj
 0002:00000b48       _uiLog$initializer$        10019b48     moc_DNAStatMSAProfileDialog.obj
 0002:00000b4c       _userActLog$initializer$   10019b4c     moc_DNAStatMSAProfileDialog.obj
 0002:00000b50       ?staticMetaObject$initializer$@DNAStatMSAProfileDialog@U2@@2P6AXXZA 10019b50     moc_DNAStatMSAProfileDialog.obj
 0002:00000b54       ?staticMetaObject$initializer$@DNAStatMSAProfileTask@U2@@2P6AXXZA 10019b54     moc_DNAStatMSAProfileDialog.obj
 0002:00000b58       _Service_PluginViewer$initializer$ 10019b58     moc_DNAStatPlugin.obj
 0002:00000b5c       _Service_Project$initializer$ 10019b5c     moc_DNAStatPlugin.obj
 0002:00000b60       _Service_ProjectView$initializer$ 10019b60     moc_DNAStatPlugin.obj
 0002:00000b64       _Service_DNAGraphPack$initializer$ 10019b64     moc_DNAStatPlugin.obj
 0002:00000b68       _Service_DNAExport$initializer$ 10019b68     moc_DNAStatPlugin.obj
 0002:00000b6c       _Service_TestRunner$initializer$ 10019b6c     moc_DNAStatPlugin.obj
 0002:00000b70       _Service_ScriptRegistry$initializer$ 10019b70     moc_DNAStatPlugin.obj
 0002:00000b74       _Service_ExternalToolSupport$initializer$ 10019b74     moc_DNAStatPlugin.obj
 0002:00000b78       _Service_GUITesting$initializer$ 10019b78     moc_DNAStatPlugin.obj
 0002:00000b7c       _Service_WorkflowDesigner$initializer$ 10019b7c     moc_DNAStatPlugin.obj
 0002:00000b80       _Service_QueryDesigner$initializer$ 10019b80     moc_DNAStatPlugin.obj
 0002:00000b84       _Service_MinCoreServiceId$initializer$ 10019b84     moc_DNAStatPlugin.obj
 0002:00000b88       _Service_MaxCoreServiceId$initializer$ 10019b88     moc_DNAStatPlugin.obj
 0002:00000b8c       ?staticMetaObject$initializer$@DNAStatPlugin@U2@@2P6AXXZA 10019b8c     moc_DNAStatPlugin.obj
 0002:00000b90       ?staticMetaObject$initializer$@DNAStatMSAEditorContext@U2@@2P6AXXZA 10019b90     moc_DNAStatPlugin.obj
 0002:00000b94       ?staticMetaObject$initializer$@DistanceMatrixMSAEditorContext@U2@@2P6AXXZA 10019b94     moc_DNAStatPlugin.obj
 0002:00000b98       _algoLog$initializer$      10019b98     moc_DNAStatProfileTask.obj
 0002:00000b9c       _cmdLog$initializer$       10019b9c     moc_DNAStatProfileTask.obj
 0002:00000ba0       _coreLog$initializer$      10019ba0     moc_DNAStatProfileTask.obj
 0002:00000ba4       _ioLog$initializer$        10019ba4     moc_DNAStatProfileTask.obj
 0002:00000ba8       _perfLog$initializer$      10019ba8     moc_DNAStatProfileTask.obj
 0002:00000bac       _scriptLog$initializer$    10019bac     moc_DNAStatProfileTask.obj
 0002:00000bb0       _taskLog$initializer$      10019bb0     moc_DNAStatProfileTask.obj
 0002:00000bb4       _uiLog$initializer$        10019bb4     moc_DNAStatProfileTask.obj
 0002:00000bb8       _userActLog$initializer$   10019bb8     moc_DNAStatProfileTask.obj
 0002:00000bbc       ?staticMetaObject$initializer$@DNAStatProfileTask@U2@@2P6AXXZA 10019bbc     moc_DNAStatProfileTask.obj
 0002:00000bc0       _algoLog$initializer$      10019bc0     moc_DistanceMatrixMSAProfileDialog.obj
 0002:00000bc4       _cmdLog$initializer$       10019bc4     moc_DistanceMatrixMSAProfileDialog.obj
 0002:00000bc8       _coreLog$initializer$      10019bc8     moc_DistanceMatrixMSAProfileDialog.obj
 0002:00000bcc       _ioLog$initializer$        10019bcc     moc_DistanceMatrixMSAProfileDialog.obj
 0002:00000bd0       _perfLog$initializer$      10019bd0     moc_DistanceMatrixMSAProfileDialog.obj
 0002:00000bd4       _scriptLog$initializer$    10019bd4     moc_DistanceMatrixMSAProfileDialog.obj
 0002:00000bd8       _taskLog$initializer$      10019bd8     moc_DistanceMatrixMSAProfileDialog.obj
 0002:00000bdc       _uiLog$initializer$        10019bdc     moc_DistanceMatrixMSAProfileDialog.obj
 0002:00000be0       _userActLog$initializer$   10019be0     moc_DistanceMatrixMSAProfileDialog.obj
 0002:00000be4       ?staticMetaObject$initializer$@DistanceMatrixMSAProfileDialog@U2@@2P6AXXZA 10019be4     moc_DistanceMatrixMSAProfileDialog.obj
 0002:00000be8       ?staticMetaObject$initializer$@DistanceMatrixMSAProfileTask@U2@@2P6AXXZA 10019be8     moc_DistanceMatrixMSAProfileDialog.obj
 0002:00000bf4       _pcinit                    10019bf4     MSVCRT:crtdll.obj
 0002:00000bf8       _pinit                     10019bf8     MSVCRT:atonexit.obj
 0002:000017e8       ?qstring_literal@?6???R<lambda_332f86a55e7649bbbc7d152cfc1d46e6>@@QBE?AVQString@@XZ@4U?$QStaticStringData@$0BH@@@B 1001a7e8     DNAStatMSAProfileDialog.obj
 0002:00001828       ?qstring_literal@?7???R<lambda_459d3513592b8ff4f9b393a392f7e1dc>@@QBE?AVQString@@XZ@4U?$QStaticStringData@$0BA@@@B 1001a828     DNAStatMSAProfileDialog.obj
 0002:0000185c       ?qstring_literal@?8???R<lambda_a3a39629b9536d4dab532972692be556>@@QBE?AVQString@@XZ@4U?$QStaticStringData@$09@@B 1001a85c     DNAStatMSAProfileDialog.obj
 0002:00001884       ?qstring_literal@?9???R<lambda_9f6a8b438001a51b240e5bf18f0afdd2>@@QBE?AVQString@@XZ@4U?$QStaticStringData@$0M@@@B 1001a884     DNAStatMSAProfileDialog.obj
 0002:000018b0       ?qstring_literal@?L@???R<lambda_3f118f97850a866f6d5ae3fbb0dc2aed>@@QBE?AVQString@@XZ@4U?$QStaticStringData@$07@@B 1001a8b0     DNAStatMSAProfileDialog.obj
 0002:000018d4       ?qstring_literal@?M@???R<lambda_376d37d6abfed47a5cb9bd756b76dca8>@@QBE?AVQString@@XZ@4U?$QStaticStringData@$09@@B 1001a8d4     DNAStatMSAProfileDialog.obj
 0002:000018fc       ?qstring_literal@?N@???R<lambda_a89643c798c7c6488c2208d0e325f35b>@@QBE?AVQString@@XZ@4U?$QStaticStringData@$07@@B 1001a8fc     DNAStatMSAProfileDialog.obj
 0002:00001920       ?qstring_literal@?O@???R<lambda_3921f84164ed29f15fc743b6ab68e204>@@QBE?AVQString@@XZ@4U?$QStaticStringData@$0O@@@B 1001a920     DNAStatMSAProfileDialog.obj
 0002:00001950       ?qstring_literal@?P@???R<lambda_bd9b46c5af1ae431bf97a2b6b358b9a7>@@QBE?AVQString@@XZ@4U?$QStaticStringData@$04@@B 1001a950     DNAStatMSAProfileDialog.obj
 0002:0000196c       ?qstring_literal@?BA@???R<lambda_4a12a9b4f8aa2ea3a7fffd7d958ae388>@@QBE?AVQString@@XZ@4U?$QStaticStringData@$07@@B 1001a96c     DNAStatMSAProfileDialog.obj
 0002:00001990       ?qstring_literal@?BB@???R<lambda_545371d98571d04f1b39b4582be52899>@@QBE?AVQString@@XZ@4U?$QStaticStringData@$0BC@@@B 1001a990     DNAStatMSAProfileDialog.obj
 0002:000019c8       ?qstring_literal@?BC@???R<lambda_0b89744300e523de31da4f8ed196539f>@@QBE?AVQString@@XZ@4U?$QStaticStringData@$06@@B 1001a9c8     DNAStatMSAProfileDialog.obj
 0002:000019e8       ?qstring_literal@?BD@???R<lambda_bda637ed11183b6068483cf30a484448>@@QBE?AVQString@@XZ@4U?$QStaticStringData@$09@@B 1001a9e8     DNAStatMSAProfileDialog.obj
 0002:00001a10       ?qstring_literal@?BE@???R<lambda_664313d2fa9b135bdb11bebee3978435>@@QBE?AVQString@@XZ@4U?$QStaticStringData@$04@@B 1001aa10     DNAStatMSAProfileDialog.obj
 0002:00001a2c       ?qstring_literal@?BF@???R<lambda_fab6138414a91a0c3bced0a99c7ba19f>@@QBE?AVQString@@XZ@4U?$QStaticStringData@$07@@B 1001aa2c     DNAStatMSAProfileDialog.obj
 0002:00001a50       ?qstring_literal@?BG@???R<lambda_369cdf7999dc0faee62b5b90af0d786b>@@QBE?AVQString@@XZ@4U?$QStaticStringData@$09@@B 1001aa50     DNAStatMSAProfileDialog.obj
 0002:00001a78       ?qstring_literal@?BH@???R<lambda_59946a197341b3528bd575f770f586ea>@@QBE?AVQString@@XZ@4U?$QStaticStringData@$05@@B 1001aa78     DNAStatMSAProfileDialog.obj
 0002:00001a98       ?qstring_literal@?BI@???R<lambda_9ef6d0056c3e3c198c7a1006e54d249c>@@QBE?AVQString@@XZ@4U?$QStaticStringData@$04@@B 1001aa98     DNAStatMSAProfileDialog.obj
 0002:00001ab4       ?qstring_literal@?BJ@???R<lambda_580e10368bf5988093bdeab019318dc2>@@QBE?AVQString@@XZ@4U?$QStaticStringData@$08@@B 1001aab4     DNAStatMSAProfileDialog.obj
 0002:00002c58       ?qstring_literal@?6???R<lambda_4149c1a5601b404cb9e3099d72fa0a0a>@@QBE?AVQString@@XZ@4U?$QStaticStringData@$0BO@@@B 1001bc58     DistanceMatrixMSAProfileDialog.obj
 0002:00002ca8       ?qstring_literal@?7???R<lambda_4c9d5f56d49016978bbb8760a7e3d910>@@QBE?AVQString@@XZ@4U?$QStaticStringData@$0BA@@@B 1001bca8     DistanceMatrixMSAProfileDialog.obj
 0002:00002cdc       ?qstring_literal@?8???R<lambda_346f61b4a197c7796b06dee8cb9eb1b6>@@QBE?AVQString@@XZ@4U?$QStaticStringData@$0BC@@@B 1001bcdc     DistanceMatrixMSAProfileDialog.obj
 0002:00002d14       ?qstring_literal@?9???R<lambda_257a9ba125789c78778143779c7aa17e>@@QBE?AVQString@@XZ@4U?$QStaticStringData@$08@@B 1001bd14     DistanceMatrixMSAProfileDialog.obj
 0002:00002d38       ?qstring_literal@?L@???R<lambda_477f2371469cb72a5ef263890104105f>@@QBE?AVQString@@XZ@4U?$QStaticStringData@$08@@B 1001bd38     DistanceMatrixMSAProfileDialog.obj
 0002:00002d5c       ?qstring_literal@?M@???R<lambda_f3813fcbb1e170019aa0d3012117af7b>@@QBE?AVQString@@XZ@4U?$QStaticStringData@$09@@B 1001bd5c     DistanceMatrixMSAProfileDialog.obj
 0002:00002d84       ?qstring_literal@?N@???R<lambda_840dc314801588f3307f74f67d327cab>@@QBE?AVQString@@XZ@4U?$QStaticStringData@$0M@@@B 1001bd84     DistanceMatrixMSAProfileDialog.obj
 0002:00002db0       ?qstring_literal@?O@???R<lambda_aaa0d8f07c2dd2193aa6aadb22c08d2b>@@QBE?AVQString@@XZ@4U?$QStaticStringData@$07@@B 1001bdb0     DistanceMatrixMSAProfileDialog.obj
 0002:00002dd4       ?qstring_literal@?P@???R<lambda_22328789e56fd3e3b770fcf81371bdbf>@@QBE?AVQString@@XZ@4U?$QStaticStringData@$09@@B 1001bdd4     DistanceMatrixMSAProfileDialog.obj
 0002:00002dfc       ?qstring_literal@?BA@???R<lambda_667cf19c3b93807e72a75e35313c6da5>@@QBE?AVQString@@XZ@4U?$QStaticStringData@$07@@B 1001bdfc     DistanceMatrixMSAProfileDialog.obj
 0002:00002e20       ?qstring_literal@?BB@???R<lambda_3af62e2b98c1502753882d3498ff5cca>@@QBE?AVQString@@XZ@4U?$QStaticStringData@$0BE@@@B 1001be20     DistanceMatrixMSAProfileDialog.obj
 0002:00002e5c       ?qstring_literal@?BC@???R<lambda_df5a57b07f782d6c431b0eadd5e7983a>@@QBE?AVQString@@XZ@4U?$QStaticStringData@$06@@B 1001be5c     DistanceMatrixMSAProfileDialog.obj
 0002:00002e7c       ?qstring_literal@?BD@???R<lambda_d91a2c0f8c8907c0767dda3038aeabd8>@@QBE?AVQString@@XZ@4U?$QStaticStringData@$09@@B 1001be7c     DistanceMatrixMSAProfileDialog.obj
 0002:00002ea4       ?qstring_literal@?BE@???R<lambda_cd3023c81d757c47026fd3c6565acb82>@@QBE?AVQString@@XZ@4U?$QStaticStringData@$04@@B 1001bea4     DistanceMatrixMSAProfileDialog.obj
 0002:00002ec0       ?qstring_literal@?BF@???R<lambda_f076482335b87e84dc878d3bc1c37823>@@QBE?AVQString@@XZ@4U?$QStaticStringData@$07@@B 1001bec0     DistanceMatrixMSAProfileDialog.obj
 0002:00002ee4       ?qstring_literal@?BG@???R<lambda_b420bad46777224f9d1a7dddab21eac2>@@QBE?AVQString@@XZ@4U?$QStaticStringData@$09@@B 1001bee4     DistanceMatrixMSAProfileDialog.obj
 0002:00002f0c       ?qstring_literal@?BH@???R<lambda_7d1f8454ec166fb6929aab69d9b35ec8>@@QBE?AVQString@@XZ@4U?$QStaticStringData@$05@@B 1001bf0c     DistanceMatrixMSAProfileDialog.obj
 0002:00002f2c       ?qstring_literal@?BI@???R<lambda_3b9e00bd2f9235c0e5410d79eb0eadce>@@QBE?AVQString@@XZ@4U?$QStaticStringData@$04@@B 1001bf2c     DistanceMatrixMSAProfileDialog.obj
 0002:00002f48       ?qstring_literal@?BJ@???R<lambda_d92ac2e6e619141498e0b5df5f617cb4>@@QBE?AVQString@@XZ@4U?$QStaticStringData@$08@@B 1001bf48     DistanceMatrixMSAProfileDialog.obj
 0002:00003350       _qt_meta_stringdata_U2__DNAStatMSAProfileDialog 1001c350     moc_DNAStatMSAProfileDialog.obj
 0002:000033ec       _qt_meta_stringdata_U2__DNAStatMSAProfileTask 1001c3ec     moc_DNAStatMSAProfileDialog.obj
 0002:00003418       _qt_meta_data_U2__DNAStatMSAProfileDialog 1001c418     moc_DNAStatMSAProfileDialog.obj
 0002:0000348c       _qt_meta_data_U2__DNAStatMSAProfileTask 1001c48c     moc_DNAStatMSAProfileDialog.obj
 0002:000034e8       _qt_meta_stringdata_U2__DNAStatPlugin 1001c4e8     moc_DNAStatPlugin.obj
 0002:0000350c       _qt_meta_data_U2__DNAStatPlugin 1001c50c     moc_DNAStatPlugin.obj
 0002:00003548       _qt_meta_stringdata_U2__DNAStatMSAEditorContext 1001c548     moc_DNAStatPlugin.obj
 0002:00003620       _qt_meta_data_U2__DNAStatMSAEditorContext 1001c620     moc_DNAStatPlugin.obj
 0002:000036a0       _qt_meta_stringdata_U2__DistanceMatrixMSAEditorContext 1001c6a0     moc_DNAStatPlugin.obj
 0002:00003788       _qt_meta_data_U2__DistanceMatrixMSAEditorContext 1001c788     moc_DNAStatPlugin.obj
 0002:00003804       _qt_meta_stringdata_U2__DNAStatProfileTask 1001c804     moc_DNAStatProfileTask.obj
 0002:0000382c       _qt_meta_data_U2__DNAStatProfileTask 1001c82c     moc_DNAStatProfileTask.obj
 0002:00003868       _qt_meta_stringdata_U2__DistanceMatrixMSAProfileDialog 1001c868     moc_DistanceMatrixMSAProfileDialog.obj
 0002:0000390c       _qt_meta_stringdata_U2__DistanceMatrixMSAProfileTask 1001c90c     moc_DistanceMatrixMSAProfileDialog.obj
 0002:00003940       _qt_meta_data_U2__DistanceMatrixMSAProfileDialog 1001c940     moc_DistanceMatrixMSAProfileDialog.obj
 0002:000039b4       _qt_meta_data_U2__DistanceMatrixMSAProfileTask 1001c9b4     moc_DistanceMatrixMSAProfileDialog.obj
 0002:00003a20       _Int32ToUInt32             1001ca20     MSVCRT:ftol3.obj
 0002:00003a30       _MantissaMask              1001ca30     MSVCRT:ftol3.obj
 0002:00003a38       _IntegerBit                1001ca38     MSVCRT:ftol3.obj
 0002:00003a40       _SignBit64                 1001ca40     MSVCRT:ftol3.obj
 0002:00003a48       _MinFP64                   1001ca48     MSVCRT:ftol3.obj
 0002:00003a50       _MinInt64                  1001ca50     MSVCRT:ftol3.obj
 0002:00003a58       _MaxInt64                  1001ca58     MSVCRT:ftol3.obj
 0002:00003a60       _MaxUInt64                 1001ca60     MSVCRT:ftol3.obj
 0002:00003a68       _MaxFP32                   1001ca68     MSVCRT:ftol3.obj
 0002:00003a70       _MinFP32                   1001ca70     MSVCRT:ftol3.obj
 0002:00003a78       _MinSubInexact             1001ca78     MSVCRT:ftol3.obj
 0002:00003a80       _FpExcptTable              1001ca80     MSVCRT:ftol3.obj
 0002:00003a90       _i1075                     1001ca90     MSVCRT:ftol3.obj
 0002:00003a94       _i1087                     1001ca94     MSVCRT:ftol3.obj
 0002:00003a98       _x0800                     1001ca98     MSVCRT:ftol3.obj
 0002:00003a9c       _x17FF                     1001ca9c     MSVCRT:ftol3.obj
 0002:00003aa0       _CWMask                    1001caa0     MSVCRT:ftol3.obj
 0002:00003aa8       _GS_ExceptionPointers      1001caa8     MSVCRT:gs_report.obj
 0002:00005090       __catchsym$?_Copy@?$basic_string@DU?$char_traits@D@std@@V?$allocator@D@2@@std@@QAEXII@Z$5 1001e090     DNAStatMSAProfileDialog.obj
 0002:000050a0       __catchsym$?_Copy@?$basic_string@DU?$char_traits@D@std@@V?$allocator@D@2@@std@@QAEXII@Z$4 1001e0a0     DNAStatMSAProfileDialog.obj
 0002:000050b0       __unwindtable$?_Copy@?$basic_string@DU?$char_traits@D@std@@V?$allocator@D@2@@std@@QAEXII@Z 1001e0b0     DNAStatMSAProfileDialog.obj
 0002:000050d0       __ehfuncinfo$?_Copy@?$basic_string@DU?$char_traits@D@std@@V?$allocator@D@2@@std@@QAEXII@Z 1001e0d0     DNAStatMSAProfileDialog.obj
 0002:000050f4       __tryblocktable$?_Copy@?$basic_string@DU?$char_traits@D@std@@V?$allocator@D@2@@std@@QAEXII@Z 1001e0f4     DNAStatMSAProfileDialog.obj
 0002:0000511c       __unwindtable$??H@YA?BVQString@@ABV0@0@Z 1001e11c     DNAStatMSAProfileDialog.obj
 0002:00005124       __ehfuncinfo$??H@YA?BVQString@@ABV0@0@Z 1001e124     DNAStatMSAProfileDialog.obj
 0002:00005148       __unwindtable$??H@YA?BVQString@@ABV0@PBD@Z 1001e148     DNAStatMSAProfileDialog.obj
 0002:00005158       __ehfuncinfo$??H@YA?BVQString@@ABV0@PBD@Z 1001e158     DNAStatMSAProfileDialog.obj
 0002:0000517c       __unwindtable$??H@YA?BVQString@@PBDABV0@@Z 1001e17c     DNAStatMSAProfileDialog.obj
 0002:00005184       __ehfuncinfo$??H@YA?BVQString@@PBDABV0@@Z 1001e184     DNAStatMSAProfileDialog.obj
 0002:000051a8       __catchsym$?append@?$QList@VQString@@@@QAEXABVQString@@@Z$13 1001e1a8     DNAStatMSAProfileDialog.obj
 0002:000051b8       __catchsym$?append@?$QList@VQString@@@@QAEXABVQString@@@Z$12 1001e1b8     DNAStatMSAProfileDialog.obj
 0002:000051c8       __ehfuncinfo$?append@?$QList@VQString@@@@QAEXABVQString@@@Z 1001e1c8     DNAStatMSAProfileDialog.obj
 0002:000051ec       __tryblocktable$?append@?$QList@VQString@@@@QAEXABVQString@@@Z 1001e1ec     DNAStatMSAProfileDialog.obj
 0002:00005214       __unwindtable$?append@?$QList@VQString@@@@QAEXABVQString@@@Z 1001e214     DNAStatMSAProfileDialog.obj
 0002:00005274       __catchsym$?detach_helper_grow@?$QList@VQString@@@@AAEPAUNode@1@HH@Z$5 1001e274     DNAStatMSAProfileDialog.obj
 0002:00005284       __catchsym$?detach_helper_grow@?$QList@VQString@@@@AAEPAUNode@1@HH@Z$4 1001e284     DNAStatMSAProfileDialog.obj
 0002:00005294       __unwindtable$?detach_helper_grow@?$QList@VQString@@@@AAEPAUNode@1@HH@Z 1001e294     DNAStatMSAProfileDialog.obj
 0002:000052b4       __ehfuncinfo$?detach_helper_grow@?$QList@VQString@@@@AAEPAUNode@1@HH@Z 1001e2b4     DNAStatMSAProfileDialog.obj
 0002:000052d8       __tryblocktable$?detach_helper_grow@?$QList@VQString@@@@AAEPAUNode@1@HH@Z 1001e2d8     DNAStatMSAProfileDialog.obj
 0002:00005300       __unwindtable$?node_construct@?$QList@VQString@@@@AAEXPAUNode@1@ABVQString@@@Z 1001e300     DNAStatMSAProfileDialog.obj
 0002:00005310       __ehfuncinfo$?node_construct@?$QList@VQString@@@@AAEXPAUNode@1@ABVQString@@@Z 1001e310     DNAStatMSAProfileDialog.obj
 0002:00005334       __catchsym$?node_copy@?$QList@VQString@@@@AAEXPAUNode@1@00@Z$6 1001e334     DNAStatMSAProfileDialog.obj
 0002:00005344       __tryblocktable$?node_copy@?$QList@VQString@@@@AAEXPAUNode@1@00@Z 1001e344     DNAStatMSAProfileDialog.obj
 0002:00005358       __ehfuncinfo$?node_copy@?$QList@VQString@@@@AAEXPAUNode@1@00@Z 1001e358     DNAStatMSAProfileDialog.obj
 0002:0000537c       __unwindtable$?node_copy@?$QList@VQString@@@@AAEXPAUNode@1@00@Z 1001e37c     DNAStatMSAProfileDialog.obj
 0002:000053ac       __unwindtable$??__EalgoLog@U2@@YAXXZ 1001e3ac     DNAStatMSAProfileDialog.obj
 0002:000053b4       __ehfuncinfo$??__EalgoLog@U2@@YAXXZ 1001e3b4     DNAStatMSAProfileDialog.obj
 0002:000053d8       __unwindtable$??__EcmdLog@U2@@YAXXZ 1001e3d8     DNAStatMSAProfileDialog.obj
 0002:000053e0       __ehfuncinfo$??__EcmdLog@U2@@YAXXZ 1001e3e0     DNAStatMSAProfileDialog.obj
 0002:00005404       __unwindtable$??__EcoreLog@U2@@YAXXZ 1001e404     DNAStatMSAProfileDialog.obj
 0002:0000540c       __ehfuncinfo$??__EcoreLog@U2@@YAXXZ 1001e40c     DNAStatMSAProfileDialog.obj
 0002:00005430       __unwindtable$??__EioLog@U2@@YAXXZ 1001e430     DNAStatMSAProfileDialog.obj
 0002:00005438       __ehfuncinfo$??__EioLog@U2@@YAXXZ 1001e438     DNAStatMSAProfileDialog.obj
 0002:0000545c       __unwindtable$??__EperfLog@U2@@YAXXZ 1001e45c     DNAStatMSAProfileDialog.obj
 0002:00005464       __ehfuncinfo$??__EperfLog@U2@@YAXXZ 1001e464     DNAStatMSAProfileDialog.obj
 0002:00005488       __unwindtable$??__EscriptLog@U2@@YAXXZ 1001e488     DNAStatMSAProfileDialog.obj
 0002:00005490       __ehfuncinfo$??__EscriptLog@U2@@YAXXZ 1001e490     DNAStatMSAProfileDialog.obj
 0002:000054b4       __unwindtable$??__EtaskLog@U2@@YAXXZ 1001e4b4     DNAStatMSAProfileDialog.obj
 0002:000054bc       __ehfuncinfo$??__EtaskLog@U2@@YAXXZ 1001e4bc     DNAStatMSAProfileDialog.obj
 0002:000054e0       __unwindtable$??__EuiLog@U2@@YAXXZ 1001e4e0     DNAStatMSAProfileDialog.obj
 0002:000054e8       __ehfuncinfo$??__EuiLog@U2@@YAXXZ 1001e4e8     DNAStatMSAProfileDialog.obj
 0002:0000550c       __unwindtable$??__EuserActLog@U2@@YAXXZ 1001e50c     DNAStatMSAProfileDialog.obj
 0002:00005514       __ehfuncinfo$??__EuserActLog@U2@@YAXXZ 1001e514     DNAStatMSAProfileDialog.obj
 0002:00005538       __catchsym$?reallocData@?$QVector@H@@AAEXHHV?$QFlags@W4AllocationOption@QArrayData@@@@@Z$5 1001e538     DNAStatMSAProfileDialog.obj
 0002:00005548       __catchsym$?reallocData@?$QVector@H@@AAEXHHV?$QFlags@W4AllocationOption@QArrayData@@@@@Z$4 1001e548     DNAStatMSAProfileDialog.obj
 0002:00005558       __unwindtable$?reallocData@?$QVector@H@@AAEXHHV?$QFlags@W4AllocationOption@QArrayData@@@@@Z 1001e558     DNAStatMSAProfileDialog.obj
 0002:00005578       __ehfuncinfo$?reallocData@?$QVector@H@@AAEXHHV?$QFlags@W4AllocationOption@QArrayData@@@@@Z 1001e578     DNAStatMSAProfileDialog.obj
 0002:0000559c       __tryblocktable$?reallocData@?$QVector@H@@AAEXHHV?$QFlags@W4AllocationOption@QArrayData@@@@@Z 1001e59c     DNAStatMSAProfileDialog.obj
 0002:000055c4       __ehfuncinfo$?setupUi@Ui_DNAStatMSAProfileDialog@@QAEXPAVQDialog@@@Z 1001e5c4     DNAStatMSAProfileDialog.obj
 0002:000055e8       __unwindtable$?setupUi@Ui_DNAStatMSAProfileDialog@@QAEXPAVQDialog@@@Z 1001e5e8     DNAStatMSAProfileDialog.obj
 0002:00005710       __ehfuncinfo$?retranslateUi@Ui_DNAStatMSAProfileDialog@@QAEXPAVQDialog@@@Z 1001e710     DNAStatMSAProfileDialog.obj
 0002:00005734       __unwindtable$?retranslateUi@Ui_DNAStatMSAProfileDialog@@QAEXPAVQDialog@@@Z 1001e734     DNAStatMSAProfileDialog.obj
 0002:0000579c       __ehfuncinfo$??0DNAStatMSAProfileDialog@U2@@QAE@PAVQWidget@@PAVMSAEditor@1@@Z 1001e79c     DNAStatMSAProfileDialog.obj
 0002:000057c0       __unwindtable$??0DNAStatMSAProfileDialog@U2@@QAE@PAVQWidget@@PAVMSAEditor@1@@Z 1001e7c0     DNAStatMSAProfileDialog.obj
 0002:000057f0       __ehfuncinfo$?accept@DNAStatMSAProfileDialog@U2@@UAEXXZ 1001e7f0     DNAStatMSAProfileDialog.obj
 0002:00005814       __unwindtable$?accept@DNAStatMSAProfileDialog@U2@@UAEXXZ 1001e814     DNAStatMSAProfileDialog.obj
 0002:0000585c       __ehfuncinfo$?initSaveController@DNAStatMSAProfileDialog@U2@@AAEXXZ 1001e85c     DNAStatMSAProfileDialog.obj
 0002:00005880       __unwindtable$?initSaveController@DNAStatMSAProfileDialog@U2@@AAEXXZ 1001e880     DNAStatMSAProfileDialog.obj
 0002:00005910       __ehfuncinfo$??0DNAStatMSAProfileTaskSettings@U2@@QAE@XZ 1001e910     DNAStatMSAProfileDialog.obj
 0002:00005934       __unwindtable$??0DNAStatMSAProfileTaskSettings@U2@@QAE@XZ 1001e934     DNAStatMSAProfileDialog.obj
 0002:0000596c       __unwindtable$??1DNAStatMSAProfileTaskSettings@U2@@QAE@XZ 1001e96c     DNAStatMSAProfileDialog.obj
 0002:00005984       __ehfuncinfo$??1DNAStatMSAProfileTaskSettings@U2@@QAE@XZ 1001e984     DNAStatMSAProfileDialog.obj
 0002:000059a8       __unwindtable$??0DNAStatMSAProfileTaskSettings@U2@@QAE@ABV01@@Z 1001e9a8     DNAStatMSAProfileDialog.obj
 0002:000059c0       __ehfuncinfo$??0DNAStatMSAProfileTaskSettings@U2@@QAE@ABV01@@Z 1001e9c0     DNAStatMSAProfileDialog.obj
 0002:000059e4       __ehfuncinfo$??0DNAStatMSAProfileTask@U2@@QAE@ABVDNAStatMSAProfileTaskSettings@1@@Z 1001e9e4     DNAStatMSAProfileDialog.obj
 0002:00005a08       __unwindtable$??0DNAStatMSAProfileTask@U2@@QAE@ABVDNAStatMSAProfileTaskSettings@1@@Z 1001ea08     DNAStatMSAProfileDialog.obj
 0002:00005a58       __catchsym$?run@DNAStatMSAProfileTask@U2@@UAEXXZ$75 1001ea58     DNAStatMSAProfileDialog.obj
 0002:00005a68       __tryblocktable$?run@DNAStatMSAProfileTask@U2@@UAEXXZ 1001ea68     DNAStatMSAProfileDialog.obj
 0002:00005a7c       __ehfuncinfo$?run@DNAStatMSAProfileTask@U2@@UAEXXZ 1001ea7c     DNAStatMSAProfileDialog.obj
 0002:00005aa0       __unwindtable$?run@DNAStatMSAProfileTask@U2@@UAEXXZ 1001eaa0     DNAStatMSAProfileDialog.obj
 0002:00005cf0       __ehfuncinfo$?generateReport@DNAStatMSAProfileTask@U2@@UBE?AVQString@@XZ 1001ecf0     DNAStatMSAProfileDialog.obj
 0002:00005d14       __unwindtable$?generateReport@DNAStatMSAProfileTask@U2@@UBE?AVQString@@XZ 1001ed14     DNAStatMSAProfileDialog.obj
 0002:00005d5c       __ehfuncinfo$?report@DNAStatMSAProfileTask@U2@@UAE?AW4ReportResult@Task@2@XZ 1001ed5c     DNAStatMSAProfileDialog.obj
 0002:00005d80       __unwindtable$?report@DNAStatMSAProfileTask@U2@@UAE?AW4ReportResult@Task@2@XZ 1001ed80     DNAStatMSAProfileDialog.obj
 0002:00005dd0       __unwindtable$?computeStats@DNAStatMSAProfileTask@U2@@AAEXXZ 1001edd0     DNAStatMSAProfileDialog.obj
 0002:00005de8       __ehfuncinfo$?computeStats@DNAStatMSAProfileTask@U2@@AAEXXZ 1001ede8     DNAStatMSAProfileDialog.obj
 0002:00005e0c       __unwindtable$?clear@?$QVector@UColumnStat@DNAStatMSAProfileTask@U2@@@@QAEXXZ 1001ee0c     DNAStatMSAProfileDialog.obj
 0002:00005e14       __ehfuncinfo$?clear@?$QVector@UColumnStat@DNAStatMSAProfileTask@U2@@@@QAEXXZ 1001ee14     DNAStatMSAProfileDialog.obj
 0002:00005e38       __catchsym$?reallocData@?$QVector@UColumnStat@DNAStatMSAProfileTask@U2@@@@AAEXHHV?$QFlags@W4AllocationOption@QArrayData@@@@@Z$7 1001ee38     DNAStatMSAProfileDialog.obj
 0002:00005e48       __catchsym$?reallocData@?$QVector@UColumnStat@DNAStatMSAProfileTask@U2@@@@AAEXHHV?$QFlags@W4AllocationOption@QArrayData@@@@@Z$6 1001ee48     DNAStatMSAProfileDialog.obj
 0002:00005e58       __ehfuncinfo$?reallocData@?$QVector@UColumnStat@DNAStatMSAProfileTask@U2@@@@AAEXHHV?$QFlags@W4AllocationOption@QArrayData@@@@@Z 1001ee58     DNAStatMSAProfileDialog.obj
 0002:00005e7c       __tryblocktable$?reallocData@?$QVector@UColumnStat@DNAStatMSAProfileTask@U2@@@@AAEXHHV?$QFlags@W4AllocationOption@QArrayData@@@@@Z 1001ee7c     DNAStatMSAProfileDialog.obj
 0002:00005ea4       __unwindtable$?reallocData@?$QVector@UColumnStat@DNAStatMSAProfileTask@U2@@@@AAEXHHV?$QFlags@W4AllocationOption@QArrayData@@@@@Z 1001eea4     DNAStatMSAProfileDialog.obj
 0002:00005ecc       __unwindtable$?copyConstruct@?$QVector@UColumnStat@DNAStatMSAProfileTask@U2@@@@AAEXPBUColumnStat@DNAStatMSAProfileTask@U2@@0PAU234@@Z 1001eecc     DNAStatMSAProfileDialog.obj
 0002:00005ed4       __ehfuncinfo$?copyConstruct@?$QVector@UColumnStat@DNAStatMSAProfileTask@U2@@@@AAEXPBUColumnStat@DNAStatMSAProfileTask@U2@@0PAU234@@Z 1001eed4     DNAStatMSAProfileDialog.obj
 0002:00005ef8       __unwindtable$?clear@?$QVector@D@@QAEXXZ 1001eef8     DNAStatMSAProfileDialog.obj
 0002:00005f00       __ehfuncinfo$?clear@?$QVector@D@@QAEXXZ 1001ef00     DNAStatMSAProfileDialog.obj
 0002:00005f24       __catchsym$?reallocData@?$QVector@D@@AAEXHHV?$QFlags@W4AllocationOption@QArrayData@@@@@Z$5 1001ef24     DNAStatMSAProfileDialog.obj
 0002:00005f34       __catchsym$?reallocData@?$QVector@D@@AAEXHHV?$QFlags@W4AllocationOption@QArrayData@@@@@Z$4 1001ef34     DNAStatMSAProfileDialog.obj
 0002:00005f44       __unwindtable$?reallocData@?$QVector@D@@AAEXHHV?$QFlags@W4AllocationOption@QArrayData@@@@@Z 1001ef44     DNAStatMSAProfileDialog.obj
 0002:00005f64       __ehfuncinfo$?reallocData@?$QVector@D@@AAEXHHV?$QFlags@W4AllocationOption@QArrayData@@@@@Z 1001ef64     DNAStatMSAProfileDialog.obj
 0002:00005f88       __tryblocktable$?reallocData@?$QVector@D@@AAEXHHV?$QFlags@W4AllocationOption@QArrayData@@@@@Z 1001ef88     DNAStatMSAProfileDialog.obj
 0002:00005fb0       __ehfuncinfo$??1DNAStatMSAProfileTask@U2@@UAE@XZ 1001efb0     DNAStatMSAProfileDialog.obj
 0002:00005fd4       __unwindtable$??1DNAStatMSAProfileTask@U2@@UAE@XZ 1001efd4     DNAStatMSAProfileDialog.obj
 0002:00006024       __unwindtable$??__EalgoLog@U2@@YAXXZ 1001f024     DNAStatPlugin.obj
 0002:0000602c       __ehfuncinfo$??__EalgoLog@U2@@YAXXZ 1001f02c     DNAStatPlugin.obj
 0002:00006050       __unwindtable$??__EcmdLog@U2@@YAXXZ 1001f050     DNAStatPlugin.obj
 0002:00006058       __ehfuncinfo$??__EcmdLog@U2@@YAXXZ 1001f058     DNAStatPlugin.obj
 0002:0000607c       __unwindtable$??__EcoreLog@U2@@YAXXZ 1001f07c     DNAStatPlugin.obj
 0002:00006084       __ehfuncinfo$??__EcoreLog@U2@@YAXXZ 1001f084     DNAStatPlugin.obj
 0002:000060a8       __unwindtable$??__EioLog@U2@@YAXXZ 1001f0a8     DNAStatPlugin.obj
 0002:000060b0       __ehfuncinfo$??__EioLog@U2@@YAXXZ 1001f0b0     DNAStatPlugin.obj
 0002:000060d4       __unwindtable$??__EperfLog@U2@@YAXXZ 1001f0d4     DNAStatPlugin.obj
 0002:000060dc       __ehfuncinfo$??__EperfLog@U2@@YAXXZ 1001f0dc     DNAStatPlugin.obj
 0002:00006100       __unwindtable$??__EscriptLog@U2@@YAXXZ 1001f100     DNAStatPlugin.obj
 0002:00006108       __ehfuncinfo$??__EscriptLog@U2@@YAXXZ 1001f108     DNAStatPlugin.obj
 0002:0000612c       __unwindtable$??__EtaskLog@U2@@YAXXZ 1001f12c     DNAStatPlugin.obj
 0002:00006134       __ehfuncinfo$??__EtaskLog@U2@@YAXXZ 1001f134     DNAStatPlugin.obj
 0002:00006158       __unwindtable$??__EuiLog@U2@@YAXXZ 1001f158     DNAStatPlugin.obj
 0002:00006160       __ehfuncinfo$??__EuiLog@U2@@YAXXZ 1001f160     DNAStatPlugin.obj
 0002:00006184       __unwindtable$??__EuserActLog@U2@@YAXXZ 1001f184     DNAStatPlugin.obj
 0002:0000618c       __ehfuncinfo$??__EuserActLog@U2@@YAXXZ 1001f18c     DNAStatPlugin.obj
 0002:000061b0       __ehfuncinfo$??0DNAStatPlugin@U2@@QAE@XZ 1001f1b0     DNAStatPlugin.obj
 0002:000061d4       __unwindtable$??0DNAStatPlugin@U2@@QAE@XZ 1001f1d4     DNAStatPlugin.obj
 0002:0000620c       __unwindtable$?sl_showMSAProfileDialog@DNAStatMSAEditorContext@U2@@IAEXXZ 1001f20c     DNAStatPlugin.obj
 0002:00006224       __ehfuncinfo$?sl_showMSAProfileDialog@DNAStatMSAEditorContext@U2@@IAEXXZ 1001f224     DNAStatPlugin.obj
 0002:00006248       __ehfuncinfo$?buildMenu@DNAStatMSAEditorContext@U2@@MAEXPAVGObjectView@2@PAVQMenu@@@Z 1001f248     DNAStatPlugin.obj
 0002:0000626c       __unwindtable$?buildMenu@DNAStatMSAEditorContext@U2@@MAEXPAVGObjectView@2@PAVQMenu@@@Z 1001f26c     DNAStatPlugin.obj
 0002:000062b4       __unwindtable$?initViewContext@DNAStatMSAEditorContext@U2@@MAEXPAVGObjectView@2@@Z 1001f2b4     DNAStatPlugin.obj
 0002:000062d4       __ehfuncinfo$?initViewContext@DNAStatMSAEditorContext@U2@@MAEXPAVGObjectView@2@@Z 1001f2d4     DNAStatPlugin.obj
 0002:000062f8       __unwindtable$?sl_showDistanceMatrixDialog@DistanceMatrixMSAEditorContext@U2@@IAEXXZ 1001f2f8     DNAStatPlugin.obj
 0002:00006310       __ehfuncinfo$?sl_showDistanceMatrixDialog@DistanceMatrixMSAEditorContext@U2@@IAEXXZ 1001f310     DNAStatPlugin.obj
 0002:00006334       __ehfuncinfo$?buildMenu@DistanceMatrixMSAEditorContext@U2@@MAEXPAVGObjectView@2@PAVQMenu@@@Z 1001f334     DNAStatPlugin.obj
 0002:00006358       __unwindtable$?buildMenu@DistanceMatrixMSAEditorContext@U2@@MAEXPAVGObjectView@2@PAVQMenu@@@Z 1001f358     DNAStatPlugin.obj
 0002:000063a0       __unwindtable$?initViewContext@DistanceMatrixMSAEditorContext@U2@@MAEXPAVGObjectView@2@@Z 1001f3a0     DNAStatPlugin.obj
 0002:000063c0       __ehfuncinfo$?initViewContext@DistanceMatrixMSAEditorContext@U2@@MAEXPAVGObjectView@2@@Z 1001f3c0     DNAStatPlugin.obj
 0002:000063e4       __catchsym$??0?$QList@PAVGObjectViewAction@U2@@@@QAE@ABV0@@Z$2 1001f3e4     DNAStatPlugin.obj
 0002:000063f4       __unwindtable$??0?$QList@PAVGObjectViewAction@U2@@@@QAE@ABV0@@Z 1001f3f4     DNAStatPlugin.obj
 0002:00006404       __tryblocktable$??0?$QList@PAVGObjectViewAction@U2@@@@QAE@ABV0@@Z 1001f404     DNAStatPlugin.obj
 0002:00006418       __ehfuncinfo$??0?$QList@PAVGObjectViewAction@U2@@@@QAE@ABV0@@Z 1001f418     DNAStatPlugin.obj
 0002:0000643c       __unwindtable$??1?$QObjectScopedPointer@VDNAStatMSAProfileDialog@U2@@@U2@@QAE@XZ 1001f43c     DNAStatPlugin.obj
 0002:00006444       __ehfuncinfo$??1?$QObjectScopedPointer@VDNAStatMSAProfileDialog@U2@@@U2@@QAE@XZ 1001f444     DNAStatPlugin.obj
 0002:00006468       __unwindtable$??1?$QObjectScopedPointer@VDistanceMatrixMSAProfileDialog@U2@@@U2@@QAE@XZ 1001f468     DNAStatPlugin.obj
 0002:00006470       __ehfuncinfo$??1?$QObjectScopedPointer@VDistanceMatrixMSAProfileDialog@U2@@@U2@@QAE@XZ 1001f470     DNAStatPlugin.obj
 0002:00006494       __unwindtable$??__EalgoLog@U2@@YAXXZ 1001f494     DNAStatProfileTask.obj
 0002:0000649c       __ehfuncinfo$??__EalgoLog@U2@@YAXXZ 1001f49c     DNAStatProfileTask.obj
 0002:000064c0       __unwindtable$??__EcmdLog@U2@@YAXXZ 1001f4c0     DNAStatProfileTask.obj
 0002:000064c8       __ehfuncinfo$??__EcmdLog@U2@@YAXXZ 1001f4c8     DNAStatProfileTask.obj
 0002:000064ec       __unwindtable$??__EcoreLog@U2@@YAXXZ 1001f4ec     DNAStatProfileTask.obj
 0002:000064f4       __ehfuncinfo$??__EcoreLog@U2@@YAXXZ 1001f4f4     DNAStatProfileTask.obj
 0002:00006518       __unwindtable$??__EioLog@U2@@YAXXZ 1001f518     DNAStatProfileTask.obj
 0002:00006520       __ehfuncinfo$??__EioLog@U2@@YAXXZ 1001f520     DNAStatProfileTask.obj
 0002:00006544       __unwindtable$??__EperfLog@U2@@YAXXZ 1001f544     DNAStatProfileTask.obj
 0002:0000654c       __ehfuncinfo$??__EperfLog@U2@@YAXXZ 1001f54c     DNAStatProfileTask.obj
 0002:00006570       __unwindtable$??__EscriptLog@U2@@YAXXZ 1001f570     DNAStatProfileTask.obj
 0002:00006578       __ehfuncinfo$??__EscriptLog@U2@@YAXXZ 1001f578     DNAStatProfileTask.obj
 0002:0000659c       __unwindtable$??__EtaskLog@U2@@YAXXZ 1001f59c     DNAStatProfileTask.obj
 0002:000065a4       __ehfuncinfo$??__EtaskLog@U2@@YAXXZ 1001f5a4     DNAStatProfileTask.obj
 0002:000065c8       __unwindtable$??__EuiLog@U2@@YAXXZ 1001f5c8     DNAStatProfileTask.obj
 0002:000065d0       __ehfuncinfo$??__EuiLog@U2@@YAXXZ 1001f5d0     DNAStatProfileTask.obj
 0002:000065f4       __unwindtable$??__EuserActLog@U2@@YAXXZ 1001f5f4     DNAStatProfileTask.obj
 0002:000065fc       __ehfuncinfo$??__EuserActLog@U2@@YAXXZ 1001f5fc     DNAStatProfileTask.obj
 0002:00006620       __catchsym$??0?$QList@UCharOccurResult@U2@@@@QAE@ABV0@@Z$2 1001f620     DNAStatProfileTask.obj
 0002:00006630       __unwindtable$??0?$QList@UCharOccurResult@U2@@@@QAE@ABV0@@Z 1001f630     DNAStatProfileTask.obj
 0002:00006640       __tryblocktable$??0?$QList@UCharOccurResult@U2@@@@QAE@ABV0@@Z 1001f640     DNAStatProfileTask.obj
 0002:00006654       __ehfuncinfo$??0?$QList@UCharOccurResult@U2@@@@QAE@ABV0@@Z 1001f654     DNAStatProfileTask.obj
 0002:00006678       __catchsym$?node_copy@?$QList@UCharOccurResult@U2@@@@AAEXPAUNode@1@00@Z$4 1001f678     DNAStatProfileTask.obj
 0002:00006688       __tryblocktable$?node_copy@?$QList@UCharOccurResult@U2@@@@AAEXPAUNode@1@00@Z 1001f688     DNAStatProfileTask.obj
 0002:0000669c       __unwindtable$?node_copy@?$QList@UCharOccurResult@U2@@@@AAEXPAUNode@1@00@Z 1001f69c     DNAStatProfileTask.obj
 0002:000066bc       __ehfuncinfo$?node_copy@?$QList@UCharOccurResult@U2@@@@AAEXPAUNode@1@00@Z 1001f6bc     DNAStatProfileTask.obj
 0002:000066e0       __ehfuncinfo$??0DNAStatProfileTask@U2@@QAE@PAVADVSequenceObjectContext@1@@Z 1001f6e0     DNAStatProfileTask.obj
 0002:00006704       __unwindtable$??0DNAStatProfileTask@U2@@QAE@PAVADVSequenceObjectContext@1@@Z 1001f704     DNAStatProfileTask.obj
 0002:0000676c       __unwindtable$?onSubTaskFinished@DNAStatProfileTask@U2@@UAE?AV?$QList@PAVTask@U2@@@@PAVTask@2@@Z 1001f76c     DNAStatProfileTask.obj
 0002:0000678c       __ehfuncinfo$?onSubTaskFinished@DNAStatProfileTask@U2@@UAE?AV?$QList@PAVTask@U2@@@@PAVTask@2@@Z 1001f78c     DNAStatProfileTask.obj
 0002:000067b0       __unwindtable$?getResult@DNAStatProfileTask@U2@@QBE?AVQString@@XZ 1001f7b0     DNAStatProfileTask.obj
 0002:000067b8       __ehfuncinfo$?getResult@DNAStatProfileTask@U2@@QBE?AVQString@@XZ 1001f7b8     DNAStatProfileTask.obj
 0002:000067dc       __ehfuncinfo$?formCharResultString@DNAStatProfileTask@U2@@ABE?AVQString@@XZ 1001f7dc     DNAStatProfileTask.obj
 0002:00006800       __unwindtable$?formCharResultString@DNAStatProfileTask@U2@@ABE?AVQString@@XZ 1001f800     DNAStatProfileTask.obj
 0002:00006878       __ehfuncinfo$?formDinucResultString@DNAStatProfileTask@U2@@ABE?AVQString@@XZ 1001f878     DNAStatProfileTask.obj
 0002:0000689c       __unwindtable$?formDinucResultString@DNAStatProfileTask@U2@@ABE?AVQString@@XZ 1001f89c     DNAStatProfileTask.obj
 0002:00006924       __ehfuncinfo$?formStatResultString@DNAStatProfileTask@U2@@ABE?AVQString@@XZ 1001f924     DNAStatProfileTask.obj
 0002:00006948       __unwindtable$?formStatResultString@DNAStatProfileTask@U2@@ABE?AVQString@@XZ 1001f948     DNAStatProfileTask.obj
 0002:00006b40       __unwindtable$??1DNAStatProfileTask@U2@@UAE@XZ 1001fb40     DNAStatProfileTask.obj
 0002:00006b58       __ehfuncinfo$??1DNAStatProfileTask@U2@@UAE@XZ 1001fb58     DNAStatProfileTask.obj
 0002:00006b7c       __unwindtable$??_GDNAStatProfileTask@U2@@UAEPAXI@Z 1001fb7c     DNAStatProfileTask.obj
 0002:00006b94       __ehfuncinfo$??_GDNAStatProfileTask@U2@@UAEPAXI@Z 1001fb94     DNAStatProfileTask.obj
 0002:00006bb8       __catchsym$?createNode@?$QMapData@VQByteArray@@_J@@QAEPAU?$QMapNode@VQByteArray@@_J@@ABVQByteArray@@AB_JPAU2@_N@Z$5 1001fbb8     DNAStatProfileTask.obj
 0002:00006bc8       __tryblocktable$?createNode@?$QMapData@VQByteArray@@_J@@QAEPAU?$QMapNode@VQByteArray@@_J@@ABVQByteArray@@AB_JPAU2@_N@Z 1001fbc8     DNAStatProfileTask.obj
 0002:00006bdc       __ehfuncinfo$?createNode@?$QMapData@VQByteArray@@_J@@QAEPAU?$QMapNode@VQByteArray@@_J@@ABVQByteArray@@AB_JPAU2@_N@Z 1001fbdc     DNAStatProfileTask.obj
 0002:00006c00       __unwindtable$?createNode@?$QMapData@VQByteArray@@_J@@QAEPAU?$QMapNode@VQByteArray@@_J@@ABVQByteArray@@AB_JPAU2@_N@Z 1001fc00     DNAStatProfileTask.obj
 0002:00006c28       __unwindtable$??__EalgoLog@U2@@YAXXZ 1001fc28     DistanceMatrixMSAProfileDialog.obj
 0002:00006c30       __ehfuncinfo$??__EalgoLog@U2@@YAXXZ 1001fc30     DistanceMatrixMSAProfileDialog.obj
 0002:00006c54       __unwindtable$??__EcmdLog@U2@@YAXXZ 1001fc54     DistanceMatrixMSAProfileDialog.obj
 0002:00006c5c       __ehfuncinfo$??__EcmdLog@U2@@YAXXZ 1001fc5c     DistanceMatrixMSAProfileDialog.obj
 0002:00006c80       __unwindtable$??__EcoreLog@U2@@YAXXZ 1001fc80     DistanceMatrixMSAProfileDialog.obj
 0002:00006c88       __ehfuncinfo$??__EcoreLog@U2@@YAXXZ 1001fc88     DistanceMatrixMSAProfileDialog.obj
 0002:00006cac       __unwindtable$??__EioLog@U2@@YAXXZ 1001fcac     DistanceMatrixMSAProfileDialog.obj
 0002:00006cb4       __ehfuncinfo$??__EioLog@U2@@YAXXZ 1001fcb4     DistanceMatrixMSAProfileDialog.obj
 0002:00006cd8       __unwindtable$??__EperfLog@U2@@YAXXZ 1001fcd8     DistanceMatrixMSAProfileDialog.obj
 0002:00006ce0       __ehfuncinfo$??__EperfLog@U2@@YAXXZ 1001fce0     DistanceMatrixMSAProfileDialog.obj
 0002:00006d04       __unwindtable$??__EscriptLog@U2@@YAXXZ 1001fd04     DistanceMatrixMSAProfileDialog.obj
 0002:00006d0c       __ehfuncinfo$??__EscriptLog@U2@@YAXXZ 1001fd0c     DistanceMatrixMSAProfileDialog.obj
 0002:00006d30       __unwindtable$??__EtaskLog@U2@@YAXXZ 1001fd30     DistanceMatrixMSAProfileDialog.obj
 0002:00006d38       __ehfuncinfo$??__EtaskLog@U2@@YAXXZ 1001fd38     DistanceMatrixMSAProfileDialog.obj
 0002:00006d5c       __unwindtable$??__EuiLog@U2@@YAXXZ 1001fd5c     DistanceMatrixMSAProfileDialog.obj
 0002:00006d64       __ehfuncinfo$??__EuiLog@U2@@YAXXZ 1001fd64     DistanceMatrixMSAProfileDialog.obj
 0002:00006d88       __unwindtable$??__EuserActLog@U2@@YAXXZ 1001fd88     DistanceMatrixMSAProfileDialog.obj
 0002:00006d90       __ehfuncinfo$??__EuserActLog@U2@@YAXXZ 1001fd90     DistanceMatrixMSAProfileDialog.obj
 0002:00006db4       __catchsym$?append@?$QList@VMultipleSequenceAlignmentRow@U2@@@@QAEXABVMultipleSequenceAlignmentRow@U2@@@Z$9 1001fdb4     DistanceMatrixMSAProfileDialog.obj
 0002:00006dc4       __catchsym$?append@?$QList@VMultipleSequenceAlignmentRow@U2@@@@QAEXABVMultipleSequenceAlignmentRow@U2@@@Z$8 1001fdc4     DistanceMatrixMSAProfileDialog.obj
 0002:00006dd4       __ehfuncinfo$?append@?$QList@VMultipleSequenceAlignmentRow@U2@@@@QAEXABVMultipleSequenceAlignmentRow@U2@@@Z 1001fdd4     DistanceMatrixMSAProfileDialog.obj
 0002:00006df8       __tryblocktable$?append@?$QList@VMultipleSequenceAlignmentRow@U2@@@@QAEXABVMultipleSequenceAlignmentRow@U2@@@Z 1001fdf8     DistanceMatrixMSAProfileDialog.obj
 0002:00006e20       __unwindtable$?append@?$QList@VMultipleSequenceAlignmentRow@U2@@@@QAEXABVMultipleSequenceAlignmentRow@U2@@@Z 1001fe20     DistanceMatrixMSAProfileDialog.obj
 0002:00006e60       __catchsym$?detach_helper_grow@?$QList@VMultipleSequenceAlignmentRow@U2@@@@AAEPAUNode@1@HH@Z$5 1001fe60     DistanceMatrixMSAProfileDialog.obj
 0002:00006e70       __catchsym$?detach_helper_grow@?$QList@VMultipleSequenceAlignmentRow@U2@@@@AAEPAUNode@1@HH@Z$4 1001fe70     DistanceMatrixMSAProfileDialog.obj
 0002:00006e80       __unwindtable$?detach_helper_grow@?$QList@VMultipleSequenceAlignmentRow@U2@@@@AAEPAUNode@1@HH@Z 1001fe80     DistanceMatrixMSAProfileDialog.obj
 0002:00006ea0       __ehfuncinfo$?detach_helper_grow@?$QList@VMultipleSequenceAlignmentRow@U2@@@@AAEPAUNode@1@HH@Z 1001fea0     DistanceMatrixMSAProfileDialog.obj
 0002:00006ec4       __tryblocktable$?detach_helper_grow@?$QList@VMultipleSequenceAlignmentRow@U2@@@@AAEPAUNode@1@HH@Z 1001fec4     DistanceMatrixMSAProfileDialog.obj
 0002:00006eec       __unwindtable$?node_construct@?$QList@VMultipleSequenceAlignmentRow@U2@@@@AAEXPAUNode@1@ABVMultipleSequenceAlignmentRow@U2@@@Z 1001feec     DistanceMatrixMSAProfileDialog.obj
 0002:00006efc       __ehfuncinfo$?node_construct@?$QList@VMultipleSequenceAlignmentRow@U2@@@@AAEXPAUNode@1@ABVMultipleSequenceAlignmentRow@U2@@@Z 1001fefc     DistanceMatrixMSAProfileDialog.obj
 0002:00006f20       __catchsym$?node_copy@?$QList@VMultipleSequenceAlignmentRow@U2@@@@AAEXPAUNode@1@00@Z$6 1001ff20     DistanceMatrixMSAProfileDialog.obj
 0002:00006f30       __tryblocktable$?node_copy@?$QList@VMultipleSequenceAlignmentRow@U2@@@@AAEXPAUNode@1@00@Z 1001ff30     DistanceMatrixMSAProfileDialog.obj
 0002:00006f44       __ehfuncinfo$?node_copy@?$QList@VMultipleSequenceAlignmentRow@U2@@@@AAEXPAUNode@1@00@Z 1001ff44     DistanceMatrixMSAProfileDialog.obj
 0002:00006f68       __unwindtable$?node_copy@?$QList@VMultipleSequenceAlignmentRow@U2@@@@AAEXPAUNode@1@00@Z 1001ff68     DistanceMatrixMSAProfileDialog.obj
 0002:00006f98       __catchsym$??0?$QList@PAVMSADistanceAlgorithmFactory@U2@@@@QAE@ABV0@@Z$2 1001ff98     DistanceMatrixMSAProfileDialog.obj
 0002:00006fa8       __unwindtable$??0?$QList@PAVMSADistanceAlgorithmFactory@U2@@@@QAE@ABV0@@Z 1001ffa8     DistanceMatrixMSAProfileDialog.obj
 0002:00006fb8       __tryblocktable$??0?$QList@PAVMSADistanceAlgorithmFactory@U2@@@@QAE@ABV0@@Z 1001ffb8     DistanceMatrixMSAProfileDialog.obj
 0002:00006fcc       __ehfuncinfo$??0?$QList@PAVMSADistanceAlgorithmFactory@U2@@@@QAE@ABV0@@Z 1001ffcc     DistanceMatrixMSAProfileDialog.obj
 0002:00006ff0       __ehfuncinfo$?setupUi@Ui_DistanceMatrixMSAProfileDialog@@QAEXPAVQDialog@@@Z 1001fff0     DistanceMatrixMSAProfileDialog.obj
 0002:00007014       __unwindtable$?setupUi@Ui_DistanceMatrixMSAProfileDialog@@QAEXPAVQDialog@@@Z 10020014     DistanceMatrixMSAProfileDialog.obj
 0002:00007144       __ehfuncinfo$?retranslateUi@Ui_DistanceMatrixMSAProfileDialog@@QAEXPAVQDialog@@@Z 10020144     DistanceMatrixMSAProfileDialog.obj
 0002:00007168       __unwindtable$?retranslateUi@Ui_DistanceMatrixMSAProfileDialog@@QAEXPAVQDialog@@@Z 10020168     DistanceMatrixMSAProfileDialog.obj
 0002:000071c8       __ehfuncinfo$??0DistanceMatrixMSAProfileDialog@U2@@QAE@PAVQWidget@@PAVMSAEditor@1@@Z 100201c8     DistanceMatrixMSAProfileDialog.obj
 0002:000071ec       __unwindtable$??0DistanceMatrixMSAProfileDialog@U2@@QAE@PAVQWidget@@PAVMSAEditor@1@@Z 100201ec     DistanceMatrixMSAProfileDialog.obj
 0002:0000725c       __ehfuncinfo$?accept@DistanceMatrixMSAProfileDialog@U2@@UAEXXZ 1002025c     DistanceMatrixMSAProfileDialog.obj
 0002:00007280       __unwindtable$?accept@DistanceMatrixMSAProfileDialog@U2@@UAEXXZ 10020280     DistanceMatrixMSAProfileDialog.obj
 0002:000072e0       __ehfuncinfo$?initSaveController@DistanceMatrixMSAProfileDialog@U2@@AAEXXZ 100202e0     DistanceMatrixMSAProfileDialog.obj
 0002:00007304       __unwindtable$?initSaveController@DistanceMatrixMSAProfileDialog@U2@@AAEXXZ 10020304     DistanceMatrixMSAProfileDialog.obj
 0002:00007394       __ehfuncinfo$??0DistanceMatrixMSAProfileTaskSettings@U2@@QAE@XZ 10020394     DistanceMatrixMSAProfileDialog.obj
 0002:000073b8       __unwindtable$??0DistanceMatrixMSAProfileTaskSettings@U2@@QAE@XZ 100203b8     DistanceMatrixMSAProfileDialog.obj
 0002:000073f8       __unwindtable$??1DistanceMatrixMSAProfileTaskSettings@U2@@QAE@XZ 100203f8     DistanceMatrixMSAProfileDialog.obj
 0002:00007418       __ehfuncinfo$??1DistanceMatrixMSAProfileTaskSettings@U2@@QAE@XZ 10020418     DistanceMatrixMSAProfileDialog.obj
 0002:0000743c       __unwindtable$??0DistanceMatrixMSAProfileTaskSettings@U2@@QAE@ABV01@@Z 1002043c     DistanceMatrixMSAProfileDialog.obj
 0002:0000745c       __ehfuncinfo$??0DistanceMatrixMSAProfileTaskSettings@U2@@QAE@ABV01@@Z 1002045c     DistanceMatrixMSAProfileDialog.obj
 0002:00007480       __ehfuncinfo$??0DistanceMatrixMSAProfileTask@U2@@QAE@ABVDistanceMatrixMSAProfileTaskSettings@1@@Z 10020480     DistanceMatrixMSAProfileDialog.obj
 0002:000074a4       __unwindtable$??0DistanceMatrixMSAProfileTask@U2@@QAE@ABVDistanceMatrixMSAProfileTaskSettings@1@@Z 100204a4     DistanceMatrixMSAProfileDialog.obj
 0002:000074cc       __ehfuncinfo$?generateReport@DistanceMatrixMSAProfileTask@U2@@UBE?AVQString@@XZ 100204cc     DistanceMatrixMSAProfileDialog.obj
 0002:000074f0       __unwindtable$?generateReport@DistanceMatrixMSAProfileTask@U2@@UBE?AVQString@@XZ 100204f0     DistanceMatrixMSAProfileDialog.obj
 0002:00007538       __ehfuncinfo$?createDistanceTable@DistanceMatrixMSAProfileTask@U2@@QAEXPAVMSADistanceAlgorithm@2@ABV?$QList@VMultipleSequenceAlignmentRow@U2@@@@PAVQFile@@@Z 10020538     DistanceMatrixMSAProfileDialog.obj
 0002:0000755c       __unwindtable$?createDistanceTable@DistanceMatrixMSAProfileTask@U2@@QAEXPAVMSADistanceAlgorithm@2@ABV?$QList@VMultipleSequenceAlignmentRow@U2@@@@PAVQFile@@@Z 1002055c     DistanceMatrixMSAProfileDialog.obj
 0002:0000762c       __catchsym$?onSubTaskFinished@DistanceMatrixMSAProfileTask@U2@@UAE?AV?$QList@PAVTask@U2@@@@PAVTask@2@@Z$103 1002062c     DistanceMatrixMSAProfileDialog.obj
 0002:0000763c       __catchsym$?onSubTaskFinished@DistanceMatrixMSAProfileTask@U2@@UAE?AV?$QList@PAVTask@U2@@@@PAVTask@2@@Z$102 1002063c     DistanceMatrixMSAProfileDialog.obj
 0002:0000764c       __ehfuncinfo$?onSubTaskFinished@DistanceMatrixMSAProfileTask@U2@@UAE?AV?$QList@PAVTask@U2@@@@PAVTask@2@@Z 1002064c     DistanceMatrixMSAProfileDialog.obj
 0002:00007670       __tryblocktable$?onSubTaskFinished@DistanceMatrixMSAProfileTask@U2@@UAE?AV?$QList@PAVTask@U2@@@@PAVTask@2@@Z 10020670     DistanceMatrixMSAProfileDialog.obj
 0002:00007698       __unwindtable$?onSubTaskFinished@DistanceMatrixMSAProfileTask@U2@@UAE?AV?$QList@PAVTask@U2@@@@PAVTask@2@@Z 10020698     DistanceMatrixMSAProfileDialog.obj
 0002:000079a0       __ehfuncinfo$?report@DistanceMatrixMSAProfileTask@U2@@UAE?AW4ReportResult@Task@2@XZ 100209a0     DistanceMatrixMSAProfileDialog.obj
 0002:000079c4       __unwindtable$?report@DistanceMatrixMSAProfileTask@U2@@UAE?AW4ReportResult@Task@2@XZ 100209c4     DistanceMatrixMSAProfileDialog.obj
 0002:00007a14       __ehfuncinfo$??1DistanceMatrixMSAProfileTask@U2@@UAE@XZ 10020a14     DistanceMatrixMSAProfileDialog.obj
 0002:00007a38       __unwindtable$??1DistanceMatrixMSAProfileTask@U2@@UAE@XZ 10020a38     DistanceMatrixMSAProfileDialog.obj
 0002:00007a68       __unwindtable$??0?$QForeachContainer@V?$QVector@VU2Region@U2@@@@@@QAE@ABV?$QVector@VU2Region@U2@@@@@Z 10020a68     DistanceMatrixMSAProfileDialog.obj
 0002:00007a70       __ehfuncinfo$??0?$QForeachContainer@V?$QVector@VU2Region@U2@@@@@@QAE@ABV?$QVector@VU2Region@U2@@@@@Z 10020a70     DistanceMatrixMSAProfileDialog.obj
 0002:00007a94       __unwindtable$??__EalgoLog@U2@@YAXXZ 10020a94     moc_DNAStatMSAProfileDialog.obj
 0002:00007a9c       __ehfuncinfo$??__EalgoLog@U2@@YAXXZ 10020a9c     moc_DNAStatMSAProfileDialog.obj
 0002:00007ac0       __unwindtable$??__EcmdLog@U2@@YAXXZ 10020ac0     moc_DNAStatMSAProfileDialog.obj
 0002:00007ac8       __ehfuncinfo$??__EcmdLog@U2@@YAXXZ 10020ac8     moc_DNAStatMSAProfileDialog.obj
 0002:00007aec       __unwindtable$??__EcoreLog@U2@@YAXXZ 10020aec     moc_DNAStatMSAProfileDialog.obj
 0002:00007af4       __ehfuncinfo$??__EcoreLog@U2@@YAXXZ 10020af4     moc_DNAStatMSAProfileDialog.obj
 0002:00007b18       __unwindtable$??__EioLog@U2@@YAXXZ 10020b18     moc_DNAStatMSAProfileDialog.obj
 0002:00007b20       __ehfuncinfo$??__EioLog@U2@@YAXXZ 10020b20     moc_DNAStatMSAProfileDialog.obj
 0002:00007b44       __unwindtable$??__EperfLog@U2@@YAXXZ 10020b44     moc_DNAStatMSAProfileDialog.obj
 0002:00007b4c       __ehfuncinfo$??__EperfLog@U2@@YAXXZ 10020b4c     moc_DNAStatMSAProfileDialog.obj
 0002:00007b70       __unwindtable$??__EscriptLog@U2@@YAXXZ 10020b70     moc_DNAStatMSAProfileDialog.obj
 0002:00007b78       __ehfuncinfo$??__EscriptLog@U2@@YAXXZ 10020b78     moc_DNAStatMSAProfileDialog.obj
 0002:00007b9c       __unwindtable$??__EtaskLog@U2@@YAXXZ 10020b9c     moc_DNAStatMSAProfileDialog.obj
 0002:00007ba4       __ehfuncinfo$??__EtaskLog@U2@@YAXXZ 10020ba4     moc_DNAStatMSAProfileDialog.obj
 0002:00007bc8       __unwindtable$??__EuiLog@U2@@YAXXZ 10020bc8     moc_DNAStatMSAProfileDialog.obj
 0002:00007bd0       __ehfuncinfo$??__EuiLog@U2@@YAXXZ 10020bd0     moc_DNAStatMSAProfileDialog.obj
 0002:00007bf4       __unwindtable$??__EuserActLog@U2@@YAXXZ 10020bf4     moc_DNAStatMSAProfileDialog.obj
 0002:00007bfc       __ehfuncinfo$??__EuserActLog@U2@@YAXXZ 10020bfc     moc_DNAStatMSAProfileDialog.obj
 0002:00007c20       __unwindtable$?qt_metatype_id@?$QMetaTypeIdQObject@PAVGObjectView@U2@@$00@@SAHXZ 10020c20     moc_DNAStatPlugin.obj
 0002:00007c28       __ehfuncinfo$?qt_metatype_id@?$QMetaTypeIdQObject@PAVGObjectView@U2@@$00@@SAHXZ 10020c28     moc_DNAStatPlugin.obj
 0002:00007c4c       __unwindtable$?qt_metatype_id@?$QMetaTypeIdQObject@PAVQMenu@@$00@@SAHXZ 10020c4c     moc_DNAStatPlugin.obj
 0002:00007c54       __ehfuncinfo$?qt_metatype_id@?$QMetaTypeIdQObject@PAVQMenu@@$00@@SAHXZ 10020c54     moc_DNAStatPlugin.obj
 0002:00007c78       __unwindtable$??__EalgoLog@U2@@YAXXZ 10020c78     moc_DNAStatProfileTask.obj
 0002:00007c80       __ehfuncinfo$??__EalgoLog@U2@@YAXXZ 10020c80     moc_DNAStatProfileTask.obj
 0002:00007ca4       __unwindtable$??__EcmdLog@U2@@YAXXZ 10020ca4     moc_DNAStatProfileTask.obj
 0002:00007cac       __ehfuncinfo$??__EcmdLog@U2@@YAXXZ 10020cac     moc_DNAStatProfileTask.obj
 0002:00007cd0       __unwindtable$??__EcoreLog@U2@@YAXXZ 10020cd0     moc_DNAStatProfileTask.obj
 0002:00007cd8       __ehfuncinfo$??__EcoreLog@U2@@YAXXZ 10020cd8     moc_DNAStatProfileTask.obj
 0002:00007cfc       __unwindtable$??__EioLog@U2@@YAXXZ 10020cfc     moc_DNAStatProfileTask.obj
 0002:00007d04       __ehfuncinfo$??__EioLog@U2@@YAXXZ 10020d04     moc_DNAStatProfileTask.obj
 0002:00007d28       __unwindtable$??__EperfLog@U2@@YAXXZ 10020d28     moc_DNAStatProfileTask.obj
 0002:00007d30       __ehfuncinfo$??__EperfLog@U2@@YAXXZ 10020d30     moc_DNAStatProfileTask.obj
 0002:00007d54       __unwindtable$??__EscriptLog@U2@@YAXXZ 10020d54     moc_DNAStatProfileTask.obj
 0002:00007d5c       __ehfuncinfo$??__EscriptLog@U2@@YAXXZ 10020d5c     moc_DNAStatProfileTask.obj
 0002:00007d80       __unwindtable$??__EtaskLog@U2@@YAXXZ 10020d80     moc_DNAStatProfileTask.obj
 0002:00007d88       __ehfuncinfo$??__EtaskLog@U2@@YAXXZ 10020d88     moc_DNAStatProfileTask.obj
 0002:00007dac       __unwindtable$??__EuiLog@U2@@YAXXZ 10020dac     moc_DNAStatProfileTask.obj
 0002:00007db4       __ehfuncinfo$??__EuiLog@U2@@YAXXZ 10020db4     moc_DNAStatProfileTask.obj
 0002:00007dd8       __unwindtable$??__EuserActLog@U2@@YAXXZ 10020dd8     moc_DNAStatProfileTask.obj
 0002:00007de0       __ehfuncinfo$??__EuserActLog@U2@@YAXXZ 10020de0     moc_DNAStatProfileTask.obj
 0002:00007e04       __unwindtable$??__EalgoLog@U2@@YAXXZ 10020e04     moc_DistanceMatrixMSAProfileDialog.obj
 0002:00007e0c       __ehfuncinfo$??__EalgoLog@U2@@YAXXZ 10020e0c     moc_DistanceMatrixMSAProfileDialog.obj
 0002:00007e30       __unwindtable$??__EcmdLog@U2@@YAXXZ 10020e30     moc_DistanceMatrixMSAProfileDialog.obj
 0002:00007e38       __ehfuncinfo$??__EcmdLog@U2@@YAXXZ 10020e38     moc_DistanceMatrixMSAProfileDialog.obj
 0002:00007e5c       __unwindtable$??__EcoreLog@U2@@YAXXZ 10020e5c     moc_DistanceMatrixMSAProfileDialog.obj
 0002:00007e64       __ehfuncinfo$??__EcoreLog@U2@@YAXXZ 10020e64     moc_DistanceMatrixMSAProfileDialog.obj
 0002:00007e88       __unwindtable$??__EioLog@U2@@YAXXZ 10020e88     moc_DistanceMatrixMSAProfileDialog.obj
 0002:00007e90       __ehfuncinfo$??__EioLog@U2@@YAXXZ 10020e90     moc_DistanceMatrixMSAProfileDialog.obj
 0002:00007eb4       __unwindtable$??__EperfLog@U2@@YAXXZ 10020eb4     moc_DistanceMatrixMSAProfileDialog.obj
 0002:00007ebc       __ehfuncinfo$??__EperfLog@U2@@YAXXZ 10020ebc     moc_DistanceMatrixMSAProfileDialog.obj
 0002:00007ee0       __unwindtable$??__EscriptLog@U2@@YAXXZ 10020ee0     moc_DistanceMatrixMSAProfileDialog.obj
 0002:00007ee8       __ehfuncinfo$??__EscriptLog@U2@@YAXXZ 10020ee8     moc_DistanceMatrixMSAProfileDialog.obj
 0002:00007f0c       __unwindtable$??__EtaskLog@U2@@YAXXZ 10020f0c     moc_DistanceMatrixMSAProfileDialog.obj
 0002:00007f14       __ehfuncinfo$??__EtaskLog@U2@@YAXXZ 10020f14     moc_DistanceMatrixMSAProfileDialog.obj
 0002:00007f38       __unwindtable$??__EuiLog@U2@@YAXXZ 10020f38     moc_DistanceMatrixMSAProfileDialog.obj
 0002:00007f40       __ehfuncinfo$??__EuiLog@U2@@YAXXZ 10020f40     moc_DistanceMatrixMSAProfileDialog.obj
 0002:00007f64       __unwindtable$??__EuserActLog@U2@@YAXXZ 10020f64     moc_DistanceMatrixMSAProfileDialog.obj
 0002:00007f6c       __ehfuncinfo$??__EuserActLog@U2@@YAXXZ 10020f6c     moc_DistanceMatrixMSAProfileDialog.obj
 0002:00007f90       __sehtable$??_M@YGXPAXIHP6EX0@Z@Z 10020f90     MSVCRT:ehvecdtr.obj
 0002:00007fb0       __sehtable$?__ArrayUnwind@@YGXPAXIHP6EX0@Z@Z 10020fb0     MSVCRT:ehvecdtr.obj
 0002:00007fd0       __sehtable$__onexit        10020fd0     MSVCRT:atonexit.obj
 0002:00007ff0       __sehtable$___DllMainCRTStartup 10020ff0     MSVCRT:crtdll.obj
 0002:00008018       __sehtable$__IsNonwritableInCurrentImage 10021018     MSVCRT:pesect.obj
 0002:00008040       .edata                     10021040     dna_stat.exp
 0002:00008068       rgpv                       10021068     dna_stat.exp
 0002:0000806c       rgszName                   1002106c     dna_stat.exp
 0002:00008070       rgwOrd                     10021070     dna_stat.exp
 0002:00008072       szName                     10021072     dna_stat.exp
 0002:0000807f       $N00001                    1002107f     dna_stat.exp
 0002:00009978       .idata$6                   10022978     U2Core:U2Core.dll
 0002:00009baa       .idata$6                   10022baa     U2Algorithm:U2Algorithm.dll
 0002:0000a7a8       .idata$6                   100237a8     U2Gui:U2Gui.dll
 0002:0000ad06       .idata$6                   10023d06     U2View:U2View.dll
 0002:0000e25a       .idata$6                   1002725a     Qt5Widgets:Qt5Widgets.dll
 0002:0000e2b2       .idata$6                   100272b2     Qt5Gui:Qt5Gui.dll
 0002:0000f4de       .idata$6                   100284de     Qt5Core:Qt5Core.dll
 0002:0000f584       .idata$6                   10028584     msvcprt:MSVCP120.dll
 0002:0000f62e       .idata$6                   1002862e     MSVCRT:MSVCR120.dll
 0002:0000f83a       .idata$6                   1002883a     kernel32:KERNEL32.dll
 0003:0000000c       _Service_PluginViewer      1002900c     DNAStatMSAProfileDialog.obj
 0003:00000014       _Service_Project           10029014     DNAStatMSAProfileDialog.obj
 0003:0000001c       _Service_ProjectView       1002901c     DNAStatMSAProfileDialog.obj
 0003:00000024       _Service_DNAGraphPack      10029024     DNAStatMSAProfileDialog.obj
 0003:0000002c       _Service_DNAExport         1002902c     DNAStatMSAProfileDialog.obj
 0003:00000034       _Service_TestRunner        10029034     DNAStatMSAProfileDialog.obj
 0003:0000003c       _Service_ScriptRegistry    1002903c     DNAStatMSAProfileDialog.obj
 0003:00000044       _Service_ExternalToolSupport 10029044     DNAStatMSAProfileDialog.obj
 0003:0000004c       _Service_GUITesting        1002904c     DNAStatMSAProfileDialog.obj
 0003:00000054       _Service_WorkflowDesigner  10029054     DNAStatMSAProfileDialog.obj
 0003:0000005c       _Service_QueryDesigner     1002905c     DNAStatMSAProfileDialog.obj
 0003:00000064       _Service_MinCoreServiceId  10029064     DNAStatMSAProfileDialog.obj
 0003:0000006c       _Service_MaxCoreServiceId  1002906c     DNAStatMSAProfileDialog.obj
 0003:00000074       _Service_PluginViewer      10029074     DNAStatPlugin.obj
 0003:0000007c       _Service_Project           1002907c     DNAStatPlugin.obj
 0003:00000084       _Service_ProjectView       10029084     DNAStatPlugin.obj
 0003:0000008c       _Service_DNAGraphPack      1002908c     DNAStatPlugin.obj
 0003:00000094       _Service_DNAExport         10029094     DNAStatPlugin.obj
 0003:0000009c       _Service_TestRunner        1002909c     DNAStatPlugin.obj
 0003:000000a4       _Service_ScriptRegistry    100290a4     DNAStatPlugin.obj
 0003:000000ac       _Service_ExternalToolSupport 100290ac     DNAStatPlugin.obj
 0003:000000b4       _Service_GUITesting        100290b4     DNAStatPlugin.obj
 0003:000000bc       _Service_WorkflowDesigner  100290bc     DNAStatPlugin.obj
 0003:000000c4       _Service_QueryDesigner     100290c4     DNAStatPlugin.obj
 0003:000000cc       _Service_MinCoreServiceId  100290cc     DNAStatPlugin.obj
 0003:000000d4       _Service_MaxCoreServiceId  100290d4     DNAStatPlugin.obj
 0003:000000dc       _Service_PluginViewer      100290dc     DNAStatProfileTask.obj
 0003:000000e4       _Service_Project           100290e4     DNAStatProfileTask.obj
 0003:000000ec       _Service_ProjectView       100290ec     DNAStatProfileTask.obj
 0003:000000f4       _Service_DNAGraphPack      100290f4     DNAStatProfileTask.obj
 0003:000000fc       _Service_DNAExport         100290fc     DNAStatProfileTask.obj
 0003:00000104       _Service_TestRunner        10029104     DNAStatProfileTask.obj
 0003:0000010c       _Service_ScriptRegistry    1002910c     DNAStatProfileTask.obj
 0003:00000114       _Service_ExternalToolSupport 10029114     DNAStatProfileTask.obj
 0003:0000011c       _Service_GUITesting        1002911c     DNAStatProfileTask.obj
 0003:00000124       _Service_WorkflowDesigner  10029124     DNAStatProfileTask.obj
 0003:0000012c       _Service_QueryDesigner     1002912c     DNAStatProfileTask.obj
 0003:00000134       _Service_MinCoreServiceId  10029134     DNAStatProfileTask.obj
 0003:0000013c       _Service_MaxCoreServiceId  1002913c     DNAStatProfileTask.obj
 0003:00000144       _Service_PluginViewer      10029144     DistanceMatrixMSAProfileDialog.obj
 0003:0000014c       _Service_Project           1002914c     DistanceMatrixMSAProfileDialog.obj
 0003:00000154       _Service_ProjectView       10029154     DistanceMatrixMSAProfileDialog.obj
 0003:0000015c       _Service_DNAGraphPack      1002915c     DistanceMatrixMSAProfileDialog.obj
 0003:00000164       _Service_DNAExport         10029164     DistanceMatrixMSAProfileDialog.obj
 0003:0000016c       _Service_TestRunner        1002916c     DistanceMatrixMSAProfileDialog.obj
 0003:00000174       _Service_ScriptRegistry    10029174     DistanceMatrixMSAProfileDialog.obj
 0003:0000017c       _Service_ExternalToolSupport 1002917c     DistanceMatrixMSAProfileDialog.obj
 0003:00000184       _Service_GUITesting        10029184     DistanceMatrixMSAProfileDialog.obj
 0003:0000018c       _Service_WorkflowDesigner  1002918c     DistanceMatrixMSAProfileDialog.obj
 0003:00000194       _Service_QueryDesigner     10029194     DistanceMatrixMSAProfileDialog.obj
 0003:0000019c       _Service_MinCoreServiceId  1002919c     DistanceMatrixMSAProfileDialog.obj
 0003:000001a4       _Service_MaxCoreServiceId  100291a4     DistanceMatrixMSAProfileDialog.obj
 0003:000001dc       _Service_PluginViewer      100291dc     moc_DNAStatPlugin.obj
 0003:000001e4       _Service_Project           100291e4     moc_DNAStatPlugin.obj
 0003:000001ec       _Service_ProjectView       100291ec     moc_DNAStatPlugin.obj
 0003:000001f4       _Service_DNAGraphPack      100291f4     moc_DNAStatPlugin.obj
 0003:000001fc       _Service_DNAExport         100291fc     moc_DNAStatPlugin.obj
 0003:00000204       _Service_TestRunner        10029204     moc_DNAStatPlugin.obj
 0003:0000020c       _Service_ScriptRegistry    1002920c     moc_DNAStatPlugin.obj
 0003:00000214       _Service_ExternalToolSupport 10029214     moc_DNAStatPlugin.obj
 0003:0000021c       _Service_GUITesting        1002921c     moc_DNAStatPlugin.obj
 0003:00000224       _Service_WorkflowDesigner  10029224     moc_DNAStatPlugin.obj
 0003:0000022c       _Service_QueryDesigner     1002922c     moc_DNAStatPlugin.obj
 0003:00000234       _Service_MinCoreServiceId  10029234     moc_DNAStatPlugin.obj
 0003:0000023c       _Service_MaxCoreServiceId  1002923c     moc_DNAStatPlugin.obj
 0003:00000b10       __Tuple_alloc              10029b10     DNAStatMSAProfileDialog.obj
 0003:00000b11       _ignore                    10029b11     DNAStatMSAProfileDialog.obj
 0003:00000b12       _allocator_arg             10029b12     DNAStatMSAProfileDialog.obj
 0003:00000b13       _piecewise_construct       10029b13     DNAStatMSAProfileDialog.obj
 0003:00000b14       _taskLog                   10029b14     DNAStatMSAProfileDialog.obj
 0003:00000b1c       _algoLog                   10029b1c     DNAStatMSAProfileDialog.obj
 0003:00000b24       _userActLog                10029b24     DNAStatMSAProfileDialog.obj
 0003:00000b2c       _ioLog                     10029b2c     DNAStatMSAProfileDialog.obj
 0003:00000b38       _coreLog                   10029b38     DNAStatMSAProfileDialog.obj
 0003:00000b40       _uiLog                     10029b40     DNAStatMSAProfileDialog.obj
 0003:00000b48       _scriptLog                 10029b48     DNAStatMSAProfileDialog.obj
 0003:00000b50       _perfLog                   10029b50     DNAStatMSAProfileDialog.obj
 0003:00000b58       _cmdLog                    10029b58     DNAStatMSAProfileDialog.obj
 0003:00000b6c       __Tuple_alloc              10029b6c     DNAStatPlugin.obj
 0003:00000b6d       _ignore                    10029b6d     DNAStatPlugin.obj
 0003:00000b6e       _allocator_arg             10029b6e     DNAStatPlugin.obj
 0003:00000b6f       _piecewise_construct       10029b6f     DNAStatPlugin.obj
 0003:00000b70       _taskLog                   10029b70     DNAStatPlugin.obj
 0003:00000b78       _algoLog                   10029b78     DNAStatPlugin.obj
 0003:00000b80       _userActLog                10029b80     DNAStatPlugin.obj
 0003:00000b88       _ioLog                     10029b88     DNAStatPlugin.obj
 0003:00000b90       _coreLog                   10029b90     DNAStatPlugin.obj
 0003:00000b98       _uiLog                     10029b98     DNAStatPlugin.obj
 0003:00000ba0       _scriptLog                 10029ba0     DNAStatPlugin.obj
 0003:00000ba8       _perfLog                   10029ba8     DNAStatPlugin.obj
 0003:00000bb0       _cmdLog                    10029bb0     DNAStatPlugin.obj
 0003:00000bb8       __Tuple_alloc              10029bb8     DNAStatProfileTask.obj
 0003:00000bb9       _ignore                    10029bb9     DNAStatProfileTask.obj
 0003:00000bba       _allocator_arg             10029bba     DNAStatProfileTask.obj
 0003:00000bbb       _piecewise_construct       10029bbb     DNAStatProfileTask.obj
 0003:00000bbc       _taskLog                   10029bbc     DNAStatProfileTask.obj
 0003:00000bc4       _algoLog                   10029bc4     DNAStatProfileTask.obj
 0003:00000bcc       _userActLog                10029bcc     DNAStatProfileTask.obj
 0003:00000bd4       _ioLog                     10029bd4     DNAStatProfileTask.obj
 0003:00000bdc       _coreLog                   10029bdc     DNAStatProfileTask.obj
 0003:00000be4       _uiLog                     10029be4     DNAStatProfileTask.obj
 0003:00000bec       _scriptLog                 10029bec     DNAStatProfileTask.obj
 0003:00000bf4       _perfLog                   10029bf4     DNAStatProfileTask.obj
 0003:00000bfc       _cmdLog                    10029bfc     DNAStatProfileTask.obj
 0003:00000c04       __Tuple_alloc              10029c04     DistanceMatrixMSAProfileDialog.obj
 0003:00000c05       _ignore                    10029c05     DistanceMatrixMSAProfileDialog.obj
 0003:00000c06       _allocator_arg             10029c06     DistanceMatrixMSAProfileDialog.obj
 0003:00000c07       _piecewise_construct       10029c07     DistanceMatrixMSAProfileDialog.obj
 0003:00000c08       _taskLog                   10029c08     DistanceMatrixMSAProfileDialog.obj
 0003:00000c10       _algoLog                   10029c10     DistanceMatrixMSAProfileDialog.obj
 0003:00000c18       _userActLog                10029c18     DistanceMatrixMSAProfileDialog.obj
 0003:00000c20       _ioLog                     10029c20     DistanceMatrixMSAProfileDialog.obj
 0003:00000c28       _coreLog                   10029c28     DistanceMatrixMSAProfileDialog.obj
 0003:00000c34       _uiLog                     10029c34     DistanceMatrixMSAProfileDialog.obj
 0003:00000c3c       _scriptLog                 10029c3c     DistanceMatrixMSAProfileDialog.obj
 0003:00000c48       _perfLog                   10029c48     DistanceMatrixMSAProfileDialog.obj
 0003:00000c50       _cmdLog                    10029c50     DistanceMatrixMSAProfileDialog.obj
 0003:00000c58       __Tuple_alloc              10029c58     moc_DNAStatMSAProfileDialog.obj
 0003:00000c59       _ignore                    10029c59     moc_DNAStatMSAProfileDialog.obj
 0003:00000c5a       _allocator_arg             10029c5a     moc_DNAStatMSAProfileDialog.obj
 0003:00000c5b       _piecewise_construct       10029c5b     moc_DNAStatMSAProfileDialog.obj
 0003:00000c5c       _taskLog                   10029c5c     moc_DNAStatMSAProfileDialog.obj
 0003:00000c64       _algoLog                   10029c64     moc_DNAStatMSAProfileDialog.obj
 0003:00000c6c       _userActLog                10029c6c     moc_DNAStatMSAProfileDialog.obj
 0003:00000c74       _ioLog                     10029c74     moc_DNAStatMSAProfileDialog.obj
 0003:00000c7c       _coreLog                   10029c7c     moc_DNAStatMSAProfileDialog.obj
 0003:00000c84       _uiLog                     10029c84     moc_DNAStatMSAProfileDialog.obj
 0003:00000c8c       _scriptLog                 10029c8c     moc_DNAStatMSAProfileDialog.obj
 0003:00000c94       _perfLog                   10029c94     moc_DNAStatMSAProfileDialog.obj
 0003:00000c9c       _cmdLog                    10029c9c     moc_DNAStatMSAProfileDialog.obj
 0003:00000ca4       __Tuple_alloc              10029ca4     moc_DNAStatPlugin.obj
 0003:00000ca5       _ignore                    10029ca5     moc_DNAStatPlugin.obj
 0003:00000ca6       _allocator_arg             10029ca6     moc_DNAStatPlugin.obj
 0003:00000ca7       _piecewise_construct       10029ca7     moc_DNAStatPlugin.obj
 0003:00000cb0       __Tuple_alloc              10029cb0     moc_DNAStatProfileTask.obj
 0003:00000cb1       _ignore                    10029cb1     moc_DNAStatProfileTask.obj
 0003:00000cb2       _allocator_arg             10029cb2     moc_DNAStatProfileTask.obj
 0003:00000cb3       _piecewise_construct       10029cb3     moc_DNAStatProfileTask.obj
 0003:00000cb4       _taskLog                   10029cb4     moc_DNAStatProfileTask.obj
 0003:00000cbc       _algoLog                   10029cbc     moc_DNAStatProfileTask.obj
 0003:00000cc4       _userActLog                10029cc4     moc_DNAStatProfileTask.obj
 0003:00000ccc       _ioLog                     10029ccc     moc_DNAStatProfileTask.obj
 0003:00000cd4       _coreLog                   10029cd4     moc_DNAStatProfileTask.obj
 0003:00000cdc       _uiLog                     10029cdc     moc_DNAStatProfileTask.obj
 0003:00000ce4       _scriptLog                 10029ce4     moc_DNAStatProfileTask.obj
 0003:00000cec       _perfLog                   10029cec     moc_DNAStatProfileTask.obj
 0003:00000cf4       _cmdLog                    10029cf4     moc_DNAStatProfileTask.obj
 0003:00000cfc       __Tuple_alloc              10029cfc     moc_DistanceMatrixMSAProfileDialog.obj
 0003:00000cfd       _ignore                    10029cfd     moc_DistanceMatrixMSAProfileDialog.obj
 0003:00000cfe       _allocator_arg             10029cfe     moc_DistanceMatrixMSAProfileDialog.obj
 0003:00000cff       _piecewise_construct       10029cff     moc_DistanceMatrixMSAProfileDialog.obj
 0003:00000d00       _taskLog                   10029d00     moc_DistanceMatrixMSAProfileDialog.obj
 0003:00000d08       _algoLog                   10029d08     moc_DistanceMatrixMSAProfileDialog.obj
 0003:00000d10       _userActLog                10029d10     moc_DistanceMatrixMSAProfileDialog.obj
 0003:00000d18       _ioLog                     10029d18     moc_DistanceMatrixMSAProfileDialog.obj
 0003:00000d20       _coreLog                   10029d20     moc_DistanceMatrixMSAProfileDialog.obj
 0003:00000d28       _uiLog                     10029d28     moc_DistanceMatrixMSAProfileDialog.obj
 0003:00000d30       _scriptLog                 10029d30     moc_DistanceMatrixMSAProfileDialog.obj
 0003:00000d38       _perfLog                   10029d38     moc_DistanceMatrixMSAProfileDialog.obj
 0003:00000d40       _cmdLog                    10029d40     moc_DistanceMatrixMSAProfileDialog.obj
 0003:00000d48       ___proc_attached           10029d48     MSVCRT:crtdll.obj
 0003:00000d50       _GS_ExceptionRecord        10029d50     MSVCRT:gs_report.obj
 0003:00000da0       _GS_ContextRecord          10029da0     MSVCRT:gs_report.obj
 0003:0000106c       _DebuggerWasPresent        1002a06c     MSVCRT:gs_report.obj
 0004:00000060       $R000000                   1002b060     * linker generated manifest res *

 Exports

  ordinal    name

        1    _ugene_plugin_init
               exported name: ugene_plugin_init
